 asx32

 Timestamp is 57c98bff (Fri Sep 02 10:26:07 2016)

 Preferred load address is 10000000

 Start         Length     Name                   Class
 0001:00000000 00002126H .text$di                CODE
 0001:00002130 000625e7H .text$mn                CODE
 0001:00064720 0000205cH .text$x                 CODE
 0001:00066780 000005d0H .text$yd                CODE
 0002:00000000 0000060cH .idata$5                DATA
 0002:0000060c 00000004H .CRT$XCA                DATA
 0002:00000610 00000154H .CRT$XCU                DATA
 0002:00000764 00000004H .CRT$XCZ                DATA
 0002:00000768 00000004H .CRT$XIA                DATA
 0002:0000076c 00000014H .CRT$XIC                DATA
 0002:00000780 00000004H .CRT$XIZ                DATA
 0002:00000784 00000004H .CRT$XPA                DATA
 0002:00000788 00000008H .CRT$XPX                DATA
 0002:00000790 00000004H .CRT$XPXA               DATA
 0002:00000794 00000004H .CRT$XPZ                DATA
 0002:00000798 00000004H .CRT$XTA                DATA
 0002:0000079c 00000004H .CRT$XTZ                DATA
 0002:000007a0 0001eb58H .rdata                  DATA
 0002:0001f2f8 00000058H .rdata$debug            DATA
 0002:0001f350 000030e8H .rdata$r                DATA
 0002:00022440 0000022cH .rdata$sxdata           DATA
 0002:0002266c 00000004H .rtc$IAA                DATA
 0002:00022670 00000004H .rtc$IZZ                DATA
 0002:00022674 00000004H .rtc$TAA                DATA
 0002:00022678 00000004H .rtc$TZZ                DATA
 0002:00022680 00002844H .xdata$x                DATA
 0002:00024ec4 00000020H .didat$2                DATA
 0002:00024ee4 00000020H .didat$3                DATA
 0002:00024f04 00000028H .didat$4                DATA
 0002:00024f2c 000001a4H .didat$6                DATA
 0002:000250d0 00000028H .didat$7                DATA
 0002:00025100 0000277bH .edata                  DATA
 0002:0002787c 000000b4H .idata$2                DATA
 0002:00027930 00000014H .idata$3                DATA
 0002:00027944 0000060cH .idata$4                DATA
 0002:00027f50 00002230H .idata$6                DATA
 0003:00000000 000046a0H .data                   DATA
 0003:000046a0 0000129aH .data$r                 DATA
 0003:0000593c 00000028H .didat$5                DATA
 0003:00005980 00003fecH .bss                    DATA
 0004:00000000 000000a0H .rsrc$01                DATA
 0004:000000a0 000004e0H .rsrc$02                DATA

  Address         Publics by Value              Rva+Base       Lib:Object

 0000:00000000       ___guard_fids_count        00000000     <absolute>
 0000:00000000       __except_list              00000000     <absolute>
 0000:00000000       ___guard_flags             00000000     <absolute>
 0000:00000000       ___guard_fids_table        00000000     <absolute>
 0000:0000008b       ___safe_se_handler_count   0000008b     <absolute>
 0000:00000000       ___ImageBase               10000000     <linker-defined>
 0001:00002130       ?AssignIpToMac@AsiAutoAssign@@QAE?AW4AsiAutoAssignNodeStatus@@PBVasiMacAddr@@PBVasiIpAddr@@@Z 10003130 f   asicndload.obj
 0001:00002160       ?CheckEntry@@YA_NW4eFuncEntry@@@Z 10003160 f   asicndload.obj
 0001:000021e0       ?CreateNotificationClient@AsiCobraNetDiscovery@@QAEPAVNotificationClient@@XZ 100031e0 f   asicndload.obj
 0001:00002200       ?FreeNotificationClient@AsiCobraNetDiscovery@@QAEXPAPAVNotificationClient@@@Z 10003200 f   asicndload.obj
 0001:00002230       ?GetEvent@NotificationClient@@QAE_NPAW4EventType@NotificationEvent@@PAVasiMacAddr@@PAVasiIpAddr@@_N@Z 10003230 f   asicndload.obj
 0001:00002270       ?GetStatusForMac@AsiAutoAssign@@QAE?AW4AsiAutoAssignNodeStatus@@PBVasiMacAddr@@@Z 10003270 f   asicndload.obj
 0001:000022a0       ?Start@AsiAutoAssign@@QAEXXZ 100032a0 f   asicndload.obj
 0001:000022c0       ?Start@AsiCobraNetDiscovery@@QAEXXZ 100032c0 f   asicndload.obj
 0001:000022e0       ?Stop@AsiAutoAssign@@QAEXXZ 100032e0 f   asicndload.obj
 0001:00002300       ?Stop@AsiCobraNetDiscovery@@QAEXXZ 10003300 f   asicndload.obj
 0001:00002320       ?createAsiAutoAssign@@YA?AW4acndERROR@@PAVPcapInterface@@PAVAsiCobraNetDiscovery@@PAVAsiAutoassignIpTracker@@PAPAVAsiAutoAssign@@@Z 10003320 f   asicndload.obj
 0001:00002350       ?createAsiAutoAssignIpTracker@@YA?AW4acndERROR@@PAPAVAsiAutoassignIpTracker@@@Z 10003350 f   asicndload.obj
 0001:00002380       ?createAsiCobraNetDiscovery@@YA?AW4acndERROR@@PAVPcapInterface@@PAPAVAsiCobraNetDiscovery@@@Z 10003380 f   asicndload.obj
 0001:000023b0       ?createPcapInterface@@YA?AW4acndERROR@@VasiIpAddr@@PAPAVPcapInterface@@@Z 100033b0 f   asicndload.obj
 0001:000023f0       ?deleteAsiAutoAssign@@YA?AW4acndERROR@@PAPAVAsiAutoAssign@@@Z 100033f0 f   asicndload.obj
 0001:00002420       ?deleteAsiAutoAssignIpTracker@@YA?AW4acndERROR@@PAPAVAsiAutoassignIpTracker@@@Z 10003420 f   asicndload.obj
 0001:00002450       ?deleteAsiCobraNetDiscovery@@YA?AW4acndERROR@@PAPAVAsiCobraNetDiscovery@@@Z 10003450 f   asicndload.obj
 0001:00002480       ?deletePcapInterface@@YA?AW4acndERROR@@PAPAVPcapInterface@@@Z 10003480 f   asicndload.obj
 0001:000024b0       ??0asiMibEntry@@QAE@PBVasiMibGroup@@PBDPBIHHW4type@0@@Z 100034b0 f   asimib.obj
 0001:000024e0       ??0asiMibGroup@@QAE@PBDPBIHPAVasiMibEntry@@H@Z 100034e0 f   asimib.obj
 0001:00002530       ?GetEntryName@asiMibEntry@@QAEXPADHPAIH@Z 10003530 f   asimib.obj
 0001:00002640       ?GetOID@asiMibEntry@@QAEHPAIHHH@Z 10003640 f   asimib.obj
 0001:000026f0       ?GetOIDLength@asiMibEntry@@QAEHXZ 100036f0 f i asimib.obj
 0001:00002700       ?GetOidPrefix@asiMibGroup@@QBEPBIXZ 10003700 f i asimib.obj
 0001:00002710       ?GetOidPrefixLen@asiMibGroup@@QBEHXZ 10003710 f i asimib.obj
 0001:00002720       ?GetPrefix@asiMibGroup@@QBEPBDXZ 10003720 f i asimib.obj
 0001:00002730       ?GetSuffix@asiMibEntry@@QBEPBDXZ 10003730 f i asimib.obj
 0001:00002740       ?GroupLookup@asiMibGroup@@SAPAV1@PBD@Z 10003740 f   asimib.obj
 0001:00002800       ?Matches@asiMibEntry@@QAEHPBIH@Z 10003800 f   asimib.obj
 0001:00002880       ?Matches@asiMibGroup@@QAEHPBIH@Z 10003880 f   asimib.obj
 0001:00002900       ?MibLookup@asiMibGroup@@SAPAVasiMibEntry@@PBD@Z 10003900 f   asimib.obj
 0001:00002940       ?MibToName@@YAXPAKHPADH@Z  10003940 f   asimib.obj
 0001:00002a50       ?ReverseGroupLookup@asiMibGroup@@SAPAV1@PBIH@Z 10003a50 f   asimib.obj
 0001:00002a90       ?ReverseMibLookup@asiMibGroup@@SAPAVasiMibEntry@@PBIH@Z 10003a90 f   asimib.obj
 0001:00002ad0       ?SetOIDLength@asiMibEntry@@QAEXXZ 10003ad0 f   asimib.obj
 0001:00002b00       ?SubMibLookup@asiMibGroup@@QAEPAVasiMibEntry@@PBD@Z 10003b00 f   asimib.obj
 0001:00002b80       ?SubReverseMibLookup@asiMibGroup@@QAEPAVasiMibEntry@@PBIH@Z 10003b80 f   asimib.obj
 0001:00002be0       ?TranslateNameString@@YAXPBDPADH@Z 10003be0 f   asimib.obj
 0001:00002c90       __InlineInterlockedExchangePointer 10003c90 f i asios.obj
 0001:00002ca0       _asios_Atomic_Create       10003ca0 f   asios.obj
 0001:00002cb0       _asios_Atomic_Dec          10003cb0 f   asios.obj
 0001:00002cc0       _asios_Atomic_Delete       10003cc0 f   asios.obj
 0001:00002cd0       _asios_Atomic_Get          10003cd0 f   asios.obj
 0001:00002ce0       _asios_Atomic_Inc          10003ce0 f   asios.obj
 0001:00002d00       _asios_Atomic_Set          10003d00 f   asios.obj
 0001:00002d10       _asios_Clock_convert_to_ms 10003d10 f   asios.obj
 0001:00002d50       _asios_Clock_monotonic     10003d50 f   asios.obj
 0001:00002d70       _asios_Config_Close        10003d70 f   asios.obj
 0001:00002da0       _asios_Config_DeleteAllEntries 10003da0 f   asios.obj
 0001:00002e20       _asios_Config_GetFirstEntry 10003e20 f   asios.obj
 0001:00002e60       _asios_Config_GetNextEntry 10003e60 f   asios.obj
 0001:00002ea0       _asios_Config_GetNumberOfEntries 10003ea0 f   asios.obj
 0001:00002ee0       _asios_Config_Open         10003ee0 f   asios.obj
 0001:00002f00       _asios_Config_Read         10003f00 f   asios.obj
 0001:00002f30       _asios_Config_SetPath      10003f30 f   asios.obj
 0001:00002f60       _asios_Config_Write        10003f60 f   asios.obj
 0001:00002fa0       _asios_Mutex_Create        10003fa0 f   asios.obj
 0001:00002fb0       _asios_Mutex_Destroy       10003fb0 f   asios.obj
 0001:00002fd0       _asios_Mutex_Lock          10003fd0 f   asios.obj
 0001:00002fe0       _asios_Mutex_TryLock       10003fe0 f   asios.obj
 0001:00003010       _asios_Mutex_UnLock        10004010 f   asios.obj
 0001:00003030       _asios_Semaphore_Create    10004030 f   asios.obj
 0001:00003050       _asios_Semaphore_Destroy   10004050 f   asios.obj
 0001:00003070       _asios_Semaphore_Pend      10004070 f   asios.obj
 0001:00003090       _asios_Semaphore_Post      10004090 f   asios.obj
 0001:000030b0       _asios_Sleep               100040b0 f   asios.obj
 0001:000030c0       _asios_Thread_Create       100040c0 f   asios.obj
 0001:000030e0       _asios_Thread_Destroy      100040e0 f   asios.obj
 0001:00003110       _asios_Thread_Self         10004110 f   asios.obj
 0001:00003120       _asios_Thread_SetPriority  10004120 f   asios.obj
 0001:00003150       _asios_printf              10004150 f   asios.obj
 0001:000031d0       ??0PendingRequestList@@QAE@XZ 100041d0 f   asisnmp.obj
 0001:000031f0       ??0PendingRequestListEntry@PendingRequestList@@QAE@PAVSnmpRequest@@J@Z 100041f0 f i asisnmp.obj
 0001:00003210       ??0SnmpGetNextRequest@@QAE@PAVSnmpSession@@PBD1PAVSnmpRequest@@@Z 10004210 f   asisnmp.obj
 0001:00003270       ??0SnmpGetRequest@@QAE@PAVSnmpSession@@PBD1@Z 10004270 f   asisnmp.obj
 0001:000032a0       ??0SnmpRequest@@QAE@PAVSnmpSession@@PBD1J@Z 100042a0 f   asisnmp.obj
 0001:000033b0       ??0SnmpSession@@QAE@XZ     100043b0 f   asisnmp.obj
 0001:000033d0       ??0SnmpSetRequest@@QAE@PAVSnmpSession@@PBD1@Z 100043d0 f   asisnmp.obj
 0001:00003400       ??0SnmpSystem@@QAE@XZ      10004400 f   asisnmp.obj
 0001:00003440       ??1PendingRequestList@@QAE@XZ 10004440 f   asisnmp.obj
 0001:00003470       ??1SnmpRequest@@QAE@XZ     10004470 f   asisnmp.obj
 0001:00003510       ??1SnmpSession@@QAE@XZ     10004510 f   asisnmp.obj
 0001:00003530       ??1SnmpSystem@@QAE@XZ      10004530 f   asisnmp.obj
 0001:00003550       ??BSnmpSession@@QAEPAXXZ   10004550 f i asisnmp.obj
 0001:00003560       ??_GSnmpRequest@@QAEPAXI@Z 10004560 f i asisnmp.obj
 0001:00003590       ?AddRequest@PendingRequestList@@QAEXPAVSnmpRequest@@J@Z 10004590 f   asisnmp.obj
 0001:000035f0       ?AddVariableToRequest@SnmpRequest@@QAEXPAVasiMibEntry@@PBUsmiVALUE@@@Z 100045f0 f   asisnmp.obj
 0001:00003650       ?AddVariableToRequest@SnmpRequest@@QAEXPAVasiOID@@PBUsmiVALUE@@@Z 10004650 f i asisnmp.obj
 0001:00003670       ?AddVariableToRequest@SnmpRequest@@UAEXPAKKPBUsmiVALUE@@@Z 10004670 f   asisnmp.obj
 0001:000036b0       ?Callback@SnmpRequest@@QAEXPAX@Z 100046b0 f   asisnmp.obj
 0001:00003710       ?Callback@SnmpSession@@QAEKPAXPAUHWND__@@IIJ@Z 10004710 f   asisnmp.obj
 0001:00003780       ?CancelPendingRequest@SnmpSession@@QAEXPAVSnmpRequest@@_N@Z 10004780 f   asisnmp.obj
 0001:000037c0       ?CreateGetNextRequest@SnmpSession@@QAEPAVSnmpRequest@@PAV2@PBD1@Z 100047c0 f   asisnmp.obj
 0001:00003820       ?CreateGetRequest@SnmpSession@@QAEPAVSnmpRequest@@PBD0@Z 10004820 f   asisnmp.obj
 0001:00003870       ?CreateSetRequest@SnmpSession@@QAEPAVSnmpRequest@@PBD0@Z 10004870 f   asisnmp.obj
 0001:000038c0       ?GetOID@asiMibEntry@@QAEHAAUsmiOID@@HH@Z 100048c0 f i asisnmp.obj
 0001:000038e0       ?GetOid@asiOID@@QBEPBIXZ   100048e0 f i asisnmp.obj
 0001:000038f0       ?GetOidLen@asiOID@@QBEHXZ  100048f0 f i asisnmp.obj
 0001:00003900       ?GetResultByIndex@SnmpRequest@@QAE_NKPAKHPAH0PAXH1@Z 10004900 f   asisnmp.obj
 0001:00003ae0       ?GetResultByIndex@SnmpRequest@@QAE_NKPAUsmiVALUE@@PAXH@Z 10004ae0 f   asisnmp.obj
 0001:00003be0       ?GetResultCount@SnmpRequest@@QAEKXZ 10004be0 f   asisnmp.obj
 0001:00003c20       ?GetResultStringsByIndex@SnmpRequest@@QAE_NKPADHPAHPAKPAXH1@Z 10004c20 f   asisnmp.obj
 0001:00004050       ?GetVbl@SnmpRequest@@QAEPAXXZ 10005050 f i asisnmp.obj
 0001:00004060       ?LogChar@@YAXDPADHPAH@Z    10005060 f   asisnmp.obj
 0001:000040a0       ?PullRequest@PendingRequestList@@AAEPAVSnmpRequest@@PAV2@PAJ@Z 100050a0 f   asisnmp.obj
 0001:00004120       ?PullRequestById@PendingRequestList@@QAEPAVSnmpRequest@@J@Z 10005120 f i asisnmp.obj
 0001:00004140       ?RegisterPendingRequest@SnmpSession@@QAEXPAVSnmpRequest@@J@Z 10005140 f   asisnmp.obj
 0001:00004150       ?RemoveRequest@PendingRequestList@@QAEJPAVSnmpRequest@@@Z 10005150 f i asisnmp.obj
 0001:00004170       ?SendRequest@SnmpGetNextRequest@@UAEXPAVSnmpRequestor@@@Z 10005170 f   asisnmp.obj
 0001:00004200       ?SendRequest@SnmpRequest@@UAEXPAVSnmpRequestor@@@Z 10005200 f   asisnmp.obj
 0001:000042a0       ?SetErrInfo_Retries@SnmpSession@@QAEXH@Z 100052a0 f i asisnmp.obj
 0001:000042b0       ?SetErrInfo_Timeout@SnmpSession@@QAEXH@Z 100052b0 f i asisnmp.obj
 0001:000042c0       ?SnmpCountElements@SnmpSession@@QAEHPBDPAVasiOID@@PAHPADH@Z 100052c0 f   asisnmp.obj
 0001:00004500       ?SnmpGetInt@SnmpSession@@QAEHPBDPAVasiOID@@PAJ@Z 10005500 f   asisnmp.obj
 0001:00004530       ?SnmpGetString@SnmpSession@@QAEHPBDPAVasiOID@@PADHPAH@Z 10005530 f   asisnmp.obj
 0001:00004590       ?SnmpGetValue@SnmpSession@@QAEHPBDPAVasiOID@@PAUsmiVALUE@@PAXH@Z 10005590 f   asisnmp.obj
 0001:00004630       ?SnmpSetInt@SnmpSession@@QAEHPBDPAVasiOID@@J@Z 10005630 f   asisnmp.obj
 0001:00004660       ?SnmpSetOctets@SnmpSession@@QAEHPBDPAVasiOID@@PBEHK@Z 10005660 f   asisnmp.obj
 0001:000046d0       ?SnmpSetString@SnmpSession@@QAEHPBDPAVasiOID@@0@Z 100056d0 f   asisnmp.obj
 0001:00004700       ?SnmpSetValue@SnmpSession@@QAEHPBDPAVasiOID@@PAUsmiVALUE@@@Z 10005700 f   asisnmp.obj
 0001:00004760       ?StartSession@SnmpSystem@@QAEPAVSnmpSession@@XZ 10005760 f   asisnmp.obj
 0001:00004780       ?TimedOut@SnmpRequest@@QAE_NXZ 10005780 f i asisnmp.obj
 0001:00004790       ?Wait@SnmpRequest@@QAEXK@Z 10005790 f   asisnmp.obj
 0001:000047d0       ?cbFunc@@YGKPAXPAUHWND__@@IIJ0@Z 100057d0 f   asisnmp.obj
 0001:00004870       ?Error_ClearCode@asxBase@@QAE?AW4asxERROR@@XZ 10005870 f i asx.obj
 0001:00004890       ?GetDestinationNode@asxControlBase@@QAE?AW4asxERROR@@PAPAVasxNode@@@Z 10005890 f i asx.obj
 0001:000048b0       ?GetGenericControlName@asxGenericControl@@QAE?AW4asxERROR@@PAD@Z 100058b0 f i asx.obj
 0001:000048e0       ?GetIndex@asxNode@@QAEHXZ  100058e0 f i asx.obj
 0001:000048f0       ?GetNvMemSizeInBytes@asxAdapter@@QAE?AW4asxERROR@@PAH@Z 100058f0 f i asx.obj
 0001:00004910       ?GetSerialNumber@asxAdapter@@QAE?AW4asxERROR@@PAK@Z 10005910 f i asx.obj
 0001:00004930       ?GetSourceNode@asxControlBase@@QAE?AW4asxERROR@@PAPAVasxNode@@@Z 10005930 f i asx.obj
 0001:00004950       ?GetSubSystem@asxControlBase@@QAE?AW4asxERROR@@PAH@Z 10005950 f i asx.obj
 0001:00004970       ?GetSubSystem@asxNode@@QAE?AW4asxERROR@@PAH@Z 10005970 f i asx.obj
 0001:00004990       ?GetType@asxControlBase@@QAE?AW4asxERROR@@PAW4asxCONTROL@@@Z 10005990 f i asx.obj
 0001:000049b0       ?GetType@asxSubSystem@@QAEHXZ 100059b0 f i asx.obj
 0001:000049c0       ?SetCallerName@asxBase@@QAEXPBD@Z 100059c0 f i asx.obj
 0001:000049d0       _ASX_AESEBUReceiver_EnumerateFormat 100059d0 f   asx.obj
 0001:00004a60       _ASX_AESEBUReceiver_GetErrorStatus 10005a60 f   asx.obj
 0001:00004ae0       _ASX_AESEBUReceiver_GetFormat 10005ae0 f   asx.obj
 0001:00004b60       _ASX_AESEBUReceiver_GetSampleRate 10005b60 f   asx.obj
 0001:00004be0       _ASX_AESEBUReceiver_SetFormat 10005be0 f   asx.obj
 0001:00004c60       _ASX_AESEBUTransmitter_EnumerateFormat 10005c60 f   asx.obj
 0001:00004cf0       _ASX_AESEBUTransmitter_GetFormat 10005cf0 f   asx.obj
 0001:00004d70       _ASX_AESEBUTransmitter_SetFormat 10005d70 f   asx.obj
 0001:00004df0       _ASX_Adapter_CheckSubSystems 10005df0 f   asx.obj
 0001:00004e70       _ASX_Adapter_EnumerateMode 10005e70 f   asx.obj
 0001:00004ef0       _ASX_Adapter_EnumerateProperty 10005ef0 f   asx.obj
 0001:00004f70       _ASX_Adapter_GetAVDECCController 10005f70 f   asx.obj
 0001:00004ff0       _ASX_Adapter_GetAVDECCSystem 10005ff0 f   asx.obj
 0001:00005070       _ASX_Adapter_GetDspUtilization 10006070 f   asx.obj
 0001:000050f0       _ASX_Adapter_GetFirmwareRevision 100060f0 f   asx.obj
 0001:00005170       _ASX_Adapter_GetHardwareRevision 10006170 f   asx.obj
 0001:000051f0       _ASX_Adapter_GetIndex      100061f0 f   asx.obj
 0001:00005270       _ASX_Adapter_GetIpAddress  10006270 f   asx.obj
 0001:000052f0       _ASX_Adapter_GetMacAddress 100062f0 f   asx.obj
 0001:00005370       _ASX_Adapter_GetMixer      10006370 f   asx.obj
 0001:000053f0       _ASX_Adapter_GetMode       100063f0 f   asx.obj
 0001:00005470       _ASX_Adapter_GetName       10006470 f   asx.obj
 0001:000054f0       _ASX_Adapter_GetNvMemSizeInBytes 100064f0 f   asx.obj
 0001:00005550       _ASX_Adapter_GetSerialNumber 10006550 f   asx.obj
 0001:000055b0       _ASX_Adapter_ReadNvMem     100065b0 f   asx.obj
 0001:00005630       _ASX_Adapter_ReadProperty  10006630 f   asx.obj
 0001:000056b0       _ASX_Adapter_SetMode       100066b0 f   asx.obj
 0001:00005730       _ASX_Adapter_WriteNvMem    10006730 f   asx.obj
 0001:000057b0       _ASX_Adapter_WriteProperty 100067b0 f   asx.obj
 0001:00005830       _ASX_Block_GetInfo         10006830 f   asx.obj
 0001:000058c0       _ASX_Block_Parameter_Get   100068c0 f   asx.obj
 0001:00005940       _ASX_Block_Parameter_GetElementCount 10006940 f   asx.obj
 0001:000059c0       _ASX_Block_Parameter_GetEnumName 100069c0 f   asx.obj
 0001:00005a50       _ASX_Block_Parameter_GetFlags 10006a50 f   asx.obj
 0001:00005ad0       _ASX_Block_Parameter_GetName 10006ad0 f   asx.obj
 0001:00005b60       _ASX_Block_Parameter_GetRange 10006b60 f   asx.obj
 0001:00005be0       _ASX_Block_Parameter_GetType 10006be0 f   asx.obj
 0001:00005c60       _ASX_Block_Parameter_GetUnits 10006c60 f   asx.obj
 0001:00005cf0       _ASX_Block_Parameter_Set   10006cf0 f   asx.obj
 0001:00005d70       _ASX_ChannelMode_Enumerate 10006d70 f   asx.obj
 0001:00005e00       _ASX_ChannelMode_Get       10006e00 f   asx.obj
 0001:00005e80       _ASX_ChannelMode_Set       10006e80 f   asx.obj
 0001:00005f00       _ASX_CobranetRx_GetBundle  10006f00 f   asx.obj
 0001:00005f80       _ASX_CobranetRx_GetChannelMap 10006f80 f   asx.obj
 0001:00006000       _ASX_CobranetRx_GetMinimumDelay 10007000 f   asx.obj
 0001:00006080       _ASX_CobranetRx_GetSourceMAC 10007080 f   asx.obj
 0001:00006100       _ASX_CobranetRx_GetStatus  10007100 f   asx.obj
 0001:00006190       _ASX_CobranetRx_SetBundle  10007190 f   asx.obj
 0001:00006210       _ASX_CobranetRx_SetChannelMap 10007210 f   asx.obj
 0001:00006290       _ASX_CobranetRx_SetMinimumDelay 10007290 f   asx.obj
 0001:00006310       _ASX_CobranetRx_SetSourceMAC 10007310 f   asx.obj
 0001:00006390       _ASX_CobranetTx_GetBundle  10007390 f   asx.obj
 0001:00006410       _ASX_CobranetTx_GetChannelCount 10007410 f   asx.obj
 0001:00006490       _ASX_CobranetTx_GetChannelMap 10007490 f   asx.obj
 0001:00006510       _ASX_CobranetTx_GetFormat  10007510 f   asx.obj
 0001:00006590       _ASX_CobranetTx_GetStatus  10007590 f   asx.obj
 0001:00006620       _ASX_CobranetTx_GetUnicastMode 10007620 f   asx.obj
 0001:000066a0       _ASX_CobranetTx_SetBundle  100076a0 f   asx.obj
 0001:00006720       _ASX_CobranetTx_SetChannelCount 10007720 f   asx.obj
 0001:000067a0       _ASX_CobranetTx_SetChannelMap 100077a0 f   asx.obj
 0001:00006820       _ASX_CobranetTx_SetFormat  10007820 f   asx.obj
 0001:000068a0       _ASX_CobranetTx_SetUnicastMode 100078a0 f   asx.obj
 0001:00006920       _ASX_Cobranet_EnumerateModes 10007920 f   asx.obj
 0001:00006930       _ASX_Cobranet_GetConductorPriority 10007930 f   asx.obj
 0001:000069b0       _ASX_Cobranet_GetConductorStatus 100079b0 f   asx.obj
 0001:00006a30       _ASX_Cobranet_GetDescription 10007a30 f   asx.obj
 0001:00006ab0       _ASX_Cobranet_GetErrorInfo 10007ab0 f   asx.obj
 0001:00006b40       _ASX_Cobranet_GetFirmwareRevision 10007b40 f   asx.obj
 0001:00006bc0       _ASX_Cobranet_GetIPAddress 10007bc0 f   asx.obj
 0001:00006c40       _ASX_Cobranet_GetIfStatus  10007c40 f   asx.obj
 0001:00006cd0       _ASX_Cobranet_GetLatencyAndSampleRate 10007cd0 f   asx.obj
 0001:00006d50       _ASX_Cobranet_GetLocation  10007d50 f   asx.obj
 0001:00006dd0       _ASX_Cobranet_GetMACAddress 10007dd0 f   asx.obj
 0001:00006e50       _ASX_Cobranet_GetMode      10007e50 f   asx.obj
 0001:00006e60       _ASX_Cobranet_GetName      10007e60 f   asx.obj
 0001:00006ee0       _ASX_Cobranet_GetPersistence 10007ee0 f   asx.obj
 0001:00006f60       _ASX_Cobranet_GetSerialConfig 10007f60 f   asx.obj
 0001:00006ff0       _ASX_Cobranet_GetSerialEnable 10007ff0 f   asx.obj
 0001:00007070       _ASX_Cobranet_GetStaticIPAddress 10008070 f   asx.obj
 0001:000070f0       _ASX_Cobranet_SetConductorPriority 100080f0 f   asx.obj
 0001:00007170       _ASX_Cobranet_SetIPAddress 10008170 f   asx.obj
 0001:000071f0       _ASX_Cobranet_SetLatencyAndSampleRate 100081f0 f   asx.obj
 0001:00007270       _ASX_Cobranet_SetLocation  10008270 f   asx.obj
 0001:000072f0       _ASX_Cobranet_SetMode      100082f0 f   asx.obj
 0001:00007300       _ASX_Cobranet_SetName      10008300 f   asx.obj
 0001:00007380       _ASX_Cobranet_SetPersistence 10008380 f   asx.obj
 0001:00007400       _ASX_Cobranet_SetSerialConfig 10008400 f   asx.obj
 0001:00007490       _ASX_Cobranet_SetSerialEnable 10008490 f   asx.obj
 0001:00007510       _ASX_Cobranet_SetStaticIPAddress 10008510 f   asx.obj
 0001:00007590       _ASX_Compander_Get         10008590 f   asx.obj
 0001:00007620       _ASX_Compander_GetAttackTimeConstant 10008620 f   asx.obj
 0001:000076a0       _ASX_Compander_GetDecayTimeConstant 100086a0 f   asx.obj
 0001:00007720       _ASX_Compander_GetEnable   10008720 f   asx.obj
 0001:000077a0       _ASX_Compander_GetMakeupGain 100087a0 f   asx.obj
 0001:00007820       _ASX_Compander_GetRatio    10008820 f   asx.obj
 0001:000078a0       _ASX_Compander_GetThreshold 100088a0 f   asx.obj
 0001:00007920       _ASX_Compander_Set         10008920 f   asx.obj
 0001:000079b0       _ASX_Compander_SetAttackTimeConstant 100089b0 f   asx.obj
 0001:00007a30       _ASX_Compander_SetDecayTimeConstant 10008a30 f   asx.obj
 0001:00007ab0       _ASX_Compander_SetEnable   10008ab0 f   asx.obj
 0001:00007b30       _ASX_Compander_SetMakeupGain 10008b30 f   asx.obj
 0001:00007bc0       _ASX_Compander_SetRatio    10008bc0 f   asx.obj
 0001:00007c50       _ASX_Compander_SetThreshold 10008c50 f   asx.obj
 0001:00007ce0       _ASX_Control_GetDestinationNode 10008ce0 f   asx.obj
 0001:00007d40       _ASX_Control_GetHpiControl 10008d40 f   asx.obj
 0001:00007dc0       _ASX_Control_GetSourceNode 10008dc0 f   asx.obj
 0001:00007e20       _ASX_Control_GetSubSystem  10008e20 f   asx.obj
 0001:00007e80       _ASX_Control_GetType       10008e80 f   asx.obj
 0001:00007ee0       _ASX_EQ_GetBand            10008ee0 f   asx.obj
 0001:00007f70       _ASX_EQ_GetInfo            10008f70 f   asx.obj
 0001:00007ff0       _ASX_EQ_SetBand            10008ff0 f   asx.obj
 0001:00008080       _ASX_EQ_SetState           10009080 f   asx.obj
 0001:00008100       _ASX_Error_Clear           10009100 f   asx.obj
 0001:00008150       _ASX_Error_GetLast         10009150 f   asx.obj
 0001:00008190       _ASX_Error_GetLastString   10009190 f   asx.obj
 0001:000081e0       _ASX_GPIO_GetProperties    100091e0 f   asx.obj
 0001:00008260       _ASX_GPIO_InputGet         10009260 f   asx.obj
 0001:000082e0       _ASX_GPIO_OutputGet        100092e0 f   asx.obj
 0001:00008360       _ASX_GPIO_OutputSet        10009360 f   asx.obj
 0001:000083e0       _ASX_GetGenericControlName 100093e0 f   asx.obj
 0001:00008450       _ASX_Handle_GetType        10009450 f   asx.obj
 0001:00008460       _ASX_Level_Get             10009460 f   asx.obj
 0001:000084e0       _ASX_Level_GetRange        100094e0 f   asx.obj
 0001:00008570       _ASX_Level_Set             10009570 f   asx.obj
 0001:00008600       _ASX_Meter_GetBallistics   10009600 f   asx.obj
 0001:00008690       _ASX_Meter_GetChannels     10009690 f   asx.obj
 0001:00008710       _ASX_Meter_GetPeak         10009710 f   asx.obj
 0001:00008790       _ASX_Meter_GetRMS          10009790 f   asx.obj
 0001:00008810       _ASX_Meter_SetBallistics   10009810 f   asx.obj
 0001:000088b0       _ASX_Mic_GetPhantomPower   100098b0 f   asx.obj
 0001:00008930       _ASX_Mic_SetPhantomPower   10009930 f   asx.obj
 0001:000089b0       _ASX_Mixer_GetBlockControlByNodeTypeAndIndex 100099b0 f   asx.obj
 0001:00008a40       _ASX_Mixer_GetControl      10009a40 f   asx.obj
 0001:00008ac0       _ASX_Mixer_GetControlByNode 10009ac0 f   asx.obj
 0001:00008b40       _ASX_Mixer_GetControlByNodeTypeAndIndex 10009b40 f   asx.obj
 0001:00008bd0       _ASX_Mixer_GetControlCount 10009bd0 f   asx.obj
 0001:00008c50       _ASX_Mixer_GetDestinationNode 10009c50 f   asx.obj
 0001:00008cd0       _ASX_Mixer_GetDestinationNodeCount 10009cd0 f   asx.obj
 0001:00008d50       _ASX_Mixer_GetNodeByType   10009d50 f   asx.obj
 0001:00008dd0       _ASX_Mixer_GetNodeIndex    10009dd0 f   asx.obj
 0001:00008de0       _ASX_Mixer_GetNodeType     10009de0 f   asx.obj
 0001:00008df0       _ASX_Mixer_GetNodeTypeCount 10009df0 f   asx.obj
 0001:00008e70       _ASX_Mixer_GetSourceNode   10009e70 f   asx.obj
 0001:00008ef0       _ASX_Mixer_GetSourceNodeCount 10009ef0 f   asx.obj
 0001:00008f70       _ASX_Mixer_ResetControls   10009f70 f   asx.obj
 0001:00008ff0       _ASX_Multiplexer_Enumerate 10009ff0 f   asx.obj
 0001:00009080       _ASX_Multiplexer_Get       1000a080 f   asx.obj
 0001:00009100       _ASX_Multiplexer_Set       1000a100 f   asx.obj
 0001:00009180       _ASX_Node_GetIndex         1000a180 f   asx.obj
 0001:000091d0       _ASX_Node_GetLocation      1000a1d0 f   asx.obj
 0001:00009250       _ASX_Node_GetName          1000a250 f   asx.obj
 0001:000092d0       _ASX_Node_GetSubSystem     1000a2d0 f   asx.obj
 0001:00009330       _ASX_Node_GetType          1000a330 f   asx.obj
 0001:00009380       _ASX_PAD_GetArtist         1000a380 f   asx.obj
 0001:00009410       _ASX_PAD_GetChannelName    1000a410 f   asx.obj
 0001:000094a0       _ASX_PAD_GetComment        1000a4a0 f   asx.obj
 0001:00009530       _ASX_PAD_GetProgramType    1000a530 f   asx.obj
 0001:000095c0       _ASX_PAD_GetProgramTypeString 1000a5c0 f   asx.obj
 0001:00009650       _ASX_PAD_GetRdsPI          1000a650 f   asx.obj
 0001:000096e0       _ASX_PAD_GetTitle          1000a6e0 f   asx.obj
 0001:00009770       _ASX_Player_Close          1000a770 f   asx.obj
 0001:000097f0       _ASX_Player_Format_GetDetails 1000a7f0 f   asx.obj
 0001:00009880       _ASX_Player_Format_GetString 1000a880 f   asx.obj
 0001:00009900       _ASX_Player_GetFilename    1000a900 f   asx.obj
 0001:00009990       _ASX_Player_GetLoopMode    1000a990 f   asx.obj
 0001:00009a10       _ASX_Player_GetPosition    1000aa10 f   asx.obj
 0001:00009a90       _ASX_Player_GetState       1000aa90 f   asx.obj
 0001:00009b10       _ASX_Player_GetTimeScale   1000ab10 f   asx.obj
 0001:00009b90       _ASX_Player_Open           1000ab90 f   asx.obj
 0001:00009c10       _ASX_Player_OpenPlaylist   1000ac10 f   asx.obj
 0001:00009c90       _ASX_Player_Pause          1000ac90 f   asx.obj
 0001:00009d10       _ASX_Player_PlaylistStatus 1000ad10 f   asx.obj
 0001:00009da0       _ASX_Player_PlaylistWait   1000ada0 f   asx.obj
 0001:00009e20       _ASX_Player_PreLoad        1000ae20 f   asx.obj
 0001:00009ea0       _ASX_Player_RegisterCallback 1000aea0 f   asx.obj
 0001:00009f30       _ASX_Player_SetLoopMode    1000af30 f   asx.obj
 0001:00009fb0       _ASX_Player_SetPosition    1000afb0 f   asx.obj
 0001:0000a030       _ASX_Player_SetTimeScale   1000b030 f   asx.obj
 0001:0000a0c0       _ASX_Player_Start          1000b0c0 f   asx.obj
 0001:0000a140       _ASX_Player_Stop           1000b140 f   asx.obj
 0001:0000a1c0       _ASX_Player_Wait           1000b1c0 f   asx.obj
 0001:0000a240       _ASX_Recorder_Close        1000b240 f   asx.obj
 0001:0000a2c0       _ASX_Recorder_EnumerateFormat 1000b2c0 f   asx.obj
 0001:0000a350       _ASX_Recorder_GetFilename  1000b350 f   asx.obj
 0001:0000a3e0       _ASX_Recorder_GetPosition  1000b3e0 f   asx.obj
 0001:0000a460       _ASX_Recorder_GetState     1000b460 f   asx.obj
 0001:0000a4e0       _ASX_Recorder_Open         1000b4e0 f   asx.obj
 0001:0000a570       _ASX_Recorder_Pause        1000b570 f   asx.obj
 0001:0000a5f0       _ASX_Recorder_Start        1000b5f0 f   asx.obj
 0001:0000a670       _ASX_Recorder_Stop         1000b670 f   asx.obj
 0001:0000a6f0       _ASX_SampleClock_EnumerateClockSource 1000b6f0 f   asx.obj
 0001:0000a780       _ASX_SampleClock_EnumerateLocalRate 1000b780 f   asx.obj
 0001:0000a810       _ASX_SampleClock_EnumerateSampleRate 1000b810 f   asx.obj
 0001:0000a820       _ASX_SampleClock_GetAutoSource 1000b820 f   asx.obj
 0001:0000a8b0       _ASX_SampleClock_GetClockSource 1000b8b0 f   asx.obj
 0001:0000a930       _ASX_SampleClock_GetLocalRate 1000b930 f   asx.obj
 0001:0000a9b0       _ASX_SampleClock_GetLocalRateLock 1000b9b0 f   asx.obj
 0001:0000aa40       _ASX_SampleClock_GetSampleRate 1000ba40 f   asx.obj
 0001:0000aac0       _ASX_SampleClock_SetAutoSource 1000bac0 f   asx.obj
 0001:0000ab50       _ASX_SampleClock_SetClockSource 1000bb50 f   asx.obj
 0001:0000abd0       _ASX_SampleClock_SetLocalRate 1000bbd0 f   asx.obj
 0001:0000ac50       _ASX_SampleClock_SetLocalRateLock 1000bc50 f   asx.obj
 0001:0000ace0       _ASX_SampleClock_SetSampleRate 1000bce0 f   asx.obj
 0001:0000acf0       _ASX_SilenceDetector_GetDelay 1000bcf0 f   asx.obj
 0001:0000ad70       _ASX_SilenceDetector_GetEnable 1000bd70 f   asx.obj
 0001:0000adf0       _ASX_SilenceDetector_GetEventEnable 1000bdf0 f   asx.obj
 0001:0000ae70       _ASX_SilenceDetector_GetState 1000be70 f   asx.obj
 0001:0000aef0       _ASX_SilenceDetector_GetThreshold 1000bef0 f   asx.obj
 0001:0000af70       _ASX_SilenceDetector_SetDelay 1000bf70 f   asx.obj
 0001:0000aff0       _ASX_SilenceDetector_SetEnable 1000bff0 f   asx.obj
 0001:0000b070       _ASX_SilenceDetector_SetEventEnable 1000c070 f   asx.obj
 0001:0000b0f0       _ASX_SilenceDetector_SetThreshold 1000c0f0 f   asx.obj
 0001:0000b180       _ASX_System_Create         1000c180 f   asx.obj
 0001:0000b1d0       _ASX_System_CreateSubSystem 1000c1d0 f   asx.obj
 0001:0000b250       _ASX_System_Delete         1000c250 f   asx.obj
 0001:0000b280       _ASX_System_GetAdapter     1000c280 f   asx.obj
 0001:0000b300       _ASX_System_GetAdapterCount 1000c300 f   asx.obj
 0001:0000b380       _ASX_System_GetCobranetAutoassignParms 1000c380 f   asx.obj
 0001:0000b390       _ASX_System_GetMessageLogging 1000c390 f   asx.obj
 0001:0000b410       _ASX_System_GetName        1000c410 f   asx.obj
 0001:0000b490       _ASX_System_GetVersion     1000c490 f   asx.obj
 0001:0000b520       _ASX_System_RegisterErrorCallback 1000c520 f   asx.obj
 0001:0000b5a0       _ASX_System_SetAvdeccInterface 1000c5a0 f   asx.obj
 0001:0000b5b0       _ASX_System_SetCobranetAutoassignParms 1000c5b0 f   asx.obj
 0001:0000b5c0       _ASX_System_SetHostNetworkInterface 1000c5c0 f   asx.obj
 0001:0000b5d0       _ASX_System_SetMessageLogging 1000c5d0 f   asx.obj
 0001:0000b650       _ASX_System_SupportsSubSystem 1000c650 f   asx.obj
 0001:0000b660       _ASX_ToneDetector_GetEnable 1000c660 f   asx.obj
 0001:0000b6e0       _ASX_ToneDetector_GetEventEnable 1000c6e0 f   asx.obj
 0001:0000b760       _ASX_ToneDetector_GetFrequency 1000c760 f   asx.obj
 0001:0000b7e0       _ASX_ToneDetector_GetState 1000c7e0 f   asx.obj
 0001:0000b860       _ASX_ToneDetector_GetThreshold 1000c860 f   asx.obj
 0001:0000b8e0       _ASX_ToneDetector_SetEnable 1000c8e0 f   asx.obj
 0001:0000b960       _ASX_ToneDetector_SetEventEnable 1000c960 f   asx.obj
 0001:0000b9e0       _ASX_ToneDetector_SetThreshold 1000c9e0 f   asx.obj
 0001:0000ba70       _ASX_Tuner_EnumerateBand   1000ca70 f   asx.obj
 0001:0000bb00       _ASX_Tuner_EnumerateDeemphasis 1000cb00 f   asx.obj
 0001:0000bb90       _ASX_Tuner_EnumerateHdBlend 1000cb90 f   asx.obj
 0001:0000bc20       _ASX_Tuner_EnumerateProgram 1000cc20 f   asx.obj
 0001:0000bcb0       _ASX_Tuner_GetBand         1000ccb0 f   asx.obj
 0001:0000bd30       _ASX_Tuner_GetDabAudioInfo 1000cd30 f   asx.obj
 0001:0000bdc0       _ASX_Tuner_GetDabAudioServiceCount 1000cdc0 f   asx.obj
 0001:0000be40       _ASX_Tuner_GetDabAudioServiceName 1000ce40 f   asx.obj
 0001:0000bed0       _ASX_Tuner_GetDabMultiplexId 1000ced0 f   asx.obj
 0001:0000bf60       _ASX_Tuner_GetDabMultiplexName 1000cf60 f   asx.obj
 0001:0000bff0       _ASX_Tuner_GetDabServiceId 1000cff0 f   asx.obj
 0001:0000c080       _ASX_Tuner_GetDeemphasis   1000d080 f   asx.obj
 0001:0000c100       _ASX_Tuner_GetDigitalSignalQuality 1000d100 f   asx.obj
 0001:0000c190       _ASX_Tuner_GetFirmwareVersion 1000d190 f   asx.obj
 0001:0000c220       _ASX_Tuner_GetFrequency    1000d220 f   asx.obj
 0001:0000c2a0       _ASX_Tuner_GetFrequencyRange 1000d2a0 f   asx.obj
 0001:0000c330       _ASX_Tuner_GetGain         1000d330 f   asx.obj
 0001:0000c3b0       _ASX_Tuner_GetGainRange    1000d3b0 f   asx.obj
 0001:0000c440       _ASX_Tuner_GetHdBlend      1000d440 f   asx.obj
 0001:0000c4d0       _ASX_Tuner_GetHdRadioDspVersion 1000d4d0 f   asx.obj
 0001:0000c4e0       _ASX_Tuner_GetHdRadioSdkVersion 1000d4e0 f   asx.obj
 0001:0000c4f0       _ASX_Tuner_GetHdRadioSignalQuality 1000d4f0 f   asx.obj
 0001:0000c500       _ASX_Tuner_GetMode         1000d500 f   asx.obj
 0001:0000c580       _ASX_Tuner_GetProgram      1000d580 f   asx.obj
 0001:0000c600       _ASX_Tuner_GetRFLevel      1000d600 f   asx.obj
 0001:0000c680       _ASX_Tuner_GetRawRFLevel   1000d680 f   asx.obj
 0001:0000c700       _ASX_Tuner_GetStatus       1000d700 f   asx.obj
 0001:0000c780       _ASX_Tuner_SetBand         1000d780 f   asx.obj
 0001:0000c800       _ASX_Tuner_SetDabAudioService 1000d800 f   asx.obj
 0001:0000c880       _ASX_Tuner_SetDeemphasis   1000d880 f   asx.obj
 0001:0000c900       _ASX_Tuner_SetFrequency    1000d900 f   asx.obj
 0001:0000c980       _ASX_Tuner_SetGain         1000d980 f   asx.obj
 0001:0000ca10       _ASX_Tuner_SetHdBlend      1000da10 f   asx.obj
 0001:0000caa0       _ASX_Tuner_SetMode         1000daa0 f   asx.obj
 0001:0000cb20       _ASX_Tuner_SetProgram      1000db20 f   asx.obj
 0001:0000cba0       _ASX_Volume_GetChannels    1000dba0 f   asx.obj
 0001:0000cc20       _ASX_Volume_GetGain        1000dc20 f   asx.obj
 0001:0000cca0       _ASX_Volume_GetMute        1000dca0 f   asx.obj
 0001:0000cd20       _ASX_Volume_GetRange       1000dd20 f   asx.obj
 0001:0000cdb0       _ASX_Volume_SetAutofade    1000ddb0 f   asx.obj
 0001:0000ce40       _ASX_Volume_SetGain        1000de40 f   asx.obj
 0001:0000cec0       _ASX_Volume_SetMute        1000dec0 f   asx.obj
 0001:0000cf40       _ASX_Vox_GetLevel          1000df40 f   asx.obj
 0001:0000cfc0       _ASX_Vox_GetRange          1000dfc0 f   asx.obj
 0001:0000d050       _ASX_Vox_SetLevel          1000e050 f   asx.obj
 0001:0000d0e0       ??$_Allocate@D@std@@YAPADIPAD@Z 1000e0e0 f i asxavdecc.obj
 0001:0000d110       ??$addressof@D@std@@YAPADAAD@Z 1000e110 f i asxavdecc.obj
 0001:0000d120       ??$construct@PADAAPAD@?$_Wrap_alloc@V?$allocator@D@std@@@std@@QAEXPAPADAAPAD@Z 1000e120 f i asxavdecc.obj
 0001:0000d140       ??$construct@PADAAPAD@?$allocator@D@std@@QAEXPAPADAAPAD@Z 1000e140 f i asxavdecc.obj
 0001:0000d160       ??$construct@PADAAPAD@?$allocator_traits@V?$allocator@D@std@@@std@@SAXAAV?$allocator@D@1@PAPADAAPAD@Z 1000e160 f i asxavdecc.obj
 0001:0000d180       ??$destroy@PAD@?$_Wrap_alloc@V?$allocator@D@std@@@std@@QAEXPAPAD@Z 1000e180 f i asxavdecc.obj
 0001:0000d190       ??$destroy@PAD@?$allocator@D@std@@QAEXPAPAD@Z 1000e190 f i asxavdecc.obj
 0001:0000d1a0       ??$destroy@PAD@?$allocator_traits@V?$allocator@D@std@@@std@@SAXAAV?$allocator@D@1@PAPAD@Z 1000e1a0 f i asxavdecc.obj
 0001:0000d1b0       ??$forward@AAPAD@std@@YAAAPADAAPAD@Z 1000e1b0 f i asxavdecc.obj
 0001:0000d1c0       ??0?$_String_alloc@$0A@U?$_String_base_types@DV?$allocator@D@std@@@std@@@std@@QAE@ABV?$allocator@D@1@@Z 1000e1c0 f i asxavdecc.obj
 0001:0000d1e0       ??0?$_String_val@U?$_Simple_types@D@std@@@std@@QAE@XZ 1000e1e0 f i asxavdecc.obj
 0001:0000d200       ??0?$_Wrap_alloc@V?$allocator@D@std@@@std@@QAE@XZ 1000e200 f i asxavdecc.obj
 0001:0000d210       ??0?$allocator@D@std@@QAE@XZ 1000e210 f i asxavdecc.obj
 0001:0000d220       ??0?$basic_string@DU?$char_traits@D@std@@V?$allocator@D@2@@std@@QAE@PBD@Z 1000e220 f i asxavdecc.obj
 0001:0000d280       ??0_Generic_error_category@std@@QAE@XZ 1000e280 f i asxavdecc.obj
 0001:0000d290       ??0_Iostream_error_category@std@@QAE@XZ 1000e290 f i asxavdecc.obj
 0001:0000d2a0       ??0_System_error_category@std@@QAE@XZ 1000e2a0 f i asxavdecc.obj
 0001:0000d2b0       ??0asiIpAddr@@QAE@XZ       1000e2b0 f i asxavdecc.obj
 0001:0000d2c0       ??0asiMacAddr@@QAE@_K@Z    1000e2c0 f i asxavdecc.obj
 0001:0000d310       ??0asxAdapterAVDECC@@QAE@PAVcontroller@avdecc_lib@@PAVsystem@2@PAVasxSystem@@PADH3@Z 1000e310 f   asxavdecc.obj
 0001:0000d3b0       ??0asxSubSystemAVDECC@@QAE@PAVasxSystem@@@Z 1000e3b0 f   asxavdecc.obj
 0001:0000d440       ??0error_category@std@@QAE@XZ 1000e440 f i asxavdecc.obj
 0001:0000d450       ??0error_condition@std@@QAE@HABVerror_category@1@@Z 1000e450 f i asxavdecc.obj
 0001:0000d470       ??0id@locale@std@@QAE@I@Z  1000e470 f i asxavdecc.obj
 0001:0000d480       ??1?$basic_string@DU?$char_traits@D@std@@V?$allocator@D@2@@std@@QAE@XZ 1000e480 f i asxavdecc.obj
 0001:0000d4b0       ??1_Generic_error_category@std@@UAE@XZ 1000e4b0 f i asxavdecc.obj
 0001:0000d4c0       ??1_Iostream_error_category@std@@UAE@XZ 1000e4c0 f i asxavdecc.obj
 0001:0000d4d0       ??1_System_error_category@std@@UAE@XZ 1000e4d0 f i asxavdecc.obj
 0001:0000d4e0       ??1asxAdapterAVDECC@@UAE@XZ 1000e4e0 f   asxavdecc.obj
 0001:0000d4f0       ??1asxSubSystemAVDECC@@UAE@XZ 1000e4f0 f   asxavdecc.obj
 0001:0000d5d0       ??1error_category@std@@UAE@XZ 1000e5d0 f i asxavdecc.obj
 0001:0000d5e0       ??2@YAPAXIPAX@Z            1000e5e0 f i asxavdecc.obj
 0001:0000d5f0       ??3@YAXPAX0@Z              1000e5f0 f i asxavdecc.obj
 0001:0000d600       ??8error_category@std@@QBE_NABV01@@Z 1000e600 f i asxavdecc.obj
 0001:0000d610       ??8error_condition@std@@QBE_NABV01@@Z 1000e610 f i asxavdecc.obj
 0001:0000d630       ??_E_Generic_error_category@std@@UAEPAXI@Z 1000e630 f i asxavdecc.obj
 0001:0000d630       ??_G_Generic_error_category@std@@UAEPAXI@Z 1000e630 f i asxavdecc.obj
 0001:0000d660       ??_E_Iostream_error_category@std@@UAEPAXI@Z 1000e660 f i asxavdecc.obj
 0001:0000d660       ??_G_Iostream_error_category@std@@UAEPAXI@Z 1000e660 f i asxavdecc.obj
 0001:0000d690       ??_E_System_error_category@std@@UAEPAXI@Z 1000e690 f i asxavdecc.obj
 0001:0000d690       ??_G_System_error_category@std@@UAEPAXI@Z 1000e690 f i asxavdecc.obj
 0001:0000d6c0       ??_EasxAdapterAVDECC@@UAEPAXI@Z 1000e6c0 f i asxavdecc.obj
 0001:0000d6c0       ??_GasxAdapterAVDECC@@UAEPAXI@Z 1000e6c0 f i asxavdecc.obj
 0001:0000d6f0       ??_EasxSubSystemAVDECC@@UAEPAXI@Z 1000e6f0 f i asxavdecc.obj
 0001:0000d6f0       ??_GasxSubSystemAVDECC@@UAEPAXI@Z 1000e6f0 f i asxavdecc.obj
 0001:0000d720       ??_Gerror_category@std@@UAEPAXI@Z 1000e720 f i asxavdecc.obj
 0001:0000d720       ??_Eerror_category@std@@UAEPAXI@Z 1000e720 f i asxavdecc.obj
 0001:0000d750       ?CheckSubSystems@asxAdapterAVDECC@@UAE?AW4asxERROR@@PAI0@Z 1000e750 f   asxavdecc.obj
 0001:0000d900       ?Count@?$TASIArray@VasxAdapter@@@@QBEHXZ 1000e900 f i asxavdecc.obj
 0001:0000d910       ?EnumerateProperty@asxAdapter@@UAE?AW4asxERROR@@HW4asxADPROPENUM_MODE@@HPAK@Z 1000e910 f i asxavdecc.obj
 0001:0000d920       ?GetAVDECCController@asxAdapterAVDECC@@UAE?AW4asxERROR@@PAPAX@Z 1000e920 f   asxavdecc.obj
 0001:0000d950       ?GetAVDECCSystem@asxAdapterAVDECC@@UAE?AW4asxERROR@@PAPAX@Z 1000e950 f   asxavdecc.obj
 0001:0000d970       ?GetDspUtilization@asxAdapter@@UAE?AW4asxERROR@@HPAH@Z 1000e970 f i asxavdecc.obj
 0001:0000d990       ?GetIpAddress@asxAdapterAVDECC@@UAE?AW4asxERROR@@PAD@Z 1000e990 f   asxavdecc.obj
 0001:0000d9a0       ?GetMacAddress@asxAdapterAVDECC@@UAE?AW4asxERROR@@PAD@Z 1000e9a0 f   asxavdecc.obj
 0001:0000d9d0       ?GetMode@asxAdapter@@UAE?AW4asxERROR@@PAW4asxADAPTERMODE@@@Z 1000e9d0 f i asxavdecc.obj
 0001:0000d9e0       ?GetParentSystem@asxSubSystem@@QAEPAVasxSystem@@XZ 1000e9e0 f i asxavdecc.obj
 0001:0000d9f0       ?GetSubType@asxBase@@UAEHXZ 1000e9f0 f i asxavdecc.obj
 0001:0000da00       ?GetType@asxBase@@UAEHXZ   1000ea00 f i asxavdecc.obj
 0001:0000da10       ?InitAVDECCController@asxSubSystemAVDECC@@AAEXPBD@Z 1000ea10 f   asxavdecc.obj
 0001:0000dad0       ?InitError@asxSubSystemAVDECC@@QAE?AW4asxERROR@@XZ 1000ead0 f   asxavdecc.obj
 0001:0000dae0       ?Predelete@asxAdapter@@UAE?AW4asxERROR@@XZ 1000eae0 f i asxavdecc.obj
 0001:0000daf0       ?ReScan@asxSubSystemAVDECC@@UAEXXZ 1000eaf0 f   asxavdecc.obj
 0001:0000df10       ?ReadNvMem@asxAdapter@@UAE?AW4asxERROR@@HPAE@Z 1000ef10 f i asxavdecc.obj
 0001:0000df20       ?ReadProperty@asxAdapter@@UAE?AW4asxERROR@@HPAG0@Z 1000ef20 f i asxavdecc.obj
 0001:0000df30       ?Scan@asxSubSystemAVDECC@@UAEXXZ 1000ef30 f   asxavdecc.obj
 0001:0000df40       ?SetDetails@asxAdapterAVDECC@@QAEXXZ 1000ef40 f   asxavdecc.obj
 0001:0000e180       ?SetMode@asxAdapter@@UAE?AW4asxERROR@@W4asxADAPTERMODE@@@Z 1000f180 f i asxavdecc.obj
 0001:0000e190       ?TranslateSpecificErrorCode@asxSubSystem@@UAEXIPAPBD@Z 1000f190 f i asxavdecc.obj
 0001:0000e1a0       ?UpdateAdapterProperties@asxAdapterAVDECC@@UAE?AW4asxERROR@@XZ 1000f1a0 f   asxavdecc.obj
 0001:0000e3e0       ?WriteNvMem@asxAdapter@@UAE?AW4asxERROR@@HE@Z 1000f3e0 f i asxavdecc.obj
 0001:0000e3f0       ?WriteProperty@asxAdapter@@UAE?AW4asxERROR@@HGG@Z 1000f3f0 f i asxavdecc.obj
 0001:0000e400       ?_Copy@?$basic_string@DU?$char_traits@D@std@@V?$allocator@D@2@@std@@QAEXII@Z 1000f400 f i asxavdecc.obj
 0001:0000e550       ?_Eos@?$basic_string@DU?$char_traits@D@std@@V?$allocator@D@2@@std@@QAEXI@Z 1000f550 f i asxavdecc.obj
 0001:0000e580       ?_Getal@?$_String_alloc@$0A@U?$_String_base_types@DV?$allocator@D@std@@@std@@@std@@QBE?AU?$_Wrap_alloc@V?$allocator@D@std@@@2@XZ 1000f580 f i asxavdecc.obj
 0001:0000e590       ?_Grow@?$basic_string@DU?$char_traits@D@std@@V?$allocator@D@2@@std@@QAE_NI_N@Z 1000f590 f i asxavdecc.obj
 0001:0000e650       ?_Inside@?$basic_string@DU?$char_traits@D@std@@V?$allocator@D@2@@std@@QAE_NPBD@Z 1000f650 f i asxavdecc.obj
 0001:0000e690       ?_Myptr@?$_String_val@U?$_Simple_types@D@std@@@std@@QAEPADXZ 1000f690 f i asxavdecc.obj
 0001:0000e6a0       ?_Myptr@?$_String_val@U?$_Simple_types@D@std@@@std@@QBEPBDXZ 1000f6a0 f i asxavdecc.obj
 0001:0000e6b0       ?_Tidy@?$basic_string@DU?$char_traits@D@std@@V?$allocator@D@2@@std@@QAEX_NI@Z 1000f6b0 f i asxavdecc.obj
 0001:0000e700       ?_Xlen@?$basic_string@DU?$char_traits@D@std@@V?$allocator@D@2@@std@@QBEXXZ 1000f700 f i asxavdecc.obj
 0001:0000e710       ?_Xran@?$basic_string@DU?$char_traits@D@std@@V?$allocator@D@2@@std@@QBEXXZ 1000f710 f i asxavdecc.obj
 0001:0000e720       ?allocate@?$_Wrap_alloc@V?$allocator@D@std@@@std@@QAEPADI@Z 1000f720 f i asxavdecc.obj
 0001:0000e750       ?allocate@?$allocator@D@std@@QAEPADI@Z 1000f750 f i asxavdecc.obj
 0001:0000e780       ?assign@?$basic_string@DU?$char_traits@D@std@@V?$allocator@D@2@@std@@QAEAAV12@ABV12@II@Z 1000f780 f i asxavdecc.obj
 0001:0000e8b0       ?assign@?$basic_string@DU?$char_traits@D@std@@V?$allocator@D@2@@std@@QAEAAV12@PBD@Z 1000f8b0 f i asxavdecc.obj
 0001:0000e8f0       ?assign@?$basic_string@DU?$char_traits@D@std@@V?$allocator@D@2@@std@@QAEAAV12@PBDI@Z 1000f8f0 f i asxavdecc.obj
 0001:0000e9f0       ?assign@?$char_traits@D@std@@SAXAADABD@Z 1000f9f0 f i asxavdecc.obj
 0001:0000ea00       ?at@?$basic_string@DU?$char_traits@D@std@@V?$allocator@D@2@@std@@QAEAADI@Z 1000fa00 f i asxavdecc.obj
 0001:0000ea30       ?c_str@?$basic_string@DU?$char_traits@D@std@@V?$allocator@D@2@@std@@QBEPBDXZ 1000fa30 f i asxavdecc.obj
 0001:0000ea40       ?category@error_code@std@@QBEABVerror_category@2@XZ 1000fa40 f i asxavdecc.obj
 0001:0000ea50       ?category@error_condition@std@@QBEABVerror_category@2@XZ 1000fa50 f i asxavdecc.obj
 0001:0000ea60       ?copy@?$char_traits@D@std@@SAPADPADPBDI@Z 1000fa60 f i asxavdecc.obj
 0001:0000ea80       ?deallocate@?$_Wrap_alloc@V?$allocator@D@std@@@std@@QAEXPADI@Z 1000fa80 f i asxavdecc.obj
 0001:0000eaa0       ?deallocate@?$allocator@D@std@@QAEXPADI@Z 1000faa0 f i asxavdecc.obj
 0001:0000eac0       ?default_error_condition@_System_error_category@std@@UBE?AVerror_condition@2@H@Z 1000fac0 f i asxavdecc.obj
 0001:0000eb00       ?default_error_condition@error_category@std@@UBE?AVerror_condition@2@H@Z 1000fb00 f i asxavdecc.obj
 0001:0000eb20       ?equivalent@error_category@std@@UBE_NABVerror_code@2@H@Z 1000fb20 f i asxavdecc.obj
 0001:0000eb40       ?equivalent@error_category@std@@UBE_NHABVerror_condition@2@@Z 1000fb40 f i asxavdecc.obj
 0001:0000eb80       ?erase@?$basic_string@DU?$char_traits@D@std@@V?$allocator@D@2@@std@@QAEAAV12@I@Z 1000fb80 f i asxavdecc.obj
 0001:0000ebc0       ?erase@?$basic_string@DU?$char_traits@D@std@@V?$allocator@D@2@@std@@QAEAAV12@II@Z 1000fbc0 f i asxavdecc.obj
 0001:0000ec60       ?generic_category@std@@YAABVerror_category@1@XZ 1000fc60 f i asxavdecc.obj
 0001:0000ec70       ?getByte@asiMacAddr@@QBEEH@Z 1000fc70 f i asxavdecc.obj
 0001:0000ecc0       ?get_current_entity_and_descriptor@@YAHPAVend_station@avdecc_lib@@PAPAVentity_descriptor@2@PAPAVconfiguration_descriptor@2@@Z 1000fcc0 f   asxavdecc.obj
 0001:0000ed30       ?get_next_notification_id@@YAIXZ 1000fd30 f   asxavdecc.obj
 0001:0000ed40       ?length@?$basic_string@DU?$char_traits@D@std@@V?$allocator@D@2@@std@@QBEIXZ 1000fd40 f i asxavdecc.obj
 0001:0000ed50       ?length@?$char_traits@D@std@@SAIPBD@Z 1000fd50 f i asxavdecc.obj
 0001:0000ed70       ?max_size@?$_Wrap_alloc@V?$allocator@D@std@@@std@@QBEIXZ 1000fd70 f i asxavdecc.obj
 0001:0000ed80       ?max_size@?$allocator@D@std@@QBEIXZ 1000fd80 f i asxavdecc.obj
 0001:0000ed90       ?max_size@?$allocator_traits@V?$allocator@D@std@@@std@@SAIABV?$allocator@D@2@@Z 1000fd90 f i asxavdecc.obj
 0001:0000eda0       ?max_size@?$basic_string@DU?$char_traits@D@std@@V?$allocator@D@2@@std@@QBEIXZ 1000fda0 f i asxavdecc.obj
 0001:0000edb0       ?message@_Generic_error_category@std@@UBE?AV?$basic_string@DU?$char_traits@D@std@@V?$allocator@D@2@@2@H@Z 1000fdb0 f i asxavdecc.obj
 0001:0000ee20       ?message@_Iostream_error_category@std@@UBE?AV?$basic_string@DU?$char_traits@D@std@@V?$allocator@D@2@@2@H@Z 1000fe20 f i asxavdecc.obj
 0001:0000ee70       ?message@_System_error_category@std@@UBE?AV?$basic_string@DU?$char_traits@D@std@@V?$allocator@D@2@@2@H@Z 1000fe70 f i asxavdecc.obj
 0001:0000eee0       ?move@?$char_traits@D@std@@SAPADPADPBDI@Z 1000fee0 f i asxavdecc.obj
 0001:0000ef00       ?name@_Generic_error_category@std@@UBEPBDXZ 1000ff00 f i asxavdecc.obj
 0001:0000ef10       ?name@_Iostream_error_category@std@@UBEPBDXZ 1000ff10 f i asxavdecc.obj
 0001:0000ef20       ?name@_System_error_category@std@@UBEPBDXZ 1000ff20 f i asxavdecc.obj
 0001:0000ef30       ?size@?$basic_string@DU?$char_traits@D@std@@V?$allocator@D@2@@std@@QBEIXZ 1000ff30 f i asxavdecc.obj
 0001:0000ef40       ?system_category@std@@YAABVerror_category@1@XZ 1000ff40 f i asxavdecc.obj
 0001:0000ef50       ?to_string@std@@YA?AV?$basic_string@DU?$char_traits@D@std@@V?$allocator@D@2@@1@_K@Z 1000ff50 f i asxavdecc.obj
 0001:0000efe0       ?tostring@asiMacAddr@@QBEXPADD@Z 1000ffe0 f i asxavdecc.obj
 0001:0000f0a0       ?value@error_code@std@@QBEHXZ 100100a0 f i asxavdecc.obj
 0001:0000f0b0       ?value@error_condition@std@@QBEHXZ 100100b0 f i asxavdecc.obj
 0001:0000f0c0       _avdecc_log_callback       100100c0 f   asxavdecc.obj
 0001:0000f160       _avdecc_notification_callback 10010160 f   asxavdecc.obj
 0001:0000f230       _hypot                     10010230 f i asxavdecc.obj
 0001:0000f260       _DllMain@12                10010260 f   asx32.obj
 0001:0000f2d0       ??0asxAdapterASIO@@QAE@PAVasxSystem@@PAU_GUID@@PBD@Z 100102d0 f   asxasio.obj
 0001:0000f400       ??0asxMixerScanner@@QAE@PAVasxSubSystem@@@Z 10010400 f i asxasio.obj
 0001:0000f420       ??0asxMixerScannerASIO@@QAE@PAVasxSubSystem@@PAVasxAdapterASIO@@@Z 10010420 f   asxasio.obj
 0001:0000f440       ??0asxSubSystemASIO@@QAE@PAVasxSystem@@@Z 10010440 f   asxasio.obj
 0001:0000f470       ??1asxAdapterASIO@@UAE@XZ  10010470 f   asxasio.obj
 0001:0000f4f0       ??1asxMixerScanner@@UAE@XZ 100104f0 f i asxasio.obj
 0001:0000f500       ??1asxMixerScannerASIO@@UAE@XZ 10010500 f   asxasio.obj
 0001:0000f510       ??1asxSubSystemASIO@@UAE@XZ 10010510 f   asxasio.obj
 0001:0000f520       ??_GasxAdapterASIO@@UAEPAXI@Z 10010520 f i asxasio.obj
 0001:0000f520       ??_EasxAdapterASIO@@UAEPAXI@Z 10010520 f i asxasio.obj
 0001:0000f550       ??_EasxMixerScanner@@UAEPAXI@Z 10010550 f i asxasio.obj
 0001:0000f550       ??_GasxMixerScanner@@UAEPAXI@Z 10010550 f i asxasio.obj
 0001:0000f580       ??_GasxMixerScannerASIO@@UAEPAXI@Z 10010580 f i asxasio.obj
 0001:0000f580       ??_EasxMixerScannerASIO@@UAEPAXI@Z 10010580 f i asxasio.obj
 0001:0000f5b0       ??_GasxSubSystemASIO@@UAEPAXI@Z 100105b0 f i asxasio.obj
 0001:0000f5b0       ??_EasxSubSystemASIO@@UAEPAXI@Z 100105b0 f i asxasio.obj
 0001:0000f5e0       ?Add@?$TASIArray@VasxControlBase@@@@QAEHPAVasxControlBase@@@Z 100105e0 f i asxasio.obj
 0001:0000f610       ?Add@?$TASIArray@VasxNode@@@@QAEHPAVasxNode@@@Z 10010610 f i asxasio.obj
 0001:0000f640       ?Add@?$TASIArray@W4asxADAPTERMODE@@@@QAEHPAW4asxADAPTERMODE@@@Z 10010640 f i asxasio.obj
 0001:0000f670       ?Allocate@asxAdapterASIO@@QAEXXZ 10010670 f   asxasio.obj
 0001:0000f740       ?BufferSwitch@asxAdapterASIO@@QAEXJ@Z 10010740 f   asxasio.obj
 0001:0000f770       ?CheckSubSystems@asxAdapterASIO@@UAE?AW4asxERROR@@PAI0@Z 10010770 f i asxasio.obj
 0001:0000f790       ?Enlarge@?$TASIArray@VasxControlBase@@@@AAEXXZ 10010790 f i asxasio.obj
 0001:0000f7f0       ?Enlarge@?$TASIArray@VasxNode@@@@AAEXXZ 100107f0 f i asxasio.obj
 0001:0000f850       ?Enlarge@?$TASIArray@W4asxADAPTERMODE@@@@AAEXXZ 10010850 f i asxasio.obj
 0001:0000f8b0       ?Free@asxAdapterASIO@@QAEXXZ 100108b0 f   asxasio.obj
 0001:0000f8f0       ?GetAVDECCController@asxAdapter@@UAE?AW4asxERROR@@PAPAX@Z 100108f0 f i asxasio.obj
 0001:0000f900       ?GetAVDECCSystem@asxAdapter@@UAE?AW4asxERROR@@PAPAX@Z 10010900 f i asxasio.obj
 0001:0000f910       ?GetDriver@asxAdapterASIO@@QAEPAVAsioDriver@@XZ 10010910 f i asxasio.obj
 0001:0000f920       ?GetIpAddress@asxAdapterASIO@@UAE?AW4asxERROR@@PAD@Z 10010920 f i asxasio.obj
 0001:0000f940       ?GetMacAddress@asxAdapterASIO@@UAE?AW4asxERROR@@PAD@Z 10010940 f i asxasio.obj
 0001:0000f950       ?GetMode@asxAdapterASIO@@UAE?AW4asxERROR@@PAW4asxADAPTERMODE@@@Z 10010950 f i asxasio.obj
 0001:0000f970       ?ReScan@asxSubSystemASIO@@UAEXXZ 10010970 f   asxasio.obj
 0001:0000f980       ?ResetControls@asxMixerScanner@@UAE?AW4asxERROR@@XZ 10010980 f i asxasio.obj
 0001:0000f990       ?Scan@asxMixerScannerASIO@@EAEXPAVasxMixer@@@Z 10010990 f   asxasio.obj
 0001:0000fb40       ?Scan@asxSubSystemASIO@@UAEXXZ 10010b40 f   asxasio.obj
 0001:0000fd10       ?SetSampleType@asxAdapterASIO@@QAE?AW4asxERROR@@J@Z 10010d10 f   asxasio.obj
 0001:0000fd50       ?UpdateAdapterProperties@asxAdapter@@UAE?AW4asxERROR@@XZ 10010d50 f i asxasio.obj
 0001:0000fd60       ??0asxPlayerASIO@@QAE@PAVasxSubSystem@@PAVasxNode@@1PAVasxAdapterASIO@@@Z 10010d60 f   asxasioplay.obj
 0001:0000fdc0       ??1asxPlayerASIO@@UAE@XZ   10010dc0 f   asxasioplay.obj
 0001:0000fe20       ??A?$TASIArray@VasxPlayerFile@@@@QBEPAVasxPlayerFile@@H@Z 10010e20 f i asxasioplay.obj
 0001:0000fe40       ??_GasxPlayerASIO@@UAEPAXI@Z 10010e40 f i asxasioplay.obj
 0001:0000fe40       ??_EasxPlayerASIO@@UAEPAXI@Z 10010e40 f i asxasioplay.obj
 0001:0000fe70       ?AllocOutput@asxAdapterASIO@@QAE?AW4asxERROR@@PAPAUASIOBufferInfo@@PAJ@Z 10010e70 f i asxasioplay.obj
 0001:0000fec0       ?AllocOutput@asxPlayerASIO@@MAE?AW4asxERROR@@XZ 10010ec0 f   asxasioplay.obj
 0001:0000ff20       ?BufferSwitch@asxPlayerASIO@@QAEXJ@Z 10010f20 f   asxasioplay.obj
 0001:00010060       ?CurrentBase@asxPlayerFileList@@QAEPAVasxPlayerFile@@XZ 10011060 f i asxasioplay.obj
 0001:00010080       ?FreeOutput@asxAdapterASIO@@QAEXXZ 10011080 f i asxasioplay.obj
 0001:000100a0       ?FreeOutput@asxPlayerASIO@@MAE?AW4asxERROR@@XZ 100110a0 f   asxasioplay.obj
 0001:000100c0       ?GetBufferSize@asxAdapterASIO@@QAEJXZ 100110c0 f i asxasioplay.obj
 0001:000100d0       ?GetHpiControl@asxControlBase@@UAE?AW4asxERROR@@PAPAXPAI@Z 100110d0 f i asxasioplay.obj
 0001:000100e0       ?GetLoopMode@asxPlayer@@UAE?AW4asxERROR@@PAH@Z 100110e0 f i asxasioplay.obj
 0001:00010100       ?GetLooping@asxPlayerFileList@@QAEHXZ 10011100 f i asxasioplay.obj
 0001:00010110       ?GetPosition@asxPlayerASIO@@UAE?AW4asxERROR@@W4asxTIMESCALE@@PAK@Z 10011110 f   asxasioplay.obj
 0001:00010140       ?GetProperty@asxControlBase@@UAE?AW4asxERROR@@W4eControlProperty@1@W4eControlPropertyType@1@HPAX@Z 10011140 f i asxasioplay.obj
 0001:00010150       ?HelperThread@asxPlayerASIO@@UAEXXZ 10011150 f   asxasioplay.obj
 0001:000101a0       ?OnFileOpen@asxPlayerASIO@@MAE?AW4asxERROR@@XZ 100111a0 f   asxasioplay.obj
 0001:00010360       ?ResetOutput@asxPlayerASIO@@MAE?AW4asxERROR@@XZ 10011360 f i asxasioplay.obj
 0001:00010380       ?SetLoopMode@asxPlayer@@UAE?AW4asxERROR@@H@Z 10011380 f i asxasioplay.obj
 0001:00010390       ?SetLooping@asxPlayerFileList@@QAEXH@Z 10011390 f i asxasioplay.obj
 0001:000103a0       ?SetProperty@asxControlBase@@UAE?AW4asxERROR@@W4eControlProperty@1@W4eControlPropertyType@1@HPAX@Z 100113a0 f i asxasioplay.obj
 0001:000103b0       ?SetTimeScale@asxPlayerASIO@@UAE?AW4asxERROR@@M@Z 100113b0 f i asxasioplay.obj
 0001:000103c0       ?StartOutput@asxPlayerASIO@@MAE?AW4asxERROR@@XZ 100113c0 f   asxasioplay.obj
 0001:00010410       ?StartPlayer@asxAdapterASIO@@QAEXPAVasxPlayerASIO@@@Z 10011410 f i asxasioplay.obj
 0001:00010440       ?StopOutput@asxPlayerASIO@@MAE?AW4asxERROR@@XZ 10011440 f   asxasioplay.obj
 0001:00010490       ?StopPlayer@asxAdapterASIO@@QAEXXZ 10011490 f i asxasioplay.obj
 0001:000104b0       ?WavFormat@TWavFmt@@QAEPBUtWAVEFORMATEX@@XZ 100114b0 f i asxasioplay.obj
 0001:000104c0       ?deinterleave1@@YAXPAEPBEHHH@Z 100114c0 f   asxasioplay.obj
 0001:00010500       ?deinterleave2@@YAXPAEPBEHHH@Z 10011500 f   asxasioplay.obj
 0001:00010540       ?deinterleave3@@YAXPAEPBEHHH@Z 10011540 f   asxasioplay.obj
 0001:00010590       ?deinterleave4@@YAXPAEPBEHHH@Z 10011590 f   asxasioplay.obj
 0001:000105d0       ?waveFormat2AsioType@@YAJPBUtWAVEFORMATEX@@@Z 100115d0 f   asxasioplay.obj
 0001:00010660       ??0asxRecorderASIO@@QAE@PAVasxSubSystem@@PAVasxNode@@1PAVasxAdapterASIO@@@Z 10011660 f   asxasiorec.obj
 0001:000106b0       ??1asxRecorderASIO@@UAE@XZ 100116b0 f   asxasiorec.obj
 0001:00010710       ??_GasxRecorderASIO@@UAEPAXI@Z 10011710 f i asxasiorec.obj
 0001:00010710       ??_EasxRecorderASIO@@UAEPAXI@Z 10011710 f i asxasiorec.obj
 0001:00010740       ?AllocInput@asxAdapterASIO@@QAE?AW4asxERROR@@PAPAUASIOBufferInfo@@PAJ@Z 10011740 f i asxasiorec.obj
 0001:000107a0       ?AllocInput@asxRecorderASIO@@MAE?AW4asxERROR@@XZ 100117a0 f   asxasiorec.obj
 0001:00010800       ?BufferSwitch@asxRecorderASIO@@QAEXJ@Z 10011800 f   asxasiorec.obj
 0001:00010900       ?EnumerateAllFormats@asxRecorderASIO@@MAEXXZ 10011900 f   asxasiorec.obj
 0001:00010910       ?FreeInput@asxAdapterASIO@@QAEXXZ 10011910 f i asxasiorec.obj
 0001:00010930       ?FreeInput@asxRecorderASIO@@MAE?AW4asxERROR@@XZ 10011930 f   asxasiorec.obj
 0001:00010950       ?GetInputPosition@asxRecorderASIO@@MAE?AW4asxERROR@@PAK@Z 10011950 f   asxasiorec.obj
 0001:00010970       ?HelperThread@asxRecorderASIO@@UAEKXZ 10011970 f   asxasiorec.obj
 0001:000109d0       ?SetInputFormat@asxRecorderASIO@@MAE?AW4asxERROR@@XZ 100119d0 f   asxasiorec.obj
 0001:000109e0       ?StartInput@asxRecorderASIO@@MAE?AW4asxERROR@@XZ 100119e0 f   asxasiorec.obj
 0001:00010a30       ?StartRecorder@asxAdapterASIO@@QAEXPAVasxRecorderASIO@@@Z 10011a30 f i asxasiorec.obj
 0001:00010a60       ?StopInput@asxRecorderASIO@@MAE?AW4asxERROR@@XZ 10011a60 f   asxasiorec.obj
 0001:00010ab0       ?StopRecorder@asxAdapterASIO@@QAEXXZ 10011ab0 f i asxasiorec.obj
 0001:00010ad0       ?interleave1@@YAXPAEPBEHHH@Z 10011ad0 f   asxasiorec.obj
 0001:00010b10       ?interleave2@@YAXPAEPBEHHH@Z 10011b10 f   asxasiorec.obj
 0001:00010b50       ?interleave3@@YAXPAEPBEHHH@Z 10011b50 f   asxasiorec.obj
 0001:00010ba0       ?interleave4@@YAXPAEPBEHHH@Z 10011ba0 f   asxasiorec.obj
 0001:00010be0       ??0?$TASIArray@VasxAdapter@@@@QAE@XZ 10011be0 f i asxclass.obj
 0001:00010c00       ??0?$TASIArray@VasxCallbackObject@@@@QAE@XZ 10011c00 f i asxclass.obj
 0001:00010c20       ??0?$TASIArray@VasxControlBase@@@@QAE@XZ 10011c20 f i asxclass.obj
 0001:00010c40       ??0?$TASIArray@VasxMixerScanner@@@@QAE@XZ 10011c40 f i asxclass.obj
 0001:00010c60       ??0?$TASIArray@VasxNode@@@@QAE@XZ 10011c60 f i asxclass.obj
 0001:00010c80       ??0?$TASIArray@VasxSubSystem@@@@QAE@XZ 10011c80 f i asxclass.obj
 0001:00010ca0       ??0?$TASIArray@W4asxADAPTERMODE@@@@QAE@XZ 10011ca0 f i asxclass.obj
 0001:00010cc0       ??0TASICString@@QAE@PBD@Z  10011cc0 f i asxclass.obj
 0001:00010ce0       ??0asxAbstractAdapter@@QAE@PAVasxAdapter@@@Z 10011ce0 f   asxclass.obj
 0001:00010dd0       ??0asxAdapter@@QAE@PAV0@@Z 10011dd0 f   asxclass.obj
 0001:00010eb0       ??0asxAdapter@@QAE@PAVasxSystem@@IPBDH1@Z 10011eb0 f   asxclass.obj
 0001:00010fa0       ??0asxBase@@QAE@HH@Z       10011fa0 f   asxclass.obj
 0001:00010fe0       ??0asxBlockProperty@@QAE@W4asxUCONTROL_PTYPE@@W4asxUCONTROL_PFLAGS@@IPBDPAUasxParameterRangeInfo@@2@Z 10011fe0 f   asxclass.obj
 0001:00011070       ??0asxControlBase@@QAE@AAV0@@Z 10012070 f   asxclass.obj
 0001:000110b0       ??0asxControlBase@@QAE@PAVasxSubSystem@@HPAVasxNode@@1@Z 100120b0 f   asxclass.obj
 0001:000110e0       ??0asxMixer@@QAE@PAVasxSystem@@@Z 100120e0 f i asxclass.obj
 0001:00011160       ??0asxNode@@QAE@PAVasxSubSystem@@HH@Z 10012160 f   asxclass.obj
 0001:000111b0       ??0asxSubSystem@@QAE@PAVasxSystem@@PBDH@Z 100121b0 f   asxclass.obj
 0001:00011250       ??0asxSystem@@QAE@PBD@Z    10012250 f   asxclass.obj
 0001:00011350       ??1?$TASIArray@VasxAdapter@@@@QAE@XZ 10012350 f i asxclass.obj
 0001:000113a0       ??1?$TASIArray@VasxCallbackObject@@@@QAE@XZ 100123a0 f i asxclass.obj
 0001:000113f0       ??1?$TASIArray@VasxControlBase@@@@QAE@XZ 100123f0 f i asxclass.obj
 0001:00011440       ??1?$TASIArray@VasxMixerScanner@@@@QAE@XZ 10012440 f i asxclass.obj
 0001:00011490       ??1?$TASIArray@VasxNode@@@@QAE@XZ 10012490 f i asxclass.obj
 0001:000114e0       ??1?$TASIArray@VasxSubSystem@@@@QAE@XZ 100124e0 f i asxclass.obj
 0001:00011530       ??1?$TASIArray@W4asxADAPTERMODE@@@@QAE@XZ 10012530 f i asxclass.obj
 0001:00011580       ??1TASICString@@QAE@XZ     10012580 f i asxclass.obj
 0001:000115a0       ??1asxAbstractAdapter@@UAE@XZ 100125a0 f   asxclass.obj
 0001:00011620       ??1asxAdapter@@UAE@XZ      10012620 f   asxclass.obj
 0001:000116b0       ??1asxBase@@UAE@XZ         100126b0 f i asxclass.obj
 0001:000116d0       ??1asxBlockProperty@@UAE@XZ 100126d0 f   asxclass.obj
 0001:00011740       ??1asxControlBase@@UAE@XZ  10012740 f i asxclass.obj
 0001:00011760       ??1asxMixer@@UAE@XZ        10012760 f   asxclass.obj
 0001:00011800       ??1asxNode@@UAE@XZ         10012800 f i asxclass.obj
 0001:00011820       ??1asxSubSystem@@UAE@XZ    10012820 f   asxclass.obj
 0001:00011850       ??1asxSystem@@UAE@XZ       10012850 f   asxclass.obj
 0001:00011980       ??8asxAdapter@@QAE_NAAV0@@Z 10012980 f   asxclass.obj
 0001:00011ab0       ??A?$TASIArray@H@@QBEPAHH@Z 10012ab0 f i asxclass.obj
 0001:00011ad0       ??A?$TASIArray@VasxAdapter@@@@QBEPAVasxAdapter@@H@Z 10012ad0 f i asxclass.obj
 0001:00011af0       ??A?$TASIArray@VasxBlockProperty@@@@QBEPAVasxBlockProperty@@H@Z 10012af0 f i asxclass.obj
 0001:00011b10       ??A?$TASIArray@VasxControlBase@@@@QBEPAVasxControlBase@@H@Z 10012b10 f i asxclass.obj
 0001:00011b30       ??A?$TASIArray@VasxMixerScanner@@@@QBEPAVasxMixerScanner@@H@Z 10012b30 f i asxclass.obj
 0001:00011b50       ??A?$TASIArray@VasxNode@@@@QBEPAVasxNode@@H@Z 10012b50 f i asxclass.obj
 0001:00011b70       ??A?$TASIArray@VasxSubSystem@@@@QBEPAVasxSubSystem@@H@Z 10012b70 f i asxclass.obj
 0001:00011b90       ??A?$TASIArray@W4asxADAPTERMODE@@@@QBEPAW4asxADAPTERMODE@@H@Z 10012b90 f i asxclass.obj
 0001:00011bb0       ??A?$TASIArray@W4asxAESEBU_FORMAT@@@@QBEPAW4asxAESEBU_FORMAT@@H@Z 10012bb0 f i asxclass.obj
 0001:00011bd0       ??A?$TASIArray@W4asxCHANNELMODE@@@@QBEPAW4asxCHANNELMODE@@H@Z 10012bd0 f i asxclass.obj
 0001:00011bf0       ??A?$TASIArray@W4asxNODE@@@@QBEPAW4asxNODE@@H@Z 10012bf0 f i asxclass.obj
 0001:00011c10       ??A?$TASIArray@W4asxSAMPLE_CLOCK_SOURCE@@@@QBEPAW4asxSAMPLE_CLOCK_SOURCE@@H@Z 10012c10 f i asxclass.obj
 0001:00011c30       ??A?$TASIArray@W4asxSAMPLE_RATE@@@@QBEPAW4asxSAMPLE_RATE@@H@Z 10012c30 f i asxclass.obj
 0001:00011c50       ??A?$TASIArray@W4asxTUNERBAND@@@@QBEPAW4asxTUNERBAND@@H@Z 10012c50 f i asxclass.obj
 0001:00011c70       ??A?$TASIArray@W4asxTUNERPROGRAM@@@@QBEPAW4asxTUNERPROGRAM@@H@Z 10012c70 f i asxclass.obj
 0001:00011c90       ??BTASICString@@QAEPBDXZ   10012c90 f i asxclass.obj
 0001:00011ca0       ??_EasxAbstractAdapter@@UAEPAXI@Z 10012ca0 f i asxclass.obj
 0001:00011ca0       ??_GasxAbstractAdapter@@UAEPAXI@Z 10012ca0 f i asxclass.obj
 0001:00011cd0       ??_GasxAdapter@@UAEPAXI@Z  10012cd0 f i asxclass.obj
 0001:00011cd0       ??_EasxAdapter@@UAEPAXI@Z  10012cd0 f i asxclass.obj
 0001:00011d00       ??_EasxBase@@UAEPAXI@Z     10012d00 f i asxclass.obj
 0001:00011d00       ??_GasxBase@@UAEPAXI@Z     10012d00 f i asxclass.obj
 0001:00011d40       ??_EasxBlockProperty@@UAEPAXI@Z 10012d40 f i asxclass.obj
 0001:00011d40       ??_GasxBlockProperty@@UAEPAXI@Z 10012d40 f i asxclass.obj
 0001:00011d70       ??_GasxControlBase@@UAEPAXI@Z 10012d70 f i asxclass.obj
 0001:00011d70       ??_EasxControlBase@@UAEPAXI@Z 10012d70 f i asxclass.obj
 0001:00011db0       ??_EasxMixer@@UAEPAXI@Z    10012db0 f i asxclass.obj
 0001:00011db0       ??_GasxMixer@@UAEPAXI@Z    10012db0 f i asxclass.obj
 0001:00011de0       ??_EasxNode@@UAEPAXI@Z     10012de0 f i asxclass.obj
 0001:00011de0       ??_GasxNode@@UAEPAXI@Z     10012de0 f i asxclass.obj
 0001:00011e20       ??_EasxSubSystem@@UAEPAXI@Z 10012e20 f i asxclass.obj
 0001:00011e20       ??_GasxSubSystem@@UAEPAXI@Z 10012e20 f i asxclass.obj
 0001:00011e50       ??_GasxSystem@@UAEPAXI@Z   10012e50 f i asxclass.obj
 0001:00011e50       ??_EasxSystem@@UAEPAXI@Z   10012e50 f i asxclass.obj
 0001:00011e80       ?AdapterExists@asxSystem@@QAE_NPAVasxAdapter@@@Z 10012e80 f   asxclass.obj
 0001:00011ea0       ?Add@?$TASIArray@VasxAdapter@@@@QAEHPAVasxAdapter@@@Z 10012ea0 f i asxclass.obj
 0001:00011ed0       ?Add@?$TASIArray@VasxCallbackObject@@@@QAEHPAVasxCallbackObject@@@Z 10012ed0 f i asxclass.obj
 0001:00011f00       ?Add@?$TASIArray@VasxMixerScanner@@@@QAEHPAVasxMixerScanner@@@Z 10012f00 f i asxclass.obj
 0001:00011f30       ?Add@?$TASIArray@VasxSubSystem@@@@QAEHPAVasxSubSystem@@@Z 10012f30 f i asxclass.obj
 0001:00011f60       ?AddAdapter@asxSystem@@QAE?AW4asxERROR@@PAVasxAdapter@@PAVasxMixerScanner@@@Z 10012f60 f   asxclass.obj
 0001:00012050       ?AddAdapterObject@asxAbstractAdapter@@QAEXPAVasxAdapter@@@Z 10013050 f   asxclass.obj
 0001:00012250       ?AddSubSystem@asxSystem@@QAE?AW4asxERROR@@H@Z 10013250 f   asxclass.obj
 0001:00012320       ?CallbackThread@asxSystem@@QAEXXZ 10013320 f   asxclass.obj
 0001:00012390       ?CheckForControlRefresh@asxAbstractAdapter@@QAEXXZ 10013390 f   asxclass.obj
 0001:000125e0       ?CheckForMixerRefresh@asxSystem@@QAEXXZ 100135e0 f   asxclass.obj
 0001:00012610       ?CheckSubSystems@asxAbstractAdapter@@UAE?AW4asxERROR@@PAI0@Z 10013610 f   asxclass.obj
 0001:00012670       ?CheckSubSystems@asxAdapter@@UAE?AW4asxERROR@@PAI0@Z 10013670 f i asxclass.obj
 0001:00012680       ?Clear@?$TASIArray@VasxAdapter@@@@QAEXXZ 10013680 f i asxclass.obj
 0001:000126c0       ?Clear@?$TASIArray@VasxCallbackObject@@@@QAEXXZ 100136c0 f i asxclass.obj
 0001:00012700       ?Clear@?$TASIArray@VasxControlBase@@@@QAEXXZ 10013700 f i asxclass.obj
 0001:00012740       ?Clear@?$TASIArray@VasxMixerScanner@@@@QAEXXZ 10013740 f i asxclass.obj
 0001:00012780       ?Clear@?$TASIArray@VasxNode@@@@QAEXXZ 10013780 f i asxclass.obj
 0001:000127c0       ?Clear@?$TASIArray@VasxSubSystem@@@@QAEXXZ 100137c0 f i asxclass.obj
 0001:00012800       ?Count@?$TASIArray@VasxBlockProperty@@@@QBEHXZ 10013800 f i asxclass.obj
 0001:00012810       ?Count@?$TASIArray@VasxControlBase@@@@QBEHXZ 10013810 f i asxclass.obj
 0001:00012820       ?Count@?$TASIArray@VasxMixerScanner@@@@QBEHXZ 10013820 f i asxclass.obj
 0001:00012830       ?Count@?$TASIArray@VasxNode@@@@QBEHXZ 10013830 f i asxclass.obj
 0001:00012840       ?Count@?$TASIArray@VasxSubSystem@@@@QBEHXZ 10013840 f i asxclass.obj
 0001:00012850       ?Count@?$TASIArray@W4asxADAPTERMODE@@@@QBEHXZ 10013850 f i asxclass.obj
 0001:00012860       ?Count@?$TASIArray@W4asxAESEBU_FORMAT@@@@QBEHXZ 10013860 f i asxclass.obj
 0001:00012870       ?Count@?$TASIArray@W4asxCHANNELMODE@@@@QBEHXZ 10013870 f i asxclass.obj
 0001:00012880       ?Count@?$TASIArray@W4asxNODE@@@@QBEHXZ 10013880 f i asxclass.obj
 0001:00012890       ?Count@?$TASIArray@W4asxSAMPLE_CLOCK_SOURCE@@@@QBEHXZ 10013890 f i asxclass.obj
 0001:000128a0       ?Count@?$TASIArray@W4asxSAMPLE_RATE@@@@QBEHXZ 100138a0 f i asxclass.obj
 0001:000128b0       ?Count@?$TASIArray@W4asxTUNERBAND@@@@QBEHXZ 100138b0 f i asxclass.obj
 0001:000128c0       ?Count@?$TASIArray@W4asxTUNERPROGRAM@@@@QBEHXZ 100138c0 f i asxclass.obj
 0001:000128d0       ?CountNodesOfType@asxMixer@@QAEHHPAVasxSubSystem@@@Z 100138d0 f   asxclass.obj
 0001:00012980       ?DeleteAll@asxSystem@@SAXXZ 10013980 f   asxclass.obj
 0001:000129b0       ?DeleteContents@asxMixer@@QAEXXZ 100139b0 f   asxclass.obj
 0001:000129d0       ?Enlarge@?$TASIArray@VasxAdapter@@@@AAEXXZ 100139d0 f i asxclass.obj
 0001:00012a30       ?Enlarge@?$TASIArray@VasxCallbackObject@@@@AAEXXZ 10013a30 f i asxclass.obj
 0001:00012a90       ?Enlarge@?$TASIArray@VasxMixerScanner@@@@AAEXXZ 10013a90 f i asxclass.obj
 0001:00012af0       ?Enlarge@?$TASIArray@VasxSubSystem@@@@AAEXXZ 10013af0 f i asxclass.obj
 0001:00012b50       ?Enumerate@asxMode@@QAE?AW4asxERROR@@HPAW4asxCHANNELMODE@@PAH@Z 10013b50 f   asxclass.obj
 0001:00012b90       ?Enumerate@asxMux@@QAE?AW4asxERROR@@HPAW4asxNODE@@PAH1@Z 10013b90 f   asxclass.obj
 0001:00012be0       ?EnumerateBand@asxTuner@@QAE?AW4asxERROR@@HPAW4asxTUNERBAND@@PAH@Z 10013be0 f   asxclass.obj
 0001:00012c20       ?EnumerateClockSource@asxSampleClock@@QAE?AW4asxERROR@@HPAW4asxSAMPLE_CLOCK_SOURCE@@PAH@Z 10013c20 f   asxclass.obj
 0001:00012c60       ?EnumerateFormat@asxAes3Rx@@QAE?AW4asxERROR@@HPAW4asxAESEBU_FORMAT@@PAH@Z 10013c60 f   asxclass.obj
 0001:00012ca0       ?EnumerateFormat@asxAes3Tx@@QAE?AW4asxERROR@@HPAW4asxAESEBU_FORMAT@@PAH@Z 10013ca0 f   asxclass.obj
 0001:00012ce0       ?EnumerateHdBlend@asxTuner@@QAE?AW4asxERROR@@HPAW4asxTUNERHDBLEND@@PAH@Z 10013ce0 f   asxclass.obj
 0001:00012d20       ?EnumerateLocalRate@asxSampleClock@@QAE?AW4asxERROR@@HPAW4asxSAMPLE_RATE@@PAH@Z 10013d20 f   asxclass.obj
 0001:00012d60       ?EnumerateMode@asxAdapter@@QAE?AW4asxERROR@@HPAW4asxADAPTERMODE@@PAH@Z 10013d60 f   asxclass.obj
 0001:00012da0       ?EnumerateProgram@asxTuner@@QAE?AW4asxERROR@@HPAW4asxTUNERPROGRAM@@PAH@Z 10013da0 f   asxclass.obj
 0001:00012df0       ?EnumerateProperty@asxAbstractAdapter@@UAE?AW4asxERROR@@HW4asxADPROPENUM_MODE@@HPAK@Z 10013df0 f   asxclass.obj
 0001:00012e60       ?Error_GetLast@asxBase@@QAE?AW4asxERROR@@PAW42@PAH@Z 10013e60 f   asxclass.obj
 0001:00012e80       ?Error_GetLastString@asxBase@@QAE?AW4asxERROR@@PADHPAH0H1@Z 10013e80 f   asxclass.obj
 0001:00012f60       ?Find@?$TASIArray@VasxAdapter@@@@QAEHPAVasxAdapter@@@Z 10013f60 f i asxclass.obj
 0001:00012fa0       ?FindASXErrorString@asxBase@@AAEPADH@Z 10013fa0 f   asxclass.obj
 0001:00013000       ?FindAdapter@asxSystem@@QAE?AW4asxERROR@@PAPAVasxAdapter@@PAV3@@Z 10014000 f   asxclass.obj
 0001:00013040       ?FindAdapterFromSubSytem@asxSystem@@QAE?AW4asxERROR@@PAPAVasxAdapter@@PAV3@@Z 10014040 f   asxclass.obj
 0001:00013080       ?GetASXErrorCode@asxBase@@QAE?AW4asxERROR@@XZ 10014080 f i asxclass.obj
 0001:00013090       ?GetASXErrorString@asxBase@@QAEXPAPAD@Z 10014090 f   asxclass.obj
 0001:000130b0       ?GetAVDECCController@asxAbstractAdapter@@UAE?AW4asxERROR@@PAPAX@Z 100140b0 f   asxclass.obj
 0001:00013110       ?GetAVDECCSystem@asxAbstractAdapter@@UAE?AW4asxERROR@@PAPAX@Z 10014110 f   asxclass.obj
 0001:00013170       ?GetAdapter@asxSystem@@QAE?AW4asxERROR@@HPAPAVasxAdapter@@@Z 10014170 f   asxclass.obj
 0001:000131a0       ?GetAdapterCount@asxSystem@@QAE?AW4asxERROR@@PAH@Z 100141a0 f   asxclass.obj
 0001:000131e0       ?GetAdapterObjectForSubSystem@asxAbstractAdapter@@QAEPAVasxAdapter@@I@Z 100141e0 f i asxclass.obj
 0001:00013200       ?GetBlockControlByNodeTypeAndIndex@asxMixer@@QAE?AW4asxERROR@@W4asxNODE@@H0HPBDPAPAVasxControlBase@@@Z 10014200 f   asxclass.obj
 0001:00013300       ?GetControl@asxMixer@@QAE?AW4asxERROR@@HHHHHPAPAVasxControlBase@@@Z 10014300 f   asxclass.obj
 0001:00013340       ?GetControl@asxMixer@@QAE?AW4asxERROR@@HHHHPAVasxSubSystem@@HPAPAVasxControlBase@@@Z 10014340 f   asxclass.obj
 0001:00013380       ?GetControl@asxMixer@@QAE?AW4asxERROR@@HHHPAPAVasxControlBase@@@Z 10014380 f   asxclass.obj
 0001:000133b0       ?GetControl@asxMixer@@QAE?AW4asxERROR@@HPAPAVasxControlBase@@@Z 100143b0 f   asxclass.obj
 0001:000133f0       ?GetControl@asxMixer@@QAE?AW4asxERROR@@PAVasxNode@@0HPAPAVasxControlBase@@@Z 100143f0 f   asxclass.obj
 0001:00013420       ?GetControlByNode@asxMixer@@QAE?AW4asxERROR@@PAVasxNode@@0W4asxCONTROL@@PAPAVasxControlBase@@@Z 10014420 f   asxclass.obj
 0001:00013430       ?GetControlByNodeTypeAndIndex@asxMixer@@QAE?AW4asxERROR@@W4asxNODE@@H0HW4asxCONTROL@@PAPAVasxControlBase@@@Z 10014430 f   asxclass.obj
 0001:00013440       ?GetControlCount@asxMixer@@QAE?AW4asxERROR@@PAH@Z 10014440 f   asxclass.obj
 0001:00013460       ?GetControlWithStartingIndex@asxMixer@@AAE?AW4asxERROR@@PAVasxNode@@0HPAPAVasxControlBase@@PAH@Z 10014460 f   asxclass.obj
 0001:00013570       ?GetDestination@asxControlBase@@QAEPAVasxNode@@XZ 10014570 f i asxclass.obj
 0001:00013580       ?GetDestinationNode@asxMixer@@QAE?AW4asxERROR@@HPAPAVasxNode@@@Z 10014580 f   asxclass.obj
 0001:000135c0       ?GetDestinationNodeCount@asxMixer@@QAE?AW4asxERROR@@PAH@Z 100145c0 f   asxclass.obj
 0001:000135e0       ?GetDspUtilization@asxAbstractAdapter@@UAE?AW4asxERROR@@HPAH@Z 100145e0 f   asxclass.obj
 0001:00013640       ?GetElementCount@asxBlock@@UAE?AW4asxERROR@@IPAI@Z 10014640 f   asxclass.obj
 0001:00013670       ?GetElementCount@asxBlockProperty@@UAE?AW4asxERROR@@PAI@Z 10014670 f   asxclass.obj
 0001:00013690       ?GetEnumName@asxBlockHPI@@UAE?AW4asxERROR@@IIPADI@Z 10014690 f   asxclass.obj
 0001:00013780       ?GetFirmwareRevision@asxAdapter@@QAE?AW4asxERROR@@PAD@Z 10014780 f   asxclass.obj
 0001:000137a0       ?GetFlags@asxBlock@@UAE?AW4asxERROR@@IPAW4asxUCONTROL_PFLAGS@@@Z 100147a0 f   asxclass.obj
 0001:000137d0       ?GetFlags@asxBlockProperty@@UAE?AW4asxERROR@@PAW4asxUCONTROL_PFLAGS@@@Z 100147d0 f   asxclass.obj
 0001:000137f0       ?GetHardwareRevision@asxAdapter@@QAE?AW4asxERROR@@PAD@Z 100147f0 f   asxclass.obj
 0001:00013810       ?GetIndex@asxAdapter@@QAE?AW4asxERROR@@PAH@Z 10014810 f   asxclass.obj
 0001:00013830       ?GetIpAddress@asxAbstractAdapter@@UAE?AW4asxERROR@@PAD@Z 10014830 f   asxclass.obj
 0001:000138e0       ?GetIpAddress@asxAdapter@@UAE?AW4asxERROR@@PAD@Z 100148e0 f i asxclass.obj
 0001:000138f0       ?GetLocation@asxNode@@QAE?AW4asxERROR@@PAH0PADH@Z 100148f0 f   asxclass.obj
 0001:00013960       ?GetMacAddress@asxAbstractAdapter@@UAE?AW4asxERROR@@PAD@Z 10014960 f   asxclass.obj
 0001:000139c0       ?GetMacAddress@asxAdapter@@UAE?AW4asxERROR@@PAD@Z 100149c0 f   asxclass.obj
 0001:00013a30       ?GetMessageLogging@asxSystem@@QAE?AW4asxERROR@@PAW4asxMSG_LOGGING@@@Z 10014a30 f   asxclass.obj
 0001:00013a50       ?GetMixer@asxAdapter@@QAE?AW4asxERROR@@PAPAVasxMixer@@@Z 10014a50 f   asxclass.obj
 0001:00013aa0       ?GetMode@asxAbstractAdapter@@UAE?AW4asxERROR@@PAW4asxADAPTERMODE@@@Z 10014aa0 f   asxclass.obj
 0001:00013b00       ?GetName@asxAdapter@@UAE?AW4asxERROR@@PADHPAH@Z 10014b00 f   asxclass.obj
 0001:00013b70       ?GetName@asxBlock@@UAE?AW4asxERROR@@IPADI@Z 10014b70 f   asxclass.obj
 0001:00013ba0       ?GetName@asxBlockProperty@@UAE?AW4asxERROR@@PADI@Z 10014ba0 f   asxclass.obj
 0001:00013bc0       ?GetName@asxNode@@QAE?AW4asxERROR@@PADH@Z 10014bc0 f   asxclass.obj
 0001:00013d80       ?GetName@asxSubSystem@@QAE?AW4asxERROR@@PADHPAH@Z 10014d80 f   asxclass.obj
 0001:00013df0       ?GetName@asxSystem@@QAE?AW4asxERROR@@PADHPAH@Z 10014df0 f   asxclass.obj
 0001:00013e60       ?GetNamePtr@asxAdapter@@QAEPADXZ 10014e60 f i asxclass.obj
 0001:00013e70       ?GetNode@asxMixer@@QAEPAVasxNode@@HHPAVasxSubSystem@@@Z 10014e70 f   asxclass.obj
 0001:00013f50       ?GetNodeByType@asxMixer@@QAE?AW4asxERROR@@W4asxNODE@@HPAPAVasxNode@@@Z 10014f50 f   asxclass.obj
 0001:00013fa0       ?GetNodeByType@asxMixer@@QAE?AW4asxERROR@@W4asxNODE@@HPAVasxSubSystem@@PAPAVasxNode@@@Z 10014fa0 f   asxclass.obj
 0001:00013ff0       ?GetNodeTypeCount@asxMixer@@QAE?AW4asxERROR@@W4asxNODE@@PAH@Z 10014ff0 f   asxclass.obj
 0001:00014010       ?GetNodeTypeCount@asxMixer@@QAE?AW4asxERROR@@W4asxNODE@@PAVasxSubSystem@@PAH@Z 10015010 f   asxclass.obj
 0001:00014030       ?GetRange@asxBlock@@UAE?AW4asxERROR@@IPAUasxParameterRangeInfo@@@Z 10015030 f   asxclass.obj
 0001:00014090       ?GetRange@asxBlockProperty@@UAE?AW4asxERROR@@PAUasxParameterRangeInfo@@@Z 10015090 f   asxclass.obj
 0001:000140b0       ?GetSource@asxControlBase@@QAEPAVasxNode@@XZ 100150b0 f i asxclass.obj
 0001:000140c0       ?GetSourceNode@asxMixer@@QAE?AW4asxERROR@@HPAPAVasxNode@@@Z 100150c0 f   asxclass.obj
 0001:00014100       ?GetSourceNodeCount@asxMixer@@QAE?AW4asxERROR@@PAH@Z 10015100 f   asxclass.obj
 0001:00014120       ?GetSubSystem@asxAdapter@@QAEIXZ 10015120 f i asxclass.obj
 0001:00014130       ?GetSubSystem@asxNode@@QAEPAVasxSubSystem@@XZ 10015130 f i asxclass.obj
 0001:00014140       ?GetSubSystem@asxSystem@@QAE?AW4asxERROR@@HPAPAVasxSubSystem@@@Z 10015140 f   asxclass.obj
 0001:00014170       ?GetSubSystemByType@asxSystem@@QAE?AW4asxERROR@@HPAPAVasxSubSystem@@@Z 10015170 f   asxclass.obj
 0001:000141e0       ?GetSubsystemErrorCode@asxBase@@QAEIXZ 100151e0 f i asxclass.obj
 0001:000141f0       ?GetSubsystemErrorString@asxBase@@QAEXPAPAD@Z 100151f0 f   asxclass.obj
 0001:00014220       ?GetType@asxBlock@@UAE?AW4asxERROR@@IPAW4asxUCONTROL_PTYPE@@@Z 10015220 f   asxclass.obj
 0001:00014250       ?GetType@asxBlockProperty@@UAE?AW4asxERROR@@PAW4asxUCONTROL_PTYPE@@@Z 10015250 f   asxclass.obj
 0001:00014270       ?GetUnits@asxBlock@@UAE?AW4asxERROR@@IPADI@Z 10015270 f   asxclass.obj
 0001:000142a0       ?GetUnits@asxBlockProperty@@UAE?AW4asxERROR@@PADI@Z 100152a0 f   asxclass.obj
 0001:000142c0       ?GetVersion@asxSubSystem@@QAE?AW4asxERROR@@PADHPAH0H1@Z 100152c0 f   asxclass.obj
 0001:00014390       ?GetVersion@asxSystem@@QAE?AW4asxERROR@@PADHPAH0H1@Z 10015390 f   asxclass.obj
 0001:00014460       ?GetVersion@asxSystem@@QAE?AW4asxERROR@@PAPAD0@Z 10015460 f   asxclass.obj
 0001:00014480       ?HasSubSystem@asxAbstractAdapter@@QAE?AW4asxERROR@@H@Z 10015480 f   asxclass.obj
 0001:000144a0       ?InvokeErrorCallback@asxBase@@QAEHPAXPBDW4asxERROR@@@Z 100154a0 f   asxclass.obj
 0001:000144e0       ?MarkedForControlRefresh@asxAdapter@@QAE_NXZ 100154e0 f i asxclass.obj
 0001:000144f0       ?Pop@?$TASIArray@VasxCallbackObject@@@@QAEPAVasxCallbackObject@@XZ 100154f0 f i asxclass.obj
 0001:00014530       ?PostCallback@asxSystem@@QAEXPAVasxCallbackObject@@@Z 10015530 f   asxclass.obj
 0001:00014590       ?Predelete@asxAbstractAdapter@@UAE?AW4asxERROR@@XZ 10015590 f   asxclass.obj
 0001:000145e0       ?Predelete@asxSystem@@QAE?AW4asxERROR@@XZ 100155e0 f   asxclass.obj
 0001:000146d0       ?ReadNvMem@asxAbstractAdapter@@UAE?AW4asxERROR@@HPAE@Z 100156d0 f   asxclass.obj
 0001:00014730       ?ReadProperty@asxAbstractAdapter@@UAE?AW4asxERROR@@HPAG0@Z 10015730 f   asxclass.obj
 0001:000147a0       ?RegisterErrorCallback@asxSystem@@QAE?AW4asxERROR@@P6AXPAXPBD00@Z00@Z 100157a0 f   asxclass.obj
 0001:000147d0       ?ResetControls@asxMixer@@QAE?AW4asxERROR@@XZ 100157d0 f   asxclass.obj
 0001:00014800       ?SetASXErrorCode@asxBase@@QAE?AW4asxERROR@@W42@@Z 10015800 f   asxclass.obj
 0001:00014840       ?SetLocationInformation@asxNode@@QAEXHHH@Z 10015840 f   asxclass.obj
 0001:00014860       ?SetMessageLogging@asxSystem@@QAE?AW4asxERROR@@W4asxMSG_LOGGING@@@Z 10015860 f   asxclass.obj
 0001:00014880       ?SetMode@asxAbstractAdapter@@UAE?AW4asxERROR@@W4asxADAPTERMODE@@@Z 10015880 f   asxclass.obj
 0001:000148e0       ?SetSubSystemErrorCode@asxBase@@QAEXHPAD@Z 100158e0 f   asxclass.obj
 0001:00014910       ?TranslateSpecificErrorCode@asxSystem@@UAEXIPAPBD@Z 10015910 f i asxclass.obj
 0001:00014920       ?WriteNvMem@asxAbstractAdapter@@UAE?AW4asxERROR@@HE@Z 10015920 f   asxclass.obj
 0001:00014980       ?WriteProperty@asxAbstractAdapter@@UAE?AW4asxERROR@@HGG@Z 10015980 f   asxclass.obj
 0001:000149f0       ?WrongObject@asxBase@@QAEHHH@Z 100159f0 f   asxclass.obj
 0001:00014a20       ?WrongType@asxBase@@QAEHH@Z 10015a20 f   asxclass.obj
 0001:00014a50       ?asxCreateSubSystem@@YA?AW4asxERROR@@PAVasxSystem@@HPAPAVasxSubSystem@@@Z 10015a50 f   asxclass.obj
 0001:00014c20       ?asxSupportsSubSystem@@YAHH@Z 10015c20 f   asxclass.obj
 0001:00014c60       ?asxSystemCallbackThreadProc@@YGKPAX@Z 10015c60 f   asxclass.obj
 0001:00014c80       ?asxSystemGetAvdeccInterface@@YAPADXZ 10015c80 f   asxclass.obj
 0001:00014c90       ?asxSystemGetCobranetAutoassignParms@@YA?AW4asxERROR@@PAUasxCobranetIpAutoassignParameters@@@Z 10015c90 f   asxclass.obj
 0001:00014df0       ?asxSystemGetNetworkInterface@@YAPADXZ 10015df0 f   asxclass.obj
 0001:00014e80       ?asxSystemSetAvdeccInterface@@YA?AW4asxERROR@@PBD@Z 10015e80 f   asxclass.obj
 0001:00014ec0       ?asxSystemSetCobranetAutoassignParms@@YA?AW4asxERROR@@PBUasxCobranetIpAutoassignParameters@@@Z 10015ec0 f   asxclass.obj
 0001:00014f90       ?asxSystemSetHostNetworkInterface@@YA?AW4asxERROR@@PBD@Z 10015f90 f   asxclass.obj
 0001:00014ff0       ?asx_to_cobra_format@asxCobranetTx@@IAEIW4asxAUDIO_FORMAT@@I@Z 10015ff0 f   asxclass.obj
 0001:00015090       ?clear@TASICString@@QAEXXZ 10016090 f i asxclass.obj
 0001:000150b0       ?cobra_to_asx_format@asxCobranetTx@@IAE?AW4asxAUDIO_FORMAT@@I@Z 100160b0 f   asxclass.obj
 0001:00015100       ?compute_latency_and_rate@asxCobranet@@IAEXIPAW4asxCOBRANET_LATENCY@@PAW4asxSAMPLE_RATE@@@Z 10016100 f   asxclass.obj
 0001:00015180       ?compute_mode_and_mask@asxCobranet@@IAE?AW4asxERROR@@W4asxCOBRANET_LATENCY@@W4asxSAMPLE_RATE@@PAHPAI@Z 10016180 f   asxclass.obj
 0001:00015200       ?set@TASICString@@QAEXPBD@Z 10016200 f i asxclass.obj
 0001:00015260       ??0asxDebugClass@@QAE@XZ   10016260 f   asxdebug.obj
 0001:000152a0       ?Get@asxDebugClass@@QAEIXZ 100162a0 f   asxdebug.obj
 0001:000152b0       ?Log@asxDebugClass@@QAAXPBDI0ZZ 100162b0 f   asxdebug.obj
 0001:00015340       ?Set@asxDebugClass@@QAEXI@Z 10016340 f   asxdebug.obj
 0001:00015350       ??0asxAdapterDSND@@QAE@PAVasxSystem@@HPBD@Z 10016350 f   asxdsnd.obj
 0001:00015380       ??0asxMixerScannerDSND@@QAE@PAVasxSubSystem@@PAVdsndAdapterListEntry@@@Z 10016380 f   asxdsnd.obj
 0001:000153a0       ??0asxSubSystemDSND@@QAE@PAVasxSystem@@@Z 100163a0 f   asxdsnd.obj
 0001:000153f0       ??0dsndAdapterList@@QAE@XZ 100163f0 f   asxdsnd.obj
 0001:00015400       ??0dsndAdapterListEntry@@QAE@PBU_GUID@@PBD1_N@Z 10016400 f   asxdsnd.obj
 0001:00015490       ??1asxAdapterDSND@@UAE@XZ  10016490 f   asxdsnd.obj
 0001:000154a0       ??1asxMixerScannerDSND@@UAE@XZ 100164a0 f   asxdsnd.obj
 0001:00015510       ??1asxSubSystemDSND@@UAE@XZ 10016510 f   asxdsnd.obj
 0001:00015520       ??1dsndAdapterList@@QAE@XZ 10016520 f   asxdsnd.obj
 0001:00015540       ??1dsndAdapterListEntry@@QAE@XZ 10016540 f   asxdsnd.obj
 0001:000155a0       ??_EasxAdapterDSND@@UAEPAXI@Z 100165a0 f i asxdsnd.obj
 0001:000155a0       ??_GasxAdapterDSND@@UAEPAXI@Z 100165a0 f i asxdsnd.obj
 0001:000155d0       ??_GasxMixerScannerDSND@@UAEPAXI@Z 100165d0 f i asxdsnd.obj
 0001:000155d0       ??_EasxMixerScannerDSND@@UAEPAXI@Z 100165d0 f i asxdsnd.obj
 0001:00015600       ??_EasxSubSystemDSND@@UAEPAXI@Z 10016600 f i asxdsnd.obj
 0001:00015600       ??_GasxSubSystemDSND@@UAEPAXI@Z 10016600 f i asxdsnd.obj
 0001:00015630       ??_GdsndAdapterListEntry@@QAEPAXI@Z 10016630 f i asxdsnd.obj
 0001:00015660       ?AddEntry@dsndAdapterList@@QAEXPBU_GUID@@PBD1@Z 10016660 f   asxdsnd.obj
 0001:000156e0       ?Append@dsndAdapterListEntry@@QAEXAAV1@@Z 100166e0 f   asxdsnd.obj
 0001:00015720       ?CheckSubSystems@asxAdapterDSND@@UAE?AW4asxERROR@@PAI0@Z 10016720 f i asxdsnd.obj
 0001:00015740       ?DSoundEnumCallback@@YGHPAU_GUID@@PAD1PAX@Z 10016740 f   asxdsnd.obj
 0001:00015770       ?GetDescription@dsndAdapterListEntry@@QAEPBDXZ 10016770 f i asxdsnd.obj
 0001:00015780       ?GetGuid@dsndAdapterListEntry@@QAEPBU_GUID@@XZ 10016780 f i asxdsnd.obj
 0001:00015790       ?GetIndex@dsndAdapterListEntry@@QAEHXZ 10016790 f i asxdsnd.obj
 0001:000157a0       ?GetNext@dsndAdapterListEntry@@QAEPAV1@XZ 100167a0 f i asxdsnd.obj
 0001:000157b0       ?IsCapture@dsndAdapterListEntry@@QAE_NXZ 100167b0 f i asxdsnd.obj
 0001:000157c0       ?Matches@dsndAdapterListEntry@@QAE_NAAV1@@Z 100167c0 f   asxdsnd.obj
 0001:00015840       ?Pop@dsndAdapterList@@QAEPAVdsndAdapterListEntry@@XZ 10016840 f i asxdsnd.obj
 0001:00015860       ?Pop@dsndAdapterListEntry@@QAEXXZ 10016860 f i asxdsnd.obj
 0001:00015870       ?ReScan@asxSubSystemDSND@@UAEXXZ 10016870 f   asxdsnd.obj
 0001:00015880       ?Scan@asxMixerScannerDSND@@EAEXPAVasxMixer@@@Z 10016880 f   asxdsnd.obj
 0001:000159f0       ?Scan@asxSubSystemDSND@@UAEXXZ 100169f0 f   asxdsnd.obj
 0001:00015af0       ?SetCaptureFlag@dsndAdapterList@@QAEX_N@Z 10016af0 f i asxdsnd.obj
 0001:00015b00       ?SetNext@dsndAdapterListEntry@@QAEXPAV1@@Z 10016b00 f i asxdsnd.obj
 0001:00015b10       ?translateSpecificErrorCode@asxSubSystemDSND@@QAEXIPAPAD@Z 10016b10 f   asxdsnd.obj
 0001:00015b20       ??0asxPlayerDSND@@QAE@PAVasxSubSystem@@PAVasxNode@@1PBU_GUID@@@Z 10016b20 f   asxdsndplay.obj
 0001:00015bf0       ??1asxPlayerDSND@@UAE@XZ   10016bf0 f   asxdsndplay.obj
 0001:00015c50       ??_EasxPlayerDSND@@UAEPAXI@Z 10016c50 f i asxdsndplay.obj
 0001:00015c50       ??_GasxPlayerDSND@@UAEPAXI@Z 10016c50 f i asxdsndplay.obj
 0001:00015c80       ?AllocOutput@asxPlayerDSND@@MAE?AW4asxERROR@@XZ 10016c80 f i asxdsndplay.obj
 0001:00015d50       ?Current@asxPlayerFileList@@QAEPAVTWavFileBase@@XZ 10016d50 f i asxdsndplay.obj
 0001:00015d70       ?EnumChildProc@@YGHPAUHWND__@@J@Z 10016d70 f   asxdsndplay.obj
 0001:00015db0       ?FreeOutput@asxPlayerDSND@@MAE?AW4asxERROR@@XZ 10016db0 f i asxdsndplay.obj
 0001:00015de0       ?GetProcWindow@@YAPAUHWND__@@XZ 10016de0 f   asxdsndplay.obj
 0001:00015e20       ?HelperThread@asxPlayerDSND@@UAEXXZ 10016e20 f   asxdsndplay.obj
 0001:000160d0       ?OnFileOpen@asxPlayer@@MAE?AW4asxERROR@@XZ 100170d0 f i asxdsndplay.obj
 0001:000160e0       ?ResetOutput@asxPlayerDSND@@MAE?AW4asxERROR@@XZ 100170e0 f i asxdsndplay.obj
 0001:000160f0       ?SetTimeScale@asxPlayerDSND@@UAE?AW4asxERROR@@M@Z 100170f0 f i asxdsndplay.obj
 0001:00016100       ?StartOutput@asxPlayerDSND@@MAE?AW4asxERROR@@XZ 10017100 f i asxdsndplay.obj
 0001:00016120       ?StopOutput@asxPlayerDSND@@MAE?AW4asxERROR@@XZ 10017120 f i asxdsndplay.obj
 0001:00016140       ??0asxRecorderDSND@@QAE@PAVasxSubSystem@@PAVasxNode@@1PBU_GUID@@@Z 10017140 f   asxdsndrec.obj
 0001:000161d0       ??1asxRecorderDSND@@UAE@XZ 100171d0 f   asxdsndrec.obj
 0001:00016230       ??_EasxRecorderDSND@@UAEPAXI@Z 10017230 f i asxdsndrec.obj
 0001:00016230       ??_GasxRecorderDSND@@UAEPAXI@Z 10017230 f i asxdsndrec.obj
 0001:00016260       ?Add@?$TASIArray@W4asxAUDIO_FORMAT@@@@QAEHPAW4asxAUDIO_FORMAT@@@Z 10017260 f i asxdsndrec.obj
 0001:00016290       ?AllocInput@asxRecorderDSND@@EAE?AW4asxERROR@@XZ 10017290 f i asxdsndrec.obj
 0001:00016350       ?Enlarge@?$TASIArray@W4asxAUDIO_FORMAT@@@@AAEXXZ 10017350 f i asxdsndrec.obj
 0001:000163b0       ?EnumerateAllFormats@asxRecorderDSND@@EAEXXZ 100173b0 f   asxdsndrec.obj
 0001:000163f0       ?FreeInput@asxRecorderDSND@@EAE?AW4asxERROR@@XZ 100173f0 f i asxdsndrec.obj
 0001:00016420       ?GetInputPosition@asxRecorderDSND@@EAE?AW4asxERROR@@PAK@Z 10017420 f   asxdsndrec.obj
 0001:00016440       ?HelperThread@asxRecorderDSND@@UAEKXZ 10017440 f   asxdsndrec.obj
 0001:00016590       ?SetInputFormat@asxRecorderDSND@@EAE?AW4asxERROR@@XZ 10017590 f i asxdsndrec.obj
 0001:000165a0       ?StartInput@asxRecorderDSND@@EAE?AW4asxERROR@@XZ 100175a0 f i asxdsndrec.obj
 0001:000165e0       ?StopInput@asxRecorderDSND@@EAE?AW4asxERROR@@XZ 100175e0 f i asxdsndrec.obj
 0001:00016600       ??0?$TASIArray@G@@QAE@XZ   10017600 f i asxhpi.obj
 0001:00016620       ??0?$TASIArray@H@@QAE@XZ   10017620 f i asxhpi.obj
 0001:00016640       ??0?$TASIArray@I@@QAE@XZ   10017640 f i asxhpi.obj
 0001:00016660       ??0?$TASIArray@VasxBlockProperty@@@@QAE@XZ 10017660 f i asxhpi.obj
 0001:00016680       ??0?$TASIArray@W4asxAESEBU_FORMAT@@@@QAE@XZ 10017680 f i asxhpi.obj
 0001:000166a0       ??0?$TASIArray@W4asxCHANNELMODE@@@@QAE@XZ 100176a0 f i asxhpi.obj
 0001:000166c0       ??0?$TASIArray@W4asxNODE@@@@QAE@XZ 100176c0 f i asxhpi.obj
 0001:000166e0       ??0?$TASIArray@W4asxSAMPLE_CLOCK_SOURCE@@@@QAE@XZ 100176e0 f i asxhpi.obj
 0001:00016700       ??0?$TASIArray@W4asxSAMPLE_RATE@@@@QAE@XZ 10017700 f i asxhpi.obj
 0001:00016720       ??0?$TASIArray@W4asxTUNERBAND@@@@QAE@XZ 10017720 f i asxhpi.obj
 0001:00016740       ??0?$TASIArray@W4asxTUNERPROGRAM@@@@QAE@XZ 10017740 f i asxhpi.obj
 0001:00016760       ??0asxAdapterHPI@@QAE@PAVasxSystem@@HPBD@Z 10017760 f   asxhpi.obj
 0001:000169e0       ??0asxAdapterHPIDuplicateIndex@@QAE@PAVasxSystem@@HHGPBD@Z 100179e0 f   asxhpi.obj
 0001:00016a60       ??0asxAes3Rx@@QAE@PAVasxSubSystem@@PAVasxNode@@1@Z 10017a60 f i asxhpi.obj
 0001:00016aa0       ??0asxAes3Tx@@QAE@PAVasxSubSystem@@PAVasxNode@@1@Z 10017aa0 f i asxhpi.obj
 0001:00016ae0       ??0asxAes3TxHPI@@QAE@PAVasxSubSystem@@PAVasxNode@@1I@Z 10017ae0 f   asxhpi.obj
 0001:00016c10       ??0asxAesebuReceiverHPI@@QAE@PAVasxSubSystem@@PAVasxNode@@1I@Z 10017c10 f   asxhpi.obj
 0001:00016d40       ??0asxBitStream@@QAE@PAVasxSubSystem@@PAVasxNode@@1@Z 10017d40 f i asxhpi.obj
 0001:00016d70       ??0asxBlock@@QAE@PAVasxSubSystem@@PAVasxNode@@1@Z 10017d70 f i asxhpi.obj
 0001:00016db0       ??0asxBlockHPI@@QAE@PAVasxSubSystem@@PAVasxNode@@1I@Z 10017db0 f   asxhpi.obj
 0001:00016f30       ??0asxBlockPropertyHPI@@QAE@W4asxUCONTROL_PTYPE@@W4asxUCONTROL_PFLAGS@@IPBDPAUasxParameterRangeInfo@@2I@Z 10017f30 f i asxhpi.obj
 0001:00016f60       ??0asxCobranet@@QAE@AAV0@@Z 10017f60 f i asxhpi.obj
 0001:00016f90       ??0asxCobranet@@QAE@PAVasxSubSystem@@PAVasxNode@@1H@Z 10017f90 f i asxhpi.obj
 0001:00016fc0       ??0asxCobranetContainer@@QAE@AAVasxCobranet@@@Z 10017fc0 f i asxhpi.obj
 0001:00016ff0       ??0asxCobranetHPI@@QAE@PAVasxSubSystem@@PAVasxNode@@1IH@Z 10017ff0 f   asxhpi.obj
 0001:00017080       ??0asxCobranetRx@@QAE@AAV0@@Z 10018080 f i asxhpi.obj
 0001:000170b0       ??0asxCobranetRx@@QAE@PAVasxSubSystem@@PAVasxNode@@1H@Z 100180b0 f i asxhpi.obj
 0001:000170e0       ??0asxCobranetRxContainer@@QAE@AAVasxCobranetRx@@@Z 100180e0 f i asxhpi.obj
 0001:00017110       ??0asxCobranetRxHPI@@QAE@PAVasxSubSystem@@PAVasxNode@@1IH@Z 10018110 f   asxhpi.obj
 0001:000171a0       ??0asxCobranetTx@@QAE@AAV0@@Z 100181a0 f i asxhpi.obj
 0001:000171d0       ??0asxCobranetTx@@QAE@PAVasxSubSystem@@PAVasxNode@@1H@Z 100181d0 f i asxhpi.obj
 0001:00017200       ??0asxCobranetTxContainer@@QAE@AAVasxCobranetTx@@@Z 10018200 f i asxhpi.obj
 0001:00017230       ??0asxCobranetTxHPI@@QAE@PAVasxSubSystem@@PAVasxNode@@1IH@Z 10018230 f   asxhpi.obj
 0001:000172c0       ??0asxCompander@@QAE@PAVasxSubSystem@@PAVasxNode@@1@Z 100182c0 f i asxhpi.obj
 0001:000172f0       ??0asxCompanderHPI@@QAE@PAVasxSubSystem@@PAVasxNode@@1I@Z 100182f0 f   asxhpi.obj
 0001:00017320       ??0asxCompanderHPI_Legacy@@QAE@PAVasxSubSystem@@PAVasxNode@@1I@Z 10018320 f   asxhpi.obj
 0001:00017390       ??0asxControlBaseHPI@@QAE@I@Z 10018390 f i asxhpi.obj
 0001:000173a0       ??0asxControlHPI@@QAE@PAVasxSubSystem@@W4asxCONTROL@@PAVasxNode@@2I@Z 100183a0 f i asxhpi.obj
 0001:000173d0       ??0asxGenericControl@@QAE@PAVasxSubSystem@@PAVasxNode@@1PBD@Z 100183d0 f i asxhpi.obj
 0001:00017400       ??0asxGenericHPI@@QAE@PAVasxSubSystem@@PAVasxNode@@1IPBD@Z 10018400 f i asxhpi.obj
 0001:00017440       ??0asxGpio@@QAE@PAVasxSubSystem@@PAVasxNode@@1@Z 10018440 f i asxhpi.obj
 0001:00017470       ??0asxGpioHPI@@QAE@PAVasxSubSystem@@PAVasxNode@@1IHH@Z 10018470 f   asxhpi.obj
 0001:00017540       ??0asxLevel@@QAE@PAVasxSubSystem@@PAVasxNode@@1@Z 10018540 f i asxhpi.obj
 0001:00017570       ??0asxLevelHPI@@QAE@PAVasxSubSystem@@PAVasxNode@@1I@Z 10018570 f i asxhpi.obj
 0001:000175a0       ??0asxMeter@@QAE@PAVasxSubSystem@@PAVasxNode@@1@Z 100185a0 f i asxhpi.obj
 0001:000175d0       ??0asxMeterHPI@@QAE@PAVasxSubSystem@@PAVasxNode@@1I@Z 100185d0 f i asxhpi.obj
 0001:00017600       ??0asxMic@@QAE@PAVasxSubSystem@@PAVasxNode@@1@Z 10018600 f i asxhpi.obj
 0001:00017630       ??0asxMicHPI@@QAE@PAVasxSubSystem@@PAVasxNode@@1I@Z 10018630 f   asxhpi.obj
 0001:00017660       ??0asxMixerScannerHPI@@QAE@PAVasxSubSystem@@I@Z 10018660 f i asxhpi.obj
 0001:00017690       ??0asxMixerScannerHPIDuplicateIndex@@QAE@PAVasxSubSystem@@@Z 10018690 f i asxhpi.obj
 0001:000176b0       ??0asxMode@@QAE@PAVasxSubSystem@@PAVasxNode@@1@Z 100186b0 f i asxhpi.obj
 0001:000176f0       ??0asxModeHPI@@QAE@PAVasxSubSystem@@PAVasxNode@@1I@Z 100186f0 f   asxhpi.obj
 0001:000179a0       ??0asxMux@@QAE@PAVasxSubSystem@@PAVasxNode@@1@Z 100189a0 f i asxhpi.obj
 0001:000179f0       ??0asxMuxHPI@@QAE@PAVasxSubSystem@@PAVasxNode@@1I@Z 100189f0 f   asxhpi.obj
 0001:00017bd0       ??0asxPad@@QAE@PAVasxSubSystem@@PAVasxNode@@1@Z 10018bd0 f i asxhpi.obj
 0001:00017c00       ??0asxPadHPI@@QAE@PAVasxSubSystem@@PAVasxNode@@1I@Z 10018c00 f   asxhpi.obj
 0001:00017c30       ??0asxParametricEQ@@QAE@PAVasxSubSystem@@PAVasxNode@@1@Z 10018c30 f i asxhpi.obj
 0001:00017c60       ??0asxParametricEqHPI@@QAE@PAVasxSubSystem@@PAVasxNode@@1I@Z 10018c60 f   asxhpi.obj
 0001:00017c90       ??0asxSampleClock@@QAE@PAVasxSubSystem@@PAVasxNode@@1@Z 10018c90 f i asxhpi.obj
 0001:00017ce0       ??0asxSampleClockHPI@@QAE@PAVasxSubSystem@@PAVasxNode@@1I@Z 10018ce0 f   asxhpi.obj
 0001:00017f70       ??0asxSilenceDetector@@QAE@PAVasxSubSystem@@PAVasxNode@@1@Z 10018f70 f i asxhpi.obj
 0001:00017fa0       ??0asxSilenceDetectorHPI@@QAE@PAVasxSubSystem@@PAVasxNode@@1I@Z 10018fa0 f   asxhpi.obj
 0001:00017fd0       ??0asxSubSystemHPI@@QAE@PAVasxSystem@@H@Z 10018fd0 f   asxhpi.obj
 0001:00018070       ??0asxToneDetector@@QAE@PAVasxSubSystem@@PAVasxNode@@1@Z 10019070 f i asxhpi.obj
 0001:000180a0       ??0asxToneDetectorHPI@@QAE@PAVasxSubSystem@@PAVasxNode@@1I@Z 100190a0 f   asxhpi.obj
 0001:000180d0       ??0asxTuner@@QAE@PAVasxSubSystem@@PAVasxNode@@1@Z 100190d0 f i asxhpi.obj
 0001:00018120       ??0asxTunerHPI@@QAE@PAVasxSubSystem@@PAVasxNode@@1I@Z 10019120 f   asxhpi.obj
 0001:00018200       ??0asxVolume@@QAE@PAVasxSubSystem@@PAVasxNode@@1@Z 10019200 f i asxhpi.obj
 0001:00018230       ??0asxVolumeHPI@@QAE@PAVasxSubSystem@@PAVasxNode@@1I@Z 10019230 f i asxhpi.obj
 0001:00018270       ??0asxVox@@QAE@PAVasxSubSystem@@PAVasxNode@@1@Z 10019270 f i asxhpi.obj
 0001:000182a0       ??0asxVoxHPI@@QAE@PAVasxSubSystem@@PAVasxNode@@1I@Z 100192a0 f   asxhpi.obj
 0001:000182d0       ??0hpiHMI@@QAE@I@Z         100192d0 f   asxhpi.obj
 0001:000182f0       ??1?$TASIArray@G@@QAE@XZ   100192f0 f i asxhpi.obj
 0001:00018340       ??1?$TASIArray@H@@QAE@XZ   10019340 f i asxhpi.obj
 0001:00018390       ??1?$TASIArray@I@@QAE@XZ   10019390 f i asxhpi.obj
 0001:000183e0       ??1?$TASIArray@VasxBlockProperty@@@@QAE@XZ 100193e0 f i asxhpi.obj
 0001:00018430       ??1?$TASIArray@W4asxAESEBU_FORMAT@@@@QAE@XZ 10019430 f i asxhpi.obj
 0001:00018480       ??1?$TASIArray@W4asxCHANNELMODE@@@@QAE@XZ 10019480 f i asxhpi.obj
 0001:000184d0       ??1?$TASIArray@W4asxNODE@@@@QAE@XZ 100194d0 f i asxhpi.obj
 0001:00018520       ??1?$TASIArray@W4asxSAMPLE_CLOCK_SOURCE@@@@QAE@XZ 10019520 f i asxhpi.obj
 0001:00018570       ??1?$TASIArray@W4asxSAMPLE_RATE@@@@QAE@XZ 10019570 f i asxhpi.obj
 0001:000185c0       ??1?$TASIArray@W4asxTUNERBAND@@@@QAE@XZ 100195c0 f i asxhpi.obj
 0001:00018610       ??1?$TASIArray@W4asxTUNERPROGRAM@@@@QAE@XZ 10019610 f i asxhpi.obj
 0001:00018660       ??1asxAdapterHPI@@UAE@XZ   10019660 f   asxhpi.obj
 0001:000186d0       ??1asxAdapterHPIDuplicateIndex@@UAE@XZ 100196d0 f i asxhpi.obj
 0001:000186e0       ??1asxAes3Rx@@UAE@XZ       100196e0 f i asxhpi.obj
 0001:00018750       ??1asxAes3Tx@@UAE@XZ       10019750 f i asxhpi.obj
 0001:000187c0       ??1asxAes3TxHPI@@UAE@XZ    100197c0 f   asxhpi.obj
 0001:00018830       ??1asxAesebuReceiverHPI@@UAE@XZ 10019830 f   asxhpi.obj
 0001:000188a0       ??1asxBitStream@@UAE@XZ    100198a0 f i asxhpi.obj
 0001:000188c0       ??1asxBlock@@UAE@XZ        100198c0 f i asxhpi.obj
 0001:00018930       ??1asxBlockHPI@@UAE@XZ     10019930 f   asxhpi.obj
 0001:000189a0       ??1asxBlockPropertyHPI@@UAE@XZ 100199a0 f i asxhpi.obj
 0001:000189b0       ??1asxCobranet@@UAE@XZ     100199b0 f i asxhpi.obj
 0001:000189d0       ??1asxCobranetContainer@@UAE@XZ 100199d0 f i asxhpi.obj
 0001:00018a40       ??1asxCobranetHPI@@UAE@XZ  10019a40 f   asxhpi.obj
 0001:00018a70       ??1asxCobranetRx@@UAE@XZ   10019a70 f i asxhpi.obj
 0001:00018a90       ??1asxCobranetRxContainer@@UAE@XZ 10019a90 f i asxhpi.obj
 0001:00018b00       ??1asxCobranetRxHPI@@UAE@XZ 10019b00 f   asxhpi.obj
 0001:00018b30       ??1asxCobranetTx@@UAE@XZ   10019b30 f i asxhpi.obj
 0001:00018b50       ??1asxCobranetTxContainer@@UAE@XZ 10019b50 f i asxhpi.obj
 0001:00018bc0       ??1asxCobranetTxHPI@@UAE@XZ 10019bc0 f   asxhpi.obj
 0001:00018bf0       ??1asxCompander@@UAE@XZ    10019bf0 f i asxhpi.obj
 0001:00018c10       ??1asxCompanderHPI@@UAE@XZ 10019c10 f   asxhpi.obj
 0001:00018c30       ??1asxCompanderHPI_Legacy@@UAE@XZ 10019c30 f   asxhpi.obj
 0001:00018c50       ??1asxControlBaseHPI@@QAE@XZ 10019c50 f i asxhpi.obj
 0001:00018c60       ??1asxControlHPI@@UAE@XZ   10019c60 f i asxhpi.obj
 0001:00018c80       ??1asxGenericControl@@UAE@XZ 10019c80 f i asxhpi.obj
 0001:00018ca0       ??1asxGenericHPI@@UAE@XZ   10019ca0 f i asxhpi.obj
 0001:00018cc0       ??1asxGpio@@UAE@XZ         10019cc0 f i asxhpi.obj
 0001:00018ce0       ??1asxGpioHPI@@UAE@XZ      10019ce0 f   asxhpi.obj
 0001:00018d50       ??1asxLevel@@UAE@XZ        10019d50 f i asxhpi.obj
 0001:00018d70       ??1asxLevelHPI@@UAE@XZ     10019d70 f i asxhpi.obj
 0001:00018d90       ??1asxMeter@@UAE@XZ        10019d90 f i asxhpi.obj
 0001:00018db0       ??1asxMeterHPI@@UAE@XZ     10019db0 f i asxhpi.obj
 0001:00018dd0       ??1asxMic@@UAE@XZ          10019dd0 f i asxhpi.obj
 0001:00018df0       ??1asxMicHPI@@UAE@XZ       10019df0 f   asxhpi.obj
 0001:00018e10       ??1asxMixerScannerHPI@@UAE@XZ 10019e10 f   asxhpi.obj
 0001:00018e40       ??1asxMixerScannerHPIDuplicateIndex@@UAE@XZ 10019e40 f i asxhpi.obj
 0001:00018e50       ??1asxMode@@UAE@XZ         10019e50 f i asxhpi.obj
 0001:00018ec0       ??1asxModeHPI@@UAE@XZ      10019ec0 f   asxhpi.obj
 0001:00018f40       ??1asxMux@@UAE@XZ          10019f40 f i asxhpi.obj
 0001:00018fb0       ??1asxMuxHPI@@UAE@XZ       10019fb0 f   asxhpi.obj
 0001:00019040       ??1asxPad@@UAE@XZ          1001a040 f i asxhpi.obj
 0001:00019060       ??1asxPadHPI@@UAE@XZ       1001a060 f   asxhpi.obj
 0001:00019080       ??1asxParametricEQ@@UAE@XZ 1001a080 f i asxhpi.obj
 0001:000190a0       ??1asxParametricEqHPI@@UAE@XZ 1001a0a0 f   asxhpi.obj
 0001:000190c0       ??1asxSampleClock@@UAE@XZ  1001a0c0 f i asxhpi.obj
 0001:00019130       ??1asxSampleClockHPI@@UAE@XZ 1001a130 f   asxhpi.obj
 0001:000191d0       ??1asxSilenceDetector@@UAE@XZ 1001a1d0 f i asxhpi.obj
 0001:000191f0       ??1asxSilenceDetectorHPI@@UAE@XZ 1001a1f0 f   asxhpi.obj
 0001:00019210       ??1asxSubSystemHPI@@UAE@XZ 1001a210 f   asxhpi.obj
 0001:00019230       ??1asxToneDetector@@UAE@XZ 1001a230 f i asxhpi.obj
 0001:00019250       ??1asxToneDetectorHPI@@UAE@XZ 1001a250 f   asxhpi.obj
 0001:00019270       ??1asxTuner@@UAE@XZ        1001a270 f i asxhpi.obj
 0001:000192e0       ??1asxTunerHPI@@UAE@XZ     1001a2e0 f   asxhpi.obj
 0001:00019350       ??1asxVolume@@UAE@XZ       1001a350 f i asxhpi.obj
 0001:00019370       ??1asxVolumeHPI@@UAE@XZ    1001a370 f i asxhpi.obj
 0001:00019390       ??1asxVox@@UAE@XZ          1001a390 f i asxhpi.obj
 0001:000193b0       ??1asxVoxHPI@@UAE@XZ       1001a3b0 f   asxhpi.obj
 0001:000193d0       ??1hpiHMI@@QAE@XZ          1001a3d0 f   asxhpi.obj
 0001:000193e0       ??4asxBase@@QAEAAV0@ABV0@@Z 1001a3e0 f i asxhpi.obj
 0001:00019410       ??4asxControlBase@@QAEAAV0@ABV0@@Z 1001a410 f i asxhpi.obj
 0001:00019460       ??8asxNode@@QAE_NAAV0@@Z   1001a460 f i asxhpi.obj
 0001:000194a0       ??A?$TASIArray@G@@QBEPAGH@Z 1001a4a0 f i asxhpi.obj
 0001:000194c0       ??A?$TASIArray@I@@QBEPAIH@Z 1001a4c0 f i asxhpi.obj
 0001:000194e0       ??_GasxAdapterHPI@@UAEPAXI@Z 1001a4e0 f i asxhpi.obj
 0001:000194e0       ??_EasxAdapterHPI@@UAEPAXI@Z 1001a4e0 f i asxhpi.obj
 0001:00019510       ??_EasxAdapterHPIDuplicateIndex@@UAEPAXI@Z 1001a510 f i asxhpi.obj
 0001:00019510       ??_GasxAdapterHPIDuplicateIndex@@UAEPAXI@Z 1001a510 f i asxhpi.obj
 0001:00019540       ??_GasxAes3Rx@@UAEPAXI@Z   1001a540 f i asxhpi.obj
 0001:00019540       ??_EasxAes3Rx@@UAEPAXI@Z   1001a540 f i asxhpi.obj
 0001:000195c0       ??_GasxAes3Tx@@UAEPAXI@Z   1001a5c0 f i asxhpi.obj
 0001:000195c0       ??_EasxAes3Tx@@UAEPAXI@Z   1001a5c0 f i asxhpi.obj
 0001:00019640       ??_EasxAes3TxHPI@@UAEPAXI@Z 1001a640 f i asxhpi.obj
 0001:00019640       ??_GasxAes3TxHPI@@UAEPAXI@Z 1001a640 f i asxhpi.obj
 0001:00019670       ??_GasxAesebuReceiverHPI@@UAEPAXI@Z 1001a670 f i asxhpi.obj
 0001:00019670       ??_EasxAesebuReceiverHPI@@UAEPAXI@Z 1001a670 f i asxhpi.obj
 0001:000196a0       ??_GasxBitStream@@UAEPAXI@Z 1001a6a0 f i asxhpi.obj
 0001:000196a0       ??_EasxBitStream@@UAEPAXI@Z 1001a6a0 f i asxhpi.obj
 0001:000196e0       ??_GasxBlock@@UAEPAXI@Z    1001a6e0 f i asxhpi.obj
 0001:000196e0       ??_EasxBlock@@UAEPAXI@Z    1001a6e0 f i asxhpi.obj
 0001:00019760       ??_GasxBlockHPI@@UAEPAXI@Z 1001a760 f i asxhpi.obj
 0001:00019760       ??_EasxBlockHPI@@UAEPAXI@Z 1001a760 f i asxhpi.obj
 0001:00019790       ??_EasxBlockPropertyHPI@@UAEPAXI@Z 1001a790 f i asxhpi.obj
 0001:00019790       ??_GasxBlockPropertyHPI@@UAEPAXI@Z 1001a790 f i asxhpi.obj
 0001:000197c0       ??_GasxCobranet@@UAEPAXI@Z 1001a7c0 f i asxhpi.obj
 0001:000197c0       ??_EasxCobranet@@UAEPAXI@Z 1001a7c0 f i asxhpi.obj
 0001:00019800       ??_EasxCobranetContainer@@UAEPAXI@Z 1001a800 f i asxhpi.obj
 0001:00019800       ??_GasxCobranetContainer@@UAEPAXI@Z 1001a800 f i asxhpi.obj
 0001:00019880       ??_EasxCobranetHPI@@UAEPAXI@Z 1001a880 f i asxhpi.obj
 0001:00019880       ??_GasxCobranetHPI@@UAEPAXI@Z 1001a880 f i asxhpi.obj
 0001:000198b0       ??_EasxCobranetRx@@UAEPAXI@Z 1001a8b0 f i asxhpi.obj
 0001:000198b0       ??_GasxCobranetRx@@UAEPAXI@Z 1001a8b0 f i asxhpi.obj
 0001:000198f0       ??_EasxCobranetRxContainer@@UAEPAXI@Z 1001a8f0 f i asxhpi.obj
 0001:000198f0       ??_GasxCobranetRxContainer@@UAEPAXI@Z 1001a8f0 f i asxhpi.obj
 0001:00019970       ??_EasxCobranetRxHPI@@UAEPAXI@Z 1001a970 f i asxhpi.obj
 0001:00019970       ??_GasxCobranetRxHPI@@UAEPAXI@Z 1001a970 f i asxhpi.obj
 0001:000199a0       ??_EasxCobranetTx@@UAEPAXI@Z 1001a9a0 f i asxhpi.obj
 0001:000199a0       ??_GasxCobranetTx@@UAEPAXI@Z 1001a9a0 f i asxhpi.obj
 0001:000199e0       ??_EasxCobranetTxContainer@@UAEPAXI@Z 1001a9e0 f i asxhpi.obj
 0001:000199e0       ??_GasxCobranetTxContainer@@UAEPAXI@Z 1001a9e0 f i asxhpi.obj
 0001:00019a60       ??_GasxCobranetTxHPI@@UAEPAXI@Z 1001aa60 f i asxhpi.obj
 0001:00019a60       ??_EasxCobranetTxHPI@@UAEPAXI@Z 1001aa60 f i asxhpi.obj
 0001:00019a90       ??_GasxCompander@@UAEPAXI@Z 1001aa90 f i asxhpi.obj
 0001:00019a90       ??_EasxCompander@@UAEPAXI@Z 1001aa90 f i asxhpi.obj
 0001:00019ad0       ??_EasxCompanderHPI@@UAEPAXI@Z 1001aad0 f i asxhpi.obj
 0001:00019ad0       ??_GasxCompanderHPI@@UAEPAXI@Z 1001aad0 f i asxhpi.obj
 0001:00019b00       ??_EasxCompanderHPI_Legacy@@UAEPAXI@Z 1001ab00 f i asxhpi.obj
 0001:00019b00       ??_GasxCompanderHPI_Legacy@@UAEPAXI@Z 1001ab00 f i asxhpi.obj
 0001:00019b30       ??_EasxControlHPI@@UAEPAXI@Z 1001ab30 f i asxhpi.obj
 0001:00019b30       ??_GasxControlHPI@@UAEPAXI@Z 1001ab30 f i asxhpi.obj
 0001:00019b70       ??_GasxGenericControl@@UAEPAXI@Z 1001ab70 f i asxhpi.obj
 0001:00019b70       ??_EasxGenericControl@@UAEPAXI@Z 1001ab70 f i asxhpi.obj
 0001:00019bb0       ??_EasxGenericHPI@@UAEPAXI@Z 1001abb0 f i asxhpi.obj
 0001:00019bb0       ??_GasxGenericHPI@@UAEPAXI@Z 1001abb0 f i asxhpi.obj
 0001:00019bf0       ??_EasxGpio@@UAEPAXI@Z     1001abf0 f i asxhpi.obj
 0001:00019bf0       ??_GasxGpio@@UAEPAXI@Z     1001abf0 f i asxhpi.obj
 0001:00019c30       ??_EasxGpioHPI@@UAEPAXI@Z  1001ac30 f i asxhpi.obj
 0001:00019c30       ??_GasxGpioHPI@@UAEPAXI@Z  1001ac30 f i asxhpi.obj
 0001:00019c60       ??_GasxLevel@@UAEPAXI@Z    1001ac60 f i asxhpi.obj
 0001:00019c60       ??_EasxLevel@@UAEPAXI@Z    1001ac60 f i asxhpi.obj
 0001:00019ca0       ??_GasxLevelHPI@@UAEPAXI@Z 1001aca0 f i asxhpi.obj
 0001:00019ca0       ??_EasxLevelHPI@@UAEPAXI@Z 1001aca0 f i asxhpi.obj
 0001:00019ce0       ??_GasxMeter@@UAEPAXI@Z    1001ace0 f i asxhpi.obj
 0001:00019ce0       ??_EasxMeter@@UAEPAXI@Z    1001ace0 f i asxhpi.obj
 0001:00019d20       ??_EasxMeterHPI@@UAEPAXI@Z 1001ad20 f i asxhpi.obj
 0001:00019d20       ??_GasxMeterHPI@@UAEPAXI@Z 1001ad20 f i asxhpi.obj
 0001:00019d60       ??_GasxMic@@UAEPAXI@Z      1001ad60 f i asxhpi.obj
 0001:00019d60       ??_EasxMic@@UAEPAXI@Z      1001ad60 f i asxhpi.obj
 0001:00019da0       ??_GasxMicHPI@@UAEPAXI@Z   1001ada0 f i asxhpi.obj
 0001:00019da0       ??_EasxMicHPI@@UAEPAXI@Z   1001ada0 f i asxhpi.obj
 0001:00019dd0       ??_GasxMixerScannerHPI@@UAEPAXI@Z 1001add0 f i asxhpi.obj
 0001:00019dd0       ??_EasxMixerScannerHPI@@UAEPAXI@Z 1001add0 f i asxhpi.obj
 0001:00019e00       ??_GasxMixerScannerHPIDuplicateIndex@@UAEPAXI@Z 1001ae00 f i asxhpi.obj
 0001:00019e00       ??_EasxMixerScannerHPIDuplicateIndex@@UAEPAXI@Z 1001ae00 f i asxhpi.obj
 0001:00019e30       ??_GasxMode@@UAEPAXI@Z     1001ae30 f i asxhpi.obj
 0001:00019e30       ??_EasxMode@@UAEPAXI@Z     1001ae30 f i asxhpi.obj
 0001:00019eb0       ??_GasxModeHPI@@UAEPAXI@Z  1001aeb0 f i asxhpi.obj
 0001:00019eb0       ??_EasxModeHPI@@UAEPAXI@Z  1001aeb0 f i asxhpi.obj
 0001:00019ee0       ??_EasxMux@@UAEPAXI@Z      1001aee0 f i asxhpi.obj
 0001:00019ee0       ??_GasxMux@@UAEPAXI@Z      1001aee0 f i asxhpi.obj
 0001:00019f70       ??_GasxMuxHPI@@UAEPAXI@Z   1001af70 f i asxhpi.obj
 0001:00019f70       ??_EasxMuxHPI@@UAEPAXI@Z   1001af70 f i asxhpi.obj
 0001:00019fa0       ??_GasxPad@@UAEPAXI@Z      1001afa0 f i asxhpi.obj
 0001:00019fa0       ??_EasxPad@@UAEPAXI@Z      1001afa0 f i asxhpi.obj
 0001:00019fe0       ??_EasxPadHPI@@UAEPAXI@Z   1001afe0 f i asxhpi.obj
 0001:00019fe0       ??_GasxPadHPI@@UAEPAXI@Z   1001afe0 f i asxhpi.obj
 0001:0001a010       ??_EasxParametricEQ@@UAEPAXI@Z 1001b010 f i asxhpi.obj
 0001:0001a010       ??_GasxParametricEQ@@UAEPAXI@Z 1001b010 f i asxhpi.obj
 0001:0001a050       ??_EasxParametricEqHPI@@UAEPAXI@Z 1001b050 f i asxhpi.obj
 0001:0001a050       ??_GasxParametricEqHPI@@UAEPAXI@Z 1001b050 f i asxhpi.obj
 0001:0001a080       ??_GasxSampleClock@@UAEPAXI@Z 1001b080 f i asxhpi.obj
 0001:0001a080       ??_EasxSampleClock@@UAEPAXI@Z 1001b080 f i asxhpi.obj
 0001:0001a110       ??_GasxSampleClockHPI@@UAEPAXI@Z 1001b110 f i asxhpi.obj
 0001:0001a110       ??_EasxSampleClockHPI@@UAEPAXI@Z 1001b110 f i asxhpi.obj
 0001:0001a140       ??_EasxSilenceDetector@@UAEPAXI@Z 1001b140 f i asxhpi.obj
 0001:0001a140       ??_GasxSilenceDetector@@UAEPAXI@Z 1001b140 f i asxhpi.obj
 0001:0001a180       ??_EasxSilenceDetectorHPI@@UAEPAXI@Z 1001b180 f i asxhpi.obj
 0001:0001a180       ??_GasxSilenceDetectorHPI@@UAEPAXI@Z 1001b180 f i asxhpi.obj
 0001:0001a1b0       ??_GasxSubSystemHPI@@UAEPAXI@Z 1001b1b0 f i asxhpi.obj
 0001:0001a1b0       ??_EasxSubSystemHPI@@UAEPAXI@Z 1001b1b0 f i asxhpi.obj
 0001:0001a1e0       ??_GasxToneDetector@@UAEPAXI@Z 1001b1e0 f i asxhpi.obj
 0001:0001a1e0       ??_EasxToneDetector@@UAEPAXI@Z 1001b1e0 f i asxhpi.obj
 0001:0001a220       ??_GasxToneDetectorHPI@@UAEPAXI@Z 1001b220 f i asxhpi.obj
 0001:0001a220       ??_EasxToneDetectorHPI@@UAEPAXI@Z 1001b220 f i asxhpi.obj
 0001:0001a250       ??_EasxTuner@@UAEPAXI@Z    1001b250 f i asxhpi.obj
 0001:0001a250       ??_GasxTuner@@UAEPAXI@Z    1001b250 f i asxhpi.obj
 0001:0001a2e0       ??_GasxTunerHPI@@UAEPAXI@Z 1001b2e0 f i asxhpi.obj
 0001:0001a2e0       ??_EasxTunerHPI@@UAEPAXI@Z 1001b2e0 f i asxhpi.obj
 0001:0001a310       ??_GasxVolume@@UAEPAXI@Z   1001b310 f i asxhpi.obj
 0001:0001a310       ??_EasxVolume@@UAEPAXI@Z   1001b310 f i asxhpi.obj
 0001:0001a350       ??_GasxVolumeHPI@@UAEPAXI@Z 1001b350 f i asxhpi.obj
 0001:0001a350       ??_EasxVolumeHPI@@UAEPAXI@Z 1001b350 f i asxhpi.obj
 0001:0001a390       ??_GasxVox@@UAEPAXI@Z      1001b390 f i asxhpi.obj
 0001:0001a390       ??_EasxVox@@UAEPAXI@Z      1001b390 f i asxhpi.obj
 0001:0001a3d0       ??_EasxVoxHPI@@UAEPAXI@Z   1001b3d0 f i asxhpi.obj
 0001:0001a3d0       ??_GasxVoxHPI@@UAEPAXI@Z   1001b3d0 f i asxhpi.obj
 0001:0001a400       ??_GhpiHMI@@QAEPAXI@Z      1001b400 f i asxhpi.obj
 0001:0001a420       ?Add@?$TASIArray@G@@QAEHPAG@Z 1001b420 f i asxhpi.obj
 0001:0001a450       ?Add@?$TASIArray@H@@QAEHPAH@Z 1001b450 f i asxhpi.obj
 0001:0001a480       ?Add@?$TASIArray@I@@QAEHPAI@Z 1001b480 f i asxhpi.obj
 0001:0001a4b0       ?Add@?$TASIArray@VasxBlockProperty@@@@QAEHPAVasxBlockProperty@@@Z 1001b4b0 f i asxhpi.obj
 0001:0001a4e0       ?Add@?$TASIArray@W4asxAESEBU_FORMAT@@@@QAEHPAW4asxAESEBU_FORMAT@@@Z 1001b4e0 f i asxhpi.obj
 0001:0001a510       ?Add@?$TASIArray@W4asxCHANNELMODE@@@@QAEHPAW4asxCHANNELMODE@@@Z 1001b510 f i asxhpi.obj
 0001:0001a540       ?Add@?$TASIArray@W4asxNODE@@@@QAEHPAW4asxNODE@@@Z 1001b540 f i asxhpi.obj
 0001:0001a570       ?Add@?$TASIArray@W4asxSAMPLE_CLOCK_SOURCE@@@@QAEHPAW4asxSAMPLE_CLOCK_SOURCE@@@Z 1001b570 f i asxhpi.obj
 0001:0001a5a0       ?Add@?$TASIArray@W4asxSAMPLE_RATE@@@@QAEHPAW4asxSAMPLE_RATE@@@Z 1001b5a0 f i asxhpi.obj
 0001:0001a5d0       ?Add@?$TASIArray@W4asxTUNERBAND@@@@QAEHPAW4asxTUNERBAND@@@Z 1001b5d0 f i asxhpi.obj
 0001:0001a600       ?Add@?$TASIArray@W4asxTUNERPROGRAM@@@@QAEHPAW4asxTUNERPROGRAM@@@Z 1001b600 f i asxhpi.obj
 0001:0001a630       ?AddDuplicateIndexAdapter@asxSubSystemHPI@@AAEXIGG@Z 1001b630 f   asxhpi.obj
 0001:0001a7d0       ?AddProperty@asxBlock@@UAEXPAVasxBlockProperty@@@Z 1001b7d0 f i asxhpi.obj
 0001:0001a7e0       ?AddProperty@asxBlockHPI@@QAE?AW4asxERROR@@I@Z 1001b7e0 f   asxhpi.obj
 0001:0001aec0       ?AddSingleAdapter@asxSubSystemHPI@@AAEHIG@Z 1001bec0 f   asxhpi.obj
 0001:0001b0b0       ?CheckIP@asxSubSystemHPI@@AAEXXZ 1001c0b0 f   asxhpi.obj
 0001:0001b0f0       ?CheckSubSystems@asxAdapterHPI@@UAE?AW4asxERROR@@PAI0@Z 1001c0f0 f   asxhpi.obj
 0001:0001b140       ?Clear@?$TASIArray@W4asxAESEBU_FORMAT@@@@QAEXXZ 1001c140 f i asxhpi.obj
 0001:0001b180       ?Clear@?$TASIArray@W4asxSAMPLE_RATE@@@@QAEXXZ 1001c180 f i asxhpi.obj
 0001:0001b1c0       ?Clear@?$TASIArray@W4asxTUNERPROGRAM@@@@QAEXXZ 1001c1c0 f i asxhpi.obj
 0001:0001b200       ?Count@?$TASIArray@G@@QBEHXZ 1001c200 f i asxhpi.obj
 0001:0001b210       ?Count@?$TASIArray@I@@QBEHXZ 1001c210 f i asxhpi.obj
 0001:0001b220       ?CreateUniversalControl@asxMixerScannerHPI@@QAEPAVasxControlBase@@PAHPAVasxNode@@1I@Z 1001c220 f   asxhpi.obj
 0001:0001b360       ?Enlarge@?$TASIArray@G@@AAEXXZ 1001c360 f i asxhpi.obj
 0001:0001b3c0       ?Enlarge@?$TASIArray@H@@AAEXXZ 1001c3c0 f i asxhpi.obj
 0001:0001b420       ?Enlarge@?$TASIArray@I@@AAEXXZ 1001c420 f i asxhpi.obj
 0001:0001b480       ?Enlarge@?$TASIArray@VasxBlockProperty@@@@AAEXXZ 1001c480 f i asxhpi.obj
 0001:0001b4e0       ?Enlarge@?$TASIArray@W4asxAESEBU_FORMAT@@@@AAEXXZ 1001c4e0 f i asxhpi.obj
 0001:0001b540       ?Enlarge@?$TASIArray@W4asxCHANNELMODE@@@@AAEXXZ 1001c540 f i asxhpi.obj
 0001:0001b5a0       ?Enlarge@?$TASIArray@W4asxNODE@@@@AAEXXZ 1001c5a0 f i asxhpi.obj
 0001:0001b600       ?Enlarge@?$TASIArray@W4asxSAMPLE_CLOCK_SOURCE@@@@AAEXXZ 1001c600 f i asxhpi.obj
 0001:0001b660       ?Enlarge@?$TASIArray@W4asxSAMPLE_RATE@@@@AAEXXZ 1001c660 f i asxhpi.obj
 0001:0001b6c0       ?Enlarge@?$TASIArray@W4asxTUNERBAND@@@@AAEXXZ 1001c6c0 f i asxhpi.obj
 0001:0001b720       ?Enlarge@?$TASIArray@W4asxTUNERPROGRAM@@@@AAEXXZ 1001c720 f i asxhpi.obj
 0001:0001b780       ?EnumerateDeemphasis@asxTuner@@UAE?AW4asxERROR@@HPAW4asxTUNERDEEMPHASIS@@PAH@Z 1001c780 f i asxhpi.obj
 0001:0001b790       ?EnumerateDeemphasis@asxTunerHPI@@UAE?AW4asxERROR@@HPAW4asxTUNERDEEMPHASIS@@PAH@Z 1001c790 f   asxhpi.obj
 0001:0001b860       ?Find@?$TASIArray@VasxNode@@@@QAEHPAVasxNode@@@Z 1001c860 f i asxhpi.obj
 0001:0001b8b0       ?Get@asxBlock@@UAE?AW4asxERROR@@IPAUasxParameterValue@@@Z 1001c8b0 f i asxhpi.obj
 0001:0001b8c0       ?Get@asxBlockHPI@@UAE?AW4asxERROR@@IPAUasxParameterValue@@@Z 1001c8c0 f   asxhpi.obj
 0001:0001b9b0       ?Get@asxCompander@@UAE?AW4asxERROR@@PAG0PAF11@Z 1001c9b0 f i asxhpi.obj
 0001:0001b9c0       ?Get@asxCompanderHPI@@UAE?AW4asxERROR@@PAG0PAF11@Z 1001c9c0 f   asxhpi.obj
 0001:0001b9d0       ?Get@asxCompanderHPI_Legacy@@UAE?AW4asxERROR@@PAG0PAF11@Z 1001c9d0 f   asxhpi.obj
 0001:0001ba30       ?Get@asxLevelHPI@@UAE?AW4asxERROR@@PAM@Z 1001ca30 f   asxhpi.obj
 0001:0001ba90       ?Get@asxModeHPI@@UAE?AW4asxERROR@@PAW4asxCHANNELMODE@@@Z 1001ca90 f   asxhpi.obj
 0001:0001bb20       ?Get@asxMuxHPI@@UAE?AW4asxERROR@@PAW4asxNODE@@PAH@Z 1001cb20 f   asxhpi.obj
 0001:0001bbd0       ?GetAttackTimeConstant@asxCompander@@UAE?AW4asxERROR@@W4asxCOMPANDER_INDEX@@PAI@Z 1001cbd0 f i asxhpi.obj
 0001:0001bbe0       ?GetAttackTimeConstant@asxCompanderHPI@@UAE?AW4asxERROR@@W4asxCOMPANDER_INDEX@@PAI@Z 1001cbe0 f   asxhpi.obj
 0001:0001bc30       ?GetAttackTimeConstant@asxCompanderHPI_Legacy@@UAE?AW4asxERROR@@W4asxCOMPANDER_INDEX@@PAI@Z 1001cc30 f   asxhpi.obj
 0001:0001bc60       ?GetBallistics@asxMeter@@UAE?AW4asxERROR@@HPAM0@Z 1001cc60 f i asxhpi.obj
 0001:0001bc70       ?GetBallistics@asxMeterHPI@@UAE?AW4asxERROR@@HPAM0@Z 1001cc70 f   asxhpi.obj
 0001:0001bd20       ?GetBand@asxParametricEQ@@UAE?AW4asxERROR@@GPAW4asxEQBANDTYPE@@PAKPAF2@Z 1001cd20 f i asxhpi.obj
 0001:0001bd30       ?GetBand@asxParametricEqHPI@@UAE?AW4asxERROR@@GPAW4asxEQBANDTYPE@@PAKPAF2@Z 1001cd30 f   asxhpi.obj
 0001:0001be10       ?GetBand@asxTuner@@UAE?AW4asxERROR@@PAW4asxTUNERBAND@@@Z 1001ce10 f i asxhpi.obj
 0001:0001be20       ?GetBand@asxTunerHPI@@UAE?AW4asxERROR@@PAW4asxTUNERBAND@@@Z 1001ce20 f   asxhpi.obj
 0001:0001be80       ?GetBundle@asxCobranetRx@@UAE?AW4asxERROR@@PAI@Z 1001ce80 f i asxhpi.obj
 0001:0001be90       ?GetBundle@asxCobranetRxContainer@@UAE?AW4asxERROR@@PAI@Z 1001ce90 f i asxhpi.obj
 0001:0001bea0       ?GetBundle@asxCobranetRxHPI@@UAE?AW4asxERROR@@PAI@Z 1001cea0 f   asxhpi.obj
 0001:0001bed0       ?GetBundle@asxCobranetTx@@UAE?AW4asxERROR@@PAI@Z 1001ced0 f i asxhpi.obj
 0001:0001bee0       ?GetBundle@asxCobranetTxContainer@@UAE?AW4asxERROR@@PAI@Z 1001cee0 f i asxhpi.obj
 0001:0001bef0       ?GetBundle@asxCobranetTxHPI@@UAE?AW4asxERROR@@PAI@Z 1001cef0 f   asxhpi.obj
 0001:0001bf20       ?GetChannelCount@asxCobranetTx@@UAE?AW4asxERROR@@PAI@Z 1001cf20 f i asxhpi.obj
 0001:0001bf30       ?GetChannelCount@asxCobranetTxContainer@@UAE?AW4asxERROR@@PAI@Z 1001cf30 f i asxhpi.obj
 0001:0001bf40       ?GetChannelCount@asxCobranetTxHPI@@UAE?AW4asxERROR@@PAI@Z 1001cf40 f   asxhpi.obj
 0001:0001bf70       ?GetChannelMap@asxCobranetRx@@UAE?AW4asxERROR@@QAI@Z 1001cf70 f i asxhpi.obj
 0001:0001bf80       ?GetChannelMap@asxCobranetRxContainer@@UAE?AW4asxERROR@@QAI@Z 1001cf80 f i asxhpi.obj
 0001:0001bf90       ?GetChannelMap@asxCobranetRxHPI@@UAE?AW4asxERROR@@QAI@Z 1001cf90 f   asxhpi.obj
 0001:0001bfc0       ?GetChannelMap@asxCobranetTx@@UAE?AW4asxERROR@@QAI@Z 1001cfc0 f i asxhpi.obj
 0001:0001bfd0       ?GetChannelMap@asxCobranetTxContainer@@UAE?AW4asxERROR@@QAI@Z 1001cfd0 f i asxhpi.obj
 0001:0001bfe0       ?GetChannelMap@asxCobranetTxHPI@@UAE?AW4asxERROR@@QAI@Z 1001cfe0 f   asxhpi.obj
 0001:0001c010       ?GetChannels@asxMeter@@UAE?AW4asxERROR@@PAH@Z 1001d010 f i asxhpi.obj
 0001:0001c030       ?GetChannels@asxMeterHPI@@UAE?AW4asxERROR@@PAH@Z 1001d030 f   asxhpi.obj
 0001:0001c070       ?GetChannels@asxVolume@@UAE?AW4asxERROR@@PAH@Z 1001d070 f i asxhpi.obj
 0001:0001c090       ?GetChannels@asxVolumeHPI@@UAE?AW4asxERROR@@PAH@Z 1001d090 f   asxhpi.obj
 0001:0001c0d0       ?GetClockSource@asxSampleClockHPI@@UAE?AW4asxERROR@@PAW4asxSAMPLE_CLOCK_SOURCE@@@Z 1001d0d0 f   asxhpi.obj
 0001:0001c190       ?GetCobranetControl@asxMixerScannerHPI@@QAEIXZ 1001d190 f i asxhpi.obj
 0001:0001c1a0       ?GetConductorPriority@asxCobranet@@UAE?AW4asxERROR@@PAI@Z 1001d1a0 f i asxhpi.obj
 0001:0001c1b0       ?GetConductorPriority@asxCobranetContainer@@UAE?AW4asxERROR@@PAI@Z 1001d1b0 f i asxhpi.obj
 0001:0001c1c0       ?GetConductorPriority@asxCobranetHPI@@UAE?AW4asxERROR@@PAI@Z 1001d1c0 f   asxhpi.obj
 0001:0001c1e0       ?GetConductorStatus@asxCobranet@@UAE?AW4asxERROR@@PAI@Z 1001d1e0 f i asxhpi.obj
 0001:0001c1f0       ?GetConductorStatus@asxCobranetContainer@@UAE?AW4asxERROR@@PAI@Z 1001d1f0 f i asxhpi.obj
 0001:0001c200       ?GetConductorStatus@asxCobranetHPI@@UAE?AW4asxERROR@@PAI@Z 1001d200 f   asxhpi.obj
 0001:0001c220       ?GetDabAudioServiceCount@asxTuner@@UAE?AW4asxERROR@@PAH0@Z 1001d220 f i asxhpi.obj
 0001:0001c230       ?GetDabAudioServiceCount@asxTunerHPI@@UAE?AW4asxERROR@@PAH0@Z 1001d230 f   asxhpi.obj
 0001:0001c2a0       ?GetDabAudioServiceName@asxTuner@@UAE?AW4asxERROR@@PADHH@Z 1001d2a0 f i asxhpi.obj
 0001:0001c2b0       ?GetDabAudioServiceName@asxTunerHPI@@UAE?AW4asxERROR@@PADHH@Z 1001d2b0 f   asxhpi.obj
 0001:0001c2e0       ?GetDecayTimeConstant@asxCompander@@UAE?AW4asxERROR@@W4asxCOMPANDER_INDEX@@PAI@Z 1001d2e0 f i asxhpi.obj
 0001:0001c2f0       ?GetDecayTimeConstant@asxCompanderHPI@@UAE?AW4asxERROR@@W4asxCOMPANDER_INDEX@@PAI@Z 1001d2f0 f   asxhpi.obj
 0001:0001c340       ?GetDecayTimeConstant@asxCompanderHPI_Legacy@@UAE?AW4asxERROR@@W4asxCOMPANDER_INDEX@@PAI@Z 1001d340 f   asxhpi.obj
 0001:0001c370       ?GetDeemphasis@asxTuner@@UAE?AW4asxERROR@@PAW4asxTUNERDEEMPHASIS@@@Z 1001d370 f i asxhpi.obj
 0001:0001c390       ?GetDeemphasis@asxTunerHPI@@UAE?AW4asxERROR@@PAW4asxTUNERDEEMPHASIS@@@Z 1001d390 f   asxhpi.obj
 0001:0001c400       ?GetDelay@asxSilenceDetector@@UAE?AW4asxERROR@@PAI@Z 1001d400 f i asxhpi.obj
 0001:0001c410       ?GetDelay@asxSilenceDetectorHPI@@UAE?AW4asxERROR@@PAI@Z 1001d410 f   asxhpi.obj
 0001:0001c450       ?GetDescription@asxCobranet@@UAE?AW4asxERROR@@PADH@Z 1001d450 f i asxhpi.obj
 0001:0001c460       ?GetDescription@asxCobranetContainer@@UAE?AW4asxERROR@@PADH@Z 1001d460 f i asxhpi.obj
 0001:0001c470       ?GetDescription@asxCobranetHPI@@UAE?AW4asxERROR@@PADH@Z 1001d470 f   asxhpi.obj
 0001:0001c4a0       ?GetDspUtilization@asxAdapterHPI@@UAE?AW4asxERROR@@HPAH@Z 1001d4a0 f   asxhpi.obj
 0001:0001c500       ?GetEnable@asxCompander@@UAE?AW4asxERROR@@PAI@Z 1001d500 f i asxhpi.obj
 0001:0001c510       ?GetEnable@asxCompanderHPI@@UAE?AW4asxERROR@@PAI@Z 1001d510 f   asxhpi.obj
 0001:0001c550       ?GetEnable@asxCompanderHPI_Legacy@@UAE?AW4asxERROR@@PAI@Z 1001d550 f   asxhpi.obj
 0001:0001c580       ?GetEnable@asxSilenceDetector@@UAE?AW4asxERROR@@PAI@Z 1001d580 f i asxhpi.obj
 0001:0001c590       ?GetEnable@asxSilenceDetectorHPI@@UAE?AW4asxERROR@@PAI@Z 1001d590 f   asxhpi.obj
 0001:0001c5d0       ?GetEnable@asxToneDetector@@UAE?AW4asxERROR@@PAI@Z 1001d5d0 f i asxhpi.obj
 0001:0001c5e0       ?GetEnable@asxToneDetectorHPI@@UAE?AW4asxERROR@@PAI@Z 1001d5e0 f   asxhpi.obj
 0001:0001c620       ?GetEnumName@asxBlock@@UAE?AW4asxERROR@@IIPADI@Z 1001d620 f i asxhpi.obj
 0001:0001c630       ?GetErrorInfo@asxCobranet@@UAE?AW4asxERROR@@PAI00@Z 1001d630 f i asxhpi.obj
 0001:0001c640       ?GetErrorInfo@asxCobranetContainer@@UAE?AW4asxERROR@@PAI00@Z 1001d640 f i asxhpi.obj
 0001:0001c650       ?GetErrorInfo@asxCobranetHPI@@UAE?AW4asxERROR@@PAI00@Z 1001d650 f   asxhpi.obj
 0001:0001c6a0       ?GetErrorStatus@asxAesebuReceiverHPI@@UAE?AW4asxERROR@@PAI0@Z 1001d6a0 f   asxhpi.obj
 0001:0001c730       ?GetEventEnable@asxSilenceDetector@@UAE?AW4asxERROR@@PAI@Z 1001d730 f i asxhpi.obj
 0001:0001c740       ?GetEventEnable@asxSilenceDetectorHPI@@UAE?AW4asxERROR@@PAI@Z 1001d740 f   asxhpi.obj
 0001:0001c7a0       ?GetEventEnable@asxToneDetector@@UAE?AW4asxERROR@@PAI@Z 1001d7a0 f i asxhpi.obj
 0001:0001c7b0       ?GetEventEnable@asxToneDetectorHPI@@UAE?AW4asxERROR@@PAI@Z 1001d7b0 f   asxhpi.obj
 0001:0001c7f0       ?GetFirmwareRevision@asxCobranet@@UAE?AW4asxERROR@@PAD@Z 1001d7f0 f i asxhpi.obj
 0001:0001c800       ?GetFirmwareRevision@asxCobranetContainer@@UAE?AW4asxERROR@@PAD@Z 1001d800 f i asxhpi.obj
 0001:0001c810       ?GetFirmwareRevision@asxCobranetHPI@@UAE?AW4asxERROR@@PAD@Z 1001d810 f   asxhpi.obj
 0001:0001c820       ?GetFormat@asxAes3TxHPI@@UAE?AW4asxERROR@@PAW4asxAESEBU_FORMAT@@@Z 1001d820 f   asxhpi.obj
 0001:0001c8b0       ?GetFormat@asxAesebuReceiverHPI@@UAE?AW4asxERROR@@PAW4asxAESEBU_FORMAT@@@Z 1001d8b0 f   asxhpi.obj
 0001:0001c940       ?GetFormat@asxCobranetTx@@UAE?AW4asxERROR@@PAW4asxAUDIO_FORMAT@@@Z 1001d940 f i asxhpi.obj
 0001:0001c950       ?GetFormat@asxCobranetTxContainer@@UAE?AW4asxERROR@@PAW4asxAUDIO_FORMAT@@@Z 1001d950 f i asxhpi.obj
 0001:0001c960       ?GetFormat@asxCobranetTxHPI@@UAE?AW4asxERROR@@PAW4asxAUDIO_FORMAT@@@Z 1001d960 f   asxhpi.obj
 0001:0001c9e0       ?GetFrequency@asxToneDetector@@UAE?AW4asxERROR@@IPAI@Z 1001d9e0 f i asxhpi.obj
 0001:0001c9f0       ?GetFrequency@asxToneDetectorHPI@@UAE?AW4asxERROR@@IPAI@Z 1001d9f0 f   asxhpi.obj
 0001:0001ca50       ?GetFrequency@asxTuner@@UAE?AW4asxERROR@@PAK@Z 1001da50 f i asxhpi.obj
 0001:0001ca60       ?GetFrequency@asxTunerHPI@@UAE?AW4asxERROR@@PAK@Z 1001da60 f   asxhpi.obj
 0001:0001cab0       ?GetFrequencyRange@asxTuner@@UAE?AW4asxERROR@@W4asxTUNERBAND@@PAK11@Z 1001dab0 f i asxhpi.obj
 0001:0001cac0       ?GetFrequencyRange@asxTunerHPI@@UAE?AW4asxERROR@@W4asxTUNERBAND@@PAK11@Z 1001dac0 f   asxhpi.obj
 0001:0001cb60       ?GetGain@asxTuner@@UAE?AW4asxERROR@@PAM@Z 1001db60 f i asxhpi.obj
 0001:0001cb70       ?GetGain@asxTunerHPI@@UAE?AW4asxERROR@@PAM@Z 1001db70 f   asxhpi.obj
 0001:0001cbf0       ?GetGain@asxVolumeHPI@@UAE?AW4asxERROR@@PAMH@Z 1001dbf0 f   asxhpi.obj
 0001:0001cd60       ?GetGainRange@asxTuner@@UAE?AW4asxERROR@@PAM00@Z 1001dd60 f i asxhpi.obj
 0001:0001cd70       ?GetGainRange@asxTunerHPI@@UAE?AW4asxERROR@@PAM00@Z 1001dd70 f   asxhpi.obj
 0001:0001cdc0       ?GetHpiControl@asxAes3TxHPI@@UAE?AW4asxERROR@@PAPAXPAI@Z 1001ddc0 f i asxhpi.obj
 0001:0001cdd0       ?GetHpiControl@asxAesebuReceiverHPI@@UAE?AW4asxERROR@@PAPAXPAI@Z 1001ddd0 f i asxhpi.obj
 0001:0001cde0       ?GetHpiControl@asxCobranetHPI@@UAE?AW4asxERROR@@PAPAXPAI@Z 1001dde0 f i asxhpi.obj
 0001:0001cdf0       ?GetHpiControl@asxCompanderHPI@@UAE?AW4asxERROR@@PAPAXPAI@Z 1001ddf0 f i asxhpi.obj
 0001:0001ce00       ?GetHpiControl@asxCompanderHPI_Legacy@@UAE?AW4asxERROR@@PAPAXPAI@Z 1001de00 f i asxhpi.obj
 0001:0001ce10       ?GetHpiControl@asxGpioHPI@@UAE?AW4asxERROR@@PAPAXPAI@Z 1001de10 f i asxhpi.obj
 0001:0001ce20       ?GetHpiControl@asxLevelHPI@@UAE?AW4asxERROR@@PAPAXPAI@Z 1001de20 f i asxhpi.obj
 0001:0001ce30       ?GetHpiControl@asxMeterHPI@@UAE?AW4asxERROR@@PAPAXPAI@Z 1001de30 f i asxhpi.obj
 0001:0001ce40       ?GetHpiControl@asxMicHPI@@UAE?AW4asxERROR@@PAPAXPAI@Z 1001de40 f i asxhpi.obj
 0001:0001ce50       ?GetHpiControl@asxModeHPI@@UAE?AW4asxERROR@@PAPAXPAI@Z 1001de50 f i asxhpi.obj
 0001:0001ce60       ?GetHpiControl@asxMuxHPI@@UAE?AW4asxERROR@@PAPAXPAI@Z 1001de60 f i asxhpi.obj
 0001:0001ce70       ?GetHpiControl@asxParametricEqHPI@@UAE?AW4asxERROR@@PAPAXPAI@Z 1001de70 f i asxhpi.obj
 0001:0001ce80       ?GetHpiControl@asxSampleClockHPI@@UAE?AW4asxERROR@@PAPAXPAI@Z 1001de80 f i asxhpi.obj
 0001:0001ce90       ?GetHpiControl@asxSilenceDetectorHPI@@UAE?AW4asxERROR@@PAPAXPAI@Z 1001de90 f i asxhpi.obj
 0001:0001cea0       ?GetHpiControl@asxToneDetectorHPI@@UAE?AW4asxERROR@@PAPAXPAI@Z 1001dea0 f i asxhpi.obj
 0001:0001ceb0       ?GetHpiControl@asxTunerHPI@@UAE?AW4asxERROR@@PAPAXPAI@Z 1001deb0 f i asxhpi.obj
 0001:0001cec0       ?GetHpiControl@asxVolumeHPI@@UAE?AW4asxERROR@@PAPAXPAI@Z 1001dec0 f i asxhpi.obj
 0001:0001ced0       ?GetHpiControl@asxVoxHPI@@UAE?AW4asxERROR@@PAPAXPAI@Z 1001ded0 f i asxhpi.obj
 0001:0001cee0       ?GetIPAddress@asxCobranet@@UAE?AW4asxERROR@@PAI@Z 1001dee0 f i asxhpi.obj
 0001:0001cef0       ?GetIPAddress@asxCobranetContainer@@UAE?AW4asxERROR@@PAI@Z 1001def0 f i asxhpi.obj
 0001:0001cf00       ?GetIPAddress@asxCobranetHPI@@UAE?AW4asxERROR@@PAI@Z 1001df00 f   asxhpi.obj
 0001:0001cf80       ?GetIfStatus@asxCobranet@@UAE?AW4asxERROR@@PAI00@Z 1001df80 f i asxhpi.obj
 0001:0001cf90       ?GetIfStatus@asxCobranetContainer@@UAE?AW4asxERROR@@PAI00@Z 1001df90 f i asxhpi.obj
 0001:0001cfa0       ?GetIfStatus@asxCobranetHPI@@UAE?AW4asxERROR@@PAI00@Z 1001dfa0 f   asxhpi.obj
 0001:0001d000       ?GetInfo@asxBlock@@UAE?AW4asxERROR@@PADIPAI@Z 1001e000 f i asxhpi.obj
 0001:0001d010       ?GetInfo@asxBlockHPI@@UAE?AW4asxERROR@@PADIPAI@Z 1001e010 f   asxhpi.obj
 0001:0001d040       ?GetInfo@asxParametricEQ@@UAE?AW4asxERROR@@PAG0@Z 1001e040 f i asxhpi.obj
 0001:0001d050       ?GetInfo@asxParametricEqHPI@@UAE?AW4asxERROR@@PAG0@Z 1001e050 f   asxhpi.obj
 0001:0001d0b0       ?GetIpAddress@asxAdapterHPI@@UAE?AW4asxERROR@@PAD@Z 1001e0b0 f   asxhpi.obj
 0001:0001d130       ?GetLatencyAndSampleRate@asxCobranet@@UAE?AW4asxERROR@@PAW4asxCOBRANET_LATENCY@@PAW4asxSAMPLE_RATE@@@Z 1001e130 f i asxhpi.obj
 0001:0001d140       ?GetLatencyAndSampleRate@asxCobranetContainer@@UAE?AW4asxERROR@@PAW4asxCOBRANET_LATENCY@@PAW4asxSAMPLE_RATE@@@Z 1001e140 f i asxhpi.obj
 0001:0001d150       ?GetLatencyAndSampleRate@asxCobranetHPI@@UAE?AW4asxERROR@@PAW4asxCOBRANET_LATENCY@@PAW4asxSAMPLE_RATE@@@Z 1001e150 f   asxhpi.obj
 0001:0001d1b0       ?GetLegacy@asxCompanderHPI_Legacy@@AAE?AW4asxERROR@@XZ 1001e1b0 f   asxhpi.obj
 0001:0001d290       ?GetLevel@asxVoxHPI@@UAE?AW4asxERROR@@PAM@Z 1001e290 f   asxhpi.obj
 0001:0001d2f0       ?GetLocalRate@asxSampleClockHPI@@UAE?AW4asxERROR@@PAH@Z 1001e2f0 f   asxhpi.obj
 0001:0001d340       ?GetLocation@asxCobranet@@UAE?AW4asxERROR@@PADH@Z 1001e340 f i asxhpi.obj
 0001:0001d350       ?GetLocation@asxCobranetContainer@@UAE?AW4asxERROR@@PADH@Z 1001e350 f i asxhpi.obj
 0001:0001d360       ?GetLocation@asxCobranetHPI@@UAE?AW4asxERROR@@PADH@Z 1001e360 f   asxhpi.obj
 0001:0001d390       ?GetMACAddress@asxCobranet@@UAE?AW4asxERROR@@PAIPAG@Z 1001e390 f i asxhpi.obj
 0001:0001d3a0       ?GetMACAddress@asxCobranetContainer@@UAE?AW4asxERROR@@PAIPAG@Z 1001e3a0 f i asxhpi.obj
 0001:0001d3b0       ?GetMACAddress@asxCobranetHPI@@UAE?AW4asxERROR@@PAIPAG@Z 1001e3b0 f   asxhpi.obj
 0001:0001d430       ?GetMacAddress@asxAdapterHPI@@UAE?AW4asxERROR@@PAD@Z 1001e430 f   asxhpi.obj
 0001:0001d490       ?GetMacAddress@asxAdapterHPIDuplicateIndex@@UAE?AW4asxERROR@@PAD@Z 1001e490 f   asxhpi.obj
 0001:0001d4c0       ?GetMakeupGain@asxCompander@@UAE?AW4asxERROR@@PAM@Z 1001e4c0 f i asxhpi.obj
 0001:0001d4d0       ?GetMakeupGain@asxCompanderHPI@@UAE?AW4asxERROR@@PAM@Z 1001e4d0 f   asxhpi.obj
 0001:0001d540       ?GetMakeupGain@asxCompanderHPI_Legacy@@UAE?AW4asxERROR@@PAM@Z 1001e540 f   asxhpi.obj
 0001:0001d570       ?GetMinimumDelay@asxCobranetRx@@UAE?AW4asxERROR@@PAI@Z 1001e570 f i asxhpi.obj
 0001:0001d580       ?GetMinimumDelay@asxCobranetRxContainer@@UAE?AW4asxERROR@@PAI@Z 1001e580 f i asxhpi.obj
 0001:0001d590       ?GetMinimumDelay@asxCobranetRxHPI@@UAE?AW4asxERROR@@PAI@Z 1001e590 f   asxhpi.obj
 0001:0001d5c0       ?GetMode@asxAdapterHPI@@UAE?AW4asxERROR@@PAW4asxADAPTERMODE@@@Z 1001e5c0 f   asxhpi.obj
 0001:0001d660       ?GetMode@asxTuner@@UAE?AW4asxERROR@@W4asxTUNERMODE@@PAW43@@Z 1001e660 f i asxhpi.obj
 0001:0001d670       ?GetMode@asxTunerHPI@@UAE?AW4asxERROR@@W4asxTUNERMODE@@PAW43@@Z 1001e670 f   asxhpi.obj
 0001:0001d6f0       ?GetMute@asxVolumeHPI@@UAE?AW4asxERROR@@PAHH@Z 1001e6f0 f   asxhpi.obj
 0001:0001d770       ?GetName@asxCobranet@@UAE?AW4asxERROR@@PADH@Z 1001e770 f i asxhpi.obj
 0001:0001d780       ?GetName@asxCobranetContainer@@UAE?AW4asxERROR@@PADH@Z 1001e780 f i asxhpi.obj
 0001:0001d790       ?GetName@asxCobranetHPI@@UAE?AW4asxERROR@@PADH@Z 1001e790 f   asxhpi.obj
 0001:0001d7c0       ?GetParamCount@asxBlockHPI@@QAEIXZ 1001e7c0 f i asxhpi.obj
 0001:0001d7d0       ?GetPeak@asxMeter@@UAE?AW4asxERROR@@PAMH@Z 1001e7d0 f i asxhpi.obj
 0001:0001d7e0       ?GetPeak@asxMeterHPI@@UAE?AW4asxERROR@@PAMH@Z 1001e7e0 f   asxhpi.obj
 0001:0001d950       ?GetPersistence@asxCobranet@@UAE?AW4asxERROR@@PAI@Z 1001e950 f i asxhpi.obj
 0001:0001d960       ?GetPersistence@asxCobranetContainer@@UAE?AW4asxERROR@@PAI@Z 1001e960 f i asxhpi.obj
 0001:0001d970       ?GetPersistence@asxCobranetHPI@@UAE?AW4asxERROR@@PAI@Z 1001e970 f   asxhpi.obj
 0001:0001d990       ?GetPhantomPower@asxMic@@UAE?AW4asxERROR@@PAH@Z 1001e990 f i asxhpi.obj
 0001:0001d9a0       ?GetPhantomPower@asxMicHPI@@UAE?AW4asxERROR@@PAH@Z 1001e9a0 f   asxhpi.obj
 0001:0001d9f0       ?GetPriority@asxCobranet@@QAEHXZ 1001e9f0 f i asxhpi.obj
 0001:0001da00       ?GetProgram@asxTuner@@UAE?AW4asxERROR@@PAW4asxTUNERPROGRAM@@@Z 1001ea00 f i asxhpi.obj
 0001:0001da20       ?GetProgram@asxTunerHPI@@UAE?AW4asxERROR@@PAW4asxTUNERPROGRAM@@@Z 1001ea20 f   asxhpi.obj
 0001:0001da80       ?GetProgramTypeString@asxPad@@UAE?AW4asxERROR@@W4asxTUNER_RDS_TYPE@@HPADH@Z 1001ea80 f i asxhpi.obj
 0001:0001da90       ?GetProgramTypeString@asxPadHPI@@UAE?AW4asxERROR@@W4asxTUNER_RDS_TYPE@@HPADH@Z 1001ea90 f   asxhpi.obj
 0001:0001dad0       ?GetProperties@asxGpioHPI@@UAE?AW4asxERROR@@PAH0@Z 1001ead0 f   asxhpi.obj
 0001:0001daf0       ?GetProperty@asxPadHPI@@UAE?AW4asxERROR@@W4eControlProperty@asxControlBase@@W4eControlPropertyType@4@HPAX@Z 1001eaf0 f i asxhpi.obj
 0001:0001db30       ?GetProperty@asxSampleClockHPI@@UAE?AW4asxERROR@@W4eControlProperty@asxControlBase@@W4eControlPropertyType@4@HPAX@Z 1001eb30 f i asxhpi.obj
 0001:0001db70       ?GetProperty@asxTunerHPI@@UAE?AW4asxERROR@@W4eControlProperty@asxControlBase@@W4eControlPropertyType@4@HPAX@Z 1001eb70 f i asxhpi.obj
 0001:0001dbb0       ?GetPropertyHPI@asxControlBaseHPI@@QAEGW4eControlProperty@asxControlBase@@W4eControlPropertyType@3@HPAX@Z 1001ebb0 f   asxhpi.obj
 0001:0001de40       ?GetRFLevel@asxTuner@@UAE?AW4asxERROR@@PAM@Z 1001ee40 f i asxhpi.obj
 0001:0001de50       ?GetRFLevel@asxTunerHPI@@UAE?AW4asxERROR@@PAM@Z 1001ee50 f   asxhpi.obj
 0001:0001ded0       ?GetRMS@asxMeter@@UAE?AW4asxERROR@@PAMH@Z 1001eed0 f i asxhpi.obj
 0001:0001dee0       ?GetRMS@asxMeterHPI@@UAE?AW4asxERROR@@PAMH@Z 1001eee0 f   asxhpi.obj
 0001:0001e070       ?GetRange@asxLevelHPI@@UAE?AW4asxERROR@@PAM00@Z 1001f070 f   asxhpi.obj
 0001:0001e140       ?GetRange@asxVolumeHPI@@UAE?AW4asxERROR@@PAM00@Z 1001f140 f   asxhpi.obj
 0001:0001e210       ?GetRange@asxVoxHPI@@UAE?AW4asxERROR@@PAM00@Z 1001f210 f   asxhpi.obj
 0001:0001e240       ?GetRatio@asxCompander@@UAE?AW4asxERROR@@W4asxCOMPANDER_INDEX@@PAM@Z 1001f240 f i asxhpi.obj
 0001:0001e250       ?GetRatio@asxCompanderHPI@@UAE?AW4asxERROR@@W4asxCOMPANDER_INDEX@@PAM@Z 1001f250 f   asxhpi.obj
 0001:0001e2e0       ?GetRatio@asxCompanderHPI_Legacy@@UAE?AW4asxERROR@@W4asxCOMPANDER_INDEX@@PAM@Z 1001f2e0 f   asxhpi.obj
 0001:0001e320       ?GetRawRFLevel@asxTuner@@UAE?AW4asxERROR@@PAH@Z 1001f320 f i asxhpi.obj
 0001:0001e330       ?GetRawRFLevel@asxTunerHPI@@UAE?AW4asxERROR@@PAH@Z 1001f330 f   asxhpi.obj
 0001:0001e380       ?GetSampleRate@asxAesebuReceiverHPI@@UAE?AW4asxERROR@@PAI@Z 1001f380 f   asxhpi.obj
 0001:0001e3f0       ?GetSampleRate@asxSampleClockHPI@@UAE?AW4asxERROR@@PAH@Z 1001f3f0 f   asxhpi.obj
 0001:0001e440       ?GetSerialConfig@asxCobranet@@UAE?AW4asxERROR@@PAI0QADPAH1@Z 1001f440 f i asxhpi.obj
 0001:0001e450       ?GetSerialConfig@asxCobranetContainer@@UAE?AW4asxERROR@@PAI0QADPAH1@Z 1001f450 f i asxhpi.obj
 0001:0001e460       ?GetSerialConfig@asxCobranetHPI@@UAE?AW4asxERROR@@PAI0QADPAH1@Z 1001f460 f   asxhpi.obj
 0001:0001e4c0       ?GetSerialEnable@asxCobranet@@UAE?AW4asxERROR@@PAH@Z 1001f4c0 f i asxhpi.obj
 0001:0001e4d0       ?GetSerialEnable@asxCobranetContainer@@UAE?AW4asxERROR@@PAH@Z 1001f4d0 f i asxhpi.obj
 0001:0001e4e0       ?GetSerialEnable@asxCobranetHPI@@UAE?AW4asxERROR@@PAH@Z 1001f4e0 f   asxhpi.obj
 0001:0001e4f0       ?GetSourceMAC@asxCobranetRx@@UAE?AW4asxERROR@@PAIPAG@Z 1001f4f0 f i asxhpi.obj
 0001:0001e500       ?GetSourceMAC@asxCobranetRxContainer@@UAE?AW4asxERROR@@PAIPAG@Z 1001f500 f i asxhpi.obj
 0001:0001e510       ?GetSourceMAC@asxCobranetRxHPI@@UAE?AW4asxERROR@@PAIPAG@Z 1001f510 f   asxhpi.obj
 0001:0001e560       ?GetState@asxSilenceDetector@@UAE?AW4asxERROR@@PAI@Z 1001f560 f i asxhpi.obj
 0001:0001e570       ?GetState@asxSilenceDetectorHPI@@UAE?AW4asxERROR@@PAI@Z 1001f570 f   asxhpi.obj
 0001:0001e5b0       ?GetState@asxToneDetector@@UAE?AW4asxERROR@@PAI@Z 1001f5b0 f i asxhpi.obj
 0001:0001e5c0       ?GetState@asxToneDetectorHPI@@UAE?AW4asxERROR@@PAI@Z 1001f5c0 f   asxhpi.obj
 0001:0001e600       ?GetStaticIPAddress@asxCobranet@@UAE?AW4asxERROR@@PAI@Z 1001f600 f i asxhpi.obj
 0001:0001e610       ?GetStaticIPAddress@asxCobranetContainer@@UAE?AW4asxERROR@@PAI@Z 1001f610 f i asxhpi.obj
 0001:0001e620       ?GetStaticIPAddress@asxCobranetHPI@@UAE?AW4asxERROR@@PAI@Z 1001f620 f   asxhpi.obj
 0001:0001e660       ?GetStatus@asxCobranetRx@@UAE?AW4asxERROR@@PAI00QAI@Z 1001f660 f i asxhpi.obj
 0001:0001e670       ?GetStatus@asxCobranetRxContainer@@UAE?AW4asxERROR@@PAI00QAI@Z 1001f670 f i asxhpi.obj
 0001:0001e680       ?GetStatus@asxCobranetRxHPI@@UAE?AW4asxERROR@@PAI00QAI@Z 1001f680 f   asxhpi.obj
 0001:0001e720       ?GetStatus@asxCobranetTx@@UAE?AW4asxERROR@@PAI00@Z 1001f720 f i asxhpi.obj
 0001:0001e730       ?GetStatus@asxCobranetTxContainer@@UAE?AW4asxERROR@@PAI00@Z 1001f730 f i asxhpi.obj
 0001:0001e740       ?GetStatus@asxCobranetTxHPI@@UAE?AW4asxERROR@@PAI00@Z 1001f740 f   asxhpi.obj
 0001:0001e7b0       ?GetStatus@asxTuner@@UAE?AW4asxERROR@@PAI0@Z 1001f7b0 f i asxhpi.obj
 0001:0001e7c0       ?GetStatus@asxTunerHPI@@UAE?AW4asxERROR@@PAI0@Z 1001f7c0 f   asxhpi.obj
 0001:0001e840       ?GetString@hpiHMI@@QAE?AW4asxERROR@@PBDPAVasxBase@@PADHII@Z 1001f840 f   asxhpi.obj
 0001:0001e920       ?GetThreshold@asxCompander@@UAE?AW4asxERROR@@W4asxCOMPANDER_INDEX@@PAM@Z 1001f920 f i asxhpi.obj
 0001:0001e930       ?GetThreshold@asxCompanderHPI@@UAE?AW4asxERROR@@W4asxCOMPANDER_INDEX@@PAM@Z 1001f930 f   asxhpi.obj
 0001:0001e9b0       ?GetThreshold@asxCompanderHPI_Legacy@@UAE?AW4asxERROR@@W4asxCOMPANDER_INDEX@@PAM@Z 1001f9b0 f   asxhpi.obj
 0001:0001e9f0       ?GetThreshold@asxSilenceDetector@@UAE?AW4asxERROR@@PAM@Z 1001f9f0 f i asxhpi.obj
 0001:0001ea00       ?GetThreshold@asxSilenceDetectorHPI@@UAE?AW4asxERROR@@PAM@Z 1001fa00 f   asxhpi.obj
 0001:0001ea60       ?GetThreshold@asxToneDetector@@UAE?AW4asxERROR@@PAM@Z 1001fa60 f i asxhpi.obj
 0001:0001ea70       ?GetThreshold@asxToneDetectorHPI@@UAE?AW4asxERROR@@PAM@Z 1001fa70 f   asxhpi.obj
 0001:0001ead0       ?GetUnicastMode@asxCobranetTx@@UAE?AW4asxERROR@@PAI0@Z 1001fad0 f i asxhpi.obj
 0001:0001eae0       ?GetUnicastMode@asxCobranetTxContainer@@UAE?AW4asxERROR@@PAI0@Z 1001fae0 f i asxhpi.obj
 0001:0001eaf0       ?GetUnicastMode@asxCobranetTxHPI@@UAE?AW4asxERROR@@PAI0@Z 1001faf0 f   asxhpi.obj
 0001:0001eb40       ?GetUnsigned@hpiHMI@@QAE?AW4asxERROR@@PBDPAVasxBase@@PAII@Z 1001fb40 f   asxhpi.obj
 0001:0001eb60       ?GetUnsignedArray@hpiHMI@@QAE?AW4asxERROR@@PBDPAVasxBase@@PAIII@Z 1001fb60 f   asxhpi.obj
 0001:0001eca0       ?HpiHandlesToIndexes@asxCompanderHPI_Legacy@@AAEGIPAG0@Z 1001fca0 f   asxhpi.obj
 0001:0001ed00       ?InputGet@asxGpioHPI@@UAE?AW4asxERROR@@PAHH@Z 1001fd00 f   asxhpi.obj
 0001:0001edd0       ?IntFloatRange@asxBlock@@UAE?AW4asxERROR@@IPAUasxParameterRangeInfo@@@Z 1001fdd0 f i asxhpi.obj
 0001:0001ede0       ?IntFloatRange@asxBlockHPI@@UAE?AW4asxERROR@@IPAUasxParameterRangeInfo@@@Z 1001fde0 f   asxhpi.obj
 0001:0001eee0       ?MarkReported@asxAdapterHPIDuplicateIndex@@QAEXXZ 1001fee0 f i asxhpi.obj
 0001:0001eef0       ?OpenNvMem@asxAdapterHPI@@AAEGXZ 1001fef0 f   asxhpi.obj
 0001:0001ef40       ?OutputGet@asxGpioHPI@@UAE?AW4asxERROR@@PAHH@Z 1001ff40 f   asxhpi.obj
 0001:0001f030       ?OutputSet@asxGpioHPI@@UAE?AW4asxERROR@@PAHH@Z 10020030 f   asxhpi.obj
 0001:0001f0b0       ?Predelete@asxAdapterHPI@@UAE?AW4asxERROR@@XZ 100200b0 f   asxhpi.obj
 0001:0001f120       ?ReEnumerateLocalRate@asxSampleClockHPI@@QAEXXZ 10020120 f   asxhpi.obj
 0001:0001f390       ?ReEnumerateProgram@asxTuner@@UAE?AW4asxERROR@@XZ 10020390 f i asxhpi.obj
 0001:0001f3a0       ?ReEnumerateProgram@asxTunerHPI@@UAE?AW4asxERROR@@XZ 100203a0 f   asxhpi.obj
 0001:0001f430       ?ReScan@asxSubSystemHPI@@UAEXXZ 10020430 f   asxhpi.obj
 0001:0001f510       ?ReadNvMem@asxAdapterHPI@@UAE?AW4asxERROR@@HPAE@Z 10020510 f   asxhpi.obj
 0001:0001f580       ?ReadProperty@asxAdapterHPI@@UAE?AW4asxERROR@@HPAG0@Z 10020580 f   asxhpi.obj
 0001:0001f690       ?Replace@asxCobranetContainer@@QAEXAAVasxCobranet@@@Z 10020690 f i asxhpi.obj
 0001:0001f700       ?ResetControls@asxMixerScannerHPI@@UAE?AW4asxERROR@@XZ 10020700 f   asxhpi.obj
 0001:0001fcf0       ?Scan@asxMixerScannerHPI@@UAEXPAVasxMixer@@@Z 10020cf0 f   asxhpi.obj
 0001:000210a0       ?Scan@asxMixerScannerHPIDuplicateIndex@@UAEXPAVasxMixer@@@Z 100220a0 f i asxhpi.obj
 0001:000210b0       ?Scan@asxSubSystemHPI@@UAEXXZ 100220b0 f   asxhpi.obj
 0001:000210c0       ?Set@asxBlock@@UAE?AW4asxERROR@@IPAUasxParameterValue@@@Z 100220c0 f i asxhpi.obj
 0001:000210d0       ?Set@asxBlockHPI@@UAE?AW4asxERROR@@IPAUasxParameterValue@@@Z 100220d0 f   asxhpi.obj
 0001:00021180       ?Set@asxCompander@@UAE?AW4asxERROR@@GGFFF@Z 10022180 f i asxhpi.obj
 0001:00021190       ?Set@asxCompanderHPI@@UAE?AW4asxERROR@@GGFFF@Z 10022190 f   asxhpi.obj
 0001:000211a0       ?Set@asxCompanderHPI_Legacy@@UAE?AW4asxERROR@@GGFFF@Z 100221a0 f   asxhpi.obj
 0001:000211e0       ?Set@asxLevelHPI@@UAE?AW4asxERROR@@M@Z 100221e0 f   asxhpi.obj
 0001:00021240       ?Set@asxModeHPI@@UAE?AW4asxERROR@@W4asxCHANNELMODE@@@Z 10022240 f   asxhpi.obj
 0001:000212d0       ?Set@asxMuxHPI@@UAE?AW4asxERROR@@W4asxNODE@@H@Z 100222d0 f   asxhpi.obj
 0001:00021360       ?SetAttackTimeConstant@asxCompander@@UAE?AW4asxERROR@@W4asxCOMPANDER_INDEX@@I@Z 10022360 f i asxhpi.obj
 0001:00021370       ?SetAttackTimeConstant@asxCompanderHPI@@UAE?AW4asxERROR@@W4asxCOMPANDER_INDEX@@I@Z 10022370 f   asxhpi.obj
 0001:000213c0       ?SetAttackTimeConstant@asxCompanderHPI_Legacy@@UAE?AW4asxERROR@@W4asxCOMPANDER_INDEX@@I@Z 100223c0 f   asxhpi.obj
 0001:000213f0       ?SetAutofade@asxVolume@@UAE?AW4asxERROR@@PBMHHW4asxVOLUME_AUTOFADE@@@Z 100223f0 f i asxhpi.obj
 0001:00021400       ?SetAutofade@asxVolumeHPI@@UAE?AW4asxERROR@@PBMHHW4asxVOLUME_AUTOFADE@@@Z 10022400 f   asxhpi.obj
 0001:000214b0       ?SetBallistics@asxMeter@@UAE?AW4asxERROR@@HMM@Z 100224b0 f i asxhpi.obj
 0001:000214c0       ?SetBallistics@asxMeterHPI@@UAE?AW4asxERROR@@HMM@Z 100224c0 f   asxhpi.obj
 0001:00021560       ?SetBand@asxParametricEQ@@UAE?AW4asxERROR@@GW4asxEQBANDTYPE@@KFF@Z 10022560 f i asxhpi.obj
 0001:00021570       ?SetBand@asxParametricEqHPI@@UAE?AW4asxERROR@@GW4asxEQBANDTYPE@@KFF@Z 10022570 f   asxhpi.obj
 0001:00021620       ?SetBand@asxTuner@@UAE?AW4asxERROR@@W4asxTUNERBAND@@@Z 10022620 f i asxhpi.obj
 0001:00021630       ?SetBand@asxTunerHPI@@UAE?AW4asxERROR@@W4asxTUNERBAND@@@Z 10022630 f   asxhpi.obj
 0001:00021680       ?SetBundle@asxCobranetRx@@UAE?AW4asxERROR@@I@Z 10022680 f i asxhpi.obj
 0001:00021690       ?SetBundle@asxCobranetRxContainer@@UAE?AW4asxERROR@@I@Z 10022690 f i asxhpi.obj
 0001:000216a0       ?SetBundle@asxCobranetRxHPI@@UAE?AW4asxERROR@@I@Z 100226a0 f   asxhpi.obj
 0001:000216d0       ?SetBundle@asxCobranetTx@@UAE?AW4asxERROR@@I@Z 100226d0 f i asxhpi.obj
 0001:000216e0       ?SetBundle@asxCobranetTxContainer@@UAE?AW4asxERROR@@I@Z 100226e0 f i asxhpi.obj
 0001:000216f0       ?SetBundle@asxCobranetTxHPI@@UAE?AW4asxERROR@@I@Z 100226f0 f   asxhpi.obj
 0001:00021720       ?SetChannelCount@asxCobranetTx@@UAE?AW4asxERROR@@I@Z 10022720 f i asxhpi.obj
 0001:00021730       ?SetChannelCount@asxCobranetTxContainer@@UAE?AW4asxERROR@@I@Z 10022730 f i asxhpi.obj
 0001:00021740       ?SetChannelCount@asxCobranetTxHPI@@UAE?AW4asxERROR@@I@Z 10022740 f   asxhpi.obj
 0001:00021770       ?SetChannelMap@asxCobranetRx@@UAE?AW4asxERROR@@QBI@Z 10022770 f i asxhpi.obj
 0001:00021780       ?SetChannelMap@asxCobranetRxContainer@@UAE?AW4asxERROR@@QBI@Z 10022780 f i asxhpi.obj
 0001:00021790       ?SetChannelMap@asxCobranetRxHPI@@UAE?AW4asxERROR@@QBI@Z 10022790 f   asxhpi.obj
 0001:000217c0       ?SetChannelMap@asxCobranetTx@@UAE?AW4asxERROR@@QBI@Z 100227c0 f i asxhpi.obj
 0001:000217d0       ?SetChannelMap@asxCobranetTxContainer@@UAE?AW4asxERROR@@QBI@Z 100227d0 f i asxhpi.obj
 0001:000217e0       ?SetChannelMap@asxCobranetTxHPI@@UAE?AW4asxERROR@@QBI@Z 100227e0 f   asxhpi.obj
 0001:00021810       ?SetChannelModification@asxNode@@QAEXH@Z 10022810 f i asxhpi.obj
 0001:00021820       ?SetClockSource@asxSampleClockHPI@@UAE?AW4asxERROR@@W4asxSAMPLE_CLOCK_SOURCE@@@Z 10022820 f   asxhpi.obj
 0001:000218f0       ?SetCobranetControl@asxAdapterHPI@@QAEXI@Z 100228f0 f i asxhpi.obj
 0001:00021910       ?SetConductorPriority@asxCobranet@@UAE?AW4asxERROR@@I@Z 10022910 f i asxhpi.obj
 0001:00021920       ?SetConductorPriority@asxCobranetContainer@@UAE?AW4asxERROR@@I@Z 10022920 f i asxhpi.obj
 0001:00021930       ?SetConductorPriority@asxCobranetHPI@@UAE?AW4asxERROR@@I@Z 10022930 f   asxhpi.obj
 0001:00021950       ?SetDabAudioService@asxTuner@@UAE?AW4asxERROR@@H@Z 10022950 f i asxhpi.obj
 0001:00021960       ?SetDabAudioService@asxTunerHPI@@UAE?AW4asxERROR@@H@Z 10022960 f   asxhpi.obj
 0001:00021990       ?SetDecayTimeConstant@asxCompander@@UAE?AW4asxERROR@@W4asxCOMPANDER_INDEX@@I@Z 10022990 f i asxhpi.obj
 0001:000219a0       ?SetDecayTimeConstant@asxCompanderHPI@@UAE?AW4asxERROR@@W4asxCOMPANDER_INDEX@@I@Z 100229a0 f   asxhpi.obj
 0001:000219f0       ?SetDecayTimeConstant@asxCompanderHPI_Legacy@@UAE?AW4asxERROR@@W4asxCOMPANDER_INDEX@@I@Z 100229f0 f   asxhpi.obj
 0001:00021a20       ?SetDeemphasis@asxTuner@@UAE?AW4asxERROR@@W4asxTUNERDEEMPHASIS@@@Z 10022a20 f i asxhpi.obj
 0001:00021a30       ?SetDeemphasis@asxTunerHPI@@UAE?AW4asxERROR@@W4asxTUNERDEEMPHASIS@@@Z 10022a30 f   asxhpi.obj
 0001:00021a90       ?SetDelay@asxSilenceDetector@@UAE?AW4asxERROR@@I@Z 10022a90 f i asxhpi.obj
 0001:00021aa0       ?SetDelay@asxSilenceDetectorHPI@@UAE?AW4asxERROR@@I@Z 10022aa0 f   asxhpi.obj
 0001:00021ae0       ?SetEnable@asxCompander@@UAE?AW4asxERROR@@I@Z 10022ae0 f i asxhpi.obj
 0001:00021af0       ?SetEnable@asxCompanderHPI@@UAE?AW4asxERROR@@I@Z 10022af0 f   asxhpi.obj
 0001:00021b30       ?SetEnable@asxCompanderHPI_Legacy@@UAE?AW4asxERROR@@I@Z 10022b30 f   asxhpi.obj
 0001:00021b50       ?SetEnable@asxSilenceDetector@@UAE?AW4asxERROR@@I@Z 10022b50 f i asxhpi.obj
 0001:00021b60       ?SetEnable@asxSilenceDetectorHPI@@UAE?AW4asxERROR@@I@Z 10022b60 f   asxhpi.obj
 0001:00021ba0       ?SetEnable@asxToneDetector@@UAE?AW4asxERROR@@I@Z 10022ba0 f i asxhpi.obj
 0001:00021bb0       ?SetEnable@asxToneDetectorHPI@@UAE?AW4asxERROR@@I@Z 10022bb0 f   asxhpi.obj
 0001:00021bf0       ?SetEventEnable@asxSilenceDetector@@UAE?AW4asxERROR@@I@Z 10022bf0 f i asxhpi.obj
 0001:00021c00       ?SetEventEnable@asxSilenceDetectorHPI@@UAE?AW4asxERROR@@I@Z 10022c00 f   asxhpi.obj
 0001:00021c60       ?SetEventEnable@asxToneDetector@@UAE?AW4asxERROR@@I@Z 10022c60 f i asxhpi.obj
 0001:00021c70       ?SetEventEnable@asxToneDetectorHPI@@UAE?AW4asxERROR@@I@Z 10022c70 f   asxhpi.obj
 0001:00021cb0       ?SetFormat@asxAes3TxHPI@@UAE?AW4asxERROR@@W4asxAESEBU_FORMAT@@@Z 10022cb0 f   asxhpi.obj
 0001:00021d30       ?SetFormat@asxAesebuReceiverHPI@@UAE?AW4asxERROR@@W4asxAESEBU_FORMAT@@@Z 10022d30 f   asxhpi.obj
 0001:00021d90       ?SetFormat@asxCobranetTx@@UAE?AW4asxERROR@@W4asxAUDIO_FORMAT@@@Z 10022d90 f i asxhpi.obj
 0001:00021da0       ?SetFormat@asxCobranetTxContainer@@UAE?AW4asxERROR@@W4asxAUDIO_FORMAT@@@Z 10022da0 f i asxhpi.obj
 0001:00021db0       ?SetFormat@asxCobranetTxHPI@@UAE?AW4asxERROR@@W4asxAUDIO_FORMAT@@@Z 10022db0 f   asxhpi.obj
 0001:00021e70       ?SetFrequency@asxTuner@@UAE?AW4asxERROR@@K@Z 10022e70 f i asxhpi.obj
 0001:00021e80       ?SetFrequency@asxTunerHPI@@UAE?AW4asxERROR@@K@Z 10022e80 f   asxhpi.obj
 0001:00021ec0       ?SetGain@asxTuner@@UAE?AW4asxERROR@@M@Z 10022ec0 f i asxhpi.obj
 0001:00021ed0       ?SetGain@asxTunerHPI@@UAE?AW4asxERROR@@M@Z 10022ed0 f   asxhpi.obj
 0001:00021f20       ?SetGain@asxVolumeHPI@@UAE?AW4asxERROR@@PBMH@Z 10022f20 f   asxhpi.obj
 0001:00021fc0       ?SetIPAddress@asxCobranet@@UAE?AW4asxERROR@@I@Z 10022fc0 f i asxhpi.obj
 0001:00021fd0       ?SetIPAddress@asxCobranetContainer@@UAE?AW4asxERROR@@I@Z 10022fd0 f i asxhpi.obj
 0001:00021fe0       ?SetIPAddress@asxCobranetHPI@@UAE?AW4asxERROR@@I@Z 10022fe0 f   asxhpi.obj
 0001:00022010       ?SetLatencyAndSampleRate@asxCobranet@@UAE?AW4asxERROR@@W4asxCOBRANET_LATENCY@@W4asxSAMPLE_RATE@@@Z 10023010 f i asxhpi.obj
 0001:00022020       ?SetLatencyAndSampleRate@asxCobranetContainer@@UAE?AW4asxERROR@@W4asxCOBRANET_LATENCY@@W4asxSAMPLE_RATE@@@Z 10023020 f i asxhpi.obj
 0001:00022030       ?SetLatencyAndSampleRate@asxCobranetHPI@@UAE?AW4asxERROR@@W4asxCOBRANET_LATENCY@@W4asxSAMPLE_RATE@@@Z 10023030 f   asxhpi.obj
 0001:000221a0       ?SetLegacy@asxCompanderHPI_Legacy@@AAE?AW4asxERROR@@XZ 100231a0 f   asxhpi.obj
 0001:00022270       ?SetLevel@asxVoxHPI@@UAE?AW4asxERROR@@M@Z 10023270 f   asxhpi.obj
 0001:000222d0       ?SetLocalRate@asxSampleClockHPI@@UAE?AW4asxERROR@@H@Z 100232d0 f   asxhpi.obj
 0001:00022310       ?SetLocation@asxCobranet@@UAE?AW4asxERROR@@PBD@Z 10023310 f i asxhpi.obj
 0001:00022320       ?SetLocation@asxCobranetContainer@@UAE?AW4asxERROR@@PBD@Z 10023320 f i asxhpi.obj
 0001:00022330       ?SetLocation@asxCobranetHPI@@UAE?AW4asxERROR@@PBD@Z 10023330 f   asxhpi.obj
 0001:00022370       ?SetMakeupGain@asxCompander@@UAE?AW4asxERROR@@M@Z 10023370 f i asxhpi.obj
 0001:00022380       ?SetMakeupGain@asxCompanderHPI@@UAE?AW4asxERROR@@M@Z 10023380 f   asxhpi.obj
 0001:000223d0       ?SetMakeupGain@asxCompanderHPI_Legacy@@UAE?AW4asxERROR@@M@Z 100233d0 f   asxhpi.obj
 0001:00022400       ?SetMinimumDelay@asxCobranetRx@@UAE?AW4asxERROR@@I@Z 10023400 f i asxhpi.obj
 0001:00022410       ?SetMinimumDelay@asxCobranetRxContainer@@UAE?AW4asxERROR@@I@Z 10023410 f i asxhpi.obj
 0001:00022420       ?SetMinimumDelay@asxCobranetRxHPI@@UAE?AW4asxERROR@@I@Z 10023420 f   asxhpi.obj
 0001:00022450       ?SetMode@asxAdapterHPI@@UAE?AW4asxERROR@@W4asxADAPTERMODE@@@Z 10023450 f   asxhpi.obj
 0001:000224e0       ?SetMode@asxTuner@@UAE?AW4asxERROR@@W4asxTUNERMODE@@0@Z 100234e0 f i asxhpi.obj
 0001:000224f0       ?SetMode@asxTunerHPI@@UAE?AW4asxERROR@@W4asxTUNERMODE@@0@Z 100234f0 f   asxhpi.obj
 0001:00022560       ?SetMute@asxVolumeHPI@@UAE?AW4asxERROR@@PAHH@Z 10023560 f   asxhpi.obj
 0001:000225d0       ?SetName@asxCobranet@@UAE?AW4asxERROR@@PBD@Z 100235d0 f i asxhpi.obj
 0001:000225e0       ?SetName@asxCobranetContainer@@UAE?AW4asxERROR@@PBD@Z 100235e0 f i asxhpi.obj
 0001:000225f0       ?SetName@asxCobranetHPI@@UAE?AW4asxERROR@@PBD@Z 100235f0 f   asxhpi.obj
 0001:00022630       ?SetPersistence@asxCobranet@@UAE?AW4asxERROR@@I@Z 10023630 f i asxhpi.obj
 0001:00022640       ?SetPersistence@asxCobranetContainer@@UAE?AW4asxERROR@@I@Z 10023640 f i asxhpi.obj
 0001:00022650       ?SetPersistence@asxCobranetHPI@@UAE?AW4asxERROR@@I@Z 10023650 f   asxhpi.obj
 0001:00022670       ?SetPhantomPower@asxMic@@UAE?AW4asxERROR@@H@Z 10023670 f i asxhpi.obj
 0001:00022680       ?SetPhantomPower@asxMicHPI@@UAE?AW4asxERROR@@H@Z 10023680 f   asxhpi.obj
 0001:000226c0       ?SetProgram@asxTuner@@UAE?AW4asxERROR@@W4asxTUNERPROGRAM@@@Z 100236c0 f i asxhpi.obj
 0001:000226d0       ?SetProgram@asxTunerHPI@@UAE?AW4asxERROR@@W4asxTUNERPROGRAM@@@Z 100236d0 f   asxhpi.obj
 0001:00022720       ?SetProperty@asxSampleClockHPI@@UAE?AW4asxERROR@@W4eControlProperty@asxControlBase@@W4eControlPropertyType@4@HPAX@Z 10023720 f i asxhpi.obj
 0001:00022760       ?SetProperty@asxTunerHPI@@UAE?AW4asxERROR@@W4eControlProperty@asxControlBase@@W4eControlPropertyType@4@HPAX@Z 10023760 f i asxhpi.obj
 0001:000227a0       ?SetPropertyHPI@asxControlBaseHPI@@QAEGW4eControlProperty@asxControlBase@@W4eControlPropertyType@3@HPAX@Z 100237a0 f   asxhpi.obj
 0001:00022820       ?SetRatio@asxCompander@@UAE?AW4asxERROR@@W4asxCOMPANDER_INDEX@@M@Z 10023820 f i asxhpi.obj
 0001:00022830       ?SetRatio@asxCompanderHPI@@UAE?AW4asxERROR@@W4asxCOMPANDER_INDEX@@M@Z 10023830 f   asxhpi.obj
 0001:00022890       ?SetRatio@asxCompanderHPI_Legacy@@UAE?AW4asxERROR@@W4asxCOMPANDER_INDEX@@M@Z 10023890 f   asxhpi.obj
 0001:000228c0       ?SetSerialConfig@asxCobranet@@UAE?AW4asxERROR@@IIQBDH0@Z 100238c0 f i asxhpi.obj
 0001:000228d0       ?SetSerialConfig@asxCobranetContainer@@UAE?AW4asxERROR@@IIQBDH0@Z 100238d0 f i asxhpi.obj
 0001:000228e0       ?SetSerialConfig@asxCobranetHPI@@UAE?AW4asxERROR@@IIQBDH0@Z 100238e0 f   asxhpi.obj
 0001:000228f0       ?SetSerialEnable@asxCobranet@@UAE?AW4asxERROR@@H@Z 100238f0 f i asxhpi.obj
 0001:00022900       ?SetSerialEnable@asxCobranetContainer@@UAE?AW4asxERROR@@H@Z 10023900 f i asxhpi.obj
 0001:00022910       ?SetSerialEnable@asxCobranetHPI@@UAE?AW4asxERROR@@H@Z 10023910 f   asxhpi.obj
 0001:00022920       ?SetSourceMAC@asxCobranetRx@@UAE?AW4asxERROR@@IG@Z 10023920 f i asxhpi.obj
 0001:00022930       ?SetSourceMAC@asxCobranetRxContainer@@UAE?AW4asxERROR@@IG@Z 10023930 f i asxhpi.obj
 0001:00022940       ?SetSourceMAC@asxCobranetRxHPI@@UAE?AW4asxERROR@@IG@Z 10023940 f   asxhpi.obj
 0001:00022950       ?SetState@asxParametricEQ@@UAE?AW4asxERROR@@G@Z 10023950 f i asxhpi.obj
 0001:00022960       ?SetState@asxParametricEqHPI@@UAE?AW4asxERROR@@G@Z 10023960 f   asxhpi.obj
 0001:000229a0       ?SetStaticIPAddress@asxCobranet@@UAE?AW4asxERROR@@I@Z 100239a0 f i asxhpi.obj
 0001:000229b0       ?SetStaticIPAddress@asxCobranetContainer@@UAE?AW4asxERROR@@I@Z 100239b0 f i asxhpi.obj
 0001:000229c0       ?SetStaticIPAddress@asxCobranetHPI@@UAE?AW4asxERROR@@I@Z 100239c0 f   asxhpi.obj
 0001:000229f0       ?SetString@hpiHMI@@QAE?AW4asxERROR@@PBDPAVasxBase@@0HII@Z 100239f0 f   asxhpi.obj
 0001:00022ac0       ?SetThreshold@asxCompander@@UAE?AW4asxERROR@@W4asxCOMPANDER_INDEX@@M@Z 10023ac0 f i asxhpi.obj
 0001:00022ad0       ?SetThreshold@asxCompanderHPI@@UAE?AW4asxERROR@@W4asxCOMPANDER_INDEX@@M@Z 10023ad0 f   asxhpi.obj
 0001:00022b20       ?SetThreshold@asxCompanderHPI_Legacy@@UAE?AW4asxERROR@@W4asxCOMPANDER_INDEX@@M@Z 10023b20 f   asxhpi.obj
 0001:00022b50       ?SetThreshold@asxSilenceDetector@@UAE?AW4asxERROR@@M@Z 10023b50 f i asxhpi.obj
 0001:00022b60       ?SetThreshold@asxSilenceDetectorHPI@@UAE?AW4asxERROR@@M@Z 10023b60 f   asxhpi.obj
 0001:00022bb0       ?SetThreshold@asxToneDetector@@UAE?AW4asxERROR@@M@Z 10023bb0 f i asxhpi.obj
 0001:00022bc0       ?SetThreshold@asxToneDetectorHPI@@UAE?AW4asxERROR@@M@Z 10023bc0 f   asxhpi.obj
 0001:00022c10       ?SetUnicastMode@asxCobranetTx@@UAE?AW4asxERROR@@II@Z 10023c10 f i asxhpi.obj
 0001:00022c20       ?SetUnicastMode@asxCobranetTxContainer@@UAE?AW4asxERROR@@II@Z 10023c20 f i asxhpi.obj
 0001:00022c30       ?SetUnicastMode@asxCobranetTxHPI@@UAE?AW4asxERROR@@II@Z 10023c30 f   asxhpi.obj
 0001:00022c80       ?SetUnsigned@hpiHMI@@QAE?AW4asxERROR@@PBDPAVasxBase@@II@Z 10023c80 f   asxhpi.obj
 0001:00022ca0       ?SetUnsignedArray@hpiHMI@@QAE?AW4asxERROR@@PBDPAVasxBase@@PAIII@Z 10023ca0 f   asxhpi.obj
 0001:00022d90       ?StatusTranslate@asxTunerHPI@@AAEII@Z 10023d90 f   asxhpi.obj
 0001:00022e50       ?UpdateAdapterProperties@asxAdapterHPI@@UAE?AW4asxERROR@@XZ 10023e50 f   asxhpi.obj
 0001:00023070       ?WasReported@asxAdapterHPIDuplicateIndex@@QAEHXZ 10024070 f i asxhpi.obj
 0001:00023080       ?WriteNvMem@asxAdapterHPI@@UAE?AW4asxERROR@@HE@Z 10024080 f   asxhpi.obj
 0001:000230e0       ?WriteProperty@asxAdapterHPI@@UAE?AW4asxERROR@@HGG@Z 100240e0 f   asxhpi.obj
 0001:00023150       ?asxhpi_GetMacAddress@@YA?AW4asxERROR@@HPAD@Z 10024150 f   asxhpi.obj
 0001:000231f0       ?asxhpi_GetMacAddress_str@@YA?AW4asxERROR@@HPAD@Z 100241f0 f   asxhpi.obj
 0001:00023260       ?asxhpi_MapError@@YA?AW4asxERROR@@G@Z 10024260 f   asxhpi.obj
 0001:000234e0       ?asxhpi_Po2@@YAII@Z        100244e0 f   asxhpi.obj
 0001:00023520       ?asxhpi_SetSubsystemError@@YA?AW4asxERROR@@PAVasxBase@@G@Z 10024520 f   asxhpi.obj
 0001:00023560       ?asxhpi_TranslateFormatAsxToHpi@@YA?AW4asxERROR@@W4asxAUDIO_FORMAT@@PAG@Z 10024560 f   asxhpi.obj
 0001:000235a0       ?asxhpi_TranslateFormatHpiToAsx@@YA?AW4asxERROR@@GPAW4asxAUDIO_FORMAT@@@Z 100245a0 f   asxhpi.obj
 0001:000235e0       ?baseGetHpiHandle@asxControlBaseHPI@@QAE?AW4asxERROR@@PAPAXPAI@Z 100245e0 f   asxhpi.obj
 0001:00023600       ?byteSwap@hpiHMI@@QAEXPAEI@Z 10024600 f   asxhpi.obj
 0001:00023640       ?ipSwap@hpiHMI@@QAEII@Z    10024640 f   asxhpi.obj
 0001:00023650       ?sizeofData@asxBlockHPI@@AAEIPBUasxParameterValue@@@Z 10024650 f   asxhpi.obj
 0001:000236b0       ?translateSpecificErrorCode@asxSubSystemHPI@@QAEXIPAPAD@Z 100246b0 f   asxhpi.obj
 0001:000236d0       ??0asxPlayerHPI@@QAE@PAVasxSubSystem@@PAVasxNode@@1G_N@Z 100246d0 f   asxhpiplay.obj
 0001:00023730       ??1asxPlayerHPI@@UAE@XZ    10024730 f   asxhpiplay.obj
 0001:00023790       ??_GasxPlayerHPI@@UAEPAXI@Z 10024790 f i asxhpiplay.obj
 0001:00023790       ??_EasxPlayerHPI@@UAEPAXI@Z 10024790 f i asxhpiplay.obj
 0001:000237c0       ?AllocOutput@asxPlayerHPI@@MAE?AW4asxERROR@@XZ 100247c0 f   asxhpiplay.obj
 0001:00023900       ?FreeOutput@asxPlayerHPI@@MAE?AW4asxERROR@@XZ 10024900 f   asxhpiplay.obj
 0001:00023940       ?HelperThread@asxPlayerHPI@@UAEXXZ 10024940 f   asxhpiplay.obj
 0001:00023ba0       ?OnFileOpen@asxPlayerHPI@@MAE?AW4asxERROR@@XZ 10024ba0 f   asxhpiplay.obj
 0001:00023c10       ?ResetOutput@asxPlayerHPI@@MAE?AW4asxERROR@@XZ 10024c10 f   asxhpiplay.obj
 0001:00023c40       ?SetTimeScale@asxPlayerHPI@@UAE?AW4asxERROR@@M@Z 10024c40 f   asxhpiplay.obj
 0001:00023cb0       ?StartOutput@asxPlayerHPI@@MAE?AW4asxERROR@@XZ 10024cb0 f   asxhpiplay.obj
 0001:00023ce0       ?StopOutput@asxPlayerHPI@@MAE?AW4asxERROR@@XZ 10024ce0 f   asxhpiplay.obj
 0001:00023d10       ??0asxPlayerHPIWithInt@@QAE@PAVasxSubSystem@@PAVasxNode@@1G_N@Z 10024d10 f   asxhpiplayi.obj
 0001:00023d40       ??1asxPlayerHPIWithInt@@UAE@XZ 10024d40 f   asxhpiplayi.obj
 0001:00023d50       ??_EasxPlayerHPIWithInt@@UAEPAXI@Z 10024d50 f i asxhpiplayi.obj
 0001:00023d50       ??_GasxPlayerHPIWithInt@@UAEPAXI@Z 10024d50 f i asxhpiplayi.obj
 0001:00023d80       ?AllocOutput@asxPlayerHPIWithInt@@MAE?AW4asxERROR@@XZ 10024d80 f   asxhpiplayi.obj
 0001:00023e50       ?DiffTime@@YAHKK@Z         10024e50 f   asxhpiplayi.obj
 0001:00023e60       ?HelperThread@asxPlayerHPIWithInt@@UAEXXZ 10024e60 f   asxhpiplayi.obj
 0001:000240e0       ??0asxRecorderHPI@@QAE@PAVasxSubSystem@@PAVasxNode@@1G_N@Z 100250e0 f   asxhpirec.obj
 0001:00024130       ??1asxRecorderHPI@@UAE@XZ  10025130 f   asxhpirec.obj
 0001:00024190       ??_EasxRecorderHPI@@UAEPAXI@Z 10025190 f i asxhpirec.obj
 0001:00024190       ??_GasxRecorderHPI@@UAEPAXI@Z 10025190 f i asxhpirec.obj
 0001:000241c0       ?AllocInput@asxRecorderHPI@@MAE?AW4asxERROR@@XZ 100251c0 f   asxhpirec.obj
 0001:00024280       ?EnumerateAllFormats@asxRecorderHPI@@MAEXXZ 10025280 f   asxhpirec.obj
 0001:00024380       ?FreeInput@asxRecorderHPI@@MAE?AW4asxERROR@@XZ 10025380 f   asxhpirec.obj
 0001:000243d0       ?GetInputPosition@asxRecorderHPI@@MAE?AW4asxERROR@@PAK@Z 100253d0 f   asxhpirec.obj
 0001:00024420       ?HelperThread@asxRecorderHPI@@UAEKXZ 10025420 f   asxhpirec.obj
 0001:00024640       ?SetInputFormat@asxRecorderHPI@@MAE?AW4asxERROR@@XZ 10025640 f   asxhpirec.obj
 0001:00024740       ?StartInput@asxRecorderHPI@@MAE?AW4asxERROR@@XZ 10025740 f   asxhpirec.obj
 0001:00024780       ?StopInput@asxRecorderHPI@@MAE?AW4asxERROR@@XZ 10025780 f   asxhpirec.obj
 0001:000247b0       ??0asxRecorderHPIWithInt@@QAE@PAVasxSubSystem@@PAVasxNode@@1G_N@Z 100257b0 f   asxhpireci.obj
 0001:000247e0       ??1asxRecorderHPIWithInt@@UAE@XZ 100257e0 f   asxhpireci.obj
 0001:000247f0       ??_EasxRecorderHPIWithInt@@UAEPAXI@Z 100257f0 f i asxhpireci.obj
 0001:000247f0       ??_GasxRecorderHPIWithInt@@UAEPAXI@Z 100257f0 f i asxhpireci.obj
 0001:00024820       ?AllocInput@asxRecorderHPIWithInt@@MAE?AW4asxERROR@@XZ 10025820 f   asxhpireci.obj
 0001:000248f0       ?HelperThread@asxRecorderHPIWithInt@@UAEKXZ 100258f0 f   asxhpireci.obj
 0001:00024b00       ?SignalThread@asxRecorderHPIWithInt@@MAEXXZ 10025b00 f   asxhpireci.obj
 0001:00024b20       ??0?$TASIArray@VasxPlayerFile@@@@QAE@XZ 10025b20 f i asxplay.obj
 0001:00024b40       ??0PlayerDoneCallback@@QAE@PAVasxPlayer@@@Z 10025b40 f i asxplay.obj
 0001:00024b60       ??0asios_Mutex_Holder@@QAE@AAPAX@Z 10025b60 f i asxplay.obj
 0001:00024b80       ??0asxCallbackObject@@QAE@XZ 10025b80 f i asxplay.obj
 0001:00024b90       ??0asxPlayer@@QAE@PAVasxSubSystem@@PAVasxNode@@1J@Z 10025b90 f   asxplay.obj
 0001:00024c20       ??0asxPlayerFile@@QAE@PBDJ@Z 10025c20 f   asxplay.obj
 0001:00024ca0       ??0asxPlayerFileList@@QAE@J@Z 10025ca0 f   asxplay.obj
 0001:00024cf0       ??0asxTimescale@@QAE@XZ    10025cf0 f i asxplay.obj
 0001:00024d20       ??1?$TASIArray@VasxPlayerFile@@@@QAE@XZ 10025d20 f i asxplay.obj
 0001:00024d70       ??1PlayerDoneCallback@@UAE@XZ 10025d70 f i asxplay.obj
 0001:00024d80       ??1asios_Mutex_Holder@@QAE@XZ 10025d80 f i asxplay.obj
 0001:00024da0       ??1asxCallbackObject@@UAE@XZ 10025da0 f i asxplay.obj
 0001:00024db0       ??1asxPlayer@@UAE@XZ       10025db0 f   asxplay.obj
 0001:00024e50       ??1asxPlayerFile@@QAE@XZ   10025e50 f   asxplay.obj
 0001:00024e80       ??1asxPlayerFileList@@QAE@XZ 10025e80 f   asxplay.obj
 0001:00024e90       ??_EPlayerDoneCallback@@UAEPAXI@Z 10025e90 f i asxplay.obj
 0001:00024e90       ??_GPlayerDoneCallback@@UAEPAXI@Z 10025e90 f i asxplay.obj
 0001:00024ec0       ??_GasxCallbackObject@@UAEPAXI@Z 10025ec0 f i asxplay.obj
 0001:00024ec0       ??_EasxCallbackObject@@UAEPAXI@Z 10025ec0 f i asxplay.obj
 0001:00024ef0       ??_GasxPlayer@@UAEPAXI@Z   10025ef0 f i asxplay.obj
 0001:00024ef0       ??_EasxPlayer@@UAEPAXI@Z   10025ef0 f i asxplay.obj
 0001:00024f20       ??_GasxPlayerFile@@QAEPAXI@Z 10025f20 f i asxplay.obj
 0001:00024f50       ?Add@?$TASIArray@VasxPlayerFile@@@@QAEHPAVasxPlayerFile@@@Z 10025f50 f i asxplay.obj
 0001:00024f80       ?AddFile@asxPlayerFileList@@QAEXPBD@Z 10025f80 f   asxplay.obj
 0001:00025040       ?AtEnd@asxPlayerFileList@@QAE_NXZ 10026040 f i asxplay.obj
 0001:00025050       ?BytesToTimescale@asxTimescale@@QAEKKW4asxTIMESCALE@@@Z 10026050 f   asxplay.obj
 0001:00025120       ?CallbackFunction@PlayerDoneCallback@@UAEXXZ 10026120 f i asxplay.obj
 0001:00025130       ?CallbackFunction@asxCallbackObject@@UAEXXZ 10026130 f i asxplay.obj
 0001:00025140       ?Clear@?$TASIArray@VasxPlayerFile@@@@QAEXXZ 10026140 f i asxplay.obj
 0001:00025190       ?Clear@asxPlayerFileList@@QAEXXZ 10026190 f   asxplay.obj
 0001:000251c0       ?Close@asxPlayer@@UAE?AW4asxERROR@@XZ 100261c0 f   asxplay.obj
 0001:000252a0       ?Count@?$TASIArray@VasxPlayerFile@@@@QBEHXZ 100262a0 f i asxplay.obj
 0001:000252b0       ?Enlarge@?$TASIArray@VasxPlayerFile@@@@AAEXXZ 100262b0 f i asxplay.obj
 0001:00025310       ?FormatEnumFromStr@@YA?AW4asxERROR@@PBDPAW4asxAUDIO_FORMAT@@@Z 10026310 f   asxplay.obj
 0001:00025380       ?FreeThreadHandle@asxPlayer@@MAEXXZ 10026380 f   asxplay.obj
 0001:00025390       ?GetCount@asxPlayerFileList@@QAEIXZ 10026390 f   asxplay.obj
 0001:000253a0       ?GetFile@asxPlayerFileList@@QAEPAVasxPlayerFile@@H@Z 100263a0 f i asxplay.obj
 0001:000253c0       ?GetFilename@asxPlayer@@UAE?AW4asxERROR@@PADHPAH@Z 100263c0 f   asxplay.obj
 0001:00025480       ?GetFormatDetails@asxPlayer@@UAE?AW4asxERROR@@PAW4asxAUDIO_FORMAT@@PAH11@Z 10026480 f   asxplay.obj
 0001:00025570       ?GetFormatString@asxPlayer@@UAE?AW4asxERROR@@PAPAD@Z 10026570 f   asxplay.obj
 0001:000255f0       ?GetIndex@asxPlayerFileList@@QAEHXZ 100265f0 f i asxplay.obj
 0001:00025600       ?GetParentSystem@asxControlBase@@QAEPAVasxSystem@@XZ 10026600 f i asxplay.obj
 0001:00025610       ?GetPlaytime@asxPlayerFileList@@QAEIXZ 10026610 f i asxplay.obj
 0001:00025620       ?GetPosition@asxPlayer@@UAE?AW4asxERROR@@W4asxTIMESCALE@@PAK@Z 10026620 f   asxplay.obj
 0001:00025700       ?GetState@asxPlayer@@UAE?AW4asxERROR@@PAW4asxPLAYER_STATE@@@Z 10026700 f   asxplay.obj
 0001:00025730       ?GetTimeScale@asxPlayer@@UAE?AW4asxERROR@@PAM@Z 10026730 f   asxplay.obj
 0001:00025750       ?KillThread@asxPlayer@@MAEXXZ 10026750 f   asxplay.obj
 0001:00025780       ?Next@asxPlayerFileList@@QAE?AW4asxERROR@@XZ 10026780 f   asxplay.obj
 0001:000257e0       ?OnFileDone@asxPlayer@@UAE?AW4asxERROR@@XZ 100267e0 f   asxplay.obj
 0001:000258a0       ?Open@asxPlayer@@UAE?AW4asxERROR@@PBD@Z 100268a0 f   asxplay.obj
 0001:000258c0       ?Open@asxPlayerFile@@QAE?AW4asxERROR@@XZ 100268c0 f   asxplay.obj
 0001:00025a40       ?Open@asxPlayerFileList@@QAE?AW4asxERROR@@XZ 10026a40 f   asxplay.obj
 0001:00025ad0       ?OpenAFile@asxPlayer@@UAE?AW4asxERROR@@XZ 10026ad0 f   asxplay.obj
 0001:00025b60       ?OpenPlaylist@asxPlayer@@UAE?AW4asxERROR@@PAPBDI@Z 10026b60 f   asxplay.obj
 0001:00025cc0       ?Pause@asxPlayer@@UAE?AW4asxERROR@@XZ 10026cc0 f   asxplay.obj
 0001:00025dd0       ?PlaylistStatus@asxPlayer@@UAE?AW4asxERROR@@PAIPAHPAPAD00@Z 10026dd0 f   asxplay.obj
 0001:00025eb0       ?PlaylistWait@asxPlayer@@UAE?AW4asxERROR@@XZ 10026eb0 f   asxplay.obj
 0001:00025f00       ?PreLoad@asxPlayer@@UAE?AW4asxERROR@@W4asxTIMESCALE@@K@Z 10026f00 f   asxplay.obj
 0001:00026100       ?Prefill@asxPlayer@@MAE?AW4asxERROR@@XZ 10027100 f   asxplay.obj
 0001:00026150       ?RegisterCallback@asxPlayer@@UAE?AW4asxERROR@@P6AXPAXW4asxPLAYER_FLAGS@@0@Z10@Z 10027150 f   asxplay.obj
 0001:00026170       ?Reopen@asxPlayerFile@@QAE?AW4asxERROR@@XZ 10027170 f   asxplay.obj
 0001:000261a0       ?SetFile@asxPlayerFileList@@QAEXH@Z 100271a0 f   asxplay.obj
 0001:000261d0       ?SetFormat@asxTimescale@@QAEXKKKK@Z 100271d0 f i asxplay.obj
 0001:00026220       ?SetPosition@asxPlayer@@UAE?AW4asxERROR@@W4asxTIMESCALE@@K@Z 10027220 f   asxplay.obj
 0001:00026250       ?SetState@asxPlayer@@MAE_NW4asxPLAYER_STATE@@@Z 10027250 f   asxplay.obj
 0001:00026370       ?SetTimeScale@asxPlayer@@UAE?AW4asxERROR@@M@Z 10027370 f   asxplay.obj
 0001:00026390       ?Start@asxPlayer@@UAE?AW4asxERROR@@XZ 10027390 f   asxplay.obj
 0001:00026520       ?StartThread@asxPlayer@@MAEXXZ 10027520 f   asxplay.obj
 0001:00026540       ?Stop@asxPlayer@@UAE?AW4asxERROR@@XZ 10027540 f   asxplay.obj
 0001:000266a0       ?Stop@asxPlayerFileList@@QAEXXZ 100276a0 f i asxplay.obj
 0001:000266b0       ?TimescaleToBytes@asxTimescale@@QAEKKW4asxTIMESCALE@@@Z 100276b0 f   asxplay.obj
 0001:000267b0       ?TranslateTWavError@@YA?AW4asxERROR@@J_N@Z 100277b0 f   asxplay.obj
 0001:00026860       ?Unplayable@asxPlayerFileList@@QAEXXZ 10027860 f   asxplay.obj
 0001:000268d0       ?Wait@asxPlayer@@UAE?AW4asxERROR@@XZ 100278d0 f   asxplay.obj
 0001:00026980       ?WaitForState@asxPlayer@@MAE_NW4asxPLAYER_STATE@@@Z 10027980 f   asxplay.obj
 0001:000269e0       ?asxPlayerThreadProc@@YGKPAX@Z 100279e0 f   asxplay.obj
 0001:00026a00       ??0?$TASIArray@W4asxAUDIO_FORMAT@@@@QAE@XZ 10027a00 f i asxrec.obj
 0001:00026a20       ??0asxRecorder@@QAE@PAVasxSubSystem@@PAVasxNode@@1J@Z 10027a20 f   asxrec.obj
 0001:00026aa0       ??1?$TASIArray@W4asxAUDIO_FORMAT@@@@QAE@XZ 10027aa0 f i asxrec.obj
 0001:00026af0       ??1asxRecorder@@UAE@XZ     10027af0 f   asxrec.obj
 0001:00026b70       ??A?$TASIArray@W4asxAUDIO_FORMAT@@@@QBEPAW4asxAUDIO_FORMAT@@H@Z 10027b70 f i asxrec.obj
 0001:00026b90       ??_GasxRecorder@@UAEPAXI@Z 10027b90 f i asxrec.obj
 0001:00026b90       ??_EasxRecorder@@UAEPAXI@Z 10027b90 f i asxrec.obj
 0001:00026bc0       ?Close@asxRecorder@@UAE?AW4asxERROR@@XZ 10027bc0 f   asxrec.obj
 0001:00026c20       ?Count@?$TASIArray@W4asxAUDIO_FORMAT@@@@QBEHXZ 10027c20 f i asxrec.obj
 0001:00026c30       ?CreateFileA@asxRecorder@@MAE?AW4asxERROR@@XZ 10027c30 f   asxrec.obj
 0001:00026f50       ?EnumerateFormat@asxRecorder@@QAE?AW4asxERROR@@HPAW4asxAUDIO_FORMAT@@PAH@Z 10027f50 f   asxrec.obj
 0001:00026fa0       ?FreeFileAndName@asxRecorder@@IAEXXZ 10027fa0 f   asxrec.obj
 0001:00026fe0       ?FreeThreadHandle@asxRecorder@@MAEXXZ 10027fe0 f   asxrec.obj
 0001:00027000       ?GetFilename@asxRecorder@@UAE?AW4asxERROR@@PADHPAH@Z 10028000 f   asxrec.obj
 0001:00027090       ?GetPosition@asxRecorder@@UAE?AW4asxERROR@@W4asxTIMESCALE@@PAK@Z 10028090 f   asxrec.obj
 0001:00027160       ?GetState@asxRecorder@@UAE?AW4asxERROR@@PAW4asxRECORDER_STATE@@@Z 10028160 f   asxrec.obj
 0001:000271b0       ?Open@asxRecorder@@UAE?AW4asxERROR@@PBDW4asxFILE_FORMAT@@W4asxFILE_MODE@@HW4asxAUDIO_FORMAT@@JJW4asxRECORD_MODE@@@Z 100281b0 f   asxrec.obj
 0001:00027330       ?Pause@asxRecorder@@UAE?AW4asxERROR@@XZ 10028330 f   asxrec.obj
 0001:000273d0       ?RecreateFile@asxRecorder@@IAE?AW4asxERROR@@XZ 100283d0 f   asxrec.obj
 0001:00027400       ?SetInputFormat@asxRecorder@@MAE?AW4asxERROR@@W4asxFILE_FORMAT@@HW4asxAUDIO_FORMAT@@JJW4asxRECORD_MODE@@@Z 10028400 f   asxrec.obj
 0001:00027510       ?SetState@asxRecorder@@MAE?AW4asxERROR@@W4asxRECORDER_STATE@@@Z 10028510 f   asxrec.obj
 0001:00027590       ?SignalThread@asxRecorder@@MAEXXZ 10028590 f   asxrec.obj
 0001:000275b0       ?Start@asxRecorder@@UAE?AW4asxERROR@@XZ 100285b0 f   asxrec.obj
 0001:00027680       ?StartThread@asxRecorder@@MAEXXZ 10028680 f   asxrec.obj
 0001:000276b0       ?StateName@asxRecorder@@IAEPBDW4asxRECORDER_STATE@@@Z 100286b0 f   asxrec.obj
 0001:00027720       ?Stop@asxRecorder@@UAE?AW4asxERROR@@XZ 10028720 f   asxrec.obj
 0001:000277d0       ?WaitForState@asxRecorder@@MAE?AW4asxERROR@@W4asxRECORDER_STATE@@@Z 100287d0 f   asxrec.obj
 0001:00027870       ?asxRecorderThreadProc@@YGKPAX@Z 10028870 f   asxrec.obj
 0001:00027890       ??0asiIpAddr@@QAE@EEEE@Z   10028890 f i asxsnmp.obj
 0001:000278b0       ??0asiIpAddr@@QAE@I@Z      100288b0 f i asxsnmp.obj
 0001:000278e0       ??0asiIpAddr@@QAE@PBD@Z    100288e0 f i asxsnmp.obj
 0001:00027900       ??0asiMacAddr@@QAE@PBD@Z   10028900 f i asxsnmp.obj
 0001:00027920       ??0asiMacAddr@@QAE@XZ      10028920 f i asxsnmp.obj
 0001:00027930       ??0asxAdapterSNMP@@QAE@PAVasxSystem@@PADPBD2PAVSnmpSession@@@Z 10028930 f   asxsnmp.obj
 0001:00027b60       ??0asxCobranetRxSNMP@@QAE@PAVasxSubSystem@@PAVasxNode@@1PAVCobraNetNode@@H@Z 10028b60 f i asxsnmp.obj
 0001:00027ba0       ??0asxCobranetSNMP@@QAE@PAVasxSubSystem@@PAVasxNode@@1PAVCobraNetNode@@PBD@Z 10028ba0 f   asxsnmp.obj
 0001:00027c90       ??0asxCobranetTxSNMP@@QAE@PAVasxSubSystem@@PAVasxNode@@1PAVCobraNetNode@@H@Z 10028c90 f i asxsnmp.obj
 0001:00027cd0       ??0asxCobranetUnreachableSNMP@@QAE@PAVasxSubSystem@@PAVasxNode@@1PBD2@Z 10028cd0 f   asxsnmp.obj
 0001:00027d30       ??0asxMixerScannerSNMP@@QAE@PAVasxSubSystem@@PAVCobraNetNode@@PBD@Z 10028d30 f i asxsnmp.obj
 0001:00027d70       ??0asxMixerScannerUnreachableSNMP@@QAE@PAVasxSubSystem@@PBD1@Z 10028d70 f   asxsnmp.obj
 0001:00027db0       ??0asxSubSystemSNMP@@QAE@PAVasxSystem@@@Z 10028db0 f   asxsnmp.obj
 0001:00027f60       ??1asxAdapterSNMP@@UAE@XZ  10028f60 f   asxsnmp.obj
 0001:00027fd0       ??1asxCobranetRxSNMP@@UAE@XZ 10028fd0 f i asxsnmp.obj
 0001:00027ff0       ??1asxCobranetSNMP@@UAE@XZ 10028ff0 f i asxsnmp.obj
 0001:00028010       ??1asxCobranetTxSNMP@@UAE@XZ 10029010 f i asxsnmp.obj
 0001:00028030       ??1asxCobranetUnreachableSNMP@@UAE@XZ 10029030 f i asxsnmp.obj
 0001:00028050       ??1asxMixerScannerSNMP@@UAE@XZ 10029050 f i asxsnmp.obj
 0001:00028060       ??1asxMixerScannerUnreachableSNMP@@UAE@XZ 10029060 f i asxsnmp.obj
 0001:00028070       ??1asxSubSystemSNMP@@UAE@XZ 10029070 f   asxsnmp.obj
 0001:00028160       ??8asiIpAddr@@QBE_NABV0@@Z 10029160 f i asxsnmp.obj
 0001:00028190       ??9asiIpAddr@@QBE_NABV0@@Z 10029190 f i asxsnmp.obj
 0001:000281e0       ??AasiIpAddr@@QAEAAEH@Z    100291e0 f i asxsnmp.obj
 0001:00028210       ??AasiMacAddr@@QAEAAEH@Z   10029210 f i asxsnmp.obj
 0001:00028260       ??BasiIpAddr@@QBEIXZ       10029260 f i asxsnmp.obj
 0001:00028270       ??_GCobraNetNode@@QAEPAXI@Z 10029270 f i asxsnmp.obj
 0001:000282a0       ??_GSnmpSession@@QAEPAXI@Z 100292a0 f i asxsnmp.obj
 0001:000282d0       ??_GasxAdapterSNMP@@UAEPAXI@Z 100292d0 f i asxsnmp.obj
 0001:000282d0       ??_EasxAdapterSNMP@@UAEPAXI@Z 100292d0 f i asxsnmp.obj
 0001:00028300       ??_EasxCobranetRxSNMP@@UAEPAXI@Z 10029300 f i asxsnmp.obj
 0001:00028300       ??_GasxCobranetRxSNMP@@UAEPAXI@Z 10029300 f i asxsnmp.obj
 0001:00028340       ??_GasxCobranetSNMP@@UAEPAXI@Z 10029340 f i asxsnmp.obj
 0001:00028340       ??_EasxCobranetSNMP@@UAEPAXI@Z 10029340 f i asxsnmp.obj
 0001:00028380       ??_EasxCobranetTxSNMP@@UAEPAXI@Z 10029380 f i asxsnmp.obj
 0001:00028380       ??_GasxCobranetTxSNMP@@UAEPAXI@Z 10029380 f i asxsnmp.obj
 0001:000283c0       ??_EasxCobranetUnreachableSNMP@@UAEPAXI@Z 100293c0 f i asxsnmp.obj
 0001:000283c0       ??_GasxCobranetUnreachableSNMP@@UAEPAXI@Z 100293c0 f i asxsnmp.obj
 0001:00028400       ??_GasxMixerScannerSNMP@@UAEPAXI@Z 10029400 f i asxsnmp.obj
 0001:00028400       ??_EasxMixerScannerSNMP@@UAEPAXI@Z 10029400 f i asxsnmp.obj
 0001:00028430       ??_EasxMixerScannerUnreachableSNMP@@UAEPAXI@Z 10029430 f i asxsnmp.obj
 0001:00028430       ??_GasxMixerScannerUnreachableSNMP@@UAEPAXI@Z 10029430 f i asxsnmp.obj
 0001:00028460       ??_GasxSubSystemSNMP@@UAEPAXI@Z 10029460 f i asxsnmp.obj
 0001:00028460       ??_EasxSubSystemSNMP@@UAEPAXI@Z 10029460 f i asxsnmp.obj
 0001:00028490       ?CheckSubSystems@asxAdapterSNMP@@UAE?AW4asxERROR@@PAI0@Z 10029490 f   asxsnmp.obj
 0001:000284b0       ?GetBundle@asxCobranetRxSNMP@@UAE?AW4asxERROR@@PAI@Z 100294b0 f   asxsnmp.obj
 0001:000284e0       ?GetBundle@asxCobranetTxSNMP@@UAE?AW4asxERROR@@PAI@Z 100294e0 f   asxsnmp.obj
 0001:00028510       ?GetCNNode@asxAdapterSNMP@@QAEPAVCobraNetNode@@XZ 10029510 f i asxsnmp.obj
 0001:00028520       ?GetChannelCount@asxCobranetTxSNMP@@UAE?AW4asxERROR@@PAI@Z 10029520 f   asxsnmp.obj
 0001:00028550       ?GetChannelMap@asxCobranetRxSNMP@@UAE?AW4asxERROR@@QAI@Z 10029550 f   asxsnmp.obj
 0001:000285a0       ?GetChannelMap@asxCobranetTxSNMP@@UAE?AW4asxERROR@@QAI@Z 100295a0 f   asxsnmp.obj
 0001:000285f0       ?GetConductorPriority@CobraNetNode@@QAEHPAI@Z 100295f0 f i asxsnmp.obj
 0001:00028610       ?GetConductorPriority@asxCobranetSNMP@@UAE?AW4asxERROR@@PAI@Z 10029610 f   asxsnmp.obj
 0001:00028630       ?GetConductorStatus@CobraNetNode@@QAEHPAI@Z 10029630 f i asxsnmp.obj
 0001:00028650       ?GetConductorStatus@asxCobranetSNMP@@UAE?AW4asxERROR@@PAI@Z 10029650 f   asxsnmp.obj
 0001:00028670       ?GetDescription@asxCobranetSNMP@@UAE?AW4asxERROR@@PADH@Z 10029670 f   asxsnmp.obj
 0001:000286a0       ?GetDescription@asxCobranetUnreachableSNMP@@UAE?AW4asxERROR@@PADH@Z 100296a0 f   asxsnmp.obj
 0001:000286e0       ?GetDescriptionString@CobraNetNode@@QAEHPADHPAH@Z 100296e0 f i asxsnmp.obj
 0001:00028700       ?GetDisplayError@CobraNetNode@@QAEHPAI@Z 10029700 f i asxsnmp.obj
 0001:00028720       ?GetErrorCount@CobraNetNode@@QAEHPAI@Z 10029720 f i asxsnmp.obj
 0001:00028740       ?GetErrorInfo@asxCobranetSNMP@@UAE?AW4asxERROR@@PAI00@Z 10029740 f   asxsnmp.obj
 0001:000287a0       ?GetFirmwareRevision@asxCobranetSNMP@@UAE?AW4asxERROR@@PAD@Z 100297a0 f   asxsnmp.obj
 0001:000287b0       ?GetFormat@asxCobranetTxSNMP@@UAE?AW4asxERROR@@PAW4asxAUDIO_FORMAT@@@Z 100297b0 f   asxsnmp.obj
 0001:00028800       ?GetIPAddress@asxCobranetSNMP@@UAE?AW4asxERROR@@PAI@Z 10029800 f   asxsnmp.obj
 0001:00028870       ?GetIPAddress@asxCobranetUnreachableSNMP@@UAE?AW4asxERROR@@PAI@Z 10029870 f   asxsnmp.obj
 0001:000288a0       ?GetIpAddrString@CobraNetNode@@QAEHPADHPAH@Z 100298a0 f i asxsnmp.obj
 0001:000288e0       ?GetIpAddress@asxAdapterSNMP@@UAE?AW4asxERROR@@PAD@Z 100298e0 f   asxsnmp.obj
 0001:00028a30       ?GetIpAssignStatus@asxSubSystemSNMP@@QAEHPBD@Z 10029a30 f   asxsnmp.obj
 0001:00028a70       ?GetLastError@CobraNetNode@@QAEHPAI@Z 10029a70 f i asxsnmp.obj
 0001:00028a90       ?GetLatencyAndSampleRate@asxCobranetSNMP@@UAE?AW4asxERROR@@PAW4asxCOBRANET_LATENCY@@PAW4asxSAMPLE_RATE@@@Z 10029a90 f   asxsnmp.obj
 0001:00028ad0       ?GetLocation@asxCobranetSNMP@@UAE?AW4asxERROR@@PADH@Z 10029ad0 f   asxsnmp.obj
 0001:00028b00       ?GetLocationString@CobraNetNode@@QAEHPADHPAH@Z 10029b00 f i asxsnmp.obj
 0001:00028b20       ?GetMACAddress@asxCobranetSNMP@@UAE?AW4asxERROR@@PAIPAG@Z 10029b20 f   asxsnmp.obj
 0001:00028c00       ?GetMACAddress@asxCobranetUnreachableSNMP@@UAE?AW4asxERROR@@PAIPAG@Z 10029c00 f   asxsnmp.obj
 0001:00028c60       ?GetMacAddrString@CobraNetNode@@QAEHPADHPAH@Z 10029c60 f i asxsnmp.obj
 0001:00028ca0       ?GetMacAddress@asxAdapterSNMP@@UAE?AW4asxERROR@@PAD@Z 10029ca0 f   asxsnmp.obj
 0001:00028cd0       ?GetMinimumDelay@asxCobranetRxSNMP@@UAE?AW4asxERROR@@PAI@Z 10029cd0 f   asxsnmp.obj
 0001:00028ce0       ?GetModeRateControl@CobraNetNode@@QAEHPAJ@Z 10029ce0 f i asxsnmp.obj
 0001:00028d00       ?GetName@asxCobranetSNMP@@UAE?AW4asxERROR@@PADH@Z 10029d00 f   asxsnmp.obj
 0001:00028d30       ?GetNameString@CobraNetNode@@QAEHPADHPAH@Z 10029d30 f i asxsnmp.obj
 0001:00028d50       ?GetNumReceivers@CobraNetNode@@QAEHXZ 10029d50 f i asxsnmp.obj
 0001:00028d60       ?GetNumTransmitters@CobraNetNode@@QAEHXZ 10029d60 f i asxsnmp.obj
 0001:00028d70       ?GetPcapError@asxSubSystemSNMP@@QAE?AW4asxERROR@@XZ 10029d70 f   asxsnmp.obj
 0001:00028dd0       ?GetPersistence@CobraNetNode@@QAEHPAH@Z 10029dd0 f i asxsnmp.obj
 0001:00028df0       ?GetPersistence@asxCobranetSNMP@@UAE?AW4asxERROR@@PAI@Z 10029df0 f   asxsnmp.obj
 0001:00028e20       ?GetPriority@asxCobranetRx@@QAEHXZ 10029e20 f i asxsnmp.obj
 0001:00028e30       ?GetPriority@asxCobranetTx@@QAEHXZ 10029e30 f i asxsnmp.obj
 0001:00028e40       ?GetRxBundle@CobraNetNode@@QAEHHPAH@Z 10029e40 f i asxsnmp.obj
 0001:00028e60       ?GetRxDelay@CobraNetNode@@QAEHHPAH@Z 10029e60 f i asxsnmp.obj
 0001:00028e80       ?GetRxDropouts@CobraNetNode@@QAEHHPAH@Z 10029e80 f i asxsnmp.obj
 0001:00028ea0       ?GetRxStatus@CobraNetNode@@QAEHHPAI@Z 10029ea0 f i asxsnmp.obj
 0001:00028ec0       ?GetRxSubFormat@CobraNetNode@@QAEHHHPAI@Z 10029ec0 f i asxsnmp.obj
 0001:00028ee0       ?GetRxSubmap@CobraNetNode@@QAEHHHPAH@Z 10029ee0 f i asxsnmp.obj
 0001:00028f00       ?GetSerialBaud@CobraNetNode@@QAEHPAI@Z 10029f00 f i asxsnmp.obj
 0001:00028f20       ?GetSerialConfig@asxCobranetSNMP@@UAE?AW4asxERROR@@PAI0QADPAH1@Z 10029f20 f   asxsnmp.obj
 0001:00028fc0       ?GetSerialEnable@asxCobranetSNMP@@UAE?AW4asxERROR@@PAH@Z 10029fc0 f   asxsnmp.obj
 0001:00029010       ?GetSerialFormat@CobraNetNode@@QAEHPAI@Z 1002a010 f i asxsnmp.obj
 0001:00029030       ?GetSerialPPeriod@CobraNetNode@@QAEHPAI@Z 1002a030 f i asxsnmp.obj
 0001:00029050       ?GetSerialRxMAC@CobraNetNode@@QAEHPAD@Z 1002a050 f i asxsnmp.obj
 0001:00029070       ?GetSerialTxMAC@CobraNetNode@@QAEHPAD@Z 1002a070 f i asxsnmp.obj
 0001:00029090       ?GetStaticIPAddress@asxCobranetSNMP@@UAE?AW4asxERROR@@PAI@Z 1002a090 f   asxsnmp.obj
 0001:000290c0       ?GetStaticIpAddr@CobraNetNode@@QAEHPAI@Z 1002a0c0 f i asxsnmp.obj
 0001:00029130       ?GetStatus@asxCobranetRxSNMP@@UAE?AW4asxERROR@@PAI00QAI@Z 1002a130 f   asxsnmp.obj
 0001:000291e0       ?GetStatus@asxCobranetTxSNMP@@UAE?AW4asxERROR@@PAI00@Z 1002a1e0 f   asxsnmp.obj
 0001:00029250       ?GetTxBundle@CobraNetNode@@QAEHHPAH@Z 1002a250 f i asxsnmp.obj
 0001:00029270       ?GetTxDropouts@CobraNetNode@@QAEHHPAH@Z 1002a270 f i asxsnmp.obj
 0001:00029290       ?GetTxMaxUnicast@CobraNetNode@@QAEHHPAH@Z 1002a290 f i asxsnmp.obj
 0001:000292b0       ?GetTxPosition@CobraNetNode@@QAEHHPAH@Z 1002a2b0 f i asxsnmp.obj
 0001:000292d0       ?GetTxReceivers@CobraNetNode@@QAEHHPAH@Z 1002a2d0 f i asxsnmp.obj
 0001:000292f0       ?GetTxSubCount@CobraNetNode@@QAEHHPAH@Z 1002a2f0 f i asxsnmp.obj
 0001:00029310       ?GetTxSubFormat@CobraNetNode@@QAEHHHPAI@Z 1002a310 f i asxsnmp.obj
 0001:00029330       ?GetTxSubmap@CobraNetNode@@QAEHHHPAH@Z 1002a330 f i asxsnmp.obj
 0001:00029350       ?GetTxUnicastMode@CobraNetNode@@QAEHHPAH@Z 1002a350 f i asxsnmp.obj
 0001:00029370       ?GetUnicastMode@asxCobranetTxSNMP@@UAE?AW4asxERROR@@PAI0@Z 1002a370 f   asxsnmp.obj
 0001:000293c0       ?LogEvent@@YAXW4EventType@NotificationEvent@@PBVasiMacAddr@@PBVasiIpAddr@@@Z 1002a3c0 f   asxsnmp.obj
 0001:00029470       ?NewIpAddress@CobraNetNode@@QAEXPBD@Z 1002a470 f i asxsnmp.obj
 0001:00029500       ?NewIpAddress@asxAdapterSNMP@@QAEXPBD@Z 1002a500 f   asxsnmp.obj
 0001:000296e0       ?ReScan@asxSubSystemSNMP@@UAEXXZ 1002a6e0 f   asxsnmp.obj
 0001:00029c00       ?ReadProperty@asxAdapterSNMP@@UAE?AW4asxERROR@@HPAG0@Z 1002ac00 f   asxsnmp.obj
 0001:00029c30       ?Replace@asxCobranetRxContainer@@QAEXAAVasxCobranetRx@@@Z 1002ac30 f i asxsnmp.obj
 0001:00029ca0       ?Replace@asxCobranetTxContainer@@QAEXAAVasxCobranetTx@@@Z 1002aca0 f i asxsnmp.obj
 0001:00029d10       ?Scan@asxMixerScannerSNMP@@UAEXPAVasxMixer@@@Z 1002ad10 f   asxsnmp.obj
 0001:0002a390       ?Scan@asxMixerScannerUnreachableSNMP@@UAEXPAVasxMixer@@@Z 1002b390 f   asxsnmp.obj
 0001:0002a510       ?Scan@asxSubSystemSNMP@@UAEXXZ 1002b510 f   asxsnmp.obj
 0001:0002a520       ?SetAutoAssignRange@AsiAutoassignIpTracker@@QAEXPBVasiIpAddr@@0@Z 1002b520 f i asxsnmp.obj
 0001:0002a540       ?SetBundle@asxCobranetRxSNMP@@UAE?AW4asxERROR@@I@Z 1002b540 f   asxsnmp.obj
 0001:0002a560       ?SetBundle@asxCobranetTxSNMP@@UAE?AW4asxERROR@@I@Z 1002b560 f   asxsnmp.obj
 0001:0002a590       ?SetChannelCount@asxCobranetTxSNMP@@UAE?AW4asxERROR@@I@Z 1002b590 f   asxsnmp.obj
 0001:0002a5b0       ?SetChannelMap@asxCobranetRxSNMP@@UAE?AW4asxERROR@@QBI@Z 1002b5b0 f   asxsnmp.obj
 0001:0002a5f0       ?SetChannelMap@asxCobranetTxSNMP@@UAE?AW4asxERROR@@QBI@Z 1002b5f0 f   asxsnmp.obj
 0001:0002a640       ?SetConductorPriority@CobraNetNode@@QAEHI@Z 1002b640 f i asxsnmp.obj
 0001:0002a660       ?SetConductorPriority@asxCobranetSNMP@@UAE?AW4asxERROR@@I@Z 1002b660 f   asxsnmp.obj
 0001:0002a680       ?SetFormat@asxCobranetTxSNMP@@UAE?AW4asxERROR@@W4asxAUDIO_FORMAT@@@Z 1002b680 f   asxsnmp.obj
 0001:0002a6d0       ?SetIPAddress@asxCobranetSNMP@@UAE?AW4asxERROR@@I@Z 1002b6d0 f   asxsnmp.obj
 0001:0002a740       ?SetIPAddress@asxCobranetUnreachableSNMP@@UAE?AW4asxERROR@@I@Z 1002b740 f   asxsnmp.obj
 0001:0002a7a0       ?SetIpAddr@CobraNetNode@@QAEHI@Z 1002b7a0 f i asxsnmp.obj
 0001:0002a870       ?SetIpAddressForMac@asxSubSystemSNMP@@QAEHPBD0@Z 1002b870 f   asxsnmp.obj
 0001:0002a920       ?SetLatencyAndSampleRate@asxCobranetSNMP@@UAE?AW4asxERROR@@W4asxCOBRANET_LATENCY@@W4asxSAMPLE_RATE@@@Z 1002b920 f   asxsnmp.obj
 0001:0002a9b0       ?SetLocation@asxCobranetSNMP@@UAE?AW4asxERROR@@PBD@Z 1002b9b0 f   asxsnmp.obj
 0001:0002a9d0       ?SetLocationString@CobraNetNode@@QAEHPBD@Z 1002b9d0 f i asxsnmp.obj
 0001:0002a9f0       ?SetMinimumDelay@asxCobranetRxSNMP@@UAE?AW4asxERROR@@I@Z 1002b9f0 f   asxsnmp.obj
 0001:0002aa00       ?SetModeRateControl@CobraNetNode@@QAEHJ@Z 1002ba00 f i asxsnmp.obj
 0001:0002aa20       ?SetName@asxCobranetSNMP@@UAE?AW4asxERROR@@PBD@Z 1002ba20 f   asxsnmp.obj
 0001:0002aa40       ?SetNameString@CobraNetNode@@QAEHPBD@Z 1002ba40 f i asxsnmp.obj
 0001:0002aa60       ?SetPersistence@CobraNetNode@@QAEHH@Z 1002ba60 f i asxsnmp.obj
 0001:0002aa80       ?SetPersistence@asxCobranetSNMP@@UAE?AW4asxERROR@@I@Z 1002ba80 f   asxsnmp.obj
 0001:0002aaa0       ?SetPresent@asxAdapterSNMP@@QAEX_N@Z 1002baa0 f i asxsnmp.obj
 0001:0002aab0       ?SetRxBundle@CobraNetNode@@QAEHHH@Z 1002bab0 f i asxsnmp.obj
 0001:0002aad0       ?SetRxSubmap@CobraNetNode@@QAEHHHH@Z 1002bad0 f i asxsnmp.obj
 0001:0002aaf0       ?SetSerialBaud@CobraNetNode@@QAEHI@Z 1002baf0 f i asxsnmp.obj
 0001:0002ab10       ?SetSerialConfig@asxCobranetSNMP@@UAE?AW4asxERROR@@IIQBDH0@Z 1002bb10 f   asxsnmp.obj
 0001:0002abc0       ?SetSerialEnable@asxCobranetSNMP@@UAE?AW4asxERROR@@H@Z 1002bbc0 f   asxsnmp.obj
 0001:0002ac30       ?SetSerialFormat@CobraNetNode@@QAEHI@Z 1002bc30 f i asxsnmp.obj
 0001:0002ac50       ?SetSerialPPeriod@CobraNetNode@@QAEHI@Z 1002bc50 f i asxsnmp.obj
 0001:0002ac70       ?SetSerialRxMAC@CobraNetNode@@QAEHPBD@Z 1002bc70 f i asxsnmp.obj
 0001:0002ac90       ?SetSerialTxMAC@CobraNetNode@@QAEHPBD@Z 1002bc90 f i asxsnmp.obj
 0001:0002acb0       ?SetSnmpCacheMode@CobraNetNode@@QAEXW4snmpCacheMode@1@@Z 1002bcb0 f i asxsnmp.obj
 0001:0002ace0       ?SetStaticIPAddress@asxCobranetSNMP@@UAE?AW4asxERROR@@I@Z 1002bce0 f   asxsnmp.obj
 0001:0002ad00       ?SetStaticIpAddr@CobraNetNode@@QAEHI@Z 1002bd00 f i asxsnmp.obj
 0001:0002add0       ?SetTxBundle@CobraNetNode@@QAEHHH@Z 1002bdd0 f i asxsnmp.obj
 0001:0002adf0       ?SetTxMaxUnicast@CobraNetNode@@QAEHHH@Z 1002bdf0 f i asxsnmp.obj
 0001:0002ae10       ?SetTxSubCount@CobraNetNode@@QAEHHH@Z 1002be10 f i asxsnmp.obj
 0001:0002ae30       ?SetTxSubFormat@CobraNetNode@@QAEHHHI@Z 1002be30 f i asxsnmp.obj
 0001:0002ae50       ?SetTxSubmap@CobraNetNode@@QAEHHHH@Z 1002be50 f i asxsnmp.obj
 0001:0002ae70       ?SetTxUnicastMode@CobraNetNode@@QAEHHH@Z 1002be70 f i asxsnmp.obj
 0001:0002ae90       ?SetUnicastMode@asxCobranetTxSNMP@@UAE?AW4asxERROR@@II@Z 1002be90 f   asxsnmp.obj
 0001:0002aed0       ?fromstring@asiIpAddr@@QAE_NPBD@Z 1002bed0 f i asxsnmp.obj
 0001:0002af70       ?fromstring@asiMacAddr@@QAE_NPBD@Z 1002bf70 f i asxsnmp.obj
 0001:0002b070       ?getByte@asiIpAddr@@QBEEH@Z 1002c070 f i asxsnmp.obj
 0001:0002b0a0       ?strstr@@YAPADPADPBD@Z     1002c0a0 f i asxsnmp.obj
 0001:0002b0b0       ?tostring@asiIpAddr@@QBEXPAD@Z 1002c0b0 f i asxsnmp.obj
 0001:0002b180       _ASXSTRING_EnumToString    1002c180 f   asxstring.obj
 0001:0002b250       _ASXSTRING_StringToEnum    1002c250 f   asxstring.obj
 0001:0002b2e0       ??0asxBlockTR800OptoMode@@QAE@PAVasxSubSystem@@PAVasxTR800helperthread@@PAVasxNode@@2@Z 1002c2e0 f   asxtr800.obj
 0001:0002b440       ??0asxBlockTR800Status@@QAE@PAVasxSubSystem@@PAVasxNode@@1_N@Z 1002c440 f   asxtr800.obj
 0001:0002b550       ??0asxControlBaseTR800@@QAE@PAVasxTR800helperthread@@@Z 1002c550 f i asxtr800.obj
 0001:0002b560       ??0asxGpioTR800@@QAE@PAVasxSubSystem@@PAVasxTR800helperthread@@PAVasxNode@@2@Z 1002c560 f   asxtr800.obj
 0001:0002b5a0       ??0asxLevelTR800@@QAE@PAVasxSubSystem@@PAVasxTR800helperthread@@PAVasxNode@@2@Z 1002c5a0 f   asxtr800.obj
 0001:0002b660       ??0asxMeterTR800@@QAE@PAVasxSubSystem@@PAVasxTR800helperthread@@PAVasxNode@@2@Z 1002c660 f   asxtr800.obj
 0001:0002b6b0       ??0asxTR800helperthread@@QAE@PAVCobraNetNode@@@Z 1002c6b0 f   asxtr800.obj
 0001:0002b730       ??1asxBlockTR800OptoMode@@UAE@XZ 1002c730 f i asxtr800.obj
 0001:0002b7a0       ??1asxBlockTR800Status@@UAE@XZ 1002c7a0 f i asxtr800.obj
 0001:0002b810       ??1asxControlBaseTR800@@QAE@XZ 1002c810 f i asxtr800.obj
 0001:0002b820       ??1asxGpioTR800@@UAE@XZ    1002c820 f i asxtr800.obj
 0001:0002b840       ??1asxLevelTR800@@UAE@XZ   1002c840 f i asxtr800.obj
 0001:0002b860       ??1asxMeterTR800@@UAE@XZ   1002c860 f   asxtr800.obj
 0001:0002b8b0       ??1asxTR800helperthread@@QAE@XZ 1002c8b0 f   asxtr800.obj
 0001:0002b900       ??_EasxBlockTR800OptoMode@@UAEPAXI@Z 1002c900 f i asxtr800.obj
 0001:0002b900       ??_GasxBlockTR800OptoMode@@UAEPAXI@Z 1002c900 f i asxtr800.obj
 0001:0002b980       ??_EasxBlockTR800Status@@UAEPAXI@Z 1002c980 f i asxtr800.obj
 0001:0002b980       ??_GasxBlockTR800Status@@UAEPAXI@Z 1002c980 f i asxtr800.obj
 0001:0002ba00       ??_GasxGpioTR800@@UAEPAXI@Z 1002ca00 f i asxtr800.obj
 0001:0002ba00       ??_EasxGpioTR800@@UAEPAXI@Z 1002ca00 f i asxtr800.obj
 0001:0002ba40       ??_GasxLevelTR800@@UAEPAXI@Z 1002ca40 f i asxtr800.obj
 0001:0002ba40       ??_EasxLevelTR800@@UAEPAXI@Z 1002ca40 f i asxtr800.obj
 0001:0002ba80       ??_EasxMeterTR800@@UAEPAXI@Z 1002ca80 f i asxtr800.obj
 0001:0002ba80       ??_GasxMeterTR800@@UAEPAXI@Z 1002ca80 f i asxtr800.obj
 0001:0002bab0       ??_GasxTR800helperthread@@QAEPAXI@Z 1002cab0 f i asxtr800.obj
 0001:0002bae0       ?Get@asxBlockTR800OptoMode@@UAE?AW4asxERROR@@IPAUasxParameterValue@@@Z 1002cae0 f   asxtr800.obj
 0001:0002bb30       ?Get@asxBlockTR800Status@@UAE?AW4asxERROR@@IPAUasxParameterValue@@@Z 1002cb30 f   asxtr800.obj
 0001:0002bb70       ?Get@asxLevelTR800@@UAE?AW4asxERROR@@PAM@Z 1002cb70 f   asxtr800.obj
 0001:0002bb90       ?GetAudioMeter@CobraNetNode@@QAEHIPAI@Z 1002cb90 f i asxtr800.obj
 0001:0002bbb0       ?GetChannels@asxMeterTR800@@UAE?AW4asxERROR@@PAH@Z 1002cbb0 f   asxtr800.obj
 0001:0002bbd0       ?GetCobraNetMeter@asxTR800helperthread@@QAEII@Z 1002cbd0 f   asxtr800.obj
 0001:0002bc00       ?GetGpioRelay@asxTR800helperthread@@QAEII@Z 1002cc00 f   asxtr800.obj
 0001:0002bc20       ?GetInfo@asxBlockTR800OptoMode@@UAE?AW4asxERROR@@PADIPAI@Z 1002cc20 f   asxtr800.obj
 0001:0002bc60       ?GetInfo@asxBlockTR800Status@@UAE?AW4asxERROR@@PADIPAI@Z 1002cc60 f   asxtr800.obj
 0001:0002bc90       ?GetMicGain@asxTR800helperthread@@QAEII@Z 1002cc90 f   asxtr800.obj
 0001:0002bcc0       ?GetOptoAction@asxTR800helperthread@@QAEII@Z 1002ccc0 f   asxtr800.obj
 0001:0002bce0       ?GetPeak@asxMeterTR800@@UAE?AW4asxERROR@@PAMH@Z 1002cce0 f   asxtr800.obj
 0001:0002bd40       ?GetProperties@asxGpioTR800@@UAE?AW4asxERROR@@PAH0@Z 1002cd40 f   asxtr800.obj
 0001:0002bd60       ?GetRMS@asxMeterTR800@@UAE?AW4asxERROR@@PAMH@Z 1002cd60 f   asxtr800.obj
 0001:0002bd70       ?GetRange@asxLevelTR800@@UAE?AW4asxERROR@@PAM00@Z 1002cd70 f   asxtr800.obj
 0001:0002bda0       ?GetStdUserInteger@CobraNetNode@@QAEHIPAI@Z 1002cda0 f i asxtr800.obj
 0001:0002bdc0       ?HelperThread@asxTR800helperthread@@QAEXXZ 1002cdc0 f   asxtr800.obj
 0001:0002bef0       ?InputGet@asxGpioTR800@@UAE?AW4asxERROR@@PAHH@Z 1002cef0 f   asxtr800.obj
 0001:0002bf00       ?OutputGet@asxGpioTR800@@UAE?AW4asxERROR@@PAHH@Z 1002cf00 f   asxtr800.obj
 0001:0002bf40       ?OutputSet@asxGpioTR800@@UAE?AW4asxERROR@@PAHH@Z 1002cf40 f   asxtr800.obj
 0001:0002bf90       ?ReadGpioRelay@asxTR800helperthread@@QAEXI@Z 1002cf90 f   asxtr800.obj
 0001:0002bfc0       ?ReadOptoAction@asxTR800helperthread@@QAEXI@Z 1002cfc0 f   asxtr800.obj
 0001:0002bff0       ?Set@asxBlockTR800OptoMode@@UAE?AW4asxERROR@@IPAUasxParameterValue@@@Z 1002cff0 f   asxtr800.obj
 0001:0002c040       ?Set@asxLevelTR800@@UAE?AW4asxERROR@@M@Z 1002d040 f   asxtr800.obj
 0001:0002c0b0       ?SetGpioRelay@asxTR800helperthread@@QAEXII@Z 1002d0b0 f   asxtr800.obj
 0001:0002c0f0       ?SetMicGain@asxTR800helperthread@@QAEXII@Z 1002d0f0 f   asxtr800.obj
 0001:0002c120       ?SetOptoAction@asxTR800helperthread@@QAEXII@Z 1002d120 f   asxtr800.obj
 0001:0002c160       ?SetStdUserInteger@CobraNetNode@@QAEHII@Z 1002d160 f i asxtr800.obj
 0001:0002c180       ?asxTR800ThreadProc@@YGKPAX@Z 1002d180 f   asxtr800.obj
 0001:0002c1a0       ?asxTR800_Create@@YAXPAVasxSubSystem@@PAVCobraNetNode@@PAVasxMixer@@@Z 1002d1a0 f   asxtr800.obj
 0001:0002c530       ?enum_to_tr800@asxBlockTR800OptoMode@@AAEII@Z 1002d530 f   asxtr800.obj
 0001:0002c560       ?log10@@YAMM@Z             1002d560 f i asxtr800.obj
 0001:0002c580       ?tr800_to_enum@asxBlockTR800OptoMode@@AAEII@Z 1002d580 f   asxtr800.obj
 0001:0002c590       _log10f                    1002d590 f i asxtr800.obj
 0001:0002c5b0       ??0?$TASIArray@VwaveLineName@@@@QAE@XZ 1002d5b0 f i asxwave.obj
 0001:0002c5d0       ??0ControlTracker@@QAE@XZ  1002d5d0 f   asxwave.obj
 0001:0002c5e0       ??0ControlTrackerEntry@@QAE@PAUtagMIXERCONTROLA@@PAVasxNode@@1H@Z 1002d5e0 f i asxwave.obj
 0001:0002c620       ??0asxAdapterWAVE@@QAE@PAVasxSystem@@HPAD@Z 1002d620 f   asxwave.obj
 0001:0002c6f0       ??0asxCobranetWAVE@@QAE@PAVasxSubSystem@@PAUHMIXEROBJ__@@PAVasxNode@@2HPAUtagMIXERCONTROLA@@3@Z 1002d6f0 f   asxwave.obj
 0001:0002c810       ??0asxLevelWAVE@@QAE@PAVasxSubSystem@@PAUHMIXEROBJ__@@PAVasxNode@@2PAUtagMIXERCONTROLA@@H@Z 1002d810 f i asxwave.obj
 0001:0002c8b0       ??0asxMeterWAVE@@QAE@PAVasxSubSystem@@PAUHMIXEROBJ__@@PAVasxNode@@2PAUtagMIXERCONTROLA@@H@Z 1002d8b0 f i asxwave.obj
 0001:0002c950       ??0asxMixerScannerWAVE@@QAE@PAVasxSubSystem@@H@Z 1002d950 f   asxwave.obj
 0001:0002c9a0       ??0asxModeWAVE@@QAE@PAVasxSubSystem@@PAUHMIXEROBJ__@@PAVasxNode@@2PAUtagMIXERCONTROLA@@H@Z 1002d9a0 f   asxwave.obj
 0001:0002caf0       ??0asxMuxWAVE@@QAE@PAVasxSubSystem@@PAUHMIXEROBJ__@@PAVasxNode@@2PAUtagMIXERCONTROLA@@H@Z 1002daf0 f   asxwave.obj
 0001:0002cc80       ??0asxSilenceDetectorWAVE@@QAE@PAVasxSubSystem@@PAUHMIXEROBJ__@@PAVasxNode@@2PAUtagMIXERCONTROLA@@H@Z 1002dc80 f i asxwave.obj
 0001:0002cd20       ??0asxSubSystemWAVE@@QAE@PAVasxSystem@@@Z 1002dd20 f   asxwave.obj
 0001:0002cdb0       ??0asxToneDetectorWAVE@@QAE@PAVasxSubSystem@@PAUHMIXEROBJ__@@PAVasxNode@@2PAUtagMIXERCONTROLA@@H@Z 1002ddb0 f i asxwave.obj
 0001:0002ce50       ??0asxTunerWAVE@@QAE@PAVasxSubSystem@@PAUHMIXEROBJ__@@PAVasxNode@@2HPAUtagMIXERCONTROLA@@3333@Z 1002de50 f   asxwave.obj
 0001:0002d150       ??0asxVolumeWAVE@@QAE@PAVasxSubSystem@@PAUHMIXEROBJ__@@PAVasxNode@@2PAUtagMIXERCONTROLA@@H3@Z 1002e150 f i asxwave.obj
 0001:0002d220       ??0waveControlInfo@@QAE@PAUtagMIXERCONTROLA@@H@Z 1002e220 f i asxwave.obj
 0001:0002d250       ??0waveControlMuxHelper@@QAE@PAUHMIXEROBJ__@@PAVwaveControlInfo@@PAV?$TASIArray@VTASICString@@@@@Z 1002e250 f   asxwave.obj
 0001:0002d370       ??0waveLineName@@QAE@PAD@Z 1002e370 f i asxwave.obj
 0001:0002d3b0       ??1?$TASIArray@VwaveLineName@@@@QAE@XZ 1002e3b0 f i asxwave.obj
 0001:0002d400       ??1ControlTracker@@QAE@XZ  1002e400 f   asxwave.obj
 0001:0002d420       ??1asxAdapterWAVE@@UAE@XZ  1002e420 f   asxwave.obj
 0001:0002d490       ??1asxCobranetWAVE@@UAE@XZ 1002e490 f   asxwave.obj
 0001:0002d4d0       ??1asxLevelWAVE@@UAE@XZ    1002e4d0 f i asxwave.obj
 0001:0002d500       ??1asxMeterWAVE@@UAE@XZ    1002e500 f i asxwave.obj
 0001:0002d530       ??1asxMixerScannerWAVE@@UAE@XZ 1002e530 f   asxwave.obj
 0001:0002d5a0       ??1asxModeWAVE@@UAE@XZ     1002e5a0 f   asxwave.obj
 0001:0002d620       ??1asxMuxWAVE@@UAE@XZ      1002e620 f   asxwave.obj
 0001:0002d6b0       ??1asxSilenceDetectorWAVE@@UAE@XZ 1002e6b0 f i asxwave.obj
 0001:0002d6e0       ??1asxSubSystemWAVE@@UAE@XZ 1002e6e0 f   asxwave.obj
 0001:0002d6f0       ??1asxToneDetectorWAVE@@UAE@XZ 1002e6f0 f i asxwave.obj
 0001:0002d720       ??1asxTunerWAVE@@UAE@XZ    1002e720 f   asxwave.obj
 0001:0002d800       ??1asxVolumeWAVE@@UAE@XZ   1002e800 f i asxwave.obj
 0001:0002d840       ??1waveControlInfo@@QAE@XZ 1002e840 f i asxwave.obj
 0001:0002d850       ??1waveLineName@@QAE@XZ    1002e850 f i asxwave.obj
 0001:0002d860       ??A?$TASIArray@VwaveLineName@@@@QBEPAVwaveLineName@@H@Z 1002e860 f i asxwave.obj
 0001:0002d880       ??_GasxAdapterWAVE@@UAEPAXI@Z 1002e880 f i asxwave.obj
 0001:0002d880       ??_EasxAdapterWAVE@@UAEPAXI@Z 1002e880 f i asxwave.obj
 0001:0002d8b0       ??_GasxCobranetWAVE@@UAEPAXI@Z 1002e8b0 f i asxwave.obj
 0001:0002d8b0       ??_EasxCobranetWAVE@@UAEPAXI@Z 1002e8b0 f i asxwave.obj
 0001:0002d8e0       ??_GasxLevelWAVE@@UAEPAXI@Z 1002e8e0 f i asxwave.obj
 0001:0002d8e0       ??_EasxLevelWAVE@@UAEPAXI@Z 1002e8e0 f i asxwave.obj
 0001:0002d930       ??_GasxMeterWAVE@@UAEPAXI@Z 1002e930 f i asxwave.obj
 0001:0002d930       ??_EasxMeterWAVE@@UAEPAXI@Z 1002e930 f i asxwave.obj
 0001:0002d980       ??_GasxMixerScannerWAVE@@UAEPAXI@Z 1002e980 f i asxwave.obj
 0001:0002d980       ??_EasxMixerScannerWAVE@@UAEPAXI@Z 1002e980 f i asxwave.obj
 0001:0002d9b0       ??_EasxModeWAVE@@UAEPAXI@Z 1002e9b0 f i asxwave.obj
 0001:0002d9b0       ??_GasxModeWAVE@@UAEPAXI@Z 1002e9b0 f i asxwave.obj
 0001:0002d9e0       ??_EasxMuxWAVE@@UAEPAXI@Z  1002e9e0 f i asxwave.obj
 0001:0002d9e0       ??_GasxMuxWAVE@@UAEPAXI@Z  1002e9e0 f i asxwave.obj
 0001:0002da10       ??_EasxSilenceDetectorWAVE@@UAEPAXI@Z 1002ea10 f i asxwave.obj
 0001:0002da10       ??_GasxSilenceDetectorWAVE@@UAEPAXI@Z 1002ea10 f i asxwave.obj
 0001:0002da60       ??_EasxSubSystemWAVE@@UAEPAXI@Z 1002ea60 f i asxwave.obj
 0001:0002da60       ??_GasxSubSystemWAVE@@UAEPAXI@Z 1002ea60 f i asxwave.obj
 0001:0002da90       ??_GasxToneDetectorWAVE@@UAEPAXI@Z 1002ea90 f i asxwave.obj
 0001:0002da90       ??_EasxToneDetectorWAVE@@UAEPAXI@Z 1002ea90 f i asxwave.obj
 0001:0002dae0       ??_GasxTunerWAVE@@UAEPAXI@Z 1002eae0 f i asxwave.obj
 0001:0002dae0       ??_EasxTunerWAVE@@UAEPAXI@Z 1002eae0 f i asxwave.obj
 0001:0002db10       ??_GasxVolumeWAVE@@UAEPAXI@Z 1002eb10 f i asxwave.obj
 0001:0002db10       ??_EasxVolumeWAVE@@UAEPAXI@Z 1002eb10 f i asxwave.obj
 0001:0002db70       ??_GwaveControlInfo@@QAEPAXI@Z 1002eb70 f i asxwave.obj
 0001:0002db90       ??_GwaveLineName@@QAEPAXI@Z 1002eb90 f i asxwave.obj
 0001:0002dbc0       ?Add@?$TASIArray@VTASICString@@@@QAEHPAVTASICString@@@Z 1002ebc0 f i asxwave.obj
 0001:0002dbf0       ?Add@?$TASIArray@VwaveLineName@@@@QAEHPAVwaveLineName@@@Z 1002ebf0 f i asxwave.obj
 0001:0002dde0       ?AddControl@ControlTracker@@QAEXPAUtagMIXERCONTROLA@@PAVasxNode@@1H@Z 1002ede0 f   asxwave.obj
 0001:0002ded0       ?AddControl@asxMixerScannerWAVE@@AAEXPAVasxMixer@@PAVControlTracker@@PAUHMIXEROBJ__@@PAVasxNode@@3PAUtagMIXERCONTROLA@@H@Z 1002eed0 f   asxwave.obj
 0001:0002e920       ?CheckSubSystems@asxAdapterWAVE@@UAE?AW4asxERROR@@PAI0@Z 1002f920 f i asxwave.obj
 0001:0002e940       ?Count@?$TASIArray@VwaveLineName@@@@QBEHXZ 1002f940 f i asxwave.obj
 0001:0002e950       ?Enlarge@?$TASIArray@VTASICString@@@@AAEXXZ 1002f950 f i asxwave.obj
 0001:0002e9b0       ?Enlarge@?$TASIArray@VwaveLineName@@@@AAEXXZ 1002f9b0 f i asxwave.obj
 0001:0002ea10       ?Get@asxLevelWAVE@@UAE?AW4asxERROR@@PAM@Z 1002fa10 f   asxwave.obj
 0001:0002ea80       ?Get@asxModeWAVE@@UAE?AW4asxERROR@@PAW4asxCHANNELMODE@@@Z 1002fa80 f   asxwave.obj
 0001:0002eb40       ?Get@asxMuxWAVE@@UAE?AW4asxERROR@@PAW4asxNODE@@PAH@Z 1002fb40 f   asxwave.obj
 0001:0002ec10       ?GetBand@asxTunerWAVE@@UAE?AW4asxERROR@@PAW4asxTUNERBAND@@@Z 1002fc10 f   asxwave.obj
 0001:0002ecd0       ?GetControlOfType@ControlTracker@@QAEHPAUtagMIXERCONTROLA@@PAVasxNode@@1K@Z 1002fcd0 f   asxwave.obj
 0001:0002edb0       ?GetDelay@asxSilenceDetectorWAVE@@UAE?AW4asxERROR@@PAI@Z 1002fdb0 f   asxwave.obj
 0001:0002ee20       ?GetEnable@asxSilenceDetectorWAVE@@UAE?AW4asxERROR@@PAI@Z 1002fe20 f   asxwave.obj
 0001:0002ee90       ?GetEnable@asxToneDetectorWAVE@@UAE?AW4asxERROR@@PAI@Z 1002fe90 f   asxwave.obj
 0001:0002ef20       ?GetEventEnable@asxSilenceDetectorWAVE@@UAE?AW4asxERROR@@PAI@Z 1002ff20 f   asxwave.obj
 0001:0002ef90       ?GetEventEnable@asxToneDetectorWAVE@@UAE?AW4asxERROR@@PAI@Z 1002ff90 f   asxwave.obj
 0001:0002f020       ?GetFrequency@asxToneDetectorWAVE@@UAE?AW4asxERROR@@IPAI@Z 10030020 f   asxwave.obj
 0001:0002f0b0       ?GetFrequency@asxTunerWAVE@@UAE?AW4asxERROR@@PAK@Z 100300b0 f   asxwave.obj
 0001:0002f0f0       ?GetFrequencyRange@asxTunerWAVE@@QAE?AW4asxERROR@@XZ 100300f0 f   asxwave.obj
 0001:0002f100       ?GetGain@asxTunerWAVE@@UAE?AW4asxERROR@@PAM@Z 10030100 f   asxwave.obj
 0001:0002f120       ?GetGain@asxVolumeWAVE@@UAE?AW4asxERROR@@PAMH@Z 10030120 f   asxwave.obj
 0001:0002f1b0       ?GetGainRange@asxTunerWAVE@@UAE?AW4asxERROR@@PAM00@Z 100301b0 f   asxwave.obj
 0001:0002f1c0       ?GetIPAddress@asxCobranetWAVE@@QAE?AW4asxERROR@@PAK@Z 100301c0 f   asxwave.obj
 0001:0002f230       ?GetMACAddress@asxCobranetWAVE@@QAE?AW4asxERROR@@PAKPAG@Z 10030230 f   asxwave.obj
 0001:0002f2f0       ?GetMute@asxVolumeWAVE@@UAE?AW4asxERROR@@PAHH@Z 100302f0 f i asxwave.obj
 0001:0002f300       ?GetNextControl@ControlTracker@@QAEHPAUtagMIXERCONTROLA@@PAPAVasxNode@@1PAH@Z 10030300 f   asxwave.obj
 0001:0002f360       ?GetNextDstControl@ControlTracker@@QAEHPAVasxNode@@PAUtagMIXERCONTROLA@@PAPAV2@PAH@Z 10030360 f   asxwave.obj
 0001:0002f400       ?GetNextSrcControl@ControlTracker@@QAEHPAVasxNode@@PAUtagMIXERCONTROLA@@PAPAV2@PAH@Z 10030400 f   asxwave.obj
 0001:0002f4b0       ?GetPeak@asxMeterWAVE@@UAE?AW4asxERROR@@PAMH@Z 100304b0 f   asxwave.obj
 0001:0002f540       ?GetRFLevel@asxTunerWAVE@@UAE?AW4asxERROR@@PAM@Z 10030540 f   asxwave.obj
 0001:0002f560       ?GetRMS@asxMeterWAVE@@UAE?AW4asxERROR@@PAMH@Z 10030560 f i asxwave.obj
 0001:0002f570       ?GetRange@asxLevelWAVE@@UAE?AW4asxERROR@@PAM00@Z 10030570 f   asxwave.obj
 0001:0002f5d0       ?GetRange@asxVolumeWAVE@@UAE?AW4asxERROR@@PAM00@Z 100305d0 f   asxwave.obj
 0001:0002f610       ?GetRawRFLevel@asxTunerWAVE@@UAE?AW4asxERROR@@PAH@Z 10030610 f   asxwave.obj
 0001:0002f630       ?GetState@asxSilenceDetectorWAVE@@UAE?AW4asxERROR@@PAI@Z 10030630 f   asxwave.obj
 0001:0002f6a0       ?GetState@asxToneDetectorWAVE@@UAE?AW4asxERROR@@PAI@Z 100306a0 f   asxwave.obj
 0001:0002f730       ?GetStatus@asxTunerWAVE@@UAE?AW4asxERROR@@PAI0@Z 10030730 f   asxwave.obj
 0001:0002f810       ?GetThreshold@asxSilenceDetectorWAVE@@UAE?AW4asxERROR@@PAM@Z 10030810 f   asxwave.obj
 0001:0002f890       ?GetThreshold@asxToneDetectorWAVE@@UAE?AW4asxERROR@@PAM@Z 10030890 f   asxwave.obj
 0001:0002f930       ?MultipleItems@waveControlInfo@@QAEHXZ 10030930 f i asxwave.obj
 0001:0002f940       ?ReScan@asxSubSystemWAVE@@UAEXXZ 10030940 f   asxwave.obj
 0001:0002f950       ?Scan@asxMixerScannerWAVE@@UAEXPAVasxMixer@@@Z 10030950 f   asxwave.obj
 0001:00030330       ?Scan@asxSubSystemWAVE@@UAEXXZ 10031330 f   asxwave.obj
 0001:00030400       ?Set@asxLevelWAVE@@UAE?AW4asxERROR@@M@Z 10031400 f   asxwave.obj
 0001:00030460       ?Set@asxModeWAVE@@UAE?AW4asxERROR@@W4asxCHANNELMODE@@@Z 10031460 f   asxwave.obj
 0001:00030510       ?Set@asxMuxWAVE@@UAE?AW4asxERROR@@W4asxNODE@@H@Z 10031510 f   asxwave.obj
 0001:000305e0       ?SetBand@asxTunerWAVE@@UAE?AW4asxERROR@@W4asxTUNERBAND@@@Z 100315e0 f   asxwave.obj
 0001:000306a0       ?SetDelay@asxSilenceDetectorWAVE@@UAE?AW4asxERROR@@I@Z 100316a0 f   asxwave.obj
 0001:00030710       ?SetEnable@asxSilenceDetectorWAVE@@UAE?AW4asxERROR@@I@Z 10031710 f   asxwave.obj
 0001:00030780       ?SetEnable@asxToneDetectorWAVE@@UAE?AW4asxERROR@@I@Z 10031780 f   asxwave.obj
 0001:00030810       ?SetEventEnable@asxSilenceDetectorWAVE@@UAE?AW4asxERROR@@I@Z 10031810 f   asxwave.obj
 0001:00030880       ?SetEventEnable@asxToneDetectorWAVE@@UAE?AW4asxERROR@@I@Z 10031880 f   asxwave.obj
 0001:00030910       ?SetFrequency@asxTunerWAVE@@UAE?AW4asxERROR@@K@Z 10031910 f   asxwave.obj
 0001:00030950       ?SetGain@asxTunerWAVE@@UAE?AW4asxERROR@@M@Z 10031950 f   asxwave.obj
 0001:00030960       ?SetGain@asxVolumeWAVE@@UAE?AW4asxERROR@@PBMH@Z 10031960 f   asxwave.obj
 0001:00030a00       ?SetMode@asxTunerWAVE@@UAE?AW4asxERROR@@W4asxTUNERMODE@@0@Z 10031a00 f   asxwave.obj
 0001:00030a10       ?SetMute@asxVolumeWAVE@@UAE?AW4asxERROR@@PAHH@Z 10031a10 f i asxwave.obj
 0001:00030a20       ?SetThreshold@asxSilenceDetectorWAVE@@UAE?AW4asxERROR@@M@Z 10031a20 f   asxwave.obj
 0001:00030aa0       ?SetThreshold@asxToneDetectorWAVE@@UAE?AW4asxERROR@@M@Z 10031aa0 f   asxwave.obj
 0001:00030b30       ?addProcessedLine@asxMixerScannerWAVE@@AAEXPADH@Z 10031b30 f   asxwave.obj
 0001:00030bc0       ?alreadyProcessedThisLine@asxMixerScannerWAVE@@AAEHPADPAH@Z 10031bc0 f   asxwave.obj
 0001:00030c40       ?asxwave_MapError@@YA?AW4asxERROR@@I@Z 10031c40 f   asxwave.obj
 0001:00030d30       ?initDetails@waveControlInfo@@QAEXPAUtMIXERCONTROLDETAILS@@KPAX@Z 10031d30 f   asxwave.obj
 0001:00030e60       ??0asxPlayerWAVE@@QAE@PAVasxSubSystem@@PAVasxNode@@1I@Z 10031e60 f   asxwaveplay.obj
 0001:00030e90       ??1asxPlayerWAVE@@UAE@XZ   10031e90 f   asxwaveplay.obj
 0001:00030ef0       ??_EasxPlayerWAVE@@UAEPAXI@Z 10031ef0 f i asxwaveplay.obj
 0001:00030ef0       ??_GasxPlayerWAVE@@UAEPAXI@Z 10031ef0 f i asxwaveplay.obj
 0001:00030f20       ?AllocOutput@asxPlayerWAVE@@MAE?AW4asxERROR@@XZ 10031f20 f i asxwaveplay.obj
 0001:00030f70       ?FreeOutput@asxPlayerWAVE@@MAE?AW4asxERROR@@XZ 10031f70 f i asxwaveplay.obj
 0001:00030f90       ?GetPosition@asxPlayerWAVE@@UAE?AW4asxERROR@@W4asxTIMESCALE@@PAK@Z 10031f90 f   asxwaveplay.obj
 0001:00031030       ?HelperThread@asxPlayerWAVE@@UAEXXZ 10032030 f   asxwaveplay.obj
 0001:000311f0       ?ResetOutput@asxPlayerWAVE@@MAE?AW4asxERROR@@XZ 100321f0 f i asxwaveplay.obj
 0001:00031210       ?SetTimeScale@asxPlayerWAVE@@UAE?AW4asxERROR@@M@Z 10032210 f   asxwaveplay.obj
 0001:00031220       ?StartOutput@asxPlayerWAVE@@MAE?AW4asxERROR@@XZ 10032220 f i asxwaveplay.obj
 0001:00031240       ?StopOutput@asxPlayerWAVE@@MAE?AW4asxERROR@@XZ 10032240 f i asxwaveplay.obj
 0001:00031260       ??0asxRecorderWAVE@@QAE@PAVasxSubSystem@@PAVasxNode@@1I@Z 10032260 f   asxwaverec.obj
 0001:00031290       ??1asxRecorderWAVE@@UAE@XZ 10032290 f   asxwaverec.obj
 0001:000312f0       ??_EasxRecorderWAVE@@UAEPAXI@Z 100322f0 f i asxwaverec.obj
 0001:000312f0       ??_GasxRecorderWAVE@@UAEPAXI@Z 100322f0 f i asxwaverec.obj
 0001:00031320       ?AllocInput@asxRecorderWAVE@@EAE?AW4asxERROR@@XZ 10032320 f i asxwaverec.obj
 0001:00031350       ?EnumerateAllFormats@asxRecorderWAVE@@EAEXXZ 10032350 f   asxwaverec.obj
 0001:00031390       ?FreeInput@asxRecorderWAVE@@EAE?AW4asxERROR@@XZ 10032390 f i asxwaverec.obj
 0001:000313b0       ?GetInputPosition@asxRecorderWAVE@@EAE?AW4asxERROR@@PAK@Z 100323b0 f   asxwaverec.obj
 0001:00031400       ?HelperThread@asxRecorderWAVE@@UAEKXZ 10032400 f   asxwaverec.obj
 0001:00031580       ?SetInputFormat@asxRecorderWAVE@@EAE?AW4asxERROR@@XZ 10032580 f i asxwaverec.obj
 0001:00031590       ?StartInput@asxRecorderWAVE@@EAE?AW4asxERROR@@XZ 10032590 f i asxwaverec.obj
 0001:000315b0       ?StopInput@asxRecorderWAVE@@EAE?AW4asxERROR@@XZ 100325b0 f i asxwaverec.obj
 0001:000315d0       ??0CobraNetNode@@QAE@PBD0PAVSnmpSession@@PADH@Z 100325d0 f   cobranet.obj
 0001:000317c0       ??0CobraNetPort@@QAE@XZ    100327c0 f i cobranet.obj
 0001:000317d0       ??0CobraNetReceiver@@QAE@XZ 100327d0 f i cobranet.obj
 0001:000317e0       ??0CobraNetTransmitter@@QAE@XZ 100327e0 f i cobranet.obj
 0001:000317f0       ??0asiOID@@QAE@XZ          100327f0 f i cobranet.obj
 0001:00031810       ??1CobraNetNode@@QAE@XZ    10032810 f   cobranet.obj
 0001:00031840       ??1asiOID@@QAE@XZ          10032840 f i cobranet.obj
 0001:00031870       ??_H@YGXPAXIHP6EPAX0@Z@Z   10032870 f i cobranet.obj
 0001:000318a0       ?ClearDirtyFlag@CobraNetNode@@AAEXPAUasiCNdev_FieldEntry_@@@Z 100328a0 f   cobranet.obj
 0001:000318c0       ?ClearRxDirtyFlag@CobraNetNode@@AAEXPAUasiCNdev_FieldEntry_@@HH@Z 100328c0 f   cobranet.obj
 0001:00031950       ?ClearTxDirtyFlag@CobraNetNode@@AAEXPAUasiCNdev_FieldEntry_@@HH@Z 10032950 f   cobranet.obj
 0001:000319e0       ?ConvertMacString@CobraNetNode@@AAE_NPBD@Z 100329e0 f   cobranet.obj
 0001:00031bf0       ?GetDirtyFlag@CobraNetNode@@AAE_NKKKH@Z 10032bf0 f   cobranet.obj
 0001:00031c40       ?GetDirtyFlag@CobraNetNode@@AAE_NPAUasiCNdev_FieldEntry_@@@Z 10032c40 f   cobranet.obj
 0001:00031c60       ?GetIndexed@asiMibEntry@@QAEHXZ 10032c60 f i cobranet.obj
 0001:00031c70       ?GetIntField@CobraNetNode@@AAEHW4asiCNdev_NodeFields@1@PAH@Z 10032c70 f   cobranet.obj
 0001:00031cd0       ?GetOctetField@CobraNetNode@@AAEHW4asiCNdev_NodeFields@1@PAD@Z 10032cd0 f   cobranet.obj
 0001:00031d30       ?GetRxDirtyFlag@CobraNetNode@@AAE_NPAUasiCNdev_FieldEntry_@@HH@Z 10032d30 f   cobranet.obj
 0001:00031db0       ?GetRxIntField@CobraNetNode@@AAEHW4asiCNdev_RxFields@1@PAHHH@Z 10032db0 f   cobranet.obj
 0001:00031e40       ?GetStringField@CobraNetNode@@AAEHW4asiCNdev_NodeFields@1@PADHPAH@Z 10032e40 f   cobranet.obj
 0001:00031eb0       ?GetTxDirtyFlag@CobraNetNode@@AAE_NPAUasiCNdev_FieldEntry_@@HH@Z 10032eb0 f   cobranet.obj
 0001:00031f30       ?GetTxIntField@CobraNetNode@@AAEHW4asiCNdev_TxFields@1@PAHHH@Z 10032f30 f   cobranet.obj
 0001:00031fd0       ?InitOIDs@CobraNetNode@@CAXXZ 10032fd0 f   cobranet.obj
 0001:000323f0       ?IsIndexOid@asiMibEntry@@QAEHXZ 100333f0 f i cobranet.obj
 0001:00032400       ?NullValues@asiOID@@AAEXXZ 10033400 f i cobranet.obj
 0001:00032420       ?ReadAll@CobraNetNode@@QAEHXZ 10033420 f   cobranet.obj
 0001:00032450       ?ReadAudioMeterField@CobraNetNode@@QAEHI@Z 10033450 f   cobranet.obj
 0001:00032470       ?ReadField@CobraNetNode@@AAEHPAUasiCNdev_FieldEntry_@@@Z 10033470 f   cobranet.obj
 0001:000325e0       ?ReadIntArray64Field@CobraNetNode@@AAEHPAUasiCNdev_FieldEntry_@@PAII@Z 100335e0 f   cobranet.obj
 0001:00032640       ?ReadRx@CobraNetNode@@QAEHH@Z 10033640 f   cobranet.obj
 0001:00032690       ?ReadRxField@CobraNetNode@@AAEHPAUasiCNdev_FieldEntry_@@HH@Z 10033690 f   cobranet.obj
 0001:00032740       ?ReadStatus@CobraNetNode@@QAEHXZ 10033740 f   cobranet.obj
 0001:00032820       ?ReadStdUserIntegerField@CobraNetNode@@QAEHI@Z 10033820 f   cobranet.obj
 0001:00032840       ?ReadTx@CobraNetNode@@QAEHH@Z 10033840 f   cobranet.obj
 0001:00032890       ?ReadTxField@CobraNetNode@@AAEHPAUasiCNdev_FieldEntry_@@HH@Z 10033890 f   cobranet.obj
 0001:00032940       ?SetDirtyFlag@CobraNetNode@@AAEXPAUasiCNdev_FieldEntry_@@@Z 10033940 f   cobranet.obj
 0001:00032960       ?SetIndex@asiOID@@QAEXHH@Z 10033960 f i cobranet.obj
 0001:000329a0       ?SetIntField@CobraNetNode@@AAEHW4asiCNdev_NodeFields@1@H@Z 100339a0 f   cobranet.obj
 0001:00032a00       ?SetMibEntry@asiOID@@QAEXPAVasiMibEntry@@@Z 10033a00 f i cobranet.obj
 0001:00032ab0       ?SetOctetField@CobraNetNode@@AAEHW4asiCNdev_NodeFields@1@PBD@Z 10033ab0 f   cobranet.obj
 0001:00032b70       ?SetRxDirtyFlag@CobraNetNode@@AAEXPAUasiCNdev_FieldEntry_@@HH@Z 10033b70 f   cobranet.obj
 0001:00032bf0       ?SetRxIntField@CobraNetNode@@AAEHW4asiCNdev_RxFields@1@HHH@Z 10033bf0 f   cobranet.obj
 0001:00032ca0       ?SetStringField@CobraNetNode@@AAEHW4asiCNdev_NodeFields@1@PBD@Z 10033ca0 f   cobranet.obj
 0001:00032d40       ?SetTxDirtyFlag@CobraNetNode@@AAEXPAUasiCNdev_FieldEntry_@@HH@Z 10033d40 f   cobranet.obj
 0001:00032dc0       ?SetTxIntField@CobraNetNode@@AAEHW4asiCNdev_TxFields@1@HHH@Z 10033dc0 f   cobranet.obj
 0001:00032e70       ?WriteAll@CobraNetNode@@QAEHXZ 10033e70 f   cobranet.obj
 0001:00032ef0       ?WriteField@CobraNetNode@@AAEHPAUasiCNdev_FieldEntry_@@@Z 10033ef0 f   cobranet.obj
 0001:00033030       ?WriteIntArray64Field@CobraNetNode@@AAEHPAUasiCNdev_FieldEntry_@@PAII@Z 10034030 f   cobranet.obj
 0001:00033090       ?WriteRx@CobraNetNode@@QAEHH@Z 10034090 f   cobranet.obj
 0001:00033100       ?WriteRxField@CobraNetNode@@AAEHPAUasiCNdev_FieldEntry_@@HH@Z 10034100 f   cobranet.obj
 0001:000331c0       ?WriteStdUserIntegerField@CobraNetNode@@QAEHI@Z 100341c0 f   cobranet.obj
 0001:000331e0       ?WriteTx@CobraNetNode@@QAEHH@Z 100341e0 f   cobranet.obj
 0001:00033250       ?WriteTxField@CobraNetNode@@AAEHPAUasiCNdev_FieldEntry_@@HH@Z 10034250 f   cobranet.obj
 0001:00033300       ?cnDecodeModeRateCode@@YAHKPAH0@Z 10034300 f   cobranet.obj
 0001:00033360       ?cnDecodeSubformatCode@@YAHKPAH00@Z 10034360 f   cobranet.obj
 0001:000333e0       ?cnGetModeRateCode@@YAKHH@Z 100343e0 f   cobranet.obj
 0001:00033400       ?cnGetSubformatCode@@YAKHHH@Z 10034400 f   cobranet.obj
 0001:00033420       ?cnMaxChannelsPerBundle@@YAHHHH@Z 10034420 f   cobranet.obj
 0001:00033440       ??0RiffFile@@QAE@PBDW4eOpenMode@0@@Z 10034440 f   rifffile.obj
 0001:000334c0       ??1RiffFile@@QAE@XZ        100344c0 f   rifffile.obj
 0001:00033500       ?Ascend@RiffFile@@QAEHXZ   10034500 f   rifffile.obj
 0001:000335d0       ?CreateChunk@RiffFile@@QAEHIW4eChunkType@1@@Z 100345d0 f   rifffile.obj
 0001:000336f0       ?Descend@RiffFile@@QAEHIW4eChunkType@1@@Z 100346f0 f   rifffile.obj
 0001:00033910       ?IsOk@RiffFile@@QAEHXZ     10034910 f i rifffile.obj
 0001:00033920       ?ModifyOuterChunkLengths@RiffFile@@IAEXI@Z 10034920 f   rifffile.obj
 0001:00033950       ?Read@RiffFile@@QAEJPADJ@Z 10034950 f   rifffile.obj
 0001:00033980       ?Seek@RiffFile@@QAEJJH@Z   10034980 f   rifffile.obj
 0001:000339c0       ?Write@RiffFile@@QAEJPBDJ@Z 100349c0 f   rifffile.obj
 0001:00033a30       _tfileio_fclose            10034a30 f   tfileio.obj
 0001:00033a50       _tfileio_fopen             10034a50 f   tfileio.obj
 0001:00033ab0       _tfileio_fread             10034ab0 f   tfileio.obj
 0001:00033ae0       _tfileio_fseek             10034ae0 f   tfileio.obj
 0001:00033b20       _tfileio_ftello            10034b20 f   tfileio.obj
 0001:00033b40       _tfileio_fwrite            10034b40 f   tfileio.obj
 0001:00033b70       ??0TWavFileBase@@QAE@XZ    10034b70 f i twavfile.obj
 0001:00033b90       ??0TWavFileTypeDAF@@QAE@PBD0PAJ@Z 10034b90 f   twavfile.obj
 0001:00033bc0       ??0TWavFileTypeGenerator@@QAE@PBD0PAJ@Z 10034bc0 f   twavfile.obj
 0001:00033c70       ??0TWavFileTypeMP23@@QAE@PBD0PAJ@Z 10034c70 f   twavfile.obj
 0001:00033ca0       ??0TWavFileTypeNullRecord@@QAE@PBD0PAJ@Z 10034ca0 f   twavfile.obj
 0001:00033cd0       ??0TWavFileTypeRaw@@QAE@PBD0PAJ@Z 10034cd0 f   twavfile.obj
 0001:00033d00       ??0TWavFileTypeWav@@QAE@PBD0PAJ@Z 10034d00 f   twavfile.obj
 0001:00033d80       ??0TWavFileTypeWav@@QAE@XZ 10034d80 f   twavfile.obj
 0001:00033df0       ??1TWavFileBase@@UAE@XZ    10034df0 f i twavfile.obj
 0001:00033e00       ??1TWavFileTypeDAF@@UAE@XZ 10034e00 f i twavfile.obj
 0001:00033e20       ??1TWavFileTypeGenerator@@UAE@XZ 10034e20 f i twavfile.obj
 0001:00033e40       ??1TWavFileTypeMP23@@UAE@XZ 10034e40 f i twavfile.obj
 0001:00033e60       ??1TWavFileTypeNullRecord@@UAE@XZ 10034e60 f i twavfile.obj
 0001:00033e70       ??1TWavFileTypeRaw@@UAE@XZ 10034e70 f i twavfile.obj
 0001:00033e90       ??1TWavFileTypeWav@@UAE@XZ 10034e90 f i twavfile.obj
 0001:00033ef0       ??_ETWavFileBase@@UAEPAXI@Z 10034ef0 f i twavfile.obj
 0001:00033ef0       ??_GTWavFileBase@@UAEPAXI@Z 10034ef0 f i twavfile.obj
 0001:00033f20       ??_ETWavFileTypeDAF@@UAEPAXI@Z 10034f20 f i twavfile.obj
 0001:00033f20       ??_GTWavFileTypeDAF@@UAEPAXI@Z 10034f20 f i twavfile.obj
 0001:00033f60       ??_ETWavFileTypeGenerator@@UAEPAXI@Z 10034f60 f i twavfile.obj
 0001:00033f60       ??_GTWavFileTypeGenerator@@UAEPAXI@Z 10034f60 f i twavfile.obj
 0001:00033fa0       ??_ETWavFileTypeMP23@@UAEPAXI@Z 10034fa0 f i twavfile.obj
 0001:00033fa0       ??_GTWavFileTypeMP23@@UAEPAXI@Z 10034fa0 f i twavfile.obj
 0001:00033fe0       ??_ETWavFileTypeNullRecord@@UAEPAXI@Z 10034fe0 f i twavfile.obj
 0001:00033fe0       ??_GTWavFileTypeNullRecord@@UAEPAXI@Z 10034fe0 f i twavfile.obj
 0001:00034010       ??_ETWavFileTypeRaw@@UAEPAXI@Z 10035010 f i twavfile.obj
 0001:00034010       ??_GTWavFileTypeRaw@@UAEPAXI@Z 10035010 f i twavfile.obj
 0001:00034050       ??_GTWavFileTypeWav@@UAEPAXI@Z 10035050 f i twavfile.obj
 0001:00034050       ??_ETWavFileTypeWav@@UAEPAXI@Z 10035050 f i twavfile.obj
 0001:000340c0       ?BytesRemain@TWavFileBase@@QAEJXZ 100350c0 f   twavfile.obj
 0001:000340e0       ?Close@TWavFileBase@@UAEJXZ 100350e0 f   twavfile.obj
 0001:00034120       ?Close@TWavFileTypeGenerator@@UAEJXZ 10035120 f   twavfile.obj
 0001:00034150       ?Close@TWavFileTypeNullRecord@@UAEJXZ 10035150 f   twavfile.obj
 0001:00034160       ?Close@TWavFileTypeWav@@UAEJXZ 10035160 f   twavfile.obj
 0001:00034190       ?FindMPEGHeader@TWavFileTypeMP23@@AAEJPAK@Z 10035190 f   twavfile.obj
 0001:00034390       ?GetErrorStr@TWavFileBase@@QAEXJPAD@Z 10035390 f   twavfile.obj
 0001:00034510       ?GetFileSize@TWavFileBase@@QAEJXZ 10035510 f   twavfile.obj
 0001:00034520       ?Open@TWavFileBase@@UAEJPBDK@Z 10035520 f   twavfile.obj
 0001:00034590       ?Open@TWavFileTypeDAF@@UAEJPBDK@Z 10035590 f   twavfile.obj
 0001:00034670       ?Open@TWavFileTypeGenerator@@UAEJPBDK@Z 10035670 f   twavfile.obj
 0001:000346b0       ?Open@TWavFileTypeNullRecord@@UAEJPBDK@Z 100356b0 f   twavfile.obj
 0001:000346f0       ?Open@TWavFileTypeWav@@UAEJPBDK@Z 100356f0 f   twavfile.obj
 0001:00034750       ?OpenWavFile@@YAPAVTWavFileBase@@PBD0PAJ@Z 10035750 f   twavfile.obj
 0001:00034940       ?ParseFileName@TWavFileTypeGenerator@@QAEJPBD@Z 10035940 f   twavfile.obj
 0001:00034e50       ?ReadHeader@TWavFileBase@@UAEJH@Z 10035e50 f i twavfile.obj
 0001:00034e60       ?ReadHeader@TWavFileTypeDAF@@UAEJH@Z 10035e60 f   twavfile.obj
 0001:00034f50       ?ReadHeader@TWavFileTypeGenerator@@UAEJH@Z 10035f50 f   twavfile.obj
 0001:00034f70       ?ReadHeader@TWavFileTypeMP23@@UAEJH@Z 10035f70 f   twavfile.obj
 0001:00035000       ?ReadHeader@TWavFileTypeNullRecord@@UAEJH@Z 10036000 f   twavfile.obj
 0001:00035010       ?ReadHeader@TWavFileTypeRaw@@UAEJH@Z 10036010 f   twavfile.obj
 0001:00035040       ?ReadHeader@TWavFileTypeWav@@UAEJH@Z 10036040 f   twavfile.obj
 0001:000351e0       ?ReadMPEGHeader@TWavFileBase@@QAEJI@Z 100361e0 f   twavfile.obj
 0001:000352a0       ?ReadWavData@TWavFileBase@@UAEJPAEJ@Z 100362a0 f   twavfile.obj
 0001:000352d0       ?ReadWavData@TWavFileTypeGenerator@@UAEJPAEJ@Z 100362d0 f   twavfile.obj
 0001:000352e0       ?ReadWavData@TWavFileTypeNullRecord@@UAEJPAEJ@Z 100362e0 f   twavfile.obj
 0001:000352f0       ?ReadWavData@TWavFileTypeWav@@UAEJPAEJ@Z 100362f0 f   twavfile.obj
 0001:00035380       ?Seek@TWavFileBase@@UAEJJH@Z 10036380 f   twavfile.obj
 0001:000353c0       ?Seek@TWavFileTypeGenerator@@UAEJJH@Z 100363c0 f   twavfile.obj
 0001:000353d0       ?Seek@TWavFileTypeNullRecord@@UAEJJH@Z 100363d0 f   twavfile.obj
 0001:000353e0       ?Seek@TWavFileTypeWav@@UAEJJH@Z 100363e0 f   twavfile.obj
 0001:00035420       ?UpdateHeader@TWavFileTypeWav@@QAEJXZ 10036420 f   twavfile.obj
 0001:00035550       ?WriteHeader@TWavFileBase@@UAEJXZ 10036550 f i twavfile.obj
 0001:00035560       ?WriteHeader@TWavFileTypeGenerator@@UAEJXZ 10036560 f i twavfile.obj
 0001:00035570       ?WriteHeader@TWavFileTypeNullRecord@@UAEJXZ 10036570 f i twavfile.obj
 0001:00035580       ?WriteHeader@TWavFileTypeWav@@UAEJXZ 10036580 f   twavfile.obj
 0001:00035720       ?WriteWavData@TWavFileBase@@UAEJPAEJ@Z 10036720 f   twavfile.obj
 0001:00035760       ?WriteWavData@TWavFileTypeGenerator@@UAEJPAEJ@Z 10036760 f   twavfile.obj
 0001:00035770       ?WriteWavData@TWavFileTypeNullRecord@@UAEJPAEJ@Z 10036770 f   twavfile.obj
 0001:00035780       ?WriteWavData@TWavFileTypeWav@@UAEJPAEJ@Z 10036780 f   twavfile.obj
 0001:00035860       ??0Fifo@@QAE@J@Z           10036860 f   twavfilefifo.obj
 0001:00035890       ??0TWavFileWithFifo@@QAE@PAVTWavFileBase@@JW4FifoDirection@0@@Z 10036890 f   twavfilefifo.obj
 0001:00035930       ??1Fifo@@QAE@XZ            10036930 f   twavfilefifo.obj
 0001:00035950       ??1TWavFileWithFifo@@UAE@XZ 10036950 f   twavfilefifo.obj
 0001:000359d0       ??4TWavFileBase@@QAEAAV0@ABV0@@Z 100369d0 f i twavfilefifo.obj
 0001:00035a30       ??_GTWavFileWithFifo@@UAEPAXI@Z 10036a30 f i twavfilefifo.obj
 0001:00035a30       ??_ETWavFileWithFifo@@UAEPAXI@Z 10036a30 f i twavfilefifo.obj
 0001:00035a60       ?AdvanceReadPointer@Fifo@@AAEXJ@Z 10036a60 f   twavfilefifo.obj
 0001:00035a70       ?AdvanceWritePointer@Fifo@@AAEXJ@Z 10036a70 f   twavfilefifo.obj
 0001:00035ab0       ?Close@TWavFileWithFifo@@UAEJXZ 10036ab0 f   twavfilefifo.obj
 0001:00035ad0       ?DataAvailable@Fifo@@QAEJXZ 10036ad0 f   twavfilefifo.obj
 0001:00035ae0       ?FileIoThread@TWavFileWithFifo@@IAGKXZ 10036ae0 f   twavfilefifo.obj
 0001:00035b50       ?FileIoThreadEntry@TWavFileWithFifo@@KGKPAX@Z 10036b50 f   twavfilefifo.obj
 0001:00035b60       ?GetReadOffset@Fifo@@AAEJXZ 10036b60 f   twavfilefifo.obj
 0001:00035ba0       ?Open@TWavFileWithFifo@@UAEJPBDK@Z 10036ba0 f   twavfilefifo.obj
 0001:00035bd0       ?Read@Fifo@@QAEJPAEJ@Z     10036bd0 f   twavfilefifo.obj
 0001:00035c40       ?ReadFromFile@Fifo@@QAEXPAVTWavFileBase@@@Z 10036c40 f   twavfilefifo.obj
 0001:00035ca0       ?ReadHeader@TWavFileWithFifo@@UAEJH@Z 10036ca0 f   twavfilefifo.obj
 0001:00035cb0       ?ReadWavData@TWavFileWithFifo@@UAEJPAEJ@Z 10036cb0 f   twavfilefifo.obj
 0001:00035d00       ?Reset@Fifo@@QAEXXZ        10036d00 f   twavfilefifo.obj
 0001:00035d10       ?Seek@TWavFileWithFifo@@UAEJJH@Z 10036d10 f   twavfilefifo.obj
 0001:00035d80       ?SpaceAvailable@Fifo@@QAEJXZ 10036d80 f   twavfilefifo.obj
 0001:00035d90       ?StartFifo@TWavFileWithFifo@@IAEXXZ 10036d90 f   twavfilefifo.obj
 0001:00035e00       ?StartIoThread@TWavFileWithFifo@@IAEXXZ 10036e00 f   twavfilefifo.obj
 0001:00035e50       ?StopFifo@TWavFileWithFifo@@IAEXXZ 10036e50 f   twavfilefifo.obj
 0001:00035e80       ?StopIoThread@TWavFileWithFifo@@IAEXXZ 10036e80 f   twavfilefifo.obj
 0001:00035ec0       ?Write@Fifo@@QAEJPBEJ@Z    10036ec0 f   twavfilefifo.obj
 0001:00035f30       ?WriteHeader@TWavFileWithFifo@@UAEJXZ 10036f30 f   twavfilefifo.obj
 0001:00035f40       ?WriteToFile@Fifo@@QAEXPAVTWavFileBase@@@Z 10036f40 f   twavfilefifo.obj
 0001:00035fa0       ?WriteWavData@TWavFileWithFifo@@UAEJPAEJ@Z 10036fa0 f   twavfilefifo.obj
 0001:00035ff0       ??0TWavFmt@@QAE@XZ         10036ff0 f   twavfmt.obj
 0001:00036020       ?BytesToSamples@TWavFmt@@QAEJJJ@Z 10037020 f   twavfmt.obj
 0001:00036050       ?GetFormat@TWavFmt@@QAEJPADPAJ11@Z 10037050 f   twavfmt.obj
 0001:00036090       ?GetFormat@TWavFmt@@QAEJPADPAJ1@Z 10037090 f   twavfmt.obj
 0001:00036240       ?GetFormat@TWavFmt@@QAEJPAPAD@Z 10037240 f   twavfmt.obj
 0001:000364c0       ?GetFormat@TWavFmt@@QAEJPAUmpeg1waveformat_tag@@@Z 100374c0 f   twavfmt.obj
 0001:00036500       ?GetFormatBytesPerSample@TWavFmt@@QAEKXZ 10037500 f   twavfmt.obj
 0001:00036540       ?GetFormatBytesPerSecond@TWavFmt@@QAEKXZ 10037540 f   twavfmt.obj
 0001:00036570       ?GetFormatSamplesPerSecond@TWavFmt@@QAEKXZ 10037570 f   twavfmt.obj
 0001:00036580       ?NumChannels@TWavFmt@@QAEJXZ 10037580 f   twavfmt.obj
 0001:00036590       ?SetFormat@TWavFmt@@QAEJPBDJJ@Z 10037590 f   twavfmt.obj
 0001:00036aa0       ?SetFormat@TWavFmt@@QAEJPBDJJJ@Z 10037aa0 f   twavfmt.obj
 0001:00036b30       ?SetFormat@TWavFmt@@QAEJUmpeg1waveformat_tag@@@Z 10037b30 f   twavfmt.obj
 0001:00036b80       ?SetFormatMPEG@TWavFmt@@AAEJPBDJJJ@Z 10037b80 f   twavfmt.obj
 0001:00036c80       ?FillBuffer@TWavGen@@QAEJPAEJ@Z 10037c80 f   twavgen.obj
 0001:00037040       ?SetParameters@TWavGen@@QAEJW4wsSHAPE@1@NNNGPA_ND@Z 10038040 f   twavgen.obj
 0001:000370a2       _waveOutGetNumDevs@0       100380a2 f   winmm:WINMM.dll
 0001:000370a8       _waveInGetNumDevs@0        100380a8 f   winmm:WINMM.dll
 0001:000370ae       _mixerGetNumDevs@0         100380ae f   winmm:WINMM.dll
 0001:000370b4       _mixerGetDevCapsA@12       100380b4 f   winmm:WINMM.dll
 0001:000370ba       _mixerOpen@20              100380ba f   winmm:WINMM.dll
 0001:000370c0       _mixerClose@4              100380c0 f   winmm:WINMM.dll
 0001:000370c6       _mixerGetLineInfoA@12      100380c6 f   winmm:WINMM.dll
 0001:000370cc       _mixerGetID@12             100380cc f   winmm:WINMM.dll
 0001:000370d2       _mixerGetLineControlsA@12  100380d2 f   winmm:WINMM.dll
 0001:000370d8       _mixerGetControlDetailsA@12 100380d8 f   winmm:WINMM.dll
 0001:000370de       _mixerSetControlDetails@12 100380de f   winmm:WINMM.dll
 0001:000370e4       _waveOutOpen@24            100380e4 f   winmm:WINMM.dll
 0001:000370ea       _waveOutClose@4            100380ea f   winmm:WINMM.dll
 0001:000370f0       _waveOutPrepareHeader@12   100380f0 f   winmm:WINMM.dll
 0001:000370f6       _waveOutUnprepareHeader@12 100380f6 f   winmm:WINMM.dll
 0001:000370fc       _waveOutWrite@12           100380fc f   winmm:WINMM.dll
 0001:00037102       _waveOutPause@4            10038102 f   winmm:WINMM.dll
 0001:00037108       _waveOutRestart@4          10038108 f   winmm:WINMM.dll
 0001:0003710e       _waveOutReset@4            1003810e f   winmm:WINMM.dll
 0001:00037114       _waveOutGetPosition@12     10038114 f   winmm:WINMM.dll
 0001:0003711a       _waveInOpen@24             1003811a f   winmm:WINMM.dll
 0001:00037120       _waveInClose@4             10038120 f   winmm:WINMM.dll
 0001:00037126       _waveInPrepareHeader@12    10038126 f   winmm:WINMM.dll
 0001:0003712c       _waveInUnprepareHeader@12  1003812c f   winmm:WINMM.dll
 0001:00037132       _waveInAddBuffer@12        10038132 f   winmm:WINMM.dll
 0001:00037138       _waveInStart@4             10038138 f   winmm:WINMM.dll
 0001:0003713e       _waveInStop@4              1003813e f   winmm:WINMM.dll
 0001:00037144       _waveInReset@4             10038144 f   winmm:WINMM.dll
 0001:0003714a       _waveInGetPosition@12      1003814a f   winmm:WINMM.dll
 0001:00037150       _mmioStringToFOURCCA@8     10038150 f   winmm:WINMM.dll
 0001:00037156       _mmioOpenA@12              10038156 f   winmm:WINMM.dll
 0001:0003715c       _mmioClose@8               1003815c f   winmm:WINMM.dll
 0001:00037162       _mmioRead@12               10038162 f   winmm:WINMM.dll
 0001:00037168       _mmioWrite@12              10038168 f   winmm:WINMM.dll
 0001:0003716e       _mmioSeek@12               1003816e f   winmm:WINMM.dll
 0001:00037174       _mmioFlush@8               10038174 f   winmm:WINMM.dll
 0001:0003717a       _mmioDescend@16            1003817a f   winmm:WINMM.dll
 0001:00037180       _mmioAscend@12             10038180 f   winmm:WINMM.dll
 0001:00037186       _mmioCreateChunk@12        10038186 f   winmm:WINMM.dll
 0001:0003718c       _HPI_SubSysCreate@0        1003818c f   asihpi32:ASIHPI32.dll
 0001:00037192       _HPI_SubSysGetVersionEx@8  10038192 f   asihpi32:ASIHPI32.dll
 0001:00037198       _HPI_Entity_FindNext@20    10038198 f   asihpi32:ASIHPI32.dll
 0001:0003719e       _HPI_Entity_CopyValueFrom@20 1003819e f   asihpi32:ASIHPI32.dll
 0001:000371a4       _HPI_Entity_Unpack@20      100381a4 f   asihpi32:ASIHPI32.dll
 0001:000371aa       _HPI_Entity_AllocAndPack@24 100381aa f   asihpi32:ASIHPI32.dll
 0001:000371b0       _HPI_Entity_Free@4         100381b0 f   asihpi32:ASIHPI32.dll
 0001:000371b6       _HPI_Object_GetInfo@24     100381b6 f   asihpi32:ASIHPI32.dll
 0001:000371bc       _HPI_Object_BlockHandle@28 100381bc f   asihpi32:ASIHPI32.dll
 0001:000371c2       _HPI_Object_ParameterHandle@16 100381c2 f   asihpi32:ASIHPI32.dll
 0001:000371c8       _HPI_SubSysFree@4          100381c8 f   asihpi32:ASIHPI32.dll
 0001:000371ce       _HPI_SubSysGetNumAdapters@8 100381ce f   asihpi32:ASIHPI32.dll
 0001:000371d4       _HPI_SubSysGetAdapter@16   100381d4 f   asihpi32:ASIHPI32.dll
 0001:000371da       _HPI_SubSysSetHostNetworkInterface@8 100381da f   asihpi32:ASIHPI32.dll
 0001:000371e0       _HPI_AdapterOpen@8         100381e0 f   asihpi32:ASIHPI32.dll
 0001:000371e6       _HPI_AdapterClose@8        100381e6 f   asihpi32:ASIHPI32.dll
 0001:000371ec       _HPI_AdapterGetInfo@28     100381ec f   asihpi32:ASIHPI32.dll
 0001:000371f2       _HPI_AdapterGetModuleByIndex@36 100381f2 f   asihpi32:ASIHPI32.dll
 0001:000371f8       _HPI_AdapterSetMode@12     100381f8 f   asihpi32:ASIHPI32.dll
 0001:000371fe       _HPI_AdapterSetModeEx@16   100381fe f   asihpi32:ASIHPI32.dll
 0001:00037204       _HPI_AdapterGetMode@12     10038204 f   asihpi32:ASIHPI32.dll
 0001:0003720a       _HPI_AdapterSetProperty@20 1003820a f   asihpi32:ASIHPI32.dll
 0001:00037210       _HPI_AdapterGetProperty@20 10038210 f   asihpi32:ASIHPI32.dll
 0001:00037216       _HPI_NvMemoryOpen@16       10038216 f   asihpi32:ASIHPI32.dll
 0001:0003721c       _HPI_NvMemoryReadByte@16   1003821c f   asihpi32:ASIHPI32.dll
 0001:00037222       _HPI_NvMemoryWriteByte@16  10038222 f   asihpi32:ASIHPI32.dll
 0001:00037228       _HPI_GpioOpen@20           10038228 f   asihpi32:ASIHPI32.dll
 0001:0003722e       _HPI_GpioReadAllBits@12    1003822e f   asihpi32:ASIHPI32.dll
 0001:00037234       _HPI_GpioWriteBit@16       10038234 f   asihpi32:ASIHPI32.dll
 0001:0003723a       _HPI_GpioWriteStatus@12    1003823a f   asihpi32:ASIHPI32.dll
 0001:00037240       _HPI_MixerOpen@12          10038240 f   asihpi32:ASIHPI32.dll
 0001:00037246       _HPI_MixerClose@8          10038246 f   asihpi32:ASIHPI32.dll
 0001:0003724c       _HPI_MixerGetControlByIndex@36 1003824c f   asihpi32:ASIHPI32.dll
 0001:00037252       _HPI_MixerStore@16         10038252 f   asihpi32:ASIHPI32.dll
 0001:00037258       _HPI_VolumeSetGain@12      10038258 f   asihpi32:ASIHPI32.dll
 0001:0003725e       _HPI_VolumeGetGain@12      1003825e f   asihpi32:ASIHPI32.dll
 0001:00037264       _HPI_VolumeSetMute@12      10038264 f   asihpi32:ASIHPI32.dll
 0001:0003726a       _HPI_VolumeGetMute@12      1003826a f   asihpi32:ASIHPI32.dll
 0001:00037270       _HPI_VolumeQueryRange@20   10038270 f   asihpi32:ASIHPI32.dll
 0001:00037276       _HPI_Volume_QueryChannels@12 10038276 f   asihpi32:ASIHPI32.dll
 0001:0003727c       _HPI_VolumeAutoFadeProfile@20 1003827c f   asihpi32:ASIHPI32.dll
 0001:00037282       _HPI_LevelQueryRange@20    10038282 f   asihpi32:ASIHPI32.dll
 0001:00037288       _HPI_LevelSetGain@12       10038288 f   asihpi32:ASIHPI32.dll
 0001:0003728e       _HPI_LevelGetGain@12       1003828e f   asihpi32:ASIHPI32.dll
 0001:00037294       _HPI_Meter_QueryChannels@12 10038294 f   asihpi32:ASIHPI32.dll
 0001:0003729a       _HPI_MeterGetPeak@12       1003829a f   asihpi32:ASIHPI32.dll
 0001:000372a0       _HPI_MeterGetRms@12        100382a0 f   asihpi32:ASIHPI32.dll
 0001:000372a6       _HPI_MeterSetPeakBallistics@16 100382a6 f   asihpi32:ASIHPI32.dll
 0001:000372ac       _HPI_MeterSetRmsBallistics@16 100382ac f   asihpi32:ASIHPI32.dll
 0001:000372b2       _HPI_MeterGetPeakBallistics@16 100382b2 f   asihpi32:ASIHPI32.dll
 0001:000372b8       _HPI_MeterGetRmsBallistics@16 100382b8 f   asihpi32:ASIHPI32.dll
 0001:000372be       _HPI_ChannelMode_QueryMode@16 100382be f   asihpi32:ASIHPI32.dll
 0001:000372c4       _HPI_ChannelModeSet@12     100382c4 f   asihpi32:ASIHPI32.dll
 0001:000372ca       _HPI_ChannelModeGet@12     100382ca f   asihpi32:ASIHPI32.dll
 0001:000372d0       _HPI_Tuner_QueryBand@16    100382d0 f   asihpi32:ASIHPI32.dll
 0001:000372d6       _HPI_Tuner_SetBand@12      100382d6 f   asihpi32:ASIHPI32.dll
 0001:000372dc       _HPI_Tuner_GetBand@12      100382dc f   asihpi32:ASIHPI32.dll
 0001:000372e2       _HPI_Tuner_QueryFrequency@20 100382e2 f   asihpi32:ASIHPI32.dll
 0001:000372e8       _HPI_Tuner_SetFrequency@12 100382e8 f   asihpi32:ASIHPI32.dll
 0001:000372ee       _HPI_Tuner_GetFrequency@12 100382ee f   asihpi32:ASIHPI32.dll
 0001:000372f4       _HPI_Tuner_SetGain@12      100382f4 f   asihpi32:ASIHPI32.dll
 0001:000372fa       _HPI_Tuner_GetGain@12      100382fa f   asihpi32:ASIHPI32.dll
 0001:00037300       _HPI_Tuner_GetRFLevel@12   10038300 f   asihpi32:ASIHPI32.dll
 0001:00037306       _HPI_Tuner_GetRawRFLevel@12 10038306 f   asihpi32:ASIHPI32.dll
 0001:0003730c       _HPI_Tuner_GetStatus@16    1003830c f   asihpi32:ASIHPI32.dll
 0001:00037312       _HPI_Tuner_SetMode@16      10038312 f   asihpi32:ASIHPI32.dll
 0001:00037318       _HPI_Tuner_GetMode@16      10038318 f   asihpi32:ASIHPI32.dll
 0001:0003731e       _HPI_Tuner_QueryDeemphasis@20 1003831e f   asihpi32:ASIHPI32.dll
 0001:00037324       _HPI_Tuner_SetDeemphasis@12 10038324 f   asihpi32:ASIHPI32.dll
 0001:0003732a       _HPI_Tuner_GetDeemphasis@12 1003832a f   asihpi32:ASIHPI32.dll
 0001:00037330       _HPI_Tuner_QueryProgram@12 10038330 f   asihpi32:ASIHPI32.dll
 0001:00037336       _HPI_Tuner_SetProgram@12   10038336 f   asihpi32:ASIHPI32.dll
 0001:0003733c       _HPI_Tuner_GetProgram@12   1003833c f   asihpi32:ASIHPI32.dll
 0001:00037342       _HPI_Tuner_GetFirmwareVersion@16 10038342 f   asihpi32:ASIHPI32.dll
 0001:00037348       _HPI_Tuner_GetHdRadioSignalQuality@12 10038348 f   asihpi32:ASIHPI32.dll
 0001:0003734e       _HPI_Tuner_GetHdRadioSignalBlend@12 1003834e f   asihpi32:ASIHPI32.dll
 0001:00037354       _HPI_Tuner_SetHdRadioSignalBlend@12 10038354 f   asihpi32:ASIHPI32.dll
 0001:0003735a       _HPI_Tuner_GetDabAudioServiceCount@16 1003835a f   asihpi32:ASIHPI32.dll
 0001:00037360       _HPI_Tuner_SetDabAudioService@12 10038360 f   asihpi32:ASIHPI32.dll
 0001:00037366       _HPI_Tuner_GetDabAudioServiceName@20 10038366 f   asihpi32:ASIHPI32.dll
 0001:0003736c       _HPI_Tuner_GetDabMultiplexName@16 1003836c f   asihpi32:ASIHPI32.dll
 0001:00037372       _HPI_Tuner_GetDabAudioInfo@16 10038372 f   asihpi32:ASIHPI32.dll
 0001:00037378       _HPI_PAD_GetChannelName@16 10038378 f   asihpi32:ASIHPI32.dll
 0001:0003737e       _HPI_PAD_GetArtist@16      1003837e f   asihpi32:ASIHPI32.dll
 0001:00037384       _HPI_PAD_GetTitle@16       10038384 f   asihpi32:ASIHPI32.dll
 0001:0003738a       _HPI_PAD_GetComment@16     1003838a f   asihpi32:ASIHPI32.dll
 0001:00037390       _HPI_PAD_GetProgramType@12 10038390 f   asihpi32:ASIHPI32.dll
 0001:00037396       _HPI_PAD_GetRdsPI@12       10038396 f   asihpi32:ASIHPI32.dll
 0001:0003739c       _HPI_PAD_GetProgramTypeString@24 1003839c f   asihpi32:ASIHPI32.dll
 0001:000373a2       _HPI_AESEBU_Receiver_QueryFormat@16 100383a2 f   asihpi32:ASIHPI32.dll
 0001:000373a8       _HPI_AESEBU_Receiver_SetFormat@12 100383a8 f   asihpi32:ASIHPI32.dll
 0001:000373ae       _HPI_AESEBU_Receiver_GetFormat@12 100383ae f   asihpi32:ASIHPI32.dll
 0001:000373b4       _HPI_AESEBU_Receiver_GetSampleRate@12 100383b4 f   asihpi32:ASIHPI32.dll
 0001:000373ba       _HPI_AESEBU_Receiver_GetErrorStatus@12 100383ba f   asihpi32:ASIHPI32.dll
 0001:000373c0       _HPI_AESEBU_Transmitter_SetChannelStatus@16 100383c0 f   asihpi32:ASIHPI32.dll
 0001:000373c6       _HPI_AESEBU_Transmitter_QueryFormat@16 100383c6 f   asihpi32:ASIHPI32.dll
 0001:000373cc       _HPI_AESEBU_Transmitter_SetFormat@12 100383cc f   asihpi32:ASIHPI32.dll
 0001:000373d2       _HPI_AESEBU_Transmitter_GetFormat@12 100383d2 f   asihpi32:ASIHPI32.dll
 0001:000373d8       _HPI_Multiplexer_SetSource@16 100383d8 f   asihpi32:ASIHPI32.dll
 0001:000373de       _HPI_Multiplexer_GetSource@16 100383de f   asihpi32:ASIHPI32.dll
 0001:000373e4       _HPI_Multiplexer_QuerySource@20 100383e4 f   asihpi32:ASIHPI32.dll
 0001:000373ea       _HPI_VoxSetThreshold@12    100383ea f   asihpi32:ASIHPI32.dll
 0001:000373f0       _HPI_VoxGetThreshold@12    100383f0 f   asihpi32:ASIHPI32.dll
 0001:000373f6       _HPI_SampleClock_QuerySource@16 100383f6 f   asihpi32:ASIHPI32.dll
 0001:000373fc       _HPI_SampleClock_SetSource@12 100383fc f   asihpi32:ASIHPI32.dll
 0001:00037402       _HPI_SampleClock_GetSource@12 10038402 f   asihpi32:ASIHPI32.dll
 0001:00037408       _HPI_SampleClock_QuerySourceIndex@20 10038408 f   asihpi32:ASIHPI32.dll
 0001:0003740e       _HPI_SampleClock_SetSourceIndex@12 1003840e f   asihpi32:ASIHPI32.dll
 0001:00037414       _HPI_SampleClock_GetSourceIndex@12 10038414 f   asihpi32:ASIHPI32.dll
 0001:0003741a       _HPI_SampleClock_GetSampleRate@12 1003841a f   asihpi32:ASIHPI32.dll
 0001:00037420       _HPI_SampleClock_QueryLocalRate@16 10038420 f   asihpi32:ASIHPI32.dll
 0001:00037426       _HPI_SampleClock_SetLocalRate@12 10038426 f   asihpi32:ASIHPI32.dll
 0001:0003742c       _HPI_SampleClock_GetLocalRate@12 1003842c f   asihpi32:ASIHPI32.dll
 0001:00037432       _HPI_SampleClock_SetAuto@12 10038432 f   asihpi32:ASIHPI32.dll
 0001:00037438       _HPI_SampleClock_GetAuto@12 10038438 f   asihpi32:ASIHPI32.dll
 0001:0003743e       _HPI_SampleClock_SetLocalRateLock@12 1003843e f   asihpi32:ASIHPI32.dll
 0001:00037444       _HPI_SampleClock_GetLocalRateLock@12 10038444 f   asihpi32:ASIHPI32.dll
 0001:0003744a       _HPI_Microphone_SetPhantomPower@12 1003844a f   asihpi32:ASIHPI32.dll
 0001:00037450       _HPI_Microphone_GetPhantomPower@12 10038450 f   asihpi32:ASIHPI32.dll
 0001:00037456       _HPI_ParametricEQ_GetInfo@16 10038456 f   asihpi32:ASIHPI32.dll
 0001:0003745c       _HPI_ParametricEQ_SetState@12 1003845c f   asihpi32:ASIHPI32.dll
 0001:00037462       _HPI_ParametricEQ_SetBand@28 10038462 f   asihpi32:ASIHPI32.dll
 0001:00037468       _HPI_ParametricEQ_GetBand@28 10038468 f   asihpi32:ASIHPI32.dll
 0001:0003746e       _HPI_Compander_SetEnable@12 1003846e f   asihpi32:ASIHPI32.dll
 0001:00037474       _HPI_Compander_GetEnable@12 10038474 f   asihpi32:ASIHPI32.dll
 0001:0003747a       _HPI_Compander_SetMakeupGain@12 1003847a f   asihpi32:ASIHPI32.dll
 0001:00037480       _HPI_Compander_GetMakeupGain@12 10038480 f   asihpi32:ASIHPI32.dll
 0001:00037486       _HPI_Compander_SetAttackTimeConstant@16 10038486 f   asihpi32:ASIHPI32.dll
 0001:0003748c       _HPI_Compander_GetAttackTimeConstant@16 1003848c f   asihpi32:ASIHPI32.dll
 0001:00037492       _HPI_Compander_SetDecayTimeConstant@16 10038492 f   asihpi32:ASIHPI32.dll
 0001:00037498       _HPI_Compander_GetDecayTimeConstant@16 10038498 f   asihpi32:ASIHPI32.dll
 0001:0003749e       _HPI_Compander_SetThreshold@16 1003849e f   asihpi32:ASIHPI32.dll
 0001:000374a4       _HPI_Compander_GetThreshold@16 100384a4 f   asihpi32:ASIHPI32.dll
 0001:000374aa       _HPI_Compander_SetRatio@16 100384aa f   asihpi32:ASIHPI32.dll
 0001:000374b0       _HPI_Compander_GetRatio@16 100384b0 f   asihpi32:ASIHPI32.dll
 0001:000374b6       _HPI_Cobranet_HmiWrite@20  100384b6 f   asihpi32:ASIHPI32.dll
 0001:000374bc       _HPI_Cobranet_HmiRead@24   100384bc f   asihpi32:ASIHPI32.dll
 0001:000374c2       _HPI_Cobranet_GetIPaddress@12 100384c2 f   asihpi32:ASIHPI32.dll
 0001:000374c8       _HPI_Cobranet_GetMACaddress@16 100384c8 f   asihpi32:ASIHPI32.dll
 0001:000374ce       _HPI_ToneDetector_GetState@12 100384ce f   asihpi32:ASIHPI32.dll
 0001:000374d4       _HPI_ToneDetector_SetEnable@12 100384d4 f   asihpi32:ASIHPI32.dll
 0001:000374da       _HPI_ToneDetector_GetEnable@12 100384da f   asihpi32:ASIHPI32.dll
 0001:000374e0       _HPI_ToneDetector_SetEventEnable@12 100384e0 f   asihpi32:ASIHPI32.dll
 0001:000374e6       _HPI_ToneDetector_GetEventEnable@12 100384e6 f   asihpi32:ASIHPI32.dll
 0001:000374ec       _HPI_ToneDetector_SetThreshold@12 100384ec f   asihpi32:ASIHPI32.dll
 0001:000374f2       _HPI_ToneDetector_GetThreshold@12 100384f2 f   asihpi32:ASIHPI32.dll
 0001:000374f8       _HPI_ToneDetector_GetFrequency@16 100384f8 f   asihpi32:ASIHPI32.dll
 0001:000374fe       _HPI_SilenceDetector_GetState@12 100384fe f   asihpi32:ASIHPI32.dll
 0001:00037504       _HPI_SilenceDetector_SetEnable@12 10038504 f   asihpi32:ASIHPI32.dll
 0001:0003750a       _HPI_SilenceDetector_GetEnable@12 1003850a f   asihpi32:ASIHPI32.dll
 0001:00037510       _HPI_SilenceDetector_SetEventEnable@12 10038510 f   asihpi32:ASIHPI32.dll
 0001:00037516       _HPI_SilenceDetector_GetEventEnable@12 10038516 f   asihpi32:ASIHPI32.dll
 0001:0003751c       _HPI_SilenceDetector_SetDelay@12 1003851c f   asihpi32:ASIHPI32.dll
 0001:00037522       _HPI_SilenceDetector_GetDelay@12 10038522 f   asihpi32:ASIHPI32.dll
 0001:00037528       _HPI_SilenceDetector_SetThreshold@12 10038528 f   asihpi32:ASIHPI32.dll
 0001:0003752e       _HPI_SilenceDetector_GetThreshold@12 1003852e f   asihpi32:ASIHPI32.dll
 0001:00037534       _HPI_Universal_Info@12     10038534 f   asihpi32:ASIHPI32.dll
 0001:0003753a       _HPI_Universal_Get@12      1003853a f   asihpi32:ASIHPI32.dll
 0001:00037540       _HPI_Universal_Set@12      10038540 f   asihpi32:ASIHPI32.dll
 0001:00037546       _HPI_ProfileOpenAll@20     10038546 f   asihpi32:ASIHPI32.dll
 0001:0003754c       _HPI_ProfileGetUtilization@12 1003854c f   asihpi32:ASIHPI32.dll
 0001:00037552       _HPI_GetErrorText@8        10038552 f   asihpi32:ASIHPI32.dll
 0001:00037558       _HPI_HandleToIndexes@12    10038558 f   asihpi32:ASIHPI32.dll
 0001:0003755e       _HPI_Message@8             1003855e f   asihpi32:ASIHPI32.dll
 0001:00037564       _HPI_ControlParamGet@28    10038564 f   asihpi32:ASIHPI32.dll
 0001:0003756a       _HPI_InitMessageResponse@16 1003856a f   asihpi32:ASIHPI32.dll
 0001:00037570       _HPI_OutStreamOpen@16      10038570 f   asihpi32:ASIHPI32.dll
 0001:00037576       _HPI_OutStreamClose@8      10038576 f   asihpi32:ASIHPI32.dll
 0001:0003757c       _HPI_OutStreamGetInfoEx@28 1003857c f   asihpi32:ASIHPI32.dll
 0001:00037582       _HPI_OutStreamWriteBuf@20  10038582 f   asihpi32:ASIHPI32.dll
 0001:00037588       _HPI_OutStreamStart@8      10038588 f   asihpi32:ASIHPI32.dll
 0001:0003758e       _HPI_OutStreamStop@8       1003858e f   asihpi32:ASIHPI32.dll
 0001:00037594       _HPI_OutStreamReset@8      10038594 f   asihpi32:ASIHPI32.dll
 0001:0003759a       _HPI_OutStreamQueryFormat@12 1003859a f   asihpi32:ASIHPI32.dll
 0001:000375a0       _HPI_OutStreamSetTimeScale@12 100385a0 f   asihpi32:ASIHPI32.dll
 0001:000375a6       _HPI_OutStreamHostBufferAllocate@12 100385a6 f   asihpi32:ASIHPI32.dll
 0001:000375ac       _HPI_OutStreamHostBufferFree@8 100385ac f   asihpi32:ASIHPI32.dll
 0001:000375b2       _HPI_WaveFormatToHpiFormat@8 100385b2 f   asihpi32:ASIHPI32.dll
 0001:000375b8       _HPI_OutStreamWait@12      100385b8 f   asihpi32:ASIHPI32.dll
 0001:000375be       _HPI_InStreamOpen@16       100385be f   asihpi32:ASIHPI32.dll
 0001:000375c4       _HPI_InStreamClose@8       100385c4 f   asihpi32:ASIHPI32.dll
 0001:000375ca       _HPI_InStreamQueryFormat@12 100385ca f   asihpi32:ASIHPI32.dll
 0001:000375d0       _HPI_InStreamSetFormat@12  100385d0 f   asihpi32:ASIHPI32.dll
 0001:000375d6       _HPI_InStreamReadBuf@16    100385d6 f   asihpi32:ASIHPI32.dll
 0001:000375dc       _HPI_InStreamStart@8       100385dc f   asihpi32:ASIHPI32.dll
 0001:000375e2       _HPI_InStreamStop@8        100385e2 f   asihpi32:ASIHPI32.dll
 0001:000375e8       _HPI_InStreamReset@8       100385e8 f   asihpi32:ASIHPI32.dll
 0001:000375ee       _HPI_InStreamGetInfoEx@28  100385ee f   asihpi32:ASIHPI32.dll
 0001:000375f4       _HPI_InStreamHostBufferAllocate@12 100385f4 f   asihpi32:ASIHPI32.dll
 0001:000375fa       _HPI_InStreamHostBufferFree@8 100385fa f   asihpi32:ASIHPI32.dll
 0001:00037600       _HPI_FormatCreate@24       10038600 f   asihpi32:ASIHPI32.dll
 0001:00037606       _HPI_InStreamWait@12       10038606 f   asihpi32:ASIHPI32.dll
 0001:0003760c       _SnmpSetTranslateMode@4    1003860c f   wsnmp32:wsnmp32.dll
 0001:00037612       _SnmpSetRetransmitMode@4   10038612 f   wsnmp32:wsnmp32.dll
 0001:00037618       _SnmpSetTimeout@8          10038618 f   wsnmp32:wsnmp32.dll
 0001:0003761e       _SnmpGetRetry@12           1003861e f   wsnmp32:wsnmp32.dll
 0001:00037624       _SnmpSetRetry@8            10038624 f   wsnmp32:wsnmp32.dll
 0001:0003762a       _SnmpStartup@20            1003862a f   wsnmp32:wsnmp32.dll
 0001:00037630       _SnmpCleanup@0             10038630 f   wsnmp32:wsnmp32.dll
 0001:00037636       _SnmpClose@4               10038636 f   wsnmp32:wsnmp32.dll
 0001:0003763c       _SnmpSendMsg@20            1003863c f   wsnmp32:wsnmp32.dll
 0001:00037642       _SnmpRecvMsg@20            10038642 f   wsnmp32:wsnmp32.dll
 0001:00037648       _SnmpCreateSession@16      10038648 f   wsnmp32:wsnmp32.dll
 0001:0003764e       _SnmpCancelMsg@8           1003864e f   wsnmp32:wsnmp32.dll
 0001:00037654       _SnmpStrToEntity@8         10038654 f   wsnmp32:wsnmp32.dll
 0001:0003765a       _SnmpFreeEntity@4          1003865a f   wsnmp32:wsnmp32.dll
 0001:00037660       _SnmpStrToContext@8        10038660 f   wsnmp32:wsnmp32.dll
 0001:00037666       _SnmpFreeContext@4         10038666 f   wsnmp32:wsnmp32.dll
 0001:0003766c       _SnmpCreatePdu@24          1003866c f   wsnmp32:wsnmp32.dll
 0001:00037672       _SnmpGetPduData@24         10038672 f   wsnmp32:wsnmp32.dll
 0001:00037678       _SnmpFreePdu@4             10038678 f   wsnmp32:wsnmp32.dll
 0001:0003767e       _SnmpCreateVbl@12          1003867e f   wsnmp32:wsnmp32.dll
 0001:00037684       _SnmpFreeVbl@4             10038684 f   wsnmp32:wsnmp32.dll
 0001:0003768a       _SnmpCountVbl@4            1003868a f   wsnmp32:wsnmp32.dll
 0001:00037690       _SnmpGetVb@16              10038690 f   wsnmp32:wsnmp32.dll
 0001:00037696       _SnmpSetVb@16              10038696 f   wsnmp32:wsnmp32.dll
 0001:0003769c       _SnmpGetLastError@4        1003869c f   wsnmp32:wsnmp32.dll
 0001:000376a2       _SnmpOidToStr@12           100386a2 f   wsnmp32:wsnmp32.dll
 0001:000376a8       _SnmpFreeDescriptor@8      100386a8 f   wsnmp32:wsnmp32.dll
 0001:000376ae       _inet_ntoa@4               100386ae f   wsock32:WSOCK32.dll
 0001:000376b4       _gethostbyname@4           100386b4 f   wsock32:WSOCK32.dll
 0001:000376ba       _DirectSoundEnumerateA@8   100386ba f   dsound:DSOUND.dll
 0001:000376c0       _DirectSoundCaptureEnumerateA@8 100386c0 f   dsound:DSOUND.dll
 0001:000376c6       _DirectSoundCreate@12      100386c6 f   dsound:DSOUND.dll
 0001:000376cc       _DirectSoundCaptureCreate@12 100386cc f   dsound:DSOUND.dll
 0001:000376d2       __imp_load__create_net_interface@0 100386d2 f   avdecc-lib_controller32:avdecc-lib_controller32.dll
 0001:000376dc       __tailMerge_avdecc_lib_controller32_dll 100386dc f i avdecc-lib_controller32:avdecc-lib_controller32.dll
 0001:000376ed       _create_net_interface@0    100386ed f   avdecc-lib_controller32:avdecc-lib_controller32.dll
 0001:000376f3       __imp_load__create_controller@16 100386f3 f   avdecc-lib_controller32:avdecc-lib_controller32.dll
 0001:000376fd       _create_controller@16      100386fd f   avdecc-lib_controller32:avdecc-lib_controller32.dll
 0001:00037703       __imp_load__create_system@12 10038703 f   avdecc-lib_controller32:avdecc-lib_controller32.dll
 0001:0003770d       _create_system@12          1003870d f   avdecc-lib_controller32:avdecc-lib_controller32.dll
 0001:00037713       __imp_load_?aem_cmd_value_to_name@utility@avdecc_lib@@YGPBDG@Z 10038713 f   avdecc-lib_controller32:avdecc-lib_controller32.dll
 0001:0003771d       ?aem_cmd_value_to_name@utility@avdecc_lib@@YGPBDG@Z 1003871d f   avdecc-lib_controller32:avdecc-lib_controller32.dll
 0001:00037723       __imp_load_?aem_desc_value_to_name@utility@avdecc_lib@@YGPBDG@Z 10038723 f   avdecc-lib_controller32:avdecc-lib_controller32.dll
 0001:0003772d       ?aem_desc_value_to_name@utility@avdecc_lib@@YGPBDG@Z 1003872d f   avdecc-lib_controller32:avdecc-lib_controller32.dll
 0001:00037733       __imp_load_?aem_cmd_status_value_to_name@utility@avdecc_lib@@YGPBDI@Z 10038733 f   avdecc-lib_controller32:avdecc-lib_controller32.dll
 0001:0003773d       ?aem_cmd_status_value_to_name@utility@avdecc_lib@@YGPBDI@Z 1003873d f   avdecc-lib_controller32:avdecc-lib_controller32.dll
 0001:00037743       __imp_load_?acmp_cmd_value_to_name@utility@avdecc_lib@@YGPBDI@Z 10038743 f   avdecc-lib_controller32:avdecc-lib_controller32.dll
 0001:0003774d       ?acmp_cmd_value_to_name@utility@avdecc_lib@@YGPBDI@Z 1003874d f   avdecc-lib_controller32:avdecc-lib_controller32.dll
 0001:00037753       __imp_load_?acmp_cmd_status_value_to_name@utility@avdecc_lib@@YGPBDI@Z 10038753 f   avdecc-lib_controller32:avdecc-lib_controller32.dll
 0001:0003775d       ?acmp_cmd_status_value_to_name@utility@avdecc_lib@@YGPBDI@Z 1003875d f   avdecc-lib_controller32:avdecc-lib_controller32.dll
 0001:00037763       __imp_load_?notification_value_to_name@utility@avdecc_lib@@YGPBDG@Z 10038763 f   avdecc-lib_controller32:avdecc-lib_controller32.dll
 0001:0003776d       ?notification_value_to_name@utility@avdecc_lib@@YGPBDG@Z 1003876d f   avdecc-lib_controller32:avdecc-lib_controller32.dll
 0001:00037774       _GetProcAddress@8          10038774 f   kernel32:KERNEL32.dll
 0001:0003777a       _LoadLibraryA@4            1003877a f   kernel32:KERNEL32.dll
 0001:00037780       _CloseHandle@4             10038780 f   kernel32:KERNEL32.dll
 0001:00037786       _QueryPerformanceCounter@4 10038786 f   kernel32:KERNEL32.dll
 0001:0003778c       _QueryPerformanceFrequency@4 1003878c f   kernel32:KERNEL32.dll
 0001:00037792       _ReleaseSemaphore@12       10038792 f   kernel32:KERNEL32.dll
 0001:00037798       _ReleaseMutex@4            10038798 f   kernel32:KERNEL32.dll
 0001:0003779e       _WaitForSingleObject@8     1003879e f   kernel32:KERNEL32.dll
 0001:000377a4       _CreateMutexA@12           100387a4 f   kernel32:KERNEL32.dll
 0001:000377aa       _Sleep@4                   100387aa f   kernel32:KERNEL32.dll
 0001:000377b0       _GetCurrentProcess@0       100387b0 f   kernel32:KERNEL32.dll
 0001:000377b6       _CreateThread@24           100387b6 f   kernel32:KERNEL32.dll
 0001:000377bc       _SetPriorityClass@8        100387bc f   kernel32:KERNEL32.dll
 0001:000377c2       _GetPriorityClass@4        100387c2 f   kernel32:KERNEL32.dll
 0001:000377c8       _CreateSemaphoreA@16       100387c8 f   kernel32:KERNEL32.dll
 0001:000377ce       _SetEvent@4                100387ce f   kernel32:KERNEL32.dll
 0001:000377d4       _CreateEventA@16           100387d4 f   kernel32:KERNEL32.dll
 0001:000377da       _MultiByteToWideChar@24    100387da f   kernel32:KERNEL32.dll
 0001:000377e0       _OutputDebugStringA@4      100387e0 f   kernel32:KERNEL32.dll
 0001:000377e6       _GetCurrentProcessId@0     100387e6 f   kernel32:KERNEL32.dll
 0001:000377ec       _GetCurrentThread@0        100387ec f   kernel32:KERNEL32.dll
 0001:000377f2       _SetThreadPriority@8       100387f2 f   kernel32:KERNEL32.dll
 0001:000377f8       _GetLastError@0            100387f8 f   kernel32:KERNEL32.dll
 0001:000377fe       _LocalFree@4               100387fe f   kernel32:KERNEL32.dll
 0001:00037804       _FormatMessageA@28         10038804 f   kernel32:KERNEL32.dll
 0001:0003780a       _LocalAlloc@8              1003880a f   kernel32:KERNEL32.dll
 0001:00037810       _CreateFileA@28            10038810 f   kernel32:KERNEL32.dll
 0001:00037816       _ReadFile@20               10038816 f   kernel32:KERNEL32.dll
 0001:0003781c       _SetFilePointer@16         1003881c f   kernel32:KERNEL32.dll
 0001:00037822       _WriteFile@20              10038822 f   kernel32:KERNEL32.dll
 0001:00037828       _GetDesktopWindow@0        10038828 f   user32:USER32.dll
 0001:0003782e       _EnumChildWindows@12       1003882e f   user32:USER32.dll
 0001:00037834       _GetWindowThreadProcessId@8 10038834 f   user32:USER32.dll
 0001:0003783a       _RegCloseKey@4             1003883a f   advapi32:ADVAPI32.dll
 0001:00037840       _RegCreateKeyA@12          10038840 f   advapi32:ADVAPI32.dll
 0001:00037846       _RegDeleteValueA@8         10038846 f   advapi32:ADVAPI32.dll
 0001:0003784c       _RegEnumValueA@32          1003884c f   advapi32:ADVAPI32.dll
 0001:00037852       _RegQueryInfoKeyA@48       10038852 f   advapi32:ADVAPI32.dll
 0001:00037858       _RegQueryValueExA@24       10038858 f   advapi32:ADVAPI32.dll
 0001:0003785e       _RegSetValueExA@24         1003885e f   advapi32:ADVAPI32.dll
 0001:00037864       _RegOpenKeyExA@20          10038864 f   advapi32:ADVAPI32.dll
 0001:0003786a       _CoCreateInstance@20       1003886a f   ole32:ole32.dll
 0001:00037870       _CLSIDFromString@8         10038870 f   ole32:ole32.dll
 0001:00037876       _CoInitialize@4            10038876 f   ole32:ole32.dll
 0001:0003787c       ??$PFromRva@PAP6GHXZ@@YGPAP6GHXZK@Z 1003887c f i Delayimp:delayhlp.obj
 0001:0003788e       ??$PFromRva@PAPAUHINSTANCE__@@@@YGPAPAUHINSTANCE__@@K@Z 1003888e f i Delayimp:delayhlp.obj
 0001:000378a0       ??$PFromRva@PAU_IMAGE_IMPORT_BY_NAME@@@@YGPAU_IMAGE_IMPORT_BY_NAME@@K@Z 100388a0 f i Delayimp:delayhlp.obj
 0001:000378b2       ??$PFromRva@PAU_IMAGE_THUNK_DATA32@@@@YGPAU_IMAGE_THUNK_DATA32@@K@Z 100388b2 f i Delayimp:delayhlp.obj
 0001:000378c4       ??$PFromRva@PBD@@YGPBDK@Z  100388c4 f i Delayimp:delayhlp.obj
 0001:000378d6       ??$PFromRva@PBUImgDelayDescr@@@@YGPBUImgDelayDescr@@K@Z 100388d6 f i Delayimp:delayhlp.obj
 0001:000378e8       ??$PFromRva@PBU_IMAGE_THUNK_DATA32@@@@YGPBU_IMAGE_THUNK_DATA32@@K@Z 100388e8 f i Delayimp:delayhlp.obj
 0001:000378fa       ?CountOfImports@@YGIPBU_IMAGE_THUNK_DATA32@@@Z 100388fa f i Delayimp:delayhlp.obj
 0001:0003792c       ?IndexFromPImgThunkData@@YGIPBU_IMAGE_THUNK_DATA32@@0@Z 1003892c f i Delayimp:delayhlp.obj
 0001:00037a86       _HRESULT_FROM_WIN32@4      10038a86 f i Delayimp:delayhlp.obj
 0001:00037a9e       ___FUnloadDelayLoadedDLL2@4 10038a9e f   Delayimp:delayhlp.obj
 0001:00037b12       ___HrLoadAllImportsForDll@4 10038b12 f   Delayimp:delayhlp.obj
 0001:00037b74       ___delayLoadHelper2@8      10038b74 f   Delayimp:delayhlp.obj
 0001:00037d86       ___raise_securityfailure   10038d86 f   LIBCMT:gs_report.obj
 0001:00037dc3       ___report_gsfailure        10038dc3 f   LIBCMT:gs_report.obj
 0001:00037ebe       ___report_rangecheckfailure 10038ebe f   LIBCMT:gs_report.obj
 0001:00037eca       ___report_securityfailure  10038eca f   LIBCMT:gs_report.obj
 0001:00037f9a       ___report_securityfailureEx 10038f9a f   LIBCMT:gs_report.obj
 0001:000380b0       ??0_LocaleUpdate@@QAE@PAUlocaleinfo_struct@@@Z 100390b0 f i LIBCMT:_ctype.obj
 0001:00038138       ??1_LocaleUpdate@@QAE@XZ   10039138 f i LIBCMT:_ctype.obj
 0001:00038146       ?GetLocaleT@_LocaleUpdate@@QAEPAUlocaleinfo_struct@@XZ 10039146 f i LIBCMT:_ctype.obj
 0001:00038149       ___isascii                 10039149 f i LIBCMT:_ctype.obj
 0001:00038159       ___iscsym                  10039159 f i LIBCMT:_ctype.obj
 0001:00038179       ___iscsymf                 10039179 f i LIBCMT:_ctype.obj
 0001:00038196       ___toascii                 10039196 f i LIBCMT:_ctype.obj
 0001:000381a1       __isalnum_l                100391a1 f i LIBCMT:_ctype.obj
 0001:000381f9       __isalpha_l                100391f9 f i LIBCMT:_ctype.obj
 0001:00038251       __isblank_l                10039251 f i LIBCMT:_ctype.obj
 0001:000382ab       __iscntrl_l                100392ab f i LIBCMT:_ctype.obj
 0001:000382fd       __iscsym_l                 100392fd f i LIBCMT:_ctype.obj
 0001:0003831e       __iscsymf_l                1003931e f i LIBCMT:_ctype.obj
 0001:0003833f       __isdigit_l                1003933f f i LIBCMT:_ctype.obj
 0001:00038391       __isgraph_l                10039391 f i LIBCMT:_ctype.obj
 0001:000383e9       __islower_l                100393e9 f i LIBCMT:_ctype.obj
 0001:0003843b       __isprint_l                1003943b f i LIBCMT:_ctype.obj
 0001:00038493       __ispunct_l                10039493 f i LIBCMT:_ctype.obj
 0001:000384e5       __isspace_l                100394e5 f i LIBCMT:_ctype.obj
 0001:00038537       __isupper_l                10039537 f i LIBCMT:_ctype.obj
 0001:00038589       __isxdigit_l               10039589 f i LIBCMT:_ctype.obj
 0001:000385e1       _isalnum                   100395e1 f i LIBCMT:_ctype.obj
 0001:0003860e       _isalpha                   1003960e f i LIBCMT:_ctype.obj
 0001:0003863b       _isblank                   1003963b f i LIBCMT:_ctype.obj
 0001:00038670       _iscntrl                   10039670 f i LIBCMT:_ctype.obj
 0001:0003869b       _isdigit                   1003969b f i LIBCMT:_ctype.obj
 0001:000386c6       _isgraph                   100396c6 f i LIBCMT:_ctype.obj
 0001:000386f3       _islower                   100396f3 f i LIBCMT:_ctype.obj
 0001:0003871e       _isprint                   1003971e f i LIBCMT:_ctype.obj
 0001:0003874b       _ispunct                   1003974b f i LIBCMT:_ctype.obj
 0001:00038776       _isspace                   10039776 f i LIBCMT:_ctype.obj
 0001:000387a1       _isupper                   100397a1 f i LIBCMT:_ctype.obj
 0001:000387cc       _isxdigit                  100397cc f i LIBCMT:_ctype.obj
 0001:00038800       _strncpy                   10039800 f   LIBCMT:strncpy.obj
 0001:00038b4a       __strtol_l                 10039b4a f   LIBCMT:strtol.obj
 0001:00038b65       __strtoul_l                10039b65 f   LIBCMT:strtol.obj
 0001:00038b80       _strtol                    10039b80 f   LIBCMT:strtol.obj
 0001:00038baa       _strtoul                   10039baa f   LIBCMT:strtol.obj
 0001:00038bd4       __scprintf                 10039bd4 f   LIBCMT:sprintf.obj
 0001:00038be7       __scprintf_l               10039be7 f   LIBCMT:sprintf.obj
 0001:00038bfe       __scprintf_p               10039bfe f   LIBCMT:sprintf.obj
 0001:00038c11       __scprintf_p_l             10039c11 f   LIBCMT:sprintf.obj
 0001:00038c28       __snprintf_s               10039c28 f   LIBCMT:sprintf.obj
 0001:00038c47       __snprintf_s_l             10039c47 f   LIBCMT:sprintf.obj
 0001:00038c67       __sprintf_l                10039c67 f   LIBCMT:sprintf.obj
 0001:00038c81       __sprintf_p                10039c81 f   LIBCMT:sprintf.obj
 0001:00038c9d       __sprintf_p_l              10039c9d f   LIBCMT:sprintf.obj
 0001:00038cba       __sprintf_s_l              10039cba f   LIBCMT:sprintf.obj
 0001:00038cd7       _sprintf                   10039cd7 f   LIBCMT:sprintf.obj
 0001:00038d5b       _sprintf_s                 10039d5b f   LIBCMT:sprintf.obj
 0001:00038d77       @__security_check_cookie@4 10039d77 f   LIBCMT:secchk.obj
 0001:00038d90       _memcpy                    10039d90 f   LIBCMT:memcpy.obj
 0001:000393d4       _free                      1003a3d4 f   LIBCMT:free.obj
 0001:0003940c       __heap_alloc               1003a40c f i LIBCMT:malloc.obj
 0001:00039449       _malloc                    1003a449 f   LIBCMT:malloc.obj
 0001:000394db       __get_printf_count_output  1003a4db f   LIBCMT:printf.obj
 0001:000394f0       __printf_l                 1003a4f0 f   LIBCMT:printf.obj
 0001:00039507       __printf_p                 1003a507 f   LIBCMT:printf.obj
 0001:0003951d       __printf_p_l               1003a51d f   LIBCMT:printf.obj
 0001:00039534       __printf_s_l               1003a534 f   LIBCMT:printf.obj
 0001:0003954b       __set_printf_count_output  1003a54b f   LIBCMT:printf.obj
 0001:00039573       _printf                    1003a573 f   LIBCMT:printf.obj
 0001:00039622       _printf_s                  1003a622 f   LIBCMT:printf.obj
 0001:00039638       __vprintf_l                1003a638 f   LIBCMT:vprintf.obj
 0001:00039653       __vprintf_p                1003a653 f   LIBCMT:vprintf.obj
 0001:0003966d       __vprintf_p_l              1003a66d f   LIBCMT:vprintf.obj
 0001:00039688       __vprintf_s_l              1003a688 f   LIBCMT:vprintf.obj
 0001:000396a3       _vprintf                   1003a6a3 f   LIBCMT:vprintf.obj
 0001:000396bd       _vprintf_helper            1003a6bd f   LIBCMT:vprintf.obj
 0001:0003974a       _vprintf_s                 1003a74a f   LIBCMT:vprintf.obj
 0001:00039770       __alldiv                   1003a770 f   LIBCMT:lldiv.obj
 0001:00039820       __allmul                   1003a820 f   LIBCMT:llmul.obj
 0001:00039854       ??0bad_alloc@std@@QAE@ABV01@@Z 1003a854 f i LIBCMT:new.obj
 0001:0003986f       ??0bad_alloc@std@@QAE@XZ   1003a86f f i LIBCMT:new.obj
 0001:00039895       ??1bad_alloc@std@@UAE@XZ   1003a895 f i LIBCMT:new.obj
 0001:000398a0       ??2@YAPAXI@Z               1003a8a0 f   LIBCMT:new.obj
 0001:000398f1       ??_Gbad_alloc@std@@UAEPAXI@Z 1003a8f1 f i LIBCMT:new.obj
 0001:000398f1       ??_Ebad_alloc@std@@UAEPAXI@Z 1003a8f1 f i LIBCMT:new.obj
 0001:00039916       ??3@YAXPAX@Z               1003a916 f   LIBCMT:delete.obj
 0001:00039920       _memmove                   1003a920 f   LIBCMT:memmove.obj
 0001:00039f64       ??_U@YAPAXI@Z              1003af64 f   LIBCMT:new2.obj
 0001:00039f6d       ??_V@YAXPAX@Z              1003af6d f   LIBCMT:delete2.obj
 0001:00039f72       ??0type_info@@AAE@ABV0@@Z  1003af72 f   LIBCMT:typinfo.obj
 0001:00039f7d       ??1type_info@@UAE@XZ       1003af7d f   LIBCMT:typinfo.obj
 0001:00039f8b       ??4type_info@@AAEAAV0@ABV0@@Z 1003af8b f   LIBCMT:typinfo.obj
 0001:00039f90       ??8type_info@@QBE_NABV0@@Z 1003af90 f   LIBCMT:typinfo.obj
 0001:00039fae       ??9type_info@@QBE_NABV0@@Z 1003afae f   LIBCMT:typinfo.obj
 0001:00039fcd       ??_Gtype_info@@UAEPAXI@Z   1003afcd f i LIBCMT:typinfo.obj
 0001:00039fcd       ??_Etype_info@@UAEPAXI@Z   1003afcd f i LIBCMT:typinfo.obj
 0001:00039fec       ?_name_internal_method@type_info@@QBEPBDPAU__type_info_node@@@Z 1003afec f   LIBCMT:typinfo.obj
 0001:00039ffe       ?_type_info_dtor_internal_method@type_info@@QAEXXZ 1003affe f   LIBCMT:typinfo.obj
 0001:0003a006       ?before@type_info@@QBE_NABV1@@Z 1003b006 f   LIBCMT:typinfo.obj
 0001:0003a026       ?name@type_info@@QBEPBDPAU__type_info_node@@@Z 1003b026 f   LIBCMT:typinfo.obj
 0001:0003a038       ?raw_name@type_info@@QBEPBDXZ 1003b038 f   LIBCMT:typinfo.obj
 0001:0003a03c       __fpmath                   1003b03c f   LIBCMT:fpinit.obj
 0001:0003a053       ___setfflag                1003b053 f   LIBCMT:fpinit.obj
 0001:0003a066       __cfltcvt_init             1003b066 f   LIBCMT:fpinit.obj
 0001:0003a0c6       __get_purecall_handler     1003b0c6 f   LIBCMT:purevirt.obj
 0001:0003a0d3       __purecall                 1003b0d3 f   LIBCMT:purevirt.obj
 0001:0003a0f5       __set_purecall_handler     1003b0f5 f   LIBCMT:purevirt.obj
 0001:0003a11a       ___onexitinit              1003b11a f   LIBCMT:onexit.obj
 0001:0003a149       __onexit                   1003b149 f   LIBCMT:onexit.obj
 0001:0003a245       _atexit                    1003b245 f   LIBCMT:onexit.obj
 0001:0003a260       _strstr                    1003b260 f   LIBCMT:strstr.obj
 0001:0003a733       __strtof_l                 1003b733 f   LIBCMT:strtoq.obj
 0001:0003a753       __strtoi64                 1003b753 f   LIBCMT:strtoq.obj
 0001:0003a77d       __strtoi64_l               1003b77d f   LIBCMT:strtoq.obj
 0001:0003a798       __strtoimax_l              1003b798 f   LIBCMT:strtoq.obj
 0001:0003a7a1       __strtold_l                1003b7a1 f   LIBCMT:strtoq.obj
 0001:0003a7aa       __strtoll_l                1003b7aa f   LIBCMT:strtoq.obj
 0001:0003a7b3       __strtoui64                1003b7b3 f   LIBCMT:strtoq.obj
 0001:0003a7dd       __strtoui64_l              1003b7dd f   LIBCMT:strtoq.obj
 0001:0003a7f8       __strtoull_l               1003b7f8 f   LIBCMT:strtoq.obj
 0001:0003a801       __strtoumax_l              1003b801 f   LIBCMT:strtoq.obj
 0001:0003a80a       _strtof                    1003b80a f   LIBCMT:strtoq.obj
 0001:0003a829       _strtoimax                 1003b829 f   LIBCMT:strtoq.obj
 0001:0003a832       _strtold                   1003b832 f   LIBCMT:strtoq.obj
 0001:0003a83b       _strtoll                   1003b83b f   LIBCMT:strtoq.obj
 0001:0003a844       _strtoull                  1003b844 f   LIBCMT:strtoq.obj
 0001:0003a84d       _strtoumax                 1003b84d f   LIBCMT:strtoq.obj
 0001:0003a856       __cabs                     1003b856 f   LIBCMT:hypot.obj
 0001:0003a875       __hypot                    1003b875 f   LIBCMT:hypot.obj
 0001:0003aae0       __CxxThrowException@8      1003bae0 f   LIBCMT:throw.obj
 0001:0003ac13       ?_CallCatchBlock2@@YAPAXPAUEHRegistrationNode@@PBU_s_FuncInfo@@PAXHK@Z 1003bc13 f   LIBCMT:_trnsctrl_.obj
 0001:0003ac73       ?_CallMemberFunction0@@YGXPAX0@Z 1003bc73 f   LIBCMT:_trnsctrl_.obj
 0001:0003ac7a       ?_CallMemberFunction1@@YGXPAX00@Z 1003bc7a f   LIBCMT:_trnsctrl_.obj
 0001:0003ac81       ?_CallMemberFunction2@@YGXPAX00H@Z 1003bc81 f   LIBCMT:_trnsctrl_.obj
 0001:0003ac88       ?_CallSETranslator@@YAHPAUEHExceptionRecord@@PAUEHRegistrationNode@@PAX2PBU_s_FuncInfo@@H1@Z 1003bc88 f   LIBCMT:_trnsctrl_.obj
 0001:0003ad5f       ?_GetRangeOfTrysToCheck@@YAPBU_s_TryBlockMapEntry@@PBU_s_FuncInfo@@HHPAI1@Z 1003bd5f f   LIBCMT:_trnsctrl_.obj
 0001:0003addd       ?_JumpToContinuation@@YGXPAXPAUEHRegistrationNode@@@Z 1003bddd f   LIBCMT:_trnsctrl_.obj
 0001:0003ae0f       ?_UnwindNestedFrames@@YGXPAUEHRegistrationNode@@PAUEHExceptionRecord@@@Z 1003be0f f   LIBCMT:_trnsctrl_.obj
 0001:0003ae64       __CreateFrameInfo          1003be64 f   LIBCMT:_trnsctrl_.obj
 0001:0003ae8e       __FindAndUnlinkFrame       1003be8e f   LIBCMT:_trnsctrl_.obj
 0001:0003aede       __IsExceptionObjectToBeDestroyed 1003bede f   LIBCMT:_trnsctrl_.obj
 0001:0003af07       ___CxxFrameHandler         1003bf07 f   LIBCMT:_trnsctrl_.obj
 0001:0003af3d       ___CxxFrameHandler2        1003bf3d f   LIBCMT:_trnsctrl_.obj
 0001:0003af73       ___CxxFrameHandler3        1003bf73 f   LIBCMT:_trnsctrl_.obj
 0001:0003afa9       ___CxxLongjmpUnwind@4      1003bfa9 f   LIBCMT:_trnsctrl_.obj
 0001:0003afd0       _memset                    1003bfd0 f   LIBCMT:memset.obj
 0001:0003b060       __ftoui3                   1003c060 f   LIBCMT:ftol3.obj
 0001:0003b06f       __ftoul3                   1003c06f f   LIBCMT:ftol3.obj
 0001:0003b07e       __ftol3                    1003c07e f   LIBCMT:ftol3.obj
 0001:0003b08b       __ftol3_NaN                1003c08b f   LIBCMT:ftol3.obj
 0001:0003b0a3       __ftol3_work               1003c0a3 f   LIBCMT:ftol3.obj
 0001:0003b129       __ftol3_common             1003c129 f   LIBCMT:ftol3.obj
 0001:0003b1eb       __ftol3_arg_error          1003c1eb f   LIBCMT:ftol3.obj
 0001:0003b1fd       __ftol3_except             1003c1fd f   LIBCMT:ftol3.obj
 0001:0003b23f       __dtoui3                   1003c23f f   LIBCMT:ftol3.obj
 0001:0003b24e       __dtoul3                   1003c24e f   LIBCMT:ftol3.obj
 0001:0003b25d       __dtol3                    1003c25d f   LIBCMT:ftol3.obj
 0001:0003b26a       __dtol3_NaN                1003c26a f   LIBCMT:ftol3.obj
 0001:0003b287       __dtol3_work               1003c287 f   LIBCMT:ftol3.obj
 0001:0003b36c       __ultod3                   1003c36c f   LIBCMT:ftol3.obj
 0001:0003b3fd       __ltod3                    1003c3fd f   LIBCMT:ftol3.obj
 0001:0003b42b       __snprintf                 1003c42b f   LIBCMT:snprintf.obj
 0001:0003b4d7       __snprintf_l               1003c4d7 f   LIBCMT:snprintf.obj
 0001:0003b500       _strncmp                   1003c500 f   LIBCMT:strncmp.obj
 0001:0003b8d5       ___RTCastToVoid            1003c8d5 f   LIBCMT:rtti.obj
 0001:0003b937       ___RTDynamicCast           1003c937 f   LIBCMT:rtti.obj
 0001:0003ba13       ___RTtypeid                1003ca13 f   LIBCMT:rtti.obj
 0001:0003ba8f       __vsnprintf                1003ca8f f   LIBCMT:vsnprint.obj
 0001:0003baaa       __vsnprintf_l              1003caaa f   LIBCMT:vsnprint.obj
 0001:0003bb56       __dupenv_s                 1003cb56 f   LIBCMT:getenv.obj
 0001:0003bcc9       __getenv_helper_nolock     1003ccc9 f   LIBCMT:getenv.obj
 0001:0003bde8       __invoke_watson_if_error   1003cde8 f i LIBCMT:getenv.obj
 0001:0003be08       _getenv                    1003ce08 f   LIBCMT:getenv.obj
 0001:0003be88       _getenv_s                  1003ce88 f   LIBCMT:getenv.obj
 0001:0003bf59       __strdup                   1003cf59 f   LIBCMT:strdup.obj
 0001:0003bf59       _strdup                    1003cf59 f   LIBCMT:strdup.obj
 0001:0003bfa9       _strnlen                   1003cfa9 f   LIBCMT:strlen_s.obj
 0001:0003bfd0       __aulldiv                  1003cfd0 f   LIBCMT:ulldiv.obj
 0001:0003c040       __libm_sse2_log10_precise  1003d040 f   LIBCMT:log10_sse2_precise.obj
 0001:0003c2f0       __libm_sse2_pow_precise    1003d2f0 f   LIBCMT:pow_sse2_precise.obj
 0001:0003ce60       __fclose_nolock            1003de60 f   LIBCMT:fclose.obj
 0001:0003cecc       _fclose                    1003decc f   LIBCMT:fclose.obj
 0001:0003cf43       __fsopen                   1003df43 f   LIBCMT:fopen.obj
 0001:0003d007       _fopen                     1003e007 f   LIBCMT:fopen.obj
 0001:0003d01c       _fopen_s                   1003e01c f   LIBCMT:fopen.obj
 0001:0003d061       __fread_nolock             1003e061 f   LIBCMT:fread.obj
 0001:0003d07c       __fread_nolock_s           1003e07c f   LIBCMT:fread.obj
 0001:0003d241       _fread                     1003e241 f   LIBCMT:fread.obj
 0001:0003d25c       _fread_s                   1003e25c f   LIBCMT:fread.obj
 0001:0003d2ed       __fseek_nolock             1003e2ed f   LIBCMT:fseek.obj
 0001:0003d37c       _fseek                     1003e37c f   LIBCMT:fseek.obj
 0001:0003d3ff       __ftell_nolock             1003e3ff f   LIBCMT:ftell.obj
 0001:0003d78f       _ftell                     1003e78f f   LIBCMT:ftell.obj
 0001:0003d7fb       __fwrite_nolock            1003e7fb f   LIBCMT:fwrite.obj
 0001:0003d954       _fwrite                    1003e954 f   LIBCMT:fwrite.obj
 0001:0003d9d6       ___ascii_stricmp           1003e9d6 f   LIBCMT:stricmp.obj
 0001:0003da0f       __stricmp                  1003ea0f f   LIBCMT:stricmp.obj
 0001:0003da56       __stricmp_l                1003ea56 f   LIBCMT:stricmp.obj
 0001:0003daeb       _strtok                    1003eaeb f   LIBCMT:strtok.obj
 0001:0003dbb2       __toupper                  1003ebb2 f   LIBCMT:toupper.obj
 0001:0003dbbd       __toupper_l                1003ebbd f   LIBCMT:toupper.obj
 0001:0003dd01       _toupper                   1003ed01 f   LIBCMT:toupper.obj
 0001:0003dd2d       __strtod_l                 1003ed2d f   LIBCMT:strtod.obj
 0001:0003de44       _strtod                    1003ee44 f   LIBCMT:strtod.obj
 0001:0003de60       __libm_sse2_sin_precise    1003ee60 f   LIBCMT:sin_sse2_precise.obj
 0001:0003e028       __CRT_INIT@12              1003f028 f   LIBCMT:dllcrt0.obj
 0001:0003e19a       __DllMainCRTStartup@12     1003f19a f   LIBCMT:dllcrt0.obj
 0001:0003e2cb       ___DllXcptFilter           1003f2cb f   LIBCMT:dllcrt0.obj
 0001:0003e2f0       __crt_debugger_hook        1003f2f0 f   LIBCMT:dbghook.obj
 0001:0003e325       ___crtCloseThreadpoolTimer 1003f325 f   LIBCMT:winapisupp.obj
 0001:0003e33c       ___crtCloseThreadpoolWait  1003f33c f   LIBCMT:winapisupp.obj
 0001:0003e353       ___crtCreateEventExW       1003f353 f   LIBCMT:winapisupp.obj
 0001:0003e38e       ___crtCreateSemaphoreExW   1003f38e f   LIBCMT:winapisupp.obj
 0001:0003e3c8       ___crtCreateSymbolicLinkW  1003f3c8 f   LIBCMT:winapisupp.obj
 0001:0003e3f1       ___crtCreateThreadpoolTimer 1003f3f1 f   LIBCMT:winapisupp.obj
 0001:0003e412       ___crtCreateThreadpoolWait 1003f412 f   LIBCMT:winapisupp.obj
 0001:0003e433       ___crtFlsAlloc             1003f433 f   LIBCMT:winapisupp.obj
 0001:0003e451       ___crtFlsFree              1003f451 f   LIBCMT:winapisupp.obj
 0001:0003e470       ___crtFlsGetValue          1003f470 f   LIBCMT:winapisupp.obj
 0001:0003e48f       ___crtFlsSetValue          1003f48f f   LIBCMT:winapisupp.obj
 0001:0003e4b1       ___crtFlushProcessWriteBuffers 1003f4b1 f   LIBCMT:winapisupp.obj
 0001:0003e4c1       ___crtFreeLibraryWhenCallbackReturns 1003f4c1 f   LIBCMT:winapisupp.obj
 0001:0003e4db       ___crtGetCurrentProcessorNumber 1003f4db f   LIBCMT:winapisupp.obj
 0001:0003e4ed       ___crtGetFileInformationByHandleEx 1003f4ed f   LIBCMT:winapisupp.obj
 0001:0003e519       ___crtGetLogicalProcessorInformation 1003f519 f   LIBCMT:winapisupp.obj
 0001:0003e53f       ___crtGetShowWindowMode    1003f53f f   LIBCMT:winapisupp.obj
 0001:0003e562       ___crtGetTickCount64       1003f562 f   LIBCMT:winapisupp.obj
 0001:0003e57a       ___crtInitializeCriticalSectionEx 1003f57a f   LIBCMT:winapisupp.obj
 0001:0003e5a8       ___crtIsPackagedApp        1003f5a8 f   LIBCMT:winapisupp.obj
 0001:0003e5e8       ___crtLoadWinApiPointers   1003f5e8 f   LIBCMT:winapisupp.obj
 0001:0003e873       ___crtSetFileInformationByHandle 1003f873 f   LIBCMT:winapisupp.obj
 0001:0003e89f       ___crtSetThreadStackGuarantee 1003f89f f   LIBCMT:winapisupp.obj
 0001:0003e8ba       ___crtSetThreadpoolTimer   1003f8ba f   LIBCMT:winapisupp.obj
 0001:0003e8da       ___crtSetThreadpoolWait    1003f8da f   LIBCMT:winapisupp.obj
 0001:0003e8f7       ___crtSetUnhandledExceptionFilter 1003f8f7 f   LIBCMT:winapisupp.obj
 0001:0003e905       ___crtSleep                1003f905 f   LIBCMT:winapisupp.obj
 0001:0003e913       ___crtTerminateProcess     1003f913 f   LIBCMT:winapisupp.obj
 0001:0003e928       ___crtUnhandledException   1003f928 f   LIBCMT:winapisupp.obj
 0001:0003e93e       ___crtWaitForThreadpoolTimerCallbacks 1003f93e f   LIBCMT:winapisupp.obj
 0001:0003e958       ___addlocaleref            1003f958 f   LIBCMT:localref.obj
 0001:0003e9ed       ___freetlocinfo            1003f9ed f   LIBCMT:localref.obj
 0001:0003eb47       ___removelocaleref         1003fb47 f   LIBCMT:localref.obj
 0001:0003ebe7       ___updatetlocinfo          1003fbe7 f   LIBCMT:localref.obj
 0001:0003ec67       __updatetlocinfoEx_nolock  1003fc67 f   LIBCMT:localref.obj
 0001:0003ecb2       ___initmbctable            1003fcb2 f   LIBCMT:mbctype.obj
 0001:0003ef69       ___updatetmbcinfo          1003ff69 f   LIBCMT:mbctype.obj
 0001:0003f00f       __getmbcp                  1004000f f   LIBCMT:mbctype.obj
 0001:0003f040       __setmbcp                  10040040 f   LIBCMT:mbctype.obj
 0001:0003f1e8       __setmbcp_nolock           100401e8 f   LIBCMT:mbctype.obj
 0001:0003f3d3       __isctype                  100403d3 f   LIBCMT:isctype.obj
 0001:0003f402       __isctype_l                10040402 f   LIBCMT:isctype.obj
 0001:0003f4b3       ___get_flsindex            100404b3 f   LIBCMT:tidtable.obj
 0001:0003f4b9       ___threadhandle            100404b9 f   LIBCMT:tidtable.obj
 0001:0003f4bf       ___threadid                100404bf f   LIBCMT:tidtable.obj
 0001:0003f4c5       __freefls@4                100404c5 f   LIBCMT:tidtable.obj
 0001:0003f5fa       __freeptd                  100405fa f   LIBCMT:tidtable.obj
 0001:0003f630       __getptd                   10040630 f   LIBCMT:tidtable.obj
 0001:0003f648       __getptd_noexit            10040648 f   LIBCMT:tidtable.obj
 0001:0003f6b7       __initptd                  100406b7 f   LIBCMT:tidtable.obj
 0001:0003f76a       __mtinit                   1004076a f   LIBCMT:tidtable.obj
 0001:0003f7e0       __mtterm                   100407e0 f   LIBCMT:tidtable.obj
 0001:0003f7fd       ___init_dummy              100407fd f   LIBCMT:wsetloca.obj
 0001:0003f800       __locterm                  10040800 f   LIBCMT:wsetloca.obj
 0001:0003f852       ____setlc_active_func      10040852 f   LIBCMT:wsetloca.obj
 0001:0003f858       ____unguarded_readlc_active_add_func 10040858 f   LIBCMT:wsetloca.obj
 0001:0003f85e       ___copy_locale_name        1004085e f   LIBCMT:wsetloca.obj
 0001:0003f8c2       ___create_locale           100408c2 f   LIBCMT:wsetloca.obj
 0001:0003f8cb       ___free_locale             100408cb f   LIBCMT:wsetloca.obj
 0001:0003f8d0       ___get_current_locale      100408d0 f   LIBCMT:wsetloca.obj
 0001:0003f8d5       ___lc_lctowcs              100408d5 f   LIBCMT:wsetloca.obj
 0001:0003f943       ___lc_wcstolc              10040943 f   LIBCMT:wsetloca.obj
 0001:0003fa6f       __configthreadlocale       10040a6f f   LIBCMT:wsetloca.obj
 0001:0003faf5       __create_locale            10040af5 f   LIBCMT:wsetloca.obj
 0001:0003fb57       __expandlocale             10040b57 f   LIBCMT:wsetloca.obj
 0001:0003fe4e       __free_locale              10040e4e f   LIBCMT:wsetloca.obj
 0001:0003ff05       __get_current_locale       10040f05 f   LIBCMT:wsetloca.obj
 0001:0003ffb4       __wcreate_locale           10040fb4 f   LIBCMT:wsetloca.obj
 0001:0004008b       __wcscats                  1004108b f   LIBCMT:wsetloca.obj
 0001:000400ca       __wsetlocale               100410ca f   LIBCMT:wsetloca.obj
 0001:00040a0c       ?_invalid_parameter@@YAXPBG00II@Z 10041a0c f   LIBCMT:invarg.obj
 0001:00040a11       ?_invoke_watson@@YAXPBG00II@Z 10041a11 f   LIBCMT:invarg.obj
 0001:00040a29       __call_reportfault         10041a29 f   LIBCMT:invarg.obj
 0001:00040b4e       __get_invalid_parameter_handler 10041b4e f   LIBCMT:invarg.obj
 0001:00040b5b       __initp_misc_invarg        10041b5b f   LIBCMT:invarg.obj
 0001:00040b68       __invalid_parameter        10041b68 f   LIBCMT:invarg.obj
 0001:00040b93       __invalid_parameter_noinfo 10041b93 f   LIBCMT:invarg.obj
 0001:00040ba3       __invalid_parameter_noinfo_noreturn 10041ba3 f   LIBCMT:invarg.obj
 0001:00040bbe       __invoke_watson            10041bbe f   LIBCMT:invarg.obj
 0001:00040be9       __set_invalid_parameter_handler 10041be9 f   LIBCMT:invarg.obj
 0001:00040c0e       ___doserrno                10041c0e f   LIBCMT:dosmap.obj
 0001:00040c21       __dosmaperr                10041c21 f   LIBCMT:dosmap.obj
 0001:00040c42       __errno                    10041c42 f   LIBCMT:dosmap.obj
 0001:00040c55       __get_doserrno             10041c55 f   LIBCMT:dosmap.obj
 0001:00040c78       __get_errno                10041c78 f   LIBCMT:dosmap.obj
 0001:00040c9b       __get_errno_from_oserr     10041c9b f   LIBCMT:dosmap.obj
 0001:00040cdc       __set_doserrno             10041cdc f   LIBCMT:dosmap.obj
 0001:00040cfb       __set_errno                10041cfb f   LIBCMT:dosmap.obj
 0001:00040d1a       __flsbuf                   10041d1a f   LIBCMT:_flsbuf.obj
 0001:00040e69       __vscprintf                10041e69 f   LIBCMT:vsprintf.obj
 0001:00040e83       __vscprintf_helper         10041e83 f   LIBCMT:vsprintf.obj
 0001:00040edf       __vscprintf_l              10041edf f   LIBCMT:vsprintf.obj
 0001:00040efa       __vscprintf_p              10041efa f   LIBCMT:vsprintf.obj
 0001:00040f14       __vscprintf_p_l            10041f14 f   LIBCMT:vsprintf.obj
 0001:00040f2f       __vsprintf_l               10041f2f f   LIBCMT:vsprintf.obj
 0001:00040fb3       _vsprintf                  10041fb3 f   LIBCMT:vsprintf.obj
 0001:00040fcb       __vsnprintf_c              10041fcb f   LIBCMT:vsnprnc.obj
 0001:00040ff2       __vsnprintf_c_l            10041ff2 f   LIBCMT:vsnprnc.obj
 0001:0004101a       __vsnprintf_helper         1004201a f   LIBCMT:vsnprnc.obj
 0001:000410e4       __vsnprintf_s              100420e4 f   LIBCMT:vsnprnc.obj
 0001:00041102       __vsnprintf_s_l            10042102 f   LIBCMT:vsnprnc.obj
 0001:00041202       __vsprintf_p               10042202 f   LIBCMT:vsnprnc.obj
 0001:00041229       __vsprintf_p_l             10042229 f   LIBCMT:vsnprnc.obj
 0001:00041251       __vsprintf_s_l             10042251 f   LIBCMT:vsnprnc.obj
 0001:000412c6       _vsprintf_s                100422c6 f   LIBCMT:vsnprnc.obj
 0001:000412e1       __output_l                 100422e1 f   LIBCMT:output.obj
 0001:00041e61       _get_int64_arg             10042e61 f i LIBCMT:output.obj
 0001:00041e74       _get_int_arg               10042e74 f i LIBCMT:output.obj
 0001:00041e84       _get_short_arg             10042e84 f i LIBCMT:output.obj
 0001:00041f81       ___isa_available_init      10042f81 f   LIBCMT:cpu_disp.obj
 0001:000420fa       __get_heap_handle          100430fa f   LIBCMT:heapinit.obj
 0001:00042100       __heap_init                10043100 f   LIBCMT:heapinit.obj
 0001:00042115       __heap_term                10043115 f   LIBCMT:heapinit.obj
 0001:0004211d       ?_query_new_handler@@YAP6AHI@ZXZ 1004311d f   LIBCMT:handler.obj
 0001:0004212a       ?_set_new_handler@@YAP6AHI@ZH@Z 1004312a f   LIBCMT:handler.obj
 0001:00042133       ?_set_new_handler@@YAP6AHI@ZP6AHI@Z@Z 10043133 f   LIBCMT:handler.obj
 0001:00042168       __callnewh                 10043168 f   LIBCMT:handler.obj
 0001:0004218e       __initp_heap_handler       1004318e f   LIBCMT:handler.obj
 0001:0004219b       ___copy_path_to_wide_string 1004319b f   LIBCMT:crt0dat.obj
 0001:0004224d       ___copy_to_char            1004324d f   LIBCMT:crt0dat.obj
 0001:00042302       ___crtCorExitProcess       10043302 f   LIBCMT:crt0dat.obj
 0001:00042336       ___crtExitProcess          10043336 f   LIBCMT:crt0dat.obj
 0001:0004234c       ___freeCrtMemory           1004334c f   LIBCMT:crt0dat.obj
 0001:00042459       __amsg_exit                10043459 f   LIBCMT:crt0dat.obj
 0001:00042475       __c_exit                   10043475 f   LIBCMT:crt0dat.obj
 0001:00042484       __cexit                    10043484 f   LIBCMT:crt0dat.obj
 0001:00042493       __cinit                    10043493 f   LIBCMT:crt0dat.obj
 0001:00042517       __exit                     10043517 f   LIBCMT:crt0dat.obj
 0001:0004252b       __exit_app                 1004352b f   LIBCMT:crt0dat.obj
 0001:00042539       __get_pgmptr               10043539 f   LIBCMT:crt0dat.obj
 0001:00042568       __get_wpgmptr              10043568 f   LIBCMT:crt0dat.obj
 0001:00042597       __init_pointers            10043597 f   LIBCMT:crt0dat.obj
 0001:00042605       __initterm_e               10043605 f   LIBCMT:crt0dat.obj
 0001:00042627       __lockexit                 10043627 f   LIBCMT:crt0dat.obj
 0001:00042630       __unlockexit               10043630 f   LIBCMT:crt0dat.obj
 0001:00042768       _exit                      10043768 f   LIBCMT:crt0dat.obj
 0001:0004277c       __FF_MSGBANNER             1004377c f   LIBCMT:crt0msg.obj
 0001:000427b5       __GET_RTERRMSG             100437b5 f   LIBCMT:crt0msg.obj
 0001:000427d9       __NMSG_WRITE               100437d9 f   LIBCMT:crt0msg.obj
 0001:00042996       ___initstdio               10043996 f   LIBCMT:_file.obj
 0001:00042a09       ___endstdio                10043a09 f   LIBCMT:_file.obj
 0001:00042a30       ___iob_func                10043a30 f   LIBCMT:_file.obj
 0001:00042a36       __lock_file                10043a36 f   LIBCMT:_file.obj
 0001:00042a75       __lock_file2               10043a75 f   LIBCMT:_file.obj
 0001:00042aa5       __unlock_file              10043aa5 f   LIBCMT:_file.obj
 0001:00042adf       __unlock_file2             10043adf f   LIBCMT:_file.obj
 0001:00042b0c       __ftbuf                    10043b0c f   LIBCMT:_sftbuf.obj
 0001:00042b3d       __stbuf                    10043b3d f   LIBCMT:_sftbuf.obj
 0001:00042bf0       __SEH_prolog4              10043bf0 f   LIBCMT:sehprolg4.obj
 0001:00042c35       __SEH_epilog4              10043c35 f   LIBCMT:sehprolg4.obj
 0001:00042c90       __except_handler4          10043c90 f   LIBCMT:chandler4.obj
 0001:00042e24       __output_s_l               10043e24 f   LIBCMT:outputs.obj
 0001:00043aac       __output_p_l               10044aac f   LIBCMT:outputp.obj
 0001:00044de4       __validate_param_reuseA    10045de4 f   LIBCMT:outputp.obj
 0001:00044f1a       _get_crtdouble_arg         10045f1a f i LIBCMT:outputp.obj
 0001:00045019       ??0__non_rtti_object@std@@QAE@ABV01@@Z 10046019 f   LIBCMT:stdexcpt.obj
 0001:00045034       ??0__non_rtti_object@std@@QAE@PBD@Z 10046034 f   LIBCMT:stdexcpt.obj
 0001:0004504f       ??0bad_cast@std@@QAE@ABV01@@Z 1004604f f   LIBCMT:stdexcpt.obj
 0001:0004506a       ??0bad_cast@std@@QAE@PBD@Z 1004606a f   LIBCMT:stdexcpt.obj
 0001:00045086       ??0bad_typeid@std@@QAE@ABV01@@Z 10046086 f   LIBCMT:stdexcpt.obj
 0001:000450a1       ??0bad_typeid@std@@QAE@PBD@Z 100460a1 f   LIBCMT:stdexcpt.obj
 0001:000450bd       ??0exception@std@@QAE@ABQBD@Z 100460bd f   LIBCMT:stdexcpt.obj
 0001:000450e2       ??0exception@std@@QAE@ABQBDH@Z 100460e2 f   LIBCMT:stdexcpt.obj
 0001:000450fd       ??0exception@std@@QAE@ABV01@@Z 100460fd f   LIBCMT:stdexcpt.obj
 0001:00045120       ??0exception@std@@QAE@XZ   10046120 f   LIBCMT:stdexcpt.obj
 0001:00045131       ??1__non_rtti_object@std@@UAE@XZ 10046131 f   LIBCMT:stdexcpt.obj
 0001:0004513c       ??1bad_cast@std@@UAE@XZ    1004613c f   LIBCMT:stdexcpt.obj
 0001:00045147       ??1bad_typeid@std@@UAE@XZ  10046147 f   LIBCMT:stdexcpt.obj
 0001:00045152       ??1exception@std@@UAE@XZ   10046152 f   LIBCMT:stdexcpt.obj
 0001:0004515d       ??4exception@std@@QAEAAV01@ABV01@@Z 1004615d f   LIBCMT:stdexcpt.obj
 0001:00045190       ??_G__non_rtti_object@std@@UAEPAXI@Z 10046190 f i LIBCMT:stdexcpt.obj
 0001:00045190       ??_E__non_rtti_object@std@@UAEPAXI@Z 10046190 f i LIBCMT:stdexcpt.obj
 0001:000451b5       ??_Ebad_cast@std@@UAEPAXI@Z 100461b5 f i LIBCMT:stdexcpt.obj
 0001:000451b5       ??_Gbad_cast@std@@UAEPAXI@Z 100461b5 f i LIBCMT:stdexcpt.obj
 0001:000451da       ??_Gbad_typeid@std@@UAEPAXI@Z 100461da f i LIBCMT:stdexcpt.obj
 0001:000451da       ??_Ebad_typeid@std@@UAEPAXI@Z 100461da f i LIBCMT:stdexcpt.obj
 0001:000451ff       ??_Gexception@std@@UAEPAXI@Z 100461ff f i LIBCMT:stdexcpt.obj
 0001:000451ff       ??_Eexception@std@@UAEPAXI@Z 100461ff f i LIBCMT:stdexcpt.obj
 0001:00045224       ?_Copy_str@exception@std@@AAEXPBD@Z 10046224 f   LIBCMT:stdexcpt.obj
 0001:00045262       ?_Tidy@exception@std@@AAEXXZ 10046262 f   LIBCMT:stdexcpt.obj
 0001:0004527e       ?what@exception@std@@UBEPBDXZ 1004627e f   LIBCMT:stdexcpt.obj
 0001:00045290       _strcmp                    10046290 f   LIBCMT:strcmp.obj
 0001:0004531c       ?_Name_base@type_info@@CAPBDPBV1@PAU__type_info_node@@@Z 1004631c f   LIBCMT:typname.obj
 0001:0004540d       ?_Name_base_internal@type_info@@CAPBDPBV1@PAU__type_info_node@@@Z 1004640d f   LIBCMT:typname.obj
 0001:00045517       ?_Type_info_dtor@type_info@@CAXPAV1@@Z 10046517 f   LIBCMT:typname.obj
 0001:00045588       ?_Type_info_dtor_internal@type_info@@CAXPAV1@@Z 10046588 f   LIBCMT:typname.obj
 0001:000455f9       ___clean_type_info_names_internal 100465f9 f   LIBCMT:typname.obj
 0001:0004564c       ___unDNameHelper           1004664c f   LIBCMT:typname.obj
 0001:0004567a       ?strrchr@@YAPADPADH@Z      1004667a f i LIBCMT:cvt.obj
 0001:00045683       __cfltcvt                  10046683 f   LIBCMT:cvt.obj
 0001:000456a4       __cfltcvt_l                100466a4 f   LIBCMT:cvt.obj
 0001:0004572a       __cftoa                    1004672a f   LIBCMT:cvt.obj
 0001:00045748       __cftoa_l                  10046748 f   LIBCMT:cvt.obj
 0001:00045aa4       __cftoe                    10046aa4 f   LIBCMT:cvt.obj
 0001:00045c13       __cftoe_l                  10046c13 f   LIBCMT:cvt.obj
 0001:00045ce1       __cftof                    10046ce1 f   LIBCMT:cvt.obj
 0001:00045de8       __cftof_l                  10046de8 f   LIBCMT:cvt.obj
 0001:00045ea9       __cftog                    10046ea9 f   LIBCMT:cvt.obj
 0001:00045ec7       __cftog_l                  10046ec7 f   LIBCMT:cvt.obj
 0001:00045fc6       __cropzeros                10046fc6 f   LIBCMT:cvt.obj
 0001:00045fd7       __cropzeros_l              10046fd7 f   LIBCMT:cvt.obj
 0001:00046057       __fassign                  10047057 f   LIBCMT:cvt.obj
 0001:0004606f       __fassign_l                1004706f f   LIBCMT:cvt.obj
 0001:000460b1       __forcdecpt                100470b1 f   LIBCMT:cvt.obj
 0001:000460c2       __forcdecpt_l              100470c2 f   LIBCMT:cvt.obj
 0001:00046136       __positive                 10047136 f   LIBCMT:cvt.obj
 0001:00046178       __setdefaultprecision      10047178 f   LIBCMT:fp8.obj
 0001:0004619f       __initp_misc_cfltcvt_tab   1004719f f   LIBCMT:cmiscdat.obj
 0001:000461be       __set_abort_behavior       100471be f   LIBCMT:abort.obj
 0001:000461dd       _abort                     100471dd f   LIBCMT:abort.obj
 0001:00046220       ___getlocaleinfo           10047220 f   LIBCMT:inithelp.obj
 0001:000463f9       __initp_misc_purevirt      100473f9 f   LIBCMT:inithelp.obj
 0001:00046406       __msize                    10047406 f   LIBCMT:msize.obj
 0001:00046437       __calloc_crt               10047437 f   LIBCMT:crtheap.obj
 0001:0004647f       __malloc_crt               1004747f f   LIBCMT:crtheap.obj
 0001:000464c6       __realloc_crt              100474c6 f   LIBCMT:crtheap.obj
 0001:00046510       __recalloc_crt             10047510 f   LIBCMT:crtheap.obj
 0001:0004655e       __set_malloc_crt_max_wait  1004755e f   LIBCMT:crtheap.obj
 0001:00046571       _wait_a_bit                10047571 f i LIBCMT:crtheap.obj
 0001:000465a0       _strchr                    100475a0 f   LIBCMT:strchr.obj
 0001:0004660e       ___from_strstr_to_strchr   1004760e     LIBCMT:strchr.obj
 0001:000466cb       ___crt_atoflt_l            100476cb f   LIBCMT:atodbl.obj
 0001:0004676f       __atodbl                   1004776f f   LIBCMT:atodbl.obj
 0001:00046784       __atodbl_l                 10047784 f   LIBCMT:atodbl.obj
 0001:00046812       __atoflt                   10047812 f   LIBCMT:atodbl.obj
 0001:00046827       __atoflt_l                 10047827 f   LIBCMT:atodbl.obj
 0001:0004683f       __atoldbl                  1004783f f   LIBCMT:atodbl.obj
 0001:00046854       __atoldbl_l                10047854 f   LIBCMT:atodbl.obj
 0001:000468f0       __aulldvrm                 100478f0 f   LIBCMT:ulldvrm.obj
 0001:00046990       __CIsqrt                   10047990 f   LIBCMT:sqrt.obj
 0001:000469a4       _sqrt                      100479a4     LIBCMT:sqrt.obj
 0001:00046a4a       __add_exp                  10047a4a f   LIBCMT:util.obj
 0001:00046a79       __decomp                   10047a79 f   LIBCMT:util.obj
 0001:00046b4b       __get_exp                  10047b4b f   LIBCMT:util.obj
 0001:00046b64       __set_bexp                 10047b64 f   LIBCMT:util.obj
 0001:00046b8d       __set_exp                  10047b8d f   LIBCMT:util.obj
 0001:00046bbc       __sptype                   10047bbc f   LIBCMT:util.obj
 0001:00046c17       __errcode                  10047c17 f   LIBCMT:fpexcept.obj
 0001:00046c49       __except1                  10047c49 f   LIBCMT:fpexcept.obj
 0001:00046d11       __except2                  10047d11 f   LIBCMT:fpexcept.obj
 0001:00046e11       __handle_exc               10047e11 f   LIBCMT:fpexcept.obj
 0001:00046fef       __handle_qnan1             10047fef f   LIBCMT:fpexcept.obj
 0001:0004703f       __handle_qnan2             1004803f f   LIBCMT:fpexcept.obj
 0001:0004709f       __raise_exc                1004809f f   LIBCMT:fpexcept.obj
 0001:000470c0       __raise_exc_ex             100480c0 f   LIBCMT:fpexcept.obj
 0001:000473a5       __raise_excf               100483a5 f   LIBCMT:fpexcept.obj
 0001:000473c6       __set_errno_from_matherr   100483c6 f   LIBCMT:fpexcept.obj
 0001:000473f3       __umatherr                 100483f3 f   LIBCMT:fpexcept.obj
 0001:00047493       ___clrfp_sse2              10048493 f   LIBCMT:fpctrl.obj
 0001:000474b4       ___ctrlfp_sse2             100484b4 f   LIBCMT:fpctrl.obj
 0001:000474ed       ___fclrf_sse2              100484ed f   LIBCMT:fpctrl.obj
 0001:0004750a       ___get_fpsr_sse2           1004850a f   LIBCMT:fpctrl.obj
 0001:00047526       ___set_fpsr_sse2           10048526 f   LIBCMT:fpctrl.obj
 0001:0004759c       ___set_statfp_sse2         1004859c f   LIBCMT:fpctrl.obj
 0001:000475b5       ___statfp_sse2             100485b5 f   LIBCMT:fpctrl.obj
 0001:000475ca       __clrfp                    100485ca f   LIBCMT:fpctrl.obj
 0001:000475db       __ctrlfp                   100485db f   LIBCMT:fpctrl.obj
 0001:00047606       __set_statfp               10048606 f   LIBCMT:fpctrl.obj
 0001:0004765e       __statfp                   1004865e f   LIBCMT:fpctrl.obj
 0001:00047670       __CallSettingFrame@12      10048670 f   LIBCMT:lowhelpr.obj
 0001:00047697       __NLG_Return               10048697     LIBCMT:lowhelpr.obj
 0001:000476bc       ?_inconsistency@@YAXXZ     100486bc f   LIBCMT:hooks.obj
 0001:000476f4       ?terminate@@YAXXZ          100486f4 f   LIBCMT:hooks.obj
 0001:00047728       ?unexpected@@YAXXZ         10048728 f   LIBCMT:hooks.obj
 0001:0004773b       __initp_eh_hooks           1004873b f   LIBCMT:hooks.obj
 0001:0004774c       ___DestructExceptionObject 1004874c f   LIBCMT:frame.obj
 0001:000477d7       ??0bad_exception@std@@QAE@ABV01@@Z 100487d7 f i LIBCMT:frame.obj
 0001:000477f2       ??0bad_exception@std@@QAE@PBD@Z 100487f2 f i LIBCMT:frame.obj
 0001:0004780e       ??1bad_exception@std@@UAE@XZ 1004880e f i LIBCMT:frame.obj
 0001:00047819       ??_Ebad_exception@std@@UAEPAXI@Z 10048819 f i LIBCMT:frame.obj
 0001:00047819       ??_Gbad_exception@std@@UAEPAXI@Z 10048819 f i LIBCMT:frame.obj
 0001:00048086       ?__uncaught_exception@@YA_NXZ 10049086 f   LIBCMT:frame.obj
 0001:00048097       ?_is_exception_typeof@@YAHABVtype_info@@PAU_EXCEPTION_POINTERS@@@Z 10049097 f   LIBCMT:frame.obj
 0001:0004811e       __SetWinRTOutOfMemoryExceptionCallback 1004911e f   LIBCMT:frame.obj
 0001:0004812b       ___AdjustPointer           1004912b f   LIBCMT:frame.obj
 0001:00048150       ___BuildCatchObject        10049150 f   LIBCMT:frame.obj
 0001:000481de       ___BuildCatchObjectHelper  100491de f   LIBCMT:frame.obj
 0001:000483a0       ___CxxDetectRethrow        100493a0 f   LIBCMT:frame.obj
 0001:000483ef       ___CxxExceptionFilter      100493ef f   LIBCMT:frame.obj
 0001:00048549       ___CxxQueryExceptionSize   10049549 f   LIBCMT:frame.obj
 0001:0004854d       ___CxxRegisterExceptionObject 1004954d f   LIBCMT:frame.obj
 0001:00048604       ___CxxUnregisterExceptionObject 10049604 f   LIBCMT:frame.obj
 0001:00048741       ___FrameUnwindFilter       10049741 f   LIBCMT:frame.obj
 0001:0004878f       ___FrameUnwindToState      1004978f f   LIBCMT:frame.obj
 0001:00048868       ___GetPlatformExceptionInfo 10049868 f   LIBCMT:frame.obj
 0001:000488bd       ___InternalCxxFrameHandler 100498bd f   LIBCMT:frame.obj
 0001:0004899e       ___TypeMatch               1004999e f   LIBCMT:frame.obj
 0001:00048a05       __VEC_memset               10049a05 f   LIBCMT:p4_memset.obj
 0001:00048acd       _strcpy_s                  10049acd f   LIBCMT:strcpy_s.obj
 0001:00048b30       _strlen                    10049b30 f   LIBCMT:strlen.obj
 0001:00048bbb       __lock                     10049bbb f   LIBCMT:mlock.obj
 0001:00048bef       __lockerr_exit             10049bef f   LIBCMT:mlock.obj
 0001:00048c0f       __mtdeletelocks            10049c0f f   LIBCMT:mlock.obj
 0001:00048c63       __mtinitlocknum            10049c63 f   LIBCMT:mlock.obj
 0001:00048d0c       __mtinitlocks              10049d0c f   LIBCMT:mlock.obj
 0001:00048d45       __unlock                   10049d45 f   LIBCMT:mlock.obj
 0001:00048d5a       ___wtomb_environ           10049d5a f   LIBCMT:wtombenv.obj
 0001:00048de9       _calloc                    10049de9 f   LIBCMT:calloc.obj
 0001:00048e29       __mbsnbicoll               10049e29 f   LIBCMT:mbsnbico.obj
 0001:00048e41       __mbsnbicoll_l             10049e41 f   LIBCMT:mbsnbico.obj
 0001:00048ef7       ___libm_error_support      10049ef7 f   LIBCMT:libm_error.obj
 0001:000491df       ___libm_setusermatherr     1004a1df f   LIBCMT:libm_error.obj
 0001:00049210       _log10                     1004a210 f   LIBCMT:log10.obj
 0001:00049250       __CIlog10                  1004a250 f   LIBCMT:log10.obj
 0001:0004928b       __CIlog10_default          1004a28b f   LIBCMT:log10.obj
 0001:0004929f       __log10_default            1004a29f     LIBCMT:log10.obj
 0001:00049360       _pow                       1004a360 f   LIBCMT:pow.obj
 0001:000493a0       __CIpow                    1004a3a0 f   LIBCMT:pow.obj
 0001:000493db       __CIpow_default            1004a3db f   LIBCMT:pow.obj
 0001:000493f4       __pow_default              1004a3f4     LIBCMT:pow.obj
 0001:000495ea       __fileno                   1004a5ea f   LIBCMT:fileno.obj
 0001:0004960e       __close                    1004a60e f   LIBCMT:close.obj
 0001:000496e9       __close_nolock             1004a6e9 f   LIBCMT:close.obj
 0001:00049783       __freebuf                  1004a783 f   LIBCMT:_freebuf.obj
 0001:000497b3       __fflush_nolock            1004a7b3 f   LIBCMT:fflush.obj
 0001:000497f9       __flush                    1004a7f9 f   LIBCMT:fflush.obj
 0001:0004985d       __flushall                 1004a85d f   LIBCMT:fflush.obj
 0001:00049866       _fflush                    1004a866 f   LIBCMT:fflush.obj
 0001:000499a3       __getstream                1004a9a3 f   LIBCMT:stream.obj
 0001:00049ac2       __openfile                 1004aac2 f   LIBCMT:_open.obj
 0001:00049d40       __local_unwind4            1004ad40 f   LIBCMT:exsup4.obj
 0001:00049e16       __seh_longjmp_unwind4@4    1004ae16 f   LIBCMT:exsup4.obj
 0001:00049e32       @_EH4_CallFilterFunc@8     1004ae32 f   LIBCMT:exsup4.obj
 0001:00049e49       @_EH4_TransferToHandler@8  1004ae49 f   LIBCMT:exsup4.obj
 0001:00049e62       @_EH4_GlobalUnwind2@8      1004ae62 f   LIBCMT:exsup4.obj
 0001:00049e7b       @_EH4_LocalUnwind@16       1004ae7b f   LIBCMT:exsup4.obj
 0001:00049e92       __filbuf                   1004ae92 f   LIBCMT:_filbuf.obj
 0001:00049fb3       _memcpy_s                  1004afb3 f   LIBCMT:memcpy_s.obj
 0001:0004a032       __read                     1004b032 f   LIBCMT:read.obj
 0001:0004a146       __read_nolock              1004b146 f   LIBCMT:read.obj
 0001:0004a8d7       __lseek                    1004b8d7 f   LIBCMT:lseek.obj
 0001:0004a9c6       __lseek_nolock             1004b9c6 f   LIBCMT:lseek.obj
 0001:0004aa6d       __lseeki64                 1004ba6d f   LIBCMT:lseeki64.obj
 0001:0004ab69       __lseeki64_nolock          1004bb69 f   LIBCMT:lseeki64.obj
 0001:0004abe0       __chkstk                   1004bbe0 f   LIBCMT:chkstk.obj
 0001:0004abe0       __alloca_probe             1004bbe0 f   LIBCMT:chkstk.obj
 0001:0004ac0b       __ioinit                   1004bc0b f   LIBCMT:ioinit.obj
 0001:0004aebf       __ioterm                   1004bebf f   LIBCMT:ioinit.obj
 0001:0004af11       __write                    1004bf11 f   LIBCMT:write.obj
 0001:0004b000       __write_nolock             1004c000 f   LIBCMT:write.obj
 0001:0004b865       __tolower                  1004c865 f   LIBCMT:tolower.obj
 0001:0004b870       __tolower_l                1004c870 f   LIBCMT:tolower.obj
 0001:0004b9b3       _tolower                   1004c9b3 f   LIBCMT:tolower.obj
 0001:0004b9df       ___iswcsym                 1004c9df f i LIBCMT:_wctype.obj
 0001:0004ba03       ___iswcsymf                1004ca03 f i LIBCMT:_wctype.obj
 0001:0004ba27       __isleadbyte_l             1004ca27 f i LIBCMT:_wctype.obj
 0001:0004ba61       __iswalnum_l               1004ca61 f i LIBCMT:_wctype.obj
 0001:0004ba75       __iswalpha_l               1004ca75 f i LIBCMT:_wctype.obj
 0001:0004ba89       __iswblank_l               1004ca89 f i LIBCMT:_wctype.obj
 0001:0004baa4       __iswcntrl_l               1004caa4 f i LIBCMT:_wctype.obj
 0001:0004bab5       __iswcsym_l                1004cab5 f i LIBCMT:_wctype.obj
 0001:0004bad9       __iswcsymf_l               1004cad9 f i LIBCMT:_wctype.obj
 0001:0004bafd       __iswdigit_l               1004cafd f i LIBCMT:_wctype.obj
 0001:0004bb0e       __iswgraph_l               1004cb0e f i LIBCMT:_wctype.obj
 0001:0004bb22       __iswlower_l               1004cb22 f i LIBCMT:_wctype.obj
 0001:0004bb33       __iswprint_l               1004cb33 f i LIBCMT:_wctype.obj
 0001:0004bb47       __iswpunct_l               1004cb47 f i LIBCMT:_wctype.obj
 0001:0004bb58       __iswspace_l               1004cb58 f i LIBCMT:_wctype.obj
 0001:0004bb69       __iswupper_l               1004cb69 f i LIBCMT:_wctype.obj
 0001:0004bb7a       __iswxdigit_l              1004cb7a f i LIBCMT:_wctype.obj
 0001:0004bb8e       _isleadbyte                1004cb8e f i LIBCMT:_wctype.obj
 0001:0004bb9f       _iswalnum                  1004cb9f f i LIBCMT:_wctype.obj
 0001:0004bbb3       _iswalpha                  1004cbb3 f i LIBCMT:_wctype.obj
 0001:0004bbc7       _iswascii                  1004cbc7 f i LIBCMT:_wctype.obj
 0001:0004bbd9       _iswblank                  1004cbd9 f i LIBCMT:_wctype.obj
 0001:0004bbf4       _iswcntrl                  1004cbf4 f i LIBCMT:_wctype.obj
 0001:0004bc05       _iswdigit                  1004cc05 f i LIBCMT:_wctype.obj
 0001:0004bc16       _iswgraph                  1004cc16 f i LIBCMT:_wctype.obj
 0001:0004bc2a       _iswlower                  1004cc2a f i LIBCMT:_wctype.obj
 0001:0004bc3b       _iswprint                  1004cc3b f i LIBCMT:_wctype.obj
 0001:0004bc4f       _iswpunct                  1004cc4f f i LIBCMT:_wctype.obj
 0001:0004bc60       _iswspace                  1004cc60 f i LIBCMT:_wctype.obj
 0001:0004bc71       _iswupper                  1004cc71 f i LIBCMT:_wctype.obj
 0001:0004bc82       _iswxdigit                 1004cc82 f i LIBCMT:_wctype.obj
 0001:0004beba       __MallocaIsSizeInRange     1004ceba f i LIBCMT:a_map.obj
 0001:0004becb       __MarkAllocaS              1004cecb f i LIBCMT:a_map.obj
 0001:0004bedf       ___crtLCMapStringA         1004cedf f   LIBCMT:a_map.obj
 0001:0004bf25       __freea                    1004cf25 f i LIBCMT:a_map.obj
 0001:0004bf43       __fltin2                   1004cf43 f   LIBCMT:cfin.obj
 0001:0004bff0       _sin                       1004cff0 f   LIBCMT:sin.obj
 0001:0004c030       __CIsin                    1004d030 f   LIBCMT:sin.obj
 0001:0004c06b       __CIsin_default            1004d06b f   LIBCMT:sin.obj
 0001:0004c07f       __sin_default              1004d07f     LIBCMT:sin.obj
 0001:0004c119       __XcptFilter               1004d119 f   LIBCMT:winxfltr.obj
 0001:0004c274       ___CppXcptFilter           1004d274 f   LIBCMT:winxfltr.obj
 0001:0004c2c6       __set_pgmptr               1004d2c6 f i LIBCMT:stdargv.obj
 0001:0004c2d3       __setargv                  1004d2d3 f   LIBCMT:stdargv.obj
 0001:0004c502       __setenvp                  1004d502 f   LIBCMT:stdenvp.obj
 0001:0004c5e3       ___security_init_cookie    1004d5e3 f   LIBCMT:gs_support.obj
 0001:0004c67f       ___crtGetEnvironmentStringsA 1004d67f f   LIBCMT:a_env.obj
 0001:0004c70c       __RTC_Initialize           1004d70c f   LIBCMT:initsect.obj
 0001:0004c72c       __RTC_Terminate            1004d72c f   LIBCMT:initsect.obj
 0001:0004c74c       ___free_lconv_mon          1004d74c f   LIBCMT:initmon.obj
 0001:0004c848       ___init_monetary           1004d848 f   LIBCMT:initmon.obj
 0001:0004cc21       ___free_lconv_num          1004dc21 f   LIBCMT:initnum.obj
 0001:0004cc88       ___init_numeric            1004dc88 f   LIBCMT:initnum.obj
 0001:0004cec6       ___free_lc_time            1004dec6 f   LIBCMT:inittime.obj
 0001:0004d246       ___init_time               1004e246 f   LIBCMT:inittime.obj
 0001:0004dab5       _localeconv                1004eab5 f   LIBCMT:lconv.obj
 0001:0004dbd3       ___crtGetStringTypeA       1004ebd3 f   LIBCMT:a_str.obj
 0001:0004dc13       ___pctype_func             1004ec13 f   LIBCMT:ctype.obj
 0001:0004dc3c       ___pwctype_func            1004ec3c f   LIBCMT:ctype.obj
 0001:0004dc42       ___init_collate            1004ec42 f   LIBCMT:initcoll.obj
 0001:0004dc45       ____lc_codepage_func       1004ec45 f   LIBCMT:initctyp.obj
 0001:0004dc6b       ____lc_collate_cp_func     1004ec6b f   LIBCMT:initctyp.obj
 0001:0004dc91       ____lc_locale_name_func    1004ec91 f   LIBCMT:initctyp.obj
 0001:0004dcb9       ____mb_cur_max_func        1004ecb9 f   LIBCMT:initctyp.obj
 0001:0004dcdf       ____mb_cur_max_l_func      1004ecdf f   LIBCMT:initctyp.obj
 0001:0004dcf6       ___init_ctype              1004ecf6 f   LIBCMT:initctyp.obj
 0001:0004e1ab       _memcmp                    1004f1ab f   LIBCMT:memcmp.obj
 0001:000510bf       _wcscat_s                  100520bf f   LIBCMT:wcscat_s.obj
 0001:0005112b       _wcscmp                    1005212b f   LIBCMT:wcscmp.obj
 0001:00051169       _wcscpy_s                  10052169 f   LIBCMT:wcscpy_s.obj
 0001:000511c5       _wcscspn                   100521c5 f   LIBCMT:wcscspn.obj
 0001:00051210       _wcslen                    10052210 f   LIBCMT:wcslen.obj
 0001:00051229       _wcsnlen                   10052229 f   LIBCMT:wcslen_s.obj
 0001:00051248       _wcsncmp                   10052248 f   LIBCMT:wcsncmp.obj
 0001:0005127e       _wcsncpy_s                 1005227e f   LIBCMT:wcsncpy_s.obj
 0001:0005133c       _wcspbrk                   1005233c f   LIBCMT:wcspbrk.obj
 0001:00051940       ___get_qualified_locale    10052940 f   LIBCMT:getqloc.obj
 0001:000521b0       ___get_qualified_locale_downlevel 100531b0 f   LIBCMT:getqloc_downlevel.obj
 0001:000523cc       _GetTableIndexFromLcid     100533cc f   LIBCMT:winapinls.obj
 0001:00052401       _GetTableIndexFromLocaleName 10053401 f   LIBCMT:winapinls.obj
 0001:0005244f       ___crtCompareStringEx      1005344f f   LIBCMT:winapinls.obj
 0001:0005249b       ___crtDownlevelLCIDToLocaleName 1005349b f   LIBCMT:winapinls.obj
 0001:00052517       ___crtDownlevelLocaleNameToLCID 10053517 f   LIBCMT:winapinls.obj
 0001:00052555       ___crtEnumSystemLocalesEx  10053555 f   LIBCMT:winapinls.obj
 0001:00052592       ___crtGetDateFormatEx      10053592 f   LIBCMT:winapinls.obj
 0001:000525db       ___crtGetLocaleInfoEx      100535db f   LIBCMT:winapinls.obj
 0001:0005260a       ___crtGetTimeFormatEx      1005360a f   LIBCMT:winapinls.obj
 0001:0005263f       ___crtGetUserDefaultLocaleName 1005363f f   LIBCMT:winapinls.obj
 0001:0005266a       ___crtIsValidLocaleName    1005366a f   LIBCMT:winapinls.obj
 0001:00052695       ___crtLCMapStringEx        10053695 f   LIBCMT:winapinls.obj
 0001:000526e1       ___wcsnicmp_ascii          100536e1 f   LIBCMT:winapinls.obj
 0001:0005274f       __isatty                   1005374f f   LIBCMT:isatty.obj
 0001:000527a3       __getbuf                   100537a3 f   LIBCMT:_getbuf.obj
 0001:000527e9       __wctomb_l                 100537e9 f   LIBCMT:wctomb.obj
 0001:00052838       __wctomb_s_l               10053838 f   LIBCMT:wctomb.obj
 0001:0005295c       _wctomb                    1005395c f   LIBCMT:wctomb.obj
 0001:0005298f       _wctomb_s                  1005398f f   LIBCMT:wctomb.obj
 0001:000529b0       __FindPESection            100539b0 f   LIBCMT:pesect.obj
 0001:00052a00       __IsNonwritableInCurrentImage 10053a00 f   LIBCMT:pesect.obj
 0001:00052ac0       __ValidateImageBase        10053ac0 f   LIBCMT:pesect.obj
 0001:00052af1       ___fpecode                 10053af1 f   LIBCMT:winsig.obj
 0001:00052afa       ___get_sigabrt             10053afa f   LIBCMT:winsig.obj
 0001:00052b07       ___pxcptinfoptrs           10053b07 f   LIBCMT:winsig.obj
 0001:00052b10       __initp_misc_winsig        10053b10 f   LIBCMT:winsig.obj
 0001:00052bd1       _raise                     10053bd1 f   LIBCMT:winsig.obj
 0001:00052dc6       _signal                    10053dc6 f   LIBCMT:winsig.obj
 0001:0005301d       __initp_misc_rand_s        1005401d f   LIBCMT:rand_s.obj
 0001:0005302a       _rand_s                    1005402a f   LIBCMT:rand_s.obj
 0001:00053130       ___set_app_type            10054130 f   LIBCMT:errmode.obj
 0001:0005313d       __set_error_mode           1005413d f   LIBCMT:errmode.obj
 0001:0005317d       ___crtMessageBoxW          1005417d f   LIBCMT:crtmboxw.obj
 0001:00053363       ___crtMessageBoxWaitThreadW@4 10054363 f   LIBCMT:crtmboxw.obj
 0001:00053381       __fcloseall                10054381 f   LIBCMT:closeall.obj
 0001:0005341e       ??0Block@_HeapManager@@QAE@XZ 1005441e f i LIBCMT:undname.obj
 0001:00053424       ??0DName@@QAE@AAPBDD@Z     10054424 f   LIBCMT:undname.obj
 0001:000534dd       ??0DName@@QAE@ABV0@@Z      100544dd f i LIBCMT:undname.obj
 0001:000534f3       ??0DName@@QAE@D@Z          100544f3 f   LIBCMT:undname.obj
 0001:0005351f       ??0DName@@QAE@PAV0@@Z      1005451f f   LIBCMT:undname.obj
 0001:0005356c       ??0DName@@QAE@PBD@Z        1005456c f   LIBCMT:undname.obj
 0001:000535a6       ??0DName@@QAE@W4DNameStatus@@@Z 100545a6 f   LIBCMT:undname.obj
 0001:000535e9       ??0DName@@QAE@XZ           100545e9 f i LIBCMT:undname.obj
 0001:000535fa       ??0DName@@QAE@_J@Z         100545fa f   LIBCMT:undname.obj
 0001:0005368d       ??0DName@@QAE@_K@Z         1005468d f   LIBCMT:undname.obj
 0001:000536fa       ??0DNameNode@@IAE@XZ       100546fa f   LIBCMT:undname.obj
 0001:00053703       ??0DNameStatusNode@@AAE@W4DNameStatus@@@Z 10054703 f   LIBCMT:undname.obj
 0001:00053726       ??0Replicator@@QAE@XZ      10054726 f i LIBCMT:undname.obj
 0001:0005372c       ??0UnDecorator@@QAE@PADPBDHP6APADJ@ZK@Z 1005472c f i LIBCMT:undname.obj
 0001:00053795       ??0charNode@@QAE@D@Z       10054795 f   LIBCMT:undname.obj
 0001:000537aa       ??0pDNameNode@@QAE@PAVDName@@@Z 100547aa f   LIBCMT:undname.obj
 0001:000537d2       ??0pairNode@@QAE@PAVDNameNode@@0@Z 100547d2 f   LIBCMT:undname.obj
 0001:000537f1       ??0pcharNode@@QAE@PBDH@Z   100547f1 f   LIBCMT:undname.obj
 0001:00053848       ??2@YAPAXIAAV_HeapManager@@H@Z 10054848 f i LIBCMT:undname.obj
 0001:0005385d       ??4DName@@QAEAAV0@ABV0@@Z  1005485d f   LIBCMT:undname.obj
 0001:00053873       ??4DName@@QAEAAV0@D@Z      10054873 f i LIBCMT:undname.obj
 0001:0005389f       ??4DName@@QAEAAV0@PAV0@@Z  1005489f f   LIBCMT:undname.obj
 0001:000538e8       ??4DName@@QAEAAV0@PBD@Z    100548e8 f   LIBCMT:undname.obj
 0001:0005391a       ??4DName@@QAEAAV0@W4DNameStatus@@@Z 1005491a f   LIBCMT:undname.obj
 0001:0005394f       ??AReplicator@@QBE?AVDName@@H@Z 1005494f f   LIBCMT:undname.obj
 0001:0005398b       ??BUnDecorator@@QAEPADXZ   1005498b f i LIBCMT:undname.obj
 0001:00053b0a       ??H@YA?AVDName@@DABV0@@Z   10054b0a f i LIBCMT:undname.obj
 0001:00053b2e       ??H@YA?AVDName@@PBDABV0@@Z 10054b2e f i LIBCMT:undname.obj
 0001:00053b52       ??H@YA?AVDName@@W4DNameStatus@@ABV0@@Z 10054b52 f i LIBCMT:undname.obj
 0001:00053b76       ??HDName@@QBE?AV0@ABV0@@Z  10054b76 f   LIBCMT:undname.obj
 0001:00053b98       ??HDName@@QBE?AV0@D@Z      10054b98 f   LIBCMT:undname.obj
 0001:00053bba       ??HDName@@QBE?AV0@PAV0@@Z  10054bba f   LIBCMT:undname.obj
 0001:00053bdc       ??HDName@@QBE?AV0@PBD@Z    10054bdc f   LIBCMT:undname.obj
 0001:00053bfe       ??HDName@@QBE?AV0@W4DNameStatus@@@Z 10054bfe f   LIBCMT:undname.obj
 0001:00053c20       ??YDName@@QAEAAV0@ABV0@@Z  10054c20 f   LIBCMT:undname.obj
 0001:00053c63       ??YDName@@QAEAAV0@D@Z      10054c63 f   LIBCMT:undname.obj
 0001:00053cb3       ??YDName@@QAEAAV0@PAV0@@Z  10054cb3 f   LIBCMT:undname.obj
 0001:00053d18       ??YDName@@QAEAAV0@PBD@Z    10054d18 f   LIBCMT:undname.obj
 0001:00053d79       ??YDName@@QAEAAV0@W4DNameStatus@@@Z 10054d79 f   LIBCMT:undname.obj
 0001:00053db9       ??YReplicator@@QAEAAV0@ABVDName@@@Z 10054db9 f   LIBCMT:undname.obj
 0001:00053e03       ??_5DName@@QAEAAV0@ABV0@@Z 10054e03 f   LIBCMT:undname.obj
 0001:00053e1f       ?Constructor@_HeapManager@@QAEXP6APAXI@ZP6AXPAX@Z@Z 10054e1f f i LIBCMT:undname.obj
 0001:00053e3c       ?Destructor@_HeapManager@@QAEXXZ 10054e3c f i LIBCMT:undname.obj
 0001:00053e62       ?UScore@UnDecorator@@SAPBDW4Tokens@@@Z 10054e62 f   LIBCMT:undname.obj
 0001:00053e7f       ?append@DName@@AAEXPAVDNameNode@@@Z 10054e7f f   LIBCMT:undname.obj
 0001:00053ec5       ?composeDeclaration@UnDecorator@@CA?AVDName@@ABV2@@Z 10054ec5 f i LIBCMT:undname.obj
 0001:00054bfb       ?doAccessSpecifiers@UnDecorator@@SAHXZ 10055bfb f i LIBCMT:undname.obj
 0001:00054c09       ?doAllocationLanguage@UnDecorator@@SAHXZ 10055c09 f i LIBCMT:undname.obj
 0001:00054c17       ?doAllocationModel@UnDecorator@@SAHXZ 10055c17 f i LIBCMT:undname.obj
 0001:00054c25       ?doEcsu@UnDecorator@@SAHXZ 10055c25 f i LIBCMT:undname.obj
 0001:00054c33       ?doEllipsis@UnDecorator@@SAHXZ 10055c33 f i LIBCMT:undname.obj
 0001:00054c41       ?doFunctionReturns@UnDecorator@@SAHXZ 10055c41 f i LIBCMT:undname.obj
 0001:00054c4f       ?doMSKeywords@UnDecorator@@SAHXZ 10055c4f f i LIBCMT:undname.obj
 0001:00054c5c       ?doMemberTypes@UnDecorator@@SAHXZ 10055c5c f i LIBCMT:undname.obj
 0001:00054c6a       ?doNameOnly@UnDecorator@@SAHXZ 10055c6a f i LIBCMT:undname.obj
 0001:00054c75       ?doNoIdentCharCheck@UnDecorator@@SAHXZ 10055c75 f i LIBCMT:undname.obj
 0001:00054c80       ?doPchar@DName@@AAEXPBDH@Z 10055c80 f   LIBCMT:undname.obj
 0001:00054d08       ?doPtr64@UnDecorator@@SAHXZ 10055d08 f i LIBCMT:undname.obj
 0001:00054d16       ?doRestrictionSpec@UnDecorator@@SAHXZ 10055d16 f i LIBCMT:undname.obj
 0001:00054d24       ?doThisTypes@UnDecorator@@SAHXZ 10055d24 f i LIBCMT:undname.obj
 0001:00054d36       ?doThrowTypes@UnDecorator@@SAHXZ 10055d36 f i LIBCMT:undname.obj
 0001:00054d44       ?doTypeOnly@UnDecorator@@SAHXZ 10055d44 f i LIBCMT:undname.obj
 0001:00054d4f       ?doUnderScore@UnDecorator@@SAHXZ 10055d4f f i LIBCMT:undname.obj
 0001:00054d5a       ?getArgumentList@UnDecorator@@CA?AVDName@@XZ 10055d5a f   LIBCMT:undname.obj
 0001:00054e66       ?getArgumentTypes@UnDecorator@@CA?AVDName@@XZ 10055e66 f   LIBCMT:undname.obj
 0001:00054f44       ?getArrayType@UnDecorator@@CA?AVDName@@ABV2@@Z 10055f44 f i LIBCMT:undname.obj
 0001:00055146       ?getBasedType@UnDecorator@@CA?AVDName@@XZ 10056146 f   LIBCMT:undname.obj
 0001:000551dd       ?getBasicDataType@UnDecorator@@CA?AVDName@@ABV2@@Z 100561dd f   LIBCMT:undname.obj
 0001:000555b4       ?getCallIndex@UnDecorator@@CA?AVDName@@XZ 100565b4 f i LIBCMT:undname.obj
 0001:000555c8       ?getCallingConvention@UnDecorator@@CA?AVDName@@XZ 100565c8 f   LIBCMT:undname.obj
 0001:00055687       ?getDataIndirectType@UnDecorator@@CA?AVDName@@ABV2@PBD0H@Z 10056687 f   LIBCMT:undname.obj
 0001:00055c24       ?getDataIndirectType@UnDecorator@@CA?AVDName@@XZ 10056c24 f i LIBCMT:undname.obj
 0001:00055c5d       ?getDataType@UnDecorator@@CA?AVDName@@PAV2@@Z 10056c5d f   LIBCMT:undname.obj
 0001:00055d2f       ?getDecoratedName@UnDecorator@@CA?AVDName@@XZ 10056d2f f   LIBCMT:undname.obj
 0001:00055f7b       ?getDimension@UnDecorator@@CA?AVDName@@_N@Z 10056f7b f   LIBCMT:undname.obj
 0001:000560b2       ?getDispatchTarget@UnDecorator@@CA?AVDName@@XZ 100570b2 f   LIBCMT:undname.obj
 0001:0005610d       ?getDisplacement@UnDecorator@@CA?AVDName@@XZ 1005710d f i LIBCMT:undname.obj
 0001:00056121       ?getECSUDataType@UnDecorator@@CA?AVDName@@XZ 10057121 f   LIBCMT:undname.obj
 0001:00056234       ?getECSUName@UnDecorator@@CA?AVDName@@XZ 10057234 f i LIBCMT:undname.obj
 0001:00056245       ?getEnumType@UnDecorator@@CA?AVDName@@XZ 10057245 f i LIBCMT:undname.obj
 0001:00056329       ?getExtendedDataIndirectType@UnDecorator@@CA?AVDName@@AAPBDAA_NH@Z 10057329 f   LIBCMT:undname.obj
 0001:000564ce       ?getExternalDataType@UnDecorator@@CA?AVDName@@ABV2@@Z 100574ce f i LIBCMT:undname.obj
 0001:00056547       ?getFunctionIndirectType@UnDecorator@@CA?AVDName@@ABV2@@Z 10057547 f   LIBCMT:undname.obj
 0001:0005693d       ?getGuardNumber@UnDecorator@@CA?AVDName@@XZ 1005793d f i LIBCMT:undname.obj
 0001:00056951       ?getLastChar@DName@@QBEDXZ 10057951 f i LIBCMT:undname.obj
 0001:0005695f       ?getLastChar@DNameStatusNode@@UBEDXZ 1005795f f i LIBCMT:undname.obj
 0001:0005696b       ?getLastChar@charNode@@UBEDXZ 1005796b f i LIBCMT:undname.obj
 0001:0005696f       ?getLastChar@pDNameNode@@UBEDXZ 1005796f f i LIBCMT:undname.obj
 0001:00056984       ?getLastChar@pairNode@@UBEDXZ 10057984 f i LIBCMT:undname.obj
 0001:0005699e       ?getLastChar@pcharNode@@UBEDXZ 1005799e f i LIBCMT:undname.obj
 0001:000569b0       ?getLexicalFrame@UnDecorator@@CA?AVDName@@XZ 100579b0 f i LIBCMT:undname.obj
 0001:000569ed       ?getMemory@_HeapManager@@QAEPAXIH@Z 100579ed f   LIBCMT:undname.obj
 0001:00056a72       ?getNumberOfDimensions@UnDecorator@@CAHXZ 10057a72 f   LIBCMT:undname.obj
 0001:00056ad3       ?getOperatorName@UnDecorator@@CA?AVDName@@_NPA_N@Z 10057ad3 f i LIBCMT:undname.obj
 0001:000570ad       ?getPointerType@UnDecorator@@CA?AVDName@@ABV2@0@Z 100580ad f i LIBCMT:undname.obj
 0001:000570cb       ?getPointerTypeArray@UnDecorator@@CA?AVDName@@ABV2@0@Z 100580cb f i LIBCMT:undname.obj
 0001:000570e9       ?getPrimaryDataType@UnDecorator@@CA?AVDName@@ABV2@@Z 100580e9 f   LIBCMT:undname.obj
 0001:000572a1       ?getPtrRefDataType@UnDecorator@@CA?AVDName@@ABV2@H@Z 100582a1 f i LIBCMT:undname.obj
 0001:0005738b       ?getPtrRefType@UnDecorator@@CA?AVDName@@ABV2@0PBD@Z 1005838b f   LIBCMT:undname.obj
 0001:00057487       ?getReferenceType@UnDecorator@@CA?AVDName@@ABV2@0PBD@Z 10058487 f i LIBCMT:undname.obj
 0001:000574a3       ?getRestrictionSpec@UnDecorator@@CA?AVDName@@XZ 100584a3 f   LIBCMT:undname.obj
 0001:00057591       ?getReturnType@UnDecorator@@CA?AVDName@@PAV2@@Z 10058591 f   LIBCMT:undname.obj
 0001:000575c0       ?getScope@UnDecorator@@CA?AVDName@@XZ 100585c0 f   LIBCMT:undname.obj
 0001:00057997       ?getScopedName@UnDecorator@@CA?AVDName@@XZ 10058997 f   LIBCMT:undname.obj
 0001:00057a92       ?getSignedDimension@UnDecorator@@CA?AVDName@@XZ 10058a92 f   LIBCMT:undname.obj
 0001:00057ae5       ?getStorageConvention@UnDecorator@@CA?AVDName@@XZ 10058ae5 f i LIBCMT:undname.obj
 0001:00057af6       ?getString@DName@@QBEPADPAD0@Z 10058af6 f i LIBCMT:undname.obj
 0001:00057b0c       ?getString@DName@@QBEPADPADH@Z 10058b0c f i LIBCMT:undname.obj
 0001:00057b6a       ?getString@DNameStatusNode@@UBEPADPAD0@Z 10058b6a f i LIBCMT:undname.obj
 0001:00057b91       ?getString@charNode@@UBEPADPAD0@Z 10058b91 f i LIBCMT:undname.obj
 0001:00057ba6       ?getString@pDNameNode@@UBEPADPAD0@Z 10058ba6 f i LIBCMT:undname.obj
 0001:00057bc3       ?getString@pairNode@@UBEPADPAD0@Z 10058bc3 f i LIBCMT:undname.obj
 0001:00057bed       ?getString@pcharNode@@UBEPADPAD0@Z 10058bed f i LIBCMT:undname.obj
 0001:00057c08       ?getStringEncoding@UnDecorator@@CA?AVDName@@PADH@Z 10058c08 f   LIBCMT:undname.obj
 0001:00057cab       ?getStringHelper@@YAPADPAD00H@Z 10058cab f i LIBCMT:undname.obj
 0001:00057ce0       ?getSymbolName@UnDecorator@@CA?AVDName@@XZ 10058ce0 f i LIBCMT:undname.obj
 0001:00057d28       ?getTemplateArgumentList@UnDecorator@@CA?AVDName@@XZ 10058d28 f   LIBCMT:undname.obj
 0001:00057fa1       ?getTemplateConstant@UnDecorator@@CA?AVDName@@XZ 10058fa1 f   LIBCMT:undname.obj
 0001:0005829c       ?getTemplateName@UnDecorator@@CA?AVDName@@_N@Z 1005929c f   LIBCMT:undname.obj
 0001:000583f6       ?getThisType@UnDecorator@@CA?AVDName@@XZ 100593f6 f i LIBCMT:undname.obj
 0001:00058430       ?getThrowTypes@UnDecorator@@CA?AVDName@@XZ 10059430 f   LIBCMT:undname.obj
 0001:000584ba       ?getTypeEncoding@UnDecorator@@CAHXZ 100594ba f i LIBCMT:undname.obj
 0001:000589aa       ?getVCallThunkType@UnDecorator@@CA?AVDName@@XZ 100599aa f i LIBCMT:undname.obj
 0001:000589e5       ?getVbTableType@UnDecorator@@CA?AVDName@@ABV2@@Z 100599e5 f i LIBCMT:undname.obj
 0001:000589fa       ?getVdispMapType@UnDecorator@@CA?AVDName@@ABV2@@Z 100599fa f i LIBCMT:undname.obj
 0001:00058a50       ?getVfTableType@UnDecorator@@CA?AVDName@@ABV2@@Z 10059a50 f i LIBCMT:undname.obj
 0001:00058bb5       ?getZName@UnDecorator@@CA?AVDName@@_N0@Z 10059bb5 f   LIBCMT:undname.obj
 0001:00058ddf       ?haveTemplateParameters@UnDecorator@@SAHXZ 10059ddf f i LIBCMT:undname.obj
 0001:00058dea       ?isArray@DName@@QBEHXZ     10059dea f i LIBCMT:undname.obj
 0001:00058df4       ?isComArray@DName@@QBEHXZ  10059df4 f i LIBCMT:undname.obj
 0001:00058dfe       ?isEmpty@DName@@QBEHXZ     10059dfe f i LIBCMT:undname.obj
 0001:00058e06       ?isFull@Replicator@@QBEHXZ 10059e06 f i LIBCMT:undname.obj
 0001:00058e0f       ?isNoTE@DName@@QBEHXZ      10059e0f f i LIBCMT:undname.obj
 0001:00058e19       ?isPinPtr@DName@@QBEHXZ    10059e19 f i LIBCMT:undname.obj
 0001:00058e23       ?isPtrRef@DName@@QBEHXZ    10059e23 f i LIBCMT:undname.obj
 0001:00058e2d       ?isUDC@DName@@QBEHXZ       10059e2d f i LIBCMT:undname.obj
 0001:00058e3e       ?isUDTThunk@DName@@QBEHXZ  10059e3e f i LIBCMT:undname.obj
 0001:00058e4f       ?isVCallThunk@DName@@QBEHXZ 10059e4f f i LIBCMT:undname.obj
 0001:00058e59       ?isValid@DName@@QBEHXZ     10059e59 f i LIBCMT:undname.obj
 0001:00058e63       ?length@DName@@QBEHXZ      10059e63 f i LIBCMT:undname.obj
 0001:00058e70       ?length@DNameStatusNode@@UBEHXZ 10059e70 f i LIBCMT:undname.obj
 0001:00058e74       ?length@charNode@@UBEHXZ   10059e74 f i LIBCMT:undname.obj
 0001:00058e78       ?length@pDNameNode@@UBEHXZ 10059e78 f i LIBCMT:undname.obj
 0001:00058e8c       ?length@pairNode@@UBEHXZ   10059e8c f i LIBCMT:undname.obj
 0001:00058eb5       ?length@pcharNode@@UBEHXZ  10059eb5 f i LIBCMT:undname.obj
 0001:00058eb9       ?make@DNameStatusNode@@SAPAV1@W4DNameStatus@@@Z 10059eb9 f i LIBCMT:undname.obj
 0001:00058f3f       ?setIsArray@DName@@QAEXXZ  10059f3f f i LIBCMT:undname.obj
 0001:00058f47       ?setIsComArray@DName@@QAEXXZ 10059f47 f i LIBCMT:undname.obj
 0001:00058f4f       ?setIsNoTE@DName@@QAEXXZ   10059f4f f i LIBCMT:undname.obj
 0001:00058f57       ?setIsPinPtr@DName@@QAEXXZ 10059f57 f i LIBCMT:undname.obj
 0001:00058f5f       ?setIsUDC@DName@@QAEXXZ    10059f5f f i LIBCMT:undname.obj
 0001:00058f6c       ?setIsVCallThunk@DName@@QAEXXZ 10059f6c f i LIBCMT:undname.obj
 0001:00058f74       ?setPtrRef@DName@@QAEAAV1@XZ 10059f74 f i LIBCMT:undname.obj
 0001:00058f7e       ?status@DName@@QBE?AW4DNameStatus@@XZ 10059f7e f i LIBCMT:undname.obj
 0001:00058fe6       ___unDName                 10059fe6 f   LIBCMT:undname.obj
 0001:00059089       ___unDNameEx               1005a089 f   LIBCMT:undname.obj
 0001:00059130       _strrchr                   1005a130 f   LIBCMT:strrchr.obj
 0001:00059267       __fptostr                  1005a267 f   LIBCMT:_fptostr.obj
 0001:00059317       ___dtold                   1005a317 f   LIBCMT:cfout.obj
 0001:000593df       __fltout2                  1005a3df f   LIBCMT:cfout.obj
 0001:00059470       __alldvrm                  1005a470 f   LIBCMT:lldvrm.obj
 0001:00059550       __aullshr                  1005a550 f   LIBCMT:ullshr.obj
 0001:0005956f       __get_output_format        1005a56f f   LIBCMT:outputformat.obj
 0001:00059575       __set_output_format        1005a575 f   LIBCMT:outputformat.obj
 0001:000595a7       __controlfp_s              1005a5a7 f   LIBCMT:contrlfp.obj
 0001:00059604       __fptrap                   1005a604 f   LIBCMT:crt0fp.obj
 0001:0005960d       _strncpy_s                 1005a60d f   LIBCMT:strncpy_s.obj
 0001:00059795       ___crtGetLocaleInfoA       1005a795 f   LIBCMT:a_loc.obj
 0001:000597cf       _realloc                   1005a7cf f   LIBCMT:realloc.obj
 0001:0005987a       __recalloc                 1005a87a f   LIBCMT:recalloc.obj
 0001:000598e3       __calloc_impl              1005a8e3 f   LIBCMT:calloc_impl.obj
 0001:0005995d       __CopyMan                  1005a95d f i LIBCMT:intrncvt.obj
 0001:0005997a       __FillZeroMan              1005a97a f i LIBCMT:intrncvt.obj
 0001:00059989       __IncMan                   1005a989 f i LIBCMT:intrncvt.obj
 0001:000599eb       __IsZeroMan                1005a9eb f i LIBCMT:intrncvt.obj
 0001:00059a08       __RoundMan                 1005aa08 f i LIBCMT:intrncvt.obj
 0001:00059b09       __ShrMan                   1005ab09 f i LIBCMT:intrncvt.obj
 0001:00059b97       __ZeroTail                 1005ab97 f i LIBCMT:intrncvt.obj
 0001:00059bdf       ___addl                    1005abdf f i LIBCMT:intrncvt.obj
 0001:00059c03       __ld12cvt                  1005ac03 f i LIBCMT:intrncvt.obj
 0001:0005a16e       __ld12tod                  1005b16e f   LIBCMT:intrncvt.obj
 0001:0005a6e0       __ld12tof                  1005b6e0 f   LIBCMT:intrncvt.obj
 0001:0005ac52       __ld12told                 1005bc52 f   LIBCMT:intrncvt.obj
 0001:0005ad21       ___STRINGTOLD_L            1005bd21 f   LIBCMT:strgtold.obj
 0001:0005ad7c       ___ld12mul                 1005bd7c f i LIBCMT:strgtold.obj
 0001:0005b048       ___multtenpow12            1005c048 f i LIBCMT:strgtold.obj
 0001:0005b39b       ___shl_12                  1005c39b f i LIBCMT:strgtold.obj
 0001:0005b3cc       ___shr_12                  1005c3cc f i LIBCMT:strgtold.obj
 0001:0005b3fc       ___strgtold12_l            1005c3fc f   LIBCMT:strgtold.obj
 0001:0005bbb0       __trandisp1                1005cbb0 f   LIBCMT:87disp.obj
 0001:0005bc17       __trandisp2                1005cc17 f   LIBCMT:87disp.obj
 0001:0005bca3       __rttospopde               1005cca3     LIBCMT:87disp.obj
 0001:0005bca8       __rttospop                 1005cca8     LIBCMT:87disp.obj
 0001:0005bcaa       __rtnospop                 1005ccaa     LIBCMT:87disp.obj
 0001:0005bcac       __rttosnpop                1005ccac     LIBCMT:87disp.obj
 0001:0005bcad       __rtnospopde               1005ccad     LIBCMT:87disp.obj
 0001:0005bcb4       __rtzeropop                1005ccb4     LIBCMT:87disp.obj
 0001:0005bcb6       __rtzeronpop               1005ccb6     LIBCMT:87disp.obj
 0001:0005bcbb       __rtonepop                 1005ccbb     LIBCMT:87disp.obj
 0001:0005bcbd       __rtonenpop                1005ccbd     LIBCMT:87disp.obj
 0001:0005bcc2       __tosnan1                  1005ccc2     LIBCMT:87disp.obj
 0001:0005bced       __nosnan2                  1005cced     LIBCMT:87disp.obj
 0001:0005bcef       __tosnan2                  1005ccef     LIBCMT:87disp.obj
 0001:0005bd17       __nan2                     1005cd17     LIBCMT:87disp.obj
 0001:0005bd56       __rtindfpop                1005cd56     LIBCMT:87disp.obj
 0001:0005bd58       __rtindfnpop               1005cd58     LIBCMT:87disp.obj
 0001:0005bd69       __rttosnpopde              1005cd69     LIBCMT:87disp.obj
 0001:0005bd73       __rtchsifneg               1005cd73     LIBCMT:87disp.obj
 0001:0005bd80       __startTwoArgErrorHandling 1005cd80 f   LIBCMT:genexcep.obj
 0001:0005bd97       __startOneArgErrorHandling 1005cd97 f   LIBCMT:genexcep.obj
 0001:0005bde0       __twoToTOS                 1005cde0 f   LIBCMT:common.obj
 0001:0005bdf5       __load_CW                  1005cdf5 f   LIBCMT:common.obj
 0001:0005be0c       __convertTOStoQNaN         1005ce0c f   LIBCMT:common.obj
 0001:0005be25       __fload_withFB             1005ce25 f   LIBCMT:common.obj
 0001:0005be68       __checkTOS_withFB          1005ce68 f   LIBCMT:common.obj
 0001:0005be7e       __fast_exit                1005ce7e f   LIBCMT:common.obj
 0001:0005be8b       __math_exit                1005ce8b f   LIBCMT:common.obj
 0001:0005beb5       __check_overflow_exit      1005ceb5 f   LIBCMT:common.obj
 0001:0005bec9       __check_range_exit         1005cec9 f   LIBCMT:common.obj
 0001:0005bf6c       __matherr                  1005cf6c f   LIBCMT:matherr.obj
 0001:0005bf70       __global_unwind2           1005cf70 f   LIBCMT:exsup.obj
 0001:0005bfd5       __local_unwind2            1005cfd5 f   LIBCMT:exsup.obj
 0001:0005c059       __abnormal_termination     1005d059 f   LIBCMT:exsup.obj
 0001:0005c07c       __NLG_Notify1              1005d07c f   LIBCMT:exsup.obj
 0001:0005c085       __NLG_Notify               1005d085 f   LIBCMT:exsup.obj
 0001:0005c09c       __NLG_Dispatch             1005d09c     LIBCMT:exsup.obj
 0001:0005c09c       __NLG_Dispatch2            1005d09c     LIBCMT:exsup.obj
 0001:0005c0a4       __NLG_Call                 1005d0a4 f   LIBCMT:exsup.obj
 0001:0005c0a6       __NLG_Return2              1005d0a6     LIBCMT:exsup.obj
 0001:0005c0a7       ?_ValidateExecute@@YAHP6GHXZ@Z 1005d0a7 f   LIBCMT:validate.obj
 0001:0005c0b6       ?_ValidateRead@@YAHPBXI@Z  1005d0b6 f   LIBCMT:validate.obj
 0001:0005c0c5       ?_ValidateWrite@@YAHPAXI@Z 1005d0c5 f   LIBCMT:validate.obj
 0001:0005c0d4       __EH_epilog3               1005d0d4 f   LIBCMT:ehprolg3.obj
 0001:0005c0e8       __EH_epilog3_GS            1005d0e8 f   LIBCMT:ehprolg3.obj
 0001:0005c0f7       __EH_epilog3_catch_GS      1005d0f7 f   LIBCMT:ehprolg3.obj
 0001:0005c106       __EH_prolog3               1005d106 f   LIBCMT:ehprolg3.obj
 0001:0005c139       __EH_prolog3_GS            1005d139 f   LIBCMT:ehprolg3.obj
 0001:0005c16f       __EH_prolog3_catch         1005d16f f   LIBCMT:ehprolg3.obj
 0001:0005c1a5       __EH_prolog3_catch_GS      1005d1a5 f   LIBCMT:ehprolg3.obj
 0001:0005c1de       ___crtsetenv               1005d1de f   LIBCMT:setenv.obj
 0001:0005c4e1       __strnicoll                1005d4e1 f   LIBCMT:strnicol.obj
 0001:0005c508       __strnicoll_l              1005d508 f   LIBCMT:strnicol.obj
 0001:0005c871       ___crtCompareStringA       1005d871 f   LIBCMT:a_cmp.obj
 0001:0005c8b4       __sse2_mathfcns_init       1005d8b4 f   LIBCMT:mathfcns.obj
 0001:0005c8c3       __set_SSE2_enable          1005d8c3 f   LIBCMT:mathfcns.obj
 0001:0005c8f0       __CIlog10_pentium4         1005d8f0 f   LIBCMT:log10_pentium4.obj
 0001:0005c908       __log10_pentium4           1005d908     LIBCMT:log10_pentium4.obj
 0001:0005cb91       __fFEXP                    1005db91     LIBCMT:87tran.obj
 0001:0005cbe8       __rtinfpopse               1005dbe8     LIBCMT:87tran.obj
 0001:0005cbea       __rtinfnpopse              1005dbea     LIBCMT:87tran.obj
 0001:0005cbfa       __fFLN                     1005dbfa     LIBCMT:87tran.obj
 0001:0005ccaf       __rtinfpop                 1005dcaf     LIBCMT:87tran.obj
 0001:0005ccb1       __rtinfnpop                1005dcb1     LIBCMT:87tran.obj
 0001:0005ccce       __ffexpm1                  1005dcce     LIBCMT:87tran.obj
 0001:0005cd80       __CIpow_pentium4           1005dd80 f   LIBCMT:pow_pentium4.obj
 0001:0005cd99       __pow_pentium4             1005dd99     LIBCMT:pow_pentium4.obj
 0001:0005d8e0       __d_inttype                1005e8e0 f   LIBCMT:powhlp.obj
 0001:0005d948       __powhlp                   1005e948 f   LIBCMT:powhlp.obj
 0001:0005da7e       ___lock_fhandle            1005ea7e f   LIBCMT:osfinfo.obj
 0001:0005db0c       __alloc_osfhnd             1005eb0c f   LIBCMT:osfinfo.obj
 0001:0005dcb5       __free_osfhnd              1005ecb5 f   LIBCMT:osfinfo.obj
 0001:0005dd3b       __get_osfhandle            1005ed3b f   LIBCMT:osfinfo.obj
 0001:0005dda2       __open_osfhandle           1005eda2 f   LIBCMT:osfinfo.obj
 0001:0005deb8       __set_osfhnd               1005eeb8 f   LIBCMT:osfinfo.obj
 0001:0005df3a       __unlock_fhandle           1005ef3a f   LIBCMT:osfinfo.obj
 0001:0005df60       __commit                   1005ef60 f   LIBCMT:commit.obj
 0001:0005e049       __open                     1005f049 f   LIBCMT:open.obj
 0001:0005e0f9       __sopen                    1005f0f9 f   LIBCMT:open.obj
 0001:0005e12c       __sopen_helper             1005f12c f   LIBCMT:open.obj
 0001:0005e1f5       __sopen_nolock             1005f1f5 f   LIBCMT:open.obj
 0001:0005e243       __sopen_s                  1005f243 f   LIBCMT:open.obj
 0001:0005e261       __mbsnbcmp                 1005f261 f   LIBCMT:mbsnbcmp.obj
 0001:0005e279       __mbsnbcmp_l               1005f279 f   LIBCMT:mbsnbcmp.obj
 0001:0005e390       __mbsnbicmp                1005f390 f   LIBCMT:mbsnbicm.obj
 0001:0005e3a8       __mbsnbicmp_l              1005f3a8 f   LIBCMT:mbsnbicm.obj
 0001:0005e563       __mbtowc_l                 1005f563 f   LIBCMT:mbtowc.obj
 0001:0005e658       _mbtowc                    1005f658 f   LIBCMT:mbtowc.obj
 0001:0005e670       __putwch                   1005f670 f   LIBCMT:putwch.obj
 0001:0005e6bc       __putwch_nolock            1005f6bc f   LIBCMT:putwch.obj
 0001:0005e6ff       __iswctype_l               1005f6ff f   LIBCMT:iswctype.obj
 0001:0005e711       _is_wctype                 1005f711 f   LIBCMT:iswctype.obj
 0001:0005e71a       _iswctype                  1005f71a f   LIBCMT:iswctype.obj
 0001:0005e770       __alloca_probe_16          1005f770 f   LIBCMT:alloca16.obj
 0001:0005e786       __alloca_probe_8           1005f786     LIBCMT:alloca16.obj
 0001:0005e7a0       __CIsin_pentium4           1005f7a0 f   LIBCMT:sin_pentium4.obj
 0001:0005e7b8       __sin_pentium4             1005f7b8     LIBCMT:sin_pentium4.obj
 0001:0005e9c2       __ismbbalnum               1005f9c2 f   LIBCMT:ismbbyte.obj
 0001:0005e9db       __ismbbalnum_l             1005f9db f   LIBCMT:ismbbyte.obj
 0001:0005e9f5       __ismbbalpha               1005f9f5 f   LIBCMT:ismbbyte.obj
 0001:0005ea0e       __ismbbalpha_l             1005fa0e f   LIBCMT:ismbbyte.obj
 0001:0005ea28       __ismbbblank               1005fa28 f   LIBCMT:ismbbyte.obj
 0001:0005ea49       __ismbbblank_l             1005fa49 f   LIBCMT:ismbbyte.obj
 0001:0005ea6b       __ismbbgraph               1005fa6b f   LIBCMT:ismbbyte.obj
 0001:0005ea84       __ismbbgraph_l             1005fa84 f   LIBCMT:ismbbyte.obj
 0001:0005ea9e       __ismbbkalnum              1005fa9e f   LIBCMT:ismbbyte.obj
 0001:0005eab4       __ismbbkalnum_l            1005fab4 f   LIBCMT:ismbbyte.obj
 0001:0005eacb       __ismbbkana                1005facb f   LIBCMT:ismbbyte.obj
 0001:0005eadc       __ismbbkana_l              1005fadc f   LIBCMT:ismbbyte.obj
 0001:0005eb28       __ismbbkprint              1005fb28 f   LIBCMT:ismbbyte.obj
 0001:0005eb3e       __ismbbkprint_l            1005fb3e f   LIBCMT:ismbbyte.obj
 0001:0005eb55       __ismbbkpunct              1005fb55 f   LIBCMT:ismbbyte.obj
 0001:0005eb6b       __ismbbkpunct_l            1005fb6b f   LIBCMT:ismbbyte.obj
 0001:0005eb82       __ismbblead                1005fb82 f   LIBCMT:ismbbyte.obj
 0001:0005eb98       __ismbblead_l              1005fb98 f   LIBCMT:ismbbyte.obj
 0001:0005ebaf       __ismbbprint               1005fbaf f   LIBCMT:ismbbyte.obj
 0001:0005ebc8       __ismbbprint_l             1005fbc8 f   LIBCMT:ismbbyte.obj
 0001:0005ebe2       __ismbbpunct               1005fbe2 f   LIBCMT:ismbbyte.obj
 0001:0005ebf8       __ismbbpunct_l             1005fbf8 f   LIBCMT:ismbbyte.obj
 0001:0005ec0f       __ismbbtrail               1005fc0f f   LIBCMT:ismbbyte.obj
 0001:0005ec25       __ismbbtrail_l             1005fc25 f   LIBCMT:ismbbyte.obj
 0001:0005ed58       __i64tow_s                 1005fd58 f   LIBCMT:xtows.obj
 0001:0005ed89       __itow_s                   1005fd89 f   LIBCMT:xtows.obj
 0001:0005edb2       __ltow_s                   1005fdb2 f   LIBCMT:xtows.obj
 0001:0005eddc       __ui64tow_s                1005fddc f   LIBCMT:xtows.obj
 0001:0005edf7       __ultow_s                  1005fdf7 f   LIBCMT:xtows.obj
 0001:0005ef02       __wtoi                     1005ff02 f   LIBCMT:wtox.obj
 0001:0005ef0b       __wtoi64                   1005ff0b f   LIBCMT:wtox.obj
 0001:0005ef1f       __wtoi64_l                 1005ff1f f   LIBCMT:wtox.obj
 0001:0005ef36       __wtoi_l                   1005ff36 f   LIBCMT:wtox.obj
 0001:0005ef3f       __wtol                     1005ff3f f   LIBCMT:wtox.obj
 0001:0005ef53       __wtol_l                   1005ff53 f   LIBCMT:wtox.obj
 0001:0005ef6a       __wtoll                    1005ff6a f   LIBCMT:wtox.obj
 0001:0005ef7e       __wtoll_l                  1005ff7e f   LIBCMT:wtox.obj
 0001:0005ef95       _wcschr                    1005ff95 f   LIBCMT:wcschr.obj
 0001:0005f043       __wcsicmp                  10060043 f   LIBCMT:wcsicmp.obj
 0001:0005f0d6       __wcsicmp_l                100600d6 f   LIBCMT:wcsicmp.obj
 0001:0005f1b1       __wcsnicmp                 100601b1 f   LIBCMT:wcsnicmp.obj
 0001:0005f267       __wcsnicmp_l               10060267 f   LIBCMT:wcsnicmp.obj
 0001:0005f360       __atoi64                   10060360 f   LIBCMT:atox.obj
 0001:0005f374       __atoi64_l                 10060374 f   LIBCMT:atox.obj
 0001:0005f38b       __atoi_l                   1006038b f   LIBCMT:atox.obj
 0001:0005f394       __atol_l                   10060394 f   LIBCMT:atox.obj
 0001:0005f3ab       __atoll_l                  100603ab f   LIBCMT:atox.obj
 0001:0005f3c2       _atoi                      100603c2 f   LIBCMT:atox.obj
 0001:0005f3cb       _atol                      100603cb f   LIBCMT:atox.obj
 0001:0005f3df       _atoll                     100603df f   LIBCMT:atox.obj
 0001:0005f3f3       _$I10_OUTPUT               100603f3 f   LIBCMT:x10fout.obj
 0001:0005fdc7       ___add_12                  10060dc7 f i LIBCMT:x10fout.obj
 0001:0005ff73       ___control87_2             10060f73 f   LIBCMT:ieee87.obj
 0001:000605e7       __clearfp                  100615e7 f   LIBCMT:ieee87.obj
 0001:000606c7       __control87                100616c7 f i LIBCMT:ieee87.obj
 0001:000609c9       __controlfp                100619c9 f   LIBCMT:ieee87.obj
 0001:00060cd4       __fpreset                  10061cd4 f   LIBCMT:ieee87.obj
 0001:00060da1       __set_controlfp            10061da1 f   LIBCMT:ieee87.obj
 0001:00060e14       __statusfp                 10061e14 f   LIBCMT:ieee87.obj
 0001:00060eae       __statusfp2                10061eae f   LIBCMT:ieee87.obj
 0001:00060f0d       ___mtold12                 10061f0d f   LIBCMT:mantold.obj
 0001:000610ed       __87except                 100620ed f   LIBCMT:87except.obj
 0001:000611f6       __mbschr                   100621f6 f   LIBCMT:mbschr.obj
 0001:0006120b       __mbschr_l                 1006220b f   LIBCMT:mbschr.obj
 0001:000612a8       __strnicmp                 100622a8 f   LIBCMT:strnicmp.obj
 0001:00061313       __strnicmp_l               10062313 f   LIBCMT:strnicmp.obj
 0001:000613c4       __frnd                     100623c4 f   LIBCMT:frnd.obj
 0001:000613d8       __chgsign                  100623d8 f   LIBCMT:ieeemisc.obj
 0001:00061405       __chgsignf                 10062405 f   LIBCMT:ieeemisc.obj
 0001:00061426       __copysign                 10062426 f   LIBCMT:ieeemisc.obj
 0001:0006144e       __copysignf                1006244e f   LIBCMT:ieeemisc.obj
 0001:0006146a       __finite                   1006246a f   LIBCMT:ieeemisc.obj
 0001:00061482       __fpclass                  10062482 f   LIBCMT:ieeemisc.obj
 0001:0006151e       __isnan                    1006251e f   LIBCMT:ieeemisc.obj
 0001:00061551       __logb                     10062551 f   LIBCMT:ieeemisc.obj
 0001:00061632       __nextafter                10062632 f   LIBCMT:ieeemisc.obj
 0001:000618d2       __scalb                    100628d2 f   LIBCMT:ieeemisc.obj
 0001:00061972       __wopen                    10062972 f   LIBCMT:wopen.obj
 0001:00061a22       __wsopen                   10062a22 f   LIBCMT:wopen.obj
 0001:00061a55       __wsopen_helper            10062a55 f   LIBCMT:wopen.obj
 0001:00061b1e       __wsopen_nolock            10062b1e f   LIBCMT:wopen.obj
 0001:00062271       __wsopen_s                 10063271 f   LIBCMT:wopen.obj
 0001:0006228f       ___termconout              1006328f f   LIBCMT:initcon.obj
 0001:000622a6       ___initconout              100632a6 f   LIBCMT:initcon.obj
 0001:000624a6       __wcstol_l                 100634a6 f   LIBCMT:wcstol.obj
 0001:000624be       __wcstoul_l                100634be f   LIBCMT:wcstol.obj
 0001:000624d6       _wcstol                    100634d6 f   LIBCMT:wcstol.obj
 0001:000624ee       _wcstoul                   100634ee f   LIBCMT:wcstol.obj
 0001:000627d6       __wcstof_l                 100637d6 f   LIBCMT:wcstoq.obj
 0001:00062889       __wcstoi64                 10063889 f   LIBCMT:wcstoq.obj
 0001:000628b3       __wcstoi64_l               100638b3 f   LIBCMT:wcstoq.obj
 0001:000628ce       __wcstoimax_l              100638ce f   LIBCMT:wcstoq.obj
 0001:000628d7       __wcstold_l                100638d7 f   LIBCMT:wcstoq.obj
 0001:000628e0       __wcstoll_l                100638e0 f   LIBCMT:wcstoq.obj
 0001:000628e9       __wcstoui64                100638e9 f   LIBCMT:wcstoq.obj
 0001:00062913       __wcstoui64_l              10063913 f   LIBCMT:wcstoq.obj
 0001:0006292e       __wcstoull_l               1006392e f   LIBCMT:wcstoq.obj
 0001:00062937       __wcstoumax_l              10063937 f   LIBCMT:wcstoq.obj
 0001:00062940       _wcstof                    10063940 f   LIBCMT:wcstoq.obj
 0001:00062955       _wcstoimax                 10063955 f   LIBCMT:wcstoq.obj
 0001:0006295e       _wcstold                   1006395e f   LIBCMT:wcstoq.obj
 0001:00062967       _wcstoll                   10063967 f   LIBCMT:wcstoq.obj
 0001:00062970       _wcstoull                  10063970 f   LIBCMT:wcstoq.obj
 0001:00062979       _wcstoumax                 10063979 f   LIBCMT:wcstoq.obj
 0001:00062982       __towlower_l               10063982 f   LIBCMT:towlower.obj
 0001:00062a33       _towlower                  10063a33 f   LIBCMT:towlower.obj
 0001:00062a50       ___ascii_strnicmp          10063a50 f   LIBCMT:_strnicm.obj
 0001:00062ab1       _ldexp                     10063ab1 f   LIBCMT:ldexp.obj
 0001:00062c9d       __chsize                   10063c9d f   LIBCMT:chsize.obj
 0001:00062cb7       __chsize_nolock            10063cb7 f   LIBCMT:chsize.obj
 0001:00062e6d       __chsize_s                 10063e6d f   LIBCMT:chsize.obj
 0001:00062f5b       __get_fmode                10063f5b f   LIBCMT:setmode.obj
 0001:00062f85       __set_fmode                10063f85 f   LIBCMT:setmode.obj
 0001:00062fc0       __setmode                  10063fc0 f   LIBCMT:setmode.obj
 0001:000630c5       __setmode_nolock           100640c5 f   LIBCMT:setmode.obj
 0001:00063192       __wchartodigit             10064192 f   LIBCMT:wchtodig.obj
 0001:00063331       __wcstod_l                 10064331 f   LIBCMT:wcstod.obj
 0001:0006342c       _wcstod                    1006442c f   LIBCMT:wcstod.obj
 0001:00063441       ___crtLCMapStringW         10064441 f   LIBCMT:w_map.obj
 0001:00063470       __wfltin2                  10064470 f   LIBCMT:wcfin.obj
 0001:00063519       ___WSTRINGTOLD_L           10064519 f   LIBCMT:wstrgtold.obj
 0001:00063574       ___wstrgtold12_l           10064574 f   LIBCMT:wstrgtold.obj
 0001:00063dc4       ??0_Ignore@std@@QAE@XZ     10064dc4 f i libcpmt:xthrow.obj
 0001:00063dc7       ??0bad_function_call@std@@QAE@ABV01@@Z 10064dc7 f i libcpmt:xthrow.obj
 0001:00063de2       ??0bad_function_call@std@@QAE@PBD@Z 10064de2 f i libcpmt:xthrow.obj
 0001:00063df6       ??0invalid_argument@std@@QAE@ABV01@@Z 10064df6 f i libcpmt:xthrow.obj
 0001:00063e11       ??0invalid_argument@std@@QAE@PBD@Z 10064e11 f i libcpmt:xthrow.obj
 0001:00063e33       ??0length_error@std@@QAE@ABV01@@Z 10064e33 f i libcpmt:xthrow.obj
 0001:00063e4e       ??0length_error@std@@QAE@PBD@Z 10064e4e f i libcpmt:xthrow.obj
 0001:00063e70       ??0logic_error@std@@QAE@ABV01@@Z 10064e70 f i libcpmt:xthrow.obj
 0001:00063e8b       ??0logic_error@std@@QAE@PBD@Z 10064e8b f i libcpmt:xthrow.obj
 0001:00063ea7       ??0out_of_range@std@@QAE@ABV01@@Z 10064ea7 f i libcpmt:xthrow.obj
 0001:00063ec2       ??0out_of_range@std@@QAE@PBD@Z 10064ec2 f i libcpmt:xthrow.obj
 0001:00063ee4       ??0overflow_error@std@@QAE@ABV01@@Z 10064ee4 f i libcpmt:xthrow.obj
 0001:00063eff       ??0overflow_error@std@@QAE@PBD@Z 10064eff f i libcpmt:xthrow.obj
 0001:00063f21       ??0regex_error@std@@QAE@ABV01@@Z 10064f21 f i libcpmt:xthrow.obj
 0001:00063f45       ??0regex_error@std@@QAE@W4error_type@regex_constants@1@@Z 10064f45 f i libcpmt:xthrow.obj
 0001:00063f75       ??0runtime_error@std@@QAE@ABV01@@Z 10064f75 f i libcpmt:xthrow.obj
 0001:00063f90       ??0runtime_error@std@@QAE@PBD@Z 10064f90 f i libcpmt:xthrow.obj
 0001:00063fac       ??1bad_function_call@std@@UAE@XZ 10064fac f i libcpmt:xthrow.obj
 0001:00063fb1       ??1invalid_argument@std@@UAE@XZ 10064fb1 f i libcpmt:xthrow.obj
 0001:00063fb6       ??1length_error@std@@UAE@XZ 10064fb6 f i libcpmt:xthrow.obj
 0001:00063fbb       ??1logic_error@std@@UAE@XZ 10064fbb f i libcpmt:xthrow.obj
 0001:00063fc0       ??1out_of_range@std@@UAE@XZ 10064fc0 f i libcpmt:xthrow.obj
 0001:00063fc5       ??1overflow_error@std@@UAE@XZ 10064fc5 f i libcpmt:xthrow.obj
 0001:00063fca       ??1regex_error@std@@UAE@XZ 10064fca f i libcpmt:xthrow.obj
 0001:00063fcf       ??1runtime_error@std@@UAE@XZ 10064fcf f i libcpmt:xthrow.obj
 0001:00063fd4       ??_Gbad_function_call@std@@UAEPAXI@Z 10064fd4 f i libcpmt:xthrow.obj
 0001:00063fd4       ??_Ebad_function_call@std@@UAEPAXI@Z 10064fd4 f i libcpmt:xthrow.obj
 0001:00063ff3       ??_Ginvalid_argument@std@@UAEPAXI@Z 10064ff3 f i libcpmt:xthrow.obj
 0001:00063ff3       ??_Einvalid_argument@std@@UAEPAXI@Z 10064ff3 f i libcpmt:xthrow.obj
 0001:00064012       ??_Glength_error@std@@UAEPAXI@Z 10065012 f i libcpmt:xthrow.obj
 0001:00064012       ??_Elength_error@std@@UAEPAXI@Z 10065012 f i libcpmt:xthrow.obj
 0001:00064031       ??_Elogic_error@std@@UAEPAXI@Z 10065031 f i libcpmt:xthrow.obj
 0001:00064031       ??_Glogic_error@std@@UAEPAXI@Z 10065031 f i libcpmt:xthrow.obj
 0001:00064050       ??_Gout_of_range@std@@UAEPAXI@Z 10065050 f i libcpmt:xthrow.obj
 0001:00064050       ??_Eout_of_range@std@@UAEPAXI@Z 10065050 f i libcpmt:xthrow.obj
 0001:0006406f       ??_Eoverflow_error@std@@UAEPAXI@Z 1006506f f i libcpmt:xthrow.obj
 0001:0006406f       ??_Goverflow_error@std@@UAEPAXI@Z 1006506f f i libcpmt:xthrow.obj
 0001:0006408e       ??_Gregex_error@std@@UAEPAXI@Z 1006508e f i libcpmt:xthrow.obj
 0001:0006408e       ??_Eregex_error@std@@UAEPAXI@Z 1006508e f i libcpmt:xthrow.obj
 0001:000640ad       ??_Gruntime_error@std@@UAEPAXI@Z 100650ad f i libcpmt:xthrow.obj
 0001:000640ad       ??_Eruntime_error@std@@UAEPAXI@Z 100650ad f i libcpmt:xthrow.obj
 0001:000640cc       ?_Stringify@regex_error@std@@CAPBDW4error_type@regex_constants@2@@Z 100650cc f i libcpmt:xthrow.obj
 0001:0006418c       ?_Xbad_alloc@std@@YAXXZ    1006518c f   libcpmt:xthrow.obj
 0001:000641bd       ?_Xbad_function_call@std@@YAXXZ 100651bd f   libcpmt:xthrow.obj
 0001:000641e1       ?_Xinvalid_argument@std@@YAXPBD@Z 100651e1 f   libcpmt:xthrow.obj
 0001:0006420f       ?_Xlength_error@std@@YAXPBD@Z 1006520f f   libcpmt:xthrow.obj
 0001:0006423d       ?_Xout_of_range@std@@YAXPBD@Z 1006523d f   libcpmt:xthrow.obj
 0001:0006426b       ?_Xoverflow_error@std@@YAXPBD@Z 1006526b f   libcpmt:xthrow.obj
 0001:00064299       ?_Xregex_error@std@@YAXW4error_type@regex_constants@1@@Z 10065299 f   libcpmt:xthrow.obj
 0001:000642b9       ?_Xruntime_error@std@@YAXPBD@Z 100652b9 f   libcpmt:xthrow.obj
 0001:000642e7       ?what@bad_function_call@std@@UBEPBDXZ 100652e7 f i libcpmt:xthrow.obj
 0001:000642ed       ?_Syserror_map@std@@YAPBDH@Z 100652ed f   libcpmt:syserror.obj
 0001:00064317       ?_Winerror_map@std@@YAPBDH@Z 10065317 f   libcpmt:syserror.obj
 0001:00064342       _RaiseException@16         10065342 f   kernel32:KERNEL32.dll
 0001:00064348       _FreeLibrary@4             10065348 f   kernel32:KERNEL32.dll
 0001:0006434e       _LoadLibraryExA@12         1006534e f   kernel32:KERNEL32.dll
 0001:00064354       _IsDebuggerPresent@0       10065354 f   kernel32:KERNEL32.dll
 0001:0006435a       _IsProcessorFeaturePresent@4 1006535a f   kernel32:KERNEL32.dll
 0001:00064360       _HeapFree@12               10065360 f   kernel32:KERNEL32.dll
 0001:00064366       _HeapAlloc@12              10065366 f   kernel32:KERNEL32.dll
 0001:0006436c       _EncodePointer@4           1006536c f   kernel32:KERNEL32.dll
 0001:00064372       _DecodePointer@4           10065372 f   kernel32:KERNEL32.dll
 0001:00064378       _RtlUnwind@16              10065378 f   kernel32:KERNEL32.dll
 0001:0006437e       _GetCommandLineA@0         1006537e f   kernel32:KERNEL32.dll
 0001:00064384       _GetCurrentThreadId@0      10065384 f   kernel32:KERNEL32.dll
 0001:0006438a       _UnhandledExceptionFilter@4 1006538a f   kernel32:KERNEL32.dll
 0001:00064390       _SetUnhandledExceptionFilter@4 10065390 f   kernel32:KERNEL32.dll
 0001:00064396       _SetLastError@4            10065396 f   kernel32:KERNEL32.dll
 0001:0006439c       _InitializeCriticalSectionAndSpinCount@8 1006539c f   kernel32:KERNEL32.dll
 0001:000643a2       _CreateEventW@16           100653a2 f   kernel32:KERNEL32.dll
 0001:000643a8       _TerminateProcess@8        100653a8 f   kernel32:KERNEL32.dll
 0001:000643ae       _TlsAlloc@0                100653ae f   kernel32:KERNEL32.dll
 0001:000643b4       _TlsGetValue@4             100653b4 f   kernel32:KERNEL32.dll
 0001:000643ba       _TlsSetValue@8             100653ba f   kernel32:KERNEL32.dll
 0001:000643c0       _TlsFree@4                 100653c0 f   kernel32:KERNEL32.dll
 0001:000643c6       _GetStartupInfoW@4         100653c6 f   kernel32:KERNEL32.dll
 0001:000643cc       _GetTickCount@0            100653cc f   kernel32:KERNEL32.dll
 0001:000643d2       _GetModuleHandleW@4        100653d2 f   kernel32:KERNEL32.dll
 0001:000643d8       _CreateSemaphoreW@16       100653d8 f   kernel32:KERNEL32.dll
 0001:000643de       _IsValidCodePage@4         100653de f   kernel32:KERNEL32.dll
 0001:000643e4       _GetACP@0                  100653e4 f   kernel32:KERNEL32.dll
 0001:000643ea       _GetOEMCP@0                100653ea f   kernel32:KERNEL32.dll
 0001:000643f0       _GetCPInfo@8               100653f0 f   kernel32:KERNEL32.dll
 0001:000643f6       _GetProcessHeap@0          100653f6 f   kernel32:KERNEL32.dll
 0001:000643fc       _ExitProcess@4             100653fc f   kernel32:KERNEL32.dll
 0001:00064402       _GetModuleHandleExW@12     10065402 f   kernel32:KERNEL32.dll
 0001:00064408       _AreFileApisANSI@0         10065408 f   kernel32:KERNEL32.dll
 0001:0006440e       _WideCharToMultiByte@32    1006540e f   kernel32:KERNEL32.dll
 0001:00064414       _GetStdHandle@4            10065414 f   kernel32:KERNEL32.dll
 0001:0006441a       _GetModuleFileNameW@12     1006541a f   kernel32:KERNEL32.dll
 0001:00064420       _EnterCriticalSection@4    10065420 f   kernel32:KERNEL32.dll
 0001:00064426       _LeaveCriticalSection@4    10065426 f   kernel32:KERNEL32.dll
 0001:0006442c       _HeapSize@12               1006542c f   kernel32:KERNEL32.dll
 0001:00064432       _DeleteCriticalSection@4   10065432 f   kernel32:KERNEL32.dll
 0001:00064438       _FatalAppExitA@8           10065438 f   kernel32:KERNEL32.dll
 0001:0006443e       _GetConsoleMode@8          1006543e f   kernel32:KERNEL32.dll
 0001:00064444       _ReadConsoleW@20           10065444 f   kernel32:KERNEL32.dll
 0001:0006444a       _SetFilePointerEx@20       1006544a f   kernel32:KERNEL32.dll
 0001:00064450       _GetFileType@4             10065450 f   kernel32:KERNEL32.dll
 0001:00064456       _GetConsoleCP@0            10065456 f   kernel32:KERNEL32.dll
 0001:0006445c       _GetModuleFileNameA@12     1006545c f   kernel32:KERNEL32.dll
 0001:00064462       _GetSystemTimeAsFileTime@4 10065462 f   kernel32:KERNEL32.dll
 0001:00064468       _GetEnvironmentStringsW@0  10065468 f   kernel32:KERNEL32.dll
 0001:0006446e       _FreeEnvironmentStringsW@4 1006546e f   kernel32:KERNEL32.dll
 0001:00064474       _GetStringTypeW@16         10065474 f   kernel32:KERNEL32.dll
 0001:0006447a       _GetLocaleInfoW@16         1006547a f   kernel32:KERNEL32.dll
 0001:00064480       _IsValidLocale@8           10065480 f   kernel32:KERNEL32.dll
 0001:00064486       _GetUserDefaultLCID@0      10065486 f   kernel32:KERNEL32.dll
 0001:0006448c       _EnumSystemLocalesW@8      1006548c f   kernel32:KERNEL32.dll
 0001:00064492       _GetDateFormatW@24         10065492 f   kernel32:KERNEL32.dll
 0001:00064498       _GetTimeFormatW@24         10065498 f   kernel32:KERNEL32.dll
 0001:0006449e       _CompareStringW@24         1006549e f   kernel32:KERNEL32.dll
 0001:000644a4       _LCMapStringW@24           100654a4 f   kernel32:KERNEL32.dll
 0001:000644aa       _SetConsoleCtrlHandler@8   100654aa f   kernel32:KERNEL32.dll
 0001:000644b0       _LoadLibraryExW@12         100654b0 f   kernel32:KERNEL32.dll
 0001:000644b6       _OutputDebugStringW@4      100654b6 f   kernel32:KERNEL32.dll
 0001:000644bc       _HeapReAlloc@16            100654bc f   kernel32:KERNEL32.dll
 0001:000644c2       _SetEnvironmentVariableA@8 100654c2 f   kernel32:KERNEL32.dll
 0001:000644c8       _SetStdHandle@8            100654c8 f   kernel32:KERNEL32.dll
 0001:000644ce       _FlushFileBuffers@4        100654ce f   kernel32:KERNEL32.dll
 0001:000644d4       _WriteConsoleW@20          100654d4 f   kernel32:KERNEL32.dll
 0001:000644da       _CreateFileW@28            100654da f   kernel32:KERNEL32.dll
 0001:000644e0       _SetEndOfFile@4            100654e0 f   kernel32:KERNEL32.dll
 0001:0006465b       _strupr                    1006565b f   LIBCMT:strupr.obj
 0001:0006465b       __strupr                   1006565b f   LIBCMT:strupr.obj
 0001:000646b6       __strupr_l                 100656b6 f   LIBCMT:strupr.obj
 0001:000646ce       __strupr_s                 100656ce f   LIBCMT:strupr.obj
 0001:000646e3       __strupr_s_l               100656e3 f   LIBCMT:strupr.obj
 0002:00000000       __imp__RegEnumValueA@32    10068000     advapi32:ADVAPI32.dll
 0002:00000004       __imp__RegDeleteValueA@8   10068004     advapi32:ADVAPI32.dll
 0002:00000008       __imp__RegCreateKeyA@12    10068008     advapi32:ADVAPI32.dll
 0002:0000000c       __imp__RegCloseKey@4       1006800c     advapi32:ADVAPI32.dll
 0002:00000010       __imp__RegQueryInfoKeyA@48 10068010     advapi32:ADVAPI32.dll
 0002:00000014       __imp__RegQueryValueExA@24 10068014     advapi32:ADVAPI32.dll
 0002:00000018       __imp__RegSetValueExA@24   10068018     advapi32:ADVAPI32.dll
 0002:0000001c       __imp__RegOpenKeyExA@20    1006801c     advapi32:ADVAPI32.dll
 0002:00000020       \177ADVAPI32_NULL_THUNK_DATA 10068020     advapi32:ADVAPI32.dll
 0002:00000024       __imp__HPI_InStreamWait@12 10068024     asihpi32:ASIHPI32.dll
 0002:00000028       __imp__HPI_FormatCreate@24 10068028     asihpi32:ASIHPI32.dll
 0002:0000002c       __imp__HPI_InStreamHostBufferFree@8 1006802c     asihpi32:ASIHPI32.dll
 0002:00000030       __imp__HPI_InStreamHostBufferAllocate@12 10068030     asihpi32:ASIHPI32.dll
 0002:00000034       __imp__HPI_InStreamGetInfoEx@28 10068034     asihpi32:ASIHPI32.dll
 0002:00000038       __imp__HPI_InStreamReset@8 10068038     asihpi32:ASIHPI32.dll
 0002:0000003c       __imp__HPI_InStreamStop@8  1006803c     asihpi32:ASIHPI32.dll
 0002:00000040       __imp__HPI_InStreamStart@8 10068040     asihpi32:ASIHPI32.dll
 0002:00000044       __imp__HPI_InStreamReadBuf@16 10068044     asihpi32:ASIHPI32.dll
 0002:00000048       __imp__HPI_InStreamSetFormat@12 10068048     asihpi32:ASIHPI32.dll
 0002:0000004c       __imp__HPI_InStreamQueryFormat@12 1006804c     asihpi32:ASIHPI32.dll
 0002:00000050       __imp__HPI_InStreamClose@8 10068050     asihpi32:ASIHPI32.dll
 0002:00000054       __imp__HPI_InStreamOpen@16 10068054     asihpi32:ASIHPI32.dll
 0002:00000058       __imp__HPI_OutStreamWait@12 10068058     asihpi32:ASIHPI32.dll
 0002:0000005c       __imp__HPI_WaveFormatToHpiFormat@8 1006805c     asihpi32:ASIHPI32.dll
 0002:00000060       __imp__HPI_OutStreamHostBufferFree@8 10068060     asihpi32:ASIHPI32.dll
 0002:00000064       __imp__HPI_OutStreamHostBufferAllocate@12 10068064     asihpi32:ASIHPI32.dll
 0002:00000068       __imp__HPI_OutStreamSetTimeScale@12 10068068     asihpi32:ASIHPI32.dll
 0002:0000006c       __imp__HPI_OutStreamQueryFormat@12 1006806c     asihpi32:ASIHPI32.dll
 0002:00000070       __imp__HPI_OutStreamReset@8 10068070     asihpi32:ASIHPI32.dll
 0002:00000074       __imp__HPI_OutStreamStop@8 10068074     asihpi32:ASIHPI32.dll
 0002:00000078       __imp__HPI_OutStreamStart@8 10068078     asihpi32:ASIHPI32.dll
 0002:0000007c       __imp__HPI_OutStreamWriteBuf@20 1006807c     asihpi32:ASIHPI32.dll
 0002:00000080       __imp__HPI_OutStreamGetInfoEx@28 10068080     asihpi32:ASIHPI32.dll
 0002:00000084       __imp__HPI_OutStreamClose@8 10068084     asihpi32:ASIHPI32.dll
 0002:00000088       __imp__HPI_OutStreamOpen@16 10068088     asihpi32:ASIHPI32.dll
 0002:0000008c       __imp__HPI_InitMessageResponse@16 1006808c     asihpi32:ASIHPI32.dll
 0002:00000090       __imp__HPI_ControlParamGet@28 10068090     asihpi32:ASIHPI32.dll
 0002:00000094       __imp__HPI_Message@8       10068094     asihpi32:ASIHPI32.dll
 0002:00000098       __imp__HPI_HandleToIndexes@12 10068098     asihpi32:ASIHPI32.dll
 0002:0000009c       __imp__HPI_SubSysCreate@0  1006809c     asihpi32:ASIHPI32.dll
 0002:000000a0       __imp__HPI_SubSysGetVersionEx@8 100680a0     asihpi32:ASIHPI32.dll
 0002:000000a4       __imp__HPI_Entity_FindNext@20 100680a4     asihpi32:ASIHPI32.dll
 0002:000000a8       __imp__HPI_Entity_CopyValueFrom@20 100680a8     asihpi32:ASIHPI32.dll
 0002:000000ac       __imp__HPI_Entity_Unpack@20 100680ac     asihpi32:ASIHPI32.dll
 0002:000000b0       __imp__HPI_Entity_AllocAndPack@24 100680b0     asihpi32:ASIHPI32.dll
 0002:000000b4       __imp__HPI_Entity_Free@4   100680b4     asihpi32:ASIHPI32.dll
 0002:000000b8       __imp__HPI_Object_GetInfo@24 100680b8     asihpi32:ASIHPI32.dll
 0002:000000bc       __imp__HPI_Object_BlockHandle@28 100680bc     asihpi32:ASIHPI32.dll
 0002:000000c0       __imp__HPI_Object_ParameterHandle@16 100680c0     asihpi32:ASIHPI32.dll
 0002:000000c4       __imp__HPI_SubSysFree@4    100680c4     asihpi32:ASIHPI32.dll
 0002:000000c8       __imp__HPI_SubSysGetNumAdapters@8 100680c8     asihpi32:ASIHPI32.dll
 0002:000000cc       __imp__HPI_SubSysGetAdapter@16 100680cc     asihpi32:ASIHPI32.dll
 0002:000000d0       __imp__HPI_SubSysSetHostNetworkInterface@8 100680d0     asihpi32:ASIHPI32.dll
 0002:000000d4       __imp__HPI_AdapterOpen@8   100680d4     asihpi32:ASIHPI32.dll
 0002:000000d8       __imp__HPI_AdapterClose@8  100680d8     asihpi32:ASIHPI32.dll
 0002:000000dc       __imp__HPI_AdapterGetInfo@28 100680dc     asihpi32:ASIHPI32.dll
 0002:000000e0       __imp__HPI_AdapterGetModuleByIndex@36 100680e0     asihpi32:ASIHPI32.dll
 0002:000000e4       __imp__HPI_AdapterSetMode@12 100680e4     asihpi32:ASIHPI32.dll
 0002:000000e8       __imp__HPI_AdapterSetModeEx@16 100680e8     asihpi32:ASIHPI32.dll
 0002:000000ec       __imp__HPI_AdapterGetMode@12 100680ec     asihpi32:ASIHPI32.dll
 0002:000000f0       __imp__HPI_AdapterSetProperty@20 100680f0     asihpi32:ASIHPI32.dll
 0002:000000f4       __imp__HPI_AdapterGetProperty@20 100680f4     asihpi32:ASIHPI32.dll
 0002:000000f8       __imp__HPI_NvMemoryOpen@16 100680f8     asihpi32:ASIHPI32.dll
 0002:000000fc       __imp__HPI_NvMemoryReadByte@16 100680fc     asihpi32:ASIHPI32.dll
 0002:00000100       __imp__HPI_NvMemoryWriteByte@16 10068100     asihpi32:ASIHPI32.dll
 0002:00000104       __imp__HPI_GpioOpen@20     10068104     asihpi32:ASIHPI32.dll
 0002:00000108       __imp__HPI_GpioReadAllBits@12 10068108     asihpi32:ASIHPI32.dll
 0002:0000010c       __imp__HPI_GpioWriteBit@16 1006810c     asihpi32:ASIHPI32.dll
 0002:00000110       __imp__HPI_GpioWriteStatus@12 10068110     asihpi32:ASIHPI32.dll
 0002:00000114       __imp__HPI_MixerOpen@12    10068114     asihpi32:ASIHPI32.dll
 0002:00000118       __imp__HPI_MixerClose@8    10068118     asihpi32:ASIHPI32.dll
 0002:0000011c       __imp__HPI_MixerGetControlByIndex@36 1006811c     asihpi32:ASIHPI32.dll
 0002:00000120       __imp__HPI_MixerStore@16   10068120     asihpi32:ASIHPI32.dll
 0002:00000124       __imp__HPI_VolumeSetGain@12 10068124     asihpi32:ASIHPI32.dll
 0002:00000128       __imp__HPI_VolumeGetGain@12 10068128     asihpi32:ASIHPI32.dll
 0002:0000012c       __imp__HPI_VolumeSetMute@12 1006812c     asihpi32:ASIHPI32.dll
 0002:00000130       __imp__HPI_VolumeGetMute@12 10068130     asihpi32:ASIHPI32.dll
 0002:00000134       __imp__HPI_VolumeQueryRange@20 10068134     asihpi32:ASIHPI32.dll
 0002:00000138       __imp__HPI_Volume_QueryChannels@12 10068138     asihpi32:ASIHPI32.dll
 0002:0000013c       __imp__HPI_VolumeAutoFadeProfile@20 1006813c     asihpi32:ASIHPI32.dll
 0002:00000140       __imp__HPI_LevelQueryRange@20 10068140     asihpi32:ASIHPI32.dll
 0002:00000144       __imp__HPI_LevelSetGain@12 10068144     asihpi32:ASIHPI32.dll
 0002:00000148       __imp__HPI_LevelGetGain@12 10068148     asihpi32:ASIHPI32.dll
 0002:0000014c       __imp__HPI_Meter_QueryChannels@12 1006814c     asihpi32:ASIHPI32.dll
 0002:00000150       __imp__HPI_MeterGetPeak@12 10068150     asihpi32:ASIHPI32.dll
 0002:00000154       __imp__HPI_MeterGetRms@12  10068154     asihpi32:ASIHPI32.dll
 0002:00000158       __imp__HPI_MeterSetPeakBallistics@16 10068158     asihpi32:ASIHPI32.dll
 0002:0000015c       __imp__HPI_MeterSetRmsBallistics@16 1006815c     asihpi32:ASIHPI32.dll
 0002:00000160       __imp__HPI_MeterGetPeakBallistics@16 10068160     asihpi32:ASIHPI32.dll
 0002:00000164       __imp__HPI_MeterGetRmsBallistics@16 10068164     asihpi32:ASIHPI32.dll
 0002:00000168       __imp__HPI_ChannelMode_QueryMode@16 10068168     asihpi32:ASIHPI32.dll
 0002:0000016c       __imp__HPI_ChannelModeSet@12 1006816c     asihpi32:ASIHPI32.dll
 0002:00000170       __imp__HPI_ChannelModeGet@12 10068170     asihpi32:ASIHPI32.dll
 0002:00000174       __imp__HPI_Tuner_QueryBand@16 10068174     asihpi32:ASIHPI32.dll
 0002:00000178       __imp__HPI_Tuner_SetBand@12 10068178     asihpi32:ASIHPI32.dll
 0002:0000017c       __imp__HPI_Tuner_GetBand@12 1006817c     asihpi32:ASIHPI32.dll
 0002:00000180       __imp__HPI_Tuner_QueryFrequency@20 10068180     asihpi32:ASIHPI32.dll
 0002:00000184       __imp__HPI_Tuner_SetFrequency@12 10068184     asihpi32:ASIHPI32.dll
 0002:00000188       __imp__HPI_Tuner_GetFrequency@12 10068188     asihpi32:ASIHPI32.dll
 0002:0000018c       __imp__HPI_Tuner_SetGain@12 1006818c     asihpi32:ASIHPI32.dll
 0002:00000190       __imp__HPI_Tuner_GetGain@12 10068190     asihpi32:ASIHPI32.dll
 0002:00000194       __imp__HPI_Tuner_GetRFLevel@12 10068194     asihpi32:ASIHPI32.dll
 0002:00000198       __imp__HPI_Tuner_GetRawRFLevel@12 10068198     asihpi32:ASIHPI32.dll
 0002:0000019c       __imp__HPI_Tuner_GetStatus@16 1006819c     asihpi32:ASIHPI32.dll
 0002:000001a0       __imp__HPI_Tuner_SetMode@16 100681a0     asihpi32:ASIHPI32.dll
 0002:000001a4       __imp__HPI_Tuner_GetMode@16 100681a4     asihpi32:ASIHPI32.dll
 0002:000001a8       __imp__HPI_Tuner_QueryDeemphasis@20 100681a8     asihpi32:ASIHPI32.dll
 0002:000001ac       __imp__HPI_Tuner_SetDeemphasis@12 100681ac     asihpi32:ASIHPI32.dll
 0002:000001b0       __imp__HPI_Tuner_GetDeemphasis@12 100681b0     asihpi32:ASIHPI32.dll
 0002:000001b4       __imp__HPI_Tuner_QueryProgram@12 100681b4     asihpi32:ASIHPI32.dll
 0002:000001b8       __imp__HPI_Tuner_SetProgram@12 100681b8     asihpi32:ASIHPI32.dll
 0002:000001bc       __imp__HPI_Tuner_GetProgram@12 100681bc     asihpi32:ASIHPI32.dll
 0002:000001c0       __imp__HPI_Tuner_GetFirmwareVersion@16 100681c0     asihpi32:ASIHPI32.dll
 0002:000001c4       __imp__HPI_Tuner_GetHdRadioSignalQuality@12 100681c4     asihpi32:ASIHPI32.dll
 0002:000001c8       __imp__HPI_Tuner_GetHdRadioSignalBlend@12 100681c8     asihpi32:ASIHPI32.dll
 0002:000001cc       __imp__HPI_Tuner_SetHdRadioSignalBlend@12 100681cc     asihpi32:ASIHPI32.dll
 0002:000001d0       __imp__HPI_Tuner_GetDabAudioServiceCount@16 100681d0     asihpi32:ASIHPI32.dll
 0002:000001d4       __imp__HPI_Tuner_SetDabAudioService@12 100681d4     asihpi32:ASIHPI32.dll
 0002:000001d8       __imp__HPI_Tuner_GetDabAudioServiceName@20 100681d8     asihpi32:ASIHPI32.dll
 0002:000001dc       __imp__HPI_Tuner_GetDabMultiplexName@16 100681dc     asihpi32:ASIHPI32.dll
 0002:000001e0       __imp__HPI_Tuner_GetDabAudioInfo@16 100681e0     asihpi32:ASIHPI32.dll
 0002:000001e4       __imp__HPI_PAD_GetChannelName@16 100681e4     asihpi32:ASIHPI32.dll
 0002:000001e8       __imp__HPI_PAD_GetArtist@16 100681e8     asihpi32:ASIHPI32.dll
 0002:000001ec       __imp__HPI_PAD_GetTitle@16 100681ec     asihpi32:ASIHPI32.dll
 0002:000001f0       __imp__HPI_PAD_GetComment@16 100681f0     asihpi32:ASIHPI32.dll
 0002:000001f4       __imp__HPI_PAD_GetProgramType@12 100681f4     asihpi32:ASIHPI32.dll
 0002:000001f8       __imp__HPI_PAD_GetRdsPI@12 100681f8     asihpi32:ASIHPI32.dll
 0002:000001fc       __imp__HPI_PAD_GetProgramTypeString@24 100681fc     asihpi32:ASIHPI32.dll
 0002:00000200       __imp__HPI_AESEBU_Receiver_QueryFormat@16 10068200     asihpi32:ASIHPI32.dll
 0002:00000204       __imp__HPI_AESEBU_Receiver_SetFormat@12 10068204     asihpi32:ASIHPI32.dll
 0002:00000208       __imp__HPI_AESEBU_Receiver_GetFormat@12 10068208     asihpi32:ASIHPI32.dll
 0002:0000020c       __imp__HPI_AESEBU_Receiver_GetSampleRate@12 1006820c     asihpi32:ASIHPI32.dll
 0002:00000210       __imp__HPI_AESEBU_Receiver_GetErrorStatus@12 10068210     asihpi32:ASIHPI32.dll
 0002:00000214       __imp__HPI_AESEBU_Transmitter_SetChannelStatus@16 10068214     asihpi32:ASIHPI32.dll
 0002:00000218       __imp__HPI_AESEBU_Transmitter_QueryFormat@16 10068218     asihpi32:ASIHPI32.dll
 0002:0000021c       __imp__HPI_AESEBU_Transmitter_SetFormat@12 1006821c     asihpi32:ASIHPI32.dll
 0002:00000220       __imp__HPI_AESEBU_Transmitter_GetFormat@12 10068220     asihpi32:ASIHPI32.dll
 0002:00000224       __imp__HPI_Multiplexer_SetSource@16 10068224     asihpi32:ASIHPI32.dll
 0002:00000228       __imp__HPI_Multiplexer_GetSource@16 10068228     asihpi32:ASIHPI32.dll
 0002:0000022c       __imp__HPI_Multiplexer_QuerySource@20 1006822c     asihpi32:ASIHPI32.dll
 0002:00000230       __imp__HPI_VoxSetThreshold@12 10068230     asihpi32:ASIHPI32.dll
 0002:00000234       __imp__HPI_VoxGetThreshold@12 10068234     asihpi32:ASIHPI32.dll
 0002:00000238       __imp__HPI_SampleClock_QuerySource@16 10068238     asihpi32:ASIHPI32.dll
 0002:0000023c       __imp__HPI_SampleClock_SetSource@12 1006823c     asihpi32:ASIHPI32.dll
 0002:00000240       __imp__HPI_SampleClock_GetSource@12 10068240     asihpi32:ASIHPI32.dll
 0002:00000244       __imp__HPI_SampleClock_QuerySourceIndex@20 10068244     asihpi32:ASIHPI32.dll
 0002:00000248       __imp__HPI_SampleClock_SetSourceIndex@12 10068248     asihpi32:ASIHPI32.dll
 0002:0000024c       __imp__HPI_SampleClock_GetSourceIndex@12 1006824c     asihpi32:ASIHPI32.dll
 0002:00000250       __imp__HPI_SampleClock_GetSampleRate@12 10068250     asihpi32:ASIHPI32.dll
 0002:00000254       __imp__HPI_SampleClock_QueryLocalRate@16 10068254     asihpi32:ASIHPI32.dll
 0002:00000258       __imp__HPI_SampleClock_SetLocalRate@12 10068258     asihpi32:ASIHPI32.dll
 0002:0000025c       __imp__HPI_SampleClock_GetLocalRate@12 1006825c     asihpi32:ASIHPI32.dll
 0002:00000260       __imp__HPI_SampleClock_SetAuto@12 10068260     asihpi32:ASIHPI32.dll
 0002:00000264       __imp__HPI_SampleClock_GetAuto@12 10068264     asihpi32:ASIHPI32.dll
 0002:00000268       __imp__HPI_SampleClock_SetLocalRateLock@12 10068268     asihpi32:ASIHPI32.dll
 0002:0000026c       __imp__HPI_SampleClock_GetLocalRateLock@12 1006826c     asihpi32:ASIHPI32.dll
 0002:00000270       __imp__HPI_Microphone_SetPhantomPower@12 10068270     asihpi32:ASIHPI32.dll
 0002:00000274       __imp__HPI_Microphone_GetPhantomPower@12 10068274     asihpi32:ASIHPI32.dll
 0002:00000278       __imp__HPI_ParametricEQ_GetInfo@16 10068278     asihpi32:ASIHPI32.dll
 0002:0000027c       __imp__HPI_ParametricEQ_SetState@12 1006827c     asihpi32:ASIHPI32.dll
 0002:00000280       __imp__HPI_ParametricEQ_SetBand@28 10068280     asihpi32:ASIHPI32.dll
 0002:00000284       __imp__HPI_ParametricEQ_GetBand@28 10068284     asihpi32:ASIHPI32.dll
 0002:00000288       __imp__HPI_Compander_SetEnable@12 10068288     asihpi32:ASIHPI32.dll
 0002:0000028c       __imp__HPI_Compander_GetEnable@12 1006828c     asihpi32:ASIHPI32.dll
 0002:00000290       __imp__HPI_Compander_SetMakeupGain@12 10068290     asihpi32:ASIHPI32.dll
 0002:00000294       __imp__HPI_Compander_GetMakeupGain@12 10068294     asihpi32:ASIHPI32.dll
 0002:00000298       __imp__HPI_Compander_SetAttackTimeConstant@16 10068298     asihpi32:ASIHPI32.dll
 0002:0000029c       __imp__HPI_Compander_GetAttackTimeConstant@16 1006829c     asihpi32:ASIHPI32.dll
 0002:000002a0       __imp__HPI_Compander_SetDecayTimeConstant@16 100682a0     asihpi32:ASIHPI32.dll
 0002:000002a4       __imp__HPI_Compander_GetDecayTimeConstant@16 100682a4     asihpi32:ASIHPI32.dll
 0002:000002a8       __imp__HPI_Compander_SetThreshold@16 100682a8     asihpi32:ASIHPI32.dll
 0002:000002ac       __imp__HPI_Compander_GetThreshold@16 100682ac     asihpi32:ASIHPI32.dll
 0002:000002b0       __imp__HPI_Compander_SetRatio@16 100682b0     asihpi32:ASIHPI32.dll
 0002:000002b4       __imp__HPI_Compander_GetRatio@16 100682b4     asihpi32:ASIHPI32.dll
 0002:000002b8       __imp__HPI_Cobranet_HmiWrite@20 100682b8     asihpi32:ASIHPI32.dll
 0002:000002bc       __imp__HPI_Cobranet_HmiRead@24 100682bc     asihpi32:ASIHPI32.dll
 0002:000002c0       __imp__HPI_Cobranet_GetIPaddress@12 100682c0     asihpi32:ASIHPI32.dll
 0002:000002c4       __imp__HPI_Cobranet_GetMACaddress@16 100682c4     asihpi32:ASIHPI32.dll
 0002:000002c8       __imp__HPI_ToneDetector_GetState@12 100682c8     asihpi32:ASIHPI32.dll
 0002:000002cc       __imp__HPI_ToneDetector_SetEnable@12 100682cc     asihpi32:ASIHPI32.dll
 0002:000002d0       __imp__HPI_ToneDetector_GetEnable@12 100682d0     asihpi32:ASIHPI32.dll
 0002:000002d4       __imp__HPI_ToneDetector_SetEventEnable@12 100682d4     asihpi32:ASIHPI32.dll
 0002:000002d8       __imp__HPI_ToneDetector_GetEventEnable@12 100682d8     asihpi32:ASIHPI32.dll
 0002:000002dc       __imp__HPI_ToneDetector_SetThreshold@12 100682dc     asihpi32:ASIHPI32.dll
 0002:000002e0       __imp__HPI_ToneDetector_GetThreshold@12 100682e0     asihpi32:ASIHPI32.dll
 0002:000002e4       __imp__HPI_ToneDetector_GetFrequency@16 100682e4     asihpi32:ASIHPI32.dll
 0002:000002e8       __imp__HPI_SilenceDetector_GetState@12 100682e8     asihpi32:ASIHPI32.dll
 0002:000002ec       __imp__HPI_SilenceDetector_SetEnable@12 100682ec     asihpi32:ASIHPI32.dll
 0002:000002f0       __imp__HPI_SilenceDetector_GetEnable@12 100682f0     asihpi32:ASIHPI32.dll
 0002:000002f4       __imp__HPI_SilenceDetector_SetEventEnable@12 100682f4     asihpi32:ASIHPI32.dll
 0002:000002f8       __imp__HPI_SilenceDetector_GetEventEnable@12 100682f8     asihpi32:ASIHPI32.dll
 0002:000002fc       __imp__HPI_SilenceDetector_SetDelay@12 100682fc     asihpi32:ASIHPI32.dll
 0002:00000300       __imp__HPI_GetErrorText@8  10068300     asihpi32:ASIHPI32.dll
 0002:00000304       __imp__HPI_SilenceDetector_SetThreshold@12 10068304     asihpi32:ASIHPI32.dll
 0002:00000308       __imp__HPI_SilenceDetector_GetThreshold@12 10068308     asihpi32:ASIHPI32.dll
 0002:0000030c       __imp__HPI_Universal_Info@12 1006830c     asihpi32:ASIHPI32.dll
 0002:00000310       __imp__HPI_Universal_Get@12 10068310     asihpi32:ASIHPI32.dll
 0002:00000314       __imp__HPI_Universal_Set@12 10068314     asihpi32:ASIHPI32.dll
 0002:00000318       __imp__HPI_ProfileOpenAll@20 10068318     asihpi32:ASIHPI32.dll
 0002:0000031c       __imp__HPI_ProfileGetUtilization@12 1006831c     asihpi32:ASIHPI32.dll
 0002:00000320       __imp__HPI_SilenceDetector_GetDelay@12 10068320     asihpi32:ASIHPI32.dll
 0002:00000324       \177ASIHPI32_NULL_THUNK_DATA 10068324     asihpi32:ASIHPI32.dll
 0002:00000328       __imp__DirectSoundCaptureCreate@12 10068328     dsound:DSOUND.dll
 0002:0000032c       __imp__DirectSoundCreate@12 1006832c     dsound:DSOUND.dll
 0002:00000330       __imp__DirectSoundCaptureEnumerateA@8 10068330     dsound:DSOUND.dll
 0002:00000334       __imp__DirectSoundEnumerateA@8 10068334     dsound:DSOUND.dll
 0002:00000338       \177DSOUND_NULL_THUNK_DATA 10068338     dsound:DSOUND.dll
 0002:0000033c       __imp__GetStdHandle@4      1006833c     kernel32:KERNEL32.dll
 0002:00000340       __imp__GetModuleFileNameW@12 10068340     kernel32:KERNEL32.dll
 0002:00000344       __imp__EnterCriticalSection@4 10068344     kernel32:KERNEL32.dll
 0002:00000348       __imp__LeaveCriticalSection@4 10068348     kernel32:KERNEL32.dll
 0002:0000034c       __imp__HeapSize@12         1006834c     kernel32:KERNEL32.dll
 0002:00000350       __imp__DeleteCriticalSection@4 10068350     kernel32:KERNEL32.dll
 0002:00000354       __imp__FatalAppExitA@8     10068354     kernel32:KERNEL32.dll
 0002:00000358       __imp__GetConsoleMode@8    10068358     kernel32:KERNEL32.dll
 0002:0000035c       __imp__ReadConsoleW@20     1006835c     kernel32:KERNEL32.dll
 0002:00000360       __imp__SetFilePointerEx@20 10068360     kernel32:KERNEL32.dll
 0002:00000364       __imp__GetFileType@4       10068364     kernel32:KERNEL32.dll
 0002:00000368       __imp__GetConsoleCP@0      10068368     kernel32:KERNEL32.dll
 0002:0000036c       __imp__GetModuleFileNameA@12 1006836c     kernel32:KERNEL32.dll
 0002:00000370       __imp__GetSystemTimeAsFileTime@4 10068370     kernel32:KERNEL32.dll
 0002:00000374       __imp__GetEnvironmentStringsW@0 10068374     kernel32:KERNEL32.dll
 0002:00000378       __imp__FreeEnvironmentStringsW@4 10068378     kernel32:KERNEL32.dll
 0002:0000037c       __imp__GetStringTypeW@16   1006837c     kernel32:KERNEL32.dll
 0002:00000380       __imp__GetLocaleInfoW@16   10068380     kernel32:KERNEL32.dll
 0002:00000384       __imp__IsValidLocale@8     10068384     kernel32:KERNEL32.dll
 0002:00000388       __imp__GetUserDefaultLCID@0 10068388     kernel32:KERNEL32.dll
 0002:0000038c       __imp__EnumSystemLocalesW@8 1006838c     kernel32:KERNEL32.dll
 0002:00000390       __imp__GetDateFormatW@24   10068390     kernel32:KERNEL32.dll
 0002:00000394       __imp__GetTimeFormatW@24   10068394     kernel32:KERNEL32.dll
 0002:00000398       __imp__CompareStringW@24   10068398     kernel32:KERNEL32.dll
 0002:0000039c       __imp__LCMapStringW@24     1006839c     kernel32:KERNEL32.dll
 0002:000003a0       __imp__SetConsoleCtrlHandler@8 100683a0     kernel32:KERNEL32.dll
 0002:000003a4       __imp__GetCPInfo@8         100683a4     kernel32:KERNEL32.dll
 0002:000003a8       __imp__GetOEMCP@0          100683a8     kernel32:KERNEL32.dll
 0002:000003ac       __imp__WideCharToMultiByte@32 100683ac     kernel32:KERNEL32.dll
 0002:000003b0       __imp__IsValidCodePage@4   100683b0     kernel32:KERNEL32.dll
 0002:000003b4       __imp__CreateSemaphoreW@16 100683b4     kernel32:KERNEL32.dll
 0002:000003b8       __imp__GetModuleHandleW@4  100683b8     kernel32:KERNEL32.dll
 0002:000003bc       __imp__GetTickCount@0      100683bc     kernel32:KERNEL32.dll
 0002:000003c0       __imp__GetStartupInfoW@4   100683c0     kernel32:KERNEL32.dll
 0002:000003c4       __imp__TlsFree@4           100683c4     kernel32:KERNEL32.dll
 0002:000003c8       __imp__TlsSetValue@8       100683c8     kernel32:KERNEL32.dll
 0002:000003cc       __imp__TlsGetValue@4       100683cc     kernel32:KERNEL32.dll
 0002:000003d0       __imp__TlsAlloc@0          100683d0     kernel32:KERNEL32.dll
 0002:000003d4       __imp__TerminateProcess@8  100683d4     kernel32:KERNEL32.dll
 0002:000003d8       __imp__CreateEventW@16     100683d8     kernel32:KERNEL32.dll
 0002:000003dc       __imp__InitializeCriticalSectionAndSpinCount@8 100683dc     kernel32:KERNEL32.dll
 0002:000003e0       __imp__SetLastError@4      100683e0     kernel32:KERNEL32.dll
 0002:000003e4       __imp__SetUnhandledExceptionFilter@4 100683e4     kernel32:KERNEL32.dll
 0002:000003e8       __imp__UnhandledExceptionFilter@4 100683e8     kernel32:KERNEL32.dll
 0002:000003ec       __imp__GetCurrentThreadId@0 100683ec     kernel32:KERNEL32.dll
 0002:000003f0       __imp__GetCommandLineA@0   100683f0     kernel32:KERNEL32.dll
 0002:000003f4       __imp__RtlUnwind@16        100683f4     kernel32:KERNEL32.dll
 0002:000003f8       __imp__DecodePointer@4     100683f8     kernel32:KERNEL32.dll
 0002:000003fc       __imp__EncodePointer@4     100683fc     kernel32:KERNEL32.dll
 0002:00000400       __imp__HeapAlloc@12        10068400     kernel32:KERNEL32.dll
 0002:00000404       __imp__HeapFree@12         10068404     kernel32:KERNEL32.dll
 0002:00000408       __imp__IsProcessorFeaturePresent@4 10068408     kernel32:KERNEL32.dll
 0002:0000040c       __imp__IsDebuggerPresent@0 1006840c     kernel32:KERNEL32.dll
 0002:00000410       __imp__LoadLibraryExA@12   10068410     kernel32:KERNEL32.dll
 0002:00000414       __imp__FreeLibrary@4       10068414     kernel32:KERNEL32.dll
 0002:00000418       __imp__RaiseException@16   10068418     kernel32:KERNEL32.dll
 0002:0000041c       __imp__LoadLibraryExW@12   1006841c     kernel32:KERNEL32.dll
 0002:00000420       __imp__AreFileApisANSI@0   10068420     kernel32:KERNEL32.dll
 0002:00000424       __imp__GetModuleHandleExW@12 10068424     kernel32:KERNEL32.dll
 0002:00000428       __imp__ExitProcess@4       10068428     kernel32:KERNEL32.dll
 0002:0000042c       __imp__GetProcessHeap@0    1006842c     kernel32:KERNEL32.dll
 0002:00000430       __imp__GetACP@0            10068430     kernel32:KERNEL32.dll
 0002:00000434       __imp__GetProcAddress@8    10068434     kernel32:KERNEL32.dll
 0002:00000438       __imp__LoadLibraryA@4      10068438     kernel32:KERNEL32.dll
 0002:0000043c       __imp__CloseHandle@4       1006843c     kernel32:KERNEL32.dll
 0002:00000440       __imp__QueryPerformanceCounter@4 10068440     kernel32:KERNEL32.dll
 0002:00000444       __imp__QueryPerformanceFrequency@4 10068444     kernel32:KERNEL32.dll
 0002:00000448       __imp__ReleaseSemaphore@12 10068448     kernel32:KERNEL32.dll
 0002:0000044c       __imp__ReleaseMutex@4      1006844c     kernel32:KERNEL32.dll
 0002:00000450       __imp__WaitForSingleObject@8 10068450     kernel32:KERNEL32.dll
 0002:00000454       __imp__CreateMutexA@12     10068454     kernel32:KERNEL32.dll
 0002:00000458       __imp__Sleep@4             10068458     kernel32:KERNEL32.dll
 0002:0000045c       __imp__GetCurrentProcess@0 1006845c     kernel32:KERNEL32.dll
 0002:00000460       __imp__CreateThread@24     10068460     kernel32:KERNEL32.dll
 0002:00000464       __imp__SetPriorityClass@8  10068464     kernel32:KERNEL32.dll
 0002:00000468       __imp__GetPriorityClass@4  10068468     kernel32:KERNEL32.dll
 0002:0000046c       __imp__CreateSemaphoreA@16 1006846c     kernel32:KERNEL32.dll
 0002:00000470       __imp__SetEvent@4          10068470     kernel32:KERNEL32.dll
 0002:00000474       __imp__CreateEventA@16     10068474     kernel32:KERNEL32.dll
 0002:00000478       __imp__MultiByteToWideChar@24 10068478     kernel32:KERNEL32.dll
 0002:0000047c       __imp__OutputDebugStringA@4 1006847c     kernel32:KERNEL32.dll
 0002:00000480       __imp__GetCurrentProcessId@0 10068480     kernel32:KERNEL32.dll
 0002:00000484       __imp__GetCurrentThread@0  10068484     kernel32:KERNEL32.dll
 0002:00000488       __imp__SetThreadPriority@8 10068488     kernel32:KERNEL32.dll
 0002:0000048c       __imp__GetLastError@0      1006848c     kernel32:KERNEL32.dll
 0002:00000490       __imp__LocalFree@4         10068490     kernel32:KERNEL32.dll
 0002:00000494       __imp__FormatMessageA@28   10068494     kernel32:KERNEL32.dll
 0002:00000498       __imp__LocalAlloc@8        10068498     kernel32:KERNEL32.dll
 0002:0000049c       __imp__CreateFileA@28      1006849c     kernel32:KERNEL32.dll
 0002:000004a0       __imp__ReadFile@20         100684a0     kernel32:KERNEL32.dll
 0002:000004a4       __imp__SetFilePointer@16   100684a4     kernel32:KERNEL32.dll
 0002:000004a8       __imp__WriteFile@20        100684a8     kernel32:KERNEL32.dll
 0002:000004ac       __imp__OutputDebugStringW@4 100684ac     kernel32:KERNEL32.dll
 0002:000004b0       __imp__HeapReAlloc@16      100684b0     kernel32:KERNEL32.dll
 0002:000004b4       __imp__SetEnvironmentVariableA@8 100684b4     kernel32:KERNEL32.dll
 0002:000004b8       __imp__SetStdHandle@8      100684b8     kernel32:KERNEL32.dll
 0002:000004bc       __imp__FlushFileBuffers@4  100684bc     kernel32:KERNEL32.dll
 0002:000004c0       __imp__WriteConsoleW@20    100684c0     kernel32:KERNEL32.dll
 0002:000004c4       __imp__CreateFileW@28      100684c4     kernel32:KERNEL32.dll
 0002:000004c8       __imp__SetEndOfFile@4      100684c8     kernel32:KERNEL32.dll
 0002:000004cc       \177KERNEL32_NULL_THUNK_DATA 100684cc     kernel32:KERNEL32.dll
 0002:000004d0       __imp__GetWindowThreadProcessId@8 100684d0     user32:USER32.dll
 0002:000004d4       __imp__EnumChildWindows@12 100684d4     user32:USER32.dll
 0002:000004d8       __imp__GetDesktopWindow@0  100684d8     user32:USER32.dll
 0002:000004dc       \177USER32_NULL_THUNK_DATA 100684dc     user32:USER32.dll
 0002:000004e0       __imp__waveInGetNumDevs@0  100684e0     winmm:WINMM.dll
 0002:000004e4       __imp__mixerGetNumDevs@0   100684e4     winmm:WINMM.dll
 0002:000004e8       __imp__mixerGetDevCapsA@12 100684e8     winmm:WINMM.dll
 0002:000004ec       __imp__mixerOpen@20        100684ec     winmm:WINMM.dll
 0002:000004f0       __imp__mixerClose@4        100684f0     winmm:WINMM.dll
 0002:000004f4       __imp__mixerGetLineInfoA@12 100684f4     winmm:WINMM.dll
 0002:000004f8       __imp__mixerGetID@12       100684f8     winmm:WINMM.dll
 0002:000004fc       __imp__mixerGetLineControlsA@12 100684fc     winmm:WINMM.dll
 0002:00000500       __imp__mixerGetControlDetailsA@12 10068500     winmm:WINMM.dll
 0002:00000504       __imp__mixerSetControlDetails@12 10068504     winmm:WINMM.dll
 0002:00000508       __imp__waveOutOpen@24      10068508     winmm:WINMM.dll
 0002:0000050c       __imp__waveOutClose@4      1006850c     winmm:WINMM.dll
 0002:00000510       __imp__waveOutPrepareHeader@12 10068510     winmm:WINMM.dll
 0002:00000514       __imp__waveOutUnprepareHeader@12 10068514     winmm:WINMM.dll
 0002:00000518       __imp__waveOutWrite@12     10068518     winmm:WINMM.dll
 0002:0000051c       __imp__waveOutPause@4      1006851c     winmm:WINMM.dll
 0002:00000520       __imp__waveOutRestart@4    10068520     winmm:WINMM.dll
 0002:00000524       __imp__waveOutReset@4      10068524     winmm:WINMM.dll
 0002:00000528       __imp__waveOutGetPosition@12 10068528     winmm:WINMM.dll
 0002:0000052c       __imp__waveInOpen@24       1006852c     winmm:WINMM.dll
 0002:00000530       __imp__waveInClose@4       10068530     winmm:WINMM.dll
 0002:00000534       __imp__waveInPrepareHeader@12 10068534     winmm:WINMM.dll
 0002:00000538       __imp__waveInUnprepareHeader@12 10068538     winmm:WINMM.dll
 0002:0000053c       __imp__waveInAddBuffer@12  1006853c     winmm:WINMM.dll
 0002:00000540       __imp__waveInStart@4       10068540     winmm:WINMM.dll
 0002:00000544       __imp__waveInStop@4        10068544     winmm:WINMM.dll
 0002:00000548       __imp__waveInReset@4       10068548     winmm:WINMM.dll
 0002:0000054c       __imp__waveInGetPosition@12 1006854c     winmm:WINMM.dll
 0002:00000550       __imp__mmioStringToFOURCCA@8 10068550     winmm:WINMM.dll
 0002:00000554       __imp__mmioOpenA@12        10068554     winmm:WINMM.dll
 0002:00000558       __imp__mmioClose@8         10068558     winmm:WINMM.dll
 0002:0000055c       __imp__mmioRead@12         1006855c     winmm:WINMM.dll
 0002:00000560       __imp__mmioWrite@12        10068560     winmm:WINMM.dll
 0002:00000564       __imp__mmioSeek@12         10068564     winmm:WINMM.dll
 0002:00000568       __imp__mmioFlush@8         10068568     winmm:WINMM.dll
 0002:0000056c       __imp__mmioCreateChunk@12  1006856c     winmm:WINMM.dll
 0002:00000570       __imp__mmioAscend@12       10068570     winmm:WINMM.dll
 0002:00000574       __imp__mmioDescend@16      10068574     winmm:WINMM.dll
 0002:00000578       __imp__waveOutGetNumDevs@0 10068578     winmm:WINMM.dll
 0002:0000057c       \177WINMM_NULL_THUNK_DATA  1006857c     winmm:WINMM.dll
 0002:00000580       __imp__gethostbyname@4     10068580     wsock32:WSOCK32.dll
 0002:00000584       __imp__inet_ntoa@4         10068584     wsock32:WSOCK32.dll
 0002:00000588       \177WSOCK32_NULL_THUNK_DATA 10068588     wsock32:WSOCK32.dll
 0002:0000058c       __imp__CoCreateInstance@20 1006858c     ole32:ole32.dll
 0002:00000590       __imp__CoInitialize@4      10068590     ole32:ole32.dll
 0002:00000594       __imp__CLSIDFromString@8   10068594     ole32:ole32.dll
 0002:00000598       \177ole32_NULL_THUNK_DATA  10068598     ole32:ole32.dll
 0002:0000059c       __imp__SnmpSendMsg@20      1006859c     wsnmp32:wsnmp32.dll
 0002:000005a0       __imp__SnmpRecvMsg@20      100685a0     wsnmp32:wsnmp32.dll
 0002:000005a4       __imp__SnmpCreateSession@16 100685a4     wsnmp32:wsnmp32.dll
 0002:000005a8       __imp__SnmpCancelMsg@8     100685a8     wsnmp32:wsnmp32.dll
 0002:000005ac       __imp__SnmpStrToEntity@8   100685ac     wsnmp32:wsnmp32.dll
 0002:000005b0       __imp__SnmpFreeEntity@4    100685b0     wsnmp32:wsnmp32.dll
 0002:000005b4       __imp__SnmpStrToContext@8  100685b4     wsnmp32:wsnmp32.dll
 0002:000005b8       __imp__SnmpFreeContext@4   100685b8     wsnmp32:wsnmp32.dll
 0002:000005bc       __imp__SnmpCreatePdu@24    100685bc     wsnmp32:wsnmp32.dll
 0002:000005c0       __imp__SnmpGetRetry@12     100685c0     wsnmp32:wsnmp32.dll
 0002:000005c4       __imp__SnmpClose@4         100685c4     wsnmp32:wsnmp32.dll
 0002:000005c8       __imp__SnmpCreateVbl@12    100685c8     wsnmp32:wsnmp32.dll
 0002:000005cc       __imp__SnmpFreeVbl@4       100685cc     wsnmp32:wsnmp32.dll
 0002:000005d0       __imp__SnmpCountVbl@4      100685d0     wsnmp32:wsnmp32.dll
 0002:000005d4       __imp__SnmpGetVb@16        100685d4     wsnmp32:wsnmp32.dll
 0002:000005d8       __imp__SnmpSetVb@16        100685d8     wsnmp32:wsnmp32.dll
 0002:000005dc       __imp__SnmpGetLastError@4  100685dc     wsnmp32:wsnmp32.dll
 0002:000005e0       __imp__SnmpOidToStr@12     100685e0     wsnmp32:wsnmp32.dll
 0002:000005e4       __imp__SnmpFreeDescriptor@8 100685e4     wsnmp32:wsnmp32.dll
 0002:000005e8       __imp__SnmpSetTimeout@8    100685e8     wsnmp32:wsnmp32.dll
 0002:000005ec       __imp__SnmpSetRetransmitMode@4 100685ec     wsnmp32:wsnmp32.dll
 0002:000005f0       __imp__SnmpCleanup@0       100685f0     wsnmp32:wsnmp32.dll
 0002:000005f4       __imp__SnmpStartup@20      100685f4     wsnmp32:wsnmp32.dll
 0002:000005f8       __imp__SnmpFreePdu@4       100685f8     wsnmp32:wsnmp32.dll
 0002:000005fc       __imp__SnmpSetRetry@8      100685fc     wsnmp32:wsnmp32.dll
 0002:00000600       __imp__SnmpGetPduData@24   10068600     wsnmp32:wsnmp32.dll
 0002:00000604       __imp__SnmpSetTranslateMode@4 10068604     wsnmp32:wsnmp32.dll
 0002:00000608       \177wsnmp32_NULL_THUNK_DATA 10068608     wsnmp32:wsnmp32.dll
 0002:0000060c       ___xc_a                    1006860c     LIBCMT:crt0init.obj
 0002:00000764       ___xc_z                    10068764     LIBCMT:crt0init.obj
 0002:00000768       ___xi_a                    10068768     LIBCMT:crt0init.obj
 0002:00000780       ___xi_z                    10068780     LIBCMT:crt0init.obj
 0002:00000784       ___xp_a                    10068784     LIBCMT:crt0init.obj
 0002:00000794       ___xp_z                    10068794     LIBCMT:crt0init.obj
 0002:00000798       ___xt_a                    10068798     LIBCMT:crt0init.obj
 0002:0000079c       ___xt_z                    1006879c     LIBCMT:crt0init.obj
 0002:000007d8       ?strlen@asiIpAddr@@2HB     100687d8     asicndload.obj
 0002:000007dc       ?strlen@asiMacAddr@@2HB    100687dc     asicndload.obj
 0002:000007e0       ??_C@_0BE@KOAFJOFJ@createPcapInterface?$AA@ 100687e0     asicndload.obj
 0002:000007f4       ??_C@_0BE@JNDGLHKJ@deletePcapInterface?$AA@ 100687f4     asicndload.obj
 0002:00000808       ??_C@_0BL@IJCEDNBB@createAsiCobraNetDiscovery?$AA@ 10068808     asicndload.obj
 0002:00000824       ??_C@_0BL@MJOGMGCP@deleteAsiCobraNetDiscovery?$AA@ 10068824     asicndload.obj
 0002:00000840       ??_C@_0BN@CPCBBJIC@createAsiAutoAssignIpTracker?$AA@ 10068840     asicndload.obj
 0002:00000860       ??_C@_0BN@EEILGJKJ@deleteAsiAutoAssignIpTracker?$AA@ 10068860     asicndload.obj
 0002:00000880       ??_C@_0BE@BNEAAPLP@createAsiAutoAssign?$AA@ 10068880     asicndload.obj
 0002:00000894       ??_C@_0BE@COHDCGEP@deleteAsiAutoAssign?$AA@ 10068894     asicndload.obj
 0002:000008a8       ??_C@_0BA@MIMAKHBM@asiCnDiscoStart?$AA@ 100688a8     asicndload.obj
 0002:000008b8       ??_C@_0P@HIDGGGJP@asiCnDiscoStop?$AA@ 100688b8     asicndload.obj
 0002:000008c8       ??_C@_0CD@LMMENHIA@asiCnDiscoCreateNotificationClie@ 100688c8     asicndload.obj
 0002:000008ec       ??_C@_0CB@OMINLBKK@asiCnDiscoFreeNotificationClient@ 100688ec     asicndload.obj
 0002:00000910       ??_C@_0BL@LJLINCEL@notificationClientGetEvent?$AA@ 10068910     asicndload.obj
 0002:0000092c       ??_C@_0BA@FCBNALEB@autoAssignStart?$AA@ 1006892c     asicndload.obj
 0002:0000093c       ??_C@_0P@BKCJINBO@autoAssignStop?$AA@ 1006893c     asicndload.obj
 0002:0000094c       ??_C@_0BK@CGGMPDOL@autoAssignGetStatusForMac?$AA@ 1006894c     asicndload.obj
 0002:00000968       ??_C@_0BI@ONLEAPMM@autoAssignAssignIpToMac?$AA@ 10068968     asicndload.obj
 0002:00000980       ??_C@_0BB@OHIHILOE@asicndisco32?4dll?$AA@ 10068980     asicndload.obj
 0002:00000994       ??_C@_06LHGBEIMP@?4?$CFu?4?$CFu?$AA@ 10068994     asimib.obj
 0002:0000099c       ??_C@_03PCJIPBFG@?4?$CFu?$AA@ 1006899c     asimib.obj
 0002:000009a0       ??_C@_04CMEBGENP@?$CFuld?$AA@ 100689a0     asimib.obj
 0002:000009a8       ??_C@_01LFCBOECM@?4?$AA@   100689a8     asimib.obj
 0002:000009ac       ??_C@_04DCHGMGIO@ERR?5?$AA@ 100689ac     asios.obj
 0002:000009b4       ??_C@_04DNGKFIHI@WRN?5?$AA@ 100689b4     asios.obj
 0002:000009bc       ??_C@_04ODFIAEGP@NOT?5?$AA@ 100689bc     asios.obj
 0002:000009c4       ??_C@_04PGGGMIAE@INF?5?$AA@ 100689c4     asios.obj
 0002:000009cc       ??_C@_04EFOCNJDK@DBG?5?$AA@ 100689cc     asios.obj
 0002:000009d4       ??_C@_04JBAIIKM@VRB?5?$AA@ 100689d4     asios.obj
 0002:000009dc       ??_C@_0BJ@DOMENDPD@Unknown?5ASIOS?5Log?5Level?5?$AA@ 100689dc     asios.obj
 0002:000009fc       ??_7SnmpRequest@@6B@       100689fc     asisnmp.obj
 0002:00000a08       ??_7SnmpGetRequest@@6B@    10068a08     asisnmp.obj
 0002:00000a14       ??_7SnmpGetNextRequest@@6B@ 10068a14     asisnmp.obj
 0002:00000a20       ??_7SnmpSetRequest@@6B@    10068a20     asisnmp.obj
 0002:00000a28       ??_C@_06EOMAMIIF@public?$AA@ 10068a28     asisnmp.obj
 0002:00000a30       ??_C@_07NMPLPEPB@private?$AA@ 10068a30     asisnmp.obj
 0002:00000a38       ??_C@_03JALODAI@?$CFld?$AA@ 10068a38     asisnmp.obj
 0002:00000a3c       ??_C@_03FKNCMABI@?$CFlu?$AA@ 10068a3c     asisnmp.obj
 0002:00000a40       ??_C@_05OINFJHGD@?$CFI64u?$AA@ 10068a40     asisnmp.obj
 0002:00000a48       ??_C@_02NJNOFBBI@?$CFx?$AA@ 10068a48     asisnmp.obj
 0002:00000a4c       ??_C@_03EHDGIPBL@?4?$CFx?$AA@ 10068a4c     asisnmp.obj
 0002:00000a50       ??_C@_0M@CDHNGIPM@?$CFu?4?$CFu?4?$CFu?4?$CFu?$AA@ 10068a50     asisnmp.obj
 0002:00000a5c       ??_C@_0BF@NKHODJP@ASX_Cobranet_SetName?$AA@ 10068a5c     asx.obj
 0002:00000a74       ??_C@_0BH@LNMCKAAD@ASX_Cobranet_SetName?$CI?$CJ?$AA@ 10068a74     asx.obj
 0002:00000a8c       ??_C@_0M@GBOPHLFA@asx?4cpp?343?5?$AA@ 10068a8c     asx.obj
 0002:00000a98       ??_C@_0CD@DKLKBLGA@?$CIASX_Cobranet_SetName?$CJ?5ERROR?5?9?$DO?5@ 10068a98     asx.obj
 0002:00000abc       ??_C@_0M@GNLKJELB@asx?4cpp?348?5?$AA@ 10068abc     asx.obj
 0002:00000ac8       ??_C@_0CB@MDHJBGMO@ASX_Cobranet_GetFirmwareRevision@ 10068ac8     asx.obj
 0002:00000aec       ??_C@_0CD@NDLFAEFL@ASX_Cobranet_GetFirmwareRevision@ 10068aec     asx.obj
 0002:00000b10       ??_C@_0M@NOFKLEOJ@asx?4cpp?357?5?$AA@ 10068b10     asx.obj
 0002:00000b1c       ??_C@_0CP@ENCICFKP@?$CIASX_Cobranet_GetFirmwareRevisio@ 10068b1c     asx.obj
 0002:00000b4c       ??_C@_0M@MKCENJOM@asx?4cpp?362?5?$AA@ 10068b4c     asx.obj
 0002:00000b58       ??_C@_0BN@PKJGEMCM@ASX_Cobranet_SetSerialConfig?$AA@ 10068b58     asx.obj
 0002:00000b78       ??_C@_0BP@DEEDBEDA@ASX_Cobranet_SetSerialConfig?$CI?$CJ?$AA@ 10068b78     asx.obj
 0002:00000b98       ??_C@_0M@HHNHKIAM@asx?4cpp?375?5?$AA@ 10068b98     asx.obj
 0002:00000ba4       ??_C@_0CL@OKOEEJLB@?$CIASX_Cobranet_SetSerialConfig?$CJ?5E@ 10068ba4     asx.obj
 0002:00000bd0       ??_C@_0M@CJHPHKLB@asx?4cpp?380?5?$AA@ 10068bd0     asx.obj
 0002:00000bdc       ??_C@_0BL@PEFNCFFF@ASX_Cobranet_GetMACAddress?$AA@ 10068bdc     asx.obj
 0002:00000bf8       ??_C@_0BN@PONAABLI@ASX_Cobranet_GetMACAddress?$CI?$CJ?$AA@ 10068bf8     asx.obj
 0002:00000c18       ??_C@_0M@CGKOEBDO@asx?4cpp?389?5?$AA@ 10068c18     asx.obj
 0002:00000c24       ??_C@_0CJ@CHGNGPBI@?$CIASX_Cobranet_GetMACAddress?$CJ?5ERR@ 10068c24     asx.obj
 0002:00000c50       ??_C@_0M@JGMKLFAI@asx?4cpp?394?5?$AA@ 10068c50     asx.obj
 0002:00000c5c       ??_C@_0CA@OOMCJOLC@ASX_Cobranet_SetStaticIPAddress?$AA@ 10068c5c     asx.obj
 0002:00000c7c       ??_C@_0CC@LDFMBEAI@ASX_Cobranet_SetStaticIPAddress?$CI@ 10068c7c     asx.obj
 0002:00000ca0       ??_C@_0N@DKLLKHJK@asx?4cpp?3103?5?$AA@ 10068ca0     asx.obj
 0002:00000cb0       ??_C@_0CO@OAPICHAL@?$CIASX_Cobranet_SetStaticIPAddress@ 10068cb0     asx.obj
 0002:00000ce0       ??_C@_0N@DGOOEIHL@asx?4cpp?3108?5?$AA@ 10068ce0     asx.obj
 0002:00000cf0       ??_C@_0CC@NLKJHHKD@ASX_Cobranet_SetConductorPriorit@ 10068cf0     asx.obj
 0002:00000d14       ??_C@_0CE@DJFDFIKP@ASX_Cobranet_SetConductorPriorit@ 10068d14     asx.obj
 0002:00000d38       ??_C@_0N@IFAOGICD@asx?4cpp?3117?5?$AA@ 10068d38     asx.obj
 0002:00000d48       ??_C@_0DA@CPLHMKJE@?$CIASX_Cobranet_SetConductorPriori@ 10068d48     asx.obj
 0002:00000d78       ??_C@_0N@JBHAAFCG@asx?4cpp?3122?5?$AA@ 10068d78     asx.obj
 0002:00000d88       ??_C@_0BJ@NDCLPONF@ASX_Cobranet_SetLocation?$AA@ 10068d88     asx.obj
 0002:00000da4       ??_C@_0BL@NEFCLFNJ@ASX_Cobranet_SetLocation?$CI?$CJ?$AA@ 10068da4     asx.obj
 0002:00000dc0       ??_C@_0N@CLIKNMBK@asx?4cpp?3131?5?$AA@ 10068dc0     asx.obj
 0002:00000dd0       ??_C@_0CH@GIHJGMOH@?$CIASX_Cobranet_SetLocation?$CJ?5ERROR@ 10068dd0     asx.obj
 0002:00000df8       ??_C@_0N@COMFMKJP@asx?4cpp?3136?5?$AA@ 10068df8     asx.obj
 0002:00000e08       ??_C@_0CC@ICLEGBPE@ASX_Cobranet_GetConductorPriorit@ 10068e08     asx.obj
 0002:00000e2c       ??_C@_0CE@DIHNHPHA@ASX_Cobranet_GetConductorPriorit@ 10068e2c     asx.obj
 0002:00000e50       ??_C@_0N@LBFEEMHP@asx?4cpp?3145?5?$AA@ 10068e50     asx.obj
 0002:00000e60       ??_C@_0DA@JIAIJHOP@?$CIASX_Cobranet_GetConductorPriori@ 10068e60     asx.obj
 0002:00000e90       ??_C@_0N@PCDOJPB@asx?4cpp?3150?5?$AA@ 10068e90     asx.obj
 0002:00000ea0       ??_C@_0BK@GDBHNNBE@ASX_Cobranet_SetIPAddress?$AA@ 10068ea0     asx.obj
 0002:00000ebc       ??_C@_0BM@KENEJCJI@ASX_Cobranet_SetIPAddress?$CI?$CJ?$AA@ 10068ebc     asx.obj
 0002:00000ed8       ??_C@_0N@PCNCHO@asx?4cpp?3159?5?$AA@ 10068ed8     asx.obj
 0002:00000ee8       ??_C@_0CI@CMEOHFND@?$CIASX_Cobranet_SetIPAddress?$CJ?5ERRO@ 10068ee8     asx.obj
 0002:00000f10       ??_C@_0N@BKJPOOMD@asx?4cpp?3164?5?$AA@ 10068f10     asx.obj
 0002:00000f20       ??_C@_0BF@PFFGNMEO@ASX_Cobranet_GetName?$AA@ 10068f20     asx.obj
 0002:00000f38       ??_C@_0BH@JDIHIBJB@ASX_Cobranet_GetName?$CI?$CJ?$AA@ 10068f38     asx.obj
 0002:00000f50       ??_C@_0N@KHGMJPCD@asx?4cpp?3173?5?$AA@ 10068f50     asx.obj
 0002:00000f60       ??_C@_0CD@GDKHANDH@?$CIASX_Cobranet_GetName?$CJ?5ERROR?5?9?$DO?5@ 10068f60     asx.obj
 0002:00000f84       ??_C@_0N@KLDJHAMC@asx?4cpp?3178?5?$AA@ 10068f84     asx.obj
 0002:00000f94       ??_C@_0CA@EBGFHHGM@ASX_Cobranet_GetConductorStatus?$AA@ 10068f94     asx.obj
 0002:00000fb4       ??_C@_0CC@HFDBAJOC@ASX_Cobranet_GetConductorStatus?$CI@ 10068fb4     asx.obj
 0002:00000fd8       ??_C@_0N@PIAGCHKJ@asx?4cpp?3187?5?$AA@ 10068fd8     asx.obj
 0002:00000fe8       ??_C@_0CO@OGNHPODD@?$CIASX_Cobranet_GetConductorStatus@ 10068fe8     asx.obj
 0002:00001018       ??_C@_0N@EGHBICCH@asx?4cpp?3192?5?$AA@ 10069018     asx.obj
 0002:00001028       ??_C@_0CF@HNEHJFLM@ASX_Cobranet_SetLatencyAndSample@ 10069028     asx.obj
 0002:00001050       ??_C@_0CH@LKANHDIL@ASX_Cobranet_SetLatencyAndSample@ 10069050     asx.obj
 0002:00001078       ??_C@_0N@HOJPAJCE@asx?4cpp?3201?5?$AA@ 10069078     asx.obj
 0002:00001088       ??_C@_0DD@MIACIFFJ@?$CIASX_Cobranet_SetLatencyAndSampl@ 10069088     asx.obj
 0002:000010bc       ??_C@_0N@HLNABPKB@asx?4cpp?3206?5?$AA@ 100690bc     asx.obj
 0002:000010cc       ??_C@_0BK@BHKJBBFI@ASX_Cobranet_GetIPAddress?$AA@ 100690cc     asx.obj
 0002:000010e8       ??_C@_0BM@GKMKGILE@ASX_Cobranet_GetIPAddress?$CI?$CJ?$AA@ 100690e8     asx.obj
 0002:00001104       ??_C@_0N@MIDADPPJ@asx?4cpp?3219?5?$AA@ 10069104     asx.obj
 0002:00001114       ??_C@_0CI@KMIILIHF@?$CIASX_Cobranet_GetIPAddress?$CJ?5ERRO@ 10069114     asx.obj
 0002:0000113c       ??_C@_0N@NCFNADEE@asx?4cpp?3224?5?$AA@ 1006913c     asx.obj
 0002:0000114c       ??_C@_0CF@GLCKHENO@ASX_Cobranet_GetLatencyAndSample@ 1006914c     asx.obj
 0002:00001174       ??_C@_0CH@DKMLLOCN@ASX_Cobranet_GetLatencyAndSample@ 10069174     asx.obj
 0002:0000119c       ??_C@_0N@GPKOHCKE@asx?4cpp?3233?5?$AA@ 1006919c     asx.obj
 0002:000011ac       ??_C@_0DD@MEGNIPFL@?$CIASX_Cobranet_GetLatencyAndSampl@ 100691ac     asx.obj
 0002:000011e0       ??_C@_0N@GDPLJNEF@asx?4cpp?3238?5?$AA@ 100691e0     asx.obj
 0002:000011f0       ??_C@_0BN@MIIADODF@ASX_Cobranet_GetSerialConfig?$AA@ 100691f0     asx.obj
 0002:00001210       ??_C@_0BP@BBEIJPCO@ASX_Cobranet_GetSerialConfig?$CI?$CJ?$AA@ 10069210     asx.obj
 0002:00001230       ??_C@_0N@PFHAOCMB@asx?4cpp?3247?5?$AA@ 10069230     asx.obj
 0002:00001240       ??_C@_0CL@DLECKGGF@?$CIASX_Cobranet_GetSerialConfig?$CJ?5E@ 10069240     asx.obj
 0002:0000126c       ??_C@_0N@ELAHEHEP@asx?4cpp?3252?5?$AA@ 1006926c     asx.obj
 0002:0000127c       ??_C@_0BM@HBALAOBH@ASX_Cobranet_GetPersistence?$AA@ 1006927c     asx.obj
 0002:00001298       ??_C@_0BO@JACDFACJ@ASX_Cobranet_GetPersistence?$CI?$CJ?$AA@ 10069298     asx.obj
 0002:000012b8       ??_C@_0N@FLPEFGPI@asx?4cpp?3261?5?$AA@ 100692b8     asx.obj
 0002:000012c8       ??_C@_0CK@LJNGPODB@?$CIASX_Cobranet_GetPersistence?$CJ?5ER@ 100692c8     asx.obj
 0002:000012f4       ??_C@_0N@FOLLEAHN@asx?4cpp?3266?5?$AA@ 100692f4     asx.obj
 0002:00001304       ??_C@_0BK@IADCIIEB@ASX_Cobranet_GetErrorInfo?$AA@ 10069304     asx.obj
 0002:00001320       ??_C@_0BM@HIBJHNNH@ASX_Cobranet_GetErrorInfo?$CI?$CJ?$AA@ 10069320     asx.obj
 0002:0000133c       ??_C@_0N@OEEBJJEB@asx?4cpp?3275?5?$AA@ 1006933c     asx.obj
 0002:0000134c       ??_C@_0CI@LHCNEJEK@?$CIASX_Cobranet_GetErrorInfo?$CJ?5ERRO@ 1006934c     asx.obj
 0002:00001374       ??_C@_0N@LKOJELPM@asx?4cpp?3280?5?$AA@ 10069374     asx.obj
 0002:00001384       ??_C@_0CA@BEOIKIFK@ASX_Cobranet_GetStaticIPAddress?$AA@ 10069384     asx.obj
 0002:000013a4       ??_C@_0CC@OKEBACFP@ASX_Cobranet_GetStaticIPAddress?$CI@ 100693a4     asx.obj
 0002:000013c8       ??_C@_0N@LFDIHAHD@asx?4cpp?3289?5?$AA@ 100693c8     asx.obj
 0002:000013d8       ??_C@_0CO@IMCLFDMI@?$CIASX_Cobranet_GetStaticIPAddress@ 100693d8     asx.obj
 0002:00001408       ??_C@_0N@FFMIEEF@asx?4cpp?3294?5?$AA@ 10069408     asx.obj
 0002:00001418       ??_C@_0BJ@NMDFCIFG@ASX_Cobranet_GetLocation?$AA@ 10069418     asx.obj
 0002:00001434       ??_C@_0BL@KLEMAGKO@ASX_Cobranet_GetLocation?$CI?$CJ?$AA@ 10069434     asx.obj
 0002:00001450       ??_C@_0N@EAHLPEPK@asx?4cpp?3303?5?$AA@ 10069450     asx.obj
 0002:00001460       ??_C@_0CH@MLNDABHC@?$CIASX_Cobranet_GetLocation?$CJ?5ERROR@ 10069460     asx.obj
 0002:00001488       ??_C@_0N@EMCOBLBL@asx?4cpp?3308?5?$AA@ 10069488     asx.obj
 0002:00001498       ??_C@_0BN@GLNFAKFM@ASX_Cobranet_SetSerialEnable?$AA@ 10069498     asx.obj
 0002:000014b8       ??_C@_0BP@IEMDBICA@ASX_Cobranet_SetSerialEnable?$CI?$CJ?$AA@ 100694b8     asx.obj
 0002:000014d8       ??_C@_0N@PPMODLED@asx?4cpp?3317?5?$AA@ 100694d8     asx.obj
 0002:000014e8       ??_C@_0CL@OOINLLBM@?$CIASX_Cobranet_SetSerialEnable?$CJ?5E@ 100694e8     asx.obj
 0002:00001514       ??_C@_0N@OLLAFGEG@asx?4cpp?3322?5?$AA@ 10069514     asx.obj
 0002:00001524       ??_C@_0BM@LPBFPEDL@ASX_Cobranet_SetPersistence?$AA@ 10069524     asx.obj
 0002:00001540       ??_C@_0BO@PEHKOOJL@ASX_Cobranet_SetPersistence?$CI?$CJ?$AA@ 10069540     asx.obj
 0002:00001560       ??_C@_0N@FBEKIPHK@asx?4cpp?3331?5?$AA@ 10069560     asx.obj
 0002:00001570       ??_C@_0CK@KEFONLJF@?$CIASX_Cobranet_SetPersistence?$CJ?5ER@ 10069570     asx.obj
 0002:0000159c       ??_C@_0N@FEAFJJPP@asx?4cpp?3336?5?$AA@ 1006959c     asx.obj
 0002:000015ac       ??_C@_0BN@FJMDHIEF@ASX_Cobranet_GetSerialEnable?$AA@ 100695ac     asx.obj
 0002:000015cc       ??_C@_0BP@KBMIJDDO@ASX_Cobranet_GetSerialEnable?$CI?$CJ?$AA@ 100695cc     asx.obj
 0002:000015ec       ??_C@_0N@MLJEBPBP@asx?4cpp?3345?5?$AA@ 100695ec     asx.obj
 0002:000015fc       ??_C@_0CL@DPCLFEMI@?$CIASX_Cobranet_GetSerialEnable?$CJ?5E@ 100695fc     asx.obj
 0002:00001628       ??_C@_0N@HFODLKJB@asx?4cpp?3350?5?$AA@ 10069628     asx.obj
 0002:00001638       ??_C@_0BJ@JGDLJNEC@ASX_Cobranet_GetIfStatus?$AA@ 10069638     asx.obj
 0002:00001654       ??_C@_0BL@DOOJNMPG@ASX_Cobranet_GetIfStatus?$CI?$CJ?$AA@ 10069654     asx.obj
 0002:00001670       ??_C@_0N@HKDCIBBO@asx?4cpp?3359?5?$AA@ 10069670     asx.obj
 0002:00001680       ??_C@_0CH@IIMOFPKF@?$CIASX_Cobranet_GetIfStatus?$CJ?5ERROR@ 10069680     asx.obj
 0002:000016a8       ??_C@_0N@GAFPLNKD@asx?4cpp?3364?5?$AA@ 100696a8     asx.obj
 0002:000016b8       ??_C@_0BM@GOEAPLBE@ASX_Cobranet_GetDescription?$AA@ 100696b8     asx.obj
 0002:000016d4       ??_C@_0BO@HGNJBKDC@ASX_Cobranet_GetDescription?$CI?$CJ?$AA@ 100696d4     asx.obj
 0002:000016f4       ??_C@_0N@NKKFGEJP@asx?4cpp?3377?5?$AA@ 100696f4     asx.obj
 0002:00001704       ??_C@_0CK@PLPOEPDF@?$CIASX_Cobranet_GetDescription?$CJ?5ER@ 10069704     asx.obj
 0002:00001730       ??_C@_0N@IEANLGCC@asx?4cpp?3382?5?$AA@ 10069730     asx.obj
 0002:00001740       ??_C@_0BN@HGHGJGNF@ASX_SampleClock_SetLocalRate?$AA@ 10069740     asx.obj
 0002:00001760       ??_C@_0BP@JHDLPJOO@ASX_SampleClock_SetLocalRate?$CI?$CJ?$AA@ 10069760     asx.obj
 0002:00001780       ??_C@_0N@DIDMKNPF@asx?4cpp?3394?5?$AA@ 10069780     asx.obj
 0002:00001790       ??_C@_0CL@BKGIINGP@?$CIASX_SampleClock_SetLocalRate?$CJ?5E@ 10069790     asx.obj
 0002:000017bc       ??_C@_0N@DAOEDOKG@asx?4cpp?3399?5?$AA@ 100697bc     asx.obj
 0002:000017cc       ??_C@_0BO@JKDPHNGH@ASX_SampleClock_SetAutoSource?$AA@ 100697cc     asx.obj
 0002:000017ec       ??_C@_0CA@HGBAOCGN@ASX_SampleClock_SetAutoSource?$CI?$CJ?$AA@ 100697ec     asx.obj
 0002:0000180c       ??_C@_0N@POAOMHAL@asx?4cpp?3408?5?$AA@ 1006980c     asx.obj
 0002:0000181c       ??_C@_0CM@BGJPEGGI@?$CIASX_SampleClock_SetAutoSource?$CJ?5@ 1006981c     asx.obj
 0002:00001848       ??_C@_0N@EKOHEPIP@asx?4cpp?3413?5?$AA@ 10069848     asx.obj
 0002:00001858       ??_C@_0BP@MAIMHFNJ@ASX_SampleClock_GetClockSource?$AA@ 10069858     asx.obj
 0002:00001878       ??_C@_0CB@CINLDNK@ASX_SampleClock_GetClockSource?$CI?$CJ@ 10069878     asx.obj
 0002:0000189c       ??_C@_0N@FJJAIKFG@asx?4cpp?3422?5?$AA@ 1006989c     asx.obj
 0002:000018ac       ??_C@_0CN@LLCPALGF@?$CIASX_SampleClock_GetClockSource?$CJ@ 100698ac     asx.obj
 0002:000018dc       ??_C@_0N@FPFLEILN@asx?4cpp?3427?5?$AA@ 100698dc     asx.obj
 0002:000018ec       ??_C@_0CB@BKMJBCJI@ASX_SampleClock_SetLocalRateLock@ 100698ec     asx.obj
 0002:00001910       ??_C@_0CD@DIDJODCA@ASX_SampleClock_SetLocalRateLock@ 10069910     asx.obj
 0002:00001934       ??_C@_0N@OGCFEFOP@asx?4cpp?3436?5?$AA@ 10069934     asx.obj
 0002:00001944       ??_C@_0CP@BLMOCMHM@?$CIASX_SampleClock_SetLocalRateLoc@ 10069944     asx.obj
 0002:00001974       ??_C@_0N@HOLNGLND@asx?4cpp?3441?5?$AA@ 10069974     asx.obj
 0002:00001984       ??_C@_0CD@FCEHDFFP@ASX_SampleClock_EnumerateLocalRa@ 10069984     asx.obj
 0002:000019a8       ??_C@_0CF@BJIIFPEM@ASX_SampleClock_EnumerateLocalRa@ 100699a8     asx.obj
 0002:000019d0       ??_C@_0N@MHMDGGIB@asx?4cpp?3450?5?$AA@ 100699d0     asx.obj
 0002:000019e0       ??_C@_0DB@NDKDDPJ@?$CIASX_SampleClock_EnumerateLocalR@ 100699e0     asx.obj
 0002:00001a14       ??_C@_0N@MBAIKEGK@asx?4cpp?3455?5?$AA@ 10069a14     asx.obj
 0002:00001a24       ??_C@_0CF@IACBCJFH@ASX_SampleClock_EnumerateClockSo@ 10069a24     asx.obj
 0002:00001a4c       ??_C@_0CH@MFFAFLGN@ASX_SampleClock_EnumerateClockSo@ 10069a4c     asx.obj
 0002:00001a74       ??_C@_0N@NLGFJINH@asx?4cpp?3468?5?$AA@ 10069a74     asx.obj
 0002:00001a84       ??_C@_0DD@KNGFIKIE@?$CIASX_SampleClock_EnumerateClockS@ 10069a84     asx.obj
 0002:00001ab8       ??_C@_0N@GPIMBAFD@asx?4cpp?3473?5?$AA@ 10069ab8     asx.obj
 0002:00001ac8       ??_C@_0BP@OJCIPPF@ASX_SampleClock_SetClockSource?$AA@ 10069ac8     asx.obj
 0002:00001ae8       ??_C@_0CB@GGNEANGI@ASX_SampleClock_SetClockSource?$CI?$CJ@ 10069ae8     asx.obj
 0002:00001b0c       ??_C@_0N@DGCNGKDC@asx?4cpp?3482?5?$AA@ 10069b0c     asx.obj
 0002:00001b1c       ??_C@_0CN@KGKHCOMB@?$CIASX_SampleClock_SetClockSource?$CJ@ 10069b1c     asx.obj
 0002:00001b4c       ??_C@_0N@DAOGKINJ@asx?4cpp?3487?5?$AA@ 10069b4c     asx.obj
 0002:00001b5c       ??_C@_0BN@CMIFKJJ@ASX_SampleClock_GetLocalRate?$AA@ 10069b5c     asx.obj
 0002:00001b7c       ??_C@_0BP@FJCFADMC@ASX_SampleClock_GetLocalRate?$CI?$CJ?$AA@ 10069b7c     asx.obj
 0002:00001b9c       ??_C@_0N@IJJIKFIL@asx?4cpp?3496?5?$AA@ 10069b9c     asx.obj
 0002:00001bac       ??_C@_0CL@JKKOEAMJ@?$CIASX_SampleClock_GetLocalRate?$CJ?5E@ 10069bac     asx.obj
 0002:00001bd8       ??_C@_0N@MMLPNFDE@asx?4cpp?3501?5?$AA@ 10069bd8     asx.obj
 0002:00001be8       ??_C@_0CB@HOJAKMCK@ASX_SampleClock_GetLocalRateLock@ 10069be8     asx.obj
 0002:00001c0c       ??_C@_0CD@MCBDNFMI@ASX_SampleClock_GetLocalRateLock@ 10069c0c     asx.obj
 0002:00001c30       ??_C@_0N@HCMIHALK@asx?4cpp?3514?5?$AA@ 10069c30     asx.obj
 0002:00001c40       ??_C@_0CP@JKKBJMFO@?$CIASX_SampleClock_GetLocalRateLoc@ 10069c40     asx.obj
 0002:00001c70       ??_C@_0N@HKBAODOJ@asx?4cpp?3519?5?$AA@ 10069c70     asx.obj
 0002:00001c80       ??_C@_0BO@EPJCANGI@ASX_SampleClock_GetSampleRate?$AA@ 10069c80     asx.obj
 0002:00001ca0       ??_C@_0CA@KBINFKDD@ASX_SampleClock_GetSampleRate?$CI?$CJ?$AA@ 10069ca0     asx.obj
 0002:00001cc0       ??_C@_0N@GJGHCGDA@asx?4cpp?3528?5?$AA@ 10069cc0     asx.obj
 0002:00001cd0       ??_C@_0CM@JGHEKBOL@?$CIASX_SampleClock_GetSampleRate?$CJ?5@ 10069cd0     asx.obj
 0002:00001cfc       ??_C@_0N@NNIOKOLE@asx?4cpp?3533?5?$AA@ 10069cfc     asx.obj
 0002:00001d0c       ??_C@_0BO@OFCBMOBA@ASX_SampleClock_GetAutoSource?$AA@ 10069d0c     asx.obj
 0002:00001d2c       ??_C@_0CA@EEAGJAHE@ASX_SampleClock_GetAutoSource?$CI?$CJ?$AA@ 10069d2c     asx.obj
 0002:00001d4c       ??_C@_0N@EBJLPMDK@asx?4cpp?3542?5?$AA@ 10069d4c     asx.obj
 0002:00001d5c       ??_C@_0CM@CJKKIGHI@?$CIASX_SampleClock_GetAutoSource?$CJ?5@ 10069d5c     asx.obj
 0002:00001d88       ??_C@_0N@EHFADONB@asx?4cpp?3547?5?$AA@ 10069d88     asx.obj
 0002:00001d98       ??_C@_0BJ@JMGCHDEP@ASX_Control_GetSubSystem?$AA@ 10069d98     asx.obj
 0002:00001db4       ??_C@_0BL@MMPFGHJN@ASX_Control_GetSubSystem?$CI?$CJ?$AA@ 10069db4     asx.obj
 0002:00001dd0       ??_C@_0N@PFHCHELO@asx?4cpp?3559?5?$AA@ 10069dd0     asx.obj
 0002:00001de0       ??_C@_0BK@MPKLDOBN@ASX_Control_GetHpiControl?$AA@ 10069de0     asx.obj
 0002:00001dfc       ??_C@_0BM@EMBFDGKP@ASX_Control_GetHpiControl?$CI?$CJ?$AA@ 10069dfc     asx.obj
 0002:00001e18       ??_C@_0N@FCOMDJOD@asx?4cpp?3573?5?$AA@ 10069e18     asx.obj
 0002:00001e28       ??_C@_0CI@HCCFKIDI@?$CIASX_Control_GetHpiControl?$CJ?5ERRO@ 10069e28     asx.obj
 0002:00001e50       ??_C@_0N@FOLJNGAC@asx?4cpp?3578?5?$AA@ 10069e50     asx.obj
 0002:00001e60       ??_C@_0BP@EEIIEMLI@ASX_Control_GetDestinationNode?$AA@ 10069e60     asx.obj
 0002:00001e80       ??_C@_0CB@CBGOOFDA@ASX_Control_GetDestinationNode?$CI?$CJ@ 10069e80     asx.obj
 0002:00001ea4       ??_C@_0N@NIGIBGJ@asx?4cpp?3587?5?$AA@ 10069ea4     asx.obj
 0002:00001eb4       ??_C@_0BE@OOJPGKEO@ASX_Control_GetType?$AA@ 10069eb4     asx.obj
 0002:00001ec8       ??_C@_0BG@LBIFIMOB@ASX_Control_GetType?$CI?$CJ?$AA@ 10069ec8     asx.obj
 0002:00001ee0       ??_C@_0N@ILBPKPOE@asx?4cpp?3601?5?$AA@ 10069ee0     asx.obj
 0002:00001ef0       ??_C@_0BK@KOFIKEAL@ASX_Control_GetSourceNode?$AA@ 10069ef0     asx.obj
 0002:00001f0c       ??_C@_0BM@EAFHJINB@ASX_Control_GetSourceNode?$CI?$CJ?$AA@ 10069f0c     asx.obj
 0002:00001f28       ??_C@_0N@DEKKGAFN@asx?4cpp?3615?5?$AA@ 10069f28     asx.obj
 0002:00001f38       ??_C@_0CB@NHKDONGP@ASX_System_RegisterErrorCallback@ 10069f38     asx.obj
 0002:00001f5c       ??_C@_0CD@EOMGLGLN@ASX_System_RegisterErrorCallback@ 10069f5c     asx.obj
 0002:00001f80       ??_C@_0N@JMOFBGIP@asx?4cpp?3636?5?$AA@ 10069f80     asx.obj
 0002:00001f90       ??_C@_0CP@HFAAEJHP@?$CIASX_System_RegisterErrorCallbac@ 10069f90     asx.obj
 0002:00001fc0       ??_C@_0N@EHNDILD@asx?4cpp?3641?5?$AA@ 10069fc0     asx.obj
 0002:00001fd0       ??_C@_0BL@BMLOJAJE@ASX_System_GetAdapterCount?$AA@ 10069fd0     asx.obj
 0002:00001fec       ??_C@_0BN@JHDKEIFH@ASX_System_GetAdapterCount?$CI?$CJ?$AA@ 10069fec     asx.obj
 0002:0000200c       ??_C@_0N@LNADDFOB@asx?4cpp?3650?5?$AA@ 1006a00c     asx.obj
 0002:0000201c       ??_C@_0CJ@JBLDKEPG@?$CIASX_System_GetAdapterCount?$CJ?5ERR@ 1006a01c     asx.obj
 0002:00002048       ??_C@_0N@LLMIPHAK@asx?4cpp?3655?5?$AA@ 1006a048     asx.obj
 0002:00002058       ??_C@_0BG@DMIHFJOI@ASX_System_GetVersion?$AA@ 1006a058     asx.obj
 0002:00002070       ??_C@_0BI@PGAICEIA@ASX_System_GetVersion?$CI?$CJ?$AA@ 1006a070     asx.obj
 0002:00002088       ??_C@_0N@BEIOCJAE@asx?4cpp?3672?5?$AA@ 1006a088     asx.obj
 0002:00002098       ??_C@_0CE@HFGMDCFD@?$CIASX_System_GetVersion?$CJ?5ERROR?5?9?$DO@ 1006a098     asx.obj
 0002:000020bc       ??_C@_0N@BCEFOLOP@asx?4cpp?3677?5?$AA@ 1006a0bc     asx.obj
 0002:000020cc       ??_C@_0P@JHNDNCLA@Default?5System?$AA@ 1006a0cc     asx.obj
 0002:000020dc       ??_C@_0BD@COGGLCJP@ASX_System_GetName?$AA@ 1006a0dc     asx.obj
 0002:000020f0       ??_C@_0BF@KBKOOCKA@ASX_System_GetName?$CI?$CJ?$AA@ 1006a0f0     asx.obj
 0002:00002108       ??_C@_0N@LIGMNHOM@asx?4cpp?3709?5?$AA@ 1006a108     asx.obj
 0002:00002118       ??_C@_0CB@CDGFLLDC@?$CIASX_System_GetName?$CJ?5ERROR?5?9?$DO?5?$CFd@ 1006a118     asx.obj
 0002:0000213c       ??_C@_0N@IAICDNK@asx?4cpp?3714?5?$AA@ 1006a13c     asx.obj
 0002:0000214c       ??_C@_0BN@PIELBCEA@ASX_System_SetMessageLogging?$AA@ 1006a14c     asx.obj
 0002:0000216c       ??_C@_0BP@HBNIEOLF@ASX_System_SetMessageLogging?$CI?$CJ?$AA@ 1006a16c     asx.obj
 0002:0000218c       ??_C@_0N@KEMKCJLK@asx?4cpp?3731?5?$AA@ 1006a18c     asx.obj
 0002:0000219c       ??_C@_0CL@GLNJNGIH@?$CIASX_System_SetMessageLogging?$CJ?5E@ 1006a19c     asx.obj
 0002:000021c8       ??_C@_0N@KBIFDPDP@asx?4cpp?3736?5?$AA@ 1006a1c8     asx.obj
 0002:000021d8       ??_C@_0BG@GHPPDHEC@ASX_System_GetAdapter?$AA@ 1006a1d8     asx.obj
 0002:000021f0       ??_C@_0BI@IOKGHME@ASX_System_GetAdapter?$CI?$CJ?$AA@ 1006a1f0     asx.obj
 0002:00002208       ??_C@_0N@JCNGLDLP@asx?4cpp?3760?5?$AA@ 1006a208     asx.obj
 0002:00002218       ??_C@_0CE@JIFBELII@?$CIASX_System_GetAdapter?$CJ?5ERROR?5?9?$DO@ 1006a218     asx.obj
 0002:0000223c       ??_C@_0N@JEBNHBFE@asx?4cpp?3765?5?$AA@ 1006a23c     asx.obj
 0002:0000224c       ??_C@_0BN@NNEAJJFO@ASX_System_GetMessageLogging?$AA@ 1006a24c     asx.obj
 0002:0000226c       ??_C@_0BP@NPPDAOMJ@ASX_System_GetMessageLogging?$CI?$CJ?$AA@ 1006a26c     asx.obj
 0002:0000228c       ??_C@_0N@CEHJIFGC@asx?4cpp?3778?5?$AA@ 1006a28c     asx.obj
 0002:0000229c       ??_C@_0CL@LODIPIND@?$CIASX_System_GetMessageLogging?$CJ?5E@ 1006a29c     asx.obj
 0002:000022c8       ??_C@_0N@HAEPHKNF@asx?4cpp?3783?5?$AA@ 1006a2c8     asx.obj
 0002:000022d8       ??_C@_0P@LECNIEF@ASX_EQ_GetInfo?$AA@ 1006a2d8     asx.obj
 0002:000022e8       ??_C@_0BB@HHBOGCFH@ASX_EQ_GetInfo?$CI?$CJ?$AA@ 1006a2e8     asx.obj
 0002:000022fc       ??_C@_0N@MFGEJIGG@asx?4cpp?3799?5?$AA@ 1006a2fc     asx.obj
 0002:0000230c       ??_C@_0BN@HJOCPLCA@?$CIASX_EQ_GetInfo?$CJ?5ERROR?5?9?$DO?5?$CFd?$AA@ 1006a30c     asx.obj
 0002:0000232c       ??_C@_0N@DCOENDGO@asx?4cpp?3804?5?$AA@ 1006a32c     asx.obj
 0002:0000233c       ??_C@_0P@MJBGHBHB@ASX_EQ_GetBand?$AA@ 1006a33c     asx.obj
 0002:0000234c       ??_C@_0BB@GDDOEILI@ASX_EQ_GetBand?$CI?$CJ?$AA@ 1006a34c     asx.obj
 0002:00002360       ??_C@_0N@IPBHKCIO@asx?4cpp?3813?5?$AA@ 1006a360     asx.obj
 0002:00002370       ??_C@_0BN@OPFAICCK@?$CIASX_EQ_GetBand?$CJ?5ERROR?5?9?$DO?5?$CFd?$AA@ 1006a370     asx.obj
 0002:00002390       ??_C@_0N@IDECENGP@asx?4cpp?3818?5?$AA@ 1006a390     asx.obj
 0002:000023a0       ??_C@_0BA@OKKCKBKO@ASX_EQ_SetState?$AA@ 1006a3a0     asx.obj
 0002:000023b0       ??_C@_0BC@ODENGAAI@ASX_EQ_SetState?$CI?$CJ?$AA@ 1006a3b0     asx.obj
 0002:000023c4       ??_C@_0N@JKKLKFLM@asx?4cpp?3827?5?$AA@ 1006a3c4     asx.obj
 0002:000023d4       ??_C@_0BO@FHKCDDPH@?$CIASX_EQ_SetState?$CJ?5ERROR?5?9?$DO?5?$CFd?$AA@ 1006a3d4     asx.obj
 0002:000023f4       ??_C@_0N@CENMAADC@asx?4cpp?3832?5?$AA@ 1006a3f4     asx.obj
 0002:00002404       ??_C@_0P@DBOHEOKA@ASX_EQ_SetBand?$AA@ 1006a404     asx.obj
 0002:00002414       ??_C@_0BB@ENHLGJCK@ASX_EQ_SetBand?$CI?$CJ?$AA@ 1006a414     asx.obj
 0002:00002428       ??_C@_0N@LLENIGNC@asx?4cpp?3841?5?$AA@ 1006a428     asx.obj
 0002:00002438       ??_C@_0BN@LGENJEHN@?$CIASX_EQ_SetBand?$CJ?5ERROR?5?9?$DO?5?$CFd?$AA@ 1006a438     asx.obj
 0002:00002458       ??_C@_0N@LOACJAFH@asx?4cpp?3846?5?$AA@ 1006a458     asx.obj
 0002:00002468       ??_C@_0BB@DFNEABGC@ASX_PAD_GetTitle?$AA@ 1006a468     asx.obj
 0002:0000247c       ??_C@_0BD@FCNEIENE@ASX_PAD_GetTitle?$CI?$CJ?$AA@ 1006a47c     asx.obj
 0002:00002490       ??_C@_0N@MCANKDI@asx?4cpp?3858?5?$AA@ 1006a490     asx.obj
 0002:000024a0       ??_C@_0BP@NLMEJDKG@?$CIASX_PAD_GetTitle?$CJ?5ERROR?5?9?$DO?5?$CFd?$AA@ 1006a4a0     asx.obj
 0002:000024c0       ??_C@_0N@BCMAJKDH@asx?4cpp?3863?5?$AA@ 1006a4c0     asx.obj
 0002:000024d0       ??_C@_0BH@GCLLDGCH@ASX_PAD_GetChannelName?$AA@ 1006a4d0     asx.obj
 0002:000024e8       ??_C@_0BJ@GHGHMNPE@ASX_PAD_GetChannelName?$CI?$CJ?$AA@ 1006a4e8     asx.obj
 0002:00002504       ??_C@_0N@KLLOJHGF@asx?4cpp?3872?5?$AA@ 1006a504     asx.obj
 0002:00002514       ??_C@_0CF@MMDEIAAD@?$CIASX_PAD_GetChannelName?$CJ?5ERROR?5?9@ 1006a514     asx.obj
 0002:0000253c       ??_C@_0N@KNHFFFIO@asx?4cpp?3877?5?$AA@ 1006a53c     asx.obj
 0002:0000254c       ??_C@_0BB@JCIKGJCN@ASX_PAD_GetRdsPI?$AA@ 1006a54c     asx.obj
 0002:00002560       ??_C@_0BD@GGFMJJCK@ASX_PAD_GetRdsPI?$CI?$CJ?$AA@ 1006a560     asx.obj
 0002:00002574       ??_C@_0N@PENECPOP@asx?4cpp?3886?5?$AA@ 1006a574     asx.obj
 0002:00002584       ??_C@_0BP@OCLCKEE@?$CIASX_PAD_GetRdsPI?$CJ?5ERROR?5?9?$DO?5?$CFd?$AA@ 1006a584     asx.obj
 0002:000025a4       ??_C@_0N@EJCHFOAP@asx?4cpp?3891?5?$AA@ 1006a5a4     asx.obj
 0002:000025b4       ??_C@_0BC@JLFIAGEG@ASX_PAD_GetArtist?$AA@ 1006a5b4     asx.obj
 0002:000025c8       ??_C@_0BE@DNFIFOFN@ASX_PAD_GetArtist?$CI?$CJ?$AA@ 1006a5c8     asx.obj
 0002:000025dc       ??_C@_0N@IINFCAC@asx?4cpp?3900?5?$AA@ 1006a5dc     asx.obj
 0002:000025ec       ??_C@_0CA@KGOKBOAH@?$CIASX_PAD_GetArtist?$CJ?5ERROR?5?9?$DO?5?$CFd?$AA@ 1006a5ec     asx.obj
 0002:0000260c       ??_C@_0N@OEGJAOJ@asx?4cpp?3905?5?$AA@ 1006a60c     asx.obj
 0002:0000261c       ??_C@_0BN@BPPDFHLL@ASX_PAD_GetProgramTypeString?$AA@ 1006a61c     asx.obj
 0002:0000263c       ??_C@_0BP@IACGCEGE@ASX_PAD_GetProgramTypeString?$CI?$CJ?$AA@ 1006a63c     asx.obj
 0002:0000265c       ??_C@_0N@LHDIJNLL@asx?4cpp?3914?5?$AA@ 1006a65c     asx.obj
 0002:0000266c       ??_C@_0CL@ODIHJJJ@?$CIASX_PAD_GetProgramTypeString?$CJ?5E@ 1006a66c     asx.obj
 0002:00002698       ??_C@_0N@LPOAAOOI@asx?4cpp?3919?5?$AA@ 1006a698     asx.obj
 0002:000026a8       ??_C@_0BH@FIAKAACO@ASX_PAD_GetProgramType?$AA@ 1006a6a8     asx.obj
 0002:000026c0       ??_C@_0BJ@HJBPNJJF@ASX_PAD_GetProgramType?$CI?$CJ?$AA@ 1006a6c0     asx.obj
 0002:000026dc       ??_C@_0N@KMJHMLDB@asx?4cpp?3928?5?$AA@ 1006a6dc     asx.obj
 0002:000026ec       ??_C@_0CF@FBGBKKLN@?$CIASX_PAD_GetProgramType?$CJ?5ERROR?5?9@ 1006a6ec     asx.obj
 0002:00002714       ??_C@_0N@BIHOEDLF@asx?4cpp?3933?5?$AA@ 1006a714     asx.obj
 0002:00002724       ??_C@_0BD@CFMBCBFE@ASX_PAD_GetComment?$AA@ 1006a724     asx.obj
 0002:00002738       ??_C@_0BF@OAKGCFHM@ASX_PAD_GetComment?$CI?$CJ?$AA@ 1006a738     asx.obj
 0002:00002750       ??_C@_0N@IEGLBBDL@asx?4cpp?3942?5?$AA@ 1006a750     asx.obj
 0002:00002760       ??_C@_0CB@OCKMLEPN@?$CIASX_PAD_GetComment?$CJ?5ERROR?5?9?$DO?5?$CFd@ 1006a760     asx.obj
 0002:00002784       ??_C@_0N@ICKANDNA@asx?4cpp?3947?5?$AA@ 1006a784     asx.obj
 0002:00002794       ??_C@_0BI@PBHBGMIL@ASX_Mic_SetPhantomPower?$AA@ 1006a794     asx.obj
 0002:000027ac       ??_C@_0BK@OOGLBFDB@ASX_Mic_SetPhantomPower?$CI?$CJ?$AA@ 1006a7ac     asx.obj
 0002:000027c8       ??_C@_0N@DAICJJLP@asx?4cpp?3959?5?$AA@ 1006a7c8     asx.obj
 0002:000027d8       ??_C@_0CG@BHKIIFAG@?$CIASX_Mic_SetPhantomPower?$CJ?5ERROR?5@ 1006a7d8     asx.obj
 0002:00002800       ??_C@_0N@CKOPKFAC@asx?4cpp?3964?5?$AA@ 1006a800     asx.obj
 0002:00002810       ??_C@_0BI@MDGHBOJC@ASX_Mic_GetPhantomPower?$AA@ 1006a810     asx.obj
 0002:00002828       ??_C@_0BK@MLGAJOCP@ASX_Mic_GetPhantomPower?$CI?$CJ?$AA@ 1006a828     asx.obj
 0002:00002844       ??_C@_0N@JHBMNEOC@asx?4cpp?3973?5?$AA@ 1006a844     asx.obj
 0002:00002854       ??_C@_0CG@MGAOGKNC@?$CIASX_Mic_GetPhantomPower?$CJ?5ERROR?5@ 1006a854     asx.obj
 0002:0000287c       ??_C@_0N@JLEJDLAD@asx?4cpp?3978?5?$AA@ 1006a87c     asx.obj
 0002:0000288c       ??_C@_0BD@FMBINJC@ASX_Recorder_Pause?$AA@ 1006a88c     asx.obj
 0002:000028a0       ??_C@_0BF@KCGGJKHH@ASX_Recorder_Pause?$CI?$CJ?$AA@ 1006a8a0     asx.obj
 0002:000028b8       ??_C@_0N@HFIFBNII@asx?4cpp?3990?5?$AA@ 1006a8b8     asx.obj
 0002:000028c8       ??_C@_0CB@GNAPCFNF@?$CIASX_Recorder_Pause?$CJ?5ERROR?5?9?$DO?5?$CFd@ 1006a8c8     asx.obj
 0002:000028ec       ??_C@_0N@HDEONPGD@asx?4cpp?3995?5?$AA@ 1006a8ec     asx.obj
 0002:000028fc       ??_C@_0BD@EHLHIOON@ASX_Recorder_Close?$AA@ 1006a8fc     asx.obj
 0002:00002910       ??_C@_0BF@JDMIOMIC@ASX_Recorder_Close?$CI?$CJ?$AA@ 1006a910     asx.obj
 0002:00002928       ??_C@_0O@IMPOEBBN@asx?4cpp?31004?5?$AA@ 1006a928     asx.obj
 0002:00002938       ??_C@_0CB@LMNBBLJ@?$CIASX_Recorder_Close?$CJ?5ERROR?5?9?$DO?5?$CFd@ 1006a938     asx.obj
 0002:0000295c       ??_C@_0O@IECGNCEO@asx?4cpp?31009?5?$AA@ 1006a95c     asx.obj
 0002:0000296c       ??_C@_0BC@BFFNOLNF@ASX_Recorder_Open?$AA@ 1006a96c     asx.obj
 0002:00002980       ??_C@_0BE@LJIPJHEE@ASX_Recorder_Open?$CI?$CJ?$AA@ 1006a980     asx.obj
 0002:00002994       ??_C@_0O@DNFINPBM@asx?4cpp?31018?5?$AA@ 1006a994     asx.obj
 0002:000029a4       ??_C@_0CA@FAOMGGPC@?$CIASX_Recorder_Open?$CJ?5ERROR?5?9?$DO?5?$CFd?$AA@ 1006a9a4     asx.obj
 0002:000029c4       ??_C@_0O@CDLIJPBD@asx?4cpp?31023?5?$AA@ 1006a9c4     asx.obj
 0002:000029d4       ??_C@_0BN@LCJJJJP@ASX_Recorder_EnumerateFormat?$AA@ 1006a9d4     asx.obj
 0002:000029f4       ??_C@_0BP@NBCDOKP@ASX_Recorder_EnumerateFormat?$CI?$CJ?$AA@ 1006a9f4     asx.obj
 0002:00002a14       ??_C@_0O@JKMGJCEB@asx?4cpp?31032?5?$AA@ 1006aa14     asx.obj
 0002:00002a24       ??_C@_0CL@HNPMCFJ@?$CIASX_Recorder_EnumerateFormat?$CJ?5E@ 1006aa24     asx.obj
 0002:00002a50       ??_C@_0O@JMANFAKK@asx?4cpp?31037?5?$AA@ 1006aa50     asx.obj
 0002:00002a60       ??_C@_0BD@KGDFGOCB@ASX_Recorder_Start?$AA@ 1006aa60     asx.obj
 0002:00002a74       ??_C@_0BF@FEINHHDK@ASX_Recorder_Start?$CI?$CJ?$AA@ 1006aa74     asx.obj
 0002:00002a8c       ??_C@_0O@BIACCE@asx?4cpp?31046?5?$AA@ 1006aa8c     asx.obj
 0002:00002a9c       ??_C@_0CB@DDKIPFAH@?$CIASX_Recorder_Start?$CJ?5ERROR?5?9?$DO?5?$CFd@ 1006aa9c     asx.obj
 0002:00002ac0       ??_C@_0O@LNOLHDME@asx?4cpp?31051?5?$AA@ 1006aac0     asx.obj
 0002:00002ad0       ??_C@_0BC@OGPJLMAI@ASX_Recorder_Stop?$AA@ 1006aad0     asx.obj
 0002:00002ae4       ??_C@_0BE@HIBGBLOF@ASX_Recorder_Stop?$CI?$CJ?$AA@ 1006aae4     asx.obj
 0002:00002af8       ??_C@_0O@KOJMLGBN@asx?4cpp?31060?5?$AA@ 1006aaf8     asx.obj
 0002:00002b08       ??_C@_0CA@EMBMFJDJ@?$CIASX_Recorder_Stop?$CJ?5ERROR?5?9?$DO?5?$CFd?$AA@ 1006ab08     asx.obj
 0002:00002b28       ??_C@_0O@KIFHHEPG@asx?4cpp?31065?5?$AA@ 1006ab28     asx.obj
 0002:00002b38       ??_C@_0BJ@NMDHJGBE@ASX_Recorder_GetPosition?$AA@ 1006ab38     asx.obj
 0002:00002b54       ??_C@_0BL@EFNKLFKA@ASX_Recorder_GetPosition?$CI?$CJ?$AA@ 1006ab54     asx.obj
 0002:00002b70       ??_C@_0O@BBCJHJKE@asx?4cpp?31074?5?$AA@ 1006ab70     asx.obj
 0002:00002b80       ??_C@_0CH@NDLBBGKJ@?$CIASX_Recorder_GetPosition?$CJ?5ERROR@ 1006ab80     asx.obj
 0002:00002ba8       ??_C@_0O@BJPBOKPH@asx?4cpp?31079?5?$AA@ 1006aba8     asx.obj
 0002:00002bb8       ??_C@_0BJ@CMECCCFN@ASX_Recorder_GetFilename?$AA@ 1006abb8     asx.obj
 0002:00002bd4       ??_C@_0BL@KIGNMGAM@ASX_Recorder_GetFilename?$CI?$CJ?$AA@ 1006abd4     asx.obj
 0002:00002bf0       ??_C@_0O@EAFAJAJG@asx?4cpp?31088?5?$AA@ 1006abf0     asx.obj
 0002:00002c00       ??_C@_0CH@BHIJNFJ@?$CIASX_Recorder_GetFilename?$CJ?5ERROR@ 1006ac00     asx.obj
 0002:00002c28       ??_C@_0O@PELJBIBC@asx?4cpp?31093?5?$AA@ 1006ac28     asx.obj
 0002:00002c38       ??_C@_0BG@OEIBCGEB@ASX_Recorder_GetState?$AA@ 1006ac38     asx.obj
 0002:00002c50       ??_C@_0BI@EJHHJHIL@ASX_Recorder_GetState?$CI?$CJ?$AA@ 1006ac50     asx.obj
 0002:00002c68       ??_C@_0O@LFBDBEBP@asx?4cpp?31102?5?$AA@ 1006ac68     asx.obj
 0002:00002c78       ??_C@_0CE@BDEAENCC@?$CIASX_Recorder_GetState?$CJ?5ERROR?5?9?$DO@ 1006ac78     asx.obj
 0002:00002c9c       ??_C@_0O@LDNINGPE@asx?4cpp?31107?5?$AA@ 1006ac9c     asx.obj
 0002:00002cac       ??_C@_0BO@PACJBNE@ASX_CobranetTx_GetUnicastMode?$AA@ 1006acac     asx.obj
 0002:00002ccc       ??_C@_0CA@BAEECEHI@ASX_CobranetTx_GetUnicastMode?$CI?$CJ?$AA@ 1006accc     asx.obj
 0002:00002cec       ??_C@_0O@BPKJMJL@asx?4cpp?31119?5?$AA@ 1006acec     asx.obj
 0002:00002cfc       ??_C@_0CM@IFKFOJEB@?$CIASX_CobranetTx_GetUnicastMode?$CJ?5@ 1006acfc     asx.obj
 0002:00002d28       ??_C@_0O@BLJHKACG@asx?4cpp?31124?5?$AA@ 1006ad28     asx.obj
 0002:00002d38       ??_C@_0BN@DFHALOL@ASX_CobranetTx_GetChannelMap?$AA@ 1006ad38     asx.obj
 0002:00002d58       ??_C@_0BP@FIEAHIEL@ASX_CobranetTx_GetChannelMap?$CI?$CJ?$AA@ 1006ad58     asx.obj
 0002:00002d78       ??_C@_0O@KGGENBMG@asx?4cpp?31133?5?$AA@ 1006ad78     asx.obj
 0002:00002d88       ??_C@_0CL@ECPFPBMJ@?$CIASX_CobranetTx_GetChannelMap?$CJ?5E@ 1006ad88     asx.obj
 0002:00002db4       ??_C@_0O@KKDBDOCH@asx?4cpp?31138?5?$AA@ 1006adb4     asx.obj
 0002:00002dc4       ??_C@_0BO@MBBMGLPI@ASX_CobranetTx_SetUnicastMode?$AA@ 1006adc4     asx.obj
 0002:00002de4       ??_C@_0CA@HEBNJKMK@ASX_CobranetTx_SetUnicastMode?$CI?$CJ?$AA@ 1006ade4     asx.obj
 0002:00002e04       ??_C@_0O@DMLKEBKD@asx?4cpp?31147?5?$AA@ 1006ae04     asx.obj
 0002:00002e14       ??_C@_0CM@JICNMMOF@?$CIASX_CobranetTx_SetUnicastMode?$CJ?5@ 1006ae14     asx.obj
 0002:00002e40       ??_C@_0O@ICMNOECN@asx?4cpp?31152?5?$AA@ 1006ae40     asx.obj
 0002:00002e50       ??_C@_0BP@JBKGIFAD@ASX_CobranetTx_GetChannelCount?$AA@ 1006ae50     asx.obj
 0002:00002e70       ??_C@_0CB@MEOHDNHJ@ASX_CobranetTx_GetChannelCount?$CI?$CJ@ 1006ae70     asx.obj
 0002:00002e94       ??_C@_0O@JCDOPFJK@asx?4cpp?31161?5?$AA@ 1006ae94     asx.obj
 0002:00002ea4       ??_C@_0CN@FOPIKLBE@?$CIASX_CobranetTx_GetChannelCount?$CJ@ 1006aea4     asx.obj
 0002:00002ed4       ??_C@_0O@JHHBODBP@asx?4cpp?31166?5?$AA@ 1006aed4     asx.obj
 0002:00002ee4       ??_C@_0BJ@PNIDGOPN@ASX_CobranetTx_SetBundle?$AA@ 1006aee4     asx.obj
 0002:00002f00       ??_C@_0BL@HJAAKGJP@ASX_CobranetTx_SetBundle?$CI?$CJ?$AA@ 1006af00     asx.obj
 0002:00002f1c       ??_C@_0O@CNILDKCD@asx?4cpp?31175?5?$AA@ 1006af1c     asx.obj
 0002:00002f2c       ??_C@_0CH@PHPBBOAN@?$CIASX_CobranetTx_SetBundle?$CJ?5ERROR@ 1006af2c     asx.obj
 0002:00002f54       ??_C@_0O@HDCDOIJO@asx?4cpp?31180?5?$AA@ 1006af54     asx.obj
 0002:00002f64       ??_C@_0BJ@CIJIOOFJ@ASX_CobranetTx_SetFormat?$AA@ 1006af64     asx.obj
 0002:00002f80       ??_C@_0BL@FONDIJEJ@ASX_CobranetTx_SetFormat?$CI?$CJ?$AA@ 1006af80     asx.obj
 0002:00002f9c       ??_C@_0O@HMPCNDBB@asx?4cpp?31189?5?$AA@ 1006af9c     asx.obj
 0002:00002fac       ??_C@_0CH@HAHEHCBL@?$CIASX_CobranetTx_SetFormat?$CJ?5ERROR@ 1006afac     asx.obj
 0002:00002fd4       ??_C@_0O@MMJGCHCH@asx?4cpp?31194?5?$AA@ 1006afd4     asx.obj
 0002:00002fe4       ??_C@_0BJ@EBFOGNG@ASX_CobranetTx_GetStatus?$AA@ 1006afe4     asx.obj
 0002:00003000       ??_C@_0BL@OMBDKJHC@ASX_CobranetTx_GetStatus?$CI?$CJ?$AA@ 1006b000     asx.obj
 0002:0000301c       ??_C@_0O@PDHBAEPI@asx?4cpp?31203?5?$AA@ 1006b01c     asx.obj
 0002:0000302c       ??_C@_0CH@BIHGGPAB@?$CIASX_CobranetTx_GetStatus?$CJ?5ERROR@ 1006b02c     asx.obj
 0002:00003054       ??_C@_0O@PPCEOLBJ@asx?4cpp?31208?5?$AA@ 1006b054     asx.obj
 0002:00003064       ??_C@_0BJ@NDMGEPGP@ASX_CobranetTx_GetBundle?$AA@ 1006b064     asx.obj
 0002:00003080       ??_C@_0BL@HGBOHABM@ASX_CobranetTx_GetBundle?$CI?$CJ?$AA@ 1006b080     asx.obj
 0002:0000309c       ??_C@_0O@EMMEMLEB@asx?4cpp?31217?5?$AA@ 1006b09c     asx.obj
 0002:000030ac       ??_C@_0CH@PGNPDJNC@?$CIASX_CobranetTx_GetBundle?$CJ?5ERROR@ 1006b0ac     asx.obj
 0002:000030d4       ??_C@_0O@FILKKGEE@asx?4cpp?31222?5?$AA@ 1006b0d4     asx.obj
 0002:000030e4       ??_C@_0BJ@GNNMPML@ASX_CobranetTx_GetFormat?$AA@ 1006b0e4     asx.obj
 0002:00003100       ??_C@_0BL@FBMNFPMK@ASX_CobranetTx_GetFormat?$CI?$CJ?$AA@ 1006b100     asx.obj
 0002:0000311c       ??_C@_0O@OCEAHPHI@asx?4cpp?31231?5?$AA@ 1006b11c     asx.obj
 0002:0000312c       ??_C@_0CH@HBFKFFME@?$CIASX_CobranetTx_GetFormat?$CJ?5ERROR@ 1006b12c     asx.obj
 0002:00003154       ??_C@_0O@OHAPGJPN@asx?4cpp?31236?5?$AA@ 1006b154     asx.obj
 0002:00003164       ??_C@_0BP@KDLAPHBK@ASX_CobranetTx_SetChannelCount?$AA@ 1006b164     asx.obj
 0002:00003184       ??_C@_0CB@OBOMLGGH@ASX_CobranetTx_SetChannelCount?$CI?$CJ@ 1006b184     asx.obj
 0002:000031a8       ??_C@_0O@HIJOOPBN@asx?4cpp?31245?5?$AA@ 1006b1a8     asx.obj
 0002:000031b8       ??_C@_0CN@IPFOEEMA@?$CIASX_CobranetTx_SetChannelCount?$CJ@ 1006b1b8     asx.obj
 0002:000031e8       ??_C@_0O@MGOJEKJD@asx?4cpp?31250?5?$AA@ 1006b1e8     asx.obj
 0002:000031f8       ??_C@_0BN@HMEJLIJM@ASX_CobranetTx_SetChannelMap?$AA@ 1006b1f8     asx.obj
 0002:00003218       ??_C@_0BP@GKFGAKFC@ASX_CobranetTx_SetChannelMap?$CI?$CJ?$AA@ 1006b218     asx.obj
 0002:00003238       ??_C@_0O@MJDIHBBM@asx?4cpp?31259?5?$AA@ 1006b238     asx.obj
 0002:00003248       ??_C@_0CL@HNMADBNJ@?$CIASX_CobranetTx_SetChannelMap?$CJ?5E@ 1006b248     asx.obj
 0002:00003274       ??_C@_0O@NDFFENKB@asx?4cpp?31264?5?$AA@ 1006b274     asx.obj
 0002:00003284       ??_C@_0BB@MNCBHEI@ASX_Node_GetName?$AA@ 1006b284     asx.obj
 0002:00003298       ??_C@_0BD@MJGLMEKL@ASX_Node_GetName?$CI?$CJ?$AA@ 1006b298     asx.obj
 0002:000032ac       ??_C@_0O@GIGNPOKK@asx?4cpp?31276?5?$AA@ 1006b2ac     asx.obj
 0002:000032bc       ??_C@_0BP@MNJDJFNI@?$CIASX_Node_GetName?$CJ?5ERROR?5?9?$DO?5?$CFd?$AA@ 1006b2bc     asx.obj
 0002:000032dc       ??_C@_0O@DFEBPIHJ@asx?4cpp?31281?5?$AA@ 1006b2dc     asx.obj
 0002:000032ec       ??_C@_0BB@KHNBNHDI@ASX_Node_GetType?$AA@ 1006b2ec     asx.obj
 0002:00003300       ??_C@_0BC@HNLAAAKI@ASX_Node_GetIndex?$AA@ 1006b300     asx.obj
 0002:00003314       ??_C@_0BG@FOFHKEOB@ASX_Node_GetSubSystem?$AA@ 1006b314     asx.obj
 0002:0000332c       ??_C@_0BI@OEMGHDLI@ASX_Node_GetSubSystem?$CI?$CJ?$AA@ 1006b32c     asx.obj
 0002:00003344       ??_C@_0O@NNGGOIJB@asx?4cpp?31332?5?$AA@ 1006b344     asx.obj
 0002:00003354       ??_C@_0BF@PPCKBJNM@ASX_Node_GetLocation?$AA@ 1006b354     asx.obj
 0002:0000336c       ??_C@_0BH@DLPOFFEK@ASX_Node_GetLocation?$CI?$CJ?$AA@ 1006b36c     asx.obj
 0002:00003384       ??_C@_0O@EHLIHIPE@asx?4cpp?31346?5?$AA@ 1006b384     asx.obj
 0002:00003394       ??_C@_0CD@DMILMEEM@?$CIASX_Node_GetLocation?$CJ?5ERROR?5?9?$DO?5@ 1006b394     asx.obj
 0002:000033b8       ??_C@_0O@PKELAJBE@asx?4cpp?31351?5?$AA@ 1006b3b8     asx.obj
 0002:000033c8       ??_C@_0BA@PPPEAKAI@ASX_Error_Clear?$AA@ 1006b3c8     asx.obj
 0002:000033d8       ??_C@_0BC@FKBEBEFB@ASX_Error_Clear?$CI?$CJ?$AA@ 1006b3d8     asx.obj
 0002:000033ec       ??_C@_0O@FAECMBJP@asx?4cpp?31371?5?$AA@ 1006b3ec     asx.obj
 0002:000033fc       ??_C@_0BI@HFJEMIMI@ASX_Error_GetLastString?$AA@ 1006b3fc     asx.obj
 0002:00003414       ??_C@_0BK@OEIEOKOD@ASX_Error_GetLastString?$CI?$CJ?$AA@ 1006b414     asx.obj
 0002:00003430       ??_C@_0O@LKFAFKH@asx?4cpp?31383?5?$AA@ 1006b430     asx.obj
 0002:00003440       ??_C@_0BC@JHENHPMK@ASX_Error_GetLast?$AA@ 1006b440     asx.obj
 0002:00003454       ??_C@_0BE@IDLHEMJH@ASX_Error_GetLast?$CI?$CJ?$AA@ 1006b454     asx.obj
 0002:00003468       ??_C@_0O@LDBJGCMC@asx?4cpp?31393?5?$AA@ 1006b468     asx.obj
 0002:00003478       ??_C@_0BK@OANENMHH@ASX_GetGenericControlName?$AA@ 1006b478     asx.obj
 0002:00003494       ??_C@_0BM@JNADBJKJ@ASX_GetGenericControlName?$CI?$CJ?$AA@ 1006b494     asx.obj
 0002:000034b0       ??_C@_0O@HKPKDDLD@asx?4cpp?31406?5?$AA@ 1006b4b0     asx.obj
 0002:000034c0       ??_C@_0BD@FBIKPIMJ@ASX_Volume_SetMute?$AA@ 1006b4c0     asx.obj
 0002:000034d4       ??_C@_0BF@NLEGMPBA@ASX_Volume_SetMute?$CI?$CJ?$AA@ 1006b4d4     asx.obj
 0002:000034ec       ??_C@_0O@NGDIDJND@asx?4cpp?31423?5?$AA@ 1006b4ec     asx.obj
 0002:000034fc       ??_C@_0CB@HKDDODHK@?$CIASX_Volume_SetMute?$CJ?5ERROR?5?9?$DO?5?$CFd@ 1006b4fc     asx.obj
 0002:00003520       ??_C@_0O@NKGNNGDC@asx?4cpp?31428?5?$AA@ 1006b520     asx.obj
 0002:00003530       ??_C@_0BD@KJHLMHBI@ASX_Volume_GetMute?$AA@ 1006b530     asx.obj
 0002:00003544       ??_C@_0BF@PFADOOIC@ASX_Volume_GetMute?$CI?$CJ?$AA@ 1006b544     asx.obj
 0002:0000355c       ??_C@_0O@GJINPGGK@asx?4cpp?31437?5?$AA@ 1006b55c     asx.obj
 0002:0000356c       ??_C@_0CB@CDCOPFCN@?$CIASX_Volume_GetMute?$CJ?5ERROR?5?9?$DO?5?$CFd@ 1006b56c     asx.obj
 0002:00003590       ??_C@_0O@PCJBAMDI@asx?4cpp?31442?5?$AA@ 1006b590     asx.obj
 0002:000035a0       ??_C@_0BE@FAIPJOOK@ASX_Volume_GetRange?$AA@ 1006b5a0     asx.obj
 0002:000035b4       ??_C@_0BG@MBDOHNBJ@ASX_Volume_GetRange?$CI?$CJ?$AA@ 1006b5b4     asx.obj
 0002:000035cc       ??_C@_0O@EIGLNFAE@asx?4cpp?31451?5?$AA@ 1006b5cc     asx.obj
 0002:000035dc       ??_C@_0CC@MFALMPBJ@?$CIASX_Volume_GetRange?$CJ?5ERROR?5?9?$DO?5?$CF@ 1006b5dc     asx.obj
 0002:00003600       ??_C@_0O@ENCEMDIB@asx?4cpp?31456?5?$AA@ 1006b600     asx.obj
 0002:00003610       ??_C@_0BD@DDELMJEI@ASX_Volume_SetGain?$AA@ 1006b610     asx.obj
 0002:00003624       ??_C@_0BF@KIAAAEOB@ASX_Volume_SetGain?$CI?$CJ?$AA@ 1006b624     asx.obj
 0002:0000363c       ??_C@_0O@FNNHNCDG@asx?4cpp?31465?5?$AA@ 1006b63c     asx.obj
 0002:0000364c       ??_C@_0CB@DNHGECHO@?$CIASX_Volume_SetGain?$CJ?5ERROR?5?9?$DO?5?$CFd@ 1006b64c     asx.obj
 0002:00003670       ??_C@_0O@ODKAHHLI@asx?4cpp?31470?5?$AA@ 1006b670     asx.obj
 0002:00003680       ??_C@_0BD@MLLKPGJJ@ASX_Volume_GetGain?$AA@ 1006b680     asx.obj
 0002:00003694       ??_C@_0BF@IGEFCFHD@ASX_Volume_GetGain?$CI?$CJ?$AA@ 1006b694     asx.obj
 0002:000036ac       ??_C@_0O@OMHBEMDH@asx?4cpp?31479?5?$AA@ 1006b6ac     asx.obj
 0002:000036bc       ??_C@_0CB@GEGLFECJ@?$CIASX_Volume_GetGain?$CJ?5ERROR?5?9?$DO?5?$CFd@ 1006b6bc     asx.obj
 0002:000036e0       ??_C@_0O@LMMKMPDC@asx?4cpp?31484?5?$AA@ 1006b6e0     asx.obj
 0002:000036f0       ??_C@_0BH@HNPECOGK@ASX_Volume_GetChannels?$AA@ 1006b6f0     asx.obj
 0002:00003708       ??_C@_0BJ@DBNMHLKF@ASX_Volume_GetChannels?$CI?$CJ?$AA@ 1006b708     asx.obj
 0002:00003724       ??_C@_0O@BDJLONC@asx?4cpp?31493?5?$AA@ 1006b724     asx.obj
 0002:00003734       ??_C@_0CF@KPJENNJI@?$CIASX_Volume_GetChannels?$CJ?5ERROR?5?9@ 1006b734     asx.obj
 0002:0000375c       ??_C@_0O@NGMFBDD@asx?4cpp?31498?5?$AA@ 1006b75c     asx.obj
 0002:0000376c       ??_C@_0BH@OIIBKMKA@ASX_Volume_SetAutofade?$AA@ 1006b76c     asx.obj
 0002:00003784       ??_C@_0BJ@DHPDDBI@ASX_Volume_SetAutofade?$CI?$CJ?$AA@ 1006b784     asx.obj
 0002:000037a0       ??_C@_0O@EGFIHADE@asx?4cpp?31507?5?$AA@ 1006b7a0     asx.obj
 0002:000037b0       ??_C@_0CF@KMCHEDGB@?$CIASX_Volume_SetAutofade?$CJ?5ERROR?5?9@ 1006b7b0     asx.obj
 0002:000037d8       ??_C@_0O@PICPNFLK@asx?4cpp?31512?5?$AA@ 1006b7d8     asx.obj
 0002:000037e8       ??_C@_0BN@DFMEBGBE@ASX_SilenceDetector_GetDelay?$AA@ 1006b7e8     asx.obj
 0002:00003808       ??_C@_0BP@KIGCNPHD@ASX_SilenceDetector_GetDelay?$CI?$CJ?$AA@ 1006b808     asx.obj
 0002:00003828       ??_C@_0O@OOBHAGOG@asx?4cpp?31524?5?$AA@ 1006b828     asx.obj
 0002:00003838       ??_C@_0CL@MILEPEFH@?$CIASX_SilenceDetector_GetDelay?$CJ?5E@ 1006b838     asx.obj
 0002:00003864       ??_C@_0O@OGMPJFLF@asx?4cpp?31529?5?$AA@ 1006b864     asx.obj
 0002:00003874       ??_C@_0CB@CKBEAAMC@ASX_SilenceDetector_SetThreshold@ 1006b874     asx.obj
 0002:00003898       ??_C@_0CD@ILNEBHGL@ASX_SilenceDetector_SetThreshold@ 1006b898     asx.obj
 0002:000038bc       ??_C@_0O@FPLBJIOH@asx?4cpp?31538?5?$AA@ 1006b8bc     asx.obj
 0002:000038cc       ??_C@_0CP@GEAACJMM@?$CIASX_SilenceDetector_SetThreshol@ 1006b8cc     asx.obj
 0002:000038fc       ??_C@_0O@MODDEPLP@asx?4cpp?31543?5?$AA@ 1006b8fc     asx.obj
 0002:0000390c       ??_C@_0BO@DOBNHODK@ASX_SilenceDetector_GetEnable?$AA@ 1006b90c     asx.obj
 0002:0000392c       ??_C@_0CA@OAAMDEOM@ASX_SilenceDetector_GetEnable?$CI?$CJ?$AA@ 1006b92c     asx.obj
 0002:0000394c       ??_C@_0O@HHENECON@asx?4cpp?31552?5?$AA@ 1006b94c     asx.obj
 0002:0000395c       ??_C@_0CM@FBOEFPCK@?$CIASX_SilenceDetector_GetEnable?$CJ?5@ 1006b95c     asx.obj
 0002:00003988       ??_C@_0O@HBIGIAAG@asx?4cpp?31557?5?$AA@ 1006b988     asx.obj
 0002:00003998       ??_C@_0CB@FOKKMMIO@ASX_SilenceDetector_GetThreshold@ 1006b998     asx.obj
 0002:000039bc       ??_C@_0CD@EFMKONEH@ASX_SilenceDetector_GetThreshold@ 1006b9bc     asx.obj
 0002:000039e0       ??_C@_0O@GCPBEFNP@asx?4cpp?31566?5?$AA@ 1006b9e0     asx.obj
 0002:000039f0       ??_C@_0CP@OEMGOEGK@?$CIASX_SilenceDetector_GetThreshol@ 1006b9f0     asx.obj
 0002:00003a20       ??_C@_0O@NPACDEDP@asx?4cpp?31571?5?$AA@ 1006ba20     asx.obj
 0002:00003a30       ??_C@_0BN@MEOIAFGJ@ASX_SilenceDetector_SetDelay?$AA@ 1006ba30     asx.obj
 0002:00003a50       ??_C@_0BP@LGENGIDK@ASX_SilenceDetector_SetDelay?$CI?$CJ?$AA@ 1006ba50     asx.obj
 0002:00003a70       ??_C@_0O@IGKDEOFO@asx?4cpp?31580?5?$AA@ 1006ba70     asx.obj
 0002:00003a80       ??_C@_0CL@DNOCCNBG@?$CIASX_SilenceDetector_SetDelay?$CJ?5E@ 1006ba80     asx.obj
 0002:00003aac       ??_C@_0O@IAGIIMLF@asx?4cpp?31585?5?$AA@ 1006baac     asx.obj
 0002:00003abc       ??_C@_0CD@PAIHJLMN@ASX_SilenceDetector_GetEventEnab@ 1006babc     asx.obj
 0002:00003ae0       ??_C@_0CF@GLJBJLPL@ASX_SilenceDetector_GetEventEnab@ 1006bae0     asx.obj
 0002:00003b08       ??_C@_0O@DJBGIBOH@asx?4cpp?31594?5?$AA@ 1006bb08     asx.obj
 0002:00003b18       ??_C@_0DB@OEMIJEOF@?$CIASX_SilenceDetector_GetEventEna@ 1006bb18     asx.obj
 0002:00003b4c       ??_C@_0O@DBMOBCLE@asx?4cpp?31599?5?$AA@ 1006bb4c     asx.obj
 0002:00003b5c       ??_C@_0CD@DOJJGBOB@ASX_SilenceDetector_SetEventEnab@ 1006bb5c     asx.obj
 0002:00003b80       ??_C@_0CF@PMICFEJ@ASX_SilenceDetector_SetEventEnab@ 1006bb80     asx.obj
 0002:00003ba8       ??_C@_0O@KKEENNJ@asx?4cpp?31608?5?$AA@ 1006bba8     asx.obj
 0002:00003bb8       ??_C@_0DB@PJEALBEB@?$CIASX_SilenceDetector_SetEventEna@ 1006bbb8     asx.obj
 0002:00003bec       ??_C@_0O@LOENMFFN@asx?4cpp?31613?5?$AA@ 1006bbec     asx.obj
 0002:00003bfc       ??_C@_0BN@HIGHHOBO@ASX_SilenceDetector_GetState?$AA@ 1006bbfc     asx.obj
 0002:00003c1c       ??_C@_0BP@BBOEJDDA@ASX_SilenceDetector_GetState?$CI?$CJ?$AA@ 1006bc1c     asx.obj
 0002:00003c3c       ??_C@_0O@KNDKAAIE@asx?4cpp?31622?5?$AA@ 1006bc3c     asx.obj
 0002:00003c4c       ??_C@_0CL@NPGONINO@?$CIASX_SilenceDetector_GetState?$CJ?5E@ 1006bc4c     asx.obj
 0002:00003c78       ??_C@_0O@KLPBMCGP@asx?4cpp?31627?5?$AA@ 1006bc78     asx.obj
 0002:00003c88       ??_C@_0BO@BAFIFPKI@ASX_SilenceDetector_SetEnable?$AA@ 1006bc88     asx.obj
 0002:00003ca8       ??_C@_0CA@OPBCOCGP@ASX_SilenceDetector_SetEnable?$CI?$CJ?$AA@ 1006bca8     asx.obj
 0002:00003cc8       ??_C@_0O@BCIPMPDN@asx?4cpp?31636?5?$AA@ 1006bcc8     asx.obj
 0002:00003cd8       ??_C@_0CM@FAMKHIPF@?$CIASX_SilenceDetector_SetEnable?$CJ?5@ 1006bcd8     asx.obj
 0002:00003d04       ??_C@_0O@IKBHOBAB@asx?4cpp?31641?5?$AA@ 1006bd04     asx.obj
 0002:00003d14       ??_C@_0BM@FHIDJGEB@ASX_Block_Parameter_GetType?$AA@ 1006bd14     asx.obj
 0002:00003d30       ??_C@_0BO@ICBGJHAF@ASX_Block_Parameter_GetType?$CI?$CJ?$AA@ 1006bd30     asx.obj
 0002:00003d50       ??_C@_0O@DBCPFCAK@asx?4cpp?31653?5?$AA@ 1006bd50     asx.obj
 0002:00003d60       ??_C@_0CK@PFALEFDC@?$CIASX_Block_Parameter_GetType?$CJ?5ER@ 1006bd60     asx.obj
 0002:00003d8c       ??_C@_0O@DNHKLNOL@asx?4cpp?31658?5?$AA@ 1006bd8c     asx.obj
 0002:00003d9c       ??_C@_0BM@PMIAFGDB@ASX_Block_Parameter_GetName?$AA@ 1006bd9c     asx.obj
 0002:00003db8       ??_C@_0BO@DGENIHEA@ASX_Block_Parameter_GetName?$CI?$CJ?$AA@ 1006bdb8     asx.obj
 0002:00003dd8       ??_C@_0O@CEJDFFDI@asx?4cpp?31667?5?$AA@ 1006bdd8     asx.obj
 0002:00003de8       ??_C@_0CK@NHABHGIB@?$CIASX_Block_Parameter_GetName?$CJ?5ER@ 1006bde8     asx.obj
 0002:00003e14       ??_C@_0O@JKOEPALG@asx?4cpp?31672?5?$AA@ 1006be14     asx.obj
 0002:00003e24       ??_C@_0BN@CMINKGOO@ASX_Block_Parameter_GetRange?$AA@ 1006be24     asx.obj
 0002:00003e44       ??_C@_0BP@INFAHMIB@ASX_Block_Parameter_GetRange?$CI?$CJ?$AA@ 1006be44     asx.obj
 0002:00003e64       ??_C@_0O@MAMBFOLJ@asx?4cpp?31681?5?$AA@ 1006be64     asx.obj
 0002:00003e74       ??_C@_0CL@OKCFBPEO@?$CIASX_Block_Parameter_GetRange?$CJ?5E@ 1006be74     asx.obj
 0002:00003ea0       ??_C@_0O@MFIOEIDM@asx?4cpp?31686?5?$AA@ 1006bea0     asx.obj
 0002:00003eb0       ??_C@_0BI@MNFKCGOE@ASX_Block_Parameter_Get?$AA@ 1006beb0     asx.obj
 0002:00003ec8       ??_C@_0BK@JKAHPGPM@ASX_Block_Parameter_Get?$CI?$CJ?$AA@ 1006bec8     asx.obj
 0002:00003ee4       ??_C@_0O@HPHEJBAA@asx?4cpp?31695?5?$AA@ 1006bee4     asx.obj
 0002:00003ef4       ??_C@_0CG@DDANLPNJ@?$CIASX_Block_Parameter_Get?$CJ?5ERROR?5@ 1006bef4     asx.obj
 0002:00003f1c       ??_C@_0O@DJNHDFNB@asx?4cpp?31700?5?$AA@ 1006bf1c     asx.obj
 0002:00003f2c       ??_C@_0BN@IKBIHFD@ASX_Block_Parameter_GetFlags?$AA@ 1006bf2c     asx.obj
 0002:00003f4c       ??_C@_0BP@JAFCJIAG@ASX_Block_Parameter_GetFlags?$CI?$CJ?$AA@ 1006bf4c     asx.obj
 0002:00003f6c       ??_C@_0O@DGAGAOFO@asx?4cpp?31709?5?$AA@ 1006bf6c     asx.obj
 0002:00003f7c       ??_C@_0CL@EDLOJOCF@?$CIASX_Block_Parameter_GetFlags?$CJ?5E@ 1006bf7c     asx.obj
 0002:00003fa8       ??_C@_0O@IGGCPKGI@asx?4cpp?31714?5?$AA@ 1006bfa8     asx.obj
 0002:00003fb8       ??_C@_0BC@NMCPJOLA@ASX_Block_GetInfo?$AA@ 1006bfb8     asx.obj
 0002:00003fcc       ??_C@_0BE@IBGKEEGH@ASX_Block_GetInfo?$CI?$CJ?$AA@ 1006bfcc     asx.obj
 0002:00003fe0       ??_C@_0O@JBJIEDAD@asx?4cpp?31723?5?$AA@ 1006bfe0     asx.obj
 0002:00003ff0       ??_C@_0CA@NNDNDHAC@?$CIASX_Block_GetInfo?$CJ?5ERROR?5?9?$DO?5?$CFd?$AA@ 1006bff0     asx.obj
 0002:00004010       ??_C@_0O@JNMNKMOC@asx?4cpp?31728?5?$AA@ 1006c010     asx.obj
 0002:00004020       ??_C@_0BI@BCCBOGCM@ASX_Block_Parameter_Set?$AA@ 1006c020     asx.obj
 0002:00004038       ??_C@_0BK@CEALGHB@ASX_Block_Parameter_Set?$CI?$CJ?$AA@ 1006c038     asx.obj
 0002:00004054       ??_C@_0O@COCNIMLK@asx?4cpp?31737?5?$AA@ 1006c054     asx.obj
 0002:00004064       ??_C@_0CG@FHFEABGL@?$CIASX_Block_Parameter_Set?$CJ?5ERROR?5@ 1006c064     asx.obj
 0002:0000408c       ??_C@_0O@LFDBHGOI@asx?4cpp?31742?5?$AA@ 1006c08c     asx.obj
 0002:0000409c       ??_C@_0BN@CMPHJBMA@ASX_Block_Parameter_GetUnits?$AA@ 1006c09c     asx.obj
 0002:000040bc       ??_C@_0BP@DOOKNANI@ASX_Block_Parameter_GetUnits?$CI?$CJ?$AA@ 1006c0bc     asx.obj
 0002:000040dc       ??_C@_0O@PMLKPNE@asx?4cpp?31751?5?$AA@ 1006c0dc     asx.obj
 0002:000040ec       ??_C@_0CL@NPIBINPH@?$CIASX_Block_Parameter_GetUnits?$CJ?5E@ 1006c0ec     asx.obj
 0002:00004118       ??_C@_0O@KIELJFB@asx?4cpp?31756?5?$AA@ 1006c118     asx.obj
 0002:00004128       ??_C@_0CE@EGIDCJGE@ASX_Block_Parameter_GetElementCo@ 1006c128     asx.obj
 0002:0000414c       ??_C@_0CG@DBDLPIPP@ASX_Block_Parameter_GetElementCo@ 1006c14c     asx.obj
 0002:00004174       ??_C@_0O@BKHHKIOG@asx?4cpp?31765?5?$AA@ 1006c174     asx.obj
 0002:00004184       ??_C@_0DC@NLLMBNPC@?$CIASX_Block_Parameter_GetElementC@ 1006c184     asx.obj
 0002:000041b8       ??_C@_0O@KEAAANGI@asx?4cpp?31770?5?$AA@ 1006c1b8     asx.obj
 0002:000041c8       ??_C@_0CA@HAOFIGNA@ASX_Block_Parameter_GetEnumName?$AA@ 1006c1c8     asx.obj
 0002:000041e8       ??_C@_0CC@PHPLBLFM@ASX_Block_Parameter_GetEnumName?$CI@ 1006c1e8     asx.obj
 0002:0000420c       ??_C@_0O@KLNBDGOH@asx?4cpp?31779?5?$AA@ 1006c20c     asx.obj
 0002:0000421c       ??_C@_0CO@PEIGPBBC@?$CIASX_Block_Parameter_GetEnumName@ 1006c21c     asx.obj
 0002:0000424c       ??_C@_0O@PLGKLFOC@asx?4cpp?31784?5?$AA@ 1006c24c     asx.obj
 0002:0000425c       ??_C@_0CB@MIKFLHLA@ASX_AESEBUReceiver_GetSampleRate@ 1006c25c     asx.obj
 0002:00004280       ??_C@_0CD@MDNIMIIB@ASX_AESEBUReceiver_GetSampleRate@ 1006c280     asx.obj
 0002:000042a4       ??_C@_0O@EAFCAGOJ@asx?4cpp?31796?5?$AA@ 1006c2a4     asx.obj
 0002:000042b4       ??_C@_0CP@BDMMCMGH@?$CIASX_AESEBUReceiver_GetSampleRat@ 1006c2b4     asx.obj
 0002:000042e4       ??_C@_0O@LKEFMIDH@asx?4cpp?31801?5?$AA@ 1006c2e4     asx.obj
 0002:000042f4       ??_C@_0CC@NBAHHHDH@ASX_AESEBUReceiver_GetErrorStatu@ 1006c2f4     asx.obj
 0002:00004318       ??_C@_0CE@CMHOBNBP@ASX_AESEBUReceiver_GetErrorStatu@ 1006c318     asx.obj
 0002:0000433c       ??_C@_0O@DDLMFGF@asx?4cpp?31810?5?$AA@ 1006c33c     asx.obj
 0002:0000434c       ??_C@_0DA@EPEKCCEI@?$CIASX_AESEBUReceiver_GetErrorStat@ 1006c34c     asx.obj
 0002:0000437c       ??_C@_0O@FPAAHIO@asx?4cpp?31815?5?$AA@ 1006c37c     asx.obj
 0002:0000438c       ??_C@_0BN@NMNPFIO@ASX_AESEBUReceiver_GetFormat?$AA@ 1006c38c     asx.obj
 0002:000043ac       ??_C@_0BP@BKMPDGCI@ASX_AESEBUReceiver_GetFormat?$CI?$CJ?$AA@ 1006c3ac     asx.obj
 0002:000043cc       ??_C@_0O@BGIHMCFH@asx?4cpp?31824?5?$AA@ 1006c3cc     asx.obj
 0002:000043dc       ??_C@_0CL@NJOEDMON@?$CIASX_AESEBUReceiver_GetFormat?$CJ?5E@ 1006c3dc     asx.obj
 0002:00004408       ??_C@_0O@BOFPFBAE@asx?4cpp?31829?5?$AA@ 1006c408     asx.obj
 0002:00004418       ??_C@_0CD@IIFBNLIM@ASX_AESEBUReceiver_EnumerateForm@ 1006c418     asx.obj
 0002:0000443c       ??_C@_0CF@PECPNMPJ@ASX_AESEBUReceiver_EnumerateForm@ 1006c43c     asx.obj
 0002:00004464       ??_C@_0O@KHCBFMFG@asx?4cpp?31838?5?$AA@ 1006c464     asx.obj
 0002:00004474       ??_C@_0DB@LGMEIMKP@?$CIASX_AESEBUReceiver_EnumerateFor@ 1006c474     asx.obj
 0002:000044a8       ??_C@_0O@DGKDILAO@asx?4cpp?31843?5?$AA@ 1006c4a8     asx.obj
 0002:000044b8       ??_C@_0BN@CDIINEBM@ASX_AESEBUReceiver_SetFormat?$AA@ 1006c4b8     asx.obj
 0002:000044d8       ??_C@_0BP@BFNBOAKL@ASX_AESEBUReceiver_SetFormat?$CI?$CJ?$AA@ 1006c4d8     asx.obj
 0002:000044f8       ??_C@_0O@IPNNIGFM@asx?4cpp?31852?5?$AA@ 1006c4f8     asx.obj
 0002:00004508       ??_C@_0CL@NIMKBLDC@?$CIASX_AESEBUReceiver_SetFormat?$CJ?5E@ 1006c508     asx.obj
 0002:00004534       ??_C@_0O@IJBGEELH@asx?4cpp?31857?5?$AA@ 1006c534     asx.obj
 0002:00004544       ??_C@_0BE@HBNMBMPJ@ASX_ChannelMode_Set?$AA@ 1006c544     asx.obj
 0002:00004558       ??_C@_0BG@KDGHPPNE@ASX_ChannelMode_Set?$CI?$CJ?$AA@ 1006c558     asx.obj
 0002:00004570       ??_C@_0O@JBDNMGFD@asx?4cpp?31869?5?$AA@ 1006c570     asx.obj
 0002:00004580       ??_C@_0CC@BPJCHLJ@?$CIASX_ChannelMode_Set?$CJ?5ERROR?5?9?$DO?5?$CF@ 1006c580     asx.obj
 0002:000045a4       ??_C@_0O@CBFJDCGF@asx?4cpp?31874?5?$AA@ 1006c5a4     asx.obj
 0002:000045b4       ??_C@_0BE@KOKHNMDB@ASX_ChannelMode_Get?$AA@ 1006c5b4     asx.obj
 0002:000045c8       ??_C@_0BG@DLCALPFJ@ASX_ChannelMode_Get?$CI?$CJ?$AA@ 1006c5c8     asx.obj
 0002:000045e0       ??_C@_0O@HMHFDELG@asx?4cpp?31883?5?$AA@ 1006c5e0     asx.obj
 0002:000045f0       ??_C@_0CC@GFKAJJAL@?$CIASX_ChannelMode_Get?$CJ?5ERROR?5?9?$DO?5?$CF@ 1006c5f0     asx.obj
 0002:00004614       ??_C@_0O@HACANLFH@asx?4cpp?31888?5?$AA@ 1006c614     asx.obj
 0002:00004624       ??_C@_0BK@DDNBJGJD@ASX_ChannelMode_Enumerate?$AA@ 1006c624     asx.obj
 0002:00004640       ??_C@_0BM@DBBIFEMK@ASX_ChannelMode_Enumerate?$CI?$CJ?$AA@ 1006c640     asx.obj
 0002:0000465c       ??_C@_0O@MDMAPLAP@asx?4cpp?31897?5?$AA@ 1006c65c     asx.obj
 0002:0000466c       ??_C@_0CI@EAKOCFBJ@?$CIASX_ChannelMode_Enumerate?$CJ?5ERRO@ 1006c66c     asx.obj
 0002:00004694       ??_C@_0O@IFGDFPNO@asx?4cpp?31902?5?$AA@ 1006c694     asx.obj
 0002:000046a4       ??_C@_0CG@DAACLCJB@ASX_AESEBUTransmitter_EnumerateF@ 1006c6a4     asx.obj
 0002:000046cc       ??_C@_0CI@DPCNNBEK@ASX_AESEBUTransmitter_EnumerateF@ 1006c6cc     asx.obj
 0002:000046f4       ??_C@_0O@DJFCEEAJ@asx?4cpp?31914?5?$AA@ 1006c6f4     asx.obj
 0002:00004704       ??_C@_0DE@CPNEAFFN@?$CIASX_AESEBUTransmitter_Enumerate@ 1006c704     asx.obj
 0002:00004738       ??_C@_0O@DBIKNHFK@asx?4cpp?31919?5?$AA@ 1006c738     asx.obj
 0002:00004748       ??_C@_0CA@OBCEBOHP@ASX_AESEBUTransmitter_SetFormat?$AA@ 1006c748     asx.obj
 0002:00004768       ??_C@_0CC@CALADBMN@ASX_AESEBUTransmitter_SetFormat?$CI@ 1006c768     asx.obj
 0002:0000478c       ??_C@_0O@CCPNBCID@asx?4cpp?31928?5?$AA@ 1006c78c     asx.obj
 0002:0000479c       ??_C@_0CO@OEHPKOEA@?$CIASX_AESEBUTransmitter_SetFormat@ 1006c79c     asx.obj
 0002:000047cc       ??_C@_0O@JGBEJKAH@asx?4cpp?31933?5?$AA@ 1006c7cc     asx.obj
 0002:000047dc       ??_C@_0CA@MPGBDPON@ASX_AESEBUTransmitter_GetFormat?$AA@ 1006c7dc     asx.obj
 0002:000047fc       ??_C@_0CC@CPKOOHEO@ASX_AESEBUTransmitter_GetFormat?$CI@ 1006c7fc     asx.obj
 0002:00004820       ??_C@_0O@KABMIIJ@asx?4cpp?31942?5?$AA@ 1006c820     asx.obj
 0002:00004830       ??_C@_0CO@OFFBIJJP@?$CIASX_AESEBUTransmitter_GetFormat@ 1006c830     asx.obj
 0002:00004860       ??_C@_0O@MMKAKGC@asx?4cpp?31947?5?$AA@ 1006c860     asx.obj
 0002:00004870       ??_C@_0BD@EFGAOEEK@ASX_Level_GetRange?$AA@ 1006c870     asx.obj
 0002:00004884       ??_C@_0BF@NPOJEMDN@ASX_Level_GetRange?$CI?$CJ?$AA@ 1006c884     asx.obj
 0002:0000489c       ??_C@_0O@LOOIEAAN@asx?4cpp?31959?5?$AA@ 1006c89c     asx.obj
 0002:000048ac       ??_C@_0CB@IFFONAGP@?$CIASX_Level_GetRange?$CJ?5ERROR?5?9?$DO?5?$CFd@ 1006c8ac     asx.obj
 0002:000048d0       ??_C@_0O@KEIFHMLA@asx?4cpp?31964?5?$AA@ 1006c8d0     asx.obj
 0002:000048e0       ??_C@_0O@HALJFEAG@ASX_Level_Get?$AA@ 1006c8e0     asx.obj
 0002:000048f0       ??_C@_0BA@EIEEMKGB@ASX_Level_Get?$CI?$CJ?$AA@ 1006c8f0     asx.obj
 0002:00004900       ??_C@_0O@BJHGANFA@asx?4cpp?31973?5?$AA@ 1006c900     asx.obj
 0002:00004910       ??_C@_0BM@OKCBLPFH@?$CIASX_Level_Get?$CJ?5ERROR?5?9?$DO?5?$CFd?$AA@ 1006c910     asx.obj
 0002:0000492c       ??_C@_0O@BFCDOCLB@asx?4cpp?31978?5?$AA@ 1006c92c     asx.obj
 0002:0000493c       ??_C@_0O@KPMCJEMO@ASX_Level_Set?$AA@ 1006c93c     asx.obj
 0002:0000494c       ??_C@_0BA@NAADIKOM@ASX_Level_Set?$CI?$CJ?$AA@ 1006c94c     asx.obj
 0002:0000495c       ??_C@_0O@EGBMLFNK@asx?4cpp?31987?5?$AA@ 1006c95c     asx.obj
 0002:0000496c       ??_C@_0BM@IOHIABOF@?$CIASX_Level_Set?$CJ?5ERROR?5?9?$DO?5?$CFd?$AA@ 1006c96c     asx.obj
 0002:00004988       ??_C@_0O@PIGLBAFE@asx?4cpp?31992?5?$AA@ 1006c988     asx.obj
 0002:00004998       ??_C@_0CA@HBEBCAKK@ASX_Adapter_GetHardwareRevision?$AA@ 1006c998     asx.obj
 0002:000049b8       ??_C@_0CC@BNJOINFJ@ASX_Adapter_GetHardwareRevision?$CI@ 1006c9b8     asx.obj
 0002:000049dc       ??_C@_0O@KGKDDLD@asx?4cpp?32004?5?$AA@ 1006c9dc     asx.obj
 0002:000049ec       ??_C@_0CO@ENIAFILM@?$CIASX_Adapter_GetHardwareRevision@ 1006c9ec     asx.obj
 0002:00004a1c       ??_C@_0O@CLCKAOA@asx?4cpp?32009?5?$AA@ 1006ca1c     asx.obj
 0002:00004a2c       ??_C@_0BM@GJKHPCJH@ASX_Adapter_GetAVDECCSystem?$AA@ 1006ca2c     asx.obj
 0002:00004a48       ??_C@_0BO@BPKLGOPJ@ASX_Adapter_GetAVDECCSystem?$CI?$CJ?$AA@ 1006ca48     asx.obj
 0002:00004a68       ??_C@_0O@LLMMKNLC@asx?4cpp?32018?5?$AA@ 1006ca68     asx.obj
 0002:00004a78       ??_C@_0CK@JHCFJBCA@?$CIASX_Adapter_GetAVDECCSystem?$CJ?5ER@ 1006ca78     asx.obj
 0002:00004aa4       ??_C@_0O@KFCMONLN@asx?4cpp?32023?5?$AA@ 1006caa4     asx.obj
 0002:00004ab4       ??_C@_0BK@DCFGHEBH@ASX_Adapter_EnumerateMode?$AA@ 1006cab4     asx.obj
 0002:00004ad0       ??_C@_0BM@CAPDILFG@ASX_Adapter_EnumerateMode?$CI?$CJ?$AA@ 1006cad0     asx.obj
 0002:00004aec       ??_C@_0O@BMFCOAOP@asx?4cpp?32032?5?$AA@ 1006caec     asx.obj
 0002:00004afc       ??_C@_0CI@DFMLLMMN@?$CIASX_Adapter_EnumerateMode?$CJ?5ERRO@ 1006cafc     asx.obj
 0002:00004b24       ??_C@_0O@BKJJCCAE@asx?4cpp?32037?5?$AA@ 1006cb24     asx.obj
 0002:00004b34       ??_C@_0CA@ONCALIDD@ASX_Adapter_GetFirmwareRevision?$AA@ 1006cb34     asx.obj
 0002:00004b54       ??_C@_0CC@EDMJDLBN@ASX_Adapter_GetFirmwareRevision?$CI@ 1006cb54     asx.obj
 0002:00004b78       ??_C@_0O@IGIMHAIK@asx?4cpp?32046?5?$AA@ 1006cb78     asx.obj
 0002:00004b88       ??_C@_0CO@POGGAEOE@?$CIASX_Adapter_GetFirmwareRevision@ 1006cb88     asx.obj
 0002:00004bb8       ??_C@_0O@DLHPABGK@asx?4cpp?32051?5?$AA@ 1006cbb8     asx.obj
 0002:00004bc8       ??_C@_0BE@BGLOINJA@ASX_Adapter_GetMode?$AA@ 1006cbc8     asx.obj
 0002:00004bdc       ??_C@_0BG@JAFAOLIK@ASX_Adapter_GetMode?$CI?$CJ?$AA@ 1006cbdc     asx.obj
 0002:00004bf4       ??_C@_0O@CIAIMELD@asx?4cpp?32060?5?$AA@ 1006cbf4     asx.obj
 0002:00004c04       ??_C@_0CC@EEGGAJIM@?$CIASX_Adapter_GetMode?$CJ?5ERROR?5?9?$DO?5?$CF@ 1006cc04     asx.obj
 0002:00004c28       ??_C@_0O@COMDAGFI@asx?4cpp?32065?5?$AA@ 1006cc28     asx.obj
 0002:00004c38       ??_C@_0CA@LKANODA@ASX_Adapter_GetAVDECCController?$AA@ 1006cc38     asx.obj
 0002:00004c58       ??_C@_0CC@MMDFEKDD@ASX_Adapter_GetAVDECCController?$CI@ 1006cc58     asx.obj
 0002:00004c7c       ??_C@_0O@JHLNALAK@asx?4cpp?32074?5?$AA@ 1006cc7c     asx.obj
 0002:00004c8c       ??_C@_0CO@MJNOOJGL@?$CIASX_Adapter_GetAVDECCController@ 1006cc8c     asx.obj
 0002:00004cbc       ??_C@_0O@JPGFJIFJ@asx?4cpp?32079?5?$AA@ 1006ccbc     asx.obj
 0002:00004ccc       ??_C@_0BO@GMMMNAOP@ASX_Adapter_EnumerateProperty?$AA@ 1006cccc     asx.obj
 0002:00004cec       ??_C@_0CA@CNCNNJII@ASX_Adapter_EnumerateProperty?$CI?$CJ?$AA@ 1006ccec     asx.obj
 0002:00004d0c       ??_C@_0O@MGMEOCDI@asx?4cpp?32088?5?$AA@ 1006cd0c     asx.obj
 0002:00004d1c       ??_C@_0CM@HNMPIFH@?$CIASX_Adapter_EnumerateProperty?$CJ?5@ 1006cd1c     asx.obj
 0002:00004d48       ??_C@_0O@HCCNGKLM@asx?4cpp?32093?5?$AA@ 1006cd48     asx.obj
 0002:00004d58       ??_C@_0BJ@BEDINFI@ASX_Adapter_ReadProperty?$AA@ 1006cd58     asx.obj
 0002:00004d74       ??_C@_0BL@JDHDKBDB@ASX_Adapter_ReadProperty?$CI?$CJ?$AA@ 1006cd74     asx.obj
 0002:00004d90       ??_C@_0O@DDIHGGLB@asx?4cpp?32102?5?$AA@ 1006cd90     asx.obj
 0002:00004da0       ??_C@_0CH@GNBIFCID@?$CIASX_Adapter_ReadProperty?$CJ?5ERROR@ 1006cda0     asx.obj
 0002:00004dc8       ??_C@_0O@DFEMKEFK@asx?4cpp?32107?5?$AA@ 1006cdc8     asx.obj
 0002:00004dd8       ??_C@_0BG@GAKIODBE@ASX_Adapter_ReadNvMem?$AA@ 1006cdd8     asx.obj
 0002:00004df0       ??_C@_0BI@GFLFIMIM@ASX_Adapter_ReadNvMem?$CI?$CJ?$AA@ 1006cdf0     asx.obj
 0002:00004e08       ??_C@_0O@IMDCKJAI@asx?4cpp?32116?5?$AA@ 1006ce08     asx.obj
 0002:00004e18       ??_C@_0CE@NNNNHOGJ@?$CIASX_Adapter_ReadNvMem?$CJ?5ERROR?5?9?$DO@ 1006ce18     asx.obj
 0002:00004e3c       ??_C@_0O@JLMIBAGD@asx?4cpp?32121?5?$AA@ 1006ce3c     asx.obj
 0002:00004e4c       ??_C@_0BM@KPAPOLNA@ASX_Adapter_CheckSubSystems?$AA@ 1006ce4c     asx.obj
 0002:00004e68       ??_C@_0BO@MEPINJFD@ASX_Adapter_CheckSubSystems?$CI?$CJ?$AA@ 1006ce68     asx.obj
 0002:00004e88       ??_C@_0O@CCLGBNDB@asx?4cpp?32130?5?$AA@ 1006ce88     asx.obj
 0002:00004e98       ??_C@_0CK@PIHFPEFF@?$CIASX_Adapter_CheckSubSystems?$CJ?5ER@ 1006ce98     asx.obj
 0002:00004ec4       ??_C@_0O@CEHNNPNK@asx?4cpp?32135?5?$AA@ 1006cec4     asx.obj
 0002:00004ed4       ??_C@_0BE@OOEPLCEB@ASX_Adapter_SetMode?$AA@ 1006ced4     asx.obj
 0002:00004ee8       ??_C@_0BG@LOBFMKBI@ASX_Adapter_SetMode?$CI?$CJ?$AA@ 1006cee8     asx.obj
 0002:00004f00       ??_C@_0O@LIGIINFE@asx?4cpp?32144?5?$AA@ 1006cf00     asx.obj
 0002:00004f10       ??_C@_0CC@BNHLBPNL@?$CIASX_Adapter_SetMode?$CJ?5ERROR?5?9?$DO?5?$CF@ 1006cf10     asx.obj
 0002:00004f34       ??_C@_0O@LALABOAH@asx?4cpp?32149?5?$AA@ 1006cf34     asx.obj
 0002:00004f44       ??_C@_0BH@CBFIHLMM@ASX_Adapter_WriteNvMem?$AA@ 1006cf44     asx.obj
 0002:00004f5c       ??_C@_0BJ@NCIAJJBN@ASX_Adapter_WriteNvMem?$CI?$CJ?$AA@ 1006cf5c     asx.obj
 0002:00004f78       ??_C@_0O@JMOBDFF@asx?4cpp?32158?5?$AA@ 1006cf78     asx.obj
 0002:00004f88       ??_C@_0CF@OAPCAPPC@?$CIASX_Adapter_WriteNvMem?$CJ?5ERROR?5?9@ 1006cf88     asx.obj
 0002:00004fb0       ??_C@_0O@BHCOFDFK@asx?4cpp?32163?5?$AA@ 1006cfb0     asx.obj
 0002:00004fc0       ??_C@_0BK@IGPMBLJP@ASX_Adapter_WriteProperty?$AA@ 1006cfc0     asx.obj
 0002:00004fdc       ??_C@_0BM@OKEFBHG@ASX_Adapter_WriteProperty?$CI?$CJ?$AA@ 1006cfdc     asx.obj
 0002:00004ff8       ??_C@_0O@KOFAFOAI@asx?4cpp?32172?5?$AA@ 1006cff8     asx.obj
 0002:00005008       ??_C@_0CI@BKLHAEB@?$CIASX_Adapter_WriteProperty?$CJ?5ERRO@ 1006d008     asx.obj
 0002:00005030       ??_C@_0O@KIJLJMOD@asx?4cpp?32177?5?$AA@ 1006d030     asx.obj
 0002:00005040       ??_C@_0BK@IHFBNIMF@ASX_Adapter_GetMacAddress?$AA@ 1006d040     asx.obj
 0002:0000505c       ??_C@_0BM@EMJNHGAP@ASX_Adapter_GetMacAddress?$CI?$CJ?$AA@ 1006d05c     asx.obj
 0002:00005078       ??_C@_0O@PBDKOGIC@asx?4cpp?32186?5?$AA@ 1006d078     asx.obj
 0002:00005088       ??_C@_0CI@MAGPLHIH@?$CIASX_Adapter_GetMacAddress?$CJ?5ERRO@ 1006d088     asx.obj
 0002:000050b0       ??_C@_0O@EMMJJHGC@asx?4cpp?32191?5?$AA@ 1006d0b0     asx.obj
 0002:000050c0       ??_C@_0BF@HIJPCLDK@ASX_Adapter_GetMixer?$AA@ 1006d0c0     asx.obj
 0002:000050d8       ??_C@_0BH@PLANNHBF@ASX_Adapter_GetMixer?$CI?$CJ?$AA@ 1006d0d8     asx.obj
 0002:000050f0       ??_C@_0O@HHKDMIAP@asx?4cpp?32200?5?$AA@ 1006d0f0     asx.obj
 0002:00005100       ??_C@_0CD@OAOAIMPK@?$CIASX_Adapter_GetMixer?$CJ?5ERROR?5?9?$DO?5@ 1006d100     asx.obj
 0002:00005124       ??_C@_0O@HBGIAKOE@asx?4cpp?32205?5?$AA@ 1006d124     asx.obj
 0002:00005134       ??_C@_0BJ@DODEGAIJ@ASX_Adapter_GetIpAddress?$AA@ 1006d134     asx.obj
 0002:00005150       ??_C@_0BL@NFOLPENN@ASX_Adapter_GetIpAddress?$CI?$CJ?$AA@ 1006d150     asx.obj
 0002:0000516c       ??_C@_0O@MIBGAHLG@asx?4cpp?32214?5?$AA@ 1006d16c     asx.obj
 0002:0000517c       ??_C@_0CH@IBLFAFKD@?$CIASX_Adapter_GetIpAddress?$CJ?5ERROR@ 1006d17c     asx.obj
 0002:000051a4       ??_C@_0O@MAMOJEOF@asx?4cpp?32219?5?$AA@ 1006d1a4     asx.obj
 0002:000051b4       ??_C@_0BF@LBAOLFJB@ASX_Adapter_GetIndex?$AA@ 1006d1b4     asx.obj
 0002:000051cc       ??_C@_0BH@KBEJMFOF@ASX_Adapter_GetIndex?$CI?$CJ?$AA@ 1006d1cc     asx.obj
 0002:000051e4       ??_C@_0O@NDLJFBDM@asx?4cpp?32228?5?$AA@ 1006d1e4     asx.obj
 0002:000051f4       ??_C@_0CD@NOAAHEG@?$CIASX_Adapter_GetIndex?$CJ?5ERROR?5?9?$DO?5@ 1006d1f4     asx.obj
 0002:00005218       ??_C@_0O@GHFANJLI@asx?4cpp?32233?5?$AA@ 1006d218     asx.obj
 0002:00005228       ??_C@_0CA@CCFIKAIJ@ASX_Adapter_GetNvMemSizeInBytes?$AA@ 1006d228     asx.obj
 0002:00005248       ??_C@_0CC@EOIPCKAB@ASX_Adapter_GetNvMemSizeInBytes?$CI@ 1006d248     asx.obj
 0002:0000526c       ??_C@_0O@PLEFILDG@asx?4cpp?32242?5?$AA@ 1006d26c     asx.obj
 0002:0000527c       ??_C@_0BM@NBJHKPGH@ASX_Adapter_GetSerialNumber?$AA@ 1006d27c     asx.obj
 0002:00005298       ??_C@_0BO@BOMNBKDN@ASX_Adapter_GetSerialNumber?$CI?$CJ?$AA@ 1006d298     asx.obj
 0002:000052b8       ??_C@_0O@EEPAEEIP@asx?4cpp?32256?5?$AA@ 1006d2b8     asx.obj
 0002:000052c8       ??_C@_0BE@LOBALLPM@ASX_Adapter_GetName?$AA@ 1006d2c8     asx.obj
 0002:000052dc       ??_C@_0BG@JGKCPCBG@ASX_Adapter_GetName?$CI?$CJ?$AA@ 1006d2dc     asx.obj
 0002:000052f4       ??_C@_0O@OKHEPALG@asx?4cpp?32270?5?$AA@ 1006d2f4     asx.obj
 0002:00005304       ??_C@_0CC@DCLPCCKG@?$CIASX_Adapter_GetName?$CJ?5ERROR?5?9?$DO?5?$CF@ 1006d304     asx.obj
 0002:00005328       ??_C@_0O@OMLPDCFN@asx?4cpp?32275?5?$AA@ 1006d328     asx.obj
 0002:00005338       ??_C@_0BO@KEKCOCDF@ASX_Adapter_GetDspUtilization?$AA@ 1006d338     asx.obj
 0002:00005358       ??_C@_0CA@JOCNGNPD@ASX_Adapter_GetDspUtilization?$CI?$CJ?$AA@ 1006d358     asx.obj
 0002:00005378       ??_C@_0O@LFBOEIDM@asx?4cpp?32284?5?$AA@ 1006d378     asx.obj
 0002:00005388       ??_C@_0CM@FLLNHOH@?$CIASX_Adapter_GetDspUtilization?$CJ?5@ 1006d388     asx.obj
 0002:000053b4       ??_C@_0O@LNMGNLGP@asx?4cpp?32289?5?$AA@ 1006d3b4     asx.obj
 0002:000053c4       ??_C@_0CM@JBLFPHOO@ASX_Mixer_GetBlockControlByNodeT@ 1006d3c4     asx.obj
 0002:000053f0       ??_C@_0CO@JBDMKANL@ASX_Mixer_GetBlockControlByNodeT@ 1006d3f0     asx.obj
 0002:00005420       ??_C@_0O@ELABILII@asx?4cpp?32301?5?$AA@ 1006d420     asx.obj
 0002:00005430       ??_C@_0DK@KMPKHMDG@?$CIASX_Mixer_GetBlockControlByNode@ 1006d430     asx.obj
 0002:0000546c       ??_C@_0O@EOEOJNAN@asx?4cpp?32306?5?$AA@ 1006d46c     asx.obj
 0002:0000547c       ??_C@_0BL@CGPMCNPA@ASX_Mixer_GetControlByNode?$AA@ 1006d47c     asx.obj
 0002:00005498       ??_C@_0BN@CDHLBDIH@ASX_Mixer_GetControlByNode?$CI?$CJ?$AA@ 1006d498     asx.obj
 0002:000054b8       ??_C@_0O@PELEEEDB@asx?4cpp?32315?5?$AA@ 1006d4b8     asx.obj
 0002:000054c8       ??_C@_0CJ@EEENPOOL@?$CIASX_Mixer_GetControlByNode?$CJ?5ERR@ 1006d4c8     asx.obj
 0002:000054f4       ??_C@_0O@OAMKCJDE@asx?4cpp?32320?5?$AA@ 1006d4f4     asx.obj
 0002:00005504       ??_C@_0BI@BFJJJBCA@ASX_Mixer_ResetControls?$AA@ 1006d504     asx.obj
 0002:0000551c       ??_C@_0BK@GAJEBKFK@ASX_Mixer_ResetControls?$CI?$CJ?$AA@ 1006d51c     asx.obj
 0002:00005538       ??_C@_0O@OPBLBCLL@asx?4cpp?32329?5?$AA@ 1006d538     asx.obj
 0002:00005548       ??_C@_0CG@JKKIFEFE@?$CIASX_Mixer_ResetControls?$CJ?5ERROR?5@ 1006d548     asx.obj
 0002:00005570       ??_C@_0O@FPHPOGIN@asx?4cpp?32334?5?$AA@ 1006d570     asx.obj
 0002:00005580       ??_C@_0BI@PJBDENFK@ASX_Mixer_GetSourceNode?$AA@ 1006d580     asx.obj
 0002:00005598       ??_C@_0BK@DKCBPJFD@ASX_Mixer_GetSourceNode?$CI?$CJ?$AA@ 1006d598     asx.obj
 0002:000055b4       ??_C@_0O@MHOHMILB@asx?4cpp?32343?5?$AA@ 1006d5b4     asx.obj
 0002:000055c4       ??_C@_0CG@PLCFLGHP@?$CIASX_Mixer_GetSourceNode?$CJ?5ERROR?5@ 1006d5c4     asx.obj
 0002:000055ec       ??_C@_0O@MLLCCHFA@asx?4cpp?32348?5?$AA@ 1006d5ec     asx.obj
 0002:000055fc       ??_C@_0BN@GDLJANMD@ASX_Mixer_GetDestinationNode?$AA@ 1006d5fc     asx.obj
 0002:0000561c       ??_C@_0BP@OMHOBDDK@ASX_Mixer_GetDestinationNode?$CI?$CJ?$AA@ 1006d61c     asx.obj
 0002:0000563c       ??_C@_0O@HIFCAHAI@asx?4cpp?32357?5?$AA@ 1006d63c     asx.obj
 0002:0000564c       ??_C@_0CL@OABBEAGA@?$CIASX_Mixer_GetDestinationNode?$CJ?5E@ 1006d64c     asx.obj
 0002:00005678       ??_C@_0O@GMCMGKAN@asx?4cpp?32362?5?$AA@ 1006d678     asx.obj
 0002:00005688       ??_C@_0BF@KOIEAODA@ASX_Mixer_GetControl?$AA@ 1006d688     asx.obj
 0002:000056a0       ??_C@_0BH@EKOGDNMD@ASX_Mixer_GetControl?$CI?$CJ?$AA@ 1006d6a0     asx.obj
 0002:000056b8       ??_C@_0O@NGNGLDDB@asx?4cpp?32371?5?$AA@ 1006d6b8     asx.obj
 0002:000056c8       ??_C@_0CD@IFPFPKLF@?$CIASX_Mixer_GetControl?$CJ?5ERROR?5?9?$DO?5@ 1006d6c8     asx.obj
 0002:000056ec       ??_C@_0O@NDJJKFLE@asx?4cpp?32376?5?$AA@ 1006d6ec     asx.obj
 0002:000056fc       ??_C@_0CH@CLLIAFGN@ASX_Mixer_GetControlByNodeTypeAn@ 1006d6fc     asx.obj
 0002:00005724       ??_C@_0CJ@NCCBECGO@ASX_Mixer_GetControlByNodeTypeAn@ 1006d724     asx.obj
 0002:00005750       ??_C@_0O@IJLMALLL@asx?4cpp?32385?5?$AA@ 1006d750     asx.obj
 0002:00005760       ??_C@_0DF@MLOJMKPJ@?$CIASX_Mixer_GetControlByNodeTypeA@ 1006d760     asx.obj
 0002:00005798       ??_C@_0O@DHMLKODF@asx?4cpp?32390?5?$AA@ 1006d798     asx.obj
 0002:000057a8       ??_C@_0CC@BPNFCFAF@ASX_Mixer_GetDestinationNodeCoun@ 1006d7a8     asx.obj
 0002:000057cc       ??_C@_0CE@EEGLLHGE@ASX_Mixer_GetDestinationNodeCoun@ 1006d7cc     asx.obj
 0002:000057f0       ??_C@_0O@DIBKJFLK@asx?4cpp?32399?5?$AA@ 1006d7f0     asx.obj
 0002:00005800       ??_C@_0DA@MJGKNBNH@?$CIASX_Mixer_GetDestinationNodeCou@ 1006d800     asx.obj
 0002:00005830       ??_C@_0O@PPOKJFHD@asx?4cpp?32404?5?$AA@ 1006d830     asx.obj
 0002:00005840       ??_C@_0BN@HJGICHP@ASX_Mixer_GetSourceNodeCount?$AA@ 1006d840     asx.obj
 0002:00005860       ??_C@_0BP@NJAJAIBA@ASX_Mixer_GetSourceNodeCount?$CI?$CJ?$AA@ 1006d860     asx.obj
 0002:00005880       ??_C@_0O@ECBJOEJD@asx?4cpp?32413?5?$AA@ 1006d880     asx.obj
 0002:00005890       ??_C@_0CL@CIDBOCJ@?$CIASX_Mixer_GetSourceNodeCount?$CJ?5E@ 1006d890     asx.obj
 0002:000058bc       ??_C@_0O@EOEMALHC@asx?4cpp?32418?5?$AA@ 1006d8bc     asx.obj
 0002:000058cc       ??_C@_0BL@JAHEPGJJ@ASX_Mixer_GetNodeTypeCount?$AA@ 1006d8cc     asx.obj
 0002:000058e8       ??_C@_0BN@IGEFHOLN@ASX_Mixer_GetNodeTypeCount?$CI?$CJ?$AA@ 1006d8e8     asx.obj
 0002:00005908       ??_C@_0O@FHKFODKB@asx?4cpp?32427?5?$AA@ 1006d908     asx.obj
 0002:00005918       ??_C@_0CJ@KOMPJABL@?$CIASX_Mixer_GetNodeTypeCount?$CJ?5ERR@ 1006d918     asx.obj
 0002:00005944       ??_C@_0O@OJNCEGCP@asx?4cpp?32432?5?$AA@ 1006d944     asx.obj
 0002:00005954       ??_C@_0BK@FABDHPKG@ASX_Mixer_GetControlCount?$AA@ 1006d954     asx.obj
 0002:00005970       ??_C@_0BM@EKPPKPGC@ASX_Mixer_GetControlCount?$CI?$CJ?$AA@ 1006d970     asx.obj
 0002:0000598c       ??_C@_0O@HGEDMAMP@asx?4cpp?32441?5?$AA@ 1006d98c     asx.obj
 0002:0000599c       ??_C@_0CI@EMNBGIJO@?$CIASX_Mixer_GetControlCount?$CJ?5ERRO@ 1006d99c     asx.obj
 0002:000059c4       ??_C@_0O@HDAMNGEK@asx?4cpp?32446?5?$AA@ 1006d9c4     asx.obj
 0002:000059d4       ??_C@_0BI@IGHNGJC@ASX_Mixer_GetNodeByType?$AA@ 1006d9d4     asx.obj
 0002:000059ec       ??_C@_0BK@FONPBPKN@ASX_Mixer_GetNodeByType?$CI?$CJ?$AA@ 1006d9ec     asx.obj
 0002:00005a08       ??_C@_0O@MJPGAPHG@asx?4cpp?32455?5?$AA@ 1006da08     asx.obj
 0002:00005a18       ??_C@_0CG@BAPJDBGK@?$CIASX_Mixer_GetNodeByType?$CJ?5ERROR?5@ 1006da18     asx.obj
 0002:00005a40       ??_C@_0O@NNIIGCHD@asx?4cpp?32460?5?$AA@ 1006da40     asx.obj
 0002:00005a50       ??_C@_0BE@IMFKBHKO@ASX_Multiplexer_Set?$AA@ 1006da50     asx.obj
 0002:00005a64       ??_C@_0BG@MBEPBAEJ@ASX_Multiplexer_Set?$CI?$CJ?$AA@ 1006da64     asx.obj
 0002:00005a7c       ??_C@_0O@GGLANBHI@asx?4cpp?32472?5?$AA@ 1006da7c     asx.obj
 0002:00005a8c       ??_C@_0CC@HOHEEKGL@?$CIASX_Multiplexer_Set?$CJ?5ERROR?5?9?$DO?5?$CF@ 1006da8c     asx.obj
 0002:00005ab0       ??_C@_0O@GAHLBDJD@asx?4cpp?32477?5?$AA@ 1006dab0     asx.obj
 0002:00005ac0       ??_C@_0BE@FDCBNHGG@ASX_Multiplexer_Get?$AA@ 1006dac0     asx.obj
 0002:00005ad4       ??_C@_0BG@FJAIFAME@ASX_Multiplexer_Get?$CI?$CJ?$AA@ 1006dad4     asx.obj
 0002:00005aec       ??_C@_0O@DJNKGJPC@asx?4cpp?32486?5?$AA@ 1006daec     asx.obj
 0002:00005afc       ??_C@_0CC@BKCNPENJ@?$CIASX_Multiplexer_Get?$CJ?5ERROR?5?9?$DO?5?$CF@ 1006dafc     asx.obj
 0002:00005b20       ??_C@_0O@IECJBIBC@asx?4cpp?32491?5?$AA@ 1006db20     asx.obj
 0002:00005b30       ??_C@_0BK@CAKEJGKJ@ASX_Multiplexer_Enumerate?$AA@ 1006db30     asx.obj
 0002:00005b4c       ??_C@_0BM@BELBJJMG@ASX_Multiplexer_Enumerate?$CI?$CJ?$AA@ 1006db4c     asx.obj
 0002:00005b68       ??_C@_0O@MFIDBEBP@asx?4cpp?32500?5?$AA@ 1006db68     asx.obj
 0002:00005b78       ??_C@_0CI@DOGEGKEK@?$CIASX_Multiplexer_Enumerate?$CJ?5ERRO@ 1006db78     asx.obj
 0002:00005ba0       ??_C@_0O@MDEINGPE@asx?4cpp?32505?5?$AA@ 1006dba0     asx.obj
 0002:00005bb0       ??_C@_0BO@GBJBJFBP@ASX_ToneDetector_SetThreshold?$AA@ 1006dbb0     asx.obj
 0002:00005bd0       ??_C@_0CA@DPCHIAHH@ASX_ToneDetector_SetThreshold?$CI?$CJ?$AA@ 1006dbd0     asx.obj
 0002:00005bf0       ??_C@_0O@HIHAGFPP@asx?4cpp?32517?5?$AA@ 1006dbf0     asx.obj
 0002:00005c00       ??_C@_0CM@PDFGHKLH@?$CIASX_ToneDetector_SetThreshold?$CJ?5@ 1006dc00     asx.obj
 0002:00005c2c       ??_C@_0O@GMAOAIPK@asx?4cpp?32522?5?$AA@ 1006dc2c     asx.obj
 0002:00005c3c       ??_C@_0CA@IKGKPGPN@ASX_ToneDetector_SetEventEnable?$AA@ 1006dc3c     asx.obj
 0002:00005c5c       ??_C@_0CC@IHNEMKAA@ASX_ToneDetector_SetEventEnable?$CI@ 1006dc5c     asx.obj
 0002:00005c80       ??_C@_0O@NGPENBMG@asx?4cpp?32531?5?$AA@ 1006dc80     asx.obj
 0002:00005c90       ??_C@_0CO@MHOJIGGE@?$CIASX_ToneDetector_SetEventEnable@ 1006dc90     asx.obj
 0002:00005cc0       ??_C@_0O@NDLLMHED@asx?4cpp?32536?5?$AA@ 1006dcc0     asx.obj
 0002:00005cd0       ??_C@_0BL@JDNKPLHB@ASX_ToneDetector_SetEnable?$AA@ 1006dcd0     asx.obj
 0002:00005cec       ??_C@_0BN@GOFDHIEK@ASX_ToneDetector_SetEnable?$CI?$CJ?$AA@ 1006dcec     asx.obj
 0002:00005d0c       ??_C@_0O@EMCKEBKD@asx?4cpp?32545?5?$AA@ 1006dd0c     asx.obj
 0002:00005d1c       ??_C@_0CJ@IMMGJHJM@?$CIASX_ToneDetector_SetEnable?$CJ?5ERR@ 1006dd1c     asx.obj
 0002:00005d48       ??_C@_0O@PCFNOECN@asx?4cpp?32550?5?$AA@ 1006dd48     asx.obj
 0002:00005d58       ??_C@_0BO@IIDACLGO@ASX_ToneDetector_GetFrequency?$AA@ 1006dd58     asx.obj
 0002:00005d78       ??_C@_0CA@CFNKLPOK@ASX_ToneDetector_GetFrequency?$CI?$CJ?$AA@ 1006dd78     asx.obj
 0002:00005d98       ??_C@_0O@PNIMNPKC@asx?4cpp?32559?5?$AA@ 1006dd98     asx.obj
 0002:00005da8       ??_C@_0CM@PCOPBGHP@?$CIASX_ToneDetector_GetFrequency?$CJ?5@ 1006dda8     asx.obj
 0002:00005dd4       ??_C@_0O@OHOBODBP@asx?4cpp?32564?5?$AA@ 1006ddd4     asx.obj
 0002:00005de4       ??_C@_0BO@BFCPFJFD@ASX_ToneDetector_GetThreshold?$AA@ 1006dde4     asx.obj
 0002:00005e04       ??_C@_0CA@PBDJHKFL@ASX_ToneDetector_GetThreshold?$CI?$CJ?$AA@ 1006de04     asx.obj
 0002:00005e24       ??_C@_0O@FKBCJCPP@asx?4cpp?32573?5?$AA@ 1006de24     asx.obj
 0002:00005e34       ??_C@_0CM@HDJALHBB@?$CIASX_ToneDetector_GetThreshold?$CJ?5@ 1006de34     asx.obj
 0002:00005e60       ??_C@_0O@FGEHHNBO@asx?4cpp?32578?5?$AA@ 1006de60     asx.obj
 0002:00005e70       ??_C@_0BK@CJEGGAAJ@ASX_ToneDetector_GetState?$AA@ 1006de70     asx.obj
 0002:00005e8c       ??_C@_0BM@OOGIHLOE@ASX_ToneDetector_GetState?$CI?$CJ?$AA@ 1006de8c     asx.obj
 0002:00005ea8       ??_C@_0O@FHICKHF@asx?4cpp?32587?5?$AA@ 1006dea8     asx.obj
 0002:00005eb8       ??_C@_0CI@FIMHOPA@?$CIASX_ToneDetector_GetState?$CJ?5ERRO@ 1006deb8     asx.obj
 0002:00005ee0       ??_C@_0O@LLAPIPPL@asx?4cpp?32592?5?$AA@ 1006dee0     asx.obj
 0002:00005ef0       ??_C@_0BL@LNJPNKOD@ASX_ToneDetector_GetEnable?$AA@ 1006def0     asx.obj
 0002:00005f0c       ??_C@_0BN@GBENKOMJ@ASX_ToneDetector_GetEnable?$CI?$CJ?$AA@ 1006df0c     asx.obj
 0002:00005f2c       ??_C@_0O@IDOBAEPI@asx?4cpp?32601?5?$AA@ 1006df2c     asx.obj
 0002:00005f3c       ??_C@_0CJ@INOILAED@?$CIASX_ToneDetector_GetEnable?$CJ?5ERR@ 1006df3c     asx.obj
 0002:00005f68       ??_C@_0O@IGKOBCHN@asx?4cpp?32606?5?$AA@ 1006df68     asx.obj
 0002:00005f78       ??_C@_0CA@EEHEAMNB@ASX_ToneDetector_GetEventEnable?$AA@ 1006df78     asx.obj
 0002:00005f98       ??_C@_0CC@ODINHELC@ASX_ToneDetector_GetEventEnable?$CI@ 1006df98     asx.obj
 0002:00005fbc       ??_C@_0O@DMFEMLEB@asx?4cpp?32615?5?$AA@ 1006dfbc     asx.obj
 0002:00005fcc       ??_C@_0CO@NKGBKDMA@?$CIASX_ToneDetector_GetEventEnable@ 1006dfcc     asx.obj
 0002:00005ffc       ??_C@_0O@CICKKGEE@asx?4cpp?32620?5?$AA@ 1006dffc     asx.obj
 0002:0000600c       ??_C@_0BJ@KEPADJAL@ASX_CobranetRx_GetStatus?$AA@ 1006e00c     asx.obj
 0002:00006028       ??_C@_0BL@MOOJHNIA@ASX_CobranetRx_GetStatus?$CI?$CJ?$AA@ 1006e028     asx.obj
 0002:00006044       ??_C@_0O@JDBCBFEP@asx?4cpp?32632?5?$AA@ 1006e044     asx.obj
 0002:00006054       ??_C@_0CH@CHKILCLA@?$CIASX_CobranetRx_GetStatus?$CJ?5ERROR@ 1006e054     asx.obj
 0002:0000607c       ??_C@_0O@JFNJNHKE@asx?4cpp?32637?5?$AA@ 1006e07c     asx.obj
 0002:0000608c       ??_C@_0BP@DLAKCOFG@ASX_CobranetRx_GetMinimumDelay?$AA@ 1006e08c     asx.obj
 0002:000060ac       ??_C@_0CB@ECCPEEKE@ASX_CobranetRx_GetMinimumDelay?$CI?$CJ@ 1006e0ac     asx.obj
 0002:000060d0       ??_C@_0O@JMMIFCK@asx?4cpp?32646?5?$AA@ 1006e0d0     asx.obj
 0002:000060e0       ??_C@_0CN@GCEINPH@?$CIASX_CobranetRx_GetMinimumDelay?$CJ@ 1006e0e0     asx.obj
 0002:00006110       ??_C@_0O@LEDPPEMK@asx?4cpp?32651?5?$AA@ 1006e110     asx.obj
 0002:00006120       ??_C@_0BM@PDIFLONB@ASX_CobranetRx_GetSourceMAC?$AA@ 1006e120     asx.obj
 0002:0000613c       ??_C@_0BO@MGOCBBOD@ASX_CobranetRx_GetSourceMAC?$CI?$CJ?$AA@ 1006e13c     asx.obj
 0002:0000615c       ??_C@_0O@KHEIDBBD@asx?4cpp?32660?5?$AA@ 1006e15c     asx.obj
 0002:0000616c       ??_C@_0CK@LHFNALBB@?$CIASX_CobranetRx_GetSourceMAC?$CJ?5ER@ 1006e16c     asx.obj
 0002:00006198       ??_C@_0O@KBIDPDPI@asx?4cpp?32665?5?$AA@ 1006e198     asx.obj
 0002:000061a8       ??_C@_0BM@IHDLHCJN@ASX_CobranetRx_SetSourceMAC?$AA@ 1006e1a8     asx.obj
 0002:000061c4       ??_C@_0BO@IPMOLMP@ASX_CobranetRx_SetSourceMAC?$CI?$CJ?$AA@ 1006e1c4     asx.obj
 0002:000061e4       ??_C@_0O@BIPNPOKK@asx?4cpp?32674?5?$AA@ 1006e1e4     asx.obj
 0002:000061f4       ??_C@_0CK@DHJLMGLH@?$CIASX_CobranetRx_SetSourceMAC?$CJ?5ER@ 1006e1f4     asx.obj
 0002:00006220       ??_C@_0O@BACFGNPJ@asx?4cpp?32679?5?$AA@ 1006e220     asx.obj
 0002:00006230       ??_C@_0BN@NLHNAPJE@ASX_CobranetRx_SetChannelMap?$AA@ 1006e230     asx.obj
 0002:00006250       ??_C@_0BP@PHIKABEB@ASX_CobranetRx_SetChannelMap?$CI?$CJ?$AA@ 1006e250     asx.obj
 0002:00006270       ??_C@_0O@EJIEBHJI@asx?4cpp?32688?5?$AA@ 1006e270     asx.obj
 0002:00006280       ??_C@_0CL@PEICHLOJ@?$CIASX_CobranetRx_SetChannelMap?$CJ?5E@ 1006e280     asx.obj
 0002:000062ac       ??_C@_0O@PNGNJPBM@asx?4cpp?32693?5?$AA@ 1006e2ac     asx.obj
 0002:000062bc       ??_C@_0BP@JBMFMEP@ASX_CobranetRx_SetMinimumDelay?$AA@ 1006e2bc     asx.obj
 0002:000062dc       ??_C@_0CB@GHCEMPLK@ASX_CobranetRx_SetMinimumDelay?$CI?$CJ@ 1006e2dc     asx.obj
 0002:00006300       ??_C@_0O@LMMHJDBB@asx?4cpp?32702?5?$AA@ 1006e300     asx.obj
 0002:00006310       ??_C@_0CN@NHICGCCD@?$CIASX_CobranetRx_SetMinimumDelay?$CJ@ 1006e310     asx.obj
 0002:00006340       ??_C@_0O@LKAMFBPK@asx?4cpp?32707?5?$AA@ 1006e340     asx.obj
 0002:00006350       ??_C@_0BN@KEGDLMOD@ASX_CobranetRx_GetChannelMap?$AA@ 1006e350     asx.obj
 0002:00006370       ??_C@_0BP@MFJMHDFI@ASX_CobranetRx_GetChannelMap?$CI?$CJ?$AA@ 1006e370     asx.obj
 0002:00006390       ??_C@_0O@DHCFMKI@asx?4cpp?32716?5?$AA@ 1006e390     asx.obj
 0002:000063a0       ??_C@_0CL@MLLHLLPJ@?$CIASX_CobranetRx_GetChannelMap?$CJ?5E@ 1006e3a0     asx.obj
 0002:000063cc       ??_C@_0O@BEIIOFMD@asx?4cpp?32721?5?$AA@ 1006e3cc     asx.obj
 0002:000063dc       ??_C@_0BJ@HDCDJALC@ASX_CobranetRx_GetBundle?$AA@ 1006e3dc     asx.obj
 0002:000063f8       ??_C@_0BL@FEOEKEOO@ASX_CobranetRx_GetBundle?$CI?$CJ?$AA@ 1006e3f8     asx.obj
 0002:00006414       ??_C@_0O@KNPGOIJB@asx?4cpp?32730?5?$AA@ 1006e414     asx.obj
 0002:00006424       ??_C@_0CH@MJABOEGD@?$CIASX_CobranetRx_GetBundle?$CJ?5ERROR@ 1006e424     asx.obj
 0002:0000644c       ??_C@_0O@KLDNCKHK@asx?4cpp?32735?5?$AA@ 1006e44c     asx.obj
 0002:0000645c       ??_C@_0BJ@FNGGLBCA@ASX_CobranetRx_SetBundle?$AA@ 1006e45c     asx.obj
 0002:00006478       ??_C@_0BL@FLPKHCGN@ASX_CobranetRx_SetBundle?$CI?$CJ?$AA@ 1006e478     asx.obj
 0002:00006494       ??_C@_0O@DHCIHIPE@asx?4cpp?32744?5?$AA@ 1006e494     asx.obj
 0002:000064a4       ??_C@_0CH@MICPMDLM@?$CIASX_CobranetRx_SetBundle?$CJ?5ERROR@ 1006e4a4     asx.obj
 0002:000064cc       ??_C@_0O@DPPAOLKH@asx?4cpp?32749?5?$AA@ 1006e4cc     asx.obj
 0002:000064dc       ??_C@_0BI@HDCBLAIA@ASX_Tuner_SetDeemphasis?$AA@ 1006e4dc     asx.obj
 0002:000064f4       ??_C@_0BK@ICPKNAFF@ASX_Tuner_SetDeemphasis?$CI?$CJ?$AA@ 1006e4f4     asx.obj
 0002:00006510       ??_C@_0O@JLOKHCJE@asx?4cpp?32761?5?$AA@ 1006e510     asx.obj
 0002:00006520       ??_C@_0CG@DDJJEGNA@?$CIASX_Tuner_SetDeemphasis?$CJ?5ERROR?5@ 1006e520     asx.obj
 0002:00006548       ??_C@_0O@JOKFGEBB@asx?4cpp?32766?5?$AA@ 1006e548     asx.obj
 0002:00006558       ??_C@_0BO@DKOOACPP@ASX_Tuner_GetDabMultiplexName?$AA@ 1006e558     asx.obj
 0002:00006578       ??_C@_0CA@PDCCOAD@ASX_Tuner_GetDabMultiplexName?$CI?$CJ?$AA@ 1006e578     asx.obj
 0002:00006598       ??_C@_0O@CEFPLNCN@asx?4cpp?32775?5?$AA@ 1006e598     asx.obj
 0002:000065a8       ??_C@_0CM@GJKGDFOH@?$CIASX_Tuner_GetDabMultiplexName?$CJ?5@ 1006e5a8     asx.obj
 0002:000065d4       ??_C@_0O@HKPHGPJA@asx?4cpp?32780?5?$AA@ 1006e5d4     asx.obj
 0002:000065e4       ??_C@_0BC@GNDBJEBH@ASX_Tuner_GetMode?$AA@ 1006e5e4     asx.obj
 0002:000065f8       ??_C@_0BE@IAPJDGEJ@ASX_Tuner_GetMode?$CI?$CJ?$AA@ 1006e5f8     asx.obj
 0002:0000660c       ??_C@_0O@HFCGFEBP@asx?4cpp?32789?5?$AA@ 1006e60c     asx.obj
 0002:0000661c       ??_C@_0CA@MENJLIBD@?$CIASX_Tuner_GetMode?$CJ?5ERROR?5?9?$DO?5?$CFd?$AA@ 1006e61c     asx.obj
 0002:0000663c       ??_C@_0O@MFECKACJ@asx?4cpp?32794?5?$AA@ 1006e63c     asx.obj
 0002:0000664c       ??_C@_0CC@LJDAMJMH@ASX_Tuner_GetDigitalSignalQualit@ 1006e64c     asx.obj
 0002:00006670       ??_C@_0CE@BEBLAKBO@ASX_Tuner_GetDigitalSignalQualit@ 1006e670     asx.obj
 0002:00006694       ??_C@_0O@DPFFGOPH@asx?4cpp?32803?5?$AA@ 1006e694     asx.obj
 0002:000066a4       ??_C@_0DA@LGKOLDK@?$CIASX_Tuner_GetDigitalSignalQuali@ 1006e6a4     asx.obj
 0002:000066d4       ??_C@_0O@DDAAIBBG@asx?4cpp?32808?5?$AA@ 1006e6d4     asx.obj
 0002:000066e4       ??_C@_0BN@OIDPKOHO@ASX_Tuner_GetFirmwareVersion?$AA@ 1006e6e4     asx.obj
 0002:00006704       ??_C@_0BP@PCMKLKBL@ASX_Tuner_GetFirmwareVersion?$CI?$CJ?$AA@ 1006e704     asx.obj
 0002:00006724       ??_C@_0O@IAOAKBEO@asx?4cpp?32817?5?$AA@ 1006e724     asx.obj
 0002:00006734       ??_C@_0CL@IOPHIDOE@?$CIASX_Tuner_GetFirmwareVersion?$CJ?5E@ 1006e734     asx.obj
 0002:00006760       ??_C@_0O@JEJOMMEL@asx?4cpp?32822?5?$AA@ 1006e760     asx.obj
 0002:00006770       ??_C@_0BM@MGKEIDPP@ASX_Tuner_GetDabMultiplexId?$AA@ 1006e770     asx.obj
 0002:0000678c       ??_C@_0BO@JFINGBPP@ASX_Tuner_GetDabMultiplexId?$CI?$CJ?$AA@ 1006e78c     asx.obj
 0002:000067ac       ??_C@_0O@COGEBFHH@asx?4cpp?32831?5?$AA@ 1006e7ac     asx.obj
 0002:000067bc       ??_C@_0CK@LNILGCNF@?$CIASX_Tuner_GetDabMultiplexId?$CJ?5ER@ 1006e7bc     asx.obj
 0002:000067e8       ??_C@_0O@CLCLADPC@asx?4cpp?32836?5?$AA@ 1006e7e8     asx.obj
 0002:000067f8       ??_C@_0BI@MDPADPH@ASX_Tuner_GetDeemphasis?$AA@ 1006e7f8     asx.obj
 0002:00006810       ??_C@_0BK@LAOMKCEM@ASX_Tuner_GetDeemphasis?$CI?$CJ?$AA@ 1006e810     asx.obj
 0002:0000682c       ??_C@_0O@LNKAHMHG@asx?4cpp?32849?5?$AA@ 1006e82c     asx.obj
 0002:0000683c       ??_C@_0CG@MKMIGMA@?$CIASX_Tuner_GetDeemphasis?$CJ?5ERROR?5@ 1006e83c     asx.obj
 0002:00006864       ??_C@_0O@NMEIIEA@asx?4cpp?32854?5?$AA@ 1006e864     asx.obj
 0002:00006874       ??_C@_0BH@IKOEBCAH@ASX_Tuner_GetFrequency?$AA@ 1006e874     asx.obj
 0002:0000688c       ??_C@_0BJ@MOOAOFNI@ASX_Tuner_GetFrequency?$CI?$CJ?$AA@ 1006e88c     asx.obj
 0002:000068a8       ??_C@_0O@BKDODBCL@asx?4cpp?32863?5?$AA@ 1006e8a8     asx.obj
 0002:000068b8       ??_C@_0CF@KLAOEPBG@?$CIASX_Tuner_GetFrequency?$CJ?5ERROR?5?9@ 1006e8b8     asx.obj
 0002:000068e0       ??_C@_0O@BGGLNOMK@asx?4cpp?32868?5?$AA@ 1006e8e0     asx.obj
 0002:000068f0       ??_C@_0CC@PGBLMDBP@ASX_Tuner_GetDabAudioServiceCoun@ 1006e8f0     asx.obj
 0002:00006914       ??_C@_0CE@LNCPODDM@ASX_Tuner_GetDabAudioServiceCoun@ 1006e914     asx.obj
 0002:00006938       ??_C@_0O@KFILPOJC@asx?4cpp?32877?5?$AA@ 1006e938     asx.obj
 0002:00006948       ??_C@_0DA@NILCJGOO@?$CIASX_Tuner_GetDabAudioServiceCou@ 1006e948     asx.obj
 0002:00006978       ??_C@_0O@PLCDCMCP@asx?4cpp?32882?5?$AA@ 1006e978     asx.obj
 0002:00006988       ??_C@_0BC@CMHCLBBN@ASX_Tuner_GetGain?$AA@ 1006e988     asx.obj
 0002:0000699c       ??_C@_0BE@DBBCELMH@ASX_Tuner_GetGain?$CI?$CJ?$AA@ 1006e99c     asx.obj
 0002:000069b0       ??_C@_0O@EBNJPFBD@asx?4cpp?32891?5?$AA@ 1006e9b0     asx.obj
 0002:000069c0       ??_C@_0CA@EAMGGBKN@?$CIASX_Tuner_GetGain?$CJ?5ERROR?5?9?$DO?5?$CFd?$AA@ 1006e9c0     asx.obj
 0002:000069e0       ??_C@_0O@EEJGODJG@asx?4cpp?32896?5?$AA@ 1006e9e0     asx.obj
 0002:000069f0       ??_C@_0BH@POFKNOEL@ASX_Tuner_SetFrequency?$AA@ 1006e9f0     asx.obj
 0002:00006a08       ??_C@_0BJ@POBPPE@ASX_Tuner_SetFrequency?$CI?$CJ?$AA@ 1006ea08     asx.obj
 0002:00006a24       ??_C@_0O@GLIDLPF@asx?4cpp?32905?5?$AA@ 1006ea24     asx.obj
 0002:00006a34       ??_C@_0CF@CLMIICLA@?$CIASX_Tuner_SetFrequency?$CJ?5ERROR?5?9@ 1006ea34     asx.obj
 0002:00006a5c       ??_C@_0O@LIMPJOHL@asx?4cpp?32910?5?$AA@ 1006ea5c     asx.obj
 0002:00006a6c       ??_C@_0BI@MMNMPAGD@ASX_Tuner_GetRawRFLevel?$AA@ 1006ea6c     asx.obj
 0002:00006a84       ??_C@_0BK@IBHFIOBH@ASX_Tuner_GetRawRFLevel?$CI?$CJ?$AA@ 1006ea84     asx.obj
 0002:00006aa0       ??_C@_0O@LHBOKFPE@asx?4cpp?32919?5?$AA@ 1006eaa0     asx.obj
 0002:00006ab0       ??_C@_0CG@CNADJIHI@?$CIASX_Tuner_GetRawRFLevel?$CJ?5ERROR?5@ 1006eab0     asx.obj
 0002:00006ad8       ??_C@_0O@KNHDJJEJ@asx?4cpp?32924?5?$AA@ 1006ead8     asx.obj
 0002:00006ae8       ??_C@_0BC@NEIDIOMM@ASX_Tuner_SetGain?$AA@ 1006eae8     asx.obj
 0002:00006afc       ??_C@_0BE@BPFHGKFF@ASX_Tuner_SetGain?$CI?$CJ?$AA@ 1006eafc     asx.obj
 0002:00006b10       ??_C@_0O@BAIAOIKJ@asx?4cpp?32933?5?$AA@ 1006eb10     asx.obj
 0002:00006b20       ??_C@_0CA@BJNLHHPK@?$CIASX_Tuner_SetGain?$CJ?5ERROR?5?9?$DO?5?$CFd?$AA@ 1006eb20     asx.obj
 0002:00006b40       ??_C@_0O@BMNFAHEI@asx?4cpp?32938?5?$AA@ 1006eb40     asx.obj
 0002:00006b50       ??_C@_0BN@KIKINMPH@ASX_Tuner_SetDabAudioService?$AA@ 1006eb50     asx.obj
 0002:00006b70       ??_C@_0BP@KGIAMJJO@ASX_Tuner_SetDabAudioService?$CI?$CJ?$AA@ 1006eb70     asx.obj
 0002:00006b90       ??_C@_0O@IKFOHIMM@asx?4cpp?32947?5?$AA@ 1006eb90     asx.obj
 0002:00006ba0       ??_C@_0CL@POPFAAH@?$CIASX_Tuner_SetDabAudioService?$CJ?5E@ 1006eba0     asx.obj
 0002:00006bcc       ??_C@_0O@DECJNNEC@asx?4cpp?32952?5?$AA@ 1006ebcc     asx.obj
 0002:00006bdc       ??_C@_0BC@JFMAKLMG@ASX_Tuner_SetMode?$AA@ 1006ebdc     asx.obj
 0002:00006bf0       ??_C@_0BE@KOLMBHNL@ASX_Tuner_SetMode?$CI?$CJ?$AA@ 1006ebf0     asx.obj
 0002:00006c04       ??_C@_0O@CENKMMPF@asx?4cpp?32961?5?$AA@ 1006ec04     asx.obj
 0002:00006c14       ??_C@_0CA@JNMEKOEE@?$CIASX_Tuner_SetMode?$CJ?5ERROR?5?9?$DO?5?$CFd?$AA@ 1006ec14     asx.obj
 0002:00006c34       ??_C@_0O@CBJFNKHA@asx?4cpp?32966?5?$AA@ 1006ec34     asx.obj
 0002:00006c44       ??_C@_0BC@ODMDPPLD@ASX_Tuner_SetBand?$AA@ 1006ec44     asx.obj
 0002:00006c58       ??_C@_0BE@JAPCHJIG@ASX_Tuner_SetBand?$CI?$CJ?$AA@ 1006ec58     asx.obj
 0002:00006c6c       ??_C@_0O@JLGPADEM@asx?4cpp?32975?5?$AA@ 1006ec6c     asx.obj
 0002:00006c7c       ??_C@_0CA@GHNHJDHO@?$CIASX_Tuner_SetBand?$CJ?5ERROR?5?9?$DO?5?$CFd?$AA@ 1006ec7c     asx.obj
 0002:00006c9c       ??_C@_0O@MFMHNBPB@asx?4cpp?32980?5?$AA@ 1006ec9c     asx.obj
 0002:00006cac       ??_C@_0BO@EBOGBBLK@ASX_Tuner_EnumerateDeemphasis?$AA@ 1006ecac     asx.obj
 0002:00006ccc       ??_C@_0CA@GICKPJF@ASX_Tuner_EnumerateDeemphasis?$CI?$CJ?$AA@ 1006eccc     asx.obj
 0002:00006cec       ??_C@_0O@MKBGOKHO@asx?4cpp?32989?5?$AA@ 1006ecec     asx.obj
 0002:00006cfc       ??_C@_0CM@GOILHHJ@?$CIASX_Tuner_EnumerateDeemphasis?$CJ?5@ 1006ecfc     asx.obj
 0002:00006d28       ??_C@_0O@HKHCBOEI@asx?4cpp?32994?5?$AA@ 1006ed28     asx.obj
 0002:00006d38       ??_C@_0BF@PEFKFMAB@ASX_Tuner_GetProgram?$AA@ 1006ed38     asx.obj
 0002:00006d50       ??_C@_0BH@JNOFAHH@ASX_Tuner_GetProgram?$CI?$CJ?$AA@ 1006ed50     asx.obj
 0002:00006d68       ??_C@_0O@MEHJPGJD@asx?4cpp?33003?5?$AA@ 1006ed68     asx.obj
 0002:00006d78       ??_C@_0CD@HMEFNPLA@?$CIASX_Tuner_GetProgram?$CJ?5ERROR?5?9?$DO?5@ 1006ed78     asx.obj
 0002:00006d9c       ??_C@_0O@MICMBJHC@asx?4cpp?33008?5?$AA@ 1006ed9c     asx.obj
 0002:00006dac       ??_C@_0BF@IANLPAAP@ASX_Tuner_GetRFLevel?$AA@ 1006edac     asx.obj
 0002:00006dc4       ??_C@_0BH@EIDNOGLL@ASX_Tuner_GetRFLevel?$CI?$CJ?$AA@ 1006edc4     asx.obj
 0002:00006ddc       ??_C@_0O@HLMMDJCK@asx?4cpp?33017?5?$AA@ 1006eddc     asx.obj
 0002:00006dec       ??_C@_0CD@LCJCOFCE@?$CIASX_Tuner_GetRFLevel?$CJ?5ERROR?5?9?$DO?5@ 1006edec     asx.obj
 0002:00006e10       ??_C@_0O@GPLCFECP@asx?4cpp?33022?5?$AA@ 1006ee10     asx.obj
 0002:00006e20       ??_C@_0BF@OKHFOLEI@ASX_Tuner_SetProgram?$AA@ 1006ee20     asx.obj
 0002:00006e38       ??_C@_0BH@HNGAJMDL@ASX_Tuner_SetProgram?$CI?$CJ?$AA@ 1006ee38     asx.obj
 0002:00006e50       ??_C@_0O@NCEBCFMP@asx?4cpp?33035?5?$AA@ 1006ee50     asx.obj
 0002:00006e60       ??_C@_0CD@GKCIDONC@?$CIASX_Tuner_SetProgram?$CJ?5ERROR?5?9?$DO?5@ 1006ee60     asx.obj
 0002:00006e84       ??_C@_0O@EJFNNPJN@asx?4cpp?33040?5?$AA@ 1006ee84     asx.obj
 0002:00006e94       ??_C@_0BH@DIAFJICK@ASX_Tuner_GetGainRange?$AA@ 1006ee94     asx.obj
 0002:00006eac       ??_C@_0BJ@ODKHGHOI@ASX_Tuner_GetGainRange?$CI?$CJ?$AA@ 1006eeac     asx.obj
 0002:00006ec8       ??_C@_0O@EGIMOEBC@asx?4cpp?33049?5?$AA@ 1006eec8     asx.obj
 0002:00006ed8       ??_C@_0CF@LJBEMEHP@?$CIASX_Tuner_GetGainRange?$CJ?5ERROR?5?9@ 1006eed8     asx.obj
 0002:00006f00       ??_C@_0O@PGOIBACE@asx?4cpp?33054?5?$AA@ 1006ef00     asx.obj
 0002:00006f10       ??_C@_0BL@HIJHLNG@ASX_Tuner_EnumerateProgram?$AA@ 1006ef10     asx.obj
 0002:00006f2c       ??_C@_0BN@GCKNEFBH@ASX_Tuner_EnumerateProgram?$CI?$CJ?$AA@ 1006ef2c     asx.obj
 0002:00006f4c       ??_C@_0O@OGBLABJD@asx?4cpp?33067?5?$AA@ 1006ef4c     asx.obj
 0002:00006f5c       ??_C@_0CJ@KLHKADHA@?$CIASX_Tuner_EnumerateProgram?$CJ?5ERR@ 1006ef5c     asx.obj
 0002:00006f88       ??_C@_0O@FIGMKEBN@asx?4cpp?33072?5?$AA@ 1006ef88     asx.obj
 0002:00006f98       ??_C@_0BI@MHIONACN@ASX_Tuner_EnumerateBand?$AA@ 1006ef98     asx.obj
 0002:00006fb0       ??_C@_0BK@NEOBMHAG@ASX_Tuner_EnumerateBand?$CI?$CJ?$AA@ 1006efb0     asx.obj
 0002:00006fcc       ??_C@_0O@CEJAKBC@asx?4cpp?33081?5?$AA@ 1006efcc     asx.obj
 0002:00006fdc       ??_C@_0CG@KKGLEBIJ@?$CIASX_Tuner_EnumerateBand?$CJ?5ERROR?5@ 1006efdc     asx.obj
 0002:00007004       ??_C@_0O@HAGBMJH@asx?4cpp?33086?5?$AA@ 1006f004     asx.obj
 0002:00007014       ??_C@_0BE@NKHMJEDF@ASX_Tuner_GetStatus?$AA@ 1006f014     asx.obj
 0002:00007028       ??_C@_0BG@CHELMHCE@ASX_Tuner_GetStatus?$CI?$CJ?$AA@ 1006f028     asx.obj
 0002:00007040       ??_C@_0O@LNPMMFKL@asx?4cpp?33095?5?$AA@ 1006f040     asx.obj
 0002:00007050       ??_C@_0CC@EAKKHIIO@?$CIASX_Tuner_GetStatus?$CJ?5ERROR?5?9?$DO?5?$CF@ 1006f050     asx.obj
 0002:00007074       ??_C@_0O@PLFPGBHK@asx?4cpp?33100?5?$AA@ 1006f074     asx.obj
 0002:00007084       ??_C@_0BF@IELIGLMA@ASX_Tuner_GetHdBlend?$AA@ 1006f084     asx.obj
 0002:0000709c       ??_C@_0BH@GDICGDJF@ASX_Tuner_GetHdBlend?$CI?$CJ?$AA@ 1006f09c     asx.obj
 0002:000070b4       ??_C@_0O@PEIOFKPF@asx?4cpp?33109?5?$AA@ 1006f0b4     asx.obj
 0002:000070c4       ??_C@_0CD@FFJFPCPM@?$CIASX_Tuner_GetHdBlend?$CJ?5ERROR?5?9?$DO?5@ 1006f0c4     asx.obj
 0002:000070e8       ??_C@_0O@EEOKKOMD@asx?4cpp?33114?5?$AA@ 1006f0e8     asx.obj
 0002:000070f8       ??_C@_0BK@CKOGFLGG@ASX_Tuner_GetDabAudioInfo?$AA@ 1006f0f8     asx.obj
 0002:00007114       ??_C@_0BM@LNAGOGAI@ASX_Tuner_GetDabAudioInfo?$CI?$CJ?$AA@ 1006f114     asx.obj
 0002:00007130       ??_C@_0O@FDBABHKI@asx?4cpp?33123?5?$AA@ 1006f130     asx.obj
 0002:00007140       ??_C@_0CI@FDPOOCNK@?$CIASX_Tuner_GetDabAudioInfo?$CJ?5ERRO@ 1006f140     asx.obj
 0002:00007168       ??_C@_0O@FPEFPIEJ@asx?4cpp?33128?5?$AA@ 1006f168     asx.obj
 0002:00007178       ??_C@_0CB@BMADGJHB@ASX_Tuner_GetDabAudioServiceName@ 1006f178     asx.obj
 0002:0000719c       ??_C@_0CD@HAFCAFPL@ASX_Tuner_GetDabAudioServiceName@ 1006f19c     asx.obj
 0002:000071c0       ??_C@_0O@OMKFNIBB@asx?4cpp?33137?5?$AA@ 1006f1c0     asx.obj
 0002:000071d0       ??_C@_0CP@CJACPIJE@?$CIASX_Tuner_GetDabAudioServiceNam@ 1006f1d0     asx.obj
 0002:00007200       ??_C@_0O@HHLJCCED@asx?4cpp?33142?5?$AA@ 1006f200     asx.obj
 0002:00007210       ??_C@_0BM@EMEIHOMP@ASX_Tuner_GetFrequencyRange?$AA@ 1006f210     asx.obj
 0002:0000722c       ??_C@_0BO@IJMHFDEB@ASX_Tuner_GetFrequencyRange?$CI?$CJ?$AA@ 1006f22c     asx.obj
 0002:0000724c       ??_C@_0O@MNEDPLHP@asx?4cpp?33151?5?$AA@ 1006f24c     asx.obj
 0002:0000725c       ??_C@_0CK@LMNIMIKI@?$CIASX_Tuner_GetFrequencyRange?$CJ?5ER@ 1006f25c     asx.obj
 0002:00007288       ??_C@_0O@MIAMONPK@asx?4cpp?33156?5?$AA@ 1006f288     asx.obj
 0002:00007298       ??_C@_0BC@BLDCMAGC@ASX_Tuner_GetBand?$AA@ 1006f298     asx.obj
 0002:000072ac       ??_C@_0BE@LOLHFIBE@ASX_Tuner_GetBand?$CI?$CJ?$AA@ 1006f2ac     asx.obj
 0002:000072c0       ??_C@_0O@NIPPPMEN@asx?4cpp?33165?5?$AA@ 1006f2c0     asx.obj
 0002:000072d0       ??_C@_0CA@DOMKIFCJ@?$CIASX_Tuner_GetBand?$CJ?5ERROR?5?9?$DO?5?$CFd?$AA@ 1006f2d0     asx.obj
 0002:000072f0       ??_C@_0O@GGIIFJMD@asx?4cpp?33170?5?$AA@ 1006f2f0     asx.obj
 0002:00007300       ??_C@_0BF@JKJHNMIJ@ASX_Tuner_SetHdBlend?$AA@ 1006f300     asx.obj
 0002:00007318       ??_C@_0BH@BHDMKPNJ@ASX_Tuner_SetHdBlend?$CI?$CJ?$AA@ 1006f318     asx.obj
 0002:00007330       ??_C@_0O@GJFJGCEM@asx?4cpp?33179?5?$AA@ 1006f330     asx.obj
 0002:00007340       ??_C@_0CD@EDPIBDJO@?$CIASX_Tuner_SetHdBlend?$CJ?5ERROR?5?9?$DO?5@ 1006f340     asx.obj
 0002:00007364       ??_C@_0O@DJOCOBEJ@asx?4cpp?33184?5?$AA@ 1006f364     asx.obj
 0002:00007374       ??_C@_0BL@HHGLEMBH@ASX_Tuner_EnumerateHdBlend?$AA@ 1006f374     asx.obj
 0002:00007390       ??_C@_0BN@IPBHGPF@ASX_Tuner_EnumerateHdBlend?$CI?$CJ?$AA@ 1006f390     asx.obj
 0002:000073b0       ??_C@_0O@IEBBJAKJ@asx?4cpp?33193?5?$AA@ 1006f3b0     asx.obj
 0002:000073c0       ??_C@_0CJ@ICKKCODM@?$CIASX_Tuner_EnumerateHdBlend?$CJ?5ERR@ 1006f3c0     asx.obj
 0002:000073ec       ??_C@_0O@IIEEHPEI@asx?4cpp?33198?5?$AA@ 1006f3ec     asx.obj
 0002:000073fc       ??_C@_0BK@NEPDBHOG@ASX_Tuner_GetDabServiceId?$AA@ 1006f3fc     asx.obj
 0002:00007418       ??_C@_0BM@PJOPINON@ASX_Tuner_GetDabServiceId?$CI?$CJ?$AA@ 1006f418     asx.obj
 0002:00007434       ??_C@_0O@LJLAANCP@asx?4cpp?33207?5?$AA@ 1006f434     asx.obj
 0002:00007444       ??_C@_0CI@BHNJOJBP@?$CIASX_Tuner_GetDabServiceId?$CJ?5ERRO@ 1006f444     asx.obj
 0002:0000746c       ??_C@_0O@HMHKIKB@asx?4cpp?33212?5?$AA@ 1006f46c     asx.obj
 0002:0000747c       ??_C@_0BC@OOJMNKDA@ASX_Compander_Set?$AA@ 1006f47c     asx.obj
 0002:00007490       ??_C@_0BE@MLFIGLBG@ASX_Compander_Set?$CI?$CJ?$AA@ 1006f490     asx.obj
 0002:000074a4       ??_C@_0O@BBPPHLPN@asx?4cpp?33224?5?$AA@ 1006f4a4     asx.obj
 0002:000074b4       ??_C@_0CA@OEFNNEBN@?$CIASX_Compander_Set?$CJ?5ERROR?5?9?$DO?5?$CFd?$AA@ 1006f4b4     asx.obj
 0002:000074d4       ??_C@_0O@BJCHOIKO@asx?4cpp?33229?5?$AA@ 1006f4d4     asx.obj
 0002:000074e4       ??_C@_0BL@NKJIAEMM@ASX_Compander_SetThreshold?$AA@ 1006f4e4     asx.obj
 0002:00007500       ??_C@_0BN@BCDKAOHA@ASX_Compander_SetThreshold?$CI?$CJ?$AA@ 1006f500     asx.obj
 0002:00007520       ??_C@_0O@KAFJOFPM@asx?4cpp?33238?5?$AA@ 1006f520     asx.obj
 0002:00007530       ??_C@_0CJ@LGGLMCPL@?$CIASX_Compander_SetThreshold?$CJ?5ERR@ 1006f530     asx.obj
 0002:0000755c       ??_C@_0O@DBNLDCKE@asx?4cpp?33243?5?$AA@ 1006f55c     asx.obj
 0002:0000756c       ??_C@_0BH@HIBGDJIA@ASX_Compander_SetRatio?$AA@ 1006f56c     asx.obj
 0002:00007584       ??_C@_0BJ@BGJOOAOG@ASX_Compander_SetRatio?$CI?$CJ?$AA@ 1006f584     asx.obj
 0002:000075a0       ??_C@_0O@IIKFDPPG@asx?4cpp?33252?5?$AA@ 1006f5a0     asx.obj
 0002:000075b0       ??_C@_0CF@NKKCJBKG@?$CIASX_Compander_SetRatio?$CJ?5ERROR?5?9@ 1006f5b0     asx.obj
 0002:000075d8       ??_C@_0O@IOGOPNBN@asx?4cpp?33257?5?$AA@ 1006f5d8     asx.obj
 0002:000075e8       ??_C@_0CE@OLAGLGJD@ASX_Compander_SetAttackTimeConst@ 1006f5e8     asx.obj
 0002:0000760c       ??_C@_0CG@KHGKMNF@ASX_Compander_SetAttackTimeConst@ 1006f60c     asx.obj
 0002:00007634       ??_C@_0O@JNBJDIME@asx?4cpp?33266?5?$AA@ 1006f634     asx.obj
 0002:00007644       ??_C@_0DC@PIAKEHOI@?$CIASX_Compander_SetAttackTimeCons@ 1006f644     asx.obj
 0002:00007678       ??_C@_0O@CAOKEJCE@asx?4cpp?33271?5?$AA@ 1006f678     asx.obj
 0002:00007688       ??_C@_0BM@MHONOPJP@ASX_Compander_SetMakeupGain?$AA@ 1006f688     asx.obj
 0002:000076a4       ??_C@_0BO@LEHECGGC@ASX_Compander_SetMakeupGain?$CI?$CJ?$AA@ 1006f6a4     asx.obj
 0002:000076c4       ??_C@_0O@HJELDDEF@asx?4cpp?33280?5?$AA@ 1006f6c4     asx.obj
 0002:000076d4       ??_C@_0CK@NMOHNFFG@?$CIASX_Compander_SetMakeupGain?$CJ?5ER@ 1006f6d4     asx.obj
 0002:00007700       ??_C@_0O@HPIAPBKO@asx?4cpp?33285?5?$AA@ 1006f700     asx.obj
 0002:00007710       ??_C@_0CD@KFKEGGDJ@ASX_Compander_SetDecayTimeConsta@ 1006f710     asx.obj
 0002:00007734       ??_C@_0CF@NIENGEMA@ASX_Compander_SetDecayTimeConsta@ 1006f734     asx.obj
 0002:0000775c       ??_C@_0O@MGPOPMPM@asx?4cpp?33294?5?$AA@ 1006f75c     asx.obj
 0002:0000776c       ??_C@_0DB@KEIOOMMA@?$CIASX_Compander_SetDecayTimeConst@ 1006f76c     asx.obj
 0002:000077a0       ??_C@_0O@MOCGGPKP@asx?4cpp?33299?5?$AA@ 1006f7a0     asx.obj
 0002:000077b0       ??_C@_0BL@KOCGMIIA@ASX_Compander_GetThreshold?$AA@ 1006f7b0     asx.obj
 0002:000077cc       ??_C@_0BN@NMCEPEFM@ASX_Compander_GetThreshold?$CI?$CJ?$AA@ 1006f7cc     asx.obj
 0002:000077ec       ??_C@_0O@IPIMGDKC@asx?4cpp?33308?5?$AA@ 1006f7ec     asx.obj
 0002:000077fc       ??_C@_0CJ@DGKNAPFN@?$CIASX_Compander_GetThreshold?$CJ?5ERR@ 1006f7fc     asx.obj
 0002:00007828       ??_C@_0O@DLGFOLCG@asx?4cpp?33313?5?$AA@ 1006f828     asx.obj
 0002:00007838       ??_C@_0CD@PMLJHAGO@ASX_Compander_GetDecayTimeConsta@ 1006f838     asx.obj
 0002:0000785c       ??_C@_0CF@NJGDEDBP@ASX_Compander_GetDecayTimeConsta@ 1006f85c     asx.obj
 0002:00007884       ??_C@_0O@CIBCCOPP@asx?4cpp?33322?5?$AA@ 1006f884     asx.obj
 0002:00007894       ??_C@_0DB@BDDBLBLL@?$CIASX_Compander_GetDecayTimeConst@ 1006f894     asx.obj
 0002:000078c8       ??_C@_0O@CONJOMBE@asx?4cpp?33327?5?$AA@ 1006f8c8     asx.obj
 0002:000078d8       ??_C@_0CE@BOFAGPNC@ASX_Compander_GetAttackTimeConst@ 1006f8d8     asx.obj
 0002:000078fc       ??_C@_0CG@BMBLENLH@ASX_Compander_GetAttackTimeConst@ 1006f8fc     asx.obj
 0002:00007924       ??_C@_0O@JHKHOBEG@asx?4cpp?33336?5?$AA@ 1006f924     asx.obj
 0002:00007934       ??_C@_0DC@DPGKFAAB@?$CIASX_Compander_GetAttackTimeCons@ 1006f934     asx.obj
 0002:00007968       ??_C@_0O@PDPMPHK@asx?4cpp?33341?5?$AA@ 1006f968     asx.obj
 0002:00007978       ??_C@_0BI@NLCCDLME@ASX_Compander_SetEnable?$AA@ 1006f978     asx.obj
 0002:00007990       ??_C@_0BK@GMIFKIPP@ASX_Compander_SetEnable?$CI?$CJ?$AA@ 1006f990     asx.obj
 0002:000079ac       ??_C@_0O@LGEBMCCI@asx?4cpp?33350?5?$AA@ 1006f9ac     asx.obj
 0002:000079bc       ??_C@_0CG@HMJFFKCH@?$CIASX_Compander_SetEnable?$CJ?5ERROR?5@ 1006f9bc     asx.obj
 0002:000079e4       ??_C@_0O@LAIKAAMD@asx?4cpp?33355?5?$AA@ 1006f9e4     asx.obj
 0002:000079f4       ??_C@_0BI@PFGHBKFG@ASX_Compander_GetEnable?$AA@ 1006f9f4     asx.obj
 0002:00007a0c       ??_C@_0BK@GDJLHOHM@ASX_Compander_GetEnable?$CI?$CJ?$AA@ 1006fa0c     asx.obj
 0002:00007a28       ??_C@_0O@KDPNMFBK@asx?4cpp?33364?5?$AA@ 1006fa28     asx.obj
 0002:00007a38       ??_C@_0CG@HNLLHNPI@?$CIASX_Compander_GetEnable?$CJ?5ERROR?5@ 1006fa38     asx.obj
 0002:00007a60       ??_C@_0O@KLCFFGEJ@asx?4cpp?33369?5?$AA@ 1006fa60     asx.obj
 0002:00007a70       ??_C@_0BH@IJDKCKPN@ASX_Compander_GetRatio?$AA@ 1006fa70     asx.obj
 0002:00007a88       ??_C@_0BJ@ILBFHKP@ASX_Compander_GetRatio?$CI?$CJ?$AA@ 1006fa88     asx.obj
 0002:00007aa4       ??_C@_0O@BCFLFLBL@asx?4cpp?33378?5?$AA@ 1006faa4     asx.obj
 0002:00007ab4       ??_C@_0CF@CPPEEIOH@?$CIASX_Compander_GetRatio?$CJ?5ERROR?5?9@ 1006fab4     asx.obj
 0002:00007adc       ??_C@_0O@EGGNKEKM@asx?4cpp?33383?5?$AA@ 1006fadc     asx.obj
 0002:00007aec       ??_C@_0BM@LIPDFMOI@ASX_Compander_GetMakeupGain?$AA@ 1006faec     asx.obj
 0002:00007b08       ??_C@_0BO@IGGCFEHL@ASX_Compander_GetMakeupGain?$CI?$CJ?$AA@ 1006fb08     asx.obj
 0002:00007b28       ??_C@_0O@PPBDKJPO@asx?4cpp?33392?5?$AA@ 1006fb28     asx.obj
 0002:00007b38       ??_C@_0CK@ODNCBFEG@?$CIASX_Compander_GetMakeupGain?$CJ?5ER@ 1006fb38     asx.obj
 0002:00007b64       ??_C@_0O@PJNIGLBF@asx?4cpp?33397?5?$AA@ 1006fb64     asx.obj
 0002:00007b74       ??_C@_0BC@DBOHBKPI@ASX_Compander_Get?$AA@ 1006fb74     asx.obj
 0002:00007b88       ??_C@_0BE@FDBPCLJL@ASX_Compander_Get?$CI?$CJ?$AA@ 1006fb88     asx.obj
 0002:00007b9c       ??_C@_0O@DHDCJCLI@asx?4cpp?33406?5?$AA@ 1006fb9c     asx.obj
 0002:00007bac       ??_C@_0CA@IAAEGKKP@?$CIASX_Compander_Get?$CJ?5ERROR?5?9?$DO?5?$CFd?$AA@ 1006fbac     asx.obj
 0002:00007bcc       ??_C@_0O@IKMBODFI@asx?4cpp?33411?5?$AA@ 1006fbcc     asx.obj
 0002:00007bdc       ??_C@_0BI@LLBCDKNN@ASX_Meter_GetBallistics?$AA@ 1006fbdc     asx.obj
 0002:00007bf4       ??_C@_0BK@IAICFBEB@ASX_Meter_GetBallistics?$CI?$CJ?$AA@ 1006fbf4     asx.obj
 0002:00007c10       ??_C@_0O@JLPAJINI@asx?4cpp?33423?5?$AA@ 1006fc10     asx.obj
 0002:00007c20       ??_C@_0CG@CNCPPFBG@?$CIASX_Meter_GetBallistics?$CJ?5ERROR?5@ 1006fc20     asx.obj
 0002:00007c48       ??_C@_0O@JHKFHHDJ@asx?4cpp?33428?5?$AA@ 1006fc48     asx.obj
 0002:00007c58       ??_C@_0BC@JIHIKIEO@ASX_Meter_GetPeak?$AA@ 1006fc58     asx.obj
 0002:00007c6c       ??_C@_0BE@MEOPFJJK@ASX_Meter_GetPeak?$CI?$CJ?$AA@ 1006fc6c     asx.obj
 0002:00007c80       ??_C@_0O@CEEFFHGB@asx?4cpp?33437?5?$AA@ 1006fc80     asx.obj
 0002:00007c90       ??_C@_0CA@IFJOLI@?$CIASX_Meter_GetPeak?$CJ?5ERROR?5?9?$DO?5?$CFd?$AA@ 1006fc90     asx.obj
 0002:00007cb0       ??_C@_0O@LPFJKNDD@asx?4cpp?33442?5?$AA@ 1006fcb0     asx.obj
 0002:00007cc0       ??_C@_0BI@MEAMIJKK@ASX_Meter_SetBallistics?$AA@ 1006fcc0     asx.obj
 0002:00007cd8       ??_C@_0BK@LCJECDFI@ASX_Meter_SetBallistics?$CI?$CJ?$AA@ 1006fcd8     asx.obj
 0002:00007cf4       ??_C@_0O@FKDHEAP@asx?4cpp?33451?5?$AA@ 1006fcf4     asx.obj
 0002:00007d04       ??_C@_0CG@BCBKDFAG@?$CIASX_Meter_SetBallistics?$CJ?5ERROR?5@ 1006fd04     asx.obj
 0002:00007d2c       ??_C@_0O@OMGCIK@asx?4cpp?33456?5?$AA@ 1006fd2c     asx.obj
 0002:00007d3c       ??_C@_0BG@IEDCOHOE@ASX_Meter_GetChannels?$AA@ 1006fd3c     asx.obj
 0002:00007d54       ??_C@_0BI@HGGEENLC@ASX_Meter_GetChannels?$CI?$CJ?$AA@ 1006fd54     asx.obj
 0002:00007d6c       ??_C@_0O@BABPHDDN@asx?4cpp?33465?5?$AA@ 1006fd6c     asx.obj
 0002:00007d7c       ??_C@_0CE@MBPEBIFO@?$CIASX_Meter_GetChannels?$CJ?5ERROR?5?9?$DO@ 1006fd7c     asx.obj
 0002:00007da0       ??_C@_0O@KOGINGLD@asx?4cpp?33470?5?$AA@ 1006fda0     asx.obj
 0002:00007db0       ??_C@_0BB@BMPMBDA@ASX_Meter_GetRMS?$AA@ 1006fdb0     asx.obj
 0002:00007dc4       ??_C@_0BD@EBDNENKJ@ASX_Meter_GetRMS?$CI?$CJ?$AA@ 1006fdc4     asx.obj
 0002:00007dd8       ??_C@_0O@KBLJONDM@asx?4cpp?33479?5?$AA@ 1006fdd8     asx.obj
 0002:00007de8       ??_C@_0BP@OHJKIEB@?$CIASX_Meter_GetRMS?$CJ?5ERROR?5?9?$DO?5?$CFd?$AA@ 1006fde8     asx.obj
 0002:00007e08       ??_C@_0O@PBACGODJ@asx?4cpp?33484?5?$AA@ 1006fe08     asx.obj
 0002:00007e18       ??_C@_0BA@NLPAIMJC@ASX_Player_Stop?$AA@ 1006fe18     asx.obj
 0002:00007e28       ??_C@_0BC@NFGBHENA@ASX_Player_Stop?$CI?$CJ?$AA@ 1006fe28     asx.obj
 0002:00007e3c       ??_C@_0O@EKDKNNDC@asx?4cpp?33496?5?$AA@ 1006fe3c     asx.obj
 0002:00007e4c       ??_C@_0BO@OLBMDANG@?$CIASX_Player_Stop?$CJ?5ERROR?5?9?$DO?5?$CFd?$AA@ 1006fe4c     asx.obj
 0002:00007e6c       ??_C@_0O@PBNKNIN@asx?4cpp?33501?5?$AA@ 1006fe6c     asx.obj
 0002:00007e7c       ??_C@_0BI@MMCFAODO@ASX_Player_OpenPlaylist?$AA@ 1006fe7c     asx.obj
 0002:00007e94       ??_C@_0BK@NEGFHCOM@ASX_Player_OpenPlaylist?$CI?$CJ?$AA@ 1006fe94     asx.obj
 0002:00007eb0       ??_C@_0O@LGGDKANP@asx?4cpp?33510?5?$AA@ 1006feb0     asx.obj
 0002:00007ec0       ??_C@_0CG@DMJHKLJE@?$CIASX_Player_OpenPlaylist?$CJ?5ERROR?5@ 1006fec0     asx.obj
 0002:00007ee8       ??_C@_0O@LAKIGCDE@asx?4cpp?33515?5?$AA@ 1006fee8     asx.obj
 0002:00007ef8       ??_C@_0BM@DPIGFCHL@ASX_Player_Format_GetString?$AA@ 1006fef8     asx.obj
 0002:00007f14       ??_C@_0BO@DLLGCHNA@ASX_Player_Format_GetString?$CI?$CJ?$AA@ 1006ff14     asx.obj
 0002:00007f34       ??_C@_0O@KDNPKHON@asx?4cpp?33524?5?$AA@ 1006ff34     asx.obj
 0002:00007f44       ??_C@_0CK@CIOIMFJC@?$CIASX_Player_Format_GetString?$CJ?5ER@ 1006ff44     asx.obj
 0002:00007f70       ??_C@_0O@KLAHDELO@asx?4cpp?33529?5?$AA@ 1006ff70     asx.obj
 0002:00007f80       ??_C@_0BA@CIFENLEP@ASX_Player_Open?$AA@ 1006ff80     asx.obj
 0002:00007f90       ??_C@_0BC@BEPIPIHB@ASX_Player_Open?$CI?$CJ?$AA@ 1006ff90     asx.obj
 0002:00007fa4       ??_C@_0O@BCHJDJOM@asx?4cpp?33538?5?$AA@ 1006ffa4     asx.obj
 0002:00007fb4       ??_C@_0BO@PHOMAPBN@?$CIASX_Player_Open?$CJ?5ERROR?5?9?$DO?5?$CFd?$AA@ 1006ffb4     asx.obj
 0002:00007fd4       ??_C@_0O@IDPLOOLE@asx?4cpp?33543?5?$AA@ 1006ffd4     asx.obj
 0002:00007fe4       ??_C@_0BN@DIGNEBP@ASX_Player_Format_GetDetails?$AA@ 1006ffe4     asx.obj
 0002:00008004       ??_C@_0BP@DOPMJDGG@ASX_Player_Format_GetDetails?$CI?$CJ?$AA@ 10070004     asx.obj
 0002:00008024       ??_C@_0O@DKIFODOG@asx?4cpp?33552?5?$AA@ 10070024     asx.obj
 0002:00008034       ??_C@_0CL@HICLFPCK@?$CIASX_Player_Format_GetDetails?$CJ?5E@ 10070034     asx.obj
 0002:00008060       ??_C@_0O@DMEOCBAN@asx?4cpp?33557?5?$AA@ 10070060     asx.obj
 0002:00008070       ??_C@_0BB@FHFAPNIH@ASX_Player_Close?$AA@ 10070070     asx.obj
 0002:00008084       ??_C@_0BD@MFNGFPMO@ASX_Player_Close?$CI?$CJ?$AA@ 10070084     asx.obj
 0002:00008098       ??_C@_0O@CPDJOENE@asx?4cpp?33566?5?$AA@ 10070098     asx.obj
 0002:000080a8       ??_C@_0BP@DLNPOODJ@?$CIASX_Player_Close?$CJ?5ERROR?5?9?$DO?5?$CFd?$AA@ 100700a8     asx.obj
 0002:000080c8       ??_C@_0O@JCMKJFDE@asx?4cpp?33571?5?$AA@ 100700c8     asx.obj
 0002:000080d8       ??_C@_0BB@BFCGPOPI@ASX_Player_Pause?$AA@ 100700d8     asx.obj
 0002:000080ec       ??_C@_0BD@PEHICJDL@ASX_Player_Pause?$CI?$CJ?$AA@ 100700ec     asx.obj
 0002:00008100       ??_C@_0O@MLGLOPFF@asx?4cpp?33580?5?$AA@ 10070100     asx.obj
 0002:00008110       ??_C@_0BP@FNBNNKFF@?$CIASX_Player_Pause?$CJ?5ERROR?5?9?$DO?5?$CFd?$AA@ 10070110     asx.obj
 0002:00008130       ??_C@_0O@MNKACNLO@asx?4cpp?33585?5?$AA@ 10070130     asx.obj
 0002:00008140       ??_C@_0BI@NDDECHC@ASX_Player_GetTimeScale?$AA@ 10070140     asx.obj
 0002:00008158       ??_C@_0BK@PHMDLOEI@ASX_Player_GetTimeScale?$CI?$CJ?$AA@ 10070158     asx.obj
 0002:00008174       ??_C@_0O@HENOCAOM@asx?4cpp?33594?5?$AA@ 10070174     asx.obj
 0002:00008184       ??_C@_0CG@PPPHBCKC@?$CIASX_Player_GetTimeScale?$CJ?5ERROR?5@ 10070184     asx.obj
 0002:000081ac       ??_C@_0O@HMAGLDLP@asx?4cpp?33599?5?$AA@ 100701ac     asx.obj
 0002:000081bc       ??_C@_0BB@LGNCBNEL@ASX_Player_Start?$AA@ 100701bc     asx.obj
 0002:000081d0       ??_C@_0BD@CJDMEHG@ASX_Player_Start?$CI?$CJ?$AA@ 100701d0     asx.obj
 0002:000081e4       ??_C@_0O@EHGMOMNC@asx?4cpp?33608?5?$AA@ 100701e4     asx.obj
 0002:000081f4       ??_C@_0BP@DLKAKIH@?$CIASX_Player_Start?$CJ?5ERROR?5?9?$DO?5?$CFd?$AA@ 100701f4     asx.obj
 0002:00008214       ??_C@_0O@PDIFGEFG@asx?4cpp?33613?5?$AA@ 10070214     asx.obj
 0002:00008224       ??_C@_0BK@DCOIIIAC@ASX_Player_PlaylistStatus?$AA@ 10070224     asx.obj
 0002:00008240       ??_C@_0BM@KDENNDML@ASX_Player_PlaylistStatus?$CI?$CJ?$AA@ 10070240     asx.obj
 0002:0000825c       ??_C@_0O@OAPCKBIP@asx?4cpp?33622?5?$AA@ 1007025c     asx.obj
 0002:0000826c       ??_C@_0CI@NAJJFPBE@?$CIASX_Player_PlaylistStatus?$CJ?5ERRO@ 1007026c     asx.obj
 0002:00008294       ??_C@_0O@OGDJGDGE@asx?4cpp?33627?5?$AA@ 10070294     asx.obj
 0002:000082a4       ??_C@_0BI@HJINIODO@ASX_Player_SetTimeScale?$AA@ 100702a4     asx.obj
 0002:000082bc       ??_C@_0BK@DJNNEEGE@ASX_Player_SetTimeScale?$CI?$CJ?$AA@ 100702bc     asx.obj
 0002:000082d8       ??_C@_0O@FPEHGODG@asx?4cpp?33636?5?$AA@ 100702d8     asx.obj
 0002:000082e8       ??_C@_0CG@HPDBNPAE@?$CIASX_Player_SetTimeScale?$CJ?5ERROR?5@ 100702e8     asx.obj
 0002:00008310       ??_C@_0O@MHNPEAAK@asx?4cpp?33641?5?$AA@ 10070310     asx.obj
 0002:00008320       ??_C@_0BH@DEAMFNEL@ASX_Player_GetLoopMode?$AA@ 10070320     asx.obj
 0002:00008338       ??_C@_0BJ@HEEPAHDI@ASX_Player_GetLoopMode?$CI?$CJ?$AA@ 10070338     asx.obj
 0002:00008354       ??_C@_0O@HOKBENFI@asx?4cpp?33650?5?$AA@ 10070354     asx.obj
 0002:00008364       ??_C@_0CF@MDAHLGKP@?$CIASX_Player_GetLoopMode?$CJ?5ERROR?5?9@ 10070364     asx.obj
 0002:0000838c       ??_C@_0O@HIGKIPLD@asx?4cpp?33655?5?$AA@ 1007038c     asx.obj
 0002:0000839c       ??_C@_0BH@GMNBEOIP@ASX_Player_GetFilename?$AA@ 1007039c     asx.obj
 0002:000083b4       ??_C@_0BJ@FPGHAMHB@ASX_Player_GetFilename?$CI?$CJ?$AA@ 100703b4     asx.obj
 0002:000083d0       ??_C@_0O@GLBNEKGK@asx?4cpp?33664?5?$AA@ 100703d0     asx.obj
 0002:000083e0       ??_C@_0CF@LNHDEIJ@?$CIASX_Player_GetFilename?$CJ?5ERROR?5?9@ 100703e0     asx.obj
 0002:00008408       ??_C@_0O@GDMFNJDJ@asx?4cpp?33669?5?$AA@ 10070408     asx.obj
 0002:00008418       ??_C@_0BH@JMKEPKMG@ASX_Player_GetPosition?$AA@ 10070418     asx.obj
 0002:00008430       ??_C@_0BJ@LCNAHPNN@ASX_Player_GetPosition?$CI?$CJ?$AA@ 10070430     asx.obj
 0002:0000844c       ??_C@_0O@NKLLNEGL@asx?4cpp?33678?5?$AA@ 1007044c     asx.obj
 0002:0000845c       ??_C@_0CF@NJBOLPHJ@?$CIASX_Player_GetPosition?$CJ?5ERROR?5?9@ 1007045c     asx.obj
 0002:00008484       ??_C@_0O@IOINCLNM@asx?4cpp?33683?5?$AA@ 10070484     asx.obj
 0002:00008494       ??_C@_0BE@JLLNDFEJ@ASX_Player_GetState?$AA@ 10070494     asx.obj
 0002:000084a8       ??_C@_0BG@FBACDGB@ASX_Player_GetState?$CI?$CJ?$AA@ 100704a8     asx.obj
 0002:000084c0       ??_C@_0O@DHPDCGIO@asx?4cpp?33692?5?$AA@ 100704c0     asx.obj
 0002:000084d0       ??_C@_0CC@JCOINKKI@?$CIASX_Player_GetState?$CJ?5ERROR?5?9?$DO?5?$CF@ 100704d0     asx.obj
 0002:000084f4       ??_C@_0O@DBDIOEGF@asx?4cpp?33697?5?$AA@ 100704f4     asx.obj
 0002:00008504       ??_C@_0BI@ONCFBAPK@ASX_Player_PlaylistWait?$AA@ 10070504     asx.obj
 0002:0000851c       ??_C@_0BK@IBPMHMMF@ASX_Player_PlaylistWait?$CI?$CJ?$AA@ 1007051c     asx.obj
 0002:00008538       ??_C@_0O@HAJCOIGI@asx?4cpp?33706?5?$AA@ 10070538     asx.obj
 0002:00008548       ??_C@_0CG@KEHPCDLC@?$CIASX_Player_PlaylistWait?$CJ?5ERROR?5@ 10070548     asx.obj
 0002:00008570       ??_C@_0O@MNGBJJII@asx?4cpp?33711?5?$AA@ 10070570     asx.obj
 0002:00008580       ??_C@_0BD@NHMIOFMH@ASX_Player_PreLoad?$AA@ 10070580     asx.obj
 0002:00008594       ??_C@_0BF@CGMDAIAF@ASX_Player_PreLoad?$CI?$CJ?$AA@ 10070594     asx.obj
 0002:000085ac       ??_C@_0O@NOBGFMFB@asx?4cpp?33720?5?$AA@ 100705ac     asx.obj
 0002:000085bc       ??_C@_0CB@HHFNNKLA@?$CIASX_Player_PreLoad?$CJ?5ERROR?5?9?$DO?5?$CFd@ 100705bc     asx.obj
 0002:000085e0       ??_C@_0O@NINNJOLK@asx?4cpp?33725?5?$AA@ 100705e0     asx.obj
 0002:000085f0       ??_C@_0BH@DLBCILMI@ASX_Player_SetLoopMode?$AA@ 100705f0     asx.obj
 0002:00008608       ??_C@_0BJ@LFBLEEP@ASX_Player_SetLoopMode?$CI?$CJ?$AA@ 10070608     asx.obj
 0002:00008624       ??_C@_0O@GBKDJDOI@asx?4cpp?33734?5?$AA@ 10070624     asx.obj
 0002:00008634       ??_C@_0CF@GAKNNLDK@?$CIASX_Player_SetLoopMode?$CJ?5ERROR?5?9@ 10070634     asx.obj
 0002:0000865c       ??_C@_0O@GJHLAALL@asx?4cpp?33739?5?$AA@ 1007065c     asx.obj
 0002:0000866c       ??_C@_0BM@CEEGEDFG@ASX_Player_RegisterCallback?$AA@ 1007066c     asx.obj
 0002:00008688       ??_C@_0BO@HBCMEGAN@ASX_Player_RegisterCallback?$CI?$CJ?$AA@ 10070688     asx.obj
 0002:000086a8       ??_C@_0O@PFGOFCDF@asx?4cpp?33748?5?$AA@ 100706a8     asx.obj
 0002:000086b8       ??_C@_0CK@DFOABJOF@?$CIASX_Player_RegisterCallback?$CJ?5ER@ 100706b8     asx.obj
 0002:000086e4       ??_C@_0O@EBIHNKLB@asx?4cpp?33753?5?$AA@ 100706e4     asx.obj
 0002:000086f4       ??_C@_0BA@CJFGDEEJ@ASX_Player_Wait?$AA@ 100706f4     asx.obj
 0002:00008704       ??_C@_0BC@HCBHKBBM@ASX_Player_Wait?$CI?$CJ?$AA@ 10070704     asx.obj
 0002:00008718       ??_C@_0O@FCPABPGI@asx?4cpp?33762?5?$AA@ 10070718     asx.obj
 0002:00008728       ??_C@_0BO@NKKGJOKG@?$CIASX_Player_Wait?$CJ?5ERROR?5?9?$DO?5?$CFd?$AA@ 10070728     asx.obj
 0002:00008748       ??_C@_0O@FEDLNNID@asx?4cpp?33767?5?$AA@ 10070748     asx.obj
 0002:00008758       ??_C@_0BH@JDLKCMEF@ASX_Player_SetPosition?$AA@ 10070758     asx.obj
 0002:00008770       ??_C@_0BJ@MNMOMMKK@ASX_Player_SetPosition?$CI?$CJ?$AA@ 10070770     asx.obj
 0002:0000878c       ??_C@_0O@ONEFNANB@asx?4cpp?33776?5?$AA@ 1007078c     asx.obj
 0002:0000879c       ??_C@_0CF@HKLENCOM@?$CIASX_Player_SetPosition?$CJ?5ERROR?5?9@ 1007079c     asx.obj
 0002:000087c4       ??_C@_0O@LAGJNGAC@asx?4cpp?33781?5?$AA@ 100707c4     asx.obj
 0002:000087d4       ??_C@_0BD@ILJPAIFP@ASX_GPIO_OutputGet?$AA@ 100707d4     asx.obj
 0002:000087e8       ??_C@_0BF@EBOAMKIF@ASX_GPIO_OutputGet?$CI?$CJ?$AA@ 100707e8     asx.obj
 0002:00008800       ??_C@_0O@LFBGFAJ@asx?4cpp?33793?5?$AA@ 10070800     asx.obj
 0002:00008810       ??_C@_0CB@BNKECGHH@?$CIASX_GPIO_OutputGet?$CJ?5ERROR?5?9?$DO?5?$CFd@ 10070810     asx.obj
 0002:00008834       ??_C@_0O@HAEIKOI@asx?4cpp?33798?5?$AA@ 10070834     asx.obj
 0002:00008844       ??_C@_0BD@FEOEMIJH@ASX_GPIO_OutputSet?$AA@ 10070844     asx.obj
 0002:00008858       ??_C@_0BF@NJKHIKAI@ASX_GPIO_OutputSet?$CI?$CJ?$AA@ 10070858     asx.obj
 0002:00008870       ??_C@_0O@PDAABFIO@asx?4cpp?33807?5?$AA@ 10070870     asx.obj
 0002:00008880       ??_C@_0CB@HJPNJIMF@?$CIASX_GPIO_OutputSet?$CJ?5ERROR?5?9?$DO?5?$CFd@ 10070880     asx.obj
 0002:000088a4       ??_C@_0O@ENHHLAAA@asx?4cpp?33812?5?$AA@ 100708a4     asx.obj
 0002:000088b4       ??_C@_0BC@DHHPCOEJ@ASX_GPIO_InputGet?$AA@ 100708b4     asx.obj
 0002:000088c8       ??_C@_0BE@IPHFEGEP@ASX_GPIO_InputGet?$CI?$CJ?$AA@ 100708c8     asx.obj
 0002:000088dc       ??_C@_0O@FNIEKBLH@asx?4cpp?33821?5?$AA@ 100708dc     asx.obj
 0002:000088ec       ??_C@_0CA@IDGEBGDP@?$CIASX_GPIO_InputGet?$CJ?5ERROR?5?9?$DO?5?$CFd?$AA@ 100708ec     asx.obj
 0002:0000890c       ??_C@_0O@FIMLLHDC@asx?4cpp?33826?5?$AA@ 1007090c     asx.obj
 0002:0000891c       ??_C@_0BH@IFGGBGNO@ASX_GPIO_GetProperties?$AA@ 1007091c     asx.obj
 0002:00008934       ??_C@_0BJ@JJHHFABF@ASX_GPIO_GetProperties?$CI?$CJ?$AA@ 10070934     asx.obj
 0002:00008950       ??_C@_0O@OCDBGOAO@asx?4cpp?33835?5?$AA@ 10070950     asx.obj
 0002:00008960       ??_C@_0CF@FIPLLLDE@?$CIASX_GPIO_GetProperties?$CJ?5ERROR?5?9@ 10070960     asx.obj
 0002:00008988       ??_C@_0O@HJCNJEFM@asx?4cpp?33840?5?$AA@ 10070988     asx.obj
 0002:00008998       ??_C@_0BB@OJACDJEF@ASX_Vox_SetLevel?$AA@ 10070998     asx.obj
 0002:000089ac       ??_C@_0BD@KABDFCPJ@ASX_Vox_SetLevel?$CI?$CJ?$AA@ 100709ac     asx.obj
 0002:000089c0       ??_C@_0O@MCBFCHFH@asx?4cpp?33852?5?$AA@ 100709c0     asx.obj
 0002:000089d0       ??_C@_0BP@KFCLNDMO@?$CIASX_Vox_SetLevel?$CJ?5ERROR?5?9?$DO?5?$CFd?$AA@ 100709d0     asx.obj
 0002:000089f0       ??_C@_0O@MENOOFLM@asx?4cpp?33857?5?$AA@ 100709f0     asx.obj
 0002:00008a00       ??_C@_0BB@JDJJPPEE@ASX_Vox_GetRange?$AA@ 10070a00     asx.obj
 0002:00008a14       ??_C@_0BD@MLAPHOKG@ASX_Vox_GetRange?$CI?$CJ?$AA@ 10070a14     asx.obj
 0002:00008a28       ??_C@_0O@NHKJCAGF@asx?4cpp?33866?5?$AA@ 10070a28     asx.obj
 0002:00008a38       ??_C@_0BP@NMHJBEPK@?$CIASX_Vox_GetRange?$CJ?5ERROR?5?9?$DO?5?$CFd?$AA@ 10070a38     asx.obj
 0002:00008a58       ??_C@_0O@GKFKFBIF@asx?4cpp?33871?5?$AA@ 10070a58     asx.obj
 0002:00008a68       ??_C@_0BB@BICOCKDI@ASX_Vox_GetLevel?$AA@ 10070a68     asx.obj
 0002:00008a7c       ??_C@_0BD@LODMOFLA@ASX_Vox_GetLevel?$CI?$CJ?$AA@ 10070a7c     asx.obj
 0002:00008a90       ??_C@_0O@DDPLCLOE@asx?4cpp?33880?5?$AA@ 10070a90     asx.obj
 0002:00008aa0       ??_C@_0BP@FAHNAKIP@?$CIASX_Vox_GetLevel?$CJ?5ERROR?5?9?$DO?5?$CFd?$AA@ 10070aa0     asx.obj
 0002:00008ac0       ??_C@_0O@DFDAOJAP@asx?4cpp?33885?5?$AA@ 10070ac0     asx.obj
 0002:00008ace       ?is_bounded@_Num_int_base@std@@2_NB 10070ace     asxavdecc.obj
 0002:00008acf       ?is_exact@_Num_int_base@std@@2_NB 10070acf     asxavdecc.obj
 0002:00008ad0       ?is_integer@_Num_int_base@std@@2_NB 10070ad0     asxavdecc.obj
 0002:00008ad1       ?is_modulo@_Num_int_base@std@@2_NB 10070ad1     asxavdecc.obj
 0002:00008ad2       ?is_specialized@_Num_int_base@std@@2_NB 10070ad2     asxavdecc.obj
 0002:00008ad4       ?radix@_Num_int_base@std@@2HB 10070ad4     asxavdecc.obj
 0002:00008ad8       ?has_denorm@_Num_float_base@std@@2W4float_denorm_style@2@B 10070ad8     asxavdecc.obj
 0002:00008adc       ?has_denorm_loss@_Num_float_base@std@@2_NB 10070adc     asxavdecc.obj
 0002:00008add       ?has_infinity@_Num_float_base@std@@2_NB 10070add     asxavdecc.obj
 0002:00008ade       ?has_quiet_NaN@_Num_float_base@std@@2_NB 10070ade     asxavdecc.obj
 0002:00008adf       ?has_signaling_NaN@_Num_float_base@std@@2_NB 10070adf     asxavdecc.obj
 0002:00008ae0       ?is_bounded@_Num_float_base@std@@2_NB 10070ae0     asxavdecc.obj
 0002:00008ae1       ?is_exact@_Num_float_base@std@@2_NB 10070ae1     asxavdecc.obj
 0002:00008ae2       ?is_iec559@_Num_float_base@std@@2_NB 10070ae2     asxavdecc.obj
 0002:00008ae3       ?is_integer@_Num_float_base@std@@2_NB 10070ae3     asxavdecc.obj
 0002:00008ae4       ?is_modulo@_Num_float_base@std@@2_NB 10070ae4     asxavdecc.obj
 0002:00008ae5       ?is_signed@_Num_float_base@std@@2_NB 10070ae5     asxavdecc.obj
 0002:00008ae6       ?is_specialized@_Num_float_base@std@@2_NB 10070ae6     asxavdecc.obj
 0002:00008ae7       ?tinyness_before@_Num_float_base@std@@2_NB 10070ae7     asxavdecc.obj
 0002:00008ae8       ?traps@_Num_float_base@std@@2_NB 10070ae8     asxavdecc.obj
 0002:00008aec       ?table_size@?$ctype@D@std@@2IB 10070aec     asxavdecc.obj
 0002:00008af0       ?round_style@_Num_float_base@std@@2W4float_round_style@2@B 10070af0     asxavdecc.obj
 0002:00008af4       ?radix@_Num_float_base@std@@2HB 10070af4     asxavdecc.obj
 0002:00008af8       ?is_signed@?$numeric_limits@D@std@@2_NB 10070af8     asxavdecc.obj
 0002:00008afc       ?digits@?$numeric_limits@D@std@@2HB 10070afc     asxavdecc.obj
 0002:00008b00       ?digits10@?$numeric_limits@D@std@@2HB 10070b00     asxavdecc.obj
 0002:00008b04       ?is_signed@?$numeric_limits@_W@std@@2_NB 10070b04     asxavdecc.obj
 0002:00008b08       ?digits@?$numeric_limits@_W@std@@2HB 10070b08     asxavdecc.obj
 0002:00008b0c       ?digits10@?$numeric_limits@_W@std@@2HB 10070b0c     asxavdecc.obj
 0002:00008b10       ?is_modulo@?$numeric_limits@_N@std@@2_NB 10070b10     asxavdecc.obj
 0002:00008b11       ?is_signed@?$numeric_limits@_N@std@@2_NB 10070b11     asxavdecc.obj
 0002:00008b14       ?digits@?$numeric_limits@_N@std@@2HB 10070b14     asxavdecc.obj
 0002:00008b18       ?digits10@?$numeric_limits@_N@std@@2HB 10070b18     asxavdecc.obj
 0002:00008b1c       ?is_signed@?$numeric_limits@C@std@@2_NB 10070b1c     asxavdecc.obj
 0002:00008b20       ?digits@?$numeric_limits@C@std@@2HB 10070b20     asxavdecc.obj
 0002:00008b24       ?digits10@?$numeric_limits@C@std@@2HB 10070b24     asxavdecc.obj
 0002:00008b28       ?is_signed@?$numeric_limits@E@std@@2_NB 10070b28     asxavdecc.obj
 0002:00008b2c       ?digits@?$numeric_limits@E@std@@2HB 10070b2c     asxavdecc.obj
 0002:00008b30       ?digits10@?$numeric_limits@E@std@@2HB 10070b30     asxavdecc.obj
 0002:00008b34       ?is_signed@?$numeric_limits@F@std@@2_NB 10070b34     asxavdecc.obj
 0002:00008b38       ?digits@?$numeric_limits@F@std@@2HB 10070b38     asxavdecc.obj
 0002:00008b3c       ?digits10@?$numeric_limits@F@std@@2HB 10070b3c     asxavdecc.obj
 0002:00008b40       ?is_signed@?$numeric_limits@G@std@@2_NB 10070b40     asxavdecc.obj
 0002:00008b44       ?digits@?$numeric_limits@G@std@@2HB 10070b44     asxavdecc.obj
 0002:00008b48       ?digits10@?$numeric_limits@G@std@@2HB 10070b48     asxavdecc.obj
 0002:00008b4c       ?is_signed@?$numeric_limits@H@std@@2_NB 10070b4c     asxavdecc.obj
 0002:00008b50       ?digits@?$numeric_limits@H@std@@2HB 10070b50     asxavdecc.obj
 0002:00008b54       ?digits10@?$numeric_limits@H@std@@2HB 10070b54     asxavdecc.obj
 0002:00008b58       ?is_signed@?$numeric_limits@I@std@@2_NB 10070b58     asxavdecc.obj
 0002:00008b5c       ?digits@?$numeric_limits@I@std@@2HB 10070b5c     asxavdecc.obj
 0002:00008b60       ?value@?$integral_constant@_N$0A@@std@@2_NB 10070b60     asxavdecc.obj
 0002:00008b64       ?digits10@?$numeric_limits@I@std@@2HB 10070b64     asxavdecc.obj
 0002:00008b68       ?value@?$integral_constant@I$07@std@@2IB 10070b68     asxavdecc.obj
 0002:00008b6c       ?value@?$integral_constant@_N$00@std@@2_NB 10070b6c     asxavdecc.obj
 0002:00008b6d       ?is_signed@?$numeric_limits@J@std@@2_NB 10070b6d     asxavdecc.obj
 0002:00008b70       ?digits@?$numeric_limits@J@std@@2HB 10070b70     asxavdecc.obj
 0002:00008b74       ?digits10@?$numeric_limits@J@std@@2HB 10070b74     asxavdecc.obj
 0002:00008b78       ?value@?$integral_constant@I$03@std@@2IB 10070b78     asxavdecc.obj
 0002:00008b7c       ?is_signed@?$numeric_limits@K@std@@2_NB 10070b7c     asxavdecc.obj
 0002:00008b80       ?digits@?$numeric_limits@K@std@@2HB 10070b80     asxavdecc.obj
 0002:00008b84       ?digits10@?$numeric_limits@K@std@@2HB 10070b84     asxavdecc.obj
 0002:00008b88       ?is_signed@?$numeric_limits@_J@std@@2_NB 10070b88     asxavdecc.obj
 0002:00008b8c       ?digits@?$numeric_limits@_J@std@@2HB 10070b8c     asxavdecc.obj
 0002:00008b90       ?digits10@?$numeric_limits@_J@std@@2HB 10070b90     asxavdecc.obj
 0002:00008b94       ?value@?$integral_constant@I$01@std@@2IB 10070b94     asxavdecc.obj
 0002:00008b98       ?is_signed@?$numeric_limits@_K@std@@2_NB 10070b98     asxavdecc.obj
 0002:00008b9c       ?digits@?$numeric_limits@_K@std@@2HB 10070b9c     asxavdecc.obj
 0002:00008ba0       ?digits10@?$numeric_limits@_K@std@@2HB 10070ba0     asxavdecc.obj
 0002:00008ba4       ?digits@?$numeric_limits@M@std@@2HB 10070ba4     asxavdecc.obj
 0002:00008ba8       ?digits10@?$numeric_limits@M@std@@2HB 10070ba8     asxavdecc.obj
 0002:00008bac       ?value@?$integral_constant@I$00@std@@2IB 10070bac     asxavdecc.obj
 0002:00008bb0       ?max_digits10@?$numeric_limits@M@std@@2HB 10070bb0     asxavdecc.obj
 0002:00008bb4       ?max_exponent@?$numeric_limits@M@std@@2HB 10070bb4     asxavdecc.obj
 0002:00008bb8       ?max_exponent10@?$numeric_limits@M@std@@2HB 10070bb8     asxavdecc.obj
 0002:00008bbc       ?min_exponent@?$numeric_limits@M@std@@2HB 10070bbc     asxavdecc.obj
 0002:00008bc0       ?min_exponent10@?$numeric_limits@M@std@@2HB 10070bc0     asxavdecc.obj
 0002:00008bc4       ?value@?$_Maximum@$S@std@@2IB 10070bc4     asxavdecc.obj
 0002:00008bc8       ?skipws@?$_Iosb@H@std@@2W4_Fmtflags@12@B 10070bc8     asxavdecc.obj
 0002:00008bcc       ?unitbuf@?$_Iosb@H@std@@2W4_Fmtflags@12@B 10070bcc     asxavdecc.obj
 0002:00008bd0       ?uppercase@?$_Iosb@H@std@@2W4_Fmtflags@12@B 10070bd0     asxavdecc.obj
 0002:00008bd4       ?digits@?$numeric_limits@N@std@@2HB 10070bd4     asxavdecc.obj
 0002:00008bd8       ?showbase@?$_Iosb@H@std@@2W4_Fmtflags@12@B 10070bd8     asxavdecc.obj
 0002:00008bdc       ?digits10@?$numeric_limits@N@std@@2HB 10070bdc     asxavdecc.obj
 0002:00008be0       ?showpoint@?$_Iosb@H@std@@2W4_Fmtflags@12@B 10070be0     asxavdecc.obj
 0002:00008be4       ?max_digits10@?$numeric_limits@N@std@@2HB 10070be4     asxavdecc.obj
 0002:00008be8       ?showpos@?$_Iosb@H@std@@2W4_Fmtflags@12@B 10070be8     asxavdecc.obj
 0002:00008bec       ?value@?$integral_constant@I$0A@@std@@2IB 10070bec     asxavdecc.obj
 0002:00008bf0       ?max_exponent@?$numeric_limits@N@std@@2HB 10070bf0     asxavdecc.obj
 0002:00008bf4       ?left@?$_Iosb@H@std@@2W4_Fmtflags@12@B 10070bf4     asxavdecc.obj
 0002:00008bf8       ?right@?$_Iosb@H@std@@2W4_Fmtflags@12@B 10070bf8     asxavdecc.obj
 0002:00008bfc       ?max_exponent10@?$numeric_limits@N@std@@2HB 10070bfc     asxavdecc.obj
 0002:00008c00       ?internal@?$_Iosb@H@std@@2W4_Fmtflags@12@B 10070c00     asxavdecc.obj
 0002:00008c04       ?min_exponent@?$numeric_limits@N@std@@2HB 10070c04     asxavdecc.obj
 0002:00008c08       ?dec@?$_Iosb@H@std@@2W4_Fmtflags@12@B 10070c08     asxavdecc.obj
 0002:00008c0c       ?oct@?$_Iosb@H@std@@2W4_Fmtflags@12@B 10070c0c     asxavdecc.obj
 0002:00008c10       ?min_exponent10@?$numeric_limits@N@std@@2HB 10070c10     asxavdecc.obj
 0002:00008c14       ?hex@?$_Iosb@H@std@@2W4_Fmtflags@12@B 10070c14     asxavdecc.obj
 0002:00008c18       ?scientific@?$_Iosb@H@std@@2W4_Fmtflags@12@B 10070c18     asxavdecc.obj
 0002:00008c1c       ?fixed@?$_Iosb@H@std@@2W4_Fmtflags@12@B 10070c1c     asxavdecc.obj
 0002:00008c20       ?hexfloat@?$_Iosb@H@std@@2W4_Fmtflags@12@B 10070c20     asxavdecc.obj
 0002:00008c24       ?boolalpha@?$_Iosb@H@std@@2W4_Fmtflags@12@B 10070c24     asxavdecc.obj
 0002:00008c28       ?_Stdio@?$_Iosb@H@std@@2W4_Fmtflags@12@B 10070c28     asxavdecc.obj
 0002:00008c2c       ?adjustfield@?$_Iosb@H@std@@2W4_Fmtflags@12@B 10070c2c     asxavdecc.obj
 0002:00008c30       ?basefield@?$_Iosb@H@std@@2W4_Fmtflags@12@B 10070c30     asxavdecc.obj
 0002:00008c34       ?floatfield@?$_Iosb@H@std@@2W4_Fmtflags@12@B 10070c34     asxavdecc.obj
 0002:00008c38       ?digits@?$numeric_limits@O@std@@2HB 10070c38     asxavdecc.obj
 0002:00008c3c       ?goodbit@?$_Iosb@H@std@@2W4_Iostate@12@B 10070c3c     asxavdecc.obj
 0002:00008c40       ?digits10@?$numeric_limits@O@std@@2HB 10070c40     asxavdecc.obj
 0002:00008c44       ?eofbit@?$_Iosb@H@std@@2W4_Iostate@12@B 10070c44     asxavdecc.obj
 0002:00008c48       ?max_digits10@?$numeric_limits@O@std@@2HB 10070c48     asxavdecc.obj
 0002:00008c4c       ?failbit@?$_Iosb@H@std@@2W4_Iostate@12@B 10070c4c     asxavdecc.obj
 0002:00008c50       ?max_exponent@?$numeric_limits@O@std@@2HB 10070c50     asxavdecc.obj
 0002:00008c54       ?badbit@?$_Iosb@H@std@@2W4_Iostate@12@B 10070c54     asxavdecc.obj
 0002:00008c58       ?max_exponent10@?$numeric_limits@O@std@@2HB 10070c58     asxavdecc.obj
 0002:00008c5c       ?_Hardfail@?$_Iosb@H@std@@2W4_Iostate@12@B 10070c5c     asxavdecc.obj
 0002:00008c60       ?min_exponent@?$numeric_limits@O@std@@2HB 10070c60     asxavdecc.obj
 0002:00008c64       ?in@?$_Iosb@H@std@@2W4_Openmode@12@B 10070c64     asxavdecc.obj
 0002:00008c68       ?min_exponent10@?$numeric_limits@O@std@@2HB 10070c68     asxavdecc.obj
 0002:00008c6c       ?out@?$_Iosb@H@std@@2W4_Openmode@12@B 10070c6c     asxavdecc.obj
 0002:00008c70       ?ate@?$_Iosb@H@std@@2W4_Openmode@12@B 10070c70     asxavdecc.obj
 0002:00008c74       ?app@?$_Iosb@H@std@@2W4_Openmode@12@B 10070c74     asxavdecc.obj
 0002:00008c78       ?trunc@?$_Iosb@H@std@@2W4_Openmode@12@B 10070c78     asxavdecc.obj
 0002:00008c7c       ?_Nocreate@?$_Iosb@H@std@@2W4_Openmode@12@B 10070c7c     asxavdecc.obj
 0002:00008c80       ?_Noreplace@?$_Iosb@H@std@@2W4_Openmode@12@B 10070c80     asxavdecc.obj
 0002:00008c84       ?binary@?$_Iosb@H@std@@2W4_Openmode@12@B 10070c84     asxavdecc.obj
 0002:00008c88       ?beg@?$_Iosb@H@std@@2W4_Seekdir@12@B 10070c88     asxavdecc.obj
 0002:00008c8c       ?cur@?$_Iosb@H@std@@2W4_Seekdir@12@B 10070c8c     asxavdecc.obj
 0002:00008c90       ?end@?$_Iosb@H@std@@2W4_Seekdir@12@B 10070c90     asxavdecc.obj
 0002:00008c94       ?collate@?$_Locbase@H@std@@2HB 10070c94     asxavdecc.obj
 0002:00008c98       ?has_denorm@_Num_base@std@@2W4float_denorm_style@2@B 10070c98     asxavdecc.obj
 0002:00008c9c       ?ctype@?$_Locbase@H@std@@2HB 10070c9c     asxavdecc.obj
 0002:00008ca0       ?has_denorm_loss@_Num_base@std@@2_NB 10070ca0     asxavdecc.obj
 0002:00008ca4       ?monetary@?$_Locbase@H@std@@2HB 10070ca4     asxavdecc.obj
 0002:00008ca8       ?numeric@?$_Locbase@H@std@@2HB 10070ca8     asxavdecc.obj
 0002:00008cac       ?has_infinity@_Num_base@std@@2_NB 10070cac     asxavdecc.obj
 0002:00008cb0       ?time@?$_Locbase@H@std@@2HB 10070cb0     asxavdecc.obj
 0002:00008cb4       ?has_quiet_NaN@_Num_base@std@@2_NB 10070cb4     asxavdecc.obj
 0002:00008cb8       ?messages@?$_Locbase@H@std@@2HB 10070cb8     asxavdecc.obj
 0002:00008cbc       ?all@?$_Locbase@H@std@@2HB 10070cbc     asxavdecc.obj
 0002:00008cc0       ?has_signaling_NaN@_Num_base@std@@2_NB 10070cc0     asxavdecc.obj
 0002:00008cc4       ?none@?$_Locbase@H@std@@2HB 10070cc4     asxavdecc.obj
 0002:00008cc8       ?is_bounded@_Num_base@std@@2_NB 10070cc8     asxavdecc.obj
 0002:00008cc9       ?is_exact@_Num_base@std@@2_NB 10070cc9     asxavdecc.obj
 0002:00008cca       ?is_iec559@_Num_base@std@@2_NB 10070cca     asxavdecc.obj
 0002:00008ccb       ?is_integer@_Num_base@std@@2_NB 10070ccb     asxavdecc.obj
 0002:00008ccc       ?is_modulo@_Num_base@std@@2_NB 10070ccc     asxavdecc.obj
 0002:00008ccd       ?is_signed@_Num_base@std@@2_NB 10070ccd     asxavdecc.obj
 0002:00008cce       ?is_specialized@_Num_base@std@@2_NB 10070cce     asxavdecc.obj
 0002:00008ccf       ?tinyness_before@_Num_base@std@@2_NB 10070ccf     asxavdecc.obj
 0002:00008cd0       ?traps@_Num_base@std@@2_NB 10070cd0     asxavdecc.obj
 0002:00008cd4       ?round_style@_Num_base@std@@2W4float_round_style@2@B 10070cd4     asxavdecc.obj
 0002:00008cd8       ?digits@_Num_base@std@@2HB 10070cd8     asxavdecc.obj
 0002:00008cdc       ?digits10@_Num_base@std@@2HB 10070cdc     asxavdecc.obj
 0002:00008ce0       ?max_digits10@_Num_base@std@@2HB 10070ce0     asxavdecc.obj
 0002:00008ce4       ?max_exponent@_Num_base@std@@2HB 10070ce4     asxavdecc.obj
 0002:00008ce8       ?max_exponent10@_Num_base@std@@2HB 10070ce8     asxavdecc.obj
 0002:00008cec       ?min_exponent@_Num_base@std@@2HB 10070cec     asxavdecc.obj
 0002:00008cf0       ?min_exponent10@_Num_base@std@@2HB 10070cf0     asxavdecc.obj
 0002:00008cf4       ?radix@_Num_base@std@@2HB  10070cf4     asxavdecc.obj
 0002:00008cf8       ??_C@_0BD@FPLNHGKN@Unsupported?5System?$AA@ 10070cf8     asxavdecc.obj
 0002:00008d10       ??_7asxSubSystemAVDECC@@6B@ 10070d10     asxavdecc.obj
 0002:00008d24       ??_7asxAdapterAVDECC@@6B@  10070d24     asxavdecc.obj
 0002:00008d74       ??_7error_category@std@@6B@ 10070d74     asxavdecc.obj
 0002:00008d90       ??_7_Generic_error_category@std@@6B@ 10070d90     asxavdecc.obj
 0002:00008da8       ??_C@_07DCLBNMLN@generic?$AA@ 10070da8     asxavdecc.obj
 0002:00008db0       ??_C@_0O@BFJCFAAK@unknown?5error?$AA@ 10070db0     asxavdecc.obj
 0002:00008dc4       ??_7_Iostream_error_category@std@@6B@ 10070dc4     asxavdecc.obj
 0002:00008ddc       ??_C@_08LLGCOLLL@iostream?$AA@ 10070ddc     asxavdecc.obj
 0002:00008de8       ??_C@_0BG@PADBLCHM@iostream?5stream?5error?$AA@ 10070de8     asxavdecc.obj
 0002:00008e04       ??_7_System_error_category@std@@6B@ 10070e04     asxavdecc.obj
 0002:00008e1c       ??_C@_06FHFOAHML@system?$AA@ 10070e1c     asxavdecc.obj
 0002:00008e24       ??_C@_04HIBGFPH@NULL?$AA@  10070e24     asxavdecc.obj
 0002:00008e2c       ??_C@_0DC@IHDLMDHJ@?6?$FLNOTIFICATION?$FN?5?$CI?$CFs?0?50x?$CFllx?0?5?$CFs?0@ 10070e2c     asxavdecc.obj
 0002:00008e60       ??_C@_0DC@OLBJDABG@?6?$FLNOTIFICATION?$FN?5?$CI?$CFs?0?50x?$CFllx?0?5?$CFd?0@ 10070e60     asxavdecc.obj
 0002:00008e94       ??_C@_0CN@GJCAHKKA@wpcap?5returned?5packet?5larger?5tha@ 10070e94     asxavdecc.obj
 0002:00008ec4       ??_C@_0BM@DMLAKCLE@avdecc_log_callback?$CI?$CJ?5?9?5?5?$CFs?$AA@ 10070ec4     asxavdecc.obj
 0002:00008ee0       ??_C@_06PCAJMMHP@AVDECC?$AA@ 10070ee0     asxavdecc.obj
 0002:00008ee8       ??_C@_0L@BJGDIPJ@dummy?5name?$AA@ 10070ee8     asxavdecc.obj
 0002:00008ef4       ??_C@_0BI@CFPLBAOH@invalid?5string?5position?$AA@ 10070ef4     asxavdecc.obj
 0002:00008f0c       ??_C@_0BA@JFNIOLAK@string?5too?5long?$AA@ 10070f0c     asxavdecc.obj
 0002:00008f20       __xmm@46454443424139383736353433323130 10070f20     asxavdecc.obj
 0002:00008f34       ??_7asxMixerScanner@@6B@   10070f34     asxasio.obj
 0002:00008f44       ??_7asxSubSystemASIO@@6B@  10070f44     asxasio.obj
 0002:00008f58       ??_7asxAdapterASIO@@6B@    10070f58     asxasio.obj
 0002:00008fa4       ??_C@_04CGFJFPFD@none?$AA@ 10070fa4     asxasio.obj
 0002:00008fb0       ??_7asxMixerScannerASIO@@6B@ 10070fb0     asxasio.obj
 0002:00008fbc       ??_C@_04INFMDMNC@ASIO?$AA@ 10070fbc     asxasio.obj
 0002:00008fc4       ??_C@_0CA@LHAMPJPC@software?2asio?2AudioScience?5ASIO?$AA@ 10070fc4     asxasio.obj
 0002:00008fe4       ??_C@_05KDICOIJK@clsid?$AA@ 10070fe4     asxasio.obj
 0002:00008fec       ??_C@_0M@PPJNHBMP@description?$AA@ 10070fec     asxasio.obj
 0002:00008ffc       ??_7asxPlayerASIO@@6B@     10070ffc     asxasioplay.obj
 0002:000090b0       __xmm@41f00000000000000000000000000000 100710b0     asxasioplay.obj
 0002:000090c4       ??_7asxRecorderASIO@@6B@   100710c4     asxasiorec.obj
 0002:0000a9fc       ??_7asxBase@@6B@           100729fc     asxclass.obj
 0002:0000aa0c       ??_7asxAdapter@@6B@        10072a0c     asxclass.obj
 0002:0000aa5c       ??_7asxAbstractAdapter@@6B@ 10072a5c     asxclass.obj
 0002:0000aaac       ??_7asxSystem@@6B@         10072aac     asxclass.obj
 0002:0000aac0       ??_7asxSubSystem@@6B@      10072ac0     asxclass.obj
 0002:0000aad4       ??_7asxNode@@6B@           10072ad4     asxclass.obj
 0002:0000aae4       ??_7asxControlBase@@6B@    10072ae4     asxclass.obj
 0002:0000ab00       ??_7asxMixer@@6B@          10072b00     asxclass.obj
 0002:0000ab10       ??_7asxBlockProperty@@6B@  10072b10     asxclass.obj
 0002:0000ab2c       ??_C@_02DPKJAMEF@?$CFd?$AA@ 10072b2c     asxclass.obj
 0002:0000ab30       ??_C@_0BK@BOGCDNP@Software?2AudioScience?2ASX?$AA@ 10072b30     asxclass.obj
 0002:0000ab4c       ??_C@_0BF@GNFHCOHF@HostNetworkInterface?$AA@ 10072b4c     asxclass.obj
 0002:0000ab64       ??_C@_02LIELOMNJ@on?$AA@   10072b64     asxclass.obj
 0002:0000ab68       ??_C@_0BD@OCCHJOKD@CobraNetAutoAssign?$AA@ 10072b68     asxclass.obj
 0002:0000ab7c       ??_C@_0BI@CCKGBOCG@CobraNetAutoAssignStart?$AA@ 10072b7c     asxclass.obj
 0002:0000ab94       ??_C@_0BG@HOOEBBKC@CobraNetAutoAssignEnd?$AA@ 10072b94     asxclass.obj
 0002:0000abac       ??_C@_03MCADLMAF@off?$AA@  10072bac     asxclass.obj
 0002:0000abb0       ??_C@_07OHKHACFK@0?40?40?40?$AA@ 10072bb0     asxclass.obj
 0002:0000abb8       ??_C@_07CJLGJJPJ@4?418?408?$AA@ 10072bb8     asxclass.obj
 0002:0000abc0       ??_C@_07CIFAGBMG@unknown?$AA@ 10072bc0     asxclass.obj
 0002:0000abc8       ??_C@_0CC@NNNCPKHA@Predelete?$CI?$CJ?5ERROR?5?9?$DO?5?$CFd?0?5index?5?$CF@ 10072bc8     asxclass.obj
 0002:0000abec       ??_C@_0BC@JOBGNMOC@asxclass?4cpp?3592?5?$AA@ 10072bec     asxclass.obj
 0002:0000ac00       ??_C@_0BP@FGFGFLCA@Predelete?$CI?$CJ?5ERROR?5?9?$DO?5?$CFd?0?5ip?5?$CFs?$AA@ 10072c00     asxclass.obj
 0002:0000ac20       ??_C@_0BC@JKJLKAFA@asxclass?4cpp?3594?5?$AA@ 10072c20     asxclass.obj
 0002:0000ac34       ??_C@_0CA@NJOIJHPL@asxSystem?3?3CallbackThread?$CIvoid?$CJ?$AA@ 10072c34     asxclass.obj
 0002:0000ac54       ??_C@_0BC@JFKLNLGB@asxclass?4cpp?3657?5?$AA@ 10072c54     asxclass.obj
 0002:0000ac68       ??_C@_09MLGAJAED@undefined?$AA@ 10072c68     asxclass.obj
 0002:0000ac74       ??_C@_0BO@NIOMDKII@?$CF02X?4?$CF02X?4?$CF02X?4?$CF02X?4?$CF02X?4?$CF02X?$AA@ 10072c74     asxclass.obj
 0002:0000ac94       ??_C@_0DH@DIJBJNHK@asxAbstractAdapter?3?3Predelete?$CI?$CJ?5@ 10072c94     asxclass.obj
 0002:0000accc       ??_C@_0BD@LIFMEIOC@asxclass?4cpp?31192?5?$AA@ 10072ccc     asxclass.obj
 0002:0000ace0       ??_C@_05MKPGFCMM@ASI?$CFx?$AA@ 10072ce0     asxclass.obj
 0002:0000ace8       ??_C@_0BC@OCNMFFOH@AVB_MediaClock_In?$AA@ 10072ce8     asxclass.obj
 0002:0000acfc       ??_C@_02DKCKIIND@?$CFs?$AA@ 10072cfc     asxclass.obj
 0002:0000ad00       ??_C@_06CPDKGIA@?$CFs?5?$CF2d?$AA@ 10072d00     asxclass.obj
 0002:0000ad08       ??_C@_0BD@EAMHAEDB@AVB_MediaClock_Out?$AA@ 10072d08     asxclass.obj
 0002:0000ad1c       ??_C@_08NCNCPMHE@?$CFs?5?$CFd?0?$CFd?$AA@ 10072d1c     asxclass.obj
 0002:0000ad28       ??_C@_09BIPEJHEK@?$CFd?5?$CFs?5?$CFdL?$AA@ 10072d28     asxclass.obj
 0002:0000ad34       ??_C@_09MMLFKIJF@?$CFd?5?$CFs?5?$CFdR?$AA@ 10072d34     asxclass.obj
 0002:0000ad40       ??_C@_08DMLKDAGM@?$CFd?5?$CFs?5?$CFd?$AA@ 10072d40     asxclass.obj
 0002:0000ad4c       ??_C@_0BD@IKNPDDPA@LIBASX_DEBUG_LEVEL?$AA@ 10072d4c     asxdebug.obj
 0002:0000ad60       ??_C@_0BB@MOJIHPC@ASX32?5?$CF?920s?5?5?$CFs?6?$AA@ 10072d60     asxdebug.obj
 0002:0000ad78       ??_7asxSubSystemDSND@@6B@  10072d78     asxdsnd.obj
 0002:0000ad8c       ??_7asxAdapterDSND@@6B@    10072d8c     asxdsnd.obj
 0002:0000addc       ??_7asxMixerScannerDSND@@6B@ 10072ddc     asxdsnd.obj
 0002:0000ade8       ??_C@_06FMJGPDAJ@DSound?$AA@ 10072de8     asxdsnd.obj
 0002:0000adf4       ??_7asxPlayerDSND@@6B@     10072df4     asxdsndplay.obj
 0002:0000aea0       ??_7asxRecorderDSND@@6B@   10072ea0     asxdsndrec.obj
 0002:0000af50       ??_7asxMeter@@6B@          10072f50     asxhpi.obj
 0002:0000af80       ??_7asxVolume@@6B@         10072f80     asxhpi.obj
 0002:0000afb8       ??_7asxLevel@@6B@          10072fb8     asxhpi.obj
 0002:0000afe0       ??_7asxMux@@6B@            10072fe0     asxhpi.obj
 0002:0000b004       ??_7asxMode@@6B@           10073004     asxhpi.obj
 0002:0000b028       ??_7asxTuner@@6B@          10073028     asxhpi.obj
 0002:0000b09c       ??_7asxPad@@6B@            1007309c     asxhpi.obj
 0002:0000b0bc       ??_7asxSampleClock@@6B@    100730bc     asxhpi.obj
 0002:0000b0ec       ??_7asxAes3Tx@@6B@         100730ec     asxhpi.obj
 0002:0000b110       ??_7asxAes3Rx@@6B@         10073110     asxhpi.obj
 0002:0000b13c       ??_7asxGpio@@6B@           1007313c     asxhpi.obj
 0002:0000b168       ??_7asxVox@@6B@            10073168     asxhpi.obj
 0002:0000b190       ??_7asxBitStream@@6B@      10073190     asxhpi.obj
 0002:0000b1ac       ??_7asxMic@@6B@            100731ac     asxhpi.obj
 0002:0000b1d0       ??_7asxParametricEQ@@6B@   100731d0     asxhpi.obj
 0002:0000b1fc       ??_7asxCompander@@6B@      100731fc     asxhpi.obj
 0002:0000b250       ??_7asxCobranet@@6B@       10073250     asxhpi.obj
 0002:0000b2cc       ??_7asxCobranetContainer@@6B@ 100732cc     asxhpi.obj
 0002:0000b348       ??_7asxCobranetRx@@6B@     10073348     asxhpi.obj
 0002:0000b388       ??_7asxCobranetRxContainer@@6B@ 10073388     asxhpi.obj
 0002:0000b3c8       ??_7asxCobranetTx@@6B@     100733c8     asxhpi.obj
 0002:0000b410       ??_7asxCobranetTxContainer@@6B@ 10073410     asxhpi.obj
 0002:0000b458       ??_7asxToneDetector@@6B@   10073458     asxhpi.obj
 0002:0000b494       ??_7asxSilenceDetector@@6B@ 10073494     asxhpi.obj
 0002:0000b4d4       ??_7asxGenericControl@@6B@ 100734d4     asxhpi.obj
 0002:0000b4f0       ??_7asxBlock@@6B@          100734f0     asxhpi.obj
 0002:0000b53c       ??_7asxSubSystemHPI@@6B@   1007353c     asxhpi.obj
 0002:0000b550       ??_7asxAdapterHPI@@6B@     10073550     asxhpi.obj
 0002:0000b5a0       ??_7asxMixerScannerHPI@@6B@ 100735a0     asxhpi.obj
 0002:0000b5b0       ??_7asxAdapterHPIDuplicateIndex@@6B@ 100735b0     asxhpi.obj
 0002:0000b600       ??_7asxMixerScannerHPIDuplicateIndex@@6B@ 10073600     asxhpi.obj
 0002:0000b610       ??_7asxControlHPI@@6B@     10073610     asxhpi.obj
 0002:0000b62c       ??_7asxGenericHPI@@6B@     1007362c     asxhpi.obj
 0002:0000b648       ??_7asxVolumeHPI@@6B@      10073648     asxhpi.obj
 0002:0000b680       ??_7asxLevelHPI@@6B@       10073680     asxhpi.obj
 0002:0000b6a8       ??_7asxMeterHPI@@6B@       100736a8     asxhpi.obj
 0002:0000b6d8       ??_7asxMuxHPI@@6B@         100736d8     asxhpi.obj
 0002:0000b6fc       ??_7asxModeHPI@@6B@        100736fc     asxhpi.obj
 0002:0000b720       ??_7asxSampleClockHPI@@6B@ 10073720     asxhpi.obj
 0002:0000b750       ??_7asxTunerHPI@@6B@       10073750     asxhpi.obj
 0002:0000b7c4       ??_7asxAes3TxHPI@@6B@      100737c4     asxhpi.obj
 0002:0000b7e8       ??_7asxAesebuReceiverHPI@@6B@ 100737e8     asxhpi.obj
 0002:0000b814       ??_7asxGpioHPI@@6B@        10073814     asxhpi.obj
 0002:0000b840       ??_7asxVoxHPI@@6B@         10073840     asxhpi.obj
 0002:0000b868       ??_7asxMicHPI@@6B@         10073868     asxhpi.obj
 0002:0000b88c       ??_7asxParametricEqHPI@@6B@ 1007388c     asxhpi.obj
 0002:0000b8b8       ??_7asxCompanderHPI@@6B@   100738b8     asxhpi.obj
 0002:0000b90c       ??_7asxCompanderHPI_Legacy@@6B@ 1007390c     asxhpi.obj
 0002:0000b960       ??_7asxCobranetHPI@@6B@    10073960     asxhpi.obj
 0002:0000b9dc       ??_7asxCobranetRxHPI@@6B@  100739dc     asxhpi.obj
 0002:0000ba1c       ??_7asxCobranetTxHPI@@6B@  10073a1c     asxhpi.obj
 0002:0000ba64       ??_7asxToneDetectorHPI@@6B@ 10073a64     asxhpi.obj
 0002:0000baa0       ??_7asxSilenceDetectorHPI@@6B@ 10073aa0     asxhpi.obj
 0002:0000bae0       ??_7asxPadHPI@@6B@         10073ae0     asxhpi.obj
 0002:0000bb00       ??_7asxBlockPropertyHPI@@6B@ 10073b00     asxhpi.obj
 0002:0000bb20       ??_7asxBlockHPI@@6B@       10073b20     asxhpi.obj
 0002:0000bb68       ??_C@_03MNBMIKMN@HPI?$AA@  10073b68     asxhpi.obj
 0002:0000bb6c       ??_C@_0BK@JJBOAAMH@asxSubSystemHPI?3?3ReScan?$CI?$CJ?$AA@ 10073b6c     asxhpi.obj
 0002:0000bb88       ??_C@_05JMHIMMIL@Dummy?$AA@ 10073b88     asxhpi.obj
 0002:0000bb90       ??_C@_0BN@HBHMJKJO@DISCOVER?5?9?5about?5to?5scan?5?$CFd?5?$AA@ 10073b90     asxhpi.obj
 0002:0000bbb0       ??_C@_0BA@FNNGAELL@asxhpi?4cpp?3204?5?$AA@ 10073bb0     asxhpi.obj
 0002:0000bbc0       ??_C@_0CD@CEEIBHJN@DISCOVER?5?9?5added?5adapter?5index?5?$CF@ 10073bc0     asxhpi.obj
 0002:0000bbe4       ??_C@_0BA@PHNPMMDA@asxhpi?4cpp?3224?5?$AA@ 10073be4     asxhpi.obj
 0002:0000bbf8       ??_C@_0EL@CEBLANGC@asxSubSystemHPI?3?3ReScan?$CI?$CJ?5?9?5Dete@ 10073bf8     asxhpi.obj
 0002:0000bc44       ??_C@_04CGHINKND@?$CFc?$CFd?$AA@ 10073c44     asxhpi.obj
 0002:0000bc4c       ??_C@_0P@MAGPGIML@?$CF01d?4?$CF02d?4?$CF02d?$AA@ 10073c4c     asxhpi.obj
 0002:0000bc5c       ??_C@_05BDOHFCKE@About?$AA@ 10073c5c     asxhpi.obj
 0002:0000bc64       ??_C@_0L@EHKKKJAJ@Model?5Name?$AA@ 10073c64     asxhpi.obj
 0002:0000bc70       ??_C@_0P@JBINPBDL@ASI?$CFx?9?$CFc?$CFc?$CFc?$CFc?$AA@ 10073c70     asxhpi.obj
 0002:0000bc80       ??_C@_07HIAOKMAM@ASI?$CF04x?$AA@ 10073c80     asxhpi.obj
 0002:0000bc88       ??_C@_0CG@NHDDAEB@HPI_AdapterGetProperty?$CI?$CFd?0?$CFd?$CJ?5e?5@ 10073c88     asxhpi.obj
 0002:0000bcb0       ??_C@_0BA@KPFPAKKH@asxhpi?4cpp?3600?5?$AA@ 10073cb0     asxhpi.obj
 0002:0000bcc0       ??_C@_03JIDPIAJI@err?$AA@  10073cc0     asxhpi.obj
 0002:0000bcc4       ??_C@_09IPOHBKEM@?$CFd?5ID?5err?$AA@ 10073cc4     asxhpi.obj
 0002:0000bcd0       ??_C@_0BP@GJLFGODK@HPI_Universal_Info?$CI?$CJ?5error?5?$CFd?5?$AA@ 10073cd0     asxhpi.obj
 0002:0000bcf0       ??_C@_0BA@JCLKFCMP@asxhpi?4cpp?3914?5?$AA@ 10073cf0     asxhpi.obj
 0002:0000bd00       ??_C@_0DE@HJGNELBN@BLOCK?5?$CFs?0?5HPI?5control?5index?5?$CFd?0?5@ 10073d00     asxhpi.obj
 0002:0000bd34       ??_C@_0BA@KEKGMIMK@asxhpi?4cpp?3945?5?$AA@ 10073d34     asxhpi.obj
 0002:0000bd44       ??_C@_0M@KLCHMOKB@Diagnostics?$AA@ 10073d44     asxhpi.obj
 0002:0000bd50       ??_C@_08CLEKIHFG@LED?5Test?$AA@ 10073d50     asxhpi.obj
 0002:0000bd5c       ??_C@_0DD@PJGPBAGI@?$CFd?5?$DN?5HPI_Universal_Set?$CI?$CJ?5on?5Bloc@ 10073d5c     asxhpi.obj
 0002:0000bd90       ??_C@_0BA@OILLLFJJ@asxhpi?4cpp?3980?5?$AA@ 10073d90     asxhpi.obj
 0002:0000bda0       ??_C@_0CG@IDIIJBCL@DISCOVER?5?9?5scanning?5adapter?5inde@ 10073da0     asxhpi.obj
 0002:0000bdc8       ??_C@_0BB@MOAPHBMF@asxhpi?4cpp?31030?5?$AA@ 10073dc8     asxhpi.obj
 0002:0000bddc       ??_C@_0BI@PCEBPPAK@Error?5opening?5mixer?5?$CFd?6?$AA@ 10073ddc     asxhpi.obj
 0002:0000bdf4       ??_C@_0BB@ECOJDCPM@asxhpi?4cpp?31072?5?$AA@ 10073df4     asxhpi.obj
 0002:0000be08       ??_C@_07MLMHLOOL@Generic?$AA@ 10073e08     asxhpi.obj
 0002:0000be10       ??_C@_07NBCGADJA@Unknown?$AA@ 10073e10     asxhpi.obj
 0002:0000be18       ??_C@_0O@JNMGBHFK@?$CFs?5?9?$DO?5?$FL?$CFd?$FN?5?$CFs?$AA@ 10073e18     asxhpi.obj
 0002:0000be28       ??_C@_0BB@DPDJLLB@asxhpi?4cpp?33973?5?$AA@ 10073e28     asxhpi.obj
 0002:0000be3c       ??_C@_09CIFBDGJJ@?$CFs?5len?5?$CFd?$AA@ 10073e3c     asxhpi.obj
 0002:0000be48       ??_C@_0BB@IMHHEPJI@asxhpi?4cpp?34000?5?$AA@ 10073e48     asxhpi.obj
 0002:0000be5c       ??_C@_0BC@GKJIFHNI@?$CFs?5?9?$DO?5HMI?5read?5?$CFd?$AA@ 10073e5c     asxhpi.obj
 0002:0000be70       ??_C@_0BB@NAGIJHH@asxhpi?4cpp?34048?5?$AA@ 10073e70     asxhpi.obj
 0002:0000be84       ??_C@_0BF@MNNJLNPH@?5?5array?$FL?$CFd?$FN?5?$DN?50x?$CF08X?$AA@ 10073e84     asxhpi.obj
 0002:0000be9c       ??_C@_0BB@LLKJLPKK@asxhpi?4cpp?34050?5?$AA@ 10073e9c     asxhpi.obj
 0002:0000beb0       ??_C@_0BP@MAGCEHGE@?$CD?$CD?$CD?5HPI?5error?5?$CFd?0?5ASX?5error?5?$CFd?$AA@ 10073eb0     asxhpi.obj
 0002:0000bed0       ??_C@_0BB@LFLKOOBC@asxhpi?4cpp?34058?5?$AA@ 10073ed0     asxhpi.obj
 0002:0000bee4       ??_C@_0BD@FDLGJNGP@?$CFs?5?9?$DO?5HMI?5write?5?$CFd?$AA@ 10073ee4     asxhpi.obj
 0002:0000bef8       ??_C@_0BB@PDDJLOEL@asxhpi?4cpp?34093?5?$AA@ 10073ef8     asxhpi.obj
 0002:0000bf0c       ??_C@_0BB@PHLEMCPJ@asxhpi?4cpp?34095?5?$AA@ 10073f0c     asxhpi.obj
 0002:0000bf20       ??_C@_0BB@LDFBNIHB@asxhpi?4cpp?34103?5?$AA@ 10073f20     asxhpi.obj
 0002:0000bf34       ??_C@_0CK@DMCNPOKM@asxCobranetHPI?3?3GetMACAddress?$CI?$CJ?5@ 10073f34     asxhpi.obj
 0002:0000bf60       ??_C@_0BB@KHCPLFHE@asxhpi?4cpp?34136?5?$AA@ 10073f60     asxhpi.obj
 0002:0000bf74       ??_C@_0CE@FKEIBJBE@asxCobranetHPI?3?3GetIPAddress?$CI?$CJ?50@ 10073f74     asxhpi.obj
 0002:0000bf98       ??_C@_0BB@IDIGIAJP@asxhpi?4cpp?34157?5?$AA@ 10073f98     asxhpi.obj
 0002:0000bfac       ??_C@_0BN@PKMMMNDJ@asxCobranetHPI?3?3SetIPAddress?$AA@ 10073fac     asxhpi.obj
 0002:0000bfcc       ??_C@_0CD@MMKNJENH@asxCobranetHPI?3?3GetStaticIPAddre@ 10073fcc     asxhpi.obj
 0002:0000bff0       ??_C@_0CD@DGIHKCDP@asxCobranetHPI?3?3SetStaticIPAddre@ 10073ff0     asxhpi.obj
 0002:0000c014       ??_C@_0BP@FDNNCIEE@asxCobranetHPI?3?3GetDescription?$AA@ 10074014     asxhpi.obj
 0002:0000c034       ??_C@_0BI@KDFBBOHH@asxCobranetHPI?3?3GetName?$AA@ 10074034     asxhpi.obj
 0002:0000c04c       ??_C@_0BI@FLKACBKG@asxCobranetHPI?3?3SetName?$AA@ 1007404c     asxhpi.obj
 0002:0000c064       ??_C@_0BM@OHELPFF@asxCobranetHPI?3?3GetLocation?$AA@ 10074064     asxhpi.obj
 0002:0000c080       ??_C@_0BM@BGKGJNG@asxCobranetHPI?3?3SetLocation?$AA@ 10074080     asxhpi.obj
 0002:0000c09c       ??_C@_0CM@JILKENID@asxCobranetHPI?3?3GetErrorInfo?5cob@ 1007409c     asxhpi.obj
 0002:0000c0c8       ??_C@_0CN@NLIKALDO@asxCobranetHPI?3?3GetErrorInfo?5cob@ 100740c8     asxhpi.obj
 0002:0000c0f8       ??_C@_0DD@DKFJBJDO@asxCobranetHPI?3?3GetErrorInfo?5cob@ 100740f8     asxhpi.obj
 0002:0000c12c       ??_C@_0CI@KHBBEHNI@asxCobranetHPI?3?3GetLatencyAndSam@ 1007412c     asxhpi.obj
 0002:0000c154       ??_C@_0CI@LBHMKGLK@asxCobranetHPI?3?3SetLatencyAndSam@ 10074154     asxhpi.obj
 0002:0000c17c       ??_C@_0BP@EMJGNNEH@asxCobranetHPI?3?3GetPersistence?$AA@ 1007417c     asxhpi.obj
 0002:0000c19c       ??_C@_0BP@ICIICHGL@asxCobranetHPI?3?3SetPersistence?$AA@ 1007419c     asxhpi.obj
 0002:0000c1bc       ??_C@_0CF@CDPGCDDA@asxCobranetHPI?3?3GetConductorPrio@ 100741bc     asxhpi.obj
 0002:0000c1e4       ??_C@_0CF@HKOLDFGH@asxCobranetHPI?3?3SetConductorPrio@ 100741e4     asxhpi.obj
 0002:0000c20c       ??_C@_0CD@JJCAELOB@asxCobranetHPI?3?3GetConductorStat@ 1007420c     asxhpi.obj
 0002:0000c230       ??_C@_0DD@HOPALMHI@asxCobranetHPI?3?3GetSerialConfig?5@ 10074230     asxhpi.obj
 0002:0000c264       ??_C@_0DB@MCEBGPFH@asxCobranetHPI?3?3GetSerialConfig?5@ 10074264     asxhpi.obj
 0002:0000c298       ??_C@_0BM@EEHKAKEB@asxCobranetHPI?3?3GetIfStatus?$AA@ 10074298     asxhpi.obj
 0002:0000c2b4       ??_C@_0BM@GNDIOBGF@asxCobranetRxHPI?3?3GetStatus?$AA@ 100742b4     asxhpi.obj
 0002:0000c2d0       ??_C@_0CC@JNPGBPMC@asxCobranetRxHPI?3?3GetMinimumDela@ 100742d0     asxhpi.obj
 0002:0000c2f4       ??_C@_0CC@KPOAGNNL@asxCobranetRxHPI?3?3SetMinimumDela@ 100742f4     asxhpi.obj
 0002:0000c318       ??_C@_0CA@BNJLHPAJ@asxCobranetRxHPI?3?3GetChannelMap?$AA@ 10074318     asxhpi.obj
 0002:0000c338       ??_C@_0CA@GCIFMMHO@asxCobranetRxHPI?3?3SetChannelMap?$AA@ 10074338     asxhpi.obj
 0002:0000c358       ??_C@_0BM@LKOLEINM@asxCobranetRxHPI?3?3GetBundle?$AA@ 10074358     asxhpi.obj
 0002:0000c374       ??_C@_0BM@JEKOGJEO@asxCobranetRxHPI?3?3SetBundle?$AA@ 10074374     asxhpi.obj
 0002:0000c390       ??_C@_0BP@GNJCFNKH@asxCobranetRxHPI?3?3GetSourceMAC?$AA@ 10074390     asxhpi.obj
 0002:0000c3b0       ??_C@_0BM@MKAMFGGN@asxCobranetTxHPI?3?3GetStatus?$AA@ 100743b0     asxhpi.obj
 0002:0000c3cc       ??_C@_0BM@BNNPPPNE@asxCobranetTxHPI?3?3GetBundle?$AA@ 100743cc     asxhpi.obj
 0002:0000c3e8       ??_C@_0BM@DDJKNOEG@asxCobranetTxHPI?3?3SetBundle?$AA@ 100743e8     asxhpi.obj
 0002:0000c404       ??_C@_0CC@EHEMMNPO@asxCobranetTxHPI?3?3GetChannelCoun@ 10074404     asxhpi.obj
 0002:0000c428       ??_C@_0CC@HFFKLPOH@asxCobranetTxHPI?3?3SetChannelCoun@ 10074428     asxhpi.obj
 0002:0000c44c       ??_C@_0CA@OLKGHKMP@asxCobranetTxHPI?3?3GetChannelMap?$AA@ 1007444c     asxhpi.obj
 0002:0000c46c       ??_C@_0CA@JELIMJLI@asxCobranetTxHPI?3?3SetChannelMap?$AA@ 1007446c     asxhpi.obj
 0002:0000c48c       ??_C@_0BM@MIMEHPHA@asxCobranetTxHPI?3?3GetFormat?$AA@ 1007448c     asxhpi.obj
 0002:0000c4a8       ??_C@_0BM@OGIBFOOC@asxCobranetTxHPI?3?3SetFormat?$AA@ 100744a8     asxhpi.obj
 0002:0000c4c4       ??_C@_0CB@DDOJIEHE@asxCobranetTxHPI?3?3GetUnicastMode@ 100744c4     asxhpi.obj
 0002:0000c4e8       ??_C@_0CB@PNPHHOFI@asxCobranetTxHPI?3?3SetUnicastMode@ 100744e8     asxhpi.obj
 0002:0000c50c       __real@42c80000            1007450c     asxhpi.obj
 0002:0000c510       __xmm@0000044d000000010000045300000005 10074510     asxhpi.obj
 0002:0000c520       __xmm@0000044f000000030000044e00000002 10074520     asxhpi.obj
 0002:0000c530       __xmm@000004510000000a000004500000000b 10074530     asxhpi.obj
 0002:0000c540       __xmm@00000454000000060000045200000004 10074540     asxhpi.obj
 0002:0000c550       __xmm@00000456000000080000045500000007 10074550     asxhpi.obj
 0002:0000c560       __xmm@000004580000000c0000045700000009 10074560     asxhpi.obj
 0002:0000c570       __xmm@0000045a0000000e000004590000000d 10074570     asxhpi.obj
 0002:0000c580       __xmm@42c8000042c8000042c8000042c80000 10074580     asxhpi.obj
 0002:0000c594       ??_7asxPlayerHPI@@6B@      10074594     asxhpiplay.obj
 0002:0000c63c       ??_C@_0CK@EADBDKFP@Failed?5to?5allocate?5host?5buffer?5f@ 1007463c     asxhpiplay.obj
 0002:0000c668       ??_C@_0BD@CHBNGJEF@asxhpiplay?4cpp?361?5?$AA@ 10074668     asxhpiplay.obj
 0002:0000c67c       __real@3f800000            1007467c     asxhpiplay.obj
 0002:0000c680       __real@461c4000            10074680     asxhpiplay.obj
 0002:0000c688       ??_7asxPlayerHPIWithInt@@6B@ 10074688     asxhpiplayi.obj
 0002:0000c730       ??_C@_0BJ@OIPELHF@Error?5setting?5IRQ?5rate?4?6?$AA@ 10074730     asxhpiplayi.obj
 0002:0000c74c       ??_C@_0CB@LOPEGHEL@Set?5the?5IRQ?5rate?5to?5?$CFd?5samples?4?6@ 1007474c     asxhpiplayi.obj
 0002:0000c774       ??_7asxRecorderHPI@@6B@    10074774     asxhpirec.obj
 0002:0000c7e8       ??_C@_0CM@HMCBEKHE@Failed?5to?5allocate?5host?5buffer?5f@ 100747e8     asxhpirec.obj
 0002:0000c814       ??_C@_0BC@FJOOKHGF@asxhpirec?4cpp?351?5?$AA@ 10074814     asxhpirec.obj
 0002:0000c828       ??_C@_0BG@NHFNCNJI@ASX_Recorder?5stopping?$AA@ 10074828     asxhpirec.obj
 0002:0000c840       ??_C@_0BD@LBGOHMFI@asxhpirec?4cpp?3209?5?$AA@ 10074840     asxhpirec.obj
 0002:0000c854       ??_C@_0BF@LMECNGKH@ASX_Recorder?5data?5?$CFd?$AA@ 10074854     asxhpirec.obj
 0002:0000c86c       ??_C@_0BD@CFKDLNIF@asxhpirec?4cpp?3275?5?$AA@ 1007486c     asxhpirec.obj
 0002:0000c880       ??_C@_0BM@CPAILEEF@ASX_Recorder?5stop?5signalled?$AA@ 10074880     asxhpirec.obj
 0002:0000c89c       ??_C@_0BD@IBJJNADO@asxhpirec?4cpp?3303?5?$AA@ 1007489c     asxhpirec.obj
 0002:0000c8b4       ??_7asxRecorderHPIWithInt@@6B@ 100748b4     asxhpireci.obj
 0002:0000c928       ??_C@_0BE@KFBEHMHC@asxhpireci?4cpp?3106?5?$AA@ 10074928     asxhpireci.obj
 0002:0000c93c       ??_C@_0BE@DMEODIHJ@asxhpireci?4cpp?3170?5?$AA@ 1007493c     asxhpireci.obj
 0002:0000c950       ??_C@_04OHLCJCJC@PCM8?$AA@ 10074950     asxplay.obj
 0002:0000c958       ??_C@_05JICLOKAA@PCM16?$AA@ 10074958     asxplay.obj
 0002:0000c960       ??_C@_05KIFLDGNL@PCM24?$AA@ 10074960     asxplay.obj
 0002:0000c968       ??_C@_05PPMDPLGK@PCM32?$AA@ 10074968     asxplay.obj
 0002:0000c970       ??_C@_07OCCLKKPM@FLOAT32?$AA@ 10074970     asxplay.obj
 0002:0000c978       ??_C@_05PBIHOPBO@MPEG2?$AA@ 10074978     asxplay.obj
 0002:0000c980       ??_C@_03CPBCOLID@MP3?$AA@  10074980     asxplay.obj
 0002:0000c984       ??_C@_03GCLPHIFD@AC2?$AA@  10074984     asxplay.obj
 0002:0000c98c       ??_7asxCallbackObject@@6B@ 1007498c     asxplay.obj
 0002:0000c998       ??_7asxPlayer@@6B@         10074998     asxplay.obj
 0002:0000ca44       ??_7PlayerDoneCallback@@6B@ 10074a44     asxplay.obj
 0002:0000ca4c       ??_C@_01KDCPPGHE@r?$AA@    10074a4c     asxplay.obj
 0002:0000ca50       ??_C@_0DG@DHJKBNJI@asxPlayerFileList?3?3Open?$CIvoid?$CJ?0?5O@ 10074a50     asxplay.obj
 0002:0000ca88       ??_C@_0BB@PBPGKDE@asxplay?4cpp?3118?5?$AA@ 10074a88     asxplay.obj
 0002:0000caa0       ??_C@_0EA@IKNLEOGK@asxPlayerFileList?3?3Open?$CIvoid?$CJ?0?5C@ 10074aa0     asxplay.obj
 0002:0000cae0       ??_C@_0BB@MLIIGIFC@asxplay?4cpp?3253?5?$AA@ 10074ae0     asxplay.obj
 0002:0000caf4       ??_C@_0CM@JOALLPN@asxPlayerFileList?3?3Open?$CIvoid?$CJ?0?5m@ 10074af4     asxplay.obj
 0002:0000cb20       ??_C@_0BB@NJDNMHLM@asxplay?4cpp?3263?5?$AA@ 10074b20     asxplay.obj
 0002:0000cb34       ??_C@_04LGGJDDML@INIT?$AA@ 10074b34     asxplay.obj
 0002:0000cb3c       ??_C@_04DANIOFHI@OPEN?$AA@ 10074b3c     asxplay.obj
 0002:0000cb44       ??_C@_07DAMHHOOC@PREFILL?$AA@ 10074b44     asxplay.obj
 0002:0000cb4c       ??_C@_07NICPBLG@RUNNING?$AA@ 10074b4c     asxplay.obj
 0002:0000cb54       ??_C@_06EOENDFCC@PAUSED?$AA@ 10074b54     asxplay.obj
 0002:0000cb5c       ??_C@_07BHALEOME@DESTROY?$AA@ 10074b5c     asxplay.obj
 0002:0000cb64       ??_C@_04KANDKFIK@DONE?$AA@ 10074b64     asxplay.obj
 0002:0000cb6c       ??_C@_07CBDMFKJF@?$DMerror?$DO?$AA@ 10074b6c     asxplay.obj
 0002:0000cb74       ??_C@_0BG@LMADGKIJ@SetState?5asxPLAYER_?$CFs?$AA@ 10074b74     asxplay.obj
 0002:0000cb8c       ??_C@_0BB@LAGJIHME@asxplay?4cpp?3486?5?$AA@ 10074b8c     asxplay.obj
 0002:0000cba0       __real@408f400000000000    10074ba0     asxplay.obj
 0002:0000cbac       ??_7asxRecorder@@6B@       10074bac     asxrec.obj
 0002:0000cc20       ??_C@_0EA@LOCIIHKC@ASX_Recorder?5state?5change?5from?5a@ 10074c20     asxrec.obj
 0002:0000cc60       ??_C@_0BA@LHCPKJMB@asxrec?4cpp?3234?5?$AA@ 10074c60     asxrec.obj
 0002:0000cc70       ??_C@_01MCMALHOG@a?$AA@    10074c70     asxrec.obj
 0002:0000cc74       ??_C@_01NOFIACDB@w?$AA@    10074c74     asxrec.obj
 0002:0000cc78       ??_C@_0BI@LMEOEBCC@OpenWavFile?5failure?3?5?$CFs?$AA@ 10074c78     asxrec.obj
 0002:0000cc90       ??_C@_0BA@DGHOJLKG@asxrec?4cpp?3322?5?$AA@ 10074c90     asxrec.obj
 0002:0000cca0       ??_C@_04IBLEHOMF@?4wav?$AA@ 10074ca0     asxrec.obj
 0002:0000cca8       ??_C@_04IMEPLDLJ@?4WAV?$AA@ 10074ca8     asxrec.obj
 0002:0000ccb4       ??_7asxSubSystemSNMP@@6B@  10074cb4     asxsnmp.obj
 0002:0000ccc8       ??_7asxAdapterSNMP@@6B@    10074cc8     asxsnmp.obj
 0002:0000cd18       ??_7asxMixerScannerSNMP@@6B@ 10074d18     asxsnmp.obj
 0002:0000cd28       ??_7asxCobranetSNMP@@6B@   10074d28     asxsnmp.obj
 0002:0000cda4       ??_7asxCobranetTxSNMP@@6B@ 10074da4     asxsnmp.obj
 0002:0000cdec       ??_7asxCobranetRxSNMP@@6B@ 10074dec     asxsnmp.obj
 0002:0000ce2c       ??_7asxMixerScannerUnreachableSNMP@@6B@ 10074e2c     asxsnmp.obj
 0002:0000ce3c       ??_7asxCobranetUnreachableSNMP@@6B@ 10074e3c     asxsnmp.obj
 0002:0000ceb4       ??_C@_04PPFMNBDA@SNMP?$AA@ 10074eb4     asxsnmp.obj
 0002:0000cebc       ??_C@_0BJ@MKGDAEMA@CNDISCOEvent?5Connect?9?9?9?9?$AA@ 10074ebc     asxsnmp.obj
 0002:0000ced8       ??_C@_0BJ@DGJEDDLP@CNDISCOEvent?5Disonnect?9?9?$AA@ 10074ed8     asxsnmp.obj
 0002:0000cef4       ??_C@_0BJ@MKDJLHE@CNDISCOEvent?5Ip?5Change?9?9?$AA@ 10074ef4     asxsnmp.obj
 0002:0000cf10       ??_C@_0BJ@BGHJDMIM@CNDISCOEvent?5?9?9?9error?9?9?9?$AA@ 10074f10     asxsnmp.obj
 0002:0000cf2c       ??_C@_0CP@HMHOOCBJ@?$CFs?5?$CF02X?3?$CF02X?3?$CF02X?3?$CF02X?3?$CF02X?3?$CF02X@ 10074f2c     asxsnmp.obj
 0002:0000cf5c       ??_C@_0BB@MPLENCHI@asxsnmp?4cpp?3135?5?$AA@ 10074f5c     asxsnmp.obj
 0002:0000cf70       ??_C@_08HHDHFDEI@CobraNet?$AA@ 10074f70     asxsnmp.obj
 0002:0000cf7c       ??_C@_0BD@MNMJACNN@Found?5SNMP?5adapter?$AA@ 10074f7c     asxsnmp.obj
 0002:0000cf90       ??_C@_0BB@BBKPKMBN@asxsnmp?4cpp?3189?5?$AA@ 10074f90     asxsnmp.obj
 0002:0000cfa4       ??_C@_0BP@BJKJFPLD@Found?5unreachable?5SNMP?5adapter?$AA@ 10074fa4     asxsnmp.obj
 0002:0000cfc4       ??_C@_0BB@KBMLFICL@asxsnmp?4cpp?3194?5?$AA@ 10074fc4     asxsnmp.obj
 0002:0000cfd8       ??_C@_0P@EBPHHFGI@00?400?400?400?400?$AA@ 10074fd8     asxsnmp.obj
 0002:0000cfe8       ??_C@_0CC@MGLHIJBJ@Found?5SNMP?5adapter?5via?5HPI?5or?5UD@ 10074fe8     asxsnmp.obj
 0002:0000d00c       ??_C@_0BB@IONPGKED@asxsnmp?4cpp?3230?5?$AA@ 1007500c     asxsnmp.obj
 0002:0000d020       ??_C@_0CO@KIECLLIE@Found?5unreachable?5SNMP?5adapter?5v@ 10075020     asxsnmp.obj
 0002:0000d050       ??_C@_0BB@IIBEKIKI@asxsnmp?4cpp?3235?5?$AA@ 10075050     asxsnmp.obj
 0002:0000d064       ??_C@_0BB@CAFHDGMO@?9?$CK?$CK?$CK?$CKm?9?$CK?$CK?$CK?$CK?$CK?$CK?$CK?$CKm?$AA@ 10075064     asxsnmp.obj
 0002:0000d078       ??_C@_0CJ@BNEBFDIP@CobraNetNode?5count?5elements?5resu@ 10075078     asxsnmp.obj
 0002:0000d0a4       ??_C@_0BB@LFHEIBBI@asxsnmp?4cpp?3335?5?$AA@ 100750a4     asxsnmp.obj
 0002:0000d0b8       ??_C@_0BB@CBLLNGLK@asxsnmp?4cpp?3457?5?$AA@ 100750b8     asxsnmp.obj
 0002:0000d0cc       ??_C@_07NFICAEG@ASI2202?$AA@ 100750cc     asxsnmp.obj
 0002:0000d0d4       ??_C@_05MHBLNJCL@ASI63?$AA@ 100750d4     asxsnmp.obj
 0002:0000d0dc       ??_C@_05MFFNGHHC@ASI53?$AA@ 100750dc     asxsnmp.obj
 0002:0000d0e4       ??_C@_0BM@DFFLIBOF@?$DMUnreachable?5CobraNet?5Node?$DO?$AA@ 100750e4     asxsnmp.obj
 0002:0000d104       ??_7asxLevelTR800@@6B@     10075104     asxtr800.obj
 0002:0000d12c       ??_7asxMeterTR800@@6B@     1007512c     asxtr800.obj
 0002:0000d15c       ??_7asxGpioTR800@@6B@      1007515c     asxtr800.obj
 0002:0000d188       ??_7asxBlockTR800OptoMode@@6B@ 10075188     asxtr800.obj
 0002:0000d1d4       ??_7asxBlockTR800Status@@6B@ 100751d4     asxtr800.obj
 0002:0000d21c       ??_C@_0BM@JILHKBCK@ASI2202?5?9?5WMRST_OFST?5failed?$AA@ 1007521c     asxtr800.obj
 0002:0000d238       ??_C@_0BC@CONDHKFD@asxtr800?4cpp?3244?5?$AA@ 10075238     asxtr800.obj
 0002:0000d24c       ??_C@_06PMAGBHAK@Action?$AA@ 1007524c     asxtr800.obj
 0002:0000d254       ??_C@_0BA@DEOECKLM@MIC?5to?5LINEOUTS?$AA@ 10075254     asxtr800.obj
 0002:0000d264       ??_C@_00CNPNBAHC@?$AA@     10075264     asxtr800.obj
 0002:0000d268       ??_C@_05CIGKLKEO@Opto1?$AA@ 10075268     asxtr800.obj
 0002:0000d270       ??_C@_05DEHOJIN@Opto2?$AA@ 10075270     asxtr800.obj
 0002:0000d278       ??_C@_06PGDKHFME@Status?$AA@ 10075278     asxtr800.obj
 0002:0000d280       ??_C@_02GIPFHKNO@OK?$AA@   10075280     asxtr800.obj
 0002:0000d284       ??_C@_05MBDEGLCK@ERROR?$AA@ 10075284     asxtr800.obj
 0002:0000d28c       ??_C@_0P@GELPEJGF@Initialization?$AA@ 1007528c     asxtr800.obj
 0002:0000d29c       __real@41a00000            1007529c     asxtr800.obj
 0002:0000d2a0       __real@4efffe00            100752a0     asxtr800.obj
 0002:0000d2a4       __real@c0c00000            100752a4     asxtr800.obj
 0002:0000d548       ??_7asxSubSystemWAVE@@6B@  10075548     asxwave.obj
 0002:0000d55c       ??_7asxAdapterWAVE@@6B@    1007555c     asxwave.obj
 0002:0000d5ac       ??_7asxMixerScannerWAVE@@6B@ 100755ac     asxwave.obj
 0002:0000d5bc       ??_7asxVolumeWAVE@@6B@     100755bc     asxwave.obj
 0002:0000d5f4       ??_7asxMeterWAVE@@6B@      100755f4     asxwave.obj
 0002:0000d624       ??_7asxLevelWAVE@@6B@      10075624     asxwave.obj
 0002:0000d64c       ??_7asxMuxWAVE@@6B@        1007564c     asxwave.obj
 0002:0000d670       ??_7asxModeWAVE@@6B@       10075670     asxwave.obj
 0002:0000d694       ??_7asxTunerWAVE@@6B@      10075694     asxwave.obj
 0002:0000d708       ??_7asxCobranetWAVE@@6B@   10075708     asxwave.obj
 0002:0000d784       ??_7asxToneDetectorWAVE@@6B@ 10075784     asxwave.obj
 0002:0000d7c0       ??_7asxSilenceDetectorWAVE@@6B@ 100757c0     asxwave.obj
 0002:0000d7fc       ??_C@_04HIICAAFP@Wave?$AA@ 100757fc     asxwave.obj
 0002:0000d804       ??_C@_07LGGAIHJM@?$CFd?4?$CF02d?$AA@ 10075804     asxwave.obj
 0002:0000d80c       ??_C@_06LLDEHLAM@?5?9?5ASI?$AA@ 1007580c     asxwave.obj
 0002:0000d814       ??_C@_0BP@EGDHPCGM@MIXERCONTROL_CONTROLTYPE_FADER?$AA@ 10075814     asxwave.obj
 0002:0000d834       ??_C@_0BP@BIIBNKHI@MIXERCONTROL_CONTROLTYPE_ONOFF?$AA@ 10075834     asxwave.obj
 0002:0000d854       ??_C@_0BG@OKEGNGAM@Tuner?5frequency?5?$CIkHz?$CJ?$AA@ 10075854     asxwave.obj
 0002:0000d86c       ??_C@_0L@CPAKKAKP@IP?5address?$AA@ 1007586c     asxwave.obj
 0002:0000d878       ??_C@_0N@PKAGLIJN@Ethernet?5MAC?$AA@ 10075878     asxwave.obj
 0002:0000d888       ??_C@_0CC@HHKDOIMH@MIXERCONTROL_CONTROLTYPE_UNSIGNE@ 10075888     asxwave.obj
 0002:0000d8ac       ??_C@_0CB@PLDFPMOD@MIXERCONTROL_CONTROLTYPE_BOOLEAN@ 100758ac     asxwave.obj
 0002:0000d8d0       ??_C@_0N@JCEFFMCM@Channel?5mode?$AA@ 100758d0     asxwave.obj
 0002:0000d8e0       ??_C@_0N@NAHLLDP@Sample?5Clock?$AA@ 100758e0     asxwave.obj
 0002:0000d8f0       ??_C@_0BH@BJLDAGDC@Clock?5Source?5Selection?$AA@ 100758f0     asxwave.obj
 0002:0000d908       ??_C@_0L@BPDOGCHG@Tuner?5band?$AA@ 10075908     asxwave.obj
 0002:0000d914       ??_C@_0CG@CFFJJNGL@MIXERCONTROL_CONTROLTYPE_SINGLES@ 10075914     asxwave.obj
 0002:0000d93c       ??_C@_0BE@HNIOGFLL@Gain?5Volume?5Control?$AA@ 1007593c     asxwave.obj
 0002:0000d950       ??_C@_0CC@ODBPIJAF@MIXERCONTROL_CONTROLTYPE_DECIBEL@ 10075950     asxwave.obj
 0002:0000d974       ??_C@_0BO@GPKEHHNO@MIXERCONTROL_CONTROLTYPE_MUTE?$AA@ 10075974     asxwave.obj
 0002:0000d994       ??_C@_07EKENHEGE@RFLevel?$AA@ 10075994     asxwave.obj
 0002:0000d99c       ??_C@_0CA@IACKOJKA@MIXERCONTROL_CONTROLTYPE_SIGNED?$AA@ 1007599c     asxwave.obj
 0002:0000d9bc       ??_C@_0CI@GCPKFDHL@MIXERCONTROL_CONTROLTYPE_MULTIPL@ 100759bc     asxwave.obj
 0002:0000d9e4       ??_C@_0CD@OFINONDM@ASI_MIXERCONTROL_CONTROLTYPE_NVM@ 100759e4     asxwave.obj
 0002:0000da08       ??_C@_0CF@IHBHGDGO@ASI_MIXERCONTROL_CONTROLTYPE_AES@ 10075a08     asxwave.obj
 0002:0000da30       ??_C@_0CF@FGGLMOIA@ASI_MIXERCONTROL_CONTROLTYPE_AES@ 10075a30     asxwave.obj
 0002:0000da58       ??_C@_0CF@FCOGLCDC@ASI_MIXERCONTROL_CONTROLTYPE_AES@ 10075a58     asxwave.obj
 0002:0000da80       ??_C@_0CI@FFDFCAIE@ASI_MIXERCONTROL_CONTROLTYPE_DIG@ 10075a80     asxwave.obj
 0002:0000daa8       ??_C@_0CJ@BEPPJAE@ASI_MIXERCONTROL_CONTROLTYPE_DIG@ 10075aa8     asxwave.obj
 0002:0000dad4       ??_C@_0CH@FAIEDNAF@ASI_MIXERCONTROL_CONTROLTYPE_DSP@ 10075ad4     asxwave.obj
 0002:0000dafc       ??_C@_0DA@LOFNPJAH@ASI_MIXERCONTROL_CONTROLTYPE_ADA@ 10075afc     asxwave.obj
 0002:0000db2c       ??_C@_0CL@NILPAADA@ASI_MIXERCONTROL_CONTROLTYPE_PAR@ 10075b2c     asxwave.obj
 0002:0000db58       ??_C@_0CH@PPFKKBCM@ASI_MIXERCONTROL_CONTROLTYPE_COM@ 10075b58     asxwave.obj
 0002:0000db80       __real@4024000000000000    10075b80     asxwave.obj
 0002:0000db88       __real@4034000000000000    10075b88     asxwave.obj
 0002:0000db90       __real@40efffe000000000    10075b90     asxwave.obj
 0002:0000db98       __real@c2c80000            10075b98     asxwave.obj
 0002:0000dba0       __xmm@00000000000001c6000001c500000199 10075ba0     asxwave.obj
 0002:0000dbb0       __xmm@00000194000001c400000193000001c3 10075bb0     asxwave.obj
 0002:0000dbc0       __xmm@00000198000001960000019700000195 10075bc0     asxwave.obj
 0002:0000dbd0       __xmm@000001c7000001c20000019200000191 10075bd0     asxwave.obj
 0002:0000dbe4       ??_7asxPlayerWAVE@@6B@     10075be4     asxwaveplay.obj
 0002:0000dc90       ??_7asxRecorderWAVE@@6B@   10075c90     asxwaverec.obj
 0002:0000dd04       ??_C@_0P@BPIMIDCF@sysDescription?$AA@ 10075d04     cobranet.obj
 0002:0000dd14       ??_C@_07HAJIONKN@sysName?$AA@ 10075d14     cobranet.obj
 0002:0000dd1c       ??_C@_0M@PFPNMEEI@sysLocation?$AA@ 10075d1c     cobranet.obj
 0002:0000dd28       ??_C@_0L@FGNCKDGJ@sysContact?$AA@ 10075d28     cobranet.obj
 0002:0000dd34       ??_C@_0BF@NIPGLIJC@firmwareMajorVersion?$AA@ 10075d34     cobranet.obj
 0002:0000dd4c       ??_C@_0BF@GOCDLNOO@firmwareMinorVersion?$AA@ 10075d4c     cobranet.obj
 0002:0000dd64       ??_C@_0BD@LIJIDKIJ@flashPersistEnable?$AA@ 10075d64     cobranet.obj
 0002:0000dd78       ??_C@_0BA@LEKNOJJB@modeRateControl?$AA@ 10075d78     cobranet.obj
 0002:0000dd88       ??_C@_0N@HCFEOBFF@errorDisplay?$AA@ 10075d88     cobranet.obj
 0002:0000dd98       ??_C@_0L@CMHLCLKC@errorCount?$AA@ 10075d98     cobranet.obj
 0002:0000dda4       ??_C@_09CDPCPKBA@errorLast?$AA@ 10075da4     cobranet.obj
 0002:0000ddb0       ??_C@_0P@INPEDJBA@modeRateStatus?$AA@ 10075db0     cobranet.obj
 0002:0000ddc0       ??_C@_0BA@OPAMMPCC@conductorStatus?$AA@ 10075dc0     cobranet.obj
 0002:0000ddd0       ??_C@_0BC@CJPEJGKI@conductorPriority?$AA@ 10075dd0     cobranet.obj
 0002:0000dde4       ??_C@_0P@OCBJAPHF@ipmonCurrentIP?$AA@ 10075de4     cobranet.obj
 0002:0000ddf4       ??_C@_0O@KKDCPNJL@ipmonStaticIP?$AA@ 10075df4     cobranet.obj
 0002:0000de04       ??_C@_0N@JGMFCKOM@serialFormat?$AA@ 10075e04     cobranet.obj
 0002:0000de14       ??_C@_0L@HFHCPCDB@serialBaud?$AA@ 10075e14     cobranet.obj
 0002:0000de20       ??_C@_0O@GFOAHOMD@serialPPeriod?$AA@ 10075e20     cobranet.obj
 0002:0000de30       ??_C@_0M@OPMAMNCD@serialRxMAC?$AA@ 10075e30     cobranet.obj
 0002:0000de3c       ??_C@_0M@DJJJCODO@serialTxMAC?$AA@ 10075e3c     cobranet.obj
 0002:0000de48       ??_C@_0BB@OCBPDNP@serialTxPriority?$AA@ 10075e48     cobranet.obj
 0002:0000de5c       ??_C@_08IIHGAPFB@txBundle?$AA@ 10075e5c     cobranet.obj
 0002:0000de68       ??_C@_0L@CMIPMADJ@txPriority?$AA@ 10075e68     cobranet.obj
 0002:0000de74       ??_C@_0L@ELAOIHKN@txSubCount?$AA@ 10075e74     cobranet.obj
 0002:0000de80       ??_C@_0N@GJFKGBIG@txMaxUnicast?$AA@ 10075e80     cobranet.obj
 0002:0000de90       ??_C@_0O@BGBGLFIB@txUnicastMode?$AA@ 10075e90     cobranet.obj
 0002:0000dea0       ??_C@_08GOHIOANJ@txSubMap?$AA@ 10075ea0     cobranet.obj
 0002:0000deac       ??_C@_0M@LDPFAOC@txSubFormat?$AA@ 10075eac     cobranet.obj
 0002:0000deb8       ??_C@_0L@EEHGPJPJ@txPosition?$AA@ 10075eb8     cobranet.obj
 0002:0000dec4       ??_C@_0L@DEKDAFKO@txDropouts?$AA@ 10075ec4     cobranet.obj
 0002:0000ded0       ??_C@_0M@MNIOLMOO@txReceivers?$AA@ 10075ed0     cobranet.obj
 0002:0000dedc       ??_C@_08PLGMHGNL@rxBundle?$AA@ 10075edc     cobranet.obj
 0002:0000dee8       ??_C@_0M@FKMEEGJN@rxSourceMAC?$AA@ 10075ee8     cobranet.obj
 0002:0000def4       ??_C@_0L@MEDKAKHK@rxPriority?$AA@ 10075ef4     cobranet.obj
 0002:0000df00       ??_C@_08CMLPNPGC@rxStatus?$AA@ 10075f00     cobranet.obj
 0002:0000df0c       ??_C@_0L@NMBGMPON@rxDropouts?$AA@ 10075f0c     cobranet.obj
 0002:0000df18       ??_C@_07KICMLDGD@rxDelay?$AA@ 10075f18     cobranet.obj
 0002:0000df20       ??_C@_0L@OPFLJDGB@rxMinDelay?$AA@ 10075f20     cobranet.obj
 0002:0000df2c       ??_C@_08BNGCJJFD@rxSubMap?$AA@ 10075f2c     cobranet.obj
 0002:0000df38       ??_C@_0BC@GLJGEOMI@rxSubChannelEntry?$AA@ 10075f38     cobranet.obj
 0002:0000df4c       ??_C@_0M@LHIHJLMB@audioMeters?$AA@ 10075f4c     cobranet.obj
 0002:0000df58       ??_C@_0P@PBNJHJED@stdUserInteger?$AA@ 10075f58     cobranet.obj
 0002:0000df68       ??_C@_0BC@IMJFHLLL@00?400?400?400?400?400?$AA@ 10075f68     cobranet.obj
 0002:0000df7c       ??_C@_0M@OHKMKKDH@Description?$AA@ 10075f7c     mibtbl.obj
 0002:0000df88       ??_C@_08CMHNALBL@ObjectID?$AA@ 10075f88     mibtbl.obj
 0002:0000df94       ??_C@_06MLGEPNED@UpTime?$AA@ 10075f94     mibtbl.obj
 0002:0000df9c       ??_C@_07PMMFKIFM@Contact?$AA@ 10075f9c     mibtbl.obj
 0002:0000dfa4       ??_C@_04FABLJDN@Name?$AA@  10075fa4     mibtbl.obj
 0002:0000dfac       ??_C@_08KDOEBHGA@Location?$AA@ 10075fac     mibtbl.obj
 0002:0000dfb8       ??_C@_08JLBBHJMM@Services?$AA@ 10075fb8     mibtbl.obj
 0002:0000dfc4       ??_C@_03PIADFGHL@sys?$AA@  10075fc4     mibtbl.obj
 0002:0000dfc8       ??_C@_06IONACMBM@Number?$AA@ 10075fc8     mibtbl.obj
 0002:0000dfd0       ??_C@_05FNNGFGLF@Index?$AA@ 10075fd0     mibtbl.obj
 0002:0000dfd8       ??_C@_05KFDEIPGE@Descr?$AA@ 10075fd8     mibtbl.obj
 0002:0000dfe0       ??_C@_04KOACHJEN@Type?$AA@ 10075fe0     mibtbl.obj
 0002:0000dfe8       ??_C@_03LGHFONDM@Mtu?$AA@  10075fe8     mibtbl.obj
 0002:0000dfec       ??_C@_05HOIAGEJD@Speed?$AA@ 10075fec     mibtbl.obj
 0002:0000dff4       ??_C@_0M@EFNAOKMI@PhysAddress?$AA@ 10075ff4     mibtbl.obj
 0002:0000e000       ??_C@_0M@EKPAHIEG@AdminStatus?$AA@ 10076000     mibtbl.obj
 0002:0000e00c       ??_C@_0L@ELKJCBOB@OperStatus?$AA@ 1007600c     mibtbl.obj
 0002:0000e018       ??_C@_0L@CMMGLEFG@LastChange?$AA@ 10076018     mibtbl.obj
 0002:0000e024       ??_C@_08MFMFDPGH@InOctets?$AA@ 10076024     mibtbl.obj
 0002:0000e030       ??_C@_0M@MDDNIJJG@InUcastPkts?$AA@ 10076030     mibtbl.obj
 0002:0000e03c       ??_C@_0N@GHLBCPJI@InNUcastPkts?$AA@ 1007603c     mibtbl.obj
 0002:0000e04c       ??_C@_0L@MHMBHMEA@InDiscards?$AA@ 1007604c     mibtbl.obj
 0002:0000e058       ??_C@_08ENEPNIGB@InErrors?$AA@ 10076058     mibtbl.obj
 0002:0000e064       ??_C@_0BA@OPAFGAFE@InUnknownProtos?$AA@ 10076064     mibtbl.obj
 0002:0000e074       ??_C@_09IKIJABLH@OutOctets?$AA@ 10076074     mibtbl.obj
 0002:0000e080       ??_C@_0N@HABLKKCP@OutUcastPkts?$AA@ 10076080     mibtbl.obj
 0002:0000e090       ??_C@_0O@NFLPACJD@OutNUcastPkts?$AA@ 10076090     mibtbl.obj
 0002:0000e0a0       ??_C@_0M@IHJIOLLI@OutDiscards?$AA@ 100760a0     mibtbl.obj
 0002:0000e0ac       ??_C@_09CADOGLB@OutErrors?$AA@ 100760ac     mibtbl.obj
 0002:0000e0b8       ??_C@_07CFFAAOJA@OutQLen?$AA@ 100760b8     mibtbl.obj
 0002:0000e0c0       ??_C@_08DHCLFMFE@Spedific?$AA@ 100760c0     mibtbl.obj
 0002:0000e0cc       ??_C@_02HEBPBKGD@if?$AA@   100760cc     mibtbl.obj
 0002:0000e0d0       ??_C@_0L@NLOLCIEN@Forwarding?$AA@ 100760d0     mibtbl.obj
 0002:0000e0dc       ??_C@_0L@EIDNNLHD@DefaultTTL?$AA@ 100760dc     mibtbl.obj
 0002:0000e0e8       ??_C@_0L@EAODJLIG@InReceives?$AA@ 100760e8     mibtbl.obj
 0002:0000e0f4       ??_C@_0M@KKDMDMDL@InHdrErrors?$AA@ 100760f4     mibtbl.obj
 0002:0000e100       ??_C@_0N@MICJINKN@InAddrErrors?$AA@ 10076100     mibtbl.obj
 0002:0000e110       ??_C@_0O@CJCCOJGE@ForwDatagrams?$AA@ 10076110     mibtbl.obj
 0002:0000e120       ??_C@_0L@KHMGFNDI@InDelivers?$AA@ 10076120     mibtbl.obj
 0002:0000e12c       ??_C@_0M@BMOHFHHG@OutRequests?$AA@ 1007612c     mibtbl.obj
 0002:0000e138       ??_C@_0M@HLBIJOFL@OutNoRoutes?$AA@ 10076138     mibtbl.obj
 0002:0000e144       ??_C@_0N@FIHCNAGA@ReasmTimeout?$AA@ 10076144     mibtbl.obj
 0002:0000e154       ??_C@_0L@IIBJBEIC@ReasmReqds?$AA@ 10076154     mibtbl.obj
 0002:0000e160       ??_C@_08KHCGKHMD@ReasmOKs?$AA@ 10076160     mibtbl.obj
 0002:0000e16c       ??_C@_0L@HOGANMAH@ReasmFails?$AA@ 1007616c     mibtbl.obj
 0002:0000e178       ??_C@_07FNMIFNCD@FragOKs?$AA@ 10076178     mibtbl.obj
 0002:0000e180       ??_C@_09HNHGMOAH@FragFails?$AA@ 10076180     mibtbl.obj
 0002:0000e18c       ??_C@_0M@HFMAJDLM@FragCreates?$AA@ 1007618c     mibtbl.obj
 0002:0000e198       ??_C@_09MFMFPGHM@AdEntAddr?$AA@ 10076198     mibtbl.obj
 0002:0000e1a4       ??_C@_0N@LDOFBNGD@AdEntIfIndex?$AA@ 100761a4     mibtbl.obj
 0002:0000e1b4       ??_C@_0N@PINHCBCC@AdEntNetMask?$AA@ 100761b4     mibtbl.obj
 0002:0000e1c4       ??_C@_0P@MMLEMGPN@AdEntBcastAddr?$AA@ 100761c4     mibtbl.obj
 0002:0000e1d4       ??_C@_0BC@DNAJCEFD@AdEntReasmMaxSize?$AA@ 100761d4     mibtbl.obj
 0002:0000e1e8       ??_C@_0BA@OLHKMBLN@RoutingDiscards?$AA@ 100761e8     mibtbl.obj
 0002:0000e1f8       ??_C@_02GIIHKPLE@ip?$AA@   100761f8     mibtbl.obj
 0002:0000e1fc       ??_C@_0M@KDLEINKE@InDatagrams?$AA@ 100761fc     mibtbl.obj
 0002:0000e208       ??_C@_07FKAEKGIA@NoPorts?$AA@ 10076208     mibtbl.obj
 0002:0000e210       ??_C@_0N@BAJCKOBN@OutDatagrams?$AA@ 10076210     mibtbl.obj
 0002:0000e220       ??_C@_03OCLLGKEH@udp?$AA@  10076220     mibtbl.obj
 0002:0000e224       ??_C@_06CCACLHB@InPkts?$AA@ 10076224     mibtbl.obj
 0002:0000e22c       ??_C@_07MHFNBFPM@OutPkts?$AA@ 1007622c     mibtbl.obj
 0002:0000e234       ??_C@_0O@HOIOIKMC@InBadVersions?$AA@ 10076234     mibtbl.obj
 0002:0000e244       ??_C@_0BE@GJCLNAFH@InBadCommunityNames?$AA@ 10076244     mibtbl.obj
 0002:0000e258       ??_C@_0BD@BLLFFEPN@InBadCommunityUses?$AA@ 10076258     mibtbl.obj
 0002:0000e26c       ??_C@_0P@OHKBEAKA@InASNParseErrs?$AA@ 1007626c     mibtbl.obj
 0002:0000e27c       ??_C@_09JCNMNJFK@InTooBigs?$AA@ 1007627c     mibtbl.obj
 0002:0000e288       ??_C@_0O@DDKIHJLN@InNoSuchNames?$AA@ 10076288     mibtbl.obj
 0002:0000e298       ??_C@_0M@GHDEAMJK@InBadValues?$AA@ 10076298     mibtbl.obj
 0002:0000e2a4       ??_C@_0M@BFCBBDEG@InReadOnlys?$AA@ 100762a4     mibtbl.obj
 0002:0000e2b0       ??_C@_09CABBAOGM@InGenErrs?$AA@ 100762b0     mibtbl.obj
 0002:0000e2bc       ??_C@_0P@ODMCKNCJ@InTotalReqVars?$AA@ 100762bc     mibtbl.obj
 0002:0000e2cc       ??_C@_0P@HPKFDMAE@InTotalSetVars?$AA@ 100762cc     mibtbl.obj
 0002:0000e2dc       ??_C@_0O@FIJIELE@InGetRequests?$AA@ 100762dc     mibtbl.obj
 0002:0000e2ec       ??_C@_0L@FBGNJIHI@InGetNexts?$AA@ 100762ec     mibtbl.obj
 0002:0000e2f8       ??_C@_0O@KJHFCDH@InSetRequests?$AA@ 100762f8     mibtbl.obj
 0002:0000e308       ??_C@_0P@GEJBGLNA@InGetResponses?$AA@ 10076308     mibtbl.obj
 0002:0000e318       ??_C@_07LAPCOFKF@InTraps?$AA@ 10076318     mibtbl.obj
 0002:0000e320       ??_C@_0L@BEEAEHLA@OutTooBigs?$AA@ 10076320     mibtbl.obj
 0002:0000e32c       ??_C@_0P@KEMIKOBI@OutNoSuchNames?$AA@ 1007632c     mibtbl.obj
 0002:0000e33c       ??_C@_0N@NEBCCPCD@OutBadValues?$AA@ 1007633c     mibtbl.obj
 0002:0000e34c       ??_C@_0L@KGINJAIG@OutGenErrs?$AA@ 1007634c     mibtbl.obj
 0002:0000e358       ??_C@_0P@JCOJFDBB@OutGetRequests?$AA@ 10076358     mibtbl.obj
 0002:0000e368       ??_C@_0M@BBDEAPIA@OutGetNexts?$AA@ 10076368     mibtbl.obj
 0002:0000e374       ??_C@_0P@JNPHIFJC@OutSetRequests?$AA@ 10076374     mibtbl.obj
 0002:0000e384       ??_C@_0BA@MCLKFMGA@OutGetResponses?$AA@ 10076384     mibtbl.obj
 0002:0000e394       ??_C@_08CDDOGHAG@OutTraps?$AA@ 10076394     mibtbl.obj
 0002:0000e3a0       ??_C@_0BC@IEGLKANK@EnableAuthenTraps?$AA@ 100763a0     mibtbl.obj
 0002:0000e3b4       ??_C@_0M@MAECCBJA@SilentDrops?$AA@ 100763b4     mibtbl.obj
 0002:0000e3c0       ??_C@_0L@LPJIMJNP@ProxyDrops?$AA@ 100763c0     mibtbl.obj
 0002:0000e3cc       ??_C@_04DDGGDDEI@snmp?$AA@ 100763cc     mibtbl.obj
 0002:0000e3d4       ??_C@_0BA@JAAMMJFI@ProtocolVersion?$AA@ 100763d4     mibtbl.obj
 0002:0000e3e4       ??_C@_0N@LJJLMPLG@MajorVersion?$AA@ 100763e4     mibtbl.obj
 0002:0000e3f4       ??_C@_0N@PEOMKMK@MinorVersion?$AA@ 100763f4     mibtbl.obj
 0002:0000e404       ??_C@_0M@FKHJGCEO@BootVersion?$AA@ 10076404     mibtbl.obj
 0002:0000e410       ??_C@_05DDKCBCFF@MfgId?$AA@ 10076410     mibtbl.obj
 0002:0000e418       ??_C@_0N@LKCDALMJ@MfgProductId?$AA@ 10076418     mibtbl.obj
 0002:0000e428       ??_C@_0L@CBNLFPMK@MfgVersion?$AA@ 10076428     mibtbl.obj
 0002:0000e434       ??_C@_07EKAIBOKF@Restart?$AA@ 10076434     mibtbl.obj
 0002:0000e43c       ??_C@_08DGIDLCPF@Unknown1?$AA@ 1007643c     mibtbl.obj
 0002:0000e448       ??_C@_08BNKOOBDG@Unknown2?$AA@ 10076448     mibtbl.obj
 0002:0000e454       ??_C@_08ELFNAHH@Unknown3?$AA@ 10076454     mibtbl.obj
 0002:0000e460       ??_C@_08LBCBPKAM@firmware?$AA@ 10076460     mibtbl.obj
 0002:0000e46c       ??_C@_09CNMMJHCC@TotalSize?$AA@ 1007646c     mibtbl.obj
 0002:0000e478       ??_C@_0L@EMHLPHDJ@SectorSize?$AA@ 10076478     mibtbl.obj
 0002:0000e484       ??_C@_0BA@JBBGKBJK@PersistSequence?$AA@ 10076484     mibtbl.obj
 0002:0000e494       ??_C@_0M@LHAILMAN@PersistType?$AA@ 10076494     mibtbl.obj
 0002:0000e4a0       ??_C@_0M@FIKGLCFE@PersistSize?$AA@ 100764a0     mibtbl.obj
 0002:0000e4ac       ??_C@_0O@GLDAFHDJ@PersistStores?$AA@ 100764ac     mibtbl.obj
 0002:0000e4bc       ??_C@_0O@DBBDLIJG@PersistEnable?$AA@ 100764bc     mibtbl.obj
 0002:0000e4cc       ??_C@_0L@FHHIOJDI@PersistAck?$AA@ 100764cc     mibtbl.obj
 0002:0000e4d8       ??_C@_05LEFLIPJH@flash?$AA@ 100764d8     mibtbl.obj
 0002:0000e4e0       ??_C@_04HCJEIHPL@POST?$AA@ 100764e0     mibtbl.obj
 0002:0000e4e8       ??_C@_05NBEAGECF@Image?$AA@ 100764e8     mibtbl.obj
 0002:0000e4f0       ??_C@_04DKKAEHDH@Last?$AA@ 100764f0     mibtbl.obj
 0002:0000e4f8       ??_C@_05IJGIMMHE@Count?$AA@ 100764f8     mibtbl.obj
 0002:0000e500       ??_C@_07JLFIFBAE@Display?$AA@ 10076500     mibtbl.obj
 0002:0000e508       ??_C@_05KKCIMGE@error?$AA@ 10076508     mibtbl.obj
 0002:0000e510       ??_C@_0M@IDNDEEHE@RateControl?$AA@ 10076510     mibtbl.obj
 0002:0000e51c       ??_C@_0L@CLGCCMPL@RateStatus?$AA@ 1007651c     mibtbl.obj
 0002:0000e528       ??_C@_04GMGOKAFF@mode?$AA@ 10076528     mibtbl.obj
 0002:0000e530       ??_C@_04LDOGFLEB@Rate?$AA@ 10076530     mibtbl.obj
 0002:0000e538       ??_C@_08KGEIBGG@Priority?$AA@ 10076538     mibtbl.obj
 0002:0000e544       ??_C@_03LOFCJIIG@Gap?$AA@  10076544     mibtbl.obj
 0002:0000e548       ??_C@_0L@GILGHLP@MacAddress?$AA@ 10076548     mibtbl.obj
 0002:0000e554       ??_C@_0N@FCGJIDBI@CurrentFrame?$AA@ 10076554     mibtbl.obj
 0002:0000e564       ??_C@_09PFIIBCCH@CycleRate?$AA@ 10076564     mibtbl.obj
 0002:0000e570       ??_C@_0BA@NKKNBNHM@IsoChannelCount?$AA@ 10076570     mibtbl.obj
 0002:0000e580       ??_C@_09CAEFINLN@conductor?$AA@ 10076580     mibtbl.obj
 0002:0000e58c       ??_C@_0O@DEBGBCCL@MeterDropouts?$AA@ 1007658c     mibtbl.obj
 0002:0000e59c       ??_C@_0O@PDLHCBDM@MeterMapIndex?$AA@ 1007659c     mibtbl.obj
 0002:0000e5ac       ??_C@_08GCHICAKB@MeterMap?$AA@ 100765ac     mibtbl.obj
 0002:0000e5b8       ??_C@_0L@GOIPEGJD@MeterPeaks?$AA@ 100765b8     mibtbl.obj
 0002:0000e5c4       ??_C@_06EMLLHNOE@Meters?$AA@ 100765c4     mibtbl.obj
 0002:0000e5cc       ??_C@_03NBOPHIOC@Map?$AA@  100765cc     mibtbl.obj
 0002:0000e5d0       ??_C@_09ONGBFEAH@LoopIndex?$AA@ 100765d0     mibtbl.obj
 0002:0000e5dc       ??_C@_07FJHMLCGO@LoopSrc?$AA@ 100765dc     mibtbl.obj
 0002:0000e5e4       ??_C@_07JAPDDDOJ@LoopDst?$AA@ 100765e4     mibtbl.obj
 0002:0000e5ec       ??_C@_0M@KJNFGKLC@OutputIndex?$AA@ 100765ec     mibtbl.obj
 0002:0000e5f8       ??_C@_06PFDLEJLJ@Output?$AA@ 100765f8     mibtbl.obj
 0002:0000e600       ??_C@_0L@KLLJKDMJ@MeterDecay?$AA@ 10076600     mibtbl.obj
 0002:0000e60c       ??_C@_0BA@CGGEKDHJ@AllowedChannels?$AA@ 1007660c     mibtbl.obj
 0002:0000e61c       ??_C@_0L@CNIKFOAC@TxChannels?$AA@ 1007661c     mibtbl.obj
 0002:0000e628       ??_C@_0L@MFDPJEEB@RxChannels?$AA@ 10076628     mibtbl.obj
 0002:0000e634       ??_C@_08IBLLPOGM@DupIndex?$AA@ 10076634     mibtbl.obj
 0002:0000e640       ??_C@_06LAPHCJEA@DupSrc?$AA@ 10076640     mibtbl.obj
 0002:0000e648       ??_C@_06HJHIKIMH@DupDst?$AA@ 10076648     mibtbl.obj
 0002:0000e650       ??_C@_0O@GMBOPJPK@MeterPeaksRaw?$AA@ 10076650     mibtbl.obj
 0002:0000e660       ??_C@_09CAKGJMIA@MetersRaw?$AA@ 10076660     mibtbl.obj
 0002:0000e66c       ??_C@_09CAJBNBFA@Unknown12?$AA@ 1007666c     mibtbl.obj
 0002:0000e678       ??_C@_05KNIAAKIP@audio?$AA@ 10076678     mibtbl.obj
 0002:0000e680       ??_C@_06CBOJNMHN@Bundle?$AA@ 10076680     mibtbl.obj
 0002:0000e688       ??_C@_09EOALEEFJ@SourceMAC?$AA@ 10076688     mibtbl.obj
 0002:0000e694       ??_C@_0N@JCFPEGIK@BuddyExclude?$AA@ 10076694     mibtbl.obj
 0002:0000e6a4       ??_C@_08BCEIEEPB@Dropouts?$AA@ 100766a4     mibtbl.obj
 0002:0000e6b0       ??_C@_05ENDOMFAI@Delay?$AA@ 100766b0     mibtbl.obj
 0002:0000e6b8       ??_C@_08CBAFBIHN@MinDelay?$AA@ 100766b8     mibtbl.obj
 0002:0000e6c4       ??_C@_0BA@IJIHKHKG@SubChannelIndex?$AA@ 100766c4     mibtbl.obj
 0002:0000e6d4       ??_C@_06MHOHDDPF@SubMap?$AA@ 100766d4     mibtbl.obj
 0002:0000e6dc       ??_C@_0BA@KOCOLEPG@SubChannelEntry?$AA@ 100766dc     mibtbl.obj
 0002:0000e6ec       ??_C@_02LACNGJCN@rx?$AA@   100766ec     mibtbl.obj
 0002:0000e6f0       ??_C@_0P@MFOODJDE@DestinationMAC?$AA@ 100766f0     mibtbl.obj
 0002:0000e700       ??_C@_08GNOFMGPC@SubCount?$AA@ 10076700     mibtbl.obj
 0002:0000e70c       ??_C@_08GCJNLIKG@Position?$AA@ 1007670c     mibtbl.obj
 0002:0000e718       ??_C@_09DGHMBLMK@Receivers?$AA@ 10076718     mibtbl.obj
 0002:0000e724       ??_C@_0M@KPEMJJJO@UnicastMode?$AA@ 10076724     mibtbl.obj
 0002:0000e730       ??_C@_0L@FFKCHHPA@MaxUnicast?$AA@ 10076730     mibtbl.obj
 0002:0000e73c       ??_C@_09PAMNPHMG@SubFormat?$AA@ 1007673c     mibtbl.obj
 0002:0000e748       ??_C@_02LEKABFJP@tx?$AA@   10076748     mibtbl.obj
 0002:0000e74c       ??_C@_0P@OGKHDFJK@ConductorClock?$AA@ 1007674c     mibtbl.obj
 0002:0000e75c       ??_C@_0P@LGJPAFPC@PerformerClock?$AA@ 1007675c     mibtbl.obj
 0002:0000e76c       ??_C@_09JJPJKGDF@ClockTrim?$AA@ 1007676c     mibtbl.obj
 0002:0000e778       ??_C@_0BB@NKFKKLFA@BuddyLinkControl?$AA@ 10076778     mibtbl.obj
 0002:0000e78c       ??_C@_07IKJEKJLO@Counter?$AA@ 1007678c     mibtbl.obj
 0002:0000e794       ??_C@_05KIFHCDFD@NTime?$AA@ 10076794     mibtbl.obj
 0002:0000e79c       ??_C@_04JNABKDKF@sync?$AA@ 1007679c     mibtbl.obj
 0002:0000e7a4       ??_C@_05CCOFGJDO@Dirty?$AA@ 100767a4     mibtbl.obj
 0002:0000e7ac       ??_C@_09KFJDHLLO@SNMPDirty?$AA@ 100767ac     mibtbl.obj
 0002:0000e7b8       ??_C@_08HDGPJKLK@HMIDirty?$AA@ 100767b8     mibtbl.obj
 0002:0000e7c4       ??_C@_05BPMMLCAO@mimon?$AA@ 100767c4     mibtbl.obj
 0002:0000e7cc       ??_C@_08LPAAKHME@StaticIP?$AA@ 100767cc     mibtbl.obj
 0002:0000e7d8       ??_C@_09BJNIHBEK@CurrentIP?$AA@ 100767d8     mibtbl.obj
 0002:0000e7e4       ??_C@_05OJKNAFOL@ipmon?$AA@ 100767e4     mibtbl.obj
 0002:0000e7ec       ??_C@_09JAMEOADP@CurrentIf?$AA@ 100767ec     mibtbl.obj
 0002:0000e7f8       ??_C@_06KGOCOFMM@TIndex?$AA@ 100767f8     mibtbl.obj
 0002:0000e800       ??_C@_07NPBIIIOP@TStatus?$AA@ 10076800     mibtbl.obj
 0002:0000e808       ??_C@_0M@DOJKCKG@TLastChange?$AA@ 10076808     mibtbl.obj
 0002:0000e814       ??_C@_0L@HDOAJPLO@SwitchMode?$AA@ 10076814     mibtbl.obj
 0002:0000e820       ??_C@_03EJMDKBC@ifm?$AA@   10076820     mibtbl.obj
 0002:0000e824       ??_C@_06PEPCFMNJ@Format?$AA@ 10076824     mibtbl.obj
 0002:0000e82c       ??_C@_04MLNPJHLF@Baud?$AA@ 1007682c     mibtbl.obj
 0002:0000e834       ??_C@_07DDDBINJG@PPeriod?$AA@ 10076834     mibtbl.obj
 0002:0000e83c       ??_C@_05FKLCHHP@RxMAC?$AA@ 1007683c     mibtbl.obj
 0002:0000e844       ??_C@_0L@KKBDEPOO@TxPriority?$AA@ 10076844     mibtbl.obj
 0002:0000e850       ??_C@_09EBLNKPHJ@TxChannel?$AA@ 10076850     mibtbl.obj
 0002:0000e85c       ??_C@_05NDPCMEGC@TxMAC?$AA@ 1007685c     mibtbl.obj
 0002:0000e864       ??_C@_06KCELPKEE@serial?$AA@ 10076864     mibtbl.obj
 0002:0000e86c       ??_C@_0BB@JJBOMGCA@UserVersionMajor?$AA@ 1007686c     mibtbl.obj
 0002:0000e880       ??_C@_0BB@CGAMBKLG@UserVersionMinor?$AA@ 10076880     mibtbl.obj
 0002:0000e894       ??_C@_0L@FHCJPPHJ@UserString?$AA@ 10076894     mibtbl.obj
 0002:0000e8a0       ??_C@_0M@HHHHIAII@UserInteger?$AA@ 100768a0     mibtbl.obj
 0002:0000e8ac       ??_C@_03PFFIEBLO@std?$AA@  100768ac     mibtbl.obj
 0002:0000e8b0       ??_C@_02JDPG@rb?$AA@       100768b0     rifffile.obj
 0002:0000e8b4       ??_C@_03ELIABIOC@w?$CLb?$AA@ 100768b4     rifffile.obj
 0002:0000e8bc       ??_7TWavFileBase@@6B@      100768bc     twavfile.obj
 0002:0000e8e0       ??_7TWavFileTypeWav@@6B@   100768e0     twavfile.obj
 0002:0000e904       ??_7TWavFileTypeMP23@@6B@  10076904     twavfile.obj
 0002:0000e928       ??_7TWavFileTypeDAF@@6B@   10076928     twavfile.obj
 0002:0000e94c       ??_7TWavFileTypeRaw@@6B@   1007694c     twavfile.obj
 0002:0000e970       ??_7TWavFileTypeNullRecord@@6B@ 10076970     twavfile.obj
 0002:0000e994       ??_7TWavFileTypeGenerator@@6B@ 10076994     twavfile.obj
 0002:0000e9b4       ??_C@_03HMFOOINA@r?$CLb?$AA@ 100769b4     twavfile.obj
 0002:0000e9b8       ??_C@_0BL@DEIPHCIG@TWavFile?5?9?5Unknown?5failure?$AA@ 100769b8     twavfile.obj
 0002:0000e9d4       ??_C@_0BN@EPDLBNFB@TWavFile?5?9?5Not?5enough?5memory?$AA@ 100769d4     twavfile.obj
 0002:0000e9f4       ??_C@_0BL@KEHDPHD@TWavFile?5?9?5Not?5a?5wave?5file?$AA@ 100769f4     twavfile.obj
 0002:0000ea10       ??_C@_0CA@KGEGAHBP@TWavFile?5?9?5Wave?5file?5is?5corrupt?$AA@ 10076a10     twavfile.obj
 0002:0000ea30       ??_C@_0BL@DFMFBJJO@TWavFile?5?9?5No?5format?5chunk?$AA@ 10076a30     twavfile.obj
 0002:0000ea4c       ??_C@_0BJ@CCBIBKMO@TWavFile?5?9?5No?5data?5chunk?$AA@ 10076a4c     twavfile.obj
 0002:0000ea68       ??_C@_0BJ@IGIOLDPI@TWavFile?5?9?5No?5fact?5chunk?$AA@ 10076a68     twavfile.obj
 0002:0000ea84       ??_C@_0BK@LBADNBKI@TWavFile?5?9?5Invalid?5format?$AA@ 10076a84     twavfile.obj
 0002:0000eaa0       ??_C@_0BI@EFNKKGLP@TWavFile?5?9?5Write?5failed?$AA@ 10076aa0     twavfile.obj
 0002:0000eab8       ??_C@_0BH@KFJLMGPO@TWavFile?5?9?5Read?5failed?$AA@ 10076ab8     twavfile.obj
 0002:0000ead0       ??_C@_0BP@LNKHHGPP@TWavFile?5?9?5Could?5not?5open?5file?$AA@ 10076ad0     twavfile.obj
 0002:0000eaf0       ??_C@_0CC@OJAAPFDN@TWavFile?5?9?5Could?5not?5create?5chun@ 10076af0     twavfile.obj
 0002:0000eb14       ??_C@_0CA@FEAGFBP@TWavFile?5?9?5Could?5not?5close?5file?$AA@ 10076b14     twavfile.obj
 0002:0000eb34       ??_C@_0BJ@HACCAGMC@TWavFile?5?9?5Unknown?5error?$AA@ 10076b34     twavfile.obj
 0002:0000eb50       ??_C@_04MLLLIHIP@null?$AA@ 10076b50     twavfile.obj
 0002:0000eb58       ??_C@_04IJNKJEOF@?4daf?$AA@ 10076b58     twavfile.obj
 0002:0000eb60       ??_C@_04HFHJMNCD@WAVE?$AA@ 10076b60     twavfile.obj
 0002:0000eb68       ??_C@_04CAJPEBPP@fmt?5?$AA@ 10076b68     twavfile.obj
 0002:0000eb70       ??_C@_0DK@ILIFKAPL@TWavFileTypeWav?3?3ReadWavData?$CI?$CJ?5m@ 10076b70     twavfile.obj
 0002:0000ebac       ??_C@_0DM@IHNACAFK@TWavFileTypeWav?3?3WriteWavData?$CI?$CJ?5@ 10076bac     twavfile.obj
 0002:0000ebe8       ??_C@_01IHBHIGKO@?0?$AA@   10076be8     twavfile.obj
 0002:0000ebec       ??_C@_04FHHILBME@SINE?$AA@ 10076bec     twavfile.obj
 0002:0000ebf8       __real@0000000000000000    10076bf8     twavfile.obj
 0002:0000ec04       ??_7TWavFileWithFifo@@6B@  10076c04     twavfilefifo.obj
 0002:0000ec24       ??_C@_0L@CCCFKAPP@Mono?0?5?$CFd?0?5?$AA@ 10076c24     twavfmt.obj
 0002:0000ec30       ??_C@_0N@LJIAEMLC@Stereo?0?5?$CFd?0?5?$AA@ 10076c30     twavfmt.obj
 0002:0000ec40       ??_C@_0M@KMAAHBLG@?$CFd?9Ch?0?5?$CFd?0?5?$AA@ 10076c40     twavfmt.obj
 0002:0000ec4c       ??_C@_03CCLNCNJA@PCM?$AA@  10076c4c     twavfmt.obj
 0002:0000ec50       ??_C@_01KJLJFBPL@8?$AA@    10076c50     twavfmt.obj
 0002:0000ec54       ??_C@_02KMALDIDP@16?$AA@   10076c54     twavfmt.obj
 0002:0000ec58       ??_C@_02JMHLOEOE@24?$AA@   10076c58     twavfmt.obj
 0002:0000ec5c       ??_C@_02MLODCJFF@32?$AA@   10076c5c     twavfmt.obj
 0002:0000ec60       ??_C@_02HHFHKOHM@?$DP?$DP?$AA@ 10076c60     twavfmt.obj
 0002:0000ec64       ??_C@_07HHDPEDJ@MP3?1kb?$DN?$AA@ 10076c64     twavfmt.obj
 0002:0000ec6c       ??_C@_09CCANOEBA@MPEG2?1kb?$DN?$AA@ 10076c6c     twavfmt.obj
 0002:0000ec78       __real@401921fb54411744    10076c78     twavgen.obj
 0002:0000ec80       __real@40a88b2f704790b8    10076c80     twavgen.obj
 0002:0000ec88       __real@41dfffffffc00000    10076c88     twavgen.obj
 0002:0000ec90       __real@42fe0000            10076c90     twavgen.obj
 0002:0000ec94       __real@43000000            10076c94     twavgen.obj
 0002:0000ec98       __real@46fffe00            10076c98     twavgen.obj
 0002:0000eca0       __sz_avdecc_lib_controller32_dll 10076ca0     avdecc-lib_controller32:avdecc-lib_controller32.dll
 0002:0000ecc4       ?ProcessDetach@NativeDll@<CrtImplementationDetails>@@0IB 10076cc4     LIBCMT:strtol.obj
 0002:0000ecc8       ?ProcessAttach@NativeDll@<CrtImplementationDetails>@@0IB 10076cc8     LIBCMT:strtol.obj
 0002:0000eccc       ?ThreadAttach@NativeDll@<CrtImplementationDetails>@@0IB 10076ccc     LIBCMT:strtol.obj
 0002:0000ecd0       ?ThreadDetach@NativeDll@<CrtImplementationDetails>@@0IB 10076cd0     LIBCMT:strtol.obj
 0002:0000ecd4       ?ProcessVerifier@NativeDll@<CrtImplementationDetails>@@0IB 10076cd4     LIBCMT:strtol.obj
 0002:0000ecdc       ??_7bad_alloc@std@@6B@     10076cdc     LIBCMT:new.obj
 0002:0000ece4       ??_C@_0P@GHFPNOJB@bad?5allocation?$AA@ 10076ce4     LIBCMT:new.obj
 0002:0000ecf8       ??_7type_info@@6B@         10076cf8     LIBCMT:typinfo.obj
 0002:0000ecfc       __FPinit                   10076cfc     LIBCMT:fpinit.obj
 0002:0000eda4       ??_C@_0CB@CGKGGDFI@Access?5violation?5?9?5no?5RTTI?5data?$CB@ 10076da4     LIBCMT:rtti.obj
 0002:0000edc8       ??_C@_0CE@FFJAJLDK@Attempted?5a?5typeid?5of?5NULL?5point@ 10076dc8     LIBCMT:rtti.obj
 0002:0000edec       ??_C@_0CB@EEENAAHH@Bad?5read?5pointer?5?9?5no?5RTTI?5data?$CB@ 10076dec     LIBCMT:rtti.obj
 0002:0000ee10       ??_C@_0BC@JNJNLHBP@Bad?5dynamic_cast?$CB?$AA@ 10076e10     LIBCMT:rtti.obj
 0002:00013930       __pRawDllMain              1007b930     LIBCMT:dllcrt0.obj
 0002:00013930       __pDefaultRawDllMain       1007b930     LIBCMT:dllcrt0.obj
 0002:00013934       ??_C@_1BK@MGMFAEKH@?$AAk?$AAe?$AAr?$AAn?$AAe?$AAl?$AA3?$AA2?$AA?4?$AAd?$AAl?$AAl?$AA?$AA@ 1007b934     LIBCMT:winapisupp.obj
 0002:00013950       ??_C@_08KNHFBNJ@FlsAlloc?$AA@ 1007b950     LIBCMT:winapisupp.obj
 0002:0001395c       ??_C@_07PEJMOBNF@FlsFree?$AA@ 1007b95c     LIBCMT:winapisupp.obj
 0002:00013964       ??_C@_0M@GDNOONDI@FlsGetValue?$AA@ 1007b964     LIBCMT:winapisupp.obj
 0002:00013970       ??_C@_0M@JCPCPOEF@FlsSetValue?$AA@ 1007b970     LIBCMT:winapisupp.obj
 0002:0001397c       ??_C@_0BM@HCFOFFN@InitializeCriticalSectionEx?$AA@ 1007b97c     LIBCMT:winapisupp.obj
 0002:00013998       ??_C@_0P@DLHPPCNH@CreateEventExW?$AA@ 1007b998     LIBCMT:winapisupp.obj
 0002:000139a8       ??_C@_0BD@KIEEOEEH@CreateSemaphoreExW?$AA@ 1007b9a8     LIBCMT:winapisupp.obj
 0002:000139bc       ??_C@_0BI@BKLFFAPO@SetThreadStackGuarantee?$AA@ 1007b9bc     LIBCMT:winapisupp.obj
 0002:000139d4       ??_C@_0BG@OGFAJCKC@CreateThreadpoolTimer?$AA@ 1007b9d4     LIBCMT:winapisupp.obj
 0002:000139ec       ??_C@_0BD@LPLEMMDI@SetThreadpoolTimer?$AA@ 1007b9ec     LIBCMT:winapisupp.obj
 0002:00013a00       ??_C@_0CA@FMNJENH@WaitForThreadpoolTimerCallbacks?$AA@ 1007ba00     LIBCMT:winapisupp.obj
 0002:00013a20       ??_C@_0BF@DCFCCNOC@CloseThreadpoolTimer?$AA@ 1007ba20     LIBCMT:winapisupp.obj
 0002:00013a38       ??_C@_0BF@FLABGKKM@CreateThreadpoolWait?$AA@ 1007ba38     LIBCMT:winapisupp.obj
 0002:00013a50       ??_C@_0BC@MGCOHNA@SetThreadpoolWait?$AA@ 1007ba50     LIBCMT:winapisupp.obj
 0002:00013a64       ??_C@_0BE@OCIOMIMP@CloseThreadpoolWait?$AA@ 1007ba64     LIBCMT:winapisupp.obj
 0002:00013a78       ??_C@_0BJ@LKGHFHBO@FlushProcessWriteBuffers?$AA@ 1007ba78     LIBCMT:winapisupp.obj
 0002:00013a94       ??_C@_0BP@KALKKPMO@FreeLibraryWhenCallbackReturns?$AA@ 1007ba94     LIBCMT:winapisupp.obj
 0002:00013ab4       ??_C@_0BK@DFNBACLA@GetCurrentProcessorNumber?$AA@ 1007bab4     LIBCMT:winapisupp.obj
 0002:00013ad0       ??_C@_0BP@KHGALBC@GetLogicalProcessorInformation?$AA@ 1007bad0     LIBCMT:winapisupp.obj
 0002:00013af0       ??_C@_0BE@FKKLLFLM@CreateSymbolicLinkW?$AA@ 1007baf0     LIBCMT:winapisupp.obj
 0002:00013b04       ??_C@_0BJ@OHNKDLIJ@SetDefaultDllDirectories?$AA@ 1007bb04     LIBCMT:winapisupp.obj
 0002:00013b20       ??_C@_0BE@LJANKFHF@EnumSystemLocalesEx?$AA@ 1007bb20     LIBCMT:winapisupp.obj
 0002:00013b34       ??_C@_0BA@IHGNDAEB@CompareStringEx?$AA@ 1007bb34     LIBCMT:winapisupp.obj
 0002:00013b44       ??_C@_0BA@EPCJIIPD@GetDateFormatEx?$AA@ 1007bb44     LIBCMT:winapisupp.obj
 0002:00013b54       ??_C@_0BA@ONOKGCMP@GetLocaleInfoEx?$AA@ 1007bb54     LIBCMT:winapisupp.obj
 0002:00013b64       ??_C@_0BA@CIJJKCJJ@GetTimeFormatEx?$AA@ 1007bb64     LIBCMT:winapisupp.obj
 0002:00013b74       ??_C@_0BJ@PBCCBIPI@GetUserDefaultLocaleName?$AA@ 1007bb74     LIBCMT:winapisupp.obj
 0002:00013b90       ??_C@_0BC@CELBKLLA@IsValidLocaleName?$AA@ 1007bb90     LIBCMT:winapisupp.obj
 0002:00013ba4       ??_C@_0O@KKBNKAPF@LCMapStringEx?$AA@ 1007bba4     LIBCMT:winapisupp.obj
 0002:00013bb4       ??_C@_0BE@JOGNEJCI@GetCurrentPackageId?$AA@ 1007bbb4     LIBCMT:winapisupp.obj
 0002:00013bc8       ??_C@_0P@CDHHOHKP@GetTickCount64?$AA@ 1007bbc8     LIBCMT:winapisupp.obj
 0002:00013bd8       ??_C@_0BO@KPCLFDJJ@GetFileInformationByHandleExW?$AA@ 1007bbd8     LIBCMT:winapisupp.obj
 0002:00013bf8       ??_C@_0BM@MHIDLABK@SetFileInformationByHandleW?$AA@ 1007bbf8     LIBCMT:winapisupp.obj
 0002:00013c24       ??_C@_1M@HPNHIDJI@?$AAj?$AAa?$AA?9?$AAJ?$AAP?$AA?$AA@ 1007bc24     LIBCMT:mbctype.obj
 0002:00013c30       ??_C@_1M@BIBDDEMK@?$AAz?$AAh?$AA?9?$AAC?$AAN?$AA?$AA@ 1007bc30     LIBCMT:mbctype.obj
 0002:00013c3c       ??_C@_1M@JLOOOEGK@?$AAk?$AAo?$AA?9?$AAK?$AAR?$AA?$AA@ 1007bc3c     LIBCMT:mbctype.obj
 0002:00013c48       ??_C@_1M@CLNBBOPM@?$AAz?$AAh?$AA?9?$AAT?$AAW?$AA?$AA@ 1007bc48     LIBCMT:mbctype.obj
 0002:00013c54       ??_C@_03KOEHGMDN@Sun?$AA@  1007bc54     LIBCMT:nlsdata.obj
 0002:00013c58       ??_C@_03PDAGKDH@Mon?$AA@   1007bc58     LIBCMT:nlsdata.obj
 0002:00013c5c       ??_C@_03NAGEINEP@Tue?$AA@  1007bc5c     LIBCMT:nlsdata.obj
 0002:00013c60       ??_C@_03MHOMLAJA@Wed?$AA@  1007bc60     LIBCMT:nlsdata.obj
 0002:00013c64       ??_C@_03IOFIKPDN@Thu?$AA@  1007bc64     LIBCMT:nlsdata.obj
 0002:00013c68       ??_C@_03IDIOELNC@Fri?$AA@  1007bc68     LIBCMT:nlsdata.obj
 0002:00013c6c       ??_C@_03FEFJNEK@Sat?$AA@   1007bc6c     LIBCMT:nlsdata.obj
 0002:00013c70       ??_C@_06OOPIFAJ@Sunday?$AA@ 1007bc70     LIBCMT:nlsdata.obj
 0002:00013c78       ??_C@_06JLEDEDGH@Monday?$AA@ 1007bc78     LIBCMT:nlsdata.obj
 0002:00013c80       ??_C@_07BAAGCFCM@Tuesday?$AA@ 1007bc80     LIBCMT:nlsdata.obj
 0002:00013c88       ??_C@_09DLIGFAKA@Wednesday?$AA@ 1007bc88     LIBCMT:nlsdata.obj
 0002:00013c94       ??_C@_08HACCIKIA@Thursday?$AA@ 1007bc94     LIBCMT:nlsdata.obj
 0002:00013ca0       ??_C@_06JECMNKMI@Friday?$AA@ 1007bca0     LIBCMT:nlsdata.obj
 0002:00013ca8       ??_C@_08INBOOONO@Saturday?$AA@ 1007bca8     LIBCMT:nlsdata.obj
 0002:00013cb4       ??_C@_03JIHJHPIE@Jan?$AA@  1007bcb4     LIBCMT:nlsdata.obj
 0002:00013cb8       ??_C@_03HJBDCHOM@Feb?$AA@  1007bcb8     LIBCMT:nlsdata.obj
 0002:00013cbc       ??_C@_03ODNJBKGA@Mar?$AA@  1007bcbc     LIBCMT:nlsdata.obj
 0002:00013cc0       ??_C@_03LEOLGMJP@Apr?$AA@  1007bcc0     LIBCMT:nlsdata.obj
 0002:00013cc4       ??_C@_03CNMDKL@May?$AA@    1007bcc4     LIBCMT:nlsdata.obj
 0002:00013cc8       ??_C@_03IDFGHECI@Jun?$AA@  1007bcc8     LIBCMT:nlsdata.obj
 0002:00013ccc       ??_C@_03LBGABGKK@Jul?$AA@  1007bccc     LIBCMT:nlsdata.obj
 0002:00013cd0       ??_C@_03IFJFEIGA@Aug?$AA@  1007bcd0     LIBCMT:nlsdata.obj
 0002:00013cd4       ??_C@_03GGCAPAJC@Sep?$AA@  1007bcd4     LIBCMT:nlsdata.obj
 0002:00013cd8       ??_C@_03BMAOKBAD@Oct?$AA@  1007bcd8     LIBCMT:nlsdata.obj
 0002:00013cdc       ??_C@_03JPJOFNIA@Nov?$AA@  1007bcdc     LIBCMT:nlsdata.obj
 0002:00013ce0       ??_C@_03MKABNOCG@Dec?$AA@  1007bce0     LIBCMT:nlsdata.obj
 0002:00013ce4       ??_C@_07CGJPFGJA@January?$AA@ 1007bce4     LIBCMT:nlsdata.obj
 0002:00013cec       ??_C@_08GNJGEPFN@February?$AA@ 1007bcec     LIBCMT:nlsdata.obj
 0002:00013cf8       ??_C@_05HPCKOFNC@March?$AA@ 1007bcf8     LIBCMT:nlsdata.obj
 0002:00013d00       ??_C@_05DMJDNLEJ@April?$AA@ 1007bd00     LIBCMT:nlsdata.obj
 0002:00013d08       ??_C@_04CNLMGBGM@June?$AA@ 1007bd08     LIBCMT:nlsdata.obj
 0002:00013d10       ??_C@_04MIEPOIFP@July?$AA@ 1007bd10     LIBCMT:nlsdata.obj
 0002:00013d18       ??_C@_06LBBHFDDG@August?$AA@ 1007bd18     LIBCMT:nlsdata.obj
 0002:00013d20       ??_C@_09BHHEALKD@September?$AA@ 1007bd20     LIBCMT:nlsdata.obj
 0002:00013d2c       ??_C@_07JJNFCEND@October?$AA@ 1007bd2c     LIBCMT:nlsdata.obj
 0002:00013d34       ??_C@_08HCHEGEOA@November?$AA@ 1007bd34     LIBCMT:nlsdata.obj
 0002:00013d40       ??_C@_08EDHMEBNP@December?$AA@ 1007bd40     LIBCMT:nlsdata.obj
 0002:00013d4c       ??_C@_02DEDBPAFC@AM?$AA@   1007bd4c     LIBCMT:nlsdata.obj
 0002:00013d50       ??_C@_02CJNFDJBF@PM?$AA@   1007bd50     LIBCMT:nlsdata.obj
 0002:00013d54       ??_C@_08BPBNCDIB@MM?1dd?1yy?$AA@ 1007bd54     LIBCMT:nlsdata.obj
 0002:00013d60       ??_C@_0BE@CKGJFCPC@dddd?0?5MMMM?5dd?0?5yyyy?$AA@ 1007bd60     LIBCMT:nlsdata.obj
 0002:00013d74       ??_C@_08JCCMCCIL@HH?3mm?3ss?$AA@ 1007bd74     LIBCMT:nlsdata.obj
 0002:00013d80       ??_C@_17MBGCMIPB@?$AAS?$AAu?$AAn?$AA?$AA@ 1007bd80     LIBCMT:nlsdata.obj
 0002:00013d88       ??_C@_17KBOMKBF@?$AAM?$AAo?$AAn?$AA?$AA@ 1007bd88     LIBCMT:nlsdata.obj
 0002:00013d90       ??_C@_17BMKGEGOJ@?$AAT?$AAu?$AAe?$AA?$AA@ 1007bd90     LIBCMT:nlsdata.obj
 0002:00013d98       ??_C@_17CJEDCEPE@?$AAW?$AAe?$AAd?$AA?$AA@ 1007bd98     LIBCMT:nlsdata.obj
 0002:00013da0       ??_C@_17PDPHAADD@?$AAT?$AAh?$AAu?$AA?$AA@ 1007bda0     LIBCMT:nlsdata.obj
 0002:00013da8       ??_C@_17HFOLPPLP@?$AAF?$AAr?$AAi?$AA?$AA@ 1007bda8     LIBCMT:nlsdata.obj
 0002:00013db0       ??_C@_17GGIBDPIH@?$AAS?$AAa?$AAt?$AA?$AA@ 1007bdb0     LIBCMT:nlsdata.obj
 0002:00013db8       ??_C@_1O@IHNHDHPB@?$AAS?$AAu?$AAn?$AAd?$AAa?$AAy?$AA?$AA@ 1007bdb8     LIBCMT:nlsdata.obj
 0002:00013dc8       ??_C@_1O@MMNBFLIA@?$AAM?$AAo?$AAn?$AAd?$AAa?$AAy?$AA?$AA@ 1007bdc8     LIBCMT:nlsdata.obj
 0002:00013dd8       ??_C@_1BA@ENFBFFEK@?$AAT?$AAu?$AAe?$AAs?$AAd?$AAa?$AAy?$AA?$AA@ 1007bdd8     LIBCMT:nlsdata.obj
 0002:00013de8       ??_C@_1BE@EBOGMDOH@?$AAW?$AAe?$AAd?$AAn?$AAe?$AAs?$AAd?$AAa?$AAy?$AA?$AA@ 1007bde8     LIBCMT:nlsdata.obj
 0002:00013dfc       ??_C@_1BC@HHMNLIHE@?$AAT?$AAh?$AAu?$AAr?$AAs?$AAd?$AAa?$AAy?$AA?$AA@ 1007bdfc     LIBCMT:nlsdata.obj
 0002:00013e10       ??_C@_1O@PDICJHAG@?$AAF?$AAr?$AAi?$AAd?$AAa?$AAy?$AA?$AA@ 1007be10     LIBCMT:nlsdata.obj
 0002:00013e20       ??_C@_1BC@ENMNNPAJ@?$AAS?$AAa?$AAt?$AAu?$AAr?$AAd?$AAa?$AAy?$AA?$AA@ 1007be20     LIBCMT:nlsdata.obj
 0002:00013e34       ??_C@_17DKNBKCHM@?$AAJ?$AAa?$AAn?$AA?$AA@ 1007be34     LIBCMT:nlsdata.obj
 0002:00013e3c       ??_C@_17LMDJEKJN@?$AAF?$AAe?$AAb?$AA?$AA@ 1007be3c     LIBCMT:nlsdata.obj
 0002:00013e44       ??_C@_17CKNLEDEC@?$AAM?$AAa?$AAr?$AA?$AA@ 1007be44     LIBCMT:nlsdata.obj
 0002:00013e4c       ??_C@_17LFPOIHDD@?$AAA?$AAp?$AAr?$AA?$AA@ 1007be4c     LIBCMT:nlsdata.obj
 0002:00013e54       ??_C@_17PNNKMEED@?$AAM?$AAa?$AAy?$AA?$AA@ 1007be54     LIBCMT:nlsdata.obj
 0002:00013e5c       ??_C@_17KCJGOCPB@?$AAJ?$AAu?$AAn?$AA?$AA@ 1007be5c     LIBCMT:nlsdata.obj
 0002:00013e64       ??_C@_17IJPCKHK@?$AAJ?$AAu?$AAl?$AA?$AA@ 1007be64     LIBCMT:nlsdata.obj
 0002:00013e6c       ??_C@_17ICPELBCN@?$AAA?$AAu?$AAg?$AA?$AA@ 1007be6c     LIBCMT:nlsdata.obj
 0002:00013e74       ??_C@_17HCHCOKMG@?$AAS?$AAe?$AAp?$AA?$AA@ 1007be74     LIBCMT:nlsdata.obj
 0002:00013e7c       ??_C@_17FNLKOI@?$AAO?$AAc?$AAt?$AA?$AA@ 1007be7c     LIBCMT:nlsdata.obj
 0002:00013e84       ??_C@_17BBDMLCIG@?$AAN?$AAo?$AAv?$AA?$AA@ 1007be84     LIBCMT:nlsdata.obj
 0002:00013e8c       ??_C@_17EGKACKIF@?$AAD?$AAe?$AAc?$AA?$AA@ 1007be8c     LIBCMT:nlsdata.obj
 0002:00013e94       ??_C@_1BA@EFMEIEBA@?$AAJ?$AAa?$AAn?$AAu?$AAa?$AAr?$AAy?$AA?$AA@ 1007be94     LIBCMT:nlsdata.obj
 0002:00013ea4       ??_C@_1BC@JGDDFFAM@?$AAF?$AAe?$AAb?$AAr?$AAu?$AAa?$AAr?$AAy?$AA?$AA@ 1007bea4     LIBCMT:nlsdata.obj
 0002:00013eb8       ??_C@_1M@IKEENEDF@?$AAM?$AAa?$AAr?$AAc?$AAh?$AA?$AA@ 1007beb8     LIBCMT:nlsdata.obj
 0002:00013ec4       ??_C@_1M@GJNLMHFD@?$AAA?$AAp?$AAr?$AAi?$AAl?$AA?$AA@ 1007bec4     LIBCMT:nlsdata.obj
 0002:00013ed0       ??_C@_19EPFLPGAP@?$AAJ?$AAu?$AAn?$AAe?$AA?$AA@ 1007bed0     LIBCMT:nlsdata.obj
 0002:00013edc       ??_C@_19BIFMLPCD@?$AAJ?$AAu?$AAl?$AAy?$AA?$AA@ 1007bedc     LIBCMT:nlsdata.obj
 0002:00013ee8       ??_C@_1O@PAHLKOAC@?$AAA?$AAu?$AAg?$AAu?$AAs?$AAt?$AA?$AA@ 1007bee8     LIBCMT:nlsdata.obj
 0002:00013ef8       ??_C@_1BE@DKAAMBJL@?$AAS?$AAe?$AAp?$AAt?$AAe?$AAm?$AAb?$AAe?$AAr?$AA?$AA@ 1007bef8     LIBCMT:nlsdata.obj
 0002:00013f0c       ??_C@_1BA@EPANDLNG@?$AAO?$AAc?$AAt?$AAo?$AAb?$AAe?$AAr?$AA?$AA@ 1007bf0c     LIBCMT:nlsdata.obj
 0002:00013f1c       ??_C@_1BC@BGLIFPF@?$AAN?$AAo?$AAv?$AAe?$AAm?$AAb?$AAe?$AAr?$AA?$AA@ 1007bf1c     LIBCMT:nlsdata.obj
 0002:00013f30       ??_C@_1BC@FEMKIFH@?$AAD?$AAe?$AAc?$AAe?$AAm?$AAb?$AAe?$AAr?$AA?$AA@ 1007bf30     LIBCMT:nlsdata.obj
 0002:00013f44       ??_C@_15ODEHAHHF@?$AAA?$AAM?$AA?$AA@ 1007bf44     LIBCMT:nlsdata.obj
 0002:00013f4c       ??_C@_15CLMNNGEL@?$AAP?$AAM?$AA?$AA@ 1007bf4c     LIBCMT:nlsdata.obj
 0002:00013f54       ??_C@_1BC@IEBCMHCM@?$AAM?$AAM?$AA?1?$AAd?$AAd?$AA?1?$AAy?$AAy?$AA?$AA@ 1007bf54     LIBCMT:nlsdata.obj
 0002:00013f68       ??_C@_1CI@KNAKOEBC@?$AAd?$AAd?$AAd?$AAd?$AA?0?$AA?5?$AAM?$AAM?$AAM?$AAM?$AA?5?$AAd?$AAd?$AA?0?$AA?5?$AAy?$AAy?$AAy?$AAy?$AA?$AA@ 1007bf68     LIBCMT:nlsdata.obj
 0002:00013f90       ??_C@_1BC@GDGBMEMK@?$AAH?$AAH?$AA?3?$AAm?$AAm?$AA?3?$AAs?$AAs?$AA?$AA@ 1007bf90     LIBCMT:nlsdata.obj
 0002:00013fa4       ??_C@_1M@BMHNFIME@?$AAe?$AAn?$AA?9?$AAU?$AAS?$AA?$AA@ 1007bfa4     LIBCMT:nlsdata.obj
 0002:00013fb0       ___lc_category             1007bfb0     LIBCMT:wsetloca.obj
 0002:00013ff8       ??_C@_1O@GIFLHMA@?$AAL?$AAC?$AA_?$AAA?$AAL?$AAL?$AA?$AA@ 1007bff8     LIBCMT:wsetloca.obj
 0002:00014008       ??_C@_1BG@PPOMIBNJ@?$AAL?$AAC?$AA_?$AAC?$AAO?$AAL?$AAL?$AAA?$AAT?$AAE?$AA?$AA@ 1007c008     LIBCMT:wsetloca.obj
 0002:00014020       ??_C@_1BC@FFJGAPJM@?$AAL?$AAC?$AA_?$AAC?$AAT?$AAY?$AAP?$AAE?$AA?$AA@ 1007c020     LIBCMT:wsetloca.obj
 0002:00014034       ??_C@_1BI@PCKFNJFB@?$AAL?$AAC?$AA_?$AAM?$AAO?$AAN?$AAE?$AAT?$AAA?$AAR?$AAY?$AA?$AA@ 1007c034     LIBCMT:wsetloca.obj
 0002:0001404c       ??_C@_1BG@ENIEDKID@?$AAL?$AAC?$AA_?$AAN?$AAU?$AAM?$AAE?$AAR?$AAI?$AAC?$AA?$AA@ 1007c04c     LIBCMT:wsetloca.obj
 0002:00014064       ??_C@_1BA@HAAOMIIG@?$AAL?$AAC?$AA_?$AAT?$AAI?$AAM?$AAE?$AA?$AA@ 1007c064     LIBCMT:wsetloca.obj
 0002:000140f8       ??_C@_15NBPDDFIP@?$AA?$DN?$AA?$DL?$AA?$AA@ 1007c0f8     LIBCMT:wsetloca.obj
 0002:00014100       ??_C@_13PJJBFPED@?$AA?$DL?$AA?$AA@ 1007c100     LIBCMT:wsetloca.obj
 0002:00014104       ??_C@_13NMPKAAJP@?$AA?$DN?$AA?$AA@ 1007c104     LIBCMT:wsetloca.obj
 0002:00014108       ??_C@_13FHBKNHDA@?$AAC?$AA?$AA@ 1007c108     LIBCMT:wsetloca.obj
 0002:0001410c       ??_C@_17MBJJLFDM@?$AA_?$AA?4?$AA?0?$AA?$AA@ 1007c10c     LIBCMT:wsetloca.obj
 0002:00014114       ??_C@_13ENNFDPBH@?$AA_?$AA?$AA@ 1007c114     LIBCMT:wsetloca.obj
 0002:00014118       ??_C@_13JOFGPIOO@?$AA?4?$AA?$AA@ 1007c118     LIBCMT:wsetloca.obj
 0002:0001411c       ??_C@_06OJHGLDPL@?$CInull?$CJ?$AA@ 1007c11c     LIBCMT:output.obj
 0002:00014124       ??_C@_1O@CEDCILHN@?$AA?$CI?$AAn?$AAu?$AAl?$AAl?$AA?$CJ?$AA?$AA@ 1007c124     LIBCMT:output.obj
 0002:00014138       ___lookuptable             1007c138     LIBCMT:output.obj
 0002:00014194       ??_C@_1BI@BGOHAHKC@?$AAm?$AAs?$AAc?$AAo?$AAr?$AAe?$AAe?$AA?4?$AAd?$AAl?$AAl?$AA?$AA@ 1007c194     LIBCMT:crt0dat.obj
 0002:000141ac       ??_C@_0P@MIGLKIOC@CorExitProcess?$AA@ 1007c1ac     LIBCMT:crt0dat.obj
 0002:00014278       ??_C@_1FK@PGACCAFB@?$AAR?$AA6?$AA0?$AA0?$AA2?$AA?$AN?$AA?6?$AA?9?$AA?5?$AAf?$AAl?$AAo?$AAa?$AAt?$AAi?$AAn?$AAg?$AA?5?$AAp?$AAo?$AAi?$AAn?$AAt?$AA?5?$AAs?$AAu?$AAp?$AAp?$AAo?$AAr?$AAt?$AA?5@ 1007c278     LIBCMT:crt0msg.obj
 0002:000142d8       ??_C@_1FE@LLNEDJMD@?$AAR?$AA6?$AA0?$AA0?$AA8?$AA?$AN?$AA?6?$AA?9?$AA?5?$AAn?$AAo?$AAt?$AA?5?$AAe?$AAn?$AAo?$AAu?$AAg?$AAh?$AA?5?$AAs?$AAp?$AAa?$AAc?$AAe?$AA?5?$AAf?$AAo?$AAr?$AA?5?$AAa?$AAr@ 1007c2d8     LIBCMT:crt0msg.obj
 0002:00014330       ??_C@_1FI@HONFMGBI@?$AAR?$AA6?$AA0?$AA0?$AA9?$AA?$AN?$AA?6?$AA?9?$AA?5?$AAn?$AAo?$AAt?$AA?5?$AAe?$AAn?$AAo?$AAu?$AAg?$AAh?$AA?5?$AAs?$AAp?$AAa?$AAc?$AAe?$AA?5?$AAf?$AAo?$AAr?$AA?5?$AAe?$AAn@ 1007c330     LIBCMT:crt0msg.obj
 0002:00014388       ??_C@_1EG@BEHAGFJD@?$AAR?$AA6?$AA0?$AA1?$AA0?$AA?$AN?$AA?6?$AA?9?$AA?5?$AAa?$AAb?$AAo?$AAr?$AAt?$AA?$CI?$AA?$CJ?$AA?5?$AAh?$AAa?$AAs?$AA?5?$AAb?$AAe?$AAe?$AAn?$AA?5?$AAc?$AAa?$AAl?$AAl?$AAe?$AAd@ 1007c388     LIBCMT:crt0msg.obj
 0002:000143d0       ??_C@_1FI@LOGNIKDM@?$AAR?$AA6?$AA0?$AA1?$AA6?$AA?$AN?$AA?6?$AA?9?$AA?5?$AAn?$AAo?$AAt?$AA?5?$AAe?$AAn?$AAo?$AAu?$AAg?$AAh?$AA?5?$AAs?$AAp?$AAa?$AAc?$AAe?$AA?5?$AAf?$AAo?$AAr?$AA?5?$AAt?$AAh@ 1007c3d0     LIBCMT:crt0msg.obj
 0002:00014428       ??_C@_1FK@BEOGODMC@?$AAR?$AA6?$AA0?$AA1?$AA7?$AA?$AN?$AA?6?$AA?9?$AA?5?$AAu?$AAn?$AAe?$AAx?$AAp?$AAe?$AAc?$AAt?$AAe?$AAd?$AA?5?$AAm?$AAu?$AAl?$AAt?$AAi?$AAt?$AAh?$AAr?$AAe?$AAa?$AAd?$AA?5@ 1007c428     LIBCMT:crt0msg.obj
 0002:00014488       ??_C@_1EC@JIBHAOPH@?$AAR?$AA6?$AA0?$AA1?$AA8?$AA?$AN?$AA?6?$AA?9?$AA?5?$AAu?$AAn?$AAe?$AAx?$AAp?$AAe?$AAc?$AAt?$AAe?$AAd?$AA?5?$AAh?$AAe?$AAa?$AAp?$AA?5?$AAe?$AAr?$AAr?$AAo?$AAr?$AA?$AN?$AA?6@ 1007c488     LIBCMT:crt0msg.obj
 0002:000144d0       ??_C@_1FC@ECHBIFBC@?$AAR?$AA6?$AA0?$AA1?$AA9?$AA?$AN?$AA?6?$AA?9?$AA?5?$AAu?$AAn?$AAa?$AAb?$AAl?$AAe?$AA?5?$AAt?$AAo?$AA?5?$AAo?$AAp?$AAe?$AAn?$AA?5?$AAc?$AAo?$AAn?$AAs?$AAo?$AAl?$AAe?$AA?5@ 1007c4d0     LIBCMT:crt0msg.obj
 0002:00014528       ??_C@_1GK@FHCKBEFA@?$AAR?$AA6?$AA0?$AA2?$AA4?$AA?$AN?$AA?6?$AA?9?$AA?5?$AAn?$AAo?$AAt?$AA?5?$AAe?$AAn?$AAo?$AAu?$AAg?$AAh?$AA?5?$AAs?$AAp?$AAa?$AAc?$AAe?$AA?5?$AAf?$AAo?$AAr?$AA?5?$AA_?$AAo@ 1007c528     LIBCMT:crt0msg.obj
 0002:00014598       ??_C@_1EM@MAADIHMB@?$AAR?$AA6?$AA0?$AA2?$AA5?$AA?$AN?$AA?6?$AA?9?$AA?5?$AAp?$AAu?$AAr?$AAe?$AA?5?$AAv?$AAi?$AAr?$AAt?$AAu?$AAa?$AAl?$AA?5?$AAf?$AAu?$AAn?$AAc?$AAt?$AAi?$AAo?$AAn?$AA?5?$AAc@ 1007c598     LIBCMT:crt0msg.obj
 0002:000145e8       ??_C@_1GK@MCAAGJMO@?$AAR?$AA6?$AA0?$AA2?$AA6?$AA?$AN?$AA?6?$AA?9?$AA?5?$AAn?$AAo?$AAt?$AA?5?$AAe?$AAn?$AAo?$AAu?$AAg?$AAh?$AA?5?$AAs?$AAp?$AAa?$AAc?$AAe?$AA?5?$AAf?$AAo?$AAr?$AA?5?$AAs?$AAt@ 1007c5e8     LIBCMT:crt0msg.obj
 0002:00014658       ??_C@_1GK@MFGOKLAG@?$AAR?$AA6?$AA0?$AA2?$AA7?$AA?$AN?$AA?6?$AA?9?$AA?5?$AAn?$AAo?$AAt?$AA?5?$AAe?$AAn?$AAo?$AAu?$AAg?$AAh?$AA?5?$AAs?$AAp?$AAa?$AAc?$AAe?$AA?5?$AAf?$AAo?$AAr?$AA?5?$AAl?$AAo@ 1007c658     LIBCMT:crt0msg.obj
 0002:000146c8       ??_C@_1EK@HHFLMAOL@?$AAR?$AA6?$AA0?$AA2?$AA8?$AA?$AN?$AA?6?$AA?9?$AA?5?$AAu?$AAn?$AAa?$AAb?$AAl?$AAe?$AA?5?$AAt?$AAo?$AA?5?$AAi?$AAn?$AAi?$AAt?$AAi?$AAa?$AAl?$AAi?$AAz?$AAe?$AA?5?$AAh?$AAe@ 1007c6c8     LIBCMT:crt0msg.obj
 0002:00014714       ??_C@_1DO@BMFCDCD@?$AAR?$AA6?$AA0?$AA3?$AA0?$AA?$AN?$AA?6?$AA?9?$AA?5?$AAC?$AAR?$AAT?$AA?5?$AAn?$AAo?$AAt?$AA?5?$AAi?$AAn?$AAi?$AAt?$AAi?$AAa?$AAl?$AAi?$AAz?$AAe?$AAd?$AA?$AN?$AA?6?$AA?$AA@ 1007c714     LIBCMT:crt0msg.obj
 0002:00014758       ??_C@_1MG@ENCOOIDF@?$AAR?$AA6?$AA0?$AA3?$AA1?$AA?$AN?$AA?6?$AA?9?$AA?5?$AAA?$AAt?$AAt?$AAe?$AAm?$AAp?$AAt?$AA?5?$AAt?$AAo?$AA?5?$AAi?$AAn?$AAi?$AAt?$AAi?$AAa?$AAl?$AAi?$AAz?$AAe?$AA?5?$AAt@ 1007c758     LIBCMT:crt0msg.obj
 0002:00014820       ??_C@_1GG@GOPILAJP@?$AAR?$AA6?$AA0?$AA3?$AA2?$AA?$AN?$AA?6?$AA?9?$AA?5?$AAn?$AAo?$AAt?$AA?5?$AAe?$AAn?$AAo?$AAu?$AAg?$AAh?$AA?5?$AAs?$AAp?$AAa?$AAc?$AAe?$AA?5?$AAf?$AAo?$AAr?$AA?5?$AAl?$AAo@ 1007c820     LIBCMT:crt0msg.obj
 0002:00014888       ??_C@_1BOO@KGEDBGAJ@?$AAR?$AA6?$AA0?$AA3?$AA3?$AA?$AN?$AA?6?$AA?9?$AA?5?$AAA?$AAt?$AAt?$AAe?$AAm?$AAp?$AAt?$AA?5?$AAt?$AAo?$AA?5?$AAu?$AAs?$AAe?$AA?5?$AAM?$AAS?$AAI?$AAL?$AA?5?$AAc?$AAo?$AAd@ 1007c888     LIBCMT:crt0msg.obj
 0002:00014a78       ??_C@_1GG@MKFPEKFO@?$AAR?$AA6?$AA0?$AA3?$AA4?$AA?$AN?$AA?6?$AA?9?$AA?5?$AAi?$AAn?$AAc?$AAo?$AAn?$AAs?$AAi?$AAs?$AAt?$AAe?$AAn?$AAt?$AA?5?$AAo?$AAn?$AAe?$AAx?$AAi?$AAt?$AA?5?$AAb?$AAe?$AAg@ 1007ca78     LIBCMT:crt0msg.obj
 0002:00014ae0       ??_C@_1BO@BFCDCGC@?$AAD?$AAO?$AAM?$AAA?$AAI?$AAN?$AA?5?$AAe?$AAr?$AAr?$AAo?$AAr?$AA?$AN?$AA?6?$AA?$AA@ 1007cae0     LIBCMT:crt0msg.obj
 0002:00014b00       ??_C@_1BK@KMOMNAAI@?$AAS?$AAI?$AAN?$AAG?$AA?5?$AAe?$AAr?$AAr?$AAo?$AAr?$AA?$AN?$AA?6?$AA?$AA@ 1007cb00     LIBCMT:crt0msg.obj
 0002:00014b1c       ??_C@_1BM@JBBEPPHI@?$AAT?$AAL?$AAO?$AAS?$AAS?$AA?5?$AAe?$AAr?$AAr?$AAo?$AAr?$AA?$AN?$AA?6?$AA?$AA@ 1007cb1c     LIBCMT:crt0msg.obj
 0002:00014b38       ??_C@_15JNBOKNOG@?$AA?$AN?$AA?6?$AA?$AA@ 1007cb38     LIBCMT:crt0msg.obj
 0002:00014b40       ??_C@_1BO@BKOMIGKJ@?$AAr?$AAu?$AAn?$AAt?$AAi?$AAm?$AAe?$AA?5?$AAe?$AAr?$AAr?$AAo?$AAr?$AA?5?$AA?$AA@ 1007cb40     LIBCMT:crt0msg.obj
 0002:00014b60       ??_C@_1DE@JNGNBFGO@?$AAR?$AAu?$AAn?$AAt?$AAi?$AAm?$AAe?$AA?5?$AAE?$AAr?$AAr?$AAo?$AAr?$AA?$CB?$AA?6?$AA?6?$AAP?$AAr?$AAo?$AAg?$AAr?$AAa?$AAm?$AA?3?$AA?5?$AA?$AA@ 1007cb60     LIBCMT:crt0msg.obj
 0002:00014b94       ??_C@_1CO@EAEJAADC@?$AA?$DM?$AAp?$AAr?$AAo?$AAg?$AAr?$AAa?$AAm?$AA?5?$AAn?$AAa?$AAm?$AAe?$AA?5?$AAu?$AAn?$AAk?$AAn?$AAo?$AAw?$AAn?$AA?$DO?$AA?$AA@ 1007cb94     LIBCMT:crt0msg.obj
 0002:00014bc4       ??_C@_17LGKOMLJ@?$AA?4?$AA?4?$AA?4?$AA?$AA@ 1007cbc4     LIBCMT:crt0msg.obj
 0002:00014bcc       ??_C@_15IABLJNFO@?$AA?6?$AA?6?$AA?$AA@ 1007cbcc     LIBCMT:crt0msg.obj
 0002:00014bd8       ??_C@_1EK@MBDPDCGA@?$AAM?$AAi?$AAc?$AAr?$AAo?$AAs?$AAo?$AAf?$AAt?$AA?5?$AAV?$AAi?$AAs?$AAu?$AAa?$AAl?$AA?5?$AAC?$AA?$CL?$AA?$CL?$AA?5?$AAR?$AAu?$AAn?$AAt?$AAi?$AAm?$AAe?$AA?5?$AAL?$AAi?$AAb@ 1007cbd8     LIBCMT:crt0msg.obj
 0002:00014c28       ___lookuptable_s           1007cc28     LIBCMT:outputs.obj
 0002:00014c88       ??_7exception@std@@6B@     1007cc88     LIBCMT:stdexcpt.obj
 0002:00014c90       ??_C@_0BC@EOODALEL@Unknown?5exception?$AA@ 1007cc90     LIBCMT:stdexcpt.obj
 0002:00014ca8       ??_7bad_cast@std@@6B@      1007cca8     LIBCMT:stdexcpt.obj
 0002:00014cb4       ??_7bad_typeid@std@@6B@    1007ccb4     LIBCMT:stdexcpt.obj
 0002:00014cc0       ??_7__non_rtti_object@std@@6B@ 1007ccc0     LIBCMT:stdexcpt.obj
 0002:00014cc8       ??_C@_05KLBDPFGC@e?$CL000?$AA@ 1007ccc8     LIBCMT:cvt.obj
 0002:00014cd0       ??_C@_04FJHINJAO@tanh?$AA@ 1007ccd0     LIBCMT:fpexcept.obj
 0002:00014cd8       ??_C@_04FIHNOPOL@asin?$AA@ 1007ccd8     LIBCMT:fpexcept.obj
 0002:00014ce0       ??_C@_04PDIFKINK@acos?$AA@ 1007cce0     LIBCMT:fpexcept.obj
 0002:00014ce8       ??_C@_04MLLJIGOK@atan?$AA@ 1007cce8     LIBCMT:fpexcept.obj
 0002:00014cf0       ??_C@_05KNGEOGJB@atan2?$AA@ 1007ccf0     LIBCMT:fpexcept.obj
 0002:00014cf8       ??_C@_04EIAKFFMI@sqrt?$AA@ 1007ccf8     LIBCMT:fpexcept.obj
 0002:00014d00       ??_C@_03BLEJJJBH@sin?$AA@  1007cd00     LIBCMT:fpexcept.obj
 0002:00014d04       ??_C@_03LALBNOCG@cos?$AA@  1007cd04     LIBCMT:fpexcept.obj
 0002:00014d08       ??_C@_03IIINPABG@tan?$AA@  1007cd08     LIBCMT:fpexcept.obj
 0002:00014d0c       ??_C@_04GFPJNGEK@ceil?$AA@ 1007cd0c     LIBCMT:fpexcept.obj
 0002:00014d14       ??_C@_05PBJFFIGL@floor?$AA@ 1007cd14     LIBCMT:fpexcept.obj
 0002:00014d1c       ??_C@_04ODHECPBC@fabs?$AA@ 1007cd1c     LIBCMT:fpexcept.obj
 0002:00014d24       ??_C@_04EHEDPDJG@modf?$AA@ 1007cd24     LIBCMT:fpexcept.obj
 0002:00014d2c       ??_C@_05CEJMAHNP@ldexp?$AA@ 1007cd2c     LIBCMT:fpexcept.obj
 0002:00014d34       ??_C@_05KBKMEMPO@_cabs?$AA@ 1007cd34     LIBCMT:fpexcept.obj
 0002:00014d3c       ??_C@_06MEIMCGCF@_hypot?$AA@ 1007cd3c     LIBCMT:fpexcept.obj
 0002:00014d44       ??_C@_04KEPJIHGP@fmod?$AA@ 1007cd44     LIBCMT:fpexcept.obj
 0002:00014d4c       ??_C@_05GKKHEGJL@frexp?$AA@ 1007cd4c     LIBCMT:fpexcept.obj
 0002:00014d54       ??_C@_03MJLDFKDL@_y0?$AA@  1007cd54     LIBCMT:fpexcept.obj
 0002:00014d58       ??_C@_03NAKIGLHK@_y1?$AA@  1007cd58     LIBCMT:fpexcept.obj
 0002:00014d5c       ??_C@_03ONILCKOB@_yn?$AA@  1007cd5c     LIBCMT:fpexcept.obj
 0002:00014d60       ??_C@_05JGDBENOH@_logb?$AA@ 1007cd60     LIBCMT:fpexcept.obj
 0002:00014d68       ??_C@_0L@KDOEJCKC@_nextafter?$AA@ 1007cd68     LIBCMT:fpexcept.obj
 0002:00014d74       ??_C@_03KHJOGHMM@exp?$AA@  1007cd74     LIBCMT:fpexcept.obj
 0002:00014d78       ??_C@_03JGHBODFD@pow?$AA@  1007cd78     LIBCMT:fpexcept.obj
 0002:00014d7c       ??_C@_03MGHMBJCF@log?$AA@  1007cd7c     LIBCMT:fpexcept.obj
 0002:00014d80       ??_C@_05HGHHAHAP@log10?$AA@ 1007cd80     LIBCMT:fpexcept.obj
 0002:00014d88       ??_C@_04COOMCNPB@sinh?$AA@ 1007cd88     LIBCMT:fpexcept.obj
 0002:00014d90       ??_C@_04HPJJNFIM@cosh?$AA@ 1007cd90     LIBCMT:fpexcept.obj
 0002:00014d98       __pDestructExceptionObject 1007cd98     LIBCMT:frame.obj
 0002:00014da0       ??_7bad_exception@std@@6B@ 1007cda0     LIBCMT:frame.obj
 0002:00014da8       ??_C@_0O@DPKOEFFH@bad?5exception?$AA@ 1007cda8     LIBCMT:frame.obj
 0002:00014e20       ??_C@_05EOHGHCHD@exp10?$AA@ 1007ce20     LIBCMT:libm_error.obj
 0002:00014e28       __real@3ff0000000000000    1007ce28     LIBCMT:libm_error.obj
 0002:00014e50       __XcptActTab               1007ce50     LIBCMT:winxfltr.obj
 0002:00014ee0       __XcptActTabCount          1007cee0     LIBCMT:winxfltr.obj
 0002:00014ee4       __XcptActTabSize           1007cee4     LIBCMT:winxfltr.obj
 0002:00014ee8       __First_FPE_Indx           1007cee8     LIBCMT:winxfltr.obj
 0002:00014eec       __Num_FPE                  1007ceec     LIBCMT:winxfltr.obj
 0002:00014ef0       ___newctype                1007cef0     LIBCMT:ctype.obj
 0002:000151f0       __wctype                   1007d1f0     LIBCMT:ctype.obj
 0002:000153f8       ___newclmap                1007d3f8     LIBCMT:ctype.obj
 0002:00015578       ___newcumap                1007d578     LIBCMT:ctype.obj
 0002:000156f8       ___rg_language             1007d6f8     LIBCMT:getqloc.obj
 0002:00015a04       ??_C@_1BC@LLOKLNP@?$AAa?$AAm?$AAe?$AAr?$AAi?$AAc?$AAa?$AAn?$AA?$AA@ 1007da04     LIBCMT:getqloc.obj
 0002:00015a18       ??_C@_1CC@HEIGCDGG@?$AAa?$AAm?$AAe?$AAr?$AAi?$AAc?$AAa?$AAn?$AA?5?$AAe?$AAn?$AAg?$AAl?$AAi?$AAs?$AAh?$AA?$AA@ 1007da18     LIBCMT:getqloc.obj
 0002:00015a3c       ??_C@_1CC@IHCNOMIN@?$AAa?$AAm?$AAe?$AAr?$AAi?$AAc?$AAa?$AAn?$AA?9?$AAe?$AAn?$AAg?$AAl?$AAi?$AAs?$AAh?$AA?$AA@ 1007da3c     LIBCMT:getqloc.obj
 0002:00015a60       ??_C@_1BG@GKAGPCGG@?$AAa?$AAu?$AAs?$AAt?$AAr?$AAa?$AAl?$AAi?$AAa?$AAn?$AA?$AA@ 1007da60     LIBCMT:getqloc.obj
 0002:00015a78       ??_C@_1BA@GMENCENF@?$AAb?$AAe?$AAl?$AAg?$AAi?$AAa?$AAn?$AA?$AA@ 1007da78     LIBCMT:getqloc.obj
 0002:00015a88       ??_C@_1BC@PJMIIAAN@?$AAc?$AAa?$AAn?$AAa?$AAd?$AAi?$AAa?$AAn?$AA?$AA@ 1007da88     LIBCMT:getqloc.obj
 0002:00015a9c       ??_C@_17NOIMNFBF@?$AAc?$AAh?$AAh?$AA?$AA@ 1007da9c     LIBCMT:getqloc.obj
 0002:00015aa4       ??_C@_17GGDALCHA@?$AAc?$AAh?$AAi?$AA?$AA@ 1007daa4     LIBCMT:getqloc.obj
 0002:00015aac       ??_C@_1BA@NPNJKIBL@?$AAc?$AAh?$AAi?$AAn?$AAe?$AAs?$AAe?$AA?$AA@ 1007daac     LIBCMT:getqloc.obj
 0002:00015abc       ??_C@_1CC@DINBAMMJ@?$AAc?$AAh?$AAi?$AAn?$AAe?$AAs?$AAe?$AA?9?$AAh?$AAo?$AAn?$AAg?$AAk?$AAo?$AAn?$AAg?$AA?$AA@ 1007dabc     LIBCMT:getqloc.obj
 0002:00015ae0       ??_C@_1CG@IOBJPACO@?$AAc?$AAh?$AAi?$AAn?$AAe?$AAs?$AAe?$AA?9?$AAs?$AAi?$AAm?$AAp?$AAl?$AAi?$AAf?$AAi?$AAe?$AAd?$AA?$AA@ 1007dae0     LIBCMT:getqloc.obj
 0002:00015b08       ??_C@_1CE@GAJNDCKG@?$AAc?$AAh?$AAi?$AAn?$AAe?$AAs?$AAe?$AA?9?$AAs?$AAi?$AAn?$AAg?$AAa?$AAp?$AAo?$AAr?$AAe?$AA?$AA@ 1007db08     LIBCMT:getqloc.obj
 0002:00015b2c       ??_C@_1CI@PAJPIOOD@?$AAc?$AAh?$AAi?$AAn?$AAe?$AAs?$AAe?$AA?9?$AAt?$AAr?$AAa?$AAd?$AAi?$AAt?$AAi?$AAo?$AAn?$AAa?$AAl?$AA?$AA@ 1007db2c     LIBCMT:getqloc.obj
 0002:00015b54       ??_C@_1BM@NILJBMMD@?$AAd?$AAu?$AAt?$AAc?$AAh?$AA?9?$AAb?$AAe?$AAl?$AAg?$AAi?$AAa?$AAn?$AA?$AA@ 1007db54     LIBCMT:getqloc.obj
 0002:00015b70       ??_C@_1CC@OOJPJNEJ@?$AAe?$AAn?$AAg?$AAl?$AAi?$AAs?$AAh?$AA?9?$AAa?$AAm?$AAe?$AAr?$AAi?$AAc?$AAa?$AAn?$AA?$AA@ 1007db70     LIBCMT:getqloc.obj
 0002:00015b94       ??_C@_1BI@IOLFEEM@?$AAe?$AAn?$AAg?$AAl?$AAi?$AAs?$AAh?$AA?9?$AAa?$AAu?$AAs?$AA?$AA@ 1007db94     LIBCMT:getqloc.obj
 0002:00015bac       ??_C@_1BO@HFFNLENJ@?$AAe?$AAn?$AAg?$AAl?$AAi?$AAs?$AAh?$AA?9?$AAb?$AAe?$AAl?$AAi?$AAz?$AAe?$AA?$AA@ 1007dbac     LIBCMT:getqloc.obj
 0002:00015bcc       ??_C@_1BI@HAPKJMPO@?$AAe?$AAn?$AAg?$AAl?$AAi?$AAs?$AAh?$AA?9?$AAc?$AAa?$AAn?$AA?$AA@ 1007dbcc     LIBCMT:getqloc.obj
 0002:00015be4       ??_C@_1CE@HLNDMIOJ@?$AAe?$AAn?$AAg?$AAl?$AAi?$AAs?$AAh?$AA?9?$AAc?$AAa?$AAr?$AAi?$AAb?$AAb?$AAe?$AAa?$AAn?$AA?$AA@ 1007dbe4     LIBCMT:getqloc.obj
 0002:00015c08       ??_C@_1BI@LDHJHHAC@?$AAe?$AAn?$AAg?$AAl?$AAi?$AAs?$AAh?$AA?9?$AAi?$AAr?$AAe?$AA?$AA@ 1007dc08     LIBCMT:getqloc.obj
 0002:00015c20       ??_C@_1CA@NJMMCFOC@?$AAe?$AAn?$AAg?$AAl?$AAi?$AAs?$AAh?$AA?9?$AAj?$AAa?$AAm?$AAa?$AAi?$AAc?$AAa?$AA?$AA@ 1007dc20     LIBCMT:getqloc.obj
 0002:00015c40       ??_C@_1BG@BHJEBBGG@?$AAe?$AAn?$AAg?$AAl?$AAi?$AAs?$AAh?$AA?9?$AAn?$AAz?$AA?$AA@ 1007dc40     LIBCMT:getqloc.obj
 0002:00015c58       ??_C@_1CK@FGOEJJCO@?$AAe?$AAn?$AAg?$AAl?$AAi?$AAs?$AAh?$AA?9?$AAs?$AAo?$AAu?$AAt?$AAh?$AA?5?$AAa?$AAf?$AAr?$AAi?$AAc?$AAa?$AA?$AA@ 1007dc58     LIBCMT:getqloc.obj
 0002:00015c84       ??_C@_1DE@PDBJPCJ@?$AAe?$AAn?$AAg?$AAl?$AAi?$AAs?$AAh?$AA?9?$AAt?$AAr?$AAi?$AAn?$AAi?$AAd?$AAa?$AAd?$AA?5?$AAy?$AA?5?$AAt?$AAo?$AAb?$AAa?$AAg?$AAo?$AA?$AA@ 1007dc84     LIBCMT:getqloc.obj
 0002:00015cb8       ??_C@_1BG@JGCANDME@?$AAe?$AAn?$AAg?$AAl?$AAi?$AAs?$AAh?$AA?9?$AAu?$AAk?$AA?$AA@ 1007dcb8     LIBCMT:getqloc.obj
 0002:00015cd0       ??_C@_1BG@DINKMLE@?$AAe?$AAn?$AAg?$AAl?$AAi?$AAs?$AAh?$AA?9?$AAu?$AAs?$AA?$AA@ 1007dcd0     LIBCMT:getqloc.obj
 0002:00015ce8       ??_C@_1BI@NMFDBHJE@?$AAe?$AAn?$AAg?$AAl?$AAi?$AAs?$AAh?$AA?9?$AAu?$AAs?$AAa?$AA?$AA@ 1007dce8     LIBCMT:getqloc.obj
 0002:00015d00       ??_C@_1BO@OIHKJKII@?$AAf?$AAr?$AAe?$AAn?$AAc?$AAh?$AA?9?$AAb?$AAe?$AAl?$AAg?$AAi?$AAa?$AAn?$AA?$AA@ 1007dd00     LIBCMT:getqloc.obj
 0002:00015d20       ??_C@_1CA@NKAELJKI@?$AAf?$AAr?$AAe?$AAn?$AAc?$AAh?$AA?9?$AAc?$AAa?$AAn?$AAa?$AAd?$AAi?$AAa?$AAn?$AA?$AA@ 1007dd20     LIBCMT:getqloc.obj
 0002:00015d40       ??_C@_1CE@MGKCNLGN@?$AAf?$AAr?$AAe?$AAn?$AAc?$AAh?$AA?9?$AAl?$AAu?$AAx?$AAe?$AAm?$AAb?$AAo?$AAu?$AAr?$AAg?$AA?$AA@ 1007dd40     LIBCMT:getqloc.obj
 0002:00015d64       ??_C@_1BK@CEGEAILM@?$AAf?$AAr?$AAe?$AAn?$AAc?$AAh?$AA?9?$AAs?$AAw?$AAi?$AAs?$AAs?$AA?$AA@ 1007dd64     LIBCMT:getqloc.obj
 0002:00015d80       ??_C@_1CA@PAFKEOCC@?$AAg?$AAe?$AAr?$AAm?$AAa?$AAn?$AA?9?$AAa?$AAu?$AAs?$AAt?$AAr?$AAi?$AAa?$AAn?$AA?$AA@ 1007dd80     LIBCMT:getqloc.obj
 0002:00015da0       ??_C@_1CI@HCFHGOFD@?$AAg?$AAe?$AAr?$AAm?$AAa?$AAn?$AA?9?$AAl?$AAi?$AAc?$AAh?$AAt?$AAe?$AAn?$AAs?$AAt?$AAe?$AAi?$AAn?$AA?$AA@ 1007dda0     LIBCMT:getqloc.obj
 0002:00015dc8       ??_C@_1CE@FEDDNPDG@?$AAg?$AAe?$AAr?$AAm?$AAa?$AAn?$AA?9?$AAl?$AAu?$AAx?$AAe?$AAm?$AAb?$AAo?$AAu?$AAr?$AAg?$AA?$AA@ 1007ddc8     LIBCMT:getqloc.obj
 0002:00015dec       ??_C@_1BK@LIMINNMN@?$AAg?$AAe?$AAr?$AAm?$AAa?$AAn?$AA?9?$AAs?$AAw?$AAi?$AAs?$AAs?$AA?$AA@ 1007ddec     LIBCMT:getqloc.obj
 0002:00015e08       ??_C@_1BM@LGMDBEPD@?$AAi?$AAr?$AAi?$AAs?$AAh?$AA?9?$AAe?$AAn?$AAg?$AAl?$AAi?$AAs?$AAh?$AA?$AA@ 1007de08     LIBCMT:getqloc.obj
 0002:00015e24       ??_C@_1BM@NNCFBAEE@?$AAi?$AAt?$AAa?$AAl?$AAi?$AAa?$AAn?$AA?9?$AAs?$AAw?$AAi?$AAs?$AAs?$AA?$AA@ 1007de24     LIBCMT:getqloc.obj
 0002:00015e40       ??_C@_1BE@FEDJNPIB@?$AAn?$AAo?$AAr?$AAw?$AAe?$AAg?$AAi?$AAa?$AAn?$AA?$AA@ 1007de40     LIBCMT:getqloc.obj
 0002:00015e54       ??_C@_1CC@CILKDEIE@?$AAn?$AAo?$AAr?$AAw?$AAe?$AAg?$AAi?$AAa?$AAn?$AA?9?$AAb?$AAo?$AAk?$AAm?$AAa?$AAl?$AA?$AA@ 1007de54     LIBCMT:getqloc.obj
 0002:00015e78       ??_C@_1CE@DHMMHEPL@?$AAn?$AAo?$AAr?$AAw?$AAe?$AAg?$AAi?$AAa?$AAn?$AA?9?$AAn?$AAy?$AAn?$AAo?$AAr?$AAs?$AAk?$AA?$AA@ 1007de78     LIBCMT:getqloc.obj
 0002:00015e9c       ??_C@_1CK@OPNMHECD@?$AAp?$AAo?$AAr?$AAt?$AAu?$AAg?$AAu?$AAe?$AAs?$AAe?$AA?9?$AAb?$AAr?$AAa?$AAz?$AAi?$AAl?$AAi?$AAa?$AAn?$AA?$AA@ 1007de9c     LIBCMT:getqloc.obj
 0002:00015ec8       ??_C@_1CE@KEEHCDB@?$AAs?$AAp?$AAa?$AAn?$AAi?$AAs?$AAh?$AA?9?$AAa?$AAr?$AAg?$AAe?$AAn?$AAt?$AAi?$AAn?$AAa?$AA?$AA@ 1007dec8     LIBCMT:getqloc.obj
 0002:00015eec       ??_C@_1CA@GIAOLHJD@?$AAs?$AAp?$AAa?$AAn?$AAi?$AAs?$AAh?$AA?9?$AAb?$AAo?$AAl?$AAi?$AAv?$AAi?$AAa?$AA?$AA@ 1007deec     LIBCMT:getqloc.obj
 0002:00015f0c       ??_C@_1BM@OJNDFNPD@?$AAs?$AAp?$AAa?$AAn?$AAi?$AAs?$AAh?$AA?9?$AAc?$AAh?$AAi?$AAl?$AAe?$AA?$AA@ 1007df0c     LIBCMT:getqloc.obj
 0002:00015f28       ??_C@_1CC@OCOLPALL@?$AAs?$AAp?$AAa?$AAn?$AAi?$AAs?$AAh?$AA?9?$AAc?$AAo?$AAl?$AAo?$AAm?$AAb?$AAi?$AAa?$AA?$AA@ 1007df28     LIBCMT:getqloc.obj
 0002:00015f4c       ??_C@_1CG@BPOFMKBB@?$AAs?$AAp?$AAa?$AAn?$AAi?$AAs?$AAh?$AA?9?$AAc?$AAo?$AAs?$AAt?$AAa?$AA?5?$AAr?$AAi?$AAc?$AAa?$AA?$AA@ 1007df4c     LIBCMT:getqloc.obj
 0002:00015f74       ??_C@_1DG@IGOBAPBB@?$AAs?$AAp?$AAa?$AAn?$AAi?$AAs?$AAh?$AA?9?$AAd?$AAo?$AAm?$AAi?$AAn?$AAi?$AAc?$AAa?$AAn?$AA?5?$AAr?$AAe?$AAp?$AAu?$AAb?$AAl?$AAi?$AAc?$AA?$AA@ 1007df74     LIBCMT:getqloc.obj
 0002:00015fac       ??_C@_1CA@JHAPGEGI@?$AAs?$AAp?$AAa?$AAn?$AAi?$AAs?$AAh?$AA?9?$AAe?$AAc?$AAu?$AAa?$AAd?$AAo?$AAr?$AA?$AA@ 1007dfac     LIBCMT:getqloc.obj
 0002:00015fcc       ??_C@_1CI@LAPALJPP@?$AAs?$AAp?$AAa?$AAn?$AAi?$AAs?$AAh?$AA?9?$AAe?$AAl?$AA?5?$AAs?$AAa?$AAl?$AAv?$AAa?$AAd?$AAo?$AAr?$AA?$AA@ 1007dfcc     LIBCMT:getqloc.obj
 0002:00015ff4       ??_C@_1CE@PDGBOFOM@?$AAs?$AAp?$AAa?$AAn?$AAi?$AAs?$AAh?$AA?9?$AAg?$AAu?$AAa?$AAt?$AAe?$AAm?$AAa?$AAl?$AAa?$AA?$AA@ 1007dff4     LIBCMT:getqloc.obj
 0002:00016018       ??_C@_1CC@NBEBAODI@?$AAs?$AAp?$AAa?$AAn?$AAi?$AAs?$AAh?$AA?9?$AAh?$AAo?$AAn?$AAd?$AAu?$AAr?$AAa?$AAs?$AA?$AA@ 1007e018     LIBCMT:getqloc.obj
 0002:0001603c       ??_C@_1CA@LLKGHBMF@?$AAs?$AAp?$AAa?$AAn?$AAi?$AAs?$AAh?$AA?9?$AAm?$AAe?$AAx?$AAi?$AAc?$AAa?$AAn?$AA?$AA@ 1007e03c     LIBCMT:getqloc.obj
 0002:0001605c       ??_C@_1BO@LKNDOIGD@?$AAs?$AAp?$AAa?$AAn?$AAi?$AAs?$AAh?$AA?9?$AAm?$AAo?$AAd?$AAe?$AAr?$AAn?$AA?$AA@ 1007e05c     LIBCMT:getqloc.obj
 0002:0001607c       ??_C@_1CE@NMDMOEEB@?$AAs?$AAp?$AAa?$AAn?$AAi?$AAs?$AAh?$AA?9?$AAn?$AAi?$AAc?$AAa?$AAr?$AAa?$AAg?$AAu?$AAa?$AA?$AA@ 1007e07c     LIBCMT:getqloc.obj
 0002:000160a0       ??_C@_1BO@LLCBEJGB@?$AAs?$AAp?$AAa?$AAn?$AAi?$AAs?$AAh?$AA?9?$AAp?$AAa?$AAn?$AAa?$AAm?$AAa?$AA?$AA@ 1007e0a0     LIBCMT:getqloc.obj
 0002:000160c0       ??_C@_1CC@FKPGGIHO@?$AAs?$AAp?$AAa?$AAn?$AAi?$AAs?$AAh?$AA?9?$AAp?$AAa?$AAr?$AAa?$AAg?$AAu?$AAa?$AAy?$AA?$AA@ 1007e0c0     LIBCMT:getqloc.obj
 0002:000160e4       ??_C@_1BK@CDEIHOOP@?$AAs?$AAp?$AAa?$AAn?$AAi?$AAs?$AAh?$AA?9?$AAp?$AAe?$AAr?$AAu?$AA?$AA@ 1007e0e4     LIBCMT:getqloc.obj
 0002:00016100       ??_C@_1CI@GAHAKKGP@?$AAs?$AAp?$AAa?$AAn?$AAi?$AAs?$AAh?$AA?9?$AAp?$AAu?$AAe?$AAr?$AAt?$AAo?$AA?5?$AAr?$AAi?$AAc?$AAo?$AA?$AA@ 1007e100     LIBCMT:getqloc.obj
 0002:00016128       ??_C@_1CA@NKJBCAGP@?$AAs?$AAp?$AAa?$AAn?$AAi?$AAs?$AAh?$AA?9?$AAu?$AAr?$AAu?$AAg?$AAu?$AAa?$AAy?$AA?$AA@ 1007e128     LIBCMT:getqloc.obj
 0002:00016148       ??_C@_1CE@ODILCONM@?$AAs?$AAp?$AAa?$AAn?$AAi?$AAs?$AAh?$AA?9?$AAv?$AAe?$AAn?$AAe?$AAz?$AAu?$AAe?$AAl?$AAa?$AA?$AA@ 1007e148     LIBCMT:getqloc.obj
 0002:0001616c       ??_C@_1CA@OBNMCGFO@?$AAs?$AAw?$AAe?$AAd?$AAi?$AAs?$AAh?$AA?9?$AAf?$AAi?$AAn?$AAl?$AAa?$AAn?$AAd?$AA?$AA@ 1007e16c     LIBCMT:getqloc.obj
 0002:0001618c       ??_C@_1M@PIPDDPPI@?$AAs?$AAw?$AAi?$AAs?$AAs?$AA?$AA@ 1007e18c     LIBCMT:getqloc.obj
 0002:00016198       ??_C@_15PJPFLCCM@?$AAu?$AAk?$AA?$AA@ 1007e198     LIBCMT:getqloc.obj
 0002:000161a0       ??_C@_15GMFIMNFM@?$AAu?$AAs?$AA?$AA@ 1007e1a0     LIBCMT:getqloc.obj
 0002:000161a8       ??_C@_17HAEBFAGL@?$AAu?$AAs?$AAa?$AA?$AA@ 1007e1a8     LIBCMT:getqloc.obj
 0002:000161b0       ___rg_country              1007e1b0     LIBCMT:getqloc.obj
 0002:000162c4       ??_C@_1BA@DPFJEPHB@?$AAa?$AAm?$AAe?$AAr?$AAi?$AAc?$AAa?$AA?$AA@ 1007e2c4     LIBCMT:getqloc.obj
 0002:000162d4       ??_C@_1BA@ELOGGFK@?$AAb?$AAr?$AAi?$AAt?$AAa?$AAi?$AAn?$AA?$AA@ 1007e2d4     LIBCMT:getqloc.obj
 0002:000162e4       ??_C@_1M@GHBGIGDA@?$AAc?$AAh?$AAi?$AAn?$AAa?$AA?$AA@ 1007e2e4     LIBCMT:getqloc.obj
 0002:000162f0       ??_C@_1M@NCHEJOPO@?$AAc?$AAz?$AAe?$AAc?$AAh?$AA?$AA@ 1007e2f0     LIBCMT:getqloc.obj
 0002:000162fc       ??_C@_1BA@BKPAPBLA@?$AAe?$AAn?$AAg?$AAl?$AAa?$AAn?$AAd?$AA?$AA@ 1007e2fc     LIBCMT:getqloc.obj
 0002:0001630c       ??_C@_1BM@HKBCKIPC@?$AAg?$AAr?$AAe?$AAa?$AAt?$AA?5?$AAb?$AAr?$AAi?$AAt?$AAa?$AAi?$AAn?$AA?$AA@ 1007e30c     LIBCMT:getqloc.obj
 0002:00016328       ??_C@_1BA@PPCHPGJB@?$AAh?$AAo?$AAl?$AAl?$AAa?$AAn?$AAd?$AA?$AA@ 1007e328     LIBCMT:getqloc.obj
 0002:00016338       ??_C@_1BE@JBMPEGDG@?$AAh?$AAo?$AAn?$AAg?$AA?9?$AAk?$AAo?$AAn?$AAg?$AA?$AA@ 1007e338     LIBCMT:getqloc.obj
 0002:0001634c       ??_C@_1BI@KOELBBPJ@?$AAn?$AAe?$AAw?$AA?9?$AAz?$AAe?$AAa?$AAl?$AAa?$AAn?$AAd?$AA?$AA@ 1007e34c     LIBCMT:getqloc.obj
 0002:00016364       ??_C@_15HIEBHAIO@?$AAn?$AAz?$AA?$AA@ 1007e364     LIBCMT:getqloc.obj
 0002:0001636c       ??_C@_1BC@CHBCPFPI@?$AAp?$AAr?$AA?5?$AAc?$AAh?$AAi?$AAn?$AAa?$AA?$AA@ 1007e36c     LIBCMT:getqloc.obj
 0002:00016380       ??_C@_1BC@JAOIIFKD@?$AAp?$AAr?$AA?9?$AAc?$AAh?$AAi?$AAn?$AAa?$AA?$AA@ 1007e380     LIBCMT:getqloc.obj
 0002:00016394       ??_C@_1BI@BEHPPHKC@?$AAp?$AAu?$AAe?$AAr?$AAt?$AAo?$AA?9?$AAr?$AAi?$AAc?$AAo?$AA?$AA@ 1007e394     LIBCMT:getqloc.obj
 0002:000163ac       ??_C@_1O@PAEOFKDI@?$AAs?$AAl?$AAo?$AAv?$AAa?$AAk?$AA?$AA@ 1007e3ac     LIBCMT:getqloc.obj
 0002:000163bc       ??_C@_1BK@FIHMCKAM@?$AAs?$AAo?$AAu?$AAt?$AAh?$AA?5?$AAa?$AAf?$AAr?$AAi?$AAc?$AAa?$AA?$AA@ 1007e3bc     LIBCMT:getqloc.obj
 0002:000163d8       ??_C@_1BI@NAEOODKB@?$AAs?$AAo?$AAu?$AAt?$AAh?$AA?5?$AAk?$AAo?$AAr?$AAe?$AAa?$AA?$AA@ 1007e3d8     LIBCMT:getqloc.obj
 0002:000163f0       ??_C@_1BK@FBDGGIFF@?$AAs?$AAo?$AAu?$AAt?$AAh?$AA?9?$AAa?$AAf?$AAr?$AAi?$AAc?$AAa?$AA?$AA@ 1007e3f0     LIBCMT:getqloc.obj
 0002:0001640c       ??_C@_1BI@GHLEJDPK@?$AAs?$AAo?$AAu?$AAt?$AAh?$AA?9?$AAk?$AAo?$AAr?$AAe?$AAa?$AA?$AA@ 1007e40c     LIBCMT:getqloc.obj
 0002:00016424       ??_C@_1CE@PLHLOMJF@?$AAt?$AAr?$AAi?$AAn?$AAi?$AAd?$AAa?$AAd?$AA?5?$AA?$CG?$AA?5?$AAt?$AAo?$AAb?$AAa?$AAg?$AAo?$AA?$AA@ 1007e424     LIBCMT:getqloc.obj
 0002:00016448       ??_C@_1BO@MODIMHHI@?$AAu?$AAn?$AAi?$AAt?$AAe?$AAd?$AA?9?$AAk?$AAi?$AAn?$AAg?$AAd?$AAo?$AAm?$AA?$AA@ 1007e448     LIBCMT:getqloc.obj
 0002:00016468       ??_C@_1BM@FFHJONBJ@?$AAu?$AAn?$AAi?$AAt?$AAe?$AAd?$AA?9?$AAs?$AAt?$AAa?$AAt?$AAe?$AAs?$AA?$AA@ 1007e468     LIBCMT:getqloc.obj
 0002:00016484       ___rg_language_count       1007e484     LIBCMT:getqloc.obj
 0002:00016488       ___rg_country_count        1007e488     LIBCMT:getqloc.obj
 0002:0001648c       ??_C@_17DNCLJFIF@?$AAA?$AAC?$AAP?$AA?$AA@ 1007e48c     LIBCMT:getqloc.obj
 0002:00016494       ??_C@_17CIKBIHLH@?$AAO?$AAC?$AAP?$AA?$AA@ 1007e494     LIBCMT:getqloc.obj
 0002:0001649c       ___rglangidNotDefault      1007e49c     LIBCMT:getqloc_downlevel.obj
 0002:000164b0       _LcidToLocaleNameTable     1007e4b0     LIBCMT:winapinls.obj
 0002:00016bd0       _LocaleNameToIndexTable    1007ebd0     LIBCMT:winapinls.obj
 0002:000172f0       ??_C@_15EMKDOKLE@?$AAa?$AAr?$AA?$AA@ 1007f2f0     LIBCMT:winapinls.obj
 0002:000172f8       ??_C@_15KNPADPLH@?$AAb?$AAg?$AA?$AA@ 1007f2f8     LIBCMT:winapinls.obj
 0002:00017300       ??_C@_15EDMHLDMO@?$AAc?$AAa?$AA?$AA@ 1007f300     LIBCMT:winapinls.obj
 0002:00017308       ??_C@_1O@BPEAJADD@?$AAz?$AAh?$AA?9?$AAC?$AAH?$AAS?$AA?$AA@ 1007f308     LIBCMT:winapinls.obj
 0002:00017318       ??_C@_15LJNHCMNK@?$AAc?$AAs?$AA?$AA@ 1007f318     LIBCMT:winapinls.obj
 0002:00017320       ??_C@_15FOMCIDHG@?$AAd?$AAa?$AA?$AA@ 1007f320     LIBCMT:winapinls.obj
 0002:00017328       ??_C@_15NBKABECB@?$AAd?$AAe?$AA?$AA@ 1007f328     LIBCMT:winapinls.obj
 0002:00017330       ??_C@_15GHPEIIAO@?$AAe?$AAl?$AA?$AA@ 1007f330     LIBCMT:winapinls.obj
 0002:00017338       ??_C@_15MNPNEAIF@?$AAe?$AAn?$AA?$AA@ 1007f338     LIBCMT:winapinls.obj
 0002:00017340       ??_C@_15GPIOMPMH@?$AAe?$AAs?$AA?$AA@ 1007f340     LIBCMT:winapinls.obj
 0002:00017348       ??_C@_15NGLOAKJC@?$AAf?$AAi?$AA?$AA@ 1007f348     LIBCMT:winapinls.obj
 0002:00017350       ??_C@_15FBKGNKAM@?$AAf?$AAr?$AA?$AA@ 1007f350     LIBCMT:winapinls.obj
 0002:00017358       ??_C@_15KGGCNEFK@?$AAh?$AAe?$AA?$AA@ 1007f358     LIBCMT:winapinls.obj
 0002:00017360       ??_C@_15PGHLIDMF@?$AAh?$AAu?$AA?$AA@ 1007f360     LIBCMT:winapinls.obj
 0002:00017368       ??_C@_15BIEMAPLM@?$AAi?$AAs?$AA?$AA@ 1007f368     LIBCMT:winapinls.obj
 0002:00017370       ??_C@_15IFJLDHAF@?$AAi?$AAt?$AA?$AA@ 1007f370     LIBCMT:winapinls.obj
 0002:00017378       ??_C@_15GEMIOCAG@?$AAj?$AAa?$AA?$AA@ 1007f378     LIBCMT:winapinls.obj
 0002:00017380       ??_C@_15EPELEGJA@?$AAk?$AAo?$AA?$AA@ 1007f380     LIBCMT:winapinls.obj
 0002:00017388       ??_C@_15NDDHIMN@?$AAn?$AAl?$AA?$AA@ 1007f388     LIBCMT:winapinls.obj
 0002:00017390       ??_C@_15BPIGNHCD@?$AAn?$AAo?$AA?$AA@ 1007f390     LIBCMT:winapinls.obj
 0002:00017398       ??_C@_15DEOPBLCG@?$AAp?$AAl?$AA?$AA@ 1007f398     LIBCMT:winapinls.obj
 0002:000173a0       ??_C@_15KBECGEFG@?$AAp?$AAt?$AA?$AA@ 1007f3a0     LIBCMT:winapinls.obj
 0002:000173a8       ??_C@_15GLJCBFMD@?$AAr?$AAo?$AA?$AA@ 1007f3a8     LIBCMT:winapinls.obj
 0002:000173b0       ??_C@_15FEDGKCDI@?$AAr?$AAu?$AA?$AA@ 1007f3b0     LIBCMT:winapinls.obj
 0002:000173b8       ??_C@_15GLKMLLHM@?$AAh?$AAr?$AA?$AA@ 1007f3b8     LIBCMT:winapinls.obj
 0002:000173c0       ??_C@_15CPKMFBDB@?$AAs?$AAk?$AA?$AA@ 1007f3c0     LIBCMT:winapinls.obj
 0002:000173c8       ??_C@_15BAAIOGMK@?$AAs?$AAq?$AA?$AA@ 1007f3c8     LIBCMT:winapinls.obj
 0002:000173d0       ??_C@_15INNPNOHD@?$AAs?$AAv?$AA?$AA@ 1007f3d0     LIBCMT:winapinls.obj
 0002:000173d8       ??_C@_15CABMMOGH@?$AAt?$AAh?$AA?$AA@ 1007f3d8     LIBCMT:winapinls.obj
 0002:000173e0       ??_C@_15BPLIHJJM@?$AAt?$AAr?$AA?$AA@ 1007f3e0     LIBCMT:winapinls.obj
 0002:000173e8       ??_C@_15NEOEKKDJ@?$AAu?$AAr?$AA?$AA@ 1007f3e8     LIBCMT:winapinls.obj
 0002:000173f0       ??_C@_15NFICGAJK@?$AAi?$AAd?$AA?$AA@ 1007f3f0     LIBCMT:winapinls.obj
 0002:000173f8       ??_C@_15HPJPHDM@?$AAb?$AAe?$AA?$AA@ 1007f3f8     LIBCMT:winapinls.obj
 0002:00017400       ??_C@_15LCHLGJII@?$AAs?$AAl?$AA?$AA@ 1007f400     LIBCMT:winapinls.obj
 0002:00017408       ??_C@_15PCFJPHHO@?$AAe?$AAt?$AA?$AA@ 1007f408     LIBCMT:winapinls.obj
 0002:00017410       ??_C@_15HPFPGODN@?$AAl?$AAv?$AA?$AA@ 1007f410     LIBCMT:winapinls.obj
 0002:00017418       ??_C@_15NFFGKGLG@?$AAl?$AAt?$AA?$AA@ 1007f418     LIBCMT:winapinls.obj
 0002:00017420       ??_C@_15BDAKCCHN@?$AAf?$AAa?$AA?$AA@ 1007f420     LIBCMT:winapinls.obj
 0002:00017428       ??_C@_15NFGIAIAJ@?$AAv?$AAi?$AA?$AA@ 1007f428     LIBCMT:winapinls.obj
 0002:00017430       ??_C@_15LMKNDMHN@?$AAh?$AAy?$AA?$AA@ 1007f430     LIBCMT:winapinls.obj
 0002:00017438       ??_C@_15IJBHMCFL@?$AAa?$AAz?$AA?$AA@ 1007f438     LIBCMT:winapinls.obj
 0002:00017440       ??_C@_15EKOFJABL@?$AAe?$AAu?$AA?$AA@ 1007f440     LIBCMT:winapinls.obj
 0002:00017448       ??_C@_15BGHADCNK@?$AAm?$AAk?$AA?$AA@ 1007f448     LIBCMT:winapinls.obj
 0002:00017450       ??_C@_15JDNICKHM@?$AAa?$AAf?$AA?$AA@ 1007f450     LIBCMT:winapinls.obj
 0002:00017458       ??_C@_15KPJEDBKD@?$AAk?$AAa?$AA?$AA@ 1007f458     LIBCMT:winapinls.obj
 0002:00017460       ??_C@_15PDNFFFEO@?$AAf?$AAo?$AA?$AA@ 1007f460     LIBCMT:winapinls.obj
 0002:00017468       ??_C@_15OMLEGLOC@?$AAh?$AAi?$AA?$AA@ 1007f468     LIBCMT:winapinls.obj
 0002:00017470       ??_C@_15IDNNENKK@?$AAm?$AAs?$AA?$AA@ 1007f470     LIBCMT:winapinls.obj
 0002:00017478       ??_C@_15MACJNBMH@?$AAk?$AAk?$AA?$AA@ 1007f478     LIBCMT:winapinls.obj
 0002:00017480       ??_C@_15DKDJEOND@?$AAk?$AAy?$AA?$AA@ 1007f480     LIBCMT:winapinls.obj
 0002:00017488       ??_C@_15DFGDLJBG@?$AAs?$AAw?$AA?$AA@ 1007f488     LIBCMT:winapinls.obj
 0002:00017490       ??_C@_15BBFAICNG@?$AAu?$AAz?$AA?$AA@ 1007f490     LIBCMT:winapinls.obj
 0002:00017498       ??_C@_15DKNDCGEA@?$AAt?$AAt?$AA?$AA@ 1007f498     LIBCMT:winapinls.obj
 0002:000174a0       ??_C@_15MGIFMDPL@?$AAp?$AAa?$AA?$AA@ 1007f4a0     LIBCMT:winapinls.obj
 0002:000174a8       ??_C@_15HCNDBBA@?$AAg?$AAu?$AA?$AA@ 1007f4a8     LIBCMT:winapinls.obj
 0002:000174b0       ??_C@_15FNBEIBON@?$AAt?$AAa?$AA?$AA@ 1007f4b0     LIBCMT:winapinls.obj
 0002:000174b8       ??_C@_15NCHGBGLK@?$AAt?$AAe?$AA?$AA@ 1007f4b8     LIBCMT:winapinls.obj
 0002:000174c0       ??_C@_15PHPHCBPF@?$AAk?$AAn?$AA?$AA@ 1007f4c0     LIBCMT:winapinls.obj
 0002:000174c8       ??_C@_15DLGBCKMP@?$AAm?$AAr?$AA?$AA@ 1007f4c8     LIBCMT:winapinls.obj
 0002:000174d0       ??_C@_15EABBLBFF@?$AAs?$AAa?$AA?$AA@ 1007f4d0     LIBCMT:winapinls.obj
 0002:000174d8       ??_C@_15CBKOMCOI@?$AAm?$AAn?$AA?$AA@ 1007f4d8     LIBCMT:winapinls.obj
 0002:000174e0       ??_C@_15CKDMCJAF@?$AAg?$AAl?$AA?$AA@ 1007f4e0     LIBCMT:winapinls.obj
 0002:000174e8       ??_C@_17CNJFBPG@?$AAk?$AAo?$AAk?$AA?$AA@ 1007f4e8     LIBCMT:winapinls.obj
 0002:000174f0       ??_C@_17FFBJICPL@?$AAs?$AAy?$AAr?$AA?$AA@ 1007f4f0     LIBCMT:winapinls.obj
 0002:000174f8       ??_C@_17KPNDCPAF@?$AAd?$AAi?$AAv?$AA?$AA@ 1007f4f8     LIBCMT:winapinls.obj
 0002:00017500       ??_C@_11LOCGONAA@?$AA?$AA@ 1007f500     LIBCMT:winapinls.obj
 0002:00017504       ??_C@_1M@OKAHONE@?$AAa?$AAr?$AA?9?$AAS?$AAA?$AA?$AA@ 1007f504     LIBCMT:winapinls.obj
 0002:00017510       ??_C@_1M@FFFIGIGK@?$AAb?$AAg?$AA?9?$AAB?$AAG?$AA?$AA@ 1007f510     LIBCMT:winapinls.obj
 0002:0001751c       ??_C@_1M@BJNKEDC@?$AAc?$AAa?$AA?9?$AAE?$AAS?$AA?$AA@ 1007f51c     LIBCMT:winapinls.obj
 0002:00017528       ??_C@_1M@IJJHFJHA@?$AAc?$AAs?$AA?9?$AAC?$AAZ?$AA?$AA@ 1007f528     LIBCMT:winapinls.obj
 0002:00017534       ??_C@_1M@CLPEOBGI@?$AAd?$AAa?$AA?9?$AAD?$AAK?$AA?$AA@ 1007f534     LIBCMT:winapinls.obj
 0002:00017540       ??_C@_1M@MCMADGCB@?$AAd?$AAe?$AA?9?$AAD?$AAE?$AA?$AA@ 1007f540     LIBCMT:winapinls.obj
 0002:0001754c       ??_C@_1M@OOCKEMAM@?$AAe?$AAl?$AA?9?$AAG?$AAR?$AA?$AA@ 1007f54c     LIBCMT:winapinls.obj
 0002:00017558       ??_C@_1M@DDNJFGID@?$AAf?$AAi?$AA?9?$AAF?$AAI?$AA?$AA@ 1007f558     LIBCMT:winapinls.obj
 0002:00017564       ??_C@_1M@GLIPPMAC@?$AAf?$AAr?$AA?9?$AAF?$AAR?$AA?$AA@ 1007f564     LIBCMT:winapinls.obj
 0002:00017570       ??_C@_1M@GFMCHPE@?$AAh?$AAe?$AA?9?$AAI?$AAL?$AA?$AA@ 1007f570     LIBCMT:winapinls.obj
 0002:0001757c       ??_C@_1M@MHLPGNKM@?$AAh?$AAu?$AA?9?$AAH?$AAU?$AA?$AA@ 1007f57c     LIBCMT:winapinls.obj
 0002:00017588       ??_C@_1M@LPDDNNPN@?$AAi?$AAs?$AA?9?$AAI?$AAS?$AA?$AA@ 1007f588     LIBCMT:winapinls.obj
 0002:00017594       ??_C@_1M@MADIPODN@?$AAi?$AAt?$AA?9?$AAI?$AAT?$AA?$AA@ 1007f594     LIBCMT:winapinls.obj
 0002:000175a0       ??_C@_1M@IHBJJGG@?$AAn?$AAl?$AA?9?$AAN?$AAL?$AA?$AA@ 1007f5a0     LIBCMT:winapinls.obj
 0002:000175ac       ??_C@_1M@EANAGDL@?$AAn?$AAb?$AA?9?$AAN?$AAO?$AA?$AA@ 1007f5ac     LIBCMT:winapinls.obj
 0002:000175b8       ??_C@_1M@NEIEMEGP@?$AAp?$AAl?$AA?9?$AAP?$AAL?$AA?$AA@ 1007f5b8     LIBCMT:winapinls.obj
 0002:000175c4       ??_C@_1M@BOCFIGEP@?$AAp?$AAt?$AA?9?$AAB?$AAR?$AA?$AA@ 1007f5c4     LIBCMT:winapinls.obj
 0002:000175d0       ??_C@_1M@IMPFOPBG@?$AAr?$AAo?$AA?9?$AAR?$AAO?$AA?$AA@ 1007f5d0     LIBCMT:winapinls.obj
 0002:000175dc       ??_C@_1M@IDNNEJMM@?$AAr?$AAu?$AA?9?$AAR?$AAU?$AA?$AA@ 1007f5dc     LIBCMT:winapinls.obj
 0002:000175e8       ??_C@_1M@LILEEOGM@?$AAh?$AAr?$AA?9?$AAH?$AAR?$AA?$AA@ 1007f5e8     LIBCMT:winapinls.obj
 0002:000175f4       ??_C@_1M@FKIFEHPB@?$AAs?$AAk?$AA?9?$AAS?$AAK?$AA?$AA@ 1007f5f4     LIBCMT:winapinls.obj
 0002:00017600       ??_C@_1M@LJMAMNPJ@?$AAs?$AAq?$AA?9?$AAA?$AAL?$AA?$AA@ 1007f600     LIBCMT:winapinls.obj
 0002:0001760c       ??_C@_1M@GIAKDKJK@?$AAs?$AAv?$AA?9?$AAS?$AAE?$AA?$AA@ 1007f60c     LIBCMT:winapinls.obj
 0002:00017618       ??_C@_1M@MKJKIKCL@?$AAt?$AAh?$AA?9?$AAT?$AAH?$AA?$AA@ 1007f618     LIBCMT:winapinls.obj
 0002:00017624       ??_C@_1M@MFLCCMPB@?$AAt?$AAr?$AA?9?$AAT?$AAR?$AA?$AA@ 1007f624     LIBCMT:winapinls.obj
 0002:00017630       ??_C@_1M@OIJHDKJN@?$AAu?$AAr?$AA?9?$AAP?$AAK?$AA?$AA@ 1007f630     LIBCMT:winapinls.obj
 0002:0001763c       ??_C@_1M@LHIPCIEK@?$AAi?$AAd?$AA?9?$AAI?$AAD?$AA?$AA@ 1007f63c     LIBCMT:winapinls.obj
 0002:00017648       ??_C@_1M@MFMOBGI@?$AAu?$AAk?$AA?9?$AAU?$AAA?$AA?$AA@ 1007f648     LIBCMT:winapinls.obj
 0002:00017654       ??_C@_1M@OBGLJIPL@?$AAb?$AAe?$AA?9?$AAB?$AAY?$AA?$AA@ 1007f654     LIBCMT:winapinls.obj
 0002:00017660       ??_C@_1M@BCFAJEAD@?$AAs?$AAl?$AA?9?$AAS?$AAI?$AA?$AA@ 1007f660     LIBCMT:winapinls.obj
 0002:0001766c       ??_C@_1M@FKFFEDDN@?$AAe?$AAt?$AA?9?$AAE?$AAE?$AA?$AA@ 1007f66c     LIBCMT:winapinls.obj
 0002:00017678       ??_C@_1M@KGKKAACI@?$AAl?$AAv?$AA?9?$AAL?$AAV?$AA?$AA@ 1007f678     LIBCMT:winapinls.obj
 0002:00017684       ??_C@_1M@IFGBIJO@?$AAl?$AAt?$AA?9?$AAL?$AAT?$AA?$AA@ 1007f684     LIBCMT:winapinls.obj
 0002:00017690       ??_C@_1M@FGEAHEDM@?$AAf?$AAa?$AA?9?$AAI?$AAR?$AA?$AA@ 1007f690     LIBCMT:winapinls.obj
 0002:0001769c       ??_C@_1M@KBMAIBFN@?$AAv?$AAi?$AA?9?$AAV?$AAN?$AA?$AA@ 1007f69c     LIBCMT:winapinls.obj
 0002:000176a8       ??_C@_1M@GPCBKDJK@?$AAh?$AAy?$AA?9?$AAA?$AAM?$AA?$AA@ 1007f6a8     LIBCMT:winapinls.obj
 0002:000176b4       ??_C@_1BG@BECMDDJB@?$AAa?$AAz?$AA?9?$AAA?$AAZ?$AA?9?$AAL?$AAa?$AAt?$AAn?$AA?$AA@ 1007f6b4     LIBCMT:winapinls.obj
 0002:000176cc       ??_C@_1M@MAOFCAEA@?$AAe?$AAu?$AA?9?$AAE?$AAS?$AA?$AA@ 1007f6cc     LIBCMT:winapinls.obj
 0002:000176d8       ??_C@_1M@IGHABKPI@?$AAm?$AAk?$AA?9?$AAM?$AAK?$AA?$AA@ 1007f6d8     LIBCMT:winapinls.obj
 0002:000176e4       ??_C@_1M@IAIGNEJG@?$AAt?$AAn?$AA?9?$AAZ?$AAA?$AA?$AA@ 1007f6e4     LIBCMT:winapinls.obj
 0002:000176f0       ??_C@_1M@IIJCOJFA@?$AAx?$AAh?$AA?9?$AAZ?$AAA?$AA?$AA@ 1007f6f0     LIBCMT:winapinls.obj
 0002:000176fc       ??_C@_1M@LGPJHNJH@?$AAz?$AAu?$AA?9?$AAZ?$AAA?$AA?$AA@ 1007f6fc     LIBCMT:winapinls.obj
 0002:00017708       ??_C@_1M@HOKAOIO@?$AAa?$AAf?$AA?9?$AAZ?$AAA?$AA?$AA@ 1007f708     LIBCMT:winapinls.obj
 0002:00017714       ??_C@_1M@DPCLHLIE@?$AAk?$AAa?$AA?9?$AAG?$AAE?$AA?$AA@ 1007f714     LIBCMT:winapinls.obj
 0002:00017720       ??_C@_1M@BLKMHJBI@?$AAf?$AAo?$AA?9?$AAF?$AAO?$AA?$AA@ 1007f720     LIBCMT:winapinls.obj
 0002:0001772c       ??_C@_1M@LGGJAPPB@?$AAh?$AAi?$AA?9?$AAI?$AAN?$AA?$AA@ 1007f72c     LIBCMT:winapinls.obj
 0002:00017738       ??_C@_1M@FIKPIHFE@?$AAm?$AAt?$AA?9?$AAM?$AAT?$AA?$AA@ 1007f738     LIBCMT:winapinls.obj
 0002:00017744       ??_C@_1M@HEGGPBFA@?$AAs?$AAe?$AA?9?$AAN?$AAO?$AA?$AA@ 1007f744     LIBCMT:winapinls.obj
 0002:00017750       ??_C@_1M@EIBJEEPA@?$AAm?$AAs?$AA?9?$AAM?$AAY?$AA?$AA@ 1007f750     LIBCMT:winapinls.obj
 0002:0001775c       ??_C@_1M@FHLBGMPP@?$AAk?$AAk?$AA?9?$AAK?$AAZ?$AA?$AA@ 1007f75c     LIBCMT:winapinls.obj
 0002:00017768       ??_C@_1M@NGJJLCGI@?$AAk?$AAy?$AA?9?$AAK?$AAG?$AA?$AA@ 1007f768     LIBCMT:winapinls.obj
 0002:00017774       ??_C@_1M@GIENNBFC@?$AAs?$AAw?$AA?9?$AAK?$AAE?$AA?$AA@ 1007f774     LIBCMT:winapinls.obj
 0002:00017780       ??_C@_1BG@NDGMJIMJ@?$AAu?$AAz?$AA?9?$AAU?$AAZ?$AA?9?$AAL?$AAa?$AAt?$AAn?$AA?$AA@ 1007f780     LIBCMT:winapinls.obj
 0002:00017798       ??_C@_1M@IDCCIHBC@?$AAt?$AAt?$AA?9?$AAR?$AAU?$AA?$AA@ 1007f798     LIBCMT:winapinls.obj
 0002:000177a4       ??_C@_1M@LOICPMOJ@?$AAb?$AAn?$AA?9?$AAI?$AAN?$AA?$AA@ 1007f7a4     LIBCMT:winapinls.obj
 0002:000177b0       ??_C@_1M@KPKKNEAH@?$AAp?$AAa?$AA?9?$AAI?$AAN?$AA?$AA@ 1007f7b0     LIBCMT:winapinls.obj
 0002:000177bc       ??_C@_1M@PJGPPBOG@?$AAg?$AAu?$AA?9?$AAI?$AAN?$AA?$AA@ 1007f7bc     LIBCMT:winapinls.obj
 0002:000177c8       ??_C@_1M@KMKMOPHI@?$AAt?$AAa?$AA?9?$AAI?$AAN?$AA?$AA@ 1007f7c8     LIBCMT:winapinls.obj
 0002:000177d4       ??_C@_1M@KFEHEPAC@?$AAt?$AAe?$AA?9?$AAI?$AAN?$AA?$AA@ 1007f7d4     LIBCMT:winapinls.obj
 0002:000177e0       ??_C@_1M@CDCLMGHI@?$AAk?$AAn?$AA?9?$AAI?$AAN?$AA?$AA@ 1007f7e0     LIBCMT:winapinls.obj
 0002:000177ec       ??_C@_1M@MIODLDKF@?$AAm?$AAl?$AA?9?$AAI?$AAN?$AA?$AA@ 1007f7ec     LIBCMT:winapinls.obj
 0002:000177f8       ??_C@_1M@PBIEACPO@?$AAm?$AAr?$AA?9?$AAI?$AAN?$AA?$AA@ 1007f7f8     LIBCMT:winapinls.obj
 0002:00017804       ??_C@_1M@NIDEAGPH@?$AAs?$AAa?$AA?9?$AAI?$AAN?$AA?$AA@ 1007f804     LIBCMT:winapinls.obj
 0002:00017810       ??_C@_1M@FHIHCBIO@?$AAm?$AAn?$AA?9?$AAM?$AAN?$AA?$AA@ 1007f810     LIBCMT:winapinls.obj
 0002:0001781c       ??_C@_1M@JAIJPENP@?$AAc?$AAy?$AA?9?$AAG?$AAB?$AA?$AA@ 1007f81c     LIBCMT:winapinls.obj
 0002:00017828       ??_C@_1M@PHGFBEPN@?$AAg?$AAl?$AA?9?$AAE?$AAS?$AA?$AA@ 1007f828     LIBCMT:winapinls.obj
 0002:00017834       ??_C@_1O@KPIPDNCP@?$AAk?$AAo?$AAk?$AA?9?$AAI?$AAN?$AA?$AA@ 1007f834     LIBCMT:winapinls.obj
 0002:00017844       ??_C@_1O@KNHJLDJA@?$AAs?$AAy?$AAr?$AA?9?$AAS?$AAY?$AA?$AA@ 1007f844     LIBCMT:winapinls.obj
 0002:00017854       ??_C@_1O@MKEKBLAH@?$AAd?$AAi?$AAv?$AA?9?$AAM?$AAV?$AA?$AA@ 1007f854     LIBCMT:winapinls.obj
 0002:00017864       ??_C@_1O@OHDCKDDF@?$AAq?$AAu?$AAz?$AA?9?$AAB?$AAO?$AA?$AA@ 1007f864     LIBCMT:winapinls.obj
 0002:00017874       ??_C@_1M@LEPJNLFD@?$AAn?$AAs?$AA?9?$AAZ?$AAA?$AA?$AA@ 1007f874     LIBCMT:winapinls.obj
 0002:00017880       ??_C@_1M@OMLEIIJB@?$AAm?$AAi?$AA?9?$AAN?$AAZ?$AA?$AA@ 1007f880     LIBCMT:winapinls.obj
 0002:0001788c       ??_C@_1M@PMPEAILG@?$AAa?$AAr?$AA?9?$AAI?$AAQ?$AA?$AA@ 1007f88c     LIBCMT:winapinls.obj
 0002:00017898       ??_C@_1M@CNKPNOEE@?$AAd?$AAe?$AA?9?$AAC?$AAH?$AA?$AA@ 1007f898     LIBCMT:winapinls.obj
 0002:000178a4       ??_C@_1M@LKMGMLKO@?$AAe?$AAn?$AA?9?$AAG?$AAB?$AA?$AA@ 1007f8a4     LIBCMT:winapinls.obj
 0002:000178b0       ??_C@_1M@PGKJFFGL@?$AAe?$AAs?$AA?9?$AAM?$AAX?$AA?$AA@ 1007f8b0     LIBCMT:winapinls.obj
 0002:000178bc       ??_C@_1M@DNNANBDC@?$AAf?$AAr?$AA?9?$AAB?$AAE?$AA?$AA@ 1007f8bc     LIBCMT:winapinls.obj
 0002:000178c8       ??_C@_1M@HLGMDFHM@?$AAi?$AAt?$AA?9?$AAC?$AAH?$AA?$AA@ 1007f8c8     LIBCMT:winapinls.obj
 0002:000178d4       ??_C@_1M@CLLBGJH@?$AAn?$AAl?$AA?9?$AAB?$AAE?$AA?$AA@ 1007f8d4     LIBCMT:winapinls.obj
 0002:000178e0       ??_C@_1M@BODBOGLF@?$AAn?$AAn?$AA?9?$AAN?$AAO?$AA?$AA@ 1007f8e0     LIBCMT:winapinls.obj
 0002:000178ec       ??_C@_1M@HFFAHKAD@?$AAp?$AAt?$AA?9?$AAP?$AAT?$AA?$AA@ 1007f8ec     LIBCMT:winapinls.obj
 0002:000178f8       ??_C@_1BG@LNOAKHIE@?$AAs?$AAr?$AA?9?$AAS?$AAP?$AA?9?$AAL?$AAa?$AAt?$AAn?$AA?$AA@ 1007f8f8     LIBCMT:winapinls.obj
 0002:00017910       ??_C@_1M@HBMHBGAK@?$AAs?$AAv?$AA?9?$AAF?$AAI?$AA?$AA@ 1007f910     LIBCMT:winapinls.obj
 0002:0001791c       ??_C@_1BG@DGCJGJBE@?$AAa?$AAz?$AA?9?$AAA?$AAZ?$AA?9?$AAC?$AAy?$AAr?$AAl?$AA?$AA@ 1007f91c     LIBCMT:winapinls.obj
 0002:00017934       ??_C@_1M@KEJDAAHB@?$AAs?$AAe?$AA?9?$AAS?$AAE?$AA?$AA@ 1007f934     LIBCMT:winapinls.obj
 0002:00017940       ??_C@_1M@HEIBJJAD@?$AAm?$AAs?$AA?9?$AAB?$AAN?$AA?$AA@ 1007f940     LIBCMT:winapinls.obj
 0002:0001794c       ??_C@_1BG@PBGJMCEM@?$AAu?$AAz?$AA?9?$AAU?$AAZ?$AA?9?$AAC?$AAy?$AAr?$AAl?$AA?$AA@ 1007f94c     LIBCMT:winapinls.obj
 0002:00017964       ??_C@_1O@LAOBCMDF@?$AAq?$AAu?$AAz?$AA?9?$AAE?$AAC?$AA?$AA@ 1007f964     LIBCMT:winapinls.obj
 0002:00017974       ??_C@_1M@POEEMAIO@?$AAa?$AAr?$AA?9?$AAE?$AAG?$AA?$AA@ 1007f974     LIBCMT:winapinls.obj
 0002:00017980       ??_C@_1M@EFAKDEDL@?$AAz?$AAh?$AA?9?$AAH?$AAK?$AA?$AA@ 1007f980     LIBCMT:winapinls.obj
 0002:0001798c       ??_C@_1M@HKKIJHGI@?$AAd?$AAe?$AA?9?$AAA?$AAT?$AA?$AA@ 1007f98c     LIBCMT:winapinls.obj
 0002:00017998       ??_C@_1M@KBFBEHJF@?$AAe?$AAn?$AA?9?$AAA?$AAU?$AA?$AA@ 1007f998     LIBCMT:winapinls.obj
 0002:000179a4       ??_C@_1M@MNPLFAAH@?$AAe?$AAs?$AA?9?$AAE?$AAS?$AA?$AA@ 1007f9a4     LIBCMT:winapinls.obj
 0002:000179b0       ??_C@_1M@HJOOJFMA@?$AAf?$AAr?$AA?9?$AAC?$AAA?$AA?$AA@ 1007f9b0     LIBCMT:winapinls.obj
 0002:000179bc       ??_C@_1BG@JPOFPNAB@?$AAs?$AAr?$AA?9?$AAS?$AAP?$AA?9?$AAC?$AAy?$AAr?$AAl?$AA?$AA@ 1007f9bc     LIBCMT:winapinls.obj
 0002:000179d4       ??_C@_1M@LNFOCMOB@?$AAs?$AAe?$AA?9?$AAF?$AAI?$AA?$AA@ 1007f9d4     LIBCMT:winapinls.obj
 0002:000179e0       ??_C@_1O@MGJBOAMB@?$AAq?$AAu?$AAz?$AA?9?$AAP?$AAE?$AA?$AA@ 1007f9e0     LIBCMT:winapinls.obj
 0002:000179f0       ??_C@_1M@GJINLBOK@?$AAa?$AAr?$AA?9?$AAL?$AAY?$AA?$AA@ 1007f9f0     LIBCMT:winapinls.obj
 0002:000179fc       ??_C@_1M@GGMNHJNL@?$AAz?$AAh?$AA?9?$AAS?$AAG?$AA?$AA@ 1007f9fc     LIBCMT:winapinls.obj
 0002:00017a08       ??_C@_1M@HOIKODND@?$AAd?$AAe?$AA?9?$AAL?$AAU?$AA?$AA@ 1007fa08     LIBCMT:winapinls.obj
 0002:00017a14       ??_C@_1M@DDOCCGFG@?$AAe?$AAn?$AA?9?$AAC?$AAA?$AA?$AA@ 1007fa14     LIBCMT:winapinls.obj
 0002:00017a20       ??_C@_1M@BNOEMJLF@?$AAe?$AAs?$AA?9?$AAG?$AAT?$AA?$AA@ 1007fa20     LIBCMT:winapinls.obj
 0002:00017a2c       ??_C@_1M@EOGNKEK@?$AAf?$AAr?$AA?9?$AAC?$AAH?$AA?$AA@ 1007fa2c     LIBCMT:winapinls.obj
 0002:00017a38       ??_C@_1M@FLIDJFHL@?$AAh?$AAr?$AA?9?$AAB?$AAA?$AA?$AA@ 1007fa38     LIBCMT:winapinls.obj
 0002:00017a44       ??_C@_1O@FMCELNAJ@?$AAs?$AAm?$AAj?$AA?9?$AAN?$AAO?$AA?$AA@ 1007fa44     LIBCMT:winapinls.obj
 0002:00017a54       ??_C@_1M@JHGLJMGJ@?$AAa?$AAr?$AA?9?$AAD?$AAZ?$AA?$AA@ 1007fa54     LIBCMT:winapinls.obj
 0002:00017a60       ??_C@_1M@JKKFDCNP@?$AAz?$AAh?$AA?9?$AAM?$AAO?$AA?$AA@ 1007fa60     LIBCMT:winapinls.obj
 0002:00017a6c       ??_C@_1M@GEEFALPE@?$AAd?$AAe?$AA?9?$AAL?$AAI?$AA?$AA@ 1007fa6c     LIBCMT:winapinls.obj
 0002:00017a78       ??_C@_1M@IGEOFBG@?$AAe?$AAn?$AA?9?$AAN?$AAZ?$AA?$AA@ 1007fa78     LIBCMT:winapinls.obj
 0002:00017a84       ??_C@_1M@KDBONEHP@?$AAe?$AAs?$AA?9?$AAC?$AAR?$AA?$AA@ 1007fa84     LIBCMT:winapinls.obj
 0002:00017a90       ??_C@_1M@FHMDOHNN@?$AAf?$AAr?$AA?9?$AAL?$AAU?$AA?$AA@ 1007fa90     LIBCMT:winapinls.obj
 0002:00017a9c       ??_C@_1BG@NFKKMAFG@?$AAb?$AAs?$AA?9?$AAB?$AAA?$AA?9?$AAL?$AAa?$AAt?$AAn?$AA?$AA@ 1007fa9c     LIBCMT:winapinls.obj
 0002:00017ab4       ??_C@_1O@IMNBEMCI@?$AAs?$AAm?$AAj?$AA?9?$AAS?$AAE?$AA?$AA@ 1007fab4     LIBCMT:winapinls.obj
 0002:00017ac4       ??_C@_1M@DHHMBNDP@?$AAa?$AAr?$AA?9?$AAM?$AAA?$AA?$AA@ 1007fac4     LIBCMT:winapinls.obj
 0002:00017ad0       ??_C@_1M@BNBLJCGH@?$AAe?$AAn?$AA?9?$AAI?$AAE?$AA?$AA@ 1007fad0     LIBCMT:winapinls.obj
 0002:00017adc       ??_C@_1M@GEPAFMDL@?$AAe?$AAs?$AA?9?$AAP?$AAA?$AA?$AA@ 1007fadc     LIBCMT:winapinls.obj
 0002:00017ae8       ??_C@_1M@OJONDMDL@?$AAf?$AAr?$AA?9?$AAM?$AAC?$AA?$AA@ 1007fae8     LIBCMT:winapinls.obj
 0002:00017af4       ??_C@_1BG@OBCNFJB@?$AAs?$AAr?$AA?9?$AAB?$AAA?$AA?9?$AAL?$AAa?$AAt?$AAn?$AA?$AA@ 1007faf4     LIBCMT:winapinls.obj
 0002:00017b0c       ??_C@_1O@KEMEEGPO@?$AAs?$AAm?$AAa?$AA?9?$AAN?$AAO?$AA?$AA@ 1007fb0c     LIBCMT:winapinls.obj
 0002:00017b1c       ??_C@_1M@ELMGFODK@?$AAa?$AAr?$AA?9?$AAT?$AAN?$AA?$AA@ 1007fb1c     LIBCMT:winapinls.obj
 0002:00017b28       ??_C@_1M@BHDLHFAF@?$AAe?$AAn?$AA?9?$AAZ?$AAA?$AA?$AA@ 1007fb28     LIBCMT:winapinls.obj
 0002:00017b34       ??_C@_1M@BMGIGLIF@?$AAe?$AAs?$AA?9?$AAD?$AAO?$AA?$AA@ 1007fb34     LIBCMT:winapinls.obj
 0002:00017b40       ??_C@_1BG@CMBHIPBE@?$AAs?$AAr?$AA?9?$AAB?$AAA?$AA?9?$AAC?$AAy?$AAr?$AAl?$AA?$AA@ 1007fb40     LIBCMT:winapinls.obj
 0002:00017b58       ??_C@_1O@HEDBLHNP@?$AAs?$AAm?$AAa?$AA?9?$AAS?$AAE?$AA?$AA@ 1007fb58     LIBCMT:winapinls.obj
 0002:00017b68       ??_C@_1M@DAGCADIM@?$AAa?$AAr?$AA?9?$AAO?$AAM?$AA?$AA@ 1007fb68     LIBCMT:winapinls.obj
 0002:00017b74       ??_C@_1M@FODLMICG@?$AAe?$AAn?$AA?9?$AAJ?$AAM?$AA?$AA@ 1007fb74     LIBCMT:winapinls.obj
 0002:00017b80       ??_C@_1M@DNMLCIHB@?$AAe?$AAs?$AA?9?$AAV?$AAE?$AA?$AA@ 1007fb80     LIBCMT:winapinls.obj
 0002:00017b8c       ??_C@_1O@EOKHMKJK@?$AAs?$AAm?$AAs?$AA?9?$AAF?$AAI?$AA?$AA@ 1007fb8c     LIBCMT:winapinls.obj
 0002:00017b9c       ??_C@_1M@CAFJMKOF@?$AAa?$AAr?$AA?9?$AAY?$AAE?$AA?$AA@ 1007fb9c     LIBCMT:winapinls.obj
 0002:00017ba8       ??_C@_1M@CBFHIJLI@?$AAe?$AAn?$AA?9?$AAC?$AAB?$AA?$AA@ 1007fba8     LIBCMT:winapinls.obj
 0002:00017bb4       ??_C@_1M@BGNFLDN@?$AAe?$AAs?$AA?9?$AAC?$AAO?$AA?$AA@ 1007fbb4     LIBCMT:winapinls.obj
 0002:00017bc0       ??_C@_1O@JMPHMAMC@?$AAs?$AAm?$AAn?$AA?9?$AAF?$AAI?$AA?$AA@ 1007fbc0     LIBCMT:winapinls.obj
 0002:00017bd0       ??_C@_1M@JLANABKE@?$AAa?$AAr?$AA?9?$AAS?$AAY?$AA?$AA@ 1007fbd0     LIBCMT:winapinls.obj
 0002:00017bdc       ??_C@_1M@HPKGCFGN@?$AAe?$AAn?$AA?9?$AAB?$AAZ?$AA?$AA@ 1007fbdc     LIBCMT:winapinls.obj
 0002:00017be8       ??_C@_1M@OLJCMLGM@?$AAe?$AAs?$AA?9?$AAP?$AAE?$AA?$AA@ 1007fbe8     LIBCMT:winapinls.obj
 0002:00017bf4       ??_C@_1M@MKKGFKLE@?$AAa?$AAr?$AA?9?$AAJ?$AAO?$AA?$AA@ 1007fbf4     LIBCMT:winapinls.obj
 0002:00017c00       ??_C@_1M@EKPGLDNI@?$AAe?$AAn?$AA?9?$AAT?$AAT?$AA?$AA@ 1007fc00     LIBCMT:winapinls.obj
 0002:00017c0c       ??_C@_1M@OONGHFHE@?$AAe?$AAs?$AA?9?$AAA?$AAR?$AA?$AA@ 1007fc0c     LIBCMT:winapinls.obj
 0002:00017c18       ??_C@_1M@OOJFGBHE@?$AAa?$AAr?$AA?9?$AAL?$AAB?$AA?$AA@ 1007fc18     LIBCMT:winapinls.obj
 0002:00017c24       ??_C@_1M@GCEJHNEG@?$AAe?$AAn?$AA?9?$AAZ?$AAW?$AA?$AA@ 1007fc24     LIBCMT:winapinls.obj
 0002:00017c30       ??_C@_1M@JNOCAHJI@?$AAe?$AAs?$AA?9?$AAE?$AAC?$AA?$AA@ 1007fc30     LIBCMT:winapinls.obj
 0002:00017c3c       ??_C@_1M@JEFHPGGB@?$AAa?$AAr?$AA?9?$AAK?$AAW?$AA?$AA@ 1007fc3c     LIBCMT:winapinls.obj
 0002:00017c48       ??_C@_1M@MLKIBJOJ@?$AAe?$AAn?$AA?9?$AAP?$AAH?$AA?$AA@ 1007fc48     LIBCMT:winapinls.obj
 0002:00017c54       ??_C@_1M@BDNIPEND@?$AAe?$AAs?$AA?9?$AAC?$AAL?$AA?$AA@ 1007fc54     LIBCMT:winapinls.obj
 0002:00017c60       ??_C@_1M@MPNMEKBD@?$AAa?$AAr?$AA?9?$AAA?$AAE?$AA?$AA@ 1007fc60     LIBCMT:winapinls.obj
 0002:00017c6c       ??_C@_1M@KBJALCPI@?$AAe?$AAs?$AA?9?$AAU?$AAY?$AA?$AA@ 1007fc6c     LIBCMT:winapinls.obj
 0002:00017c78       ??_C@_1M@LLCCOAGA@?$AAa?$AAr?$AA?9?$AAB?$AAH?$AA?$AA@ 1007fc78     LIBCMT:winapinls.obj
 0002:00017c84       ??_C@_1M@PBFNCDEL@?$AAe?$AAs?$AA?9?$AAP?$AAY?$AA?$AA@ 1007fc84     LIBCMT:winapinls.obj
 0002:00017c90       ??_C@_1M@EDGINPNP@?$AAa?$AAr?$AA?9?$AAQ?$AAA?$AA?$AA@ 1007fc90     LIBCMT:winapinls.obj
 0002:00017c9c       ??_C@_1M@MKDBIIJI@?$AAe?$AAs?$AA?9?$AAB?$AAO?$AA?$AA@ 1007fc9c     LIBCMT:winapinls.obj
 0002:00017ca8       ??_C@_1M@CPKKEBLD@?$AAe?$AAs?$AA?9?$AAS?$AAV?$AA?$AA@ 1007fca8     LIBCMT:winapinls.obj
 0002:00017cb4       ??_C@_1M@NDBGMMJL@?$AAe?$AAs?$AA?9?$AAH?$AAN?$AA?$AA@ 1007fcb4     LIBCMT:winapinls.obj
 0002:00017cc0       ??_C@_1M@JIJIBHDP@?$AAe?$AAs?$AA?9?$AAN?$AAI?$AA?$AA@ 1007fcc0     LIBCMT:winapinls.obj
 0002:00017ccc       ??_C@_1M@CGFMKEEK@?$AAe?$AAs?$AA?9?$AAP?$AAR?$AA?$AA@ 1007fccc     LIBCMT:winapinls.obj
 0002:00017cd8       ??_C@_1O@ICJHKIIK@?$AAz?$AAh?$AA?9?$AAC?$AAH?$AAT?$AA?$AA@ 1007fcd8     LIBCMT:winapinls.obj
 0002:00017ce8       ??_C@_15CLNEJCE@?$AAs?$AAr?$AA?$AA@ 1007fce8     LIBCMT:winapinls.obj
 0002:00017cf0       ??_C@_1M@KAHEKEIG@?$AAa?$AAf?$AA?9?$AAz?$AAa?$AA?$AA@ 1007fcf0     LIBCMT:winapinls.obj
 0002:00017cfc       ??_C@_1M@GIECOABL@?$AAa?$AAr?$AA?9?$AAa?$AAe?$AA?$AA@ 1007fcfc     LIBCMT:winapinls.obj
 0002:00017d08       ??_C@_1M@BMLMEKGI@?$AAa?$AAr?$AA?9?$AAb?$AAh?$AA?$AA@ 1007fd08     LIBCMT:winapinls.obj
 0002:00017d14       ??_C@_1M@DAPFDGGB@?$AAa?$AAr?$AA?9?$AAd?$AAz?$AA?$AA@ 1007fd14     LIBCMT:winapinls.obj
 0002:00017d20       ??_C@_1M@FJNKGKIG@?$AAa?$AAr?$AA?9?$AAe?$AAg?$AA?$AA@ 1007fd20     LIBCMT:winapinls.obj
 0002:00017d2c       ??_C@_1M@FLGKKCLO@?$AAa?$AAr?$AA?9?$AAi?$AAq?$AA?$AA@ 1007fd2c     LIBCMT:winapinls.obj
 0002:00017d38       ??_C@_1M@GNDIPALM@?$AAa?$AAr?$AA?9?$AAj?$AAo?$AA?$AA@ 1007fd38     LIBCMT:winapinls.obj
 0002:00017d44       ??_C@_1M@DDMJFMGJ@?$AAa?$AAr?$AA?9?$AAk?$AAw?$AA?$AA@ 1007fd44     LIBCMT:winapinls.obj
 0002:00017d50       ??_C@_1M@EJALMLHM@?$AAa?$AAr?$AA?9?$AAl?$AAb?$AA?$AA@ 1007fd50     LIBCMT:winapinls.obj
 0002:00017d5c       ??_C@_1M@MOBDBLOC@?$AAa?$AAr?$AA?9?$AAl?$AAy?$AA?$AA@ 1007fd5c     LIBCMT:winapinls.obj
 0002:00017d68       ??_C@_1M@JAOCLHDH@?$AAa?$AAr?$AA?9?$AAm?$AAa?$AA?$AA@ 1007fd68     LIBCMT:winapinls.obj
 0002:00017d74       ??_C@_1M@JHPMKJIE@?$AAa?$AAr?$AA?9?$AAo?$AAm?$AA?$AA@ 1007fd74     LIBCMT:winapinls.obj
 0002:00017d80       ??_C@_1M@OEPGHFNH@?$AAa?$AAr?$AA?9?$AAq?$AAa?$AA?$AA@ 1007fd80     LIBCMT:winapinls.obj
 0002:00017d8c       ??_C@_1M@KJDONENM@?$AAa?$AAr?$AA?9?$AAs?$AAa?$AA?$AA@ 1007fd8c     LIBCMT:winapinls.obj
 0002:00017d98       ??_C@_1M@DMJDKLKM@?$AAa?$AAr?$AA?9?$AAs?$AAy?$AA?$AA@ 1007fd98     LIBCMT:winapinls.obj
 0002:00017da4       ??_C@_1M@OMFIPEDC@?$AAa?$AAr?$AA?9?$AAt?$AAn?$AA?$AA@ 1007fda4     LIBCMT:winapinls.obj
 0002:00017db0       ??_C@_1M@IHMHGAON@?$AAa?$AAr?$AA?9?$AAy?$AAe?$AA?$AA@ 1007fdb0     LIBCMT:winapinls.obj
 0002:00017dbc       ??_C@_1BG@KDCPGJGB@?$AAa?$AAz?$AA?9?$AAa?$AAz?$AA?9?$AAc?$AAy?$AAr?$AAl?$AA?$AA@ 1007fdbc     LIBCMT:winapinls.obj
 0002:00017dd4       ??_C@_1BG@IBCKDDOE@?$AAa?$AAz?$AA?9?$AAa?$AAz?$AA?9?$AAl?$AAa?$AAt?$AAn?$AA?$AA@ 1007fdd4     LIBCMT:winapinls.obj
 0002:00017dec       ??_C@_1M@EGPFDCPD@?$AAb?$AAe?$AA?9?$AAb?$AAy?$AA?$AA@ 1007fdec     LIBCMT:winapinls.obj
 0002:00017df8       ??_C@_1M@PCMGMCGC@?$AAb?$AAg?$AA?9?$AAb?$AAg?$AA?$AA@ 1007fdf8     LIBCMT:winapinls.obj
 0002:00017e04       ??_C@_1M@BJBMFGOB@?$AAb?$AAn?$AA?9?$AAi?$AAn?$AA?$AA@ 1007fe04     LIBCMT:winapinls.obj
 0002:00017e10       ??_C@_1BG@EAKMMACD@?$AAb?$AAs?$AA?9?$AAb?$AAa?$AA?9?$AAl?$AAa?$AAt?$AAn?$AA?$AA@ 1007fe10     LIBCMT:winapinls.obj
 0002:00017e28       ??_C@_1M@KGADAODK@?$AAc?$AAa?$AA?9?$AAe?$AAs?$AA?$AA@ 1007fe28     LIBCMT:winapinls.obj
 0002:00017e34       ??_C@_1M@COAJPDHI@?$AAc?$AAs?$AA?9?$AAc?$AAz?$AA?$AA@ 1007fe34     LIBCMT:winapinls.obj
 0002:00017e40       ??_C@_1M@DHBHFONH@?$AAc?$AAy?$AA?9?$AAg?$AAb?$AA?$AA@ 1007fe40     LIBCMT:winapinls.obj
 0002:00017e4c       ??_C@_1M@IMGKELGA@?$AAd?$AAa?$AA?9?$AAd?$AAk?$AA?$AA@ 1007fe4c     LIBCMT:winapinls.obj
 0002:00017e58       ??_C@_1M@NNDGDNGA@?$AAd?$AAe?$AA?9?$AAa?$AAt?$AA?$AA@ 1007fe58     LIBCMT:winapinls.obj
 0002:00017e64       ??_C@_1M@IKDBHEEM@?$AAd?$AAe?$AA?9?$AAc?$AAh?$AA?$AA@ 1007fe64     LIBCMT:winapinls.obj
 0002:00017e70       ??_C@_1M@GFFOJMCJ@?$AAd?$AAe?$AA?9?$AAd?$AAe?$AA?$AA@ 1007fe70     LIBCMT:winapinls.obj
 0002:00017e7c       ??_C@_1M@MDNLKBPM@?$AAd?$AAe?$AA?9?$AAl?$AAi?$AA?$AA@ 1007fe7c     LIBCMT:winapinls.obj
 0002:00017e88       ??_C@_1M@NJBEEJNL@?$AAd?$AAe?$AA?9?$AAl?$AAu?$AA?$AA@ 1007fe88     LIBCMT:winapinls.obj
 0002:00017e94       ??_C@_1O@GNNELBAP@?$AAd?$AAi?$AAv?$AA?9?$AAm?$AAv?$AA?$AA@ 1007fe94     LIBCMT:winapinls.obj
 0002:00017ea4       ??_C@_1M@EJLEOGAE@?$AAe?$AAl?$AA?9?$AAg?$AAr?$AA?$AA@ 1007fea4     LIBCMT:winapinls.obj
 0002:00017eb0       ??_C@_1M@GMPONJN@?$AAe?$AAn?$AA?9?$AAa?$AAu?$AA?$AA@ 1007feb0     LIBCMT:winapinls.obj
 0002:00017ebc       ??_C@_1M@NIDIIPGF@?$AAe?$AAn?$AA?9?$AAb?$AAz?$AA?$AA@ 1007febc     LIBCMT:winapinls.obj
 0002:00017ec8       ??_C@_1M@JEHMIMFO@?$AAe?$AAn?$AA?9?$AAc?$AAa?$AA?$AA@ 1007fec8     LIBCMT:winapinls.obj
 0002:00017ed4       ??_C@_1M@IGMJCDLA@?$AAe?$AAn?$AA?9?$AAc?$AAb?$AA?$AA@ 1007fed4     LIBCMT:winapinls.obj
 0002:00017ee0       ??_C@_1M@BNFIGBKG@?$AAe?$AAn?$AA?9?$AAg?$AAb?$AA?$AA@ 1007fee0     LIBCMT:winapinls.obj
 0002:00017eec       ??_C@_1M@LKIFDIGP@?$AAe?$AAn?$AA?9?$AAi?$AAe?$AA?$AA@ 1007feec     LIBCMT:winapinls.obj
 0002:00017ef8       ??_C@_1M@PJKFGCCO@?$AAe?$AAn?$AA?9?$AAj?$AAm?$AA?$AA@ 1007fef8     LIBCMT:winapinls.obj
 0002:00017f04       ??_C@_1M@KPPKEPBO@?$AAe?$AAn?$AA?9?$AAn?$AAz?$AA?$AA@ 1007ff04     LIBCMT:winapinls.obj
 0002:00017f10       ??_C@_1M@GMDGLDOB@?$AAe?$AAn?$AA?9?$AAp?$AAh?$AA?$AA@ 1007ff10     LIBCMT:winapinls.obj
 0002:00017f1c       ??_C@_1M@ONGIBJNA@?$AAe?$AAn?$AA?9?$AAt?$AAt?$AA?$AA@ 1007ff1c     LIBCMT:winapinls.obj
 0002:00017f28       ??_C@_1M@LLODPCMM@?$AAe?$AAn?$AA?9?$AAu?$AAs?$AA?$AA@ 1007ff28     LIBCMT:winapinls.obj
 0002:00017f34       ??_C@_1M@LAKFNPAN@?$AAe?$AAn?$AA?9?$AAz?$AAa?$AA?$AA@ 1007ff34     LIBCMT:winapinls.obj
 0002:00017f40       ??_C@_1M@MFNHNHEO@?$AAe?$AAn?$AA?9?$AAz?$AAw?$AA?$AA@ 1007ff40     LIBCMT:winapinls.obj
 0002:00017f4c       ??_C@_1M@EJEINPHM@?$AAe?$AAs?$AA?9?$AAa?$AAr?$AA?$AA@ 1007ff4c     LIBCMT:winapinls.obj
 0002:00017f58       ??_C@_1M@GNKPCCJA@?$AAe?$AAs?$AA?9?$AAb?$AAo?$AA?$AA@ 1007ff58     LIBCMT:winapinls.obj
 0002:00017f64       ??_C@_1M@LEEGFONL@?$AAe?$AAs?$AA?9?$AAc?$AAl?$AA?$AA@ 1007ff64     LIBCMT:winapinls.obj
 0002:00017f70       ??_C@_1M@KGPDPBDF@?$AAe?$AAs?$AA?9?$AAc?$AAo?$AA?$AA@ 1007ff70     LIBCMT:winapinls.obj
 0002:00017f7c       ??_C@_1M@EIAHOHH@?$AAe?$AAs?$AA?9?$AAc?$AAr?$AA?$AA@ 1007ff7c     LIBCMT:winapinls.obj
 0002:00017f88       ??_C@_1M@LLPGMBIN@?$AAe?$AAs?$AA?9?$AAd?$AAo?$AA?$AA@ 1007ff88     LIBCMT:winapinls.obj
 0002:00017f94       ??_C@_1M@DKHMKNJA@?$AAe?$AAs?$AA?9?$AAe?$AAc?$AA?$AA@ 1007ff94     LIBCMT:winapinls.obj
 0002:00017fa0       ??_C@_1M@GKGFPKAP@?$AAe?$AAs?$AA?9?$AAe?$AAs?$AA?$AA@ 1007ffa0     LIBCMT:winapinls.obj
 0002:00017fac       ??_C@_1M@LKHKGDLN@?$AAe?$AAs?$AA?9?$AAg?$AAt?$AA?$AA@ 1007ffac     LIBCMT:winapinls.obj
 0002:00017fb8       ??_C@_1M@HEIIGGJD@?$AAe?$AAs?$AA?9?$AAh?$AAn?$AA?$AA@ 1007ffb8     LIBCMT:winapinls.obj
 0002:00017fc4       ??_C@_1M@FBDHPPGD@?$AAe?$AAs?$AA?9?$AAm?$AAx?$AA?$AA@ 1007ffc4     LIBCMT:winapinls.obj
 0002:00017fd0       ??_C@_1M@DPAGLNDH@?$AAe?$AAs?$AA?9?$AAn?$AAi?$AA?$AA@ 1007ffd0     LIBCMT:winapinls.obj
 0002:00017fdc       ??_C@_1M@MDGOPGDD@?$AAe?$AAs?$AA?9?$AAp?$AAa?$AA?$AA@ 1007ffdc     LIBCMT:winapinls.obj
 0002:00017fe8       ??_C@_1M@EMAMGBGE@?$AAe?$AAs?$AA?9?$AAp?$AAe?$AA?$AA@ 1007ffe8     LIBCMT:winapinls.obj
 0002:00017ff4       ??_C@_1M@IBMCAOEC@?$AAe?$AAs?$AA?9?$AAp?$AAr?$AA?$AA@ 1007fff4     LIBCMT:winapinls.obj
 0002:00018000       ??_C@_1M@FGMDIJED@?$AAe?$AAs?$AA?9?$AAp?$AAy?$AA?$AA@ 10080000     LIBCMT:winapinls.obj
 0002:0001800c       ??_C@_1M@IIDEOLLL@?$AAe?$AAs?$AA?9?$AAs?$AAv?$AA?$AA@ 1008000c     LIBCMT:winapinls.obj
 0002:00018018       ??_C@_1M@GAOBIPA@?$AAe?$AAs?$AA?9?$AAu?$AAy?$AA?$AA@ 10080018     LIBCMT:winapinls.obj
 0002:00018024       ??_C@_1M@JKFFICHJ@?$AAe?$AAs?$AA?9?$AAv?$AAe?$AA?$AA@ 10080024     LIBCMT:winapinls.obj
 0002:00018030       ??_C@_1M@PNMLOJDF@?$AAe?$AAt?$AA?9?$AAe?$AAe?$AA?$AA@ 10080030     LIBCMT:winapinls.obj
 0002:0001803c       ??_C@_1M@GHHLIKEI@?$AAe?$AAu?$AA?9?$AAe?$AAs?$AA?$AA@ 1008003c     LIBCMT:winapinls.obj
 0002:00018048       ??_C@_1M@PBNONODE@?$AAf?$AAa?$AA?9?$AAi?$AAr?$AA?$AA@ 10080048     LIBCMT:winapinls.obj
 0002:00018054       ??_C@_1M@JEEHPMIL@?$AAf?$AAi?$AA?9?$AAf?$AAi?$AA?$AA@ 10080054     LIBCMT:winapinls.obj
 0002:00018060       ??_C@_1M@LMDCNDBA@?$AAf?$AAo?$AA?9?$AAf?$AAo?$AA?$AA@ 10080060     LIBCMT:winapinls.obj
 0002:0001806c       ??_C@_1M@JKEOHLDK@?$AAf?$AAr?$AA?9?$AAb?$AAe?$AA?$AA@ 1008006c     LIBCMT:winapinls.obj
 0002:00018078       ??_C@_1M@NOHADPMI@?$AAf?$AAr?$AA?9?$AAc?$AAa?$AA?$AA@ 10080078     LIBCMT:winapinls.obj
 0002:00018084       ??_C@_1M@KDHIHAEC@?$AAf?$AAr?$AA?9?$AAc?$AAh?$AA?$AA@ 10080084     LIBCMT:winapinls.obj
 0002:00018090       ??_C@_1M@MMBBFGAK@?$AAf?$AAr?$AA?9?$AAf?$AAr?$AA?$AA@ 10080090     LIBCMT:winapinls.obj
 0002:0001809c       ??_C@_1M@PAFNENNF@?$AAf?$AAr?$AA?9?$AAl?$AAu?$AA?$AA@ 1008009c     LIBCMT:winapinls.obj
 0002:000180a8       ??_C@_1M@EOHDJGDD@?$AAf?$AAr?$AA?9?$AAm?$AAc?$AA?$AA@ 100800a8     LIBCMT:winapinls.obj
 0002:000180b4       ??_C@_1M@FAPLLOPF@?$AAg?$AAl?$AA?9?$AAe?$AAs?$AA?$AA@ 100800b4     LIBCMT:winapinls.obj
 0002:000180c0       ??_C@_1M@FOPBFLOO@?$AAg?$AAu?$AA?9?$AAi?$AAn?$AA?$AA@ 100800c0     LIBCMT:winapinls.obj
 0002:000180cc       ??_C@_1M@KBMCINPM@?$AAh?$AAe?$AA?9?$AAi?$AAl?$AA?$AA@ 100800cc     LIBCMT:winapinls.obj
 0002:000180d8       ??_C@_1M@BBPHKFPJ@?$AAh?$AAi?$AA?9?$AAi?$AAn?$AA?$AA@ 100800d8     LIBCMT:winapinls.obj
 0002:000180e4       ??_C@_1M@PMBNDPHD@?$AAh?$AAr?$AA?9?$AAb?$AAa?$AA?$AA@ 100800e4     LIBCMT:winapinls.obj
 0002:000180f0       ??_C@_1M@BPCKOEGE@?$AAh?$AAr?$AA?9?$AAh?$AAr?$AA?$AA@ 100800f0     LIBCMT:winapinls.obj
 0002:000180fc       ??_C@_1M@GACBMHKE@?$AAh?$AAu?$AA?9?$AAh?$AAu?$AA?$AA@ 100800fc     LIBCMT:winapinls.obj
 0002:00018108       ??_C@_1M@MILPAJJC@?$AAh?$AAy?$AA?9?$AAa?$AAm?$AA?$AA@ 10080108     LIBCMT:winapinls.obj
 0002:00018114       ??_C@_1M@BABBICEC@?$AAi?$AAd?$AA?9?$AAi?$AAd?$AA?$AA@ 10080114     LIBCMT:winapinls.obj
 0002:00018120       ??_C@_1M@BIKNHHPF@?$AAi?$AAs?$AA?9?$AAi?$AAs?$AA?$AA@ 10080120     LIBCMT:winapinls.obj
 0002:0001812c       ??_C@_1M@NMPCJPHE@?$AAi?$AAt?$AA?9?$AAc?$AAh?$AA?$AA@ 1008012c     LIBCMT:winapinls.obj
 0002:00018138       ??_C@_1M@GHKGFEDF@?$AAi?$AAt?$AA?9?$AAi?$AAt?$AA?$AA@ 10080138     LIBCMT:winapinls.obj
 0002:00018144       ??_C@_1M@NIEJCJJA@?$AAj?$AAa?$AA?9?$AAj?$AAp?$AA?$AA@ 10080144     LIBCMT:winapinls.obj
 0002:00018150       ??_C@_1M@JILFNBIM@?$AAk?$AAa?$AA?9?$AAg?$AAe?$AA?$AA@ 10080150     LIBCMT:winapinls.obj
 0002:0001815c       ??_C@_1M@PACPMGPH@?$AAk?$AAk?$AA?9?$AAk?$AAz?$AA?$AA@ 1008015c     LIBCMT:winapinls.obj
 0002:00018168       ??_C@_1M@IELFGMHA@?$AAk?$AAn?$AA?9?$AAi?$AAn?$AA?$AA@ 10080168     LIBCMT:winapinls.obj
 0002:00018174       ??_C@_1O@IBBJHCH@?$AAk?$AAo?$AAk?$AA?9?$AAi?$AAn?$AA?$AA@ 10080174     LIBCMT:winapinls.obj
 0002:00018184       ??_C@_1M@DMHAEOGC@?$AAk?$AAo?$AA?9?$AAk?$AAr?$AA?$AA@ 10080184     LIBCMT:winapinls.obj
 0002:00018190       ??_C@_1M@HBAHBIGA@?$AAk?$AAy?$AA?9?$AAk?$AAg?$AA?$AA@ 10080190     LIBCMT:winapinls.obj
 0002:0001819c       ??_C@_1M@KPMILCJG@?$AAl?$AAt?$AA?9?$AAl?$AAt?$AA?$AA@ 1008019c     LIBCMT:winapinls.obj
 0002:000181a8       ??_C@_1M@BDEKKCA@?$AAl?$AAv?$AA?9?$AAl?$AAv?$AA?$AA@ 100801a8     LIBCMT:winapinls.obj
 0002:000181b4       ??_C@_1M@ELCKCCJJ@?$AAm?$AAi?$AA?9?$AAn?$AAz?$AA?$AA@ 100801b4     LIBCMT:winapinls.obj
 0002:000181c0       ??_C@_1M@CBOOLAPA@?$AAm?$AAk?$AA?9?$AAm?$AAk?$AA?$AA@ 100801c0     LIBCMT:winapinls.obj
 0002:000181cc       ??_C@_1M@GPHNBJKN@?$AAm?$AAl?$AA?9?$AAi?$AAn?$AA?$AA@ 100801cc     LIBCMT:winapinls.obj
 0002:000181d8       ??_C@_1M@PABJILIG@?$AAm?$AAn?$AA?9?$AAm?$AAn?$AA?$AA@ 100801d8     LIBCMT:winapinls.obj
 0002:000181e4       ??_C@_1M@FGBKKIPG@?$AAm?$AAr?$AA?9?$AAi?$AAn?$AA?$AA@ 100801e4     LIBCMT:winapinls.obj
 0002:000181f0       ??_C@_1M@NDBPDDAL@?$AAm?$AAs?$AA?9?$AAb?$AAn?$AA?$AA@ 100801f0     LIBCMT:winapinls.obj
 0002:000181fc       ??_C@_1M@OPIHOOPI@?$AAm?$AAs?$AA?9?$AAm?$AAy?$AA?$AA@ 100801fc     LIBCMT:winapinls.obj
 0002:00018208       ??_C@_1M@PPDBCNFM@?$AAm?$AAt?$AA?9?$AAm?$AAt?$AA?$AA@ 10080208     LIBCMT:winapinls.obj
 0002:00018214       ??_C@_1M@KDJDKMDD@?$AAn?$AAb?$AA?9?$AAn?$AAo?$AA?$AA@ 10080214     LIBCMT:winapinls.obj
 0002:00018220       ??_C@_1M@KFCFLMJP@?$AAn?$AAl?$AA?9?$AAb?$AAe?$AA?$AA@ 10080220     LIBCMT:winapinls.obj
 0002:0001822c       ??_C@_1M@KPOPDDGO@?$AAn?$AAl?$AA?9?$AAn?$AAl?$AA?$AA@ 1008022c     LIBCMT:winapinls.obj
 0002:00018238       ??_C@_1M@LJKPEMLN@?$AAn?$AAn?$AA?9?$AAn?$AAo?$AA?$AA@ 10080238     LIBCMT:winapinls.obj
 0002:00018244       ??_C@_1M@BDGHHBFL@?$AAn?$AAs?$AA?9?$AAz?$AAa?$AA?$AA@ 10080244     LIBCMT:winapinls.obj
 0002:00018250       ??_C@_1M@IDEHOAP@?$AAp?$AAa?$AA?9?$AAi?$AAn?$AA?$AA@ 10080250     LIBCMT:winapinls.obj
 0002:0001825c       ??_C@_1M@HDBKGOGH@?$AAp?$AAl?$AA?9?$AAp?$AAl?$AA?$AA@ 1008025c     LIBCMT:winapinls.obj
 0002:00018268       ??_C@_1M@LJLLCMEH@?$AAp?$AAt?$AA?9?$AAb?$AAr?$AA?$AA@ 10080268     LIBCMT:winapinls.obj
 0002:00018274       ??_C@_1M@NCMONAAL@?$AAp?$AAt?$AA?9?$AAp?$AAt?$AA?$AA@ 10080274     LIBCMT:winapinls.obj
 0002:00018280       ??_C@_1O@EAKMAJDN@?$AAq?$AAu?$AAz?$AA?9?$AAb?$AAo?$AA?$AA@ 10080280     LIBCMT:winapinls.obj
 0002:00018290       ??_C@_1O@BHHPIGDN@?$AAq?$AAu?$AAz?$AA?9?$AAe?$AAc?$AA?$AA@ 10080290     LIBCMT:winapinls.obj
 0002:000182a0       ??_C@_1O@GBAPEKMJ@?$AAq?$AAu?$AAz?$AA?9?$AAp?$AAe?$AA?$AA@ 100802a0     LIBCMT:winapinls.obj
 0002:000182b0       ??_C@_1M@CLGLEFBO@?$AAr?$AAo?$AA?9?$AAr?$AAo?$AA?$AA@ 100802b0     LIBCMT:winapinls.obj
 0002:000182bc       ??_C@_1M@CEEDODME@?$AAr?$AAu?$AA?9?$AAr?$AAu?$AA?$AA@ 100802bc     LIBCMT:winapinls.obj
 0002:000182c8       ??_C@_1M@HPKKKMPP@?$AAs?$AAa?$AA?9?$AAi?$AAn?$AA?$AA@ 100802c8     LIBCMT:winapinls.obj
 0002:000182d4       ??_C@_1M@BKMAIGOJ@?$AAs?$AAe?$AA?9?$AAf?$AAi?$AA?$AA@ 100802d4     LIBCMT:winapinls.obj
 0002:000182e0       ??_C@_1M@NDPIFLFI@?$AAs?$AAe?$AA?9?$AAn?$AAo?$AA?$AA@ 100802e0     LIBCMT:winapinls.obj
 0002:000182ec       ??_C@_1M@DANKKHJ@?$AAs?$AAe?$AA?9?$AAs?$AAe?$AA?$AA@ 100802ec     LIBCMT:winapinls.obj
 0002:000182f8       ??_C@_1M@PNBLONPJ@?$AAs?$AAk?$AA?9?$AAs?$AAk?$AA?$AA@ 100802f8     LIBCMT:winapinls.obj
 0002:00018304       ??_C@_1M@LFMODOAL@?$AAs?$AAl?$AA?9?$AAs?$AAi?$AA?$AA@ 10080304     LIBCMT:winapinls.obj
 0002:00018310       ??_C@_1O@DFKOMPG@?$AAs?$AAm?$AAa?$AA?9?$AAn?$AAo?$AA?$AA@ 10080310     LIBCMT:winapinls.obj
 0002:00018320       ??_C@_1O@NDKPBNNH@?$AAs?$AAm?$AAa?$AA?9?$AAs?$AAe?$AA?$AA@ 10080320     LIBCMT:winapinls.obj
 0002:00018330       ??_C@_1O@PLLKBHAB@?$AAs?$AAm?$AAj?$AA?9?$AAn?$AAo?$AA?$AA@ 10080330     LIBCMT:winapinls.obj
 0002:00018340       ??_C@_1O@CLEPOGCA@?$AAs?$AAm?$AAj?$AA?9?$AAs?$AAe?$AA?$AA@ 10080340     LIBCMT:winapinls.obj
 0002:00018350       ??_C@_1O@DLGJGKMK@?$AAs?$AAm?$AAn?$AA?9?$AAf?$AAi?$AA?$AA@ 10080350     LIBCMT:winapinls.obj
 0002:00018360       ??_C@_1O@OJDJGAJC@?$AAs?$AAm?$AAs?$AA?9?$AAf?$AAi?$AA?$AA@ 10080360     LIBCMT:winapinls.obj
 0002:00018370       ??_C@_1M@BOFOGHPB@?$AAs?$AAq?$AA?9?$AAa?$AAl?$AA?$AA@ 10080370     LIBCMT:winapinls.obj
 0002:0001837c       ??_C@_1BG@LJBBIPGB@?$AAs?$AAr?$AA?9?$AAb?$AAa?$AA?9?$AAc?$AAy?$AAr?$AAl?$AA?$AA@ 1008037c     LIBCMT:winapinls.obj
 0002:00018394       ??_C@_1BG@JLBENFOE@?$AAs?$AAr?$AA?9?$AAb?$AAa?$AA?9?$AAl?$AAa?$AAt?$AAn?$AA?$AA@ 10080394     LIBCMT:winapinls.obj
 0002:000183ac       ??_C@_1BG@KODPNHE@?$AAs?$AAr?$AA?9?$AAs?$AAp?$AA?9?$AAc?$AAy?$AAr?$AAl?$AA?$AA@ 100803ac     LIBCMT:winapinls.obj
 0002:000183c4       ??_C@_1BG@CIOGKHPB@?$AAs?$AAr?$AA?9?$AAs?$AAp?$AA?9?$AAl?$AAa?$AAt?$AAn?$AA?$AA@ 100803c4     LIBCMT:winapinls.obj
 0002:000183dc       ??_C@_1M@NGFJLMAC@?$AAs?$AAv?$AA?9?$AAf?$AAi?$AA?$AA@ 100803dc     LIBCMT:winapinls.obj
 0002:000183e8       ??_C@_1M@MPJEJAJC@?$AAs?$AAv?$AA?9?$AAs?$AAe?$AA?$AA@ 100803e8     LIBCMT:winapinls.obj
 0002:000183f4       ??_C@_1M@MPNDHLFK@?$AAs?$AAw?$AA?9?$AAk?$AAe?$AA?$AA@ 100803f4     LIBCMT:winapinls.obj
 0002:00018400       ??_C@_1O@KOHBJJI@?$AAs?$AAy?$AAr?$AA?9?$AAs?$AAy?$AA?$AA@ 10080400     LIBCMT:winapinls.obj
 0002:00018410       ??_C@_1M@LDCEFHA@?$AAt?$AAa?$AA?9?$AAi?$AAn?$AA?$AA@ 10080410     LIBCMT:winapinls.obj
 0002:0001841c       ??_C@_1M@CNJOFAK@?$AAt?$AAe?$AA?9?$AAi?$AAn?$AA?$AA@ 1008041c     LIBCMT:winapinls.obj
 0002:00018428       ??_C@_1M@GNAECACD@?$AAt?$AAh?$AA?9?$AAt?$AAh?$AA?$AA@ 10080428     LIBCMT:winapinls.obj
 0002:00018434       ??_C@_1M@CHBIHOJO@?$AAt?$AAn?$AA?9?$AAz?$AAa?$AA?$AA@ 10080434     LIBCMT:winapinls.obj
 0002:00018440       ??_C@_1M@GCCMIGPJ@?$AAt?$AAr?$AA?9?$AAt?$AAr?$AA?$AA@ 10080440     LIBCMT:winapinls.obj
 0002:0001844c       ??_C@_1M@CELMCNBK@?$AAt?$AAt?$AA?9?$AAr?$AAu?$AA?$AA@ 1008044c     LIBCMT:winapinls.obj
 0002:00018458       ??_C@_1M@KLMCELGA@?$AAu?$AAk?$AA?9?$AAu?$AAa?$AA?$AA@ 10080458     LIBCMT:winapinls.obj
 0002:00018464       ??_C@_1M@EPAJJAJF@?$AAu?$AAr?$AA?9?$AAp?$AAk?$AA?$AA@ 10080464     LIBCMT:winapinls.obj
 0002:00018470       ??_C@_1BG@GEGPMCDJ@?$AAu?$AAz?$AA?9?$AAu?$AAz?$AA?9?$AAc?$AAy?$AAr?$AAl?$AA?$AA@ 10080470     LIBCMT:winapinls.obj
 0002:00018488       ??_C@_1BG@EGGKJILM@?$AAu?$AAz?$AA?9?$AAu?$AAz?$AA?9?$AAl?$AAa?$AAt?$AAn?$AA?$AA@ 10080488     LIBCMT:winapinls.obj
 0002:000184a0       ??_C@_1M@GFOCLFF@?$AAv?$AAi?$AA?9?$AAv?$AAn?$AA?$AA@ 100804a0     LIBCMT:winapinls.obj
 0002:000184ac       ??_C@_1M@CPAMEDFI@?$AAx?$AAh?$AA?9?$AAz?$AAa?$AA?$AA@ 100804ac     LIBCMT:winapinls.obj
 0002:000184b8       ??_C@_1O@EBKIFIGN@?$AAz?$AAh?$AA?9?$AAc?$AAh?$AAs?$AA?$AA@ 100804b8     LIBCMT:winapinls.obj
 0002:000184c8       ??_C@_1O@NMHPGANE@?$AAz?$AAh?$AA?9?$AAc?$AAh?$AAt?$AA?$AA@ 100804c8     LIBCMT:winapinls.obj
 0002:000184d8       ??_C@_1M@LPINJOMC@?$AAz?$AAh?$AA?9?$AAc?$AAn?$AA?$AA@ 100804d8     LIBCMT:winapinls.obj
 0002:000184e4       ??_C@_1M@OCJEJODD@?$AAz?$AAh?$AA?9?$AAh?$AAk?$AA?$AA@ 100804e4     LIBCMT:winapinls.obj
 0002:000184f0       ??_C@_1M@DNDLJINH@?$AAz?$AAh?$AA?9?$AAm?$AAo?$AA?$AA@ 100804f0     LIBCMT:winapinls.obj
 0002:000184fc       ??_C@_1M@MBFDNDND@?$AAz?$AAh?$AA?9?$AAs?$AAg?$AA?$AA@ 100804fc     LIBCMT:winapinls.obj
 0002:00018508       ??_C@_1M@IMEPLEPE@?$AAz?$AAh?$AA?9?$AAt?$AAw?$AA?$AA@ 10080508     LIBCMT:winapinls.obj
 0002:00018514       ??_C@_1M@BBGHNHJP@?$AAz?$AAu?$AA?9?$AAz?$AAa?$AA?$AA@ 10080514     LIBCMT:winapinls.obj
 0002:00018520       ??_C@_1BK@GAEMIDIL@?$AAA?$AAD?$AAV?$AAA?$AAP?$AAI?$AA3?$AA2?$AA?4?$AAD?$AAL?$AAL?$AA?$AA@ 10080520     LIBCMT:rand_s.obj
 0002:0001853c       ??_C@_0BC@JEAENNKH@SystemFunction036?$AA@ 1008053c     LIBCMT:rand_s.obj
 0002:00018550       ??_C@_1BG@GOEBHBDC@?$AAU?$AAS?$AAE?$AAR?$AA3?$AA2?$AA?4?$AAD?$AAL?$AAL?$AA?$AA@ 10080550     LIBCMT:crtmboxw.obj
 0002:00018568       ??_C@_0M@DLDCCGNP@MessageBoxW?$AA@ 10080568     LIBCMT:crtmboxw.obj
 0002:00018574       ??_C@_0BA@HNOPNCHB@GetActiveWindow?$AA@ 10080574     LIBCMT:crtmboxw.obj
 0002:00018584       ??_C@_0BD@HHGDFDBJ@GetLastActivePopup?$AA@ 10080584     LIBCMT:crtmboxw.obj
 0002:00018598       ??_C@_0BK@DEKFELLI@GetUserObjectInformationW?$AA@ 10080598     LIBCMT:crtmboxw.obj
 0002:000185b4       ??_C@_0BI@DFKBFLJE@GetProcessWindowStation?$AA@ 100805b4     LIBCMT:crtmboxw.obj
 0002:0001875c       ??_C@_08EHJDFFNH@__based?$CI?$AA@ 1008075c     LIBCMT:undname.obj
 0002:00018768       ??_C@_07KOLFKCDI@__cdecl?$AA@ 10080768     LIBCMT:undname.obj
 0002:00018770       ??_C@_08GHMPAG@__pascal?$AA@ 10080770     LIBCMT:undname.obj
 0002:0001877c       ??_C@_09IFJBGAPI@__stdcall?$AA@ 1008077c     LIBCMT:undname.obj
 0002:00018788       ??_C@_0L@NPHFGOKO@__thiscall?$AA@ 10080788     LIBCMT:undname.obj
 0002:00018794       ??_C@_0L@JMKHOMEK@__fastcall?$AA@ 10080794     LIBCMT:undname.obj
 0002:000187a0       ??_C@_0N@BCKKPABJ@__vectorcall?$AA@ 100807a0     LIBCMT:undname.obj
 0002:000187b0       ??_C@_09HIJEGCPM@__clrcall?$AA@ 100807b0     LIBCMT:undname.obj
 0002:000187bc       ??_C@_06GHPCKEAG@__eabi?$AA@ 100807bc     LIBCMT:undname.obj
 0002:000187c4       ??_C@_07JOMMBBKO@__ptr64?$AA@ 100807c4     LIBCMT:undname.obj
 0002:000187cc       ??_C@_0L@PILCLIHE@__restrict?$AA@ 100807cc     LIBCMT:undname.obj
 0002:000187d8       ??_C@_0M@GFIIJFMG@__unaligned?$AA@ 100807d8     LIBCMT:undname.obj
 0002:000187e4       ??_C@_09DHDLOLLB@restrict?$CI?$AA@ 100807e4     LIBCMT:undname.obj
 0002:000187f0       ??_C@_04NIHEBCM@?5new?$AA@ 100807f0     LIBCMT:undname.obj
 0002:000187f8       ??_C@_07FPCDHGMM@?5delete?$AA@ 100807f8     LIBCMT:undname.obj
 0002:00018800       ??_C@_01NEMOKFLO@?$DN?$AA@ 10080800     LIBCMT:undname.obj
 0002:00018804       ??_C@_02GPIOPFAK@?$DO?$DO?$AA@ 10080804     LIBCMT:undname.obj
 0002:00018808       ??_C@_02FODMEDOG@?$DM?$DM?$AA@ 10080808     LIBCMT:undname.obj
 0002:0001880c       ??_C@_01DCLJPIOD@?$CB?$AA@ 1008080c     LIBCMT:undname.obj
 0002:00018810       ??_C@_02EGOFBIJA@?$DN?$DN?$AA@ 10080810     LIBCMT:undname.obj
 0002:00018814       ??_C@_02FDNJECIE@?$CB?$DN?$AA@ 10080814     LIBCMT:undname.obj
 0002:00018818       ??_C@_02GPECMEKF@?$FL?$FN?$AA@ 10080818     LIBCMT:undname.obj
 0002:0001881c       ??_C@_08LHJFAFGD@operator?$AA@ 1008081c     LIBCMT:undname.obj
 0002:00018828       ??_C@_02HBOOOICD@?9?$DO?$AA@ 10080828     LIBCMT:undname.obj
 0002:0001882c       ??_C@_01NBENCBCI@?$CK?$AA@ 1008082c     LIBCMT:undname.obj
 0002:00018830       ??_C@_02ECNGHCIF@?$CL?$CL?$AA@ 10080830     LIBCMT:undname.obj
 0002:00018834       ??_C@_02BAABKJLB@?9?9?$AA@ 10080834     LIBCMT:undname.obj
 0002:00018838       ??_C@_01JOAMLHOP@?9?$AA@   10080838     LIBCMT:undname.obj
 0002:0001883c       ??_C@_01MIFGBAGJ@?$CL?$AA@ 1008083c     LIBCMT:undname.obj
 0002:00018840       ??_C@_01HNPIGOCE@?$CG?$AA@ 10080840     LIBCMT:undname.obj
 0002:00018844       ??_C@_03MNHNFDLC@?9?$DO?$CK?$AA@ 10080844     LIBCMT:undname.obj
 0002:00018848       ??_C@_01KMDKNFGN@?1?$AA@   10080848     LIBCMT:undname.obj
 0002:0001884c       ??_C@_01FGNFDNOH@?$CF?$AA@ 1008084c     LIBCMT:undname.obj
 0002:00018850       ??_C@_01MNNFJEPP@?$DM?$AA@ 10080850     LIBCMT:undname.obj
 0002:00018854       ??_C@_02EHCHHCKH@?$DM?$DN?$AA@ 10080854     LIBCMT:undname.obj
 0002:00018858       ??_C@_01PPODPGHN@?$DO?$AA@ 10080858     LIBCMT:undname.obj
 0002:0001885c       ??_C@_02EEKDKGMJ@?$DO?$DN?$AA@ 1008085c     LIBCMT:undname.obj
 0002:00018860       ??_C@_02HCKGKOFO@?$CI?$CJ?$AA@ 10080860     LIBCMT:undname.obj
 0002:00018864       ??_C@_01PJKLJHI@?$HO?$AA@  10080864     LIBCMT:undname.obj
 0002:00018868       ??_C@_01JKBOJNNK@?$FO?$AA@ 10080868     LIBCMT:undname.obj
 0002:0001886c       ??_C@_01DNKMNLPK@?$HM?$AA@ 1008086c     LIBCMT:undname.obj
 0002:00018870       ??_C@_02PPKAJPJL@?$CG?$CG?$AA@ 10080870     LIBCMT:undname.obj
 0002:00018874       ??_C@_02NONPIBCD@?$HM?$HM?$AA@ 10080874     LIBCMT:undname.obj
 0002:00018878       ??_C@_02FPIMKNGF@?$CK?$DN?$AA@ 10080878     LIBCMT:undname.obj
 0002:0001887c       ??_C@_02FOEOMHFC@?$CL?$DN?$AA@ 1008087c     LIBCMT:undname.obj
 0002:00018880       ??_C@_02FKMDLLOA@?9?$DN?$AA@ 10080880     LIBCMT:undname.obj
 0002:00018884       ??_C@_02FJEHGPIO@?1?$DN?$AA@ 10080884     LIBCMT:undname.obj
 0002:00018888       ??_C@_02FENAOKFI@?$CF?$DN?$AA@ 10080888     LIBCMT:undname.obj
 0002:0001888c       ??_C@_03IKFCCPFF@?$DO?$DO?$DN?$AA@ 1008088c     LIBCMT:undname.obj
 0002:00018890       ??_C@_03CDNPDDLA@?$DM?$DM?$DN?$AA@ 10080890     LIBCMT:undname.obj
 0002:00018894       ??_C@_02FGJGFEAB@?$CG?$DN?$AA@ 10080894     LIBCMT:undname.obj
 0002:00018898       ??_C@_02DHLNPPGH@?$HM?$DN?$AA@ 10080898     LIBCMT:undname.obj
 0002:0001889c       ??_C@_02MHEGNOJ@?$FO?$DN?$AA@ 1008089c     LIBCMT:undname.obj
 0002:000188a0       ??_C@_09IFPLHPGF@?$GAvftable?8?$AA@ 100808a0     LIBCMT:undname.obj
 0002:000188ac       ??_C@_09BLBHBJP@?$GAvbtable?8?$AA@ 100808ac     LIBCMT:undname.obj
 0002:000188b8       ??_C@_07FEEIOKP@?$GAvcall?8?$AA@ 100808b8     LIBCMT:undname.obj
 0002:000188c0       ??_C@_08LLFFHHDJ@?$GAtypeof?8?$AA@ 100808c0     LIBCMT:undname.obj
 0002:000188cc       ??_C@_0BF@KDPPACIK@?$GAlocal?5static?5guard?8?$AA@ 100808cc     LIBCMT:undname.obj
 0002:000188e4       ??_C@_08OBABFOLI@?$GAstring?8?$AA@ 100808e4     LIBCMT:undname.obj
 0002:000188f0       ??_C@_0BD@JDLKDPAB@?$GAvbase?5destructor?8?$AA@ 100808f0     LIBCMT:undname.obj
 0002:00018904       ??_C@_0BN@DEGPLNFK@?$GAvector?5deleting?5destructor?8?$AA@ 10080904     LIBCMT:undname.obj
 0002:00018924       ??_C@_0BO@OBMKPJIG@?$GAdefault?5constructor?5closure?8?$AA@ 10080924     LIBCMT:undname.obj
 0002:00018944       ??_C@_0BN@IMDCHIKM@?$GAscalar?5deleting?5destructor?8?$AA@ 10080944     LIBCMT:undname.obj
 0002:00018964       ??_C@_0BO@PFGOCPJJ@?$GAvector?5constructor?5iterator?8?$AA@ 10080964     LIBCMT:undname.obj
 0002:00018984       ??_C@_0BN@LFPFMEDL@?$GAvector?5destructor?5iterator?8?$AA@ 10080984     LIBCMT:undname.obj
 0002:000189a4       ??_C@_0CE@IKBNEHA@?$GAvector?5vbase?5constructor?5iterat@ 100809a4     LIBCMT:undname.obj
 0002:000189c8       ??_C@_0BL@NILFHHPC@?$GAvirtual?5displacement?5map?8?$AA@ 100809c8     LIBCMT:undname.obj
 0002:000189e4       ??_C@_0CB@JONCMFFK@?$GAeh?5vector?5constructor?5iterator?8@ 100809e4     LIBCMT:undname.obj
 0002:00018a08       ??_C@_0CA@GCEOPDGL@?$GAeh?5vector?5destructor?5iterator?8?$AA@ 10080a08     LIBCMT:undname.obj
 0002:00018a28       ??_C@_0CH@OOJPLCPH@?$GAeh?5vector?5vbase?5constructor?5ite@ 10080a28     LIBCMT:undname.obj
 0002:00018a50       ??_C@_0BL@LLKPOHJI@?$GAcopy?5constructor?5closure?8?$AA@ 10080a50     LIBCMT:undname.obj
 0002:00018a6c       ??_C@_0BA@KBCDOMBN@?$GAudt?5returning?8?$AA@ 10080a6c     LIBCMT:undname.obj
 0002:00018a7c       ??_C@_03KLGMFNMG@?$GAEH?$AA@ 10080a7c     LIBCMT:undname.obj
 0002:00018a80       ??_C@_05KHLCHHI@?$GARTTI?$AA@ 10080a80     LIBCMT:undname.obj
 0002:00018a88       ??_C@_0BA@KKLDJDLB@?$GAlocal?5vftable?8?$AA@ 10080a88     LIBCMT:undname.obj
 0002:00018a98       ??_C@_0CE@IIHCMGGL@?$GAlocal?5vftable?5constructor?5closu@ 10080a98     LIBCMT:undname.obj
 0002:00018abc       ??_C@_06FHBGPFGH@?5new?$FL?$FN?$AA@ 10080abc     LIBCMT:undname.obj
 0002:00018ac4       ??_C@_09LBNFPBCA@?5delete?$FL?$FN?$AA@ 10080ac4     LIBCMT:undname.obj
 0002:00018ad0       ??_C@_0P@HJKNJFNN@?$GAomni?5callsig?8?$AA@ 10080ad0     LIBCMT:undname.obj
 0002:00018ae0       ??_C@_0BL@CNOONJFP@?$GAplacement?5delete?5closure?8?$AA@ 10080ae0     LIBCMT:undname.obj
 0002:00018afc       ??_C@_0BN@CKNJLHMB@?$GAplacement?5delete?$FL?$FN?5closure?8?$AA@ 10080afc     LIBCMT:undname.obj
 0002:00018b1c       ??_C@_0CG@CFDHKGGD@?$GAmanaged?5vector?5constructor?5iter@ 10080b1c     LIBCMT:undname.obj
 0002:00018b44       ??_C@_0CF@IMGKMJNO@?$GAmanaged?5vector?5destructor?5itera@ 10080b44     LIBCMT:undname.obj
 0002:00018b6c       ??_C@_0CG@HLDDJMAG@?$GAeh?5vector?5copy?5constructor?5iter@ 10080b6c     LIBCMT:undname.obj
 0002:00018b94       ??_C@_0CM@FCBBDIGB@?$GAeh?5vector?5vbase?5copy?5constructo@ 10080b94     LIBCMT:undname.obj
 0002:00018bc0       ??_C@_0BL@CLIPGLGB@?$GAdynamic?5initializer?5for?5?8?$AA@ 10080bc0     LIBCMT:undname.obj
 0002:00018bdc       ??_C@_0CB@PDBIFEP@?$GAdynamic?5atexit?5destructor?5for?5?8@ 10080bdc     LIBCMT:undname.obj
 0002:00018c00       ??_C@_0CD@CGAJBKEJ@?$GAvector?5copy?5constructor?5iterato@ 10080c00     LIBCMT:undname.obj
 0002:00018c24       ??_C@_0CJ@GJELGAMM@?$GAvector?5vbase?5copy?5constructor?5i@ 10080c24     LIBCMT:undname.obj
 0002:00018c50       ??_C@_0CL@FGIJHLCE@?$GAmanaged?5vector?5copy?5constructor@ 10080c50     LIBCMT:undname.obj
 0002:00018c7c       ??_C@_0BM@PMGGMLDN@?$GAlocal?5static?5thread?5guard?8?$AA@ 10080c7c     LIBCMT:undname.obj
 0002:00018c98       ??_C@_0BC@DAFEJGAK@?5Type?5Descriptor?8?$AA@ 10080c98     LIBCMT:undname.obj
 0002:00018cac       ??_C@_0BM@LDKODKLH@?5Base?5Class?5Descriptor?5at?5?$CI?$AA@ 10080cac     LIBCMT:undname.obj
 0002:00018cc8       ??_C@_0BD@LGICGFMM@?5Base?5Class?5Array?8?$AA@ 10080cc8     LIBCMT:undname.obj
 0002:00018cdc       ??_C@_0BN@MECKDCOJ@?5Class?5Hierarchy?5Descriptor?8?$AA@ 10080cdc     LIBCMT:undname.obj
 0002:00018cfc       ??_C@_0BK@CFCOFLF@?5Complete?5Object?5Locator?8?$AA@ 10080cfc     LIBCMT:undname.obj
 0002:00018d18       ??_C@_04HEJADOOB@CV?3?5?$AA@ 10080d18     LIBCMT:undname.obj
 0002:00018d20       ??_C@_02MOLJINC@?3?3?$AA@  10080d20     LIBCMT:undname.obj
 0002:00018d24       ??_C@_0BE@JAEOCHPE@template?9parameter?9?$AA@ 10080d24     LIBCMT:undname.obj
 0002:00018d38       ??_C@_0O@KHGCOMHP@generic?9type?9?$AA@ 10080d38     LIBCMT:undname.obj
 0002:00018d48       ??_C@_01NLNLIGKH@?$GA?$AA@ 10080d48     LIBCMT:undname.obj
 0002:00018d4c       ??_C@_01GEODFPGF@?8?$AA@   10080d4c     LIBCMT:undname.obj
 0002:00018d50       ??_C@_0BG@JNJLAMPM@?$GAanonymous?5namespace?8?$AA@ 10080d50     LIBCMT:undname.obj
 0002:00018d68       ??_C@_02OHHJMEON@?8?8?$AA@ 10080d68     LIBCMT:undname.obj
 0002:00018d6c       ??_C@_0BN@IBLMMFAP@?$GAnon?9type?9template?9parameter?$AA@ 10080d6c     LIBCMT:undname.obj
 0002:00018d8c       ??_C@_04GKJNKENE@void?$AA@ 10080d8c     LIBCMT:undname.obj
 0002:00018d94       ??_C@_0BE@EODMJLIF@?$GAtemplate?9parameter?$AA@ 10080d94     LIBCMT:undname.obj
 0002:00018da8       ??_C@_03KHICJKCI@?4?4?4?$AA@ 10080da8     LIBCMT:undname.obj
 0002:00018dac       ??_C@_03OPGICMGF@?$HN?8?5?$AA@ 10080dac     LIBCMT:undname.obj
 0002:00018db0       ??_C@_02IGFCGPIL@?$HN?8?$AA@ 10080db0     LIBCMT:undname.obj
 0002:00018db4       ??_C@_01CLKCMJKC@?5?$AA@   10080db4     LIBCMT:undname.obj
 0002:00018db8       ??_C@_0N@CBHHHENL@?$GAvtordispex?$HL?$AA@ 10080db8     LIBCMT:undname.obj
 0002:00018dc8       ??_C@_0L@GHPFDFH@?$GAvtordisp?$HL?$AA@ 10080dc8     LIBCMT:undname.obj
 0002:00018dd4       ??_C@_0L@HNGCOGAE@?$GAadjustor?$HL?$AA@ 10080dd4     LIBCMT:undname.obj
 0002:00018de0       ??_C@_0CB@KJDOOODE@?$GAlocal?5static?5destructor?5helper?8@ 10080de0     LIBCMT:undname.obj
 0002:00018e04       ??_C@_0DB@ILEFOCIJ@?$GAtemplate?5static?5data?5member?5con@ 10080e04     LIBCMT:undname.obj
 0002:00018e38       ??_C@_0DA@HGFJFBBE@?$GAtemplate?5static?5data?5member?5des@ 10080e38     LIBCMT:undname.obj
 0002:00018e68       ??_C@_07PGOEDBHP@static?5?$AA@ 10080e68     LIBCMT:undname.obj
 0002:00018e70       ??_C@_08NIEOINHE@virtual?5?$AA@ 10080e70     LIBCMT:undname.obj
 0002:00018e7c       ??_C@_09LAPHOOG@private?3?5?$AA@ 10080e7c     LIBCMT:undname.obj
 0002:00018e88       ??_C@_0M@GAIFPFIP@protected?3?5?$AA@ 10080e88     LIBCMT:undname.obj
 0002:00018e94       ??_C@_08GPDDCMKI@public?3?5?$AA@ 10080e94     LIBCMT:undname.obj
 0002:00018ea0       ??_C@_08KJLFOPNE@?$FLthunk?$FN?3?$AA@ 10080ea0     LIBCMT:undname.obj
 0002:00018eac       ??_C@_0M@DHNBOJMP@extern?5?$CCC?$CC?5?$AA@ 10080eac     LIBCMT:undname.obj
 0002:00018eb8       ??_C@_02KCKGHPCA@?$CJ?5?$AA@ 10080eb8     LIBCMT:undname.obj
 0002:00018ebc       ??_C@_05CIHEBHNO@char?5?$AA@ 10080ebc     LIBCMT:undname.obj
 0002:00018ec4       ??_C@_06EHJMALKF@short?5?$AA@ 10080ec4     LIBCMT:undname.obj
 0002:00018ecc       ??_C@_04LAHKHJMA@int?5?$AA@ 10080ecc     LIBCMT:undname.obj
 0002:00018ed4       ??_C@_05CJIMAING@long?5?$AA@ 10080ed4     LIBCMT:undname.obj
 0002:00018edc       ??_C@_09EBBEKKIH@unsigned?5?$AA@ 10080edc     LIBCMT:undname.obj
 0002:00018ee8       ??_C@_05BEFAKPML@void?5?$AA@ 10080ee8     LIBCMT:undname.obj
 0002:00018ef0       ??_C@_08PABEKFH@volatile?$AA@ 10080ef0     LIBCMT:undname.obj
 0002:00018efc       ??_C@_0P@GCOCNKDM@std?3?3nullptr_t?$AA@ 10080efc     LIBCMT:undname.obj
 0002:00018f0c       ??_C@_0L@EGPHHEKN@?$DMellipsis?$DO?$AA@ 10080f0c     LIBCMT:undname.obj
 0002:00018f18       ??_C@_04EENFHACM@?0?4?4?4?$AA@ 10080f18     LIBCMT:undname.obj
 0002:00018f20       ??_C@_0M@ELJOJFFH@?0?$DMellipsis?$DO?$AA@ 10080f20     LIBCMT:undname.obj
 0002:00018f2c       ??_C@_07HDJPLPEK@?5throw?$CI?$AA@ 10080f2c     LIBCMT:undname.obj
 0002:00018f34       ??_C@_03PBJBJNON@cpu?$AA@  10080f34     LIBCMT:undname.obj
 0002:00018f38       ??_C@_03DCBBJBAA@amp?$AA@  10080f38     LIBCMT:undname.obj
 0002:00018f3c       ??_C@_02KEGNLNML@?0?5?$AA@ 10080f3c     LIBCMT:undname.obj
 0002:00018f40       ??_C@_04ENMBGAPA@char?$AA@ 10080f40     LIBCMT:undname.obj
 0002:00018f48       ??_C@_05BFKKPKCG@short?$AA@ 10080f48     LIBCMT:undname.obj
 0002:00018f50       ??_C@_03JBIPMCLC@int?$AA@  10080f50     LIBCMT:undname.obj
 0002:00018f54       ??_C@_04GOKPGOLB@long?$AA@ 10080f54     LIBCMT:undname.obj
 0002:00018f5c       ??_C@_05KNFBNCOH@float?$AA@ 10080f5c     LIBCMT:undname.obj
 0002:00018f64       ??_C@_06BNJCAIGJ@double?$AA@ 10080f64     LIBCMT:undname.obj
 0002:00018f6c       ??_C@_04DDKJGDCM@bool?$AA@ 10080f6c     LIBCMT:undname.obj
 0002:00018f74       ??_C@_06EBGKOKIG@__int8?$AA@ 10080f74     LIBCMT:undname.obj
 0002:00018f7c       ??_C@_07ICFHOGAF@__int16?$AA@ 10080f7c     LIBCMT:undname.obj
 0002:00018f84       ??_C@_07OFLPPHGP@__int32?$AA@ 10080f84     LIBCMT:undname.obj
 0002:00018f8c       ??_C@_07LFCOJCAC@__int64?$AA@ 10080f8c     LIBCMT:undname.obj
 0002:00018f94       ??_C@_08GAHOLHEO@__int128?$AA@ 10080f94     LIBCMT:undname.obj
 0002:00018fa0       ??_C@_09EEKGDCPH@?$DMunknown?$DO?$AA@ 10080fa0     LIBCMT:undname.obj
 0002:00018fac       ??_C@_07CLGGIAMF@wchar_t?$AA@ 10080fac     LIBCMT:undname.obj
 0002:00018fb4       ??_C@_06GCICPBLB@__w64?5?$AA@ 10080fb4     LIBCMT:undname.obj
 0002:00018fbc       ??_C@_07NFANNNEC@UNKNOWN?$AA@ 10080fbc     LIBCMT:undname.obj
 0002:00018fc4       ??_C@_07EDHNAJHC@signed?5?$AA@ 10080fc4     LIBCMT:undname.obj
 0002:00018fcc       ??_C@_05BNCCCJPP@const?$AA@ 10080fcc     LIBCMT:undname.obj
 0002:00018fd4       ??_C@_09EFNPDFFP@?5volatile?$AA@ 10080fd4     LIBCMT:undname.obj
 0002:00018fe0       ??_C@_0P@GCIFDJCJ@?$GAunknown?5ecsu?8?$AA@ 10080fe0     LIBCMT:undname.obj
 0002:00018ff0       ??_C@_06MOJHIBMG@union?5?$AA@ 10080ff0     LIBCMT:undname.obj
 0002:00018ff8       ??_C@_07DIBCDNGL@struct?5?$AA@ 10080ff8     LIBCMT:undname.obj
 0002:00019000       ??_C@_06LJBABKPM@class?5?$AA@ 10081000     LIBCMT:undname.obj
 0002:00019008       ??_C@_08KOFANOFK@coclass?5?$AA@ 10081008     LIBCMT:undname.obj
 0002:00019014       ??_C@_0N@DLIEFKNA@cointerface?5?$AA@ 10081014     LIBCMT:undname.obj
 0002:00019024       ??_C@_05LJGMCFOG@enum?5?$AA@ 10081024     LIBCMT:undname.obj
 0002:0001902c       ??_C@_09GAIEOBLP@volatile?5?$AA@ 1008102c     LIBCMT:undname.obj
 0002:00019038       ??_C@_06LIJLOJAG@const?5?$AA@ 10081038     LIBCMT:undname.obj
 0002:00019040       ??_C@_0M@EALIELKG@cli?3?3array?$DM?$AA@ 10081040     LIBCMT:undname.obj
 0002:0001904c       ??_C@_0O@GKABPPIF@cli?3?3pin_ptr?$DM?$AA@ 1008104c     LIBCMT:undname.obj
 0002:0001905c       ??_C@_02GOGNNPBN@?$CJ?$FL?$AA@ 1008105c     LIBCMT:undname.obj
 0002:00019060       ??_C@_06EEGAIFAK@?$HLflat?$HN?$AA@ 10081060     LIBCMT:undname.obj
 0002:00019068       ??_C@_05JIBOFOHK@?$HLfor?5?$AA@ 10081068     LIBCMT:undname.obj
 0002:00019070       ??_C@_02MDINNEEG@s?5?$AA@  10081070     LIBCMT:undname.obj
 0002:00019078       ??_7DNameNode@@6B@         10081078     LIBCMT:undname.obj
 0002:00019088       ??_7charNode@@6B@          10081088     LIBCMT:undname.obj
 0002:00019098       ??_7pcharNode@@6B@         10081098     LIBCMT:undname.obj
 0002:000190a8       ??_7pDNameNode@@6B@        100810a8     LIBCMT:undname.obj
 0002:000190b8       ??_7DNameStatusNode@@6B@   100810b8     LIBCMT:undname.obj
 0002:000190c8       ??_7pairNode@@6B@          100810c8     LIBCMT:undname.obj
 0002:000190d4       ??_C@_04OKOHEJBO@?5?$DP?$DP?5?$AA@ 100810d4     LIBCMT:undname.obj
 0002:000190e0       __indefinite               100810e0     LIBCMT:87disp.obj
 0002:000190ea       __piby2                    100810ea     LIBCMT:87disp.obj
 0002:00019118       __DEFAULT_CW_in_mem        10081118     LIBCMT:common.obj
 0002:0001911a       __pi_by_2_to_61            1008111a     LIBCMT:common.obj
 0002:00019a80       __infinity                 10081a80     LIBCMT:87tran.obj
 0002:00019a8a       __minfinity                10081a8a     LIBCMT:87tran.obj
 0002:00019a94       __logemax                  10081a94     LIBCMT:87tran.obj
 0002:00019aba       __OP_EXPjmptab             10081aba     LIBCMT:87tran.obj
 0002:0001d420       __real@3fe0000000000000    10085420     LIBCMT:powhlp.obj
 0002:0001dcd0       ??_C@_06PGGFOGJG@1?$CDSNAN?$AA@ 10085cd0     LIBCMT:x10fout.obj
 0002:0001dcd8       ??_C@_05PHHOCPM@1?$CDIND?$AA@ 10085cd8     LIBCMT:x10fout.obj
 0002:0001dce0       ??_C@_05DNEBIAHO@1?$CDINF?$AA@ 10085ce0     LIBCMT:x10fout.obj
 0002:0001dce8       ??_C@_06IMKFLFPG@1?$CDQNAN?$AA@ 10085ce8     LIBCMT:x10fout.obj
 0002:0001dcf0       ??_C@_0M@HHGEPIBF@CreateFile2?$AA@ 10085cf0     LIBCMT:wopen.obj
 0002:0001dcfc       ??_C@_1BA@BALFACEM@?$AAC?$AAO?$AAN?$AAO?$AAU?$AAT?$AA$?$AA?$AA@ 10085cfc     LIBCMT:initcon.obj
 0002:0001dd0c       __real@00000000            10085d0c     LIBCMT:wcstoq.obj
 0002:0001dd10       ??_C@_1M@KLMEPMCM@?$AAa?$AAl?$AAn?$AAu?$AAm?$AA?$AA@ 10085d10     libcpmt:xthrow.obj
 0002:0001dd1c       ??_C@_1M@DHGLHBMI@?$AAa?$AAl?$AAp?$AAh?$AAa?$AA?$AA@ 10085d1c     libcpmt:xthrow.obj
 0002:0001dd28       ??_C@_1M@EJAAJBPE@?$AAb?$AAl?$AAa?$AAn?$AAk?$AA?$AA@ 10085d28     libcpmt:xthrow.obj
 0002:0001dd34       ??_C@_1M@LMIMILA@?$AAc?$AAn?$AAt?$AAr?$AAl?$AA?$AA@ 10085d34     libcpmt:xthrow.obj
 0002:0001dd40       ??_C@_13GKPPEALH@?$AAd?$AA?$AA@ 10085d40     libcpmt:xthrow.obj
 0002:0001dd44       ??_C@_1M@JDAEIBKG@?$AAd?$AAi?$AAg?$AAi?$AAt?$AA?$AA@ 10085d44     libcpmt:xthrow.obj
 0002:0001dd50       ??_C@_1M@MDKNJLLK@?$AAg?$AAr?$AAa?$AAp?$AAh?$AA?$AA@ 10085d50     libcpmt:xthrow.obj
 0002:0001dd5c       ??_C@_1M@LGAECJJD@?$AAl?$AAo?$AAw?$AAe?$AAr?$AA?$AA@ 10085d5c     libcpmt:xthrow.obj
 0002:0001dd68       ??_C@_1M@ELNLAPLA@?$AAp?$AAr?$AAi?$AAn?$AAt?$AA?$AA@ 10085d68     libcpmt:xthrow.obj
 0002:0001dd74       ??_C@_1M@BPFMAOAO@?$AAp?$AAu?$AAn?$AAc?$AAt?$AA?$AA@ 10085d74     libcpmt:xthrow.obj
 0002:0001dd80       ??_C@_1M@LPGODFOM@?$AAs?$AAp?$AAa?$AAc?$AAe?$AA?$AA@ 10085d80     libcpmt:xthrow.obj
 0002:0001dd8c       ??_C@_13KHDBCPJB@?$AAs?$AA?$AA@ 10085d8c     libcpmt:xthrow.obj
 0002:0001dd90       ??_C@_1M@PLNFCNIC@?$AAu?$AAp?$AAp?$AAe?$AAr?$AA?$AA@ 10085d90     libcpmt:xthrow.obj
 0002:0001dd9c       ??_C@_13CIFDLIMG@?$AAw?$AA?$AA@ 10085d9c     libcpmt:xthrow.obj
 0002:0001dda0       ??_C@_1O@OAFMJDHN@?$AAx?$AAd?$AAi?$AAg?$AAi?$AAt?$AA?$AA@ 10085da0     libcpmt:xthrow.obj
 0002:0001ddb0       ?_VBITS@?$vector@_NV?$allocator@_N@std@@@std@@2HB 10085db0     libcpmt:xthrow.obj
 0002:0001ddb4       ?value@?$integral_constant@H$0A@@std@@2HB 10085db4     libcpmt:xthrow.obj
 0002:0001ddb8       ?_Names@?$_Regex_traits@D@std@@0QBU?$_Cl_names@D@2@B 10085db8     libcpmt:xthrow.obj
 0002:0001de78       ??_C@_05IIMHCHIO@alnum?$AA@ 10085e78     libcpmt:xthrow.obj
 0002:0001de80       ??_C@_05IAEKHIAN@alpha?$AA@ 10085e80     libcpmt:xthrow.obj
 0002:0001de88       ??_C@_05BABJKOGB@blank?$AA@ 10085e88     libcpmt:xthrow.obj
 0002:0001de90       ??_C@_05JMDPEFNK@cntrl?$AA@ 10085e90     libcpmt:xthrow.obj
 0002:0001de98       ??_C@_01LPLHEDKD@d?$AA@    10085e98     libcpmt:xthrow.obj
 0002:0001de9c       ??_C@_05ODNOIFML@digit?$AA@ 10085e9c     libcpmt:xthrow.obj
 0002:0001dea4       ??_C@_05KCJBMLII@graph?$AA@ 10085ea4     libcpmt:xthrow.obj
 0002:0001deac       ??_C@_05IPJEPLHL@lower?$AA@ 10085eac     libcpmt:xthrow.obj
 0002:0001deb4       ??_C@_05IJDJACGD@print?$AA@ 10085eb4     libcpmt:xthrow.obj
 0002:0001debc       ??_C@_05KOBGHFJJ@punct?$AA@ 10085ebc     libcpmt:xthrow.obj
 0002:0001dec4       ??_C@_05OLNILLAB@space?$AA@ 10085ec4     libcpmt:xthrow.obj
 0002:0001decc       ??_C@_01LKDEMHDF@s?$AA@    10085ecc     libcpmt:xthrow.obj
 0002:0001ded0       ??_C@_05NECKJAMC@upper?$AA@ 10085ed0     libcpmt:xthrow.obj
 0002:0001ded8       ??_C@_06BAPHGFFK@xdigit?$AA@ 10085ed8     libcpmt:xthrow.obj
 0002:0001dee0       ?_Names@?$_Regex_traits@_W@std@@0QBU?$_Cl_names@_W@2@B 10085ee0     libcpmt:xthrow.obj
 0002:0001dfa4       ??_7logic_error@std@@6B@   10085fa4     libcpmt:xthrow.obj
 0002:0001dfb0       ??_7invalid_argument@std@@6B@ 10085fb0     libcpmt:xthrow.obj
 0002:0001dfbc       ??_7length_error@std@@6B@  10085fbc     libcpmt:xthrow.obj
 0002:0001dfc8       ??_7out_of_range@std@@6B@  10085fc8     libcpmt:xthrow.obj
 0002:0001dfd4       ??_7runtime_error@std@@6B@ 10085fd4     libcpmt:xthrow.obj
 0002:0001dfe0       ??_7overflow_error@std@@6B@ 10085fe0     libcpmt:xthrow.obj
 0002:0001dfec       ??_7bad_function_call@std@@6B@ 10085fec     libcpmt:xthrow.obj
 0002:0001dff4       ??_C@_0BC@DPJNKNAF@bad?5function?5call?$AA@ 10085ff4     libcpmt:xthrow.obj
 0002:0001e00c       ??_7regex_error@std@@6B@   1008600c     libcpmt:xthrow.obj
 0002:0001e018       ??_C@_0FI@CMNGHIFF@regex_error?$CIerror_collate?$CJ?3?5The?5@ 10086018     libcpmt:xthrow.obj
 0002:0001e070       ??_C@_0FE@LJMHKIOC@regex_error?$CIerror_ctype?$CJ?3?5The?5ex@ 10086070     libcpmt:xthrow.obj
 0002:0001e0c8       ??_C@_0GI@HEGGMMDL@regex_error?$CIerror_escape?$CJ?3?5The?5e@ 100860c8     libcpmt:xthrow.obj
 0002:0001e130       ??_C@_0FA@HFMLPGNN@regex_error?$CIerror_backref?$CJ?3?5The?5@ 10086130     libcpmt:xthrow.obj
 0002:0001e180       ??_C@_0EH@LGEANNAL@regex_error?$CIerror_brack?$CJ?3?5The?5ex@ 10086180     libcpmt:xthrow.obj
 0002:0001e1c8       ??_C@_0EH@CAGOJGLE@regex_error?$CIerror_paren?$CJ?3?5The?5ex@ 100861c8     libcpmt:xthrow.obj
 0002:0001e210       ??_C@_0EH@DICJJKLO@regex_error?$CIerror_brace?$CJ?3?5The?5ex@ 10086210     libcpmt:xthrow.obj
 0002:0001e258       ??_C@_0FM@BLDIHIBB@regex_error?$CIerror_badbrace?$CJ?3?5The@ 10086258     libcpmt:xthrow.obj
 0002:0001e2b8       ??_C@_0HA@ICNJLCMC@regex_error?$CIerror_range?$CJ?3?5The?5ex@ 100862b8     libcpmt:xthrow.obj
 0002:0001e328       ??_C@_0GP@PICOBCHA@regex_error?$CIerror_space?$CJ?3?5There?5@ 10086328     libcpmt:xthrow.obj
 0002:0001e398       ??_C@_0FK@LCHHHEOA@regex_error?$CIerror_badrepeat?$CJ?3?5On@ 10086398     libcpmt:xthrow.obj
 0002:0001e3f8       ??_C@_0HL@NEKOFBJA@regex_error?$CIerror_complexity?$CJ?3?5T@ 100863f8     libcpmt:xthrow.obj
 0002:0001e478       ??_C@_0JC@HCDLJLGO@regex_error?$CIerror_stack?$CJ?3?5There?5@ 10086478     libcpmt:xthrow.obj
 0002:0001e50c       ??_C@_0BJ@CHBLKGNM@regex_error?$CIerror_parse?$CJ?$AA@ 1008650c     libcpmt:xthrow.obj
 0002:0001e528       ??_C@_0BK@DFJCACNI@regex_error?$CIerror_syntax?$CJ?$AA@ 10086528     libcpmt:xthrow.obj
 0002:0001e544       ??_C@_0M@KGKAAGCA@regex_error?$AA@ 10086544     libcpmt:xthrow.obj
 0002:0001e550       ??_C@_0BG@DHPCNBJB@address?5not?5available?$AA@ 10086550     libcpmt:syserror.obj
 0002:0001e568       ??_C@_0BC@DFIBIBIL@already?5connected?$AA@ 10086568     libcpmt:syserror.obj
 0002:0001e57c       ??_C@_0BH@CAKOHOMI@argument?5list?5too?5long?$AA@ 1008657c     libcpmt:syserror.obj
 0002:0001e594       ??_C@_0BH@CGIMPKIM@argument?5out?5of?5domain?$AA@ 10086594     libcpmt:syserror.obj
 0002:0001e5ac       ??_C@_0M@KGHGGJGL@bad?5address?$AA@ 100865ac     libcpmt:syserror.obj
 0002:0001e5b8       ??_C@_0BE@MPJPGCEO@bad?5file?5descriptor?$AA@ 100865b8     libcpmt:syserror.obj
 0002:0001e5cc       ??_C@_0M@PMMIEFCP@bad?5message?$AA@ 100865cc     libcpmt:syserror.obj
 0002:0001e5d8       ??_C@_0M@KPHOFDBE@broken?5pipe?$AA@ 100865d8     libcpmt:syserror.obj
 0002:0001e5e4       ??_C@_0BD@MGNDDEGM@connection?5aborted?$AA@ 100865e4     libcpmt:syserror.obj
 0002:0001e5f8       ??_C@_0BP@KAIHPOGN@connection?5already?5in?5progress?$AA@ 100865f8     libcpmt:syserror.obj
 0002:0001e618       ??_C@_0BD@PJLIIJEL@connection?5refused?$AA@ 10086618     libcpmt:syserror.obj
 0002:0001e62c       ??_C@_0BB@IECNJNOI@connection?5reset?$AA@ 1008662c     libcpmt:syserror.obj
 0002:0001e640       ??_C@_0BN@KDMIFEIP@destination?5address?5required?$AA@ 10086640     libcpmt:syserror.obj
 0002:0001e660       ??_C@_0BI@BNCLIGPB@executable?5format?5error?$AA@ 10086660     libcpmt:syserror.obj
 0002:0001e678       ??_C@_0P@DNAJLBJK@file?5too?5large?$AA@ 10086678     libcpmt:syserror.obj
 0002:0001e688       ??_C@_0BB@DHFDFGDM@host?5unreachable?$AA@ 10086688     libcpmt:syserror.obj
 0002:0001e69c       ??_C@_0BD@JPHBMONG@identifier?5removed?$AA@ 1008669c     libcpmt:syserror.obj
 0002:0001e6b0       ??_C@_0BG@CDNPAGJK@illegal?5byte?5sequence?$AA@ 100866b0     libcpmt:syserror.obj
 0002:0001e6c8       ??_C@_0CD@BNPLBMNA@inappropriate?5io?5control?5operati@ 100866c8     libcpmt:syserror.obj
 0002:0001e6ec       ??_C@_0N@OHAFKDEK@invalid?5seek?$AA@ 100866ec     libcpmt:syserror.obj
 0002:0001e6fc       ??_C@_0P@FLLDBIDK@is?5a?5directory?$AA@ 100866fc     libcpmt:syserror.obj
 0002:0001e70c       ??_C@_0N@IFLPBIOP@message?5size?$AA@ 1008670c     libcpmt:syserror.obj
 0002:0001e71c       ??_C@_0N@KIIEAAIO@network?5down?$AA@ 1008671c     libcpmt:syserror.obj
 0002:0001e72c       ??_C@_0O@FNPDBHEE@network?5reset?$AA@ 1008672c     libcpmt:syserror.obj
 0002:0001e73c       ??_C@_0BE@IFNCKGE@network?5unreachable?$AA@ 1008673c     libcpmt:syserror.obj
 0002:0001e750       ??_C@_0BA@PFFCAOFK@no?5buffer?5space?$AA@ 10086750     libcpmt:syserror.obj
 0002:0001e760       ??_C@_0BB@IEPBLJHK@no?5child?5process?$AA@ 10086760     libcpmt:syserror.obj
 0002:0001e774       ??_C@_07PLECNNKG@no?5link?$AA@ 10086774     libcpmt:syserror.obj
 0002:0001e77c       ??_C@_0BF@PBGGPKKE@no?5message?5available?$AA@ 1008677c     libcpmt:syserror.obj
 0002:0001e794       ??_C@_0L@EDOLMPAK@no?5message?$AA@ 10086794     libcpmt:syserror.obj
 0002:0001e7a0       ??_C@_0BD@EAMBFIDF@no?5protocol?5option?$AA@ 100867a0     libcpmt:syserror.obj
 0002:0001e7b4       ??_C@_0BE@MKFDAFMP@no?5stream?5resources?$AA@ 100867b4     libcpmt:syserror.obj
 0002:0001e7c8       ??_C@_0BK@IMCPHCBI@no?5such?5device?5or?5address?$AA@ 100867c8     libcpmt:syserror.obj
 0002:0001e7e4       ??_C@_0BA@ENLPPKBN@no?5such?5process?$AA@ 100867e4     libcpmt:syserror.obj
 0002:0001e7f4       ??_C@_0BA@DOCPFFJG@not?5a?5directory?$AA@ 100867f4     libcpmt:syserror.obj
 0002:0001e804       ??_C@_0N@POEIPGGF@not?5a?5socket?$AA@ 10086804     libcpmt:syserror.obj
 0002:0001e814       ??_C@_0N@LGAPMMPI@not?5a?5stream?$AA@ 10086814     libcpmt:syserror.obj
 0002:0001e824       ??_C@_0O@GLMIBBEG@not?5connected?$AA@ 10086824     libcpmt:syserror.obj
 0002:0001e834       ??_C@_0O@NHEDABJP@not?5supported?$AA@ 10086834     libcpmt:syserror.obj
 0002:0001e844       ??_C@_0BG@KDKHOPCO@operation?5in?5progress?$AA@ 10086844     libcpmt:syserror.obj
 0002:0001e85c       ??_C@_0BI@OHIEJAAB@operation?5not?5permitted?$AA@ 1008685c     libcpmt:syserror.obj
 0002:0001e874       ??_C@_0BI@LNEGIFLN@operation?5not?5supported?$AA@ 10086874     libcpmt:syserror.obj
 0002:0001e88c       ??_C@_0BG@OEMDKMEE@operation?5would?5block?$AA@ 1008688c     libcpmt:syserror.obj
 0002:0001e8a4       ??_C@_0L@BLPOFLNJ@owner?5dead?$AA@ 100868a4     libcpmt:syserror.obj
 0002:0001e8b0       ??_C@_0P@FNPOCJBE@protocol?5error?$AA@ 100868b0     libcpmt:syserror.obj
 0002:0001e8c0       ??_C@_0BH@JPPPLHJB@protocol?5not?5supported?$AA@ 100868c0     libcpmt:syserror.obj
 0002:0001e8d8       ??_C@_0BG@EICBIHDP@read?5only?5file?5system?$AA@ 100868d8     libcpmt:syserror.obj
 0002:0001e8f0       ??_C@_0BO@BJBOMOEJ@resource?5deadlock?5would?5occur?$AA@ 100868f0     libcpmt:syserror.obj
 0002:0001e910       ??_C@_0BE@GOIPJJHG@result?5out?5of?5range?$AA@ 10086910     libcpmt:syserror.obj
 0002:0001e924       ??_C@_0BG@MPLKFPAE@state?5not?5recoverable?$AA@ 10086924     libcpmt:syserror.obj
 0002:0001e93c       ??_C@_0P@DIIFGFCG@stream?5timeout?$AA@ 1008693c     libcpmt:syserror.obj
 0002:0001e94c       ??_C@_0P@IPFDMIFL@text?5file?5busy?$AA@ 1008694c     libcpmt:syserror.obj
 0002:0001e95c       ??_C@_09KJPPMAOI@timed?5out?$AA@ 1008695c     libcpmt:syserror.obj
 0002:0001e968       ??_C@_0BO@HACHBEKI@too?5many?5files?5open?5in?5system?$AA@ 10086968     libcpmt:syserror.obj
 0002:0001e988       ??_C@_0P@HCOMKFCC@too?5many?5links?$AA@ 10086988     libcpmt:syserror.obj
 0002:0001e998       ??_C@_0BO@EFGOJEF@too?5many?5symbolic?5link?5levels?$AA@ 10086998     libcpmt:syserror.obj
 0002:0001e9b8       ??_C@_0BA@KGKGOOJA@value?5too?5large?$AA@ 100869b8     libcpmt:syserror.obj
 0002:0001e9c8       ??_C@_0BE@MIEJDDNH@wrong?5protocol?5type?$AA@ 100869c8     libcpmt:syserror.obj
 0002:0001eeb0       ??_C@_0BC@CIJDGCDI@permission?5denied?$AA@ 10086eb0     libcpmt:syserror.obj
 0002:0001eec4       ??_C@_0M@MIDIAGJP@file?5exists?$AA@ 10086ec4     libcpmt:syserror.obj
 0002:0001eed0       ??_C@_0P@FDINDDOK@no?5such?5device?$AA@ 10086ed0     libcpmt:syserror.obj
 0002:0001eee0       ??_C@_0BC@EJHOMAAK@filename?5too?5long?$AA@ 10086ee0     libcpmt:syserror.obj
 0002:0001eef4       ??_C@_0BI@NGCEHDD@device?5or?5resource?5busy?$AA@ 10086ef4     libcpmt:syserror.obj
 0002:0001ef0c       ??_C@_08GLNPIFBN@io?5error?$AA@ 10086f0c     libcpmt:syserror.obj
 0002:0001ef18       ??_C@_0BE@JIDOCPHM@directory?5not?5empty?$AA@ 10086f18     libcpmt:syserror.obj
 0002:0001ef2c       ??_C@_0BB@FCMFBGOM@invalid?5argument?$AA@ 10086f2c     libcpmt:syserror.obj
 0002:0001ef40       ??_C@_0BD@IJDJKDEA@no?5space?5on?5device?$AA@ 10086f40     libcpmt:syserror.obj
 0002:0001ef54       ??_C@_0BK@NDOCBPGE@no?5such?5file?5or?5directory?$AA@ 10086f54     libcpmt:syserror.obj
 0002:0001ef70       ??_C@_0BH@KEFGLDAF@function?5not?5supported?$AA@ 10086f70     libcpmt:syserror.obj
 0002:0001ef88       ??_C@_0BC@NJECKMKE@no?5lock?5available?$AA@ 10086f88     libcpmt:syserror.obj
 0002:0001ef9c       ??_C@_0BC@ENOOLCNF@not?5enough?5memory?$AA@ 10086f9c     libcpmt:syserror.obj
 0002:0001efb0       ??_C@_0BP@LKNGHENJ@resource?5unavailable?5try?5again?$AA@ 10086fb0     libcpmt:syserror.obj
 0002:0001efd0       ??_C@_0BC@PPHBOELF@cross?5device?5link?$AA@ 10086fd0     libcpmt:syserror.obj
 0002:0001efe4       ??_C@_0BD@MOLBPMEA@operation?5canceled?$AA@ 10086fe4     libcpmt:syserror.obj
 0002:0001eff8       ??_C@_0BE@GHAFMPAH@too?5many?5files?5open?$AA@ 10086ff8     libcpmt:syserror.obj
 0002:0001f00c       ??_C@_0BC@FNODOBAE@permission_denied?$AA@ 1008700c     libcpmt:syserror.obj
 0002:0001f020       ??_C@_0P@LNDJPBFK@address_in_use?$AA@ 10087020     libcpmt:syserror.obj
 0002:0001f030       ??_C@_0BG@IPMGOJF@address_not_available?$AA@ 10087030     libcpmt:syserror.obj
 0002:0001f048       ??_C@_0BN@LCBDHODA@address_family_not_supported?$AA@ 10087048     libcpmt:syserror.obj
 0002:0001f068       ??_C@_0BP@FOJJHMCC@connection_already_in_progress?$AA@ 10087068     libcpmt:syserror.obj
 0002:0001f088       ??_C@_0BE@DLHHIBGN@bad_file_descriptor?$AA@ 10087088     libcpmt:syserror.obj
 0002:0001f09c       ??_C@_0BD@OJMJDIGI@connection_aborted?$AA@ 1008709c     libcpmt:syserror.obj
 0002:0001f0b0       ??_C@_0BD@NGKCIFEP@connection_refused?$AA@ 100870b0     libcpmt:syserror.obj
 0002:0001f0c4       ??_C@_0BB@JOANDNCK@connection_reset?$AA@ 100870c4     libcpmt:syserror.obj
 0002:0001f0d8       ??_C@_0BN@JLJNLKLK@destination_address_required?$AA@ 100870d8     libcpmt:syserror.obj
 0002:0001f0f8       ??_C@_0M@IJGMGFGP@bad_address?$AA@ 100870f8     libcpmt:syserror.obj
 0002:0001f104       ??_C@_0BB@KKNHPPIN@host_unreachable?$AA@ 10087104     libcpmt:syserror.obj
 0002:0001f118       ??_C@_0BG@DJGBJIIK@operation_in_progress?$AA@ 10087118     libcpmt:syserror.obj
 0002:0001f130       ??_C@_0M@EGEKIIMP@interrupted?$AA@ 10087130     libcpmt:syserror.obj
 0002:0001f13c       ??_C@_0BB@FFIHMIPJ@invalid_argument?$AA@ 1008713c     libcpmt:syserror.obj
 0002:0001f150       ??_C@_0BC@FIFLCHLO@already_connected?$AA@ 10087150     libcpmt:syserror.obj
 0002:0001f164       ??_C@_0BE@GJJJJDDA@too_many_files_open?$AA@ 10087164     libcpmt:syserror.obj
 0002:0001f178       ??_C@_0N@HPMLKHPL@message_size?$AA@ 10087178     libcpmt:syserror.obj
 0002:0001f188       ??_C@_0BC@LEEIKBAL@filename_too_long?$AA@ 10087188     libcpmt:syserror.obj
 0002:0001f19c       ??_C@_0N@FCPALPJK@network_down?$AA@ 1008719c     libcpmt:syserror.obj
 0002:0001f1ac       ??_C@_0O@EHNDLHIG@network_reset?$AA@ 100871ac     libcpmt:syserror.obj
 0002:0001f1bc       ??_C@_0BE@JFNJIDNF@network_unreachable?$AA@ 100871bc     libcpmt:syserror.obj
 0002:0001f1d0       ??_C@_0BA@FDIJKJCL@no_buffer_space?$AA@ 100871d0     libcpmt:syserror.obj
 0002:0001f1e0       ??_C@_0BD@JHIHCGKP@no_protocol_option?$AA@ 100871e0     libcpmt:syserror.obj
 0002:0001f1f4       ??_C@_0O@GBCLHHD@not_connected?$AA@ 100871f4     libcpmt:syserror.obj
 0002:0001f204       ??_C@_0N@IMHKKLEM@not_a_socket?$AA@ 10087204     libcpmt:syserror.obj
 0002:0001f214       ??_C@_0BI@ICEIDKLJ@operation_not_supported?$AA@ 10087214     libcpmt:syserror.obj
 0002:0001f22c       ??_C@_0BH@KAPBAIJF@protocol_not_supported?$AA@ 1008722c     libcpmt:syserror.obj
 0002:0001f244       ??_C@_0BE@GAOJJFPC@wrong_protocol_type?$AA@ 10087244     libcpmt:syserror.obj
 0002:0001f258       ??_C@_09NCHNLHPG@timed_out?$AA@ 10087258     libcpmt:syserror.obj
 0002:0001f264       ??_C@_0BG@GDGHKFDH@operation_would_block?$AA@ 10087264     libcpmt:syserror.obj
 0002:0001f27c       ??_C@_0BN@LKKBCCDB@address?5family?5not?5supported?$AA@ 1008727c     libcpmt:syserror.obj
 0002:0001f29c       ??_C@_0P@LDMLAFHI@address?5in?5use?$AA@ 1008729c     libcpmt:syserror.obj
 0002:0001f2b0       __load_config_used         100872b0     LIBCMT:loadcfg.obj
 0002:0001f350       ??_R4SnmpRequest@@6B@      10087350     asisnmp.obj
 0002:0001f364       ??_R3SnmpRequest@@8        10087364     asisnmp.obj
 0002:0001f374       ??_R2SnmpRequest@@8        10087374     asisnmp.obj
 0002:0001f37c       ??_R1A@?0A@EA@SnmpRequest@@8 1008737c     asisnmp.obj
 0002:0001f398       ??_R4SnmpGetRequest@@6B@   10087398     asisnmp.obj
 0002:0001f3ac       ??_R3SnmpGetRequest@@8     100873ac     asisnmp.obj
 0002:0001f3bc       ??_R2SnmpGetRequest@@8     100873bc     asisnmp.obj
 0002:0001f3c8       ??_R1A@?0A@EA@SnmpGetRequest@@8 100873c8     asisnmp.obj
 0002:0001f3e4       ??_R4SnmpGetNextRequest@@6B@ 100873e4     asisnmp.obj
 0002:0001f3f8       ??_R3SnmpGetNextRequest@@8 100873f8     asisnmp.obj
 0002:0001f408       ??_R2SnmpGetNextRequest@@8 10087408     asisnmp.obj
 0002:0001f414       ??_R1A@?0A@EA@SnmpGetNextRequest@@8 10087414     asisnmp.obj
 0002:0001f430       ??_R4SnmpSetRequest@@6B@   10087430     asisnmp.obj
 0002:0001f444       ??_R3SnmpSetRequest@@8     10087444     asisnmp.obj
 0002:0001f454       ??_R2SnmpSetRequest@@8     10087454     asisnmp.obj
 0002:0001f460       ??_R1A@?0A@EA@SnmpSetRequest@@8 10087460     asisnmp.obj
 0002:0001f47c       ??_R1A@?0A@EA@asxBase@@8   1008747c     asxavdecc.obj
 0002:0001f498       ??_R3asxBase@@8            10087498     asxavdecc.obj
 0002:0001f4a8       ??_R2asxBase@@8            100874a8     asxavdecc.obj
 0002:0001f4b0       ??_R4asxAdapterAVDECC@@6B@ 100874b0     asxavdecc.obj
 0002:0001f4c4       ??_R3asxAdapterAVDECC@@8   100874c4     asxavdecc.obj
 0002:0001f4d4       ??_R2asxAdapterAVDECC@@8   100874d4     asxavdecc.obj
 0002:0001f4e4       ??_R1A@?0A@EA@asxAdapterAVDECC@@8 100874e4     asxavdecc.obj
 0002:0001f500       ??_R1A@?0A@EA@asxAdapter@@8 10087500     asxavdecc.obj
 0002:0001f51c       ??_R3asxAdapter@@8         1008751c     asxavdecc.obj
 0002:0001f52c       ??_R2asxAdapter@@8         1008752c     asxavdecc.obj
 0002:0001f538       ??_R4asxSubSystemAVDECC@@6B@ 10087538     asxavdecc.obj
 0002:0001f54c       ??_R3asxSubSystemAVDECC@@8 1008754c     asxavdecc.obj
 0002:0001f55c       ??_R2asxSubSystemAVDECC@@8 1008755c     asxavdecc.obj
 0002:0001f568       ??_R1A@?0A@EA@asxSubSystemAVDECC@@8 10087568     asxavdecc.obj
 0002:0001f584       ??_R1A@?0A@EA@asxSubSystem@@8 10087584     asxavdecc.obj
 0002:0001f5a0       ??_R3asxSubSystem@@8       100875a0     asxavdecc.obj
 0002:0001f5b0       ??_R2asxSubSystem@@8       100875b0     asxavdecc.obj
 0002:0001f5b8       ??_R4error_category@std@@6B@ 100875b8     asxavdecc.obj
 0002:0001f5cc       ??_R3error_category@std@@8 100875cc     asxavdecc.obj
 0002:0001f5dc       ??_R2error_category@std@@8 100875dc     asxavdecc.obj
 0002:0001f5e4       ??_R1A@?0A@EA@error_category@std@@8 100875e4     asxavdecc.obj
 0002:0001f600       ??_R4_Generic_error_category@std@@6B@ 10087600     asxavdecc.obj
 0002:0001f614       ??_R3_Generic_error_category@std@@8 10087614     asxavdecc.obj
 0002:0001f624       ??_R2_Generic_error_category@std@@8 10087624     asxavdecc.obj
 0002:0001f630       ??_R1A@?0A@EA@_Generic_error_category@std@@8 10087630     asxavdecc.obj
 0002:0001f64c       ??_R4_Iostream_error_category@std@@6B@ 1008764c     asxavdecc.obj
 0002:0001f660       ??_R3_Iostream_error_category@std@@8 10087660     asxavdecc.obj
 0002:0001f670       ??_R2_Iostream_error_category@std@@8 10087670     asxavdecc.obj
 0002:0001f680       ??_R1A@?0A@EA@_Iostream_error_category@std@@8 10087680     asxavdecc.obj
 0002:0001f69c       ??_R4_System_error_category@std@@6B@ 1008769c     asxavdecc.obj
 0002:0001f6b0       ??_R3_System_error_category@std@@8 100876b0     asxavdecc.obj
 0002:0001f6c0       ??_R2_System_error_category@std@@8 100876c0     asxavdecc.obj
 0002:0001f6d0       ??_R1A@?0A@EA@_System_error_category@std@@8 100876d0     asxavdecc.obj
 0002:0001f6ec       ??_R4asxMixerScanner@@6B@  100876ec     asxasio.obj
 0002:0001f700       ??_R3asxMixerScanner@@8    10087700     asxasio.obj
 0002:0001f710       ??_R2asxMixerScanner@@8    10087710     asxasio.obj
 0002:0001f718       ??_R1A@?0A@EA@asxMixerScanner@@8 10087718     asxasio.obj
 0002:0001f734       ??_R4asxAdapterASIO@@6B@   10087734     asxasio.obj
 0002:0001f748       ??_R3asxAdapterASIO@@8     10087748     asxasio.obj
 0002:0001f758       ??_R2asxAdapterASIO@@8     10087758     asxasio.obj
 0002:0001f768       ??_R1A@?0A@EA@asxAdapterASIO@@8 10087768     asxasio.obj
 0002:0001f784       ??_R4asxSubSystemASIO@@6B@ 10087784     asxasio.obj
 0002:0001f798       ??_R3asxSubSystemASIO@@8   10087798     asxasio.obj
 0002:0001f7a8       ??_R2asxSubSystemASIO@@8   100877a8     asxasio.obj
 0002:0001f7b4       ??_R1A@?0A@EA@asxSubSystemASIO@@8 100877b4     asxasio.obj
 0002:0001f7d0       ??_R4asxMixerScannerASIO@@6B@ 100877d0     asxasio.obj
 0002:0001f7e4       ??_R3asxMixerScannerASIO@@8 100877e4     asxasio.obj
 0002:0001f7f4       ??_R2asxMixerScannerASIO@@8 100877f4     asxasio.obj
 0002:0001f800       ??_R1A@?0A@EA@asxMixerScannerASIO@@8 10087800     asxasio.obj
 0002:0001f81c       ??_R3asxControlBase@@8     1008781c     asxasioplay.obj
 0002:0001f82c       ??_R2asxControlBase@@8     1008782c     asxasioplay.obj
 0002:0001f838       ??_R1A@?0A@EA@asxControlBase@@8 10087838     asxasioplay.obj
 0002:0001f854       ??_R4asxPlayerASIO@@6B@    10087854     asxasioplay.obj
 0002:0001f868       ??_R3asxPlayerASIO@@8      10087868     asxasioplay.obj
 0002:0001f878       ??_R2asxPlayerASIO@@8      10087878     asxasioplay.obj
 0002:0001f88c       ??_R1A@?0A@EA@asxPlayerASIO@@8 1008788c     asxasioplay.obj
 0002:0001f8a8       ??_R1A@?0A@EA@asxPlayer@@8 100878a8     asxasioplay.obj
 0002:0001f8c4       ??_R3asxPlayer@@8          100878c4     asxasioplay.obj
 0002:0001f8d4       ??_R2asxPlayer@@8          100878d4     asxasioplay.obj
 0002:0001f8e4       ??_R4asxRecorderASIO@@6B@  100878e4     asxasiorec.obj
 0002:0001f8f8       ??_R3asxRecorderASIO@@8    100878f8     asxasiorec.obj
 0002:0001f908       ??_R2asxRecorderASIO@@8    10087908     asxasiorec.obj
 0002:0001f91c       ??_R1A@?0A@EA@asxRecorderASIO@@8 1008791c     asxasiorec.obj
 0002:0001f938       ??_R1A@?0A@EA@asxRecorder@@8 10087938     asxasiorec.obj
 0002:0001f954       ??_R3asxRecorder@@8        10087954     asxasiorec.obj
 0002:0001f964       ??_R2asxRecorder@@8        10087964     asxasiorec.obj
 0002:0001f974       ??_R4asxAdapter@@6B@       10087974     asxclass.obj
 0002:0001f988       ??_R4asxSystem@@6B@        10087988     asxclass.obj
 0002:0001f99c       ??_R3asxSystem@@8          1008799c     asxclass.obj
 0002:0001f9ac       ??_R2asxSystem@@8          100879ac     asxclass.obj
 0002:0001f9b8       ??_R1A@?0A@EA@asxSystem@@8 100879b8     asxclass.obj
 0002:0001f9d4       ??_R4asxSubSystem@@6B@     100879d4     asxclass.obj
 0002:0001f9e8       ??_R4asxMixer@@6B@         100879e8     asxclass.obj
 0002:0001f9fc       ??_R3asxMixer@@8           100879fc     asxclass.obj
 0002:0001fa0c       ??_R2asxMixer@@8           10087a0c     asxclass.obj
 0002:0001fa18       ??_R1A@?0A@EA@asxMixer@@8  10087a18     asxclass.obj
 0002:0001fa34       ??_R4asxNode@@6B@          10087a34     asxclass.obj
 0002:0001fa48       ??_R3asxNode@@8            10087a48     asxclass.obj
 0002:0001fa58       ??_R2asxNode@@8            10087a58     asxclass.obj
 0002:0001fa64       ??_R1A@?0A@EA@asxNode@@8   10087a64     asxclass.obj
 0002:0001fa80       ??_R4asxControlBase@@6B@   10087a80     asxclass.obj
 0002:0001fa94       ??_R4asxBase@@6B@          10087a94     asxclass.obj
 0002:0001faa8       ??_R4asxAbstractAdapter@@6B@ 10087aa8     asxclass.obj
 0002:0001fabc       ??_R3asxAbstractAdapter@@8 10087abc     asxclass.obj
 0002:0001facc       ??_R2asxAbstractAdapter@@8 10087acc     asxclass.obj
 0002:0001fadc       ??_R1A@?0A@EA@asxAbstractAdapter@@8 10087adc     asxclass.obj
 0002:0001faf8       ??_R4asxBlockProperty@@6B@ 10087af8     asxclass.obj
 0002:0001fb0c       ??_R3asxBlockProperty@@8   10087b0c     asxclass.obj
 0002:0001fb1c       ??_R2asxBlockProperty@@8   10087b1c     asxclass.obj
 0002:0001fb24       ??_R1A@?0A@EA@asxBlockProperty@@8 10087b24     asxclass.obj
 0002:0001fb40       ??_R4asxSubSystemDSND@@6B@ 10087b40     asxdsnd.obj
 0002:0001fb54       ??_R3asxSubSystemDSND@@8   10087b54     asxdsnd.obj
 0002:0001fb64       ??_R2asxSubSystemDSND@@8   10087b64     asxdsnd.obj
 0002:0001fb70       ??_R1A@?0A@EA@asxSubSystemDSND@@8 10087b70     asxdsnd.obj
 0002:0001fb8c       ??_R4asxAdapterDSND@@6B@   10087b8c     asxdsnd.obj
 0002:0001fba0       ??_R3asxAdapterDSND@@8     10087ba0     asxdsnd.obj
 0002:0001fbb0       ??_R2asxAdapterDSND@@8     10087bb0     asxdsnd.obj
 0002:0001fbc0       ??_R1A@?0A@EA@asxAdapterDSND@@8 10087bc0     asxdsnd.obj
 0002:0001fbdc       ??_R4asxMixerScannerDSND@@6B@ 10087bdc     asxdsnd.obj
 0002:0001fbf0       ??_R3asxMixerScannerDSND@@8 10087bf0     asxdsnd.obj
 0002:0001fc00       ??_R2asxMixerScannerDSND@@8 10087c00     asxdsnd.obj
 0002:0001fc0c       ??_R1A@?0A@EA@asxMixerScannerDSND@@8 10087c0c     asxdsnd.obj
 0002:0001fc28       ??_R4asxPlayerDSND@@6B@    10087c28     asxdsndplay.obj
 0002:0001fc3c       ??_R3asxPlayerDSND@@8      10087c3c     asxdsndplay.obj
 0002:0001fc4c       ??_R2asxPlayerDSND@@8      10087c4c     asxdsndplay.obj
 0002:0001fc60       ??_R1A@?0A@EA@asxPlayerDSND@@8 10087c60     asxdsndplay.obj
 0002:0001fc7c       ??_R4asxRecorderDSND@@6B@  10087c7c     asxdsndrec.obj
 0002:0001fc90       ??_R3asxRecorderDSND@@8    10087c90     asxdsndrec.obj
 0002:0001fca0       ??_R2asxRecorderDSND@@8    10087ca0     asxdsndrec.obj
 0002:0001fcb4       ??_R1A@?0A@EA@asxRecorderDSND@@8 10087cb4     asxdsndrec.obj
 0002:0001fcd0       ??_R4asxMeter@@6B@         10087cd0     asxhpi.obj
 0002:0001fce4       ??_R3asxMeter@@8           10087ce4     asxhpi.obj
 0002:0001fcf4       ??_R2asxMeter@@8           10087cf4     asxhpi.obj
 0002:0001fd04       ??_R1A@?0A@EA@asxMeter@@8  10087d04     asxhpi.obj
 0002:0001fd20       ??_R4asxVolume@@6B@        10087d20     asxhpi.obj
 0002:0001fd34       ??_R3asxVolume@@8          10087d34     asxhpi.obj
 0002:0001fd44       ??_R2asxVolume@@8          10087d44     asxhpi.obj
 0002:0001fd54       ??_R1A@?0A@EA@asxVolume@@8 10087d54     asxhpi.obj
 0002:0001fd70       ??_R4asxLevel@@6B@         10087d70     asxhpi.obj
 0002:0001fd84       ??_R3asxLevel@@8           10087d84     asxhpi.obj
 0002:0001fd94       ??_R2asxLevel@@8           10087d94     asxhpi.obj
 0002:0001fda4       ??_R1A@?0A@EA@asxLevel@@8  10087da4     asxhpi.obj
 0002:0001fdc0       ??_R4asxMux@@6B@           10087dc0     asxhpi.obj
 0002:0001fdd4       ??_R3asxMux@@8             10087dd4     asxhpi.obj
 0002:0001fde4       ??_R2asxMux@@8             10087de4     asxhpi.obj
 0002:0001fdf4       ??_R1A@?0A@EA@asxMux@@8    10087df4     asxhpi.obj
 0002:0001fe10       ??_R4asxMode@@6B@          10087e10     asxhpi.obj
 0002:0001fe24       ??_R3asxMode@@8            10087e24     asxhpi.obj
 0002:0001fe34       ??_R2asxMode@@8            10087e34     asxhpi.obj
 0002:0001fe44       ??_R1A@?0A@EA@asxMode@@8   10087e44     asxhpi.obj
 0002:0001fe60       ??_R4asxTuner@@6B@         10087e60     asxhpi.obj
 0002:0001fe74       ??_R3asxTuner@@8           10087e74     asxhpi.obj
 0002:0001fe84       ??_R2asxTuner@@8           10087e84     asxhpi.obj
 0002:0001fe94       ??_R1A@?0A@EA@asxTuner@@8  10087e94     asxhpi.obj
 0002:0001feb0       ??_R4asxPad@@6B@           10087eb0     asxhpi.obj
 0002:0001fec4       ??_R3asxPad@@8             10087ec4     asxhpi.obj
 0002:0001fed4       ??_R2asxPad@@8             10087ed4     asxhpi.obj
 0002:0001fee4       ??_R1A@?0A@EA@asxPad@@8    10087ee4     asxhpi.obj
 0002:0001ff00       ??_R4asxSampleClock@@6B@   10087f00     asxhpi.obj
 0002:0001ff14       ??_R3asxSampleClock@@8     10087f14     asxhpi.obj
 0002:0001ff24       ??_R2asxSampleClock@@8     10087f24     asxhpi.obj
 0002:0001ff34       ??_R1A@?0A@EA@asxSampleClock@@8 10087f34     asxhpi.obj
 0002:0001ff50       ??_R4asxAes3Tx@@6B@        10087f50     asxhpi.obj
 0002:0001ff64       ??_R3asxAes3Tx@@8          10087f64     asxhpi.obj
 0002:0001ff74       ??_R2asxAes3Tx@@8          10087f74     asxhpi.obj
 0002:0001ff84       ??_R1A@?0A@EA@asxAes3Tx@@8 10087f84     asxhpi.obj
 0002:0001ffa0       ??_R4asxAes3Rx@@6B@        10087fa0     asxhpi.obj
 0002:0001ffb4       ??_R3asxAes3Rx@@8          10087fb4     asxhpi.obj
 0002:0001ffc4       ??_R2asxAes3Rx@@8          10087fc4     asxhpi.obj
 0002:0001ffd4       ??_R1A@?0A@EA@asxAes3Rx@@8 10087fd4     asxhpi.obj
 0002:0001fff0       ??_R4asxGpio@@6B@          10087ff0     asxhpi.obj
 0002:00020004       ??_R3asxGpio@@8            10088004     asxhpi.obj
 0002:00020014       ??_R2asxGpio@@8            10088014     asxhpi.obj
 0002:00020024       ??_R1A@?0A@EA@asxGpio@@8   10088024     asxhpi.obj
 0002:00020040       ??_R4asxVox@@6B@           10088040     asxhpi.obj
 0002:00020054       ??_R3asxVox@@8             10088054     asxhpi.obj
 0002:00020064       ??_R2asxVox@@8             10088064     asxhpi.obj
 0002:00020074       ??_R1A@?0A@EA@asxVox@@8    10088074     asxhpi.obj
 0002:00020090       ??_R4asxBitStream@@6B@     10088090     asxhpi.obj
 0002:000200a4       ??_R3asxBitStream@@8       100880a4     asxhpi.obj
 0002:000200b4       ??_R2asxBitStream@@8       100880b4     asxhpi.obj
 0002:000200c4       ??_R1A@?0A@EA@asxBitStream@@8 100880c4     asxhpi.obj
 0002:000200e0       ??_R4asxMic@@6B@           100880e0     asxhpi.obj
 0002:000200f4       ??_R3asxMic@@8             100880f4     asxhpi.obj
 0002:00020104       ??_R2asxMic@@8             10088104     asxhpi.obj
 0002:00020114       ??_R1A@?0A@EA@asxMic@@8    10088114     asxhpi.obj
 0002:00020130       ??_R4asxParametricEQ@@6B@  10088130     asxhpi.obj
 0002:00020144       ??_R3asxParametricEQ@@8    10088144     asxhpi.obj
 0002:00020154       ??_R2asxParametricEQ@@8    10088154     asxhpi.obj
 0002:00020164       ??_R1A@?0A@EA@asxParametricEQ@@8 10088164     asxhpi.obj
 0002:00020180       ??_R4asxCompander@@6B@     10088180     asxhpi.obj
 0002:00020194       ??_R3asxCompander@@8       10088194     asxhpi.obj
 0002:000201a4       ??_R2asxCompander@@8       100881a4     asxhpi.obj
 0002:000201b4       ??_R1A@?0A@EA@asxCompander@@8 100881b4     asxhpi.obj
 0002:000201d0       ??_R4asxCobranet@@6B@      100881d0     asxhpi.obj
 0002:000201e4       ??_R3asxCobranet@@8        100881e4     asxhpi.obj
 0002:000201f4       ??_R2asxCobranet@@8        100881f4     asxhpi.obj
 0002:00020204       ??_R1A@?0A@EA@asxCobranet@@8 10088204     asxhpi.obj
 0002:00020220       ??_R4asxCobranetContainer@@6B@ 10088220     asxhpi.obj
 0002:00020234       ??_R3asxCobranetContainer@@8 10088234     asxhpi.obj
 0002:00020244       ??_R2asxCobranetContainer@@8 10088244     asxhpi.obj
 0002:00020258       ??_R1A@?0A@EA@asxCobranetContainer@@8 10088258     asxhpi.obj
 0002:00020274       ??_R4asxCobranetRx@@6B@    10088274     asxhpi.obj
 0002:00020288       ??_R3asxCobranetRx@@8      10088288     asxhpi.obj
 0002:00020298       ??_R2asxCobranetRx@@8      10088298     asxhpi.obj
 0002:000202a8       ??_R1A@?0A@EA@asxCobranetRx@@8 100882a8     asxhpi.obj
 0002:000202c4       ??_R4asxCobranetRxContainer@@6B@ 100882c4     asxhpi.obj
 0002:000202d8       ??_R3asxCobranetRxContainer@@8 100882d8     asxhpi.obj
 0002:000202e8       ??_R2asxCobranetRxContainer@@8 100882e8     asxhpi.obj
 0002:000202fc       ??_R1A@?0A@EA@asxCobranetRxContainer@@8 100882fc     asxhpi.obj
 0002:00020318       ??_R4asxCobranetTx@@6B@    10088318     asxhpi.obj
 0002:0002032c       ??_R3asxCobranetTx@@8      1008832c     asxhpi.obj
 0002:0002033c       ??_R2asxCobranetTx@@8      1008833c     asxhpi.obj
 0002:0002034c       ??_R1A@?0A@EA@asxCobranetTx@@8 1008834c     asxhpi.obj
 0002:00020368       ??_R4asxCobranetTxContainer@@6B@ 10088368     asxhpi.obj
 0002:0002037c       ??_R3asxCobranetTxContainer@@8 1008837c     asxhpi.obj
 0002:0002038c       ??_R2asxCobranetTxContainer@@8 1008838c     asxhpi.obj
 0002:000203a0       ??_R1A@?0A@EA@asxCobranetTxContainer@@8 100883a0     asxhpi.obj
 0002:000203bc       ??_R4asxToneDetector@@6B@  100883bc     asxhpi.obj
 0002:000203d0       ??_R3asxToneDetector@@8    100883d0     asxhpi.obj
 0002:000203e0       ??_R2asxToneDetector@@8    100883e0     asxhpi.obj
 0002:000203f0       ??_R1A@?0A@EA@asxToneDetector@@8 100883f0     asxhpi.obj
 0002:0002040c       ??_R4asxSilenceDetector@@6B@ 1008840c     asxhpi.obj
 0002:00020420       ??_R3asxSilenceDetector@@8 10088420     asxhpi.obj
 0002:00020430       ??_R2asxSilenceDetector@@8 10088430     asxhpi.obj
 0002:00020440       ??_R1A@?0A@EA@asxSilenceDetector@@8 10088440     asxhpi.obj
 0002:0002045c       ??_R4asxGenericControl@@6B@ 1008845c     asxhpi.obj
 0002:00020470       ??_R3asxGenericControl@@8  10088470     asxhpi.obj
 0002:00020480       ??_R2asxGenericControl@@8  10088480     asxhpi.obj
 0002:00020490       ??_R1A@?0A@EA@asxGenericControl@@8 10088490     asxhpi.obj
 0002:000204ac       ??_R4asxBlock@@6B@         100884ac     asxhpi.obj
 0002:000204c0       ??_R3asxBlock@@8           100884c0     asxhpi.obj
 0002:000204d0       ??_R2asxBlock@@8           100884d0     asxhpi.obj
 0002:000204e0       ??_R1A@?0A@EA@asxBlock@@8  100884e0     asxhpi.obj
 0002:000204fc       ??_R4asxSubSystemHPI@@6B@  100884fc     asxhpi.obj
 0002:00020510       ??_R3asxSubSystemHPI@@8    10088510     asxhpi.obj
 0002:00020520       ??_R2asxSubSystemHPI@@8    10088520     asxhpi.obj
 0002:0002052c       ??_R1A@?0A@EA@asxSubSystemHPI@@8 1008852c     asxhpi.obj
 0002:00020548       ??_R4asxAdapterHPI@@6B@    10088548     asxhpi.obj
 0002:0002055c       ??_R3asxAdapterHPI@@8      1008855c     asxhpi.obj
 0002:0002056c       ??_R2asxAdapterHPI@@8      1008856c     asxhpi.obj
 0002:0002057c       ??_R1A@?0A@EA@asxAdapterHPI@@8 1008857c     asxhpi.obj
 0002:00020598       ??_R4asxMixerScannerHPI@@6B@ 10088598     asxhpi.obj
 0002:000205ac       ??_R3asxMixerScannerHPI@@8 100885ac     asxhpi.obj
 0002:000205bc       ??_R2asxMixerScannerHPI@@8 100885bc     asxhpi.obj
 0002:000205c8       ??_R1A@?0A@EA@asxMixerScannerHPI@@8 100885c8     asxhpi.obj
 0002:000205e4       ??_R4asxAdapterHPIDuplicateIndex@@6B@ 100885e4     asxhpi.obj
 0002:000205f8       ??_R3asxAdapterHPIDuplicateIndex@@8 100885f8     asxhpi.obj
 0002:00020608       ??_R2asxAdapterHPIDuplicateIndex@@8 10088608     asxhpi.obj
 0002:00020618       ??_R1A@?0A@EA@asxAdapterHPIDuplicateIndex@@8 10088618     asxhpi.obj
 0002:00020634       ??_R4asxMixerScannerHPIDuplicateIndex@@6B@ 10088634     asxhpi.obj
 0002:00020648       ??_R3asxMixerScannerHPIDuplicateIndex@@8 10088648     asxhpi.obj
 0002:00020658       ??_R2asxMixerScannerHPIDuplicateIndex@@8 10088658     asxhpi.obj
 0002:00020664       ??_R1A@?0A@EA@asxMixerScannerHPIDuplicateIndex@@8 10088664     asxhpi.obj
 0002:00020680       ??_R4asxControlHPI@@6B@    10088680     asxhpi.obj
 0002:00020694       ??_R3asxControlHPI@@8      10088694     asxhpi.obj
 0002:000206a4       ??_R2asxControlHPI@@8      100886a4     asxhpi.obj
 0002:000206b8       ??_R1A@?0A@EA@asxControlHPI@@8 100886b8     asxhpi.obj
 0002:000206d4       ??_R1CI@?0A@EA@asxControlBaseHPI@@8 100886d4     asxhpi.obj
 0002:000206f0       ??_R3asxControlBaseHPI@@8  100886f0     asxhpi.obj
 0002:00020700       ??_R2asxControlBaseHPI@@8  10088700     asxhpi.obj
 0002:00020708       ??_R1A@?0A@EA@asxControlBaseHPI@@8 10088708     asxhpi.obj
 0002:00020724       ??_R4asxGenericHPI@@6B@    10088724     asxhpi.obj
 0002:00020738       ??_R3asxGenericHPI@@8      10088738     asxhpi.obj
 0002:00020748       ??_R2asxGenericHPI@@8      10088748     asxhpi.obj
 0002:00020760       ??_R1A@?0A@EA@asxGenericHPI@@8 10088760     asxhpi.obj
 0002:0002077c       ??_R1CM@?0A@EA@asxControlBaseHPI@@8 1008877c     asxhpi.obj
 0002:00020798       ??_R4asxVolumeHPI@@6B@     10088798     asxhpi.obj
 0002:000207ac       ??_R3asxVolumeHPI@@8       100887ac     asxhpi.obj
 0002:000207bc       ??_R2asxVolumeHPI@@8       100887bc     asxhpi.obj
 0002:000207d4       ??_R1A@?0A@EA@asxVolumeHPI@@8 100887d4     asxhpi.obj
 0002:000207f0       ??_R4asxLevelHPI@@6B@      100887f0     asxhpi.obj
 0002:00020804       ??_R3asxLevelHPI@@8        10088804     asxhpi.obj
 0002:00020814       ??_R2asxLevelHPI@@8        10088814     asxhpi.obj
 0002:0002082c       ??_R1A@?0A@EA@asxLevelHPI@@8 1008882c     asxhpi.obj
 0002:00020848       ??_R4asxMeterHPI@@6B@      10088848     asxhpi.obj
 0002:0002085c       ??_R3asxMeterHPI@@8        1008885c     asxhpi.obj
 0002:0002086c       ??_R2asxMeterHPI@@8        1008886c     asxhpi.obj
 0002:00020884       ??_R1A@?0A@EA@asxMeterHPI@@8 10088884     asxhpi.obj
 0002:000208a0       ??_R4asxMuxHPI@@6B@        100888a0     asxhpi.obj
 0002:000208b4       ??_R3asxMuxHPI@@8          100888b4     asxhpi.obj
 0002:000208c4       ??_R2asxMuxHPI@@8          100888c4     asxhpi.obj
 0002:000208dc       ??_R1A@?0A@EA@asxMuxHPI@@8 100888dc     asxhpi.obj
 0002:000208f8       ??_R1EA@?0A@EA@asxControlBaseHPI@@8 100888f8     asxhpi.obj
 0002:00020914       ??_R4asxModeHPI@@6B@       10088914     asxhpi.obj
 0002:00020928       ??_R3asxModeHPI@@8         10088928     asxhpi.obj
 0002:00020938       ??_R2asxModeHPI@@8         10088938     asxhpi.obj
 0002:00020950       ??_R1A@?0A@EA@asxModeHPI@@8 10088950     asxhpi.obj
 0002:0002096c       ??_R1DE@?0A@EA@asxControlBaseHPI@@8 1008896c     asxhpi.obj
 0002:00020988       ??_R4asxSampleClockHPI@@6B@ 10088988     asxhpi.obj
 0002:0002099c       ??_R3asxSampleClockHPI@@8  1008899c     asxhpi.obj
 0002:000209ac       ??_R2asxSampleClockHPI@@8  100889ac     asxhpi.obj
 0002:000209c4       ??_R1A@?0A@EA@asxSampleClockHPI@@8 100889c4     asxhpi.obj
 0002:000209e0       ??_R4asxTunerHPI@@6B@      100889e0     asxhpi.obj
 0002:000209f4       ??_R3asxTunerHPI@@8        100889f4     asxhpi.obj
 0002:00020a04       ??_R2asxTunerHPI@@8        10088a04     asxhpi.obj
 0002:00020a1c       ??_R1A@?0A@EA@asxTunerHPI@@8 10088a1c     asxhpi.obj
 0002:00020a38       ??_R4asxAes3TxHPI@@6B@     10088a38     asxhpi.obj
 0002:00020a4c       ??_R3asxAes3TxHPI@@8       10088a4c     asxhpi.obj
 0002:00020a5c       ??_R2asxAes3TxHPI@@8       10088a5c     asxhpi.obj
 0002:00020a74       ??_R1A@?0A@EA@asxAes3TxHPI@@8 10088a74     asxhpi.obj
 0002:00020a90       ??_R4asxAesebuReceiverHPI@@6B@ 10088a90     asxhpi.obj
 0002:00020aa4       ??_R3asxAesebuReceiverHPI@@8 10088aa4     asxhpi.obj
 0002:00020ab4       ??_R2asxAesebuReceiverHPI@@8 10088ab4     asxhpi.obj
 0002:00020acc       ??_R1A@?0A@EA@asxAesebuReceiverHPI@@8 10088acc     asxhpi.obj
 0002:00020ae8       ??_R4asxGpioHPI@@6B@       10088ae8     asxhpi.obj
 0002:00020afc       ??_R3asxGpioHPI@@8         10088afc     asxhpi.obj
 0002:00020b0c       ??_R2asxGpioHPI@@8         10088b0c     asxhpi.obj
 0002:00020b24       ??_R1A@?0A@EA@asxGpioHPI@@8 10088b24     asxhpi.obj
 0002:00020b40       ??_R1DA@?0A@EA@asxControlBaseHPI@@8 10088b40     asxhpi.obj
 0002:00020b5c       ??_R4asxVoxHPI@@6B@        10088b5c     asxhpi.obj
 0002:00020b70       ??_R3asxVoxHPI@@8          10088b70     asxhpi.obj
 0002:00020b80       ??_R2asxVoxHPI@@8          10088b80     asxhpi.obj
 0002:00020b98       ??_R1A@?0A@EA@asxVoxHPI@@8 10088b98     asxhpi.obj
 0002:00020bb4       ??_R4asxMicHPI@@6B@        10088bb4     asxhpi.obj
 0002:00020bc8       ??_R3asxMicHPI@@8          10088bc8     asxhpi.obj
 0002:00020bd8       ??_R2asxMicHPI@@8          10088bd8     asxhpi.obj
 0002:00020bf0       ??_R1A@?0A@EA@asxMicHPI@@8 10088bf0     asxhpi.obj
 0002:00020c0c       ??_R4asxParametricEqHPI@@6B@ 10088c0c     asxhpi.obj
 0002:00020c20       ??_R3asxParametricEqHPI@@8 10088c20     asxhpi.obj
 0002:00020c30       ??_R2asxParametricEqHPI@@8 10088c30     asxhpi.obj
 0002:00020c48       ??_R1A@?0A@EA@asxParametricEqHPI@@8 10088c48     asxhpi.obj
 0002:00020c64       ??_R4asxCompanderHPI@@6B@  10088c64     asxhpi.obj
 0002:00020c78       ??_R3asxCompanderHPI@@8    10088c78     asxhpi.obj
 0002:00020c88       ??_R2asxCompanderHPI@@8    10088c88     asxhpi.obj
 0002:00020ca0       ??_R1A@?0A@EA@asxCompanderHPI@@8 10088ca0     asxhpi.obj
 0002:00020cbc       ??_R4asxCompanderHPI_Legacy@@6B@ 10088cbc     asxhpi.obj
 0002:00020cd0       ??_R3asxCompanderHPI_Legacy@@8 10088cd0     asxhpi.obj
 0002:00020ce0       ??_R2asxCompanderHPI_Legacy@@8 10088ce0     asxhpi.obj
 0002:00020cf8       ??_R1A@?0A@EA@asxCompanderHPI_Legacy@@8 10088cf8     asxhpi.obj
 0002:00020d14       ??_R4asxCobranetHPI@@6B@   10088d14     asxhpi.obj
 0002:00020d28       ??_R3asxCobranetHPI@@8     10088d28     asxhpi.obj
 0002:00020d38       ??_R2asxCobranetHPI@@8     10088d38     asxhpi.obj
 0002:00020d50       ??_R1A@?0A@EA@asxCobranetHPI@@8 10088d50     asxhpi.obj
 0002:00020d6c       ??_R4asxCobranetRxHPI@@6B@ 10088d6c     asxhpi.obj
 0002:00020d80       ??_R3asxCobranetRxHPI@@8   10088d80     asxhpi.obj
 0002:00020d90       ??_R2asxCobranetRxHPI@@8   10088d90     asxhpi.obj
 0002:00020da8       ??_R1A@?0A@EA@asxCobranetRxHPI@@8 10088da8     asxhpi.obj
 0002:00020dc4       ??_R4asxCobranetTxHPI@@6B@ 10088dc4     asxhpi.obj
 0002:00020dd8       ??_R3asxCobranetTxHPI@@8   10088dd8     asxhpi.obj
 0002:00020de8       ??_R2asxCobranetTxHPI@@8   10088de8     asxhpi.obj
 0002:00020e00       ??_R1A@?0A@EA@asxCobranetTxHPI@@8 10088e00     asxhpi.obj
 0002:00020e1c       ??_R4asxToneDetectorHPI@@6B@ 10088e1c     asxhpi.obj
 0002:00020e30       ??_R3asxToneDetectorHPI@@8 10088e30     asxhpi.obj
 0002:00020e40       ??_R2asxToneDetectorHPI@@8 10088e40     asxhpi.obj
 0002:00020e58       ??_R1A@?0A@EA@asxToneDetectorHPI@@8 10088e58     asxhpi.obj
 0002:00020e74       ??_R4asxSilenceDetectorHPI@@6B@ 10088e74     asxhpi.obj
 0002:00020e88       ??_R3asxSilenceDetectorHPI@@8 10088e88     asxhpi.obj
 0002:00020e98       ??_R2asxSilenceDetectorHPI@@8 10088e98     asxhpi.obj
 0002:00020eb0       ??_R1A@?0A@EA@asxSilenceDetectorHPI@@8 10088eb0     asxhpi.obj
 0002:00020ecc       ??_R4asxPadHPI@@6B@        10088ecc     asxhpi.obj
 0002:00020ee0       ??_R3asxPadHPI@@8          10088ee0     asxhpi.obj
 0002:00020ef0       ??_R2asxPadHPI@@8          10088ef0     asxhpi.obj
 0002:00020f08       ??_R1A@?0A@EA@asxPadHPI@@8 10088f08     asxhpi.obj
 0002:00020f24       ??_R4asxBlockPropertyHPI@@6B@ 10088f24     asxhpi.obj
 0002:00020f38       ??_R3asxBlockPropertyHPI@@8 10088f38     asxhpi.obj
 0002:00020f48       ??_R2asxBlockPropertyHPI@@8 10088f48     asxhpi.obj
 0002:00020f58       ??_R1A@?0A@EA@asxBlockPropertyHPI@@8 10088f58     asxhpi.obj
 0002:00020f74       ??_R4asxBlockHPI@@6B@      10088f74     asxhpi.obj
 0002:00020f88       ??_R3asxBlockHPI@@8        10088f88     asxhpi.obj
 0002:00020f98       ??_R2asxBlockHPI@@8        10088f98     asxhpi.obj
 0002:00020fb0       ??_R1A@?0A@EA@asxBlockHPI@@8 10088fb0     asxhpi.obj
 0002:00020fcc       ??_R4asxPlayerHPI@@6B@     10088fcc     asxhpiplay.obj
 0002:00020fe0       ??_R3asxPlayerHPI@@8       10088fe0     asxhpiplay.obj
 0002:00020ff0       ??_R2asxPlayerHPI@@8       10088ff0     asxhpiplay.obj
 0002:00021004       ??_R1A@?0A@EA@asxPlayerHPI@@8 10089004     asxhpiplay.obj
 0002:00021020       ??_R4asxPlayerHPIWithInt@@6B@ 10089020     asxhpiplayi.obj
 0002:00021034       ??_R3asxPlayerHPIWithInt@@8 10089034     asxhpiplayi.obj
 0002:00021044       ??_R2asxPlayerHPIWithInt@@8 10089044     asxhpiplayi.obj
 0002:0002105c       ??_R1A@?0A@EA@asxPlayerHPIWithInt@@8 1008905c     asxhpiplayi.obj
 0002:00021078       ??_R4asxRecorderHPI@@6B@   10089078     asxhpirec.obj
 0002:0002108c       ??_R3asxRecorderHPI@@8     1008908c     asxhpirec.obj
 0002:0002109c       ??_R2asxRecorderHPI@@8     1008909c     asxhpirec.obj
 0002:000210b0       ??_R1A@?0A@EA@asxRecorderHPI@@8 100890b0     asxhpirec.obj
 0002:000210cc       ??_R4asxRecorderHPIWithInt@@6B@ 100890cc     asxhpireci.obj
 0002:000210e0       ??_R3asxRecorderHPIWithInt@@8 100890e0     asxhpireci.obj
 0002:000210f0       ??_R2asxRecorderHPIWithInt@@8 100890f0     asxhpireci.obj
 0002:00021108       ??_R1A@?0A@EA@asxRecorderHPIWithInt@@8 10089108     asxhpireci.obj
 0002:00021124       ??_R4asxCallbackObject@@6B@ 10089124     asxplay.obj
 0002:00021138       ??_R3asxCallbackObject@@8  10089138     asxplay.obj
 0002:00021148       ??_R2asxCallbackObject@@8  10089148     asxplay.obj
 0002:00021150       ??_R1A@?0A@EA@asxCallbackObject@@8 10089150     asxplay.obj
 0002:0002116c       ??_R4asxPlayer@@6B@        1008916c     asxplay.obj
 0002:00021180       ??_R4PlayerDoneCallback@@6B@ 10089180     asxplay.obj
 0002:00021194       ??_R3PlayerDoneCallback@@8 10089194     asxplay.obj
 0002:000211a4       ??_R2PlayerDoneCallback@@8 100891a4     asxplay.obj
 0002:000211b0       ??_R1A@?0A@EA@PlayerDoneCallback@@8 100891b0     asxplay.obj
 0002:000211cc       ??_R4asxRecorder@@6B@      100891cc     asxrec.obj
 0002:000211e0       ??_R4asxAdapterSNMP@@6B@   100891e0     asxsnmp.obj
 0002:000211f4       ??_R3asxAdapterSNMP@@8     100891f4     asxsnmp.obj
 0002:00021204       ??_R2asxAdapterSNMP@@8     10089204     asxsnmp.obj
 0002:00021214       ??_R1A@?0A@EA@asxAdapterSNMP@@8 10089214     asxsnmp.obj
 0002:00021230       ??_R4asxSubSystemSNMP@@6B@ 10089230     asxsnmp.obj
 0002:00021244       ??_R3asxSubSystemSNMP@@8   10089244     asxsnmp.obj
 0002:00021254       ??_R2asxSubSystemSNMP@@8   10089254     asxsnmp.obj
 0002:00021260       ??_R1A@?0A@EA@asxSubSystemSNMP@@8 10089260     asxsnmp.obj
 0002:0002127c       ??_R4asxMixerScannerSNMP@@6B@ 1008927c     asxsnmp.obj
 0002:00021290       ??_R3asxMixerScannerSNMP@@8 10089290     asxsnmp.obj
 0002:000212a0       ??_R2asxMixerScannerSNMP@@8 100892a0     asxsnmp.obj
 0002:000212ac       ??_R1A@?0A@EA@asxMixerScannerSNMP@@8 100892ac     asxsnmp.obj
 0002:000212c8       ??_R4asxCobranetSNMP@@6B@  100892c8     asxsnmp.obj
 0002:000212dc       ??_R3asxCobranetSNMP@@8    100892dc     asxsnmp.obj
 0002:000212ec       ??_R2asxCobranetSNMP@@8    100892ec     asxsnmp.obj
 0002:00021300       ??_R1A@?0A@EA@asxCobranetSNMP@@8 10089300     asxsnmp.obj
 0002:0002131c       ??_R4asxCobranetTxSNMP@@6B@ 1008931c     asxsnmp.obj
 0002:00021330       ??_R3asxCobranetTxSNMP@@8  10089330     asxsnmp.obj
 0002:00021340       ??_R2asxCobranetTxSNMP@@8  10089340     asxsnmp.obj
 0002:00021354       ??_R1A@?0A@EA@asxCobranetTxSNMP@@8 10089354     asxsnmp.obj
 0002:00021370       ??_R4asxCobranetRxSNMP@@6B@ 10089370     asxsnmp.obj
 0002:00021384       ??_R3asxCobranetRxSNMP@@8  10089384     asxsnmp.obj
 0002:00021394       ??_R2asxCobranetRxSNMP@@8  10089394     asxsnmp.obj
 0002:000213a8       ??_R1A@?0A@EA@asxCobranetRxSNMP@@8 100893a8     asxsnmp.obj
 0002:000213c4       ??_R4asxMixerScannerUnreachableSNMP@@6B@ 100893c4     asxsnmp.obj
 0002:000213d8       ??_R3asxMixerScannerUnreachableSNMP@@8 100893d8     asxsnmp.obj
 0002:000213e8       ??_R2asxMixerScannerUnreachableSNMP@@8 100893e8     asxsnmp.obj
 0002:000213f4       ??_R1A@?0A@EA@asxMixerScannerUnreachableSNMP@@8 100893f4     asxsnmp.obj
 0002:00021410       ??_R4asxCobranetUnreachableSNMP@@6B@ 10089410     asxsnmp.obj
 0002:00021424       ??_R3asxCobranetUnreachableSNMP@@8 10089424     asxsnmp.obj
 0002:00021434       ??_R2asxCobranetUnreachableSNMP@@8 10089434     asxsnmp.obj
 0002:00021448       ??_R1A@?0A@EA@asxCobranetUnreachableSNMP@@8 10089448     asxsnmp.obj
 0002:00021464       ??_R4asxLevelTR800@@6B@    10089464     asxtr800.obj
 0002:00021478       ??_R3asxLevelTR800@@8      10089478     asxtr800.obj
 0002:00021488       ??_R2asxLevelTR800@@8      10089488     asxtr800.obj
 0002:000214a0       ??_R1A@?0A@EA@asxLevelTR800@@8 100894a0     asxtr800.obj
 0002:000214bc       ??_R1CI@?0A@EA@asxControlBaseTR800@@8 100894bc     asxtr800.obj
 0002:000214d8       ??_R3asxControlBaseTR800@@8 100894d8     asxtr800.obj
 0002:000214e8       ??_R2asxControlBaseTR800@@8 100894e8     asxtr800.obj
 0002:000214f0       ??_R1A@?0A@EA@asxControlBaseTR800@@8 100894f0     asxtr800.obj
 0002:0002150c       ??_R4asxMeterTR800@@6B@    1008950c     asxtr800.obj
 0002:00021520       ??_R3asxMeterTR800@@8      10089520     asxtr800.obj
 0002:00021530       ??_R2asxMeterTR800@@8      10089530     asxtr800.obj
 0002:00021548       ??_R1A@?0A@EA@asxMeterTR800@@8 10089548     asxtr800.obj
 0002:00021564       ??_R4asxGpioTR800@@6B@     10089564     asxtr800.obj
 0002:00021578       ??_R3asxGpioTR800@@8       10089578     asxtr800.obj
 0002:00021588       ??_R2asxGpioTR800@@8       10089588     asxtr800.obj
 0002:000215a0       ??_R1A@?0A@EA@asxGpioTR800@@8 100895a0     asxtr800.obj
 0002:000215bc       ??_R1DA@?0A@EA@asxControlBaseTR800@@8 100895bc     asxtr800.obj
 0002:000215d8       ??_R4asxBlockTR800OptoMode@@6B@ 100895d8     asxtr800.obj
 0002:000215ec       ??_R3asxBlockTR800OptoMode@@8 100895ec     asxtr800.obj
 0002:000215fc       ??_R2asxBlockTR800OptoMode@@8 100895fc     asxtr800.obj
 0002:00021614       ??_R1A@?0A@EA@asxBlockTR800OptoMode@@8 10089614     asxtr800.obj
 0002:00021630       ??_R1DE@?0A@EA@asxControlBaseTR800@@8 10089630     asxtr800.obj
 0002:0002164c       ??_R4asxBlockTR800Status@@6B@ 1008964c     asxtr800.obj
 0002:00021660       ??_R3asxBlockTR800Status@@8 10089660     asxtr800.obj
 0002:00021670       ??_R2asxBlockTR800Status@@8 10089670     asxtr800.obj
 0002:00021684       ??_R1A@?0A@EA@asxBlockTR800Status@@8 10089684     asxtr800.obj
 0002:000216a0       ??_R4asxSubSystemWAVE@@6B@ 100896a0     asxwave.obj
 0002:000216b4       ??_R3asxSubSystemWAVE@@8   100896b4     asxwave.obj
 0002:000216c4       ??_R2asxSubSystemWAVE@@8   100896c4     asxwave.obj
 0002:000216d0       ??_R1A@?0A@EA@asxSubSystemWAVE@@8 100896d0     asxwave.obj
 0002:000216ec       ??_R4asxAdapterWAVE@@6B@   100896ec     asxwave.obj
 0002:00021700       ??_R3asxAdapterWAVE@@8     10089700     asxwave.obj
 0002:00021710       ??_R2asxAdapterWAVE@@8     10089710     asxwave.obj
 0002:00021720       ??_R1A@?0A@EA@asxAdapterWAVE@@8 10089720     asxwave.obj
 0002:0002173c       ??_R4asxMixerScannerWAVE@@6B@ 1008973c     asxwave.obj
 0002:00021750       ??_R3asxMixerScannerWAVE@@8 10089750     asxwave.obj
 0002:00021760       ??_R2asxMixerScannerWAVE@@8 10089760     asxwave.obj
 0002:0002176c       ??_R1A@?0A@EA@asxMixerScannerWAVE@@8 1008976c     asxwave.obj
 0002:00021788       ??_R4asxVolumeWAVE@@6B@    10089788     asxwave.obj
 0002:0002179c       ??_R3asxVolumeWAVE@@8      1008979c     asxwave.obj
 0002:000217ac       ??_R2asxVolumeWAVE@@8      100897ac     asxwave.obj
 0002:000217c0       ??_R1A@?0A@EA@asxVolumeWAVE@@8 100897c0     asxwave.obj
 0002:000217dc       ??_R4asxMeterWAVE@@6B@     100897dc     asxwave.obj
 0002:000217f0       ??_R3asxMeterWAVE@@8       100897f0     asxwave.obj
 0002:00021800       ??_R2asxMeterWAVE@@8       10089800     asxwave.obj
 0002:00021814       ??_R1A@?0A@EA@asxMeterWAVE@@8 10089814     asxwave.obj
 0002:00021830       ??_R4asxLevelWAVE@@6B@     10089830     asxwave.obj
 0002:00021844       ??_R3asxLevelWAVE@@8       10089844     asxwave.obj
 0002:00021854       ??_R2asxLevelWAVE@@8       10089854     asxwave.obj
 0002:00021868       ??_R1A@?0A@EA@asxLevelWAVE@@8 10089868     asxwave.obj
 0002:00021884       ??_R4asxMuxWAVE@@6B@       10089884     asxwave.obj
 0002:00021898       ??_R3asxMuxWAVE@@8         10089898     asxwave.obj
 0002:000218a8       ??_R2asxMuxWAVE@@8         100898a8     asxwave.obj
 0002:000218bc       ??_R1A@?0A@EA@asxMuxWAVE@@8 100898bc     asxwave.obj
 0002:000218d8       ??_R4asxModeWAVE@@6B@      100898d8     asxwave.obj
 0002:000218ec       ??_R3asxModeWAVE@@8        100898ec     asxwave.obj
 0002:000218fc       ??_R2asxModeWAVE@@8        100898fc     asxwave.obj
 0002:00021910       ??_R1A@?0A@EA@asxModeWAVE@@8 10089910     asxwave.obj
 0002:0002192c       ??_R4asxTunerWAVE@@6B@     1008992c     asxwave.obj
 0002:00021940       ??_R3asxTunerWAVE@@8       10089940     asxwave.obj
 0002:00021950       ??_R2asxTunerWAVE@@8       10089950     asxwave.obj
 0002:00021964       ??_R1A@?0A@EA@asxTunerWAVE@@8 10089964     asxwave.obj
 0002:00021980       ??_R4asxCobranetWAVE@@6B@  10089980     asxwave.obj
 0002:00021994       ??_R3asxCobranetWAVE@@8    10089994     asxwave.obj
 0002:000219a4       ??_R2asxCobranetWAVE@@8    100899a4     asxwave.obj
 0002:000219b8       ??_R1A@?0A@EA@asxCobranetWAVE@@8 100899b8     asxwave.obj
 0002:000219d4       ??_R4asxToneDetectorWAVE@@6B@ 100899d4     asxwave.obj
 0002:000219e8       ??_R3asxToneDetectorWAVE@@8 100899e8     asxwave.obj
 0002:000219f8       ??_R2asxToneDetectorWAVE@@8 100899f8     asxwave.obj
 0002:00021a0c       ??_R1A@?0A@EA@asxToneDetectorWAVE@@8 10089a0c     asxwave.obj
 0002:00021a28       ??_R4asxSilenceDetectorWAVE@@6B@ 10089a28     asxwave.obj
 0002:00021a3c       ??_R3asxSilenceDetectorWAVE@@8 10089a3c     asxwave.obj
 0002:00021a4c       ??_R2asxSilenceDetectorWAVE@@8 10089a4c     asxwave.obj
 0002:00021a60       ??_R1A@?0A@EA@asxSilenceDetectorWAVE@@8 10089a60     asxwave.obj
 0002:00021a7c       ??_R4asxPlayerWAVE@@6B@    10089a7c     asxwaveplay.obj
 0002:00021a90       ??_R3asxPlayerWAVE@@8      10089a90     asxwaveplay.obj
 0002:00021aa0       ??_R2asxPlayerWAVE@@8      10089aa0     asxwaveplay.obj
 0002:00021ab4       ??_R1A@?0A@EA@asxPlayerWAVE@@8 10089ab4     asxwaveplay.obj
 0002:00021ad0       ??_R4asxRecorderWAVE@@6B@  10089ad0     asxwaverec.obj
 0002:00021ae4       ??_R3asxRecorderWAVE@@8    10089ae4     asxwaverec.obj
 0002:00021af4       ??_R2asxRecorderWAVE@@8    10089af4     asxwaverec.obj
 0002:00021b08       ??_R1A@?0A@EA@asxRecorderWAVE@@8 10089b08     asxwaverec.obj
 0002:00021b24       ??_R4TWavFileBase@@6B@     10089b24     twavfile.obj
 0002:00021b38       ??_R3TWavFileBase@@8       10089b38     twavfile.obj
 0002:00021b48       ??_R2TWavFileBase@@8       10089b48     twavfile.obj
 0002:00021b54       ??_R1A@?0A@EA@TWavFileBase@@8 10089b54     twavfile.obj
 0002:00021b70       ??_R13?0A@EA@TWavFmt@@8    10089b70     twavfile.obj
 0002:00021b8c       ??_R3TWavFmt@@8            10089b8c     twavfile.obj
 0002:00021b9c       ??_R2TWavFmt@@8            10089b9c     twavfile.obj
 0002:00021ba4       ??_R1A@?0A@EA@TWavFmt@@8   10089ba4     twavfile.obj
 0002:00021bc0       ??_R4TWavFileTypeWav@@6B@  10089bc0     twavfile.obj
 0002:00021bd4       ??_R3TWavFileTypeWav@@8    10089bd4     twavfile.obj
 0002:00021be4       ??_R2TWavFileTypeWav@@8    10089be4     twavfile.obj
 0002:00021bf4       ??_R1A@?0A@EA@TWavFileTypeWav@@8 10089bf4     twavfile.obj
 0002:00021c10       ??_R4TWavFileTypeMP23@@6B@ 10089c10     twavfile.obj
 0002:00021c24       ??_R3TWavFileTypeMP23@@8   10089c24     twavfile.obj
 0002:00021c34       ??_R2TWavFileTypeMP23@@8   10089c34     twavfile.obj
 0002:00021c44       ??_R1A@?0A@EA@TWavFileTypeMP23@@8 10089c44     twavfile.obj
 0002:00021c60       ??_R4TWavFileTypeDAF@@6B@  10089c60     twavfile.obj
 0002:00021c74       ??_R3TWavFileTypeDAF@@8    10089c74     twavfile.obj
 0002:00021c84       ??_R2TWavFileTypeDAF@@8    10089c84     twavfile.obj
 0002:00021c94       ??_R1A@?0A@EA@TWavFileTypeDAF@@8 10089c94     twavfile.obj
 0002:00021cb0       ??_R4TWavFileTypeRaw@@6B@  10089cb0     twavfile.obj
 0002:00021cc4       ??_R3TWavFileTypeRaw@@8    10089cc4     twavfile.obj
 0002:00021cd4       ??_R2TWavFileTypeRaw@@8    10089cd4     twavfile.obj
 0002:00021ce4       ??_R1A@?0A@EA@TWavFileTypeRaw@@8 10089ce4     twavfile.obj
 0002:00021d00       ??_R4TWavFileTypeNullRecord@@6B@ 10089d00     twavfile.obj
 0002:00021d14       ??_R3TWavFileTypeNullRecord@@8 10089d14     twavfile.obj
 0002:00021d24       ??_R2TWavFileTypeNullRecord@@8 10089d24     twavfile.obj
 0002:00021d34       ??_R1A@?0A@EA@TWavFileTypeNullRecord@@8 10089d34     twavfile.obj
 0002:00021d50       ??_R4TWavFileTypeGenerator@@6B@ 10089d50     twavfile.obj
 0002:00021d64       ??_R3TWavFileTypeGenerator@@8 10089d64     twavfile.obj
 0002:00021d74       ??_R2TWavFileTypeGenerator@@8 10089d74     twavfile.obj
 0002:00021d84       ??_R1A@?0A@EA@TWavFileTypeGenerator@@8 10089d84     twavfile.obj
 0002:00021da0       ??_R4TWavFileWithFifo@@6B@ 10089da0     twavfilefifo.obj
 0002:00021db4       ??_R3TWavFileWithFifo@@8   10089db4     twavfilefifo.obj
 0002:00021dc4       ??_R2TWavFileWithFifo@@8   10089dc4     twavfilefifo.obj
 0002:00021dd4       ??_R1A@?0A@EA@TWavFileWithFifo@@8 10089dd4     twavfilefifo.obj
 0002:00021df0       ??_R1A@?0A@EA@exception@std@@8 10089df0     LIBCMT:new.obj
 0002:00021e0c       ??_R3exception@std@@8      10089e0c     LIBCMT:new.obj
 0002:00021e1c       ??_R2exception@std@@8      10089e1c     LIBCMT:new.obj
 0002:00021e24       ??_R4bad_alloc@std@@6B@    10089e24     LIBCMT:new.obj
 0002:00021e38       ??_R3bad_alloc@std@@8      10089e38     LIBCMT:new.obj
 0002:00021e48       ??_R2bad_alloc@std@@8      10089e48     LIBCMT:new.obj
 0002:00021e54       ??_R1A@?0A@EA@bad_alloc@std@@8 10089e54     LIBCMT:new.obj
 0002:00021e70       ??_R4type_info@@6B@        10089e70     LIBCMT:typinfo.obj
 0002:00021e84       ??_R3type_info@@8          10089e84     LIBCMT:typinfo.obj
 0002:00021e94       ??_R2type_info@@8          10089e94     LIBCMT:typinfo.obj
 0002:00021e9c       ??_R1A@?0A@EA@type_info@@8 10089e9c     LIBCMT:typinfo.obj
 0002:00021eb8       ??_R4exception@std@@6B@    10089eb8     LIBCMT:stdexcpt.obj
 0002:00021ecc       ??_R4bad_cast@std@@6B@     10089ecc     LIBCMT:stdexcpt.obj
 0002:00021ee0       ??_R3bad_cast@std@@8       10089ee0     LIBCMT:stdexcpt.obj
 0002:00021ef0       ??_R2bad_cast@std@@8       10089ef0     LIBCMT:stdexcpt.obj
 0002:00021efc       ??_R1A@?0A@EA@bad_cast@std@@8 10089efc     LIBCMT:stdexcpt.obj
 0002:00021f18       ??_R4bad_typeid@std@@6B@   10089f18     LIBCMT:stdexcpt.obj
 0002:00021f2c       ??_R3bad_typeid@std@@8     10089f2c     LIBCMT:stdexcpt.obj
 0002:00021f3c       ??_R2bad_typeid@std@@8     10089f3c     LIBCMT:stdexcpt.obj
 0002:00021f48       ??_R1A@?0A@EA@bad_typeid@std@@8 10089f48     LIBCMT:stdexcpt.obj
 0002:00021f64       ??_R4__non_rtti_object@std@@6B@ 10089f64     LIBCMT:stdexcpt.obj
 0002:00021f78       ??_R3__non_rtti_object@std@@8 10089f78     LIBCMT:stdexcpt.obj
 0002:00021f88       ??_R2__non_rtti_object@std@@8 10089f88     LIBCMT:stdexcpt.obj
 0002:00021f98       ??_R1A@?0A@EA@__non_rtti_object@std@@8 10089f98     LIBCMT:stdexcpt.obj
 0002:00021fb4       ??_R4bad_exception@std@@6B@ 10089fb4     LIBCMT:frame.obj
 0002:00021fc8       ??_R3bad_exception@std@@8  10089fc8     LIBCMT:frame.obj
 0002:00021fd8       ??_R2bad_exception@std@@8  10089fd8     LIBCMT:frame.obj
 0002:00021fe4       ??_R1A@?0A@EA@bad_exception@std@@8 10089fe4     LIBCMT:frame.obj
 0002:00022000       ??_R4DNameNode@@6B@        1008a000     LIBCMT:undname.obj
 0002:00022014       ??_R3DNameNode@@8          1008a014     LIBCMT:undname.obj
 0002:00022024       ??_R2DNameNode@@8          1008a024     LIBCMT:undname.obj
 0002:0002202c       ??_R1A@?0A@EA@DNameNode@@8 1008a02c     LIBCMT:undname.obj
 0002:00022048       ??_R4charNode@@6B@         1008a048     LIBCMT:undname.obj
 0002:0002205c       ??_R3charNode@@8           1008a05c     LIBCMT:undname.obj
 0002:0002206c       ??_R2charNode@@8           1008a06c     LIBCMT:undname.obj
 0002:00022078       ??_R1A@?0A@EA@charNode@@8  1008a078     LIBCMT:undname.obj
 0002:00022094       ??_R4pcharNode@@6B@        1008a094     LIBCMT:undname.obj
 0002:000220a8       ??_R3pcharNode@@8          1008a0a8     LIBCMT:undname.obj
 0002:000220b8       ??_R2pcharNode@@8          1008a0b8     LIBCMT:undname.obj
 0002:000220c4       ??_R1A@?0A@EA@pcharNode@@8 1008a0c4     LIBCMT:undname.obj
 0002:000220e0       ??_R4pDNameNode@@6B@       1008a0e0     LIBCMT:undname.obj
 0002:000220f4       ??_R3pDNameNode@@8         1008a0f4     LIBCMT:undname.obj
 0002:00022104       ??_R2pDNameNode@@8         1008a104     LIBCMT:undname.obj
 0002:00022110       ??_R1A@?0A@EA@pDNameNode@@8 1008a110     LIBCMT:undname.obj
 0002:0002212c       ??_R4DNameStatusNode@@6B@  1008a12c     LIBCMT:undname.obj
 0002:00022140       ??_R3DNameStatusNode@@8    1008a140     LIBCMT:undname.obj
 0002:00022150       ??_R2DNameStatusNode@@8    1008a150     LIBCMT:undname.obj
 0002:0002215c       ??_R1A@?0A@EA@DNameStatusNode@@8 1008a15c     LIBCMT:undname.obj
 0002:00022178       ??_R4pairNode@@6B@         1008a178     LIBCMT:undname.obj
 0002:0002218c       ??_R3pairNode@@8           1008a18c     LIBCMT:undname.obj
 0002:0002219c       ??_R2pairNode@@8           1008a19c     LIBCMT:undname.obj
 0002:000221a8       ??_R1A@?0A@EA@pairNode@@8  1008a1a8     LIBCMT:undname.obj
 0002:000221c4       ??_R4logic_error@std@@6B@  1008a1c4     libcpmt:xthrow.obj
 0002:000221d8       ??_R3logic_error@std@@8    1008a1d8     libcpmt:xthrow.obj
 0002:000221e8       ??_R2logic_error@std@@8    1008a1e8     libcpmt:xthrow.obj
 0002:000221f4       ??_R1A@?0A@EA@logic_error@std@@8 1008a1f4     libcpmt:xthrow.obj
 0002:00022210       ??_R4invalid_argument@std@@6B@ 1008a210     libcpmt:xthrow.obj
 0002:00022224       ??_R3invalid_argument@std@@8 1008a224     libcpmt:xthrow.obj
 0002:00022234       ??_R2invalid_argument@std@@8 1008a234     libcpmt:xthrow.obj
 0002:00022244       ??_R1A@?0A@EA@invalid_argument@std@@8 1008a244     libcpmt:xthrow.obj
 0002:00022260       ??_R4length_error@std@@6B@ 1008a260     libcpmt:xthrow.obj
 0002:00022274       ??_R3length_error@std@@8   1008a274     libcpmt:xthrow.obj
 0002:00022284       ??_R2length_error@std@@8   1008a284     libcpmt:xthrow.obj
 0002:00022294       ??_R1A@?0A@EA@length_error@std@@8 1008a294     libcpmt:xthrow.obj
 0002:000222b0       ??_R4out_of_range@std@@6B@ 1008a2b0     libcpmt:xthrow.obj
 0002:000222c4       ??_R3out_of_range@std@@8   1008a2c4     libcpmt:xthrow.obj
 0002:000222d4       ??_R2out_of_range@std@@8   1008a2d4     libcpmt:xthrow.obj
 0002:000222e4       ??_R1A@?0A@EA@out_of_range@std@@8 1008a2e4     libcpmt:xthrow.obj
 0002:00022300       ??_R4runtime_error@std@@6B@ 1008a300     libcpmt:xthrow.obj
 0002:00022314       ??_R3runtime_error@std@@8  1008a314     libcpmt:xthrow.obj
 0002:00022324       ??_R2runtime_error@std@@8  1008a324     libcpmt:xthrow.obj
 0002:00022330       ??_R1A@?0A@EA@runtime_error@std@@8 1008a330     libcpmt:xthrow.obj
 0002:0002234c       ??_R4overflow_error@std@@6B@ 1008a34c     libcpmt:xthrow.obj
 0002:00022360       ??_R3overflow_error@std@@8 1008a360     libcpmt:xthrow.obj
 0002:00022370       ??_R2overflow_error@std@@8 1008a370     libcpmt:xthrow.obj
 0002:00022380       ??_R1A@?0A@EA@overflow_error@std@@8 1008a380     libcpmt:xthrow.obj
 0002:0002239c       ??_R4bad_function_call@std@@6B@ 1008a39c     libcpmt:xthrow.obj
 0002:000223b0       ??_R3bad_function_call@std@@8 1008a3b0     libcpmt:xthrow.obj
 0002:000223c0       ??_R2bad_function_call@std@@8 1008a3c0     libcpmt:xthrow.obj
 0002:000223cc       ??_R1A@?0A@EA@bad_function_call@std@@8 1008a3cc     libcpmt:xthrow.obj
 0002:000223e8       ??_R4regex_error@std@@6B@  1008a3e8     libcpmt:xthrow.obj
 0002:000223fc       ??_R3regex_error@std@@8    1008a3fc     libcpmt:xthrow.obj
 0002:0002240c       ??_R2regex_error@std@@8    1008a40c     libcpmt:xthrow.obj
 0002:0002241c       ??_R1A@?0A@EA@regex_error@std@@8 1008a41c     libcpmt:xthrow.obj
 0002:00022440       ___safe_se_handler_table   1008a440     <linker-defined>
 0002:0002266c       ___rtc_iaa                 1008a66c     LIBCMT:initsect.obj
 0002:00022670       ___rtc_izz                 1008a670     LIBCMT:initsect.obj
 0002:00022674       ___rtc_taa                 1008a674     LIBCMT:initsect.obj
 0002:00022678       ___rtc_tzz                 1008a678     LIBCMT:initsect.obj
 0002:000242ec       __TI2?AVbad_alloc@std@@    1008c2ec     LIBCMT:new.obj
 0002:000242fc       __CTA2?AVbad_alloc@std@@   1008c2fc     LIBCMT:new.obj
 0002:00024308       __CT??_R0?AVbad_alloc@std@@@8??0bad_alloc@std@@QAE@ABV01@@Z12 1008c308     LIBCMT:new.obj
 0002:00024324       __CT??_R0?AVexception@std@@@8??0exception@std@@QAE@ABV01@@Z12 1008c324     LIBCMT:new.obj
 0002:000243bc       __TI3?AV__non_rtti_object@std@@ 1008c3bc     LIBCMT:rtti.obj
 0002:000243cc       __CTA3?AV__non_rtti_object@std@@ 1008c3cc     LIBCMT:rtti.obj
 0002:000243dc       __CT??_R0?AV__non_rtti_object@std@@@8??0__non_rtti_object@std@@QAE@ABV01@@Z12 1008c3dc     LIBCMT:rtti.obj
 0002:000243f8       __CT??_R0?AVbad_typeid@std@@@8??0bad_typeid@std@@QAE@ABV01@@Z12 1008c3f8     LIBCMT:rtti.obj
 0002:00024414       __TI2?AVbad_typeid@std@@   1008c414     LIBCMT:rtti.obj
 0002:00024424       __CTA2?AVbad_typeid@std@@  1008c424     LIBCMT:rtti.obj
 0002:00024430       __TI2?AVbad_cast@std@@     1008c430     LIBCMT:rtti.obj
 0002:00024440       __CTA2?AVbad_cast@std@@    1008c440     LIBCMT:rtti.obj
 0002:0002444c       __CT??_R0?AVbad_cast@std@@@8??0bad_cast@std@@QAE@ABV01@@Z12 1008c44c     LIBCMT:rtti.obj
 0002:00024944       __TI2?AVbad_exception@std@@ 1008c944     LIBCMT:frame.obj
 0002:00024954       __CTA2?AVbad_exception@std@@ 1008c954     LIBCMT:frame.obj
 0002:00024960       __CT??_R0?AVbad_exception@std@@@8??0bad_exception@std@@QAE@ABV01@@Z12 1008c960     LIBCMT:frame.obj
 0002:00024d0c       __TI3?AVinvalid_argument@std@@ 1008cd0c     libcpmt:xthrow.obj
 0002:00024d1c       __CTA3?AVinvalid_argument@std@@ 1008cd1c     libcpmt:xthrow.obj
 0002:00024d2c       __CT??_R0?AVinvalid_argument@std@@@8??0invalid_argument@std@@QAE@ABV01@@Z12 1008cd2c     libcpmt:xthrow.obj
 0002:00024d48       __CT??_R0?AVlogic_error@std@@@8??0logic_error@std@@QAE@ABV01@@Z12 1008cd48     libcpmt:xthrow.obj
 0002:00024d64       __TI3?AVlength_error@std@@ 1008cd64     libcpmt:xthrow.obj
 0002:00024d74       __CTA3?AVlength_error@std@@ 1008cd74     libcpmt:xthrow.obj
 0002:00024d84       __CT??_R0?AVlength_error@std@@@8??0length_error@std@@QAE@ABV01@@Z12 1008cd84     libcpmt:xthrow.obj
 0002:00024da0       __TI3?AVout_of_range@std@@ 1008cda0     libcpmt:xthrow.obj
 0002:00024db0       __CTA3?AVout_of_range@std@@ 1008cdb0     libcpmt:xthrow.obj
 0002:00024dc0       __CT??_R0?AVout_of_range@std@@@8??0out_of_range@std@@QAE@ABV01@@Z12 1008cdc0     libcpmt:xthrow.obj
 0002:00024ddc       __TI3?AVoverflow_error@std@@ 1008cddc     libcpmt:xthrow.obj
 0002:00024dec       __CTA3?AVoverflow_error@std@@ 1008cdec     libcpmt:xthrow.obj
 0002:00024dfc       __CT??_R0?AVoverflow_error@std@@@8??0overflow_error@std@@QAE@ABV01@@Z12 1008cdfc     libcpmt:xthrow.obj
 0002:00024e18       __CT??_R0?AVruntime_error@std@@@8??0runtime_error@std@@QAE@ABV01@@Z12 1008ce18     libcpmt:xthrow.obj
 0002:00024e34       __TI2?AVruntime_error@std@@ 1008ce34     libcpmt:xthrow.obj
 0002:00024e44       __CTA2?AVruntime_error@std@@ 1008ce44     libcpmt:xthrow.obj
 0002:00024e50       __TI2?AVbad_function_call@std@@ 1008ce50     libcpmt:xthrow.obj
 0002:00024e60       __CTA2?AVbad_function_call@std@@ 1008ce60     libcpmt:xthrow.obj
 0002:00024e6c       __CT??_R0?AVbad_function_call@std@@@8??0bad_function_call@std@@QAE@ABV01@@Z12 1008ce6c     libcpmt:xthrow.obj
 0002:00024e88       __TI3?AVregex_error@std@@  1008ce88     libcpmt:xthrow.obj
 0002:00024e98       __CTA3?AVregex_error@std@@ 1008ce98     libcpmt:xthrow.obj
 0002:00024ea8       __CT??_R0?AVregex_error@std@@@8??0regex_error@std@@QAE@ABV01@@Z16 1008cea8     libcpmt:xthrow.obj
 0002:00024ec4       __DELAY_IMPORT_DESCRIPTOR_avdecc_lib_controller32_dll 1008cec4     avdecc-lib_controller32:avdecc-lib_controller32.dll
 0002:00024ee4       __NULL_DELAY_IMPORT_DESCRIPTOR 1008cee4     avdecc-lib_controller32:avdecc-lib_controller32.dll
 0002:00024f28       \177avdecc-lib_controller32_NULL_THUNK_DATA_DLN 1008cf28     avdecc-lib_controller32:avdecc-lib_controller32.dll
 0002:000250d4       \177avdecc-lib_controller32_NULL_THUNK_DATA_DLB 1008d0d4     avdecc-lib_controller32:avdecc-lib_controller32.dll
 0002:0002787c       __IMPORT_DESCRIPTOR_WINMM  1008f87c     winmm:WINMM.dll
 0002:00027890       __IMPORT_DESCRIPTOR_ASIHPI32 1008f890     asihpi32:ASIHPI32.dll
 0002:000278a4       __IMPORT_DESCRIPTOR_wsnmp32 1008f8a4     wsnmp32:wsnmp32.dll
 0002:000278b8       __IMPORT_DESCRIPTOR_WSOCK32 1008f8b8     wsock32:WSOCK32.dll
 0002:000278cc       __IMPORT_DESCRIPTOR_DSOUND 1008f8cc     dsound:DSOUND.dll
 0002:000278e0       __IMPORT_DESCRIPTOR_KERNEL32 1008f8e0     kernel32:KERNEL32.dll
 0002:000278f4       __IMPORT_DESCRIPTOR_USER32 1008f8f4     user32:USER32.dll
 0002:00027908       __IMPORT_DESCRIPTOR_ADVAPI32 1008f908     advapi32:ADVAPI32.dll
 0002:0002791c       __IMPORT_DESCRIPTOR_ole32  1008f91c     ole32:ole32.dll
 0002:00027930       __NULL_IMPORT_DESCRIPTOR   1008f930     winmm:WINMM.dll
 0003:00000000       ?import_table@@3PAUtable_entry@@A 10093000     asicndload.obj
 0003:00000088       ?notification_id@@3HA      10093088     asxavdecc.obj
 0003:0000008c       ?_Generic_object@?$_Error_objects@H@std@@2V_Generic_error_category@2@A 1009308c     asxavdecc.obj
 0003:00000090       ?_Iostream_object@?$_Error_objects@H@std@@2V_Iostream_error_category@2@A 10093090     asxavdecc.obj
 0003:00000094       ?_System_object@?$_Error_objects@H@std@@2V_System_error_category@2@A 10093094     asxavdecc.obj
 0003:00000098       ?callbacks@@3UASIOCallbacks@@A 10093098     asxasio.obj
 0003:00000228       _aTranslationTable         10093228     asxstring.obj
 0003:000022c8       ?receiverFields@CobraNetNode@@0PAUasiCNdev_FieldEntry_@@A 100952c8     cobranet.obj
 0003:000023c4       ?ipField@CobraNetNode@@0UasiCNdev_FieldEntry_@@A 100953c4     cobranet.obj
 0003:000023e0       ?transmitterFields@CobraNetNode@@0PAUasiCNdev_FieldEntry_@@A 100953e0     cobranet.obj
 0003:000024f8       ?nodeFields@CobraNetNode@@0PAUasiCNdev_FieldEntry_@@A 100954f8     cobranet.obj
 0003:00002760       ?audioFields@CobraNetNode@@0PAUasiCNdev_FieldEntry_@@A 10095760     cobranet.obj
 0003:0000277c       ?stdUserFields@CobraNetNode@@0PAUasiCNdev_FieldEntry_@@A 1009577c     cobranet.obj
 0003:00002798       ?firmwareMfgId_OID@@3PAIA  10095798     mibtbl.obj
 0003:000027a0       ?firmwareMfgProductId_OID@@3PAIA 100957a0     mibtbl.obj
 0003:000027a8       ?firmwareMfgVersion_OID@@3PAIA 100957a8     mibtbl.obj
 0003:000027b0       ?firmwareRestart_OID@@3PAIA 100957b0     mibtbl.obj
 0003:000027b8       ?firmwareUnknown1_OID@@3PAIA 100957b8     mibtbl.obj
 0003:000027c0       ?firmwareUnknown2_OID@@3PAIA 100957c0     mibtbl.obj
 0003:000027c8       ?firmwareUnknown3_OID@@3PAIA 100957c8     mibtbl.obj
 0003:000027d0       ?flashOID@@3PAIA           100957d0     mibtbl.obj
 0003:000027f8       ?flashTotalSize_OID@@3PAIA 100957f8     mibtbl.obj
 0003:00002800       ?flashSectorSize_OID@@3PAIA 10095800     mibtbl.obj
 0003:00002808       ?flashPersistSequence_OID@@3PAIA 10095808     mibtbl.obj
 0003:00002810       ?flashPersistType_OID@@3PAIA 10095810     mibtbl.obj
 0003:00002818       ?flashPersistSize_OID@@3PAIA 10095818     mibtbl.obj
 0003:00002820       ?flashPersistStores_OID@@3PAIA 10095820     mibtbl.obj
 0003:00002828       ?flashPersistEnable_OID@@3PAIA 10095828     mibtbl.obj
 0003:00002830       ?flashPersistAck_OID@@3PAIA 10095830     mibtbl.obj
 0003:00002838       ?errorOID@@3PAIA           10095838     mibtbl.obj
 0003:00002860       ?errorPOST_OID@@3PAIA      10095860     mibtbl.obj
 0003:00002868       ?errorImage_OID@@3PAIA     10095868     mibtbl.obj
 0003:00002870       ?errorLast_OID@@3PAIA      10095870     mibtbl.obj
 0003:00002878       ?errorCount_OID@@3PAIA     10095878     mibtbl.obj
 0003:00002880       ?errorDisplay_OID@@3PAIA   10095880     mibtbl.obj
 0003:00002888       ?modeOID@@3PAIA            10095888     mibtbl.obj
 0003:000028b4       ?modeRateControl_OID@@3PAIA 100958b4     mibtbl.obj
 0003:000028bc       ?modeRateStatus_OID@@3PAIA 100958bc     mibtbl.obj
 0003:000028c4       ?conductorOID@@3PAIA       100958c4     mibtbl.obj
 0003:000028ec       ?conductorRate_OID@@3PAIA  100958ec     mibtbl.obj
 0003:000028f4       ?conductorPriority_OID@@3PAIA 100958f4     mibtbl.obj
 0003:000028fc       ?conductorGap_OID@@3PAIA   100958fc     mibtbl.obj
 0003:00002904       ?conductorStatus_OID@@3PAIA 10095904     mibtbl.obj
 0003:0000290c       ?conductorUpTime_OID@@3PAIA 1009590c     mibtbl.obj
 0003:00002914       ?conductorMacAddress_OID@@3PAIA 10095914     mibtbl.obj
 0003:0000291c       ?conductorCurrentFrame_OID@@3PAIA 1009591c     mibtbl.obj
 0003:00002924       ?conductorCycleRate_OID@@3PAIA 10095924     mibtbl.obj
 0003:0000292c       ?conductorIsoChannelCount_OID@@3PAIA 1009592c     mibtbl.obj
 0003:00002934       ?audioOID@@3PAIA           10095934     mibtbl.obj
 0003:0000295c       ?audioMeterDropouts_OID@@3PAIA 1009595c     mibtbl.obj
 0003:00002964       ?audioMeterMapIndex_OID@@3PAIA 10095964     mibtbl.obj
 0003:00002970       ?audioMeterMap_OID@@3PAIA  10095970     mibtbl.obj
 0003:0000297c       ?audioMeterPeaks_OID@@3PAIA 1009597c     mibtbl.obj
 0003:00002988       ?audioMeters_OID@@3PAIA    10095988     mibtbl.obj
 0003:00002994       ?audioMap_OID@@3PAIA       10095994     mibtbl.obj
 0003:000029a0       ?audioLoopIndex_OID@@3PAIA 100959a0     mibtbl.obj
 0003:000029ac       ?audioLoopSrc_OID@@3PAIA   100959ac     mibtbl.obj
 0003:000029b8       ?audioLoopDst_OID@@3PAIA   100959b8     mibtbl.obj
 0003:000029c4       ?audioOutputIndex_OID@@3PAIA 100959c4     mibtbl.obj
 0003:000029d0       ?audioOutput_OID@@3PAIA    100959d0     mibtbl.obj
 0003:000029dc       ?audioMeterDecay_OID@@3PAIA 100959dc     mibtbl.obj
 0003:000029e4       ?audioAllowedChannels_OID@@3PAIA 100959e4     mibtbl.obj
 0003:000029ec       ?audioTxChannels_OID@@3PAIA 100959ec     mibtbl.obj
 0003:000029f4       ?audioRxChannels_OID@@3PAIA 100959f4     mibtbl.obj
 0003:000029fc       ?audioDupIndex_OID@@3PAIA  100959fc     mibtbl.obj
 0003:00002a08       ?audioDupSrc_OID@@3PAIA    10095a08     mibtbl.obj
 0003:00002a14       ?audioDupDst_OID@@3PAIA    10095a14     mibtbl.obj
 0003:00002a20       ?audioMeterPeaksRaw_OID@@3PAIA 10095a20     mibtbl.obj
 0003:00002a28       ?audioMetersRaw_OID@@3PAIA 10095a28     mibtbl.obj
 0003:00002a30       ?audioUnknown12_OID@@3PAIA 10095a30     mibtbl.obj
 0003:00002a38       ?rxOID@@3PAIA              10095a38     mibtbl.obj
 0003:00002a60       ?rxIndex_OID@@3PAIA        10095a60     mibtbl.obj
 0003:00002a6c       ?rxBundle_OID@@3PAIA       10095a6c     mibtbl.obj
 0003:00002a78       ?rxSourceMAC_OID@@3PAIA    10095a78     mibtbl.obj
 0003:00002a84       ?rxPriority_OID@@3PAIA     10095a84     mibtbl.obj
 0003:00002a90       ?rxBuddyExclude_OID@@3PAIA 10095a90     mibtbl.obj
 0003:00002a9c       ?rxStatus_OID@@3PAIA       10095a9c     mibtbl.obj
 0003:00002aa8       ?rxDropouts_OID@@3PAIA     10095aa8     mibtbl.obj
 0003:00002ab4       ?rxDelay_OID@@3PAIA        10095ab4     mibtbl.obj
 0003:00002ac0       ?rxMinDelay_OID@@3PAIA     10095ac0     mibtbl.obj
 0003:00002acc       ?rxSubChannelIndex_OID@@3PAIA 10095acc     mibtbl.obj
 0003:00002ad8       ?rxSubMap_OID@@3PAIA       10095ad8     mibtbl.obj
 0003:00002ae4       ?rxSubChannelEntry_OID@@3PAIA 10095ae4     mibtbl.obj
 0003:00002af0       ?txOID@@3PAIA              10095af0     mibtbl.obj
 0003:00002b18       ?txIndex_OID@@3PAIA        10095b18     mibtbl.obj
 0003:00002b24       ?txBundle_OID@@3PAIA       10095b24     mibtbl.obj
 0003:00002b30       ?txDestinationMAC_OID@@3PAIA 10095b30     mibtbl.obj
 0003:00002b3c       ?txPriority_OID@@3PAIA     10095b3c     mibtbl.obj
 0003:00002b48       ?txSubCount_OID@@3PAIA     10095b48     mibtbl.obj
 0003:00002b54       ?txBuddyExclude_OID@@3PAIA 10095b54     mibtbl.obj
 0003:00002b60       ?txDropouts_OID@@3PAIA     10095b60     mibtbl.obj
 0003:00002b6c       ?txPosition_OID@@3PAIA     10095b6c     mibtbl.obj
 0003:00002b78       ?txReceivers_OID@@3PAIA    10095b78     mibtbl.obj
 0003:00002b84       ?txUnicastMode_OID@@3PAIA  10095b84     mibtbl.obj
 0003:00002b90       ?txMaxUnicast_OID@@3PAIA   10095b90     mibtbl.obj
 0003:00002b9c       ?txSubChannelIndex_OID@@3PAIA 10095b9c     mibtbl.obj
 0003:00002ba8       ?txSubMap_OID@@3PAIA       10095ba8     mibtbl.obj
 0003:00002bb4       ?txSubFormat_OID@@3PAIA    10095bb4     mibtbl.obj
 0003:00002bc0       ?syncOID@@3PAIA            10095bc0     mibtbl.obj
 0003:00002be8       ?syncConductorClock_OID@@3PAIA 10095be8     mibtbl.obj
 0003:00002bf0       ?syncPerformerClock_OID@@3PAIA 10095bf0     mibtbl.obj
 0003:00002bf8       ?syncClockTrim_OID@@3PAIA  10095bf8     mibtbl.obj
 0003:00002c00       ?syncBuddyLinkControl_OID@@3PAIA 10095c00     mibtbl.obj
 0003:00002c08       ?syncStatus_OID@@3PAIA     10095c08     mibtbl.obj
 0003:00002c10       ?syncCounter_OID@@3PAIA    10095c10     mibtbl.obj
 0003:00002c18       ?syncNTime_OID@@3PAIA      10095c18     mibtbl.obj
 0003:00002c20       ?mimonOID@@3PAIA           10095c20     mibtbl.obj
 0003:00002c4c       ?mimonDirty_OID@@3PAIA     10095c4c     mibtbl.obj
 0003:00002c54       ?mimonSNMPDirty_OID@@3PAIA 10095c54     mibtbl.obj
 0003:00002c5c       ?mimonHMIDirty_OID@@3PAIA  10095c5c     mibtbl.obj
 0003:00002c64       ?mimonUnknown_OID@@3PAIA   10095c64     mibtbl.obj
 0003:00002c6c       ?ipmonOID@@3PAIA           10095c6c     mibtbl.obj
 0003:00002c98       ?ipmonStaticIP_OID@@3PAIA  10095c98     mibtbl.obj
 0003:00002ca0       ?ipmonCurrentIP_OID@@3PAIA 10095ca0     mibtbl.obj
 0003:00002ca8       ?ipmonUnknown2_OID@@3PAIA  10095ca8     mibtbl.obj
 0003:00002cb0       ?ipmonUnknown3_OID@@3PAIA  10095cb0     mibtbl.obj
 0003:00002cb8       ?ifmOID@@3PAIA             10095cb8     mibtbl.obj
 0003:00002ce4       ?ifmCurrentIf_OID@@3PAIA   10095ce4     mibtbl.obj
 0003:00002cec       ?ifmLastChange_OID@@3PAIA  10095cec     mibtbl.obj
 0003:00002cf4       ?ifmTIndex_OID@@3PAIA      10095cf4     mibtbl.obj
 0003:00002d00       ?ifmTStatus_OID@@3PAIA     10095d00     mibtbl.obj
 0003:00002d0c       ?ifmTLastChange_OID@@3PAIA 10095d0c     mibtbl.obj
 0003:00002d18       ?ifmSwitchMode_OID@@3PAIA  10095d18     mibtbl.obj
 0003:00002d20       ?serialOID@@3PAIA          10095d20     mibtbl.obj
 0003:00002d4c       ?serialFormat_OID@@3PAIA   10095d4c     mibtbl.obj
 0003:00002d54       ?serialBaud_OID@@3PAIA     10095d54     mibtbl.obj
 0003:00002d5c       ?serialPPeriod_OID@@3PAIA  10095d5c     mibtbl.obj
 0003:00002d64       ?serialRxMAC_OID@@3PAIA    10095d64     mibtbl.obj
 0003:00002d6c       ?serialTxPriority_OID@@3PAIA 10095d6c     mibtbl.obj
 0003:00002d74       ?serialTxChannel_OID@@3PAIA 10095d74     mibtbl.obj
 0003:00002d7c       ?serialTxMAC_OID@@3PAIA    10095d7c     mibtbl.obj
 0003:00002d84       ?stdOID@@3PAIA             10095d84     mibtbl.obj
 0003:00002dac       ?stdUserVersionMajor_OID@@3PAIA 10095dac     mibtbl.obj
 0003:00002db4       ?stdUserVersionMinor_OID@@3PAIA 10095db4     mibtbl.obj
 0003:00002dbc       ?stdUserString_OID@@3PAIA  10095dbc     mibtbl.obj
 0003:00002dc8       ?stdUserInteger_OID@@3PAIA 10095dc8     mibtbl.obj
 0003:00002dd4       ?sysOID@@3PAIA             10095dd4     mibtbl.obj
 0003:00002df0       ?sysDescription_OID@@3PAIA 10095df0     mibtbl.obj
 0003:00002df8       ?sysObjectID_OID@@3PAIA    10095df8     mibtbl.obj
 0003:00002e00       ?sysUpTime_OID@@3PAIA      10095e00     mibtbl.obj
 0003:00002e08       ?sysContact_OID@@3PAIA     10095e08     mibtbl.obj
 0003:00002e10       ?sysName_OID@@3PAIA        10095e10     mibtbl.obj
 0003:00002e18       ?sysLocation_OID@@3PAIA    10095e18     mibtbl.obj
 0003:00002e20       ?sysServices_OID@@3PAIA    10095e20     mibtbl.obj
 0003:00002e28       ?ifOID@@3PAIA              10095e28     mibtbl.obj
 0003:00002e44       ?ifNumber_OID@@3PAIA       10095e44     mibtbl.obj
 0003:00002e4c       ?ifIndex_OID@@3PAIA        10095e4c     mibtbl.obj
 0003:00002e58       ?ifDescr_OID@@3PAIA        10095e58     mibtbl.obj
 0003:00002e64       ?ifType_OID@@3PAIA         10095e64     mibtbl.obj
 0003:00002e70       ?ifMtu_OID@@3PAIA          10095e70     mibtbl.obj
 0003:00002e7c       ?ifSpeed_OID@@3PAIA        10095e7c     mibtbl.obj
 0003:00002e88       ?ifPhysAddress_OID@@3PAIA  10095e88     mibtbl.obj
 0003:00002e94       ?ifAdminStatus_OID@@3PAIA  10095e94     mibtbl.obj
 0003:00002ea0       ?ifOperStatus_OID@@3PAIA   10095ea0     mibtbl.obj
 0003:00002eac       ?ifLastChange_OID@@3PAIA   10095eac     mibtbl.obj
 0003:00002eb8       ?ifInOctets_OID@@3PAIA     10095eb8     mibtbl.obj
 0003:00002ec4       ?ifInUcastPkts_OID@@3PAIA  10095ec4     mibtbl.obj
 0003:00002ed0       ?ifInNUcastPkts_OID@@3PAIA 10095ed0     mibtbl.obj
 0003:00002edc       ?ifInDiscards_OID@@3PAIA   10095edc     mibtbl.obj
 0003:00002ee8       ?ifInErrors_OID@@3PAIA     10095ee8     mibtbl.obj
 0003:00002ef4       ?ifInUnknownProtos_OID@@3PAIA 10095ef4     mibtbl.obj
 0003:00002f00       ?ifOutOctets_OID@@3PAIA    10095f00     mibtbl.obj
 0003:00002f0c       ?ifOutUcastPkts_OID@@3PAIA 10095f0c     mibtbl.obj
 0003:00002f18       ?ifOutNUcastPkts_OID@@3PAIA 10095f18     mibtbl.obj
 0003:00002f24       ?ifOutDiscards_OID@@3PAIA  10095f24     mibtbl.obj
 0003:00002f30       ?ifOutErrors_OID@@3PAIA    10095f30     mibtbl.obj
 0003:00002f3c       ?ifOutQLen_OID@@3PAIA      10095f3c     mibtbl.obj
 0003:00002f48       ?ifSpedific_OID@@3PAIA     10095f48     mibtbl.obj
 0003:00002f54       ?ipOID@@3PAIA              10095f54     mibtbl.obj
 0003:00002f70       ?ipForwarding_OID@@3PAIA   10095f70     mibtbl.obj
 0003:00002f78       ?ipDefaultTTL_OID@@3PAIA   10095f78     mibtbl.obj
 0003:00002f80       ?ipInReceives_OID@@3PAIA   10095f80     mibtbl.obj
 0003:00002f88       ?ipInHdrErrors_OID@@3PAIA  10095f88     mibtbl.obj
 0003:00002f90       ?ipInAddrErrors_OID@@3PAIA 10095f90     mibtbl.obj
 0003:00002f98       ?ipForwDatagrams_OID@@3PAIA 10095f98     mibtbl.obj
 0003:00002fa0       ?ipInUnknownProtos_OID@@3PAIA 10095fa0     mibtbl.obj
 0003:00002fa8       ?ipInDiscards_OID@@3PAIA   10095fa8     mibtbl.obj
 0003:00002fb0       ?ipInDelivers_OID@@3PAIA   10095fb0     mibtbl.obj
 0003:00002fb8       ?ipOutRequests_OID@@3PAIA  10095fb8     mibtbl.obj
 0003:00002fc0       ?ipOutDiscards_OID@@3PAIA  10095fc0     mibtbl.obj
 0003:00002fc8       ?ipOutNoRoutes_OID@@3PAIA  10095fc8     mibtbl.obj
 0003:00002fd0       ?ipReasmTimeout_OID@@3PAIA 10095fd0     mibtbl.obj
 0003:00002fd8       ?ipReasmReqds_OID@@3PAIA   10095fd8     mibtbl.obj
 0003:00002fe0       ?ipReasmOKs_OID@@3PAIA     10095fe0     mibtbl.obj
 0003:00002fe8       ?ipReasmFails_OID@@3PAIA   10095fe8     mibtbl.obj
 0003:00002ff0       ?ipFragOKs_OID@@3PAIA      10095ff0     mibtbl.obj
 0003:00002ff8       ?ipFragFails_OID@@3PAIA    10095ff8     mibtbl.obj
 0003:00003000       ?ipFragCreates_OID@@3PAIA  10096000     mibtbl.obj
 0003:00003008       ?ipAdEntAddr_OID@@3PAIA    10096008     mibtbl.obj
 0003:00003014       ?ipAdEntIfIndex_OID@@3PAIA 10096014     mibtbl.obj
 0003:00003020       ?ipAdEntNetMask_OID@@3PAIA 10096020     mibtbl.obj
 0003:0000302c       ?ipAdEntBcastAddr_OID@@3PAIA 1009602c     mibtbl.obj
 0003:00003038       ?ipAdEntReasmMaxSize_OID@@3PAIA 10096038     mibtbl.obj
 0003:00003044       ?ipRoutingDiscards_OID@@3PAIA 10096044     mibtbl.obj
 0003:0000304c       ?udpOID@@3PAIA             1009604c     mibtbl.obj
 0003:00003068       ?udpInDatagrams_OID@@3PAIA 10096068     mibtbl.obj
 0003:00003070       ?udpNoPorts_OID@@3PAIA     10096070     mibtbl.obj
 0003:00003078       ?udpInErrors_OID@@3PAIA    10096078     mibtbl.obj
 0003:00003080       ?udpOutDatagrams_OID@@3PAIA 10096080     mibtbl.obj
 0003:00003088       ?snmpOID@@3PAIA            10096088     mibtbl.obj
 0003:000030a4       ?snmpInPkts_OID@@3PAIA     100960a4     mibtbl.obj
 0003:000030ac       ?snmpOutPkts_OID@@3PAIA    100960ac     mibtbl.obj
 0003:000030b4       ?snmpInBadVersions_OID@@3PAIA 100960b4     mibtbl.obj
 0003:000030bc       ?snmpInBadCommunityNames_OID@@3PAIA 100960bc     mibtbl.obj
 0003:000030c4       ?snmpInBadCommunityUses_OID@@3PAIA 100960c4     mibtbl.obj
 0003:000030cc       ?snmpInASNParseErrs_OID@@3PAIA 100960cc     mibtbl.obj
 0003:000030d4       ?snmpInTooBigs_OID@@3PAIA  100960d4     mibtbl.obj
 0003:000030dc       ?snmpInNoSuchNames_OID@@3PAIA 100960dc     mibtbl.obj
 0003:000030e4       ?snmpInBadValues_OID@@3PAIA 100960e4     mibtbl.obj
 0003:000030ec       ?snmpInReadOnlys_OID@@3PAIA 100960ec     mibtbl.obj
 0003:000030f4       ?snmpInGenErrs_OID@@3PAIA  100960f4     mibtbl.obj
 0003:000030fc       ?snmpInTotalReqVars_OID@@3PAIA 100960fc     mibtbl.obj
 0003:00003104       ?snmpInTotalSetVars_OID@@3PAIA 10096104     mibtbl.obj
 0003:0000310c       ?snmpInGetRequests_OID@@3PAIA 1009610c     mibtbl.obj
 0003:00003114       ?snmpInGetNexts_OID@@3PAIA 10096114     mibtbl.obj
 0003:0000311c       ?snmpInSetRequests_OID@@3PAIA 1009611c     mibtbl.obj
 0003:00003124       ?snmpInGetResponses_OID@@3PAIA 10096124     mibtbl.obj
 0003:0000312c       ?snmpInTraps_OID@@3PAIA    1009612c     mibtbl.obj
 0003:00003134       ?snmpOutTooBigs_OID@@3PAIA 10096134     mibtbl.obj
 0003:0000313c       ?snmpOutNoSuchNames_OID@@3PAIA 1009613c     mibtbl.obj
 0003:00003144       ?snmpOutBadValues_OID@@3PAIA 10096144     mibtbl.obj
 0003:0000314c       ?snmpOutGenErrs_OID@@3PAIA 1009614c     mibtbl.obj
 0003:00003154       ?snmpOutGetRequests_OID@@3PAIA 10096154     mibtbl.obj
 0003:0000315c       ?snmpOutGetNexts_OID@@3PAIA 1009615c     mibtbl.obj
 0003:00003164       ?snmpOutSetRequests_OID@@3PAIA 10096164     mibtbl.obj
 0003:0000316c       ?snmpOutGetResponses_OID@@3PAIA 1009616c     mibtbl.obj
 0003:00003174       ?snmpOutTraps_OID@@3PAIA   10096174     mibtbl.obj
 0003:0000317c       ?snmpEnableAuthenTraps_OID@@3PAIA 1009617c     mibtbl.obj
 0003:00003184       ?snmpSilentDrops_OID@@3PAIA 10096184     mibtbl.obj
 0003:0000318c       ?snmpProxyDrops_OID@@3PAIA 1009618c     mibtbl.obj
 0003:00003194       ?firmwareOID@@3PAIA        10096194     mibtbl.obj
 0003:000031bc       ?firmwareProtocolVersion_OID@@3PAIA 100961bc     mibtbl.obj
 0003:000031c4       ?firmwareMajorVersion_OID@@3PAIA 100961c4     mibtbl.obj
 0003:000031cc       ?firmwareMinorVersion_OID@@3PAIA 100961cc     mibtbl.obj
 0003:000031d4       ?firmwareBootVersion_OID@@3PAIA 100961d4     mibtbl.obj
 0003:00003390       ___security_cookie         10096390     LIBCMT:gs_cookie.obj
 0003:00003394       ___security_cookie_complement 10096394     LIBCMT:gs_cookie.obj
 0003:000033a0       __fltused                  100963a0     LIBCMT:fpinit.obj
 0003:000033a4       __ldused                   100963a4     LIBCMT:fpinit.obj
 0003:000033b8       __mbctype                  100963b8     LIBCMT:mbctype.obj
 0003:000034c0       __mbcasemap                100964c0     LIBCMT:mbctype.obj
 0003:000035c0       ___initialmbcinfo          100965c0     LIBCMT:mbctype.obj
 0003:000037e4       ___ptmbcinfo               100967e4     LIBCMT:mbctype.obj
 0003:000038d8       ___flsindex                100968d8     LIBCMT:tidtable.obj
 0003:000038dc       ___mb_cur_max              100968dc     LIBCMT:nlsdata.obj
 0003:000038e0       ___wclocalestr             100968e0     LIBCMT:nlsdata.obj
 0003:000038e8       ___lc_time_c               100968e8     LIBCMT:nlsdata.obj
 0003:00003a4c       ___ptlocinfo               10096a4c     LIBCMT:nlsdata.obj
 0003:00003a50       ___initiallocinfo          10096a50     LIBCMT:nlsdata.obj
 0003:00003b08       ___initiallocalestructinfo 10096b08     LIBCMT:nlsdata.obj
 0003:00003b10       ___globallocalestatus      10096b10     LIBCMT:glstatus.obj
 0003:00003c88       ___nullstring              10096c88     LIBCMT:output.obj
 0003:00003c8c       ___wnullstring             10096c8c     LIBCMT:output.obj
 0003:00003c90       ___isa_enabled             10096c90     LIBCMT:cpu_disp.obj
 0003:00003c98       __iob                      10096c98     LIBCMT:_file.obj
 0003:00003f20       __cfltcvt_tab              10096f20     LIBCMT:cmiscdat.obj
 0003:00003f48       ___abort_behavior          10096f48     LIBCMT:abort.obj
 0003:00003f58       __d_inf                    10096f58     LIBCMT:util.obj
 0003:00003f60       __d_ind                    10096f60     LIBCMT:util.obj
 0003:00003f68       __d_max                    10096f68     LIBCMT:util.obj
 0003:00003f70       __d_min                    10096f70     LIBCMT:util.obj
 0003:00003f78       __d_mzero                  10096f78     LIBCMT:util.obj
 0003:000041c0       __half                     100971c0     LIBCMT:pow.obj
 0003:000041d0       __lookuptrailbytes         100971d0     LIBCMT:read.obj
 0003:000042d0       ___badioinfo               100972d0     LIBCMT:ioinit.obj
 0003:00004310       __HUGE                     10097310     LIBCMT:huge.obj
 0003:00004328       ___lconv                   10097328     LIBCMT:lconv.obj
 0003:0000432c       ___lconv_static_decimal    1009732c     LIBCMT:lconv.obj
 0003:00004330       ___lconv_c                 10097330     LIBCMT:lconv.obj
 0003:00004380       ___lconv_static_W_decimal  10097380     LIBCMT:lconv.obj
 0003:00004384       __pctype                   10097384     LIBCMT:ctype.obj
 0003:00004388       __pwctype                  10097388     LIBCMT:ctype.obj
 0003:000043c0       __matherr_flag             100973c0     LIBCMT:matherr.obj
 0003:000043d0       __NLG_Destination          100973d0     LIBCMT:exsup.obj
 0003:000043e0       __pow10pos                 100973e0     LIBCMT:constpow.obj
 0003:00004540       __pow10neg                 10097540     LIBCMT:constpow.obj
 0003:0000469c       __confh                    1009769c     LIBCMT:initcon.obj
 0003:000046a0       ??_R0?AVSnmpRequest@@@8    100976a0     asisnmp.obj
 0003:000046bc       ??_R0?AVSnmpGetRequest@@@8 100976bc     asisnmp.obj
 0003:000046dc       ??_R0?AVSnmpGetNextRequest@@@8 100976dc     asisnmp.obj
 0003:00004700       ??_R0?AVSnmpSetRequest@@@8 10097700     asisnmp.obj
 0003:00004720       ??_R0?AVasxBase@@@8        10097720     asxavdecc.obj
 0003:00004738       ??_R0?AVasxAdapterAVDECC@@@8 10097738     asxavdecc.obj
 0003:00004758       ??_R0?AVasxAdapter@@@8     10097758     asxavdecc.obj
 0003:00004774       ??_R0?AVasxSubSystemAVDECC@@@8 10097774     asxavdecc.obj
 0003:00004798       ??_R0?AVasxSubSystem@@@8   10097798     asxavdecc.obj
 0003:000047b4       ??_R0?AVerror_category@std@@@8 100977b4     asxavdecc.obj
 0003:000047d8       ??_R0?AV_Generic_error_category@std@@@8 100977d8     asxavdecc.obj
 0003:00004804       ??_R0?AV_Iostream_error_category@std@@@8 10097804     asxavdecc.obj
 0003:00004830       ??_R0?AV_System_error_category@std@@@8 10097830     asxavdecc.obj
 0003:0000485c       ??_R0?AVasxMixerScanner@@@8 1009785c     asxasio.obj
 0003:0000487c       ??_R0?AVasxAdapterASIO@@@8 1009787c     asxasio.obj
 0003:0000489c       ??_R0?AVasxSubSystemASIO@@@8 1009789c     asxasio.obj
 0003:000048bc       ??_R0?AVasxMixerScannerASIO@@@8 100978bc     asxasio.obj
 0003:000048e0       ??_R0?AVasxControlBase@@@8 100978e0     asxasioplay.obj
 0003:00004900       ??_R0?AVasxPlayerASIO@@@8  10097900     asxasioplay.obj
 0003:0000491c       ??_R0?AVasxPlayer@@@8      1009791c     asxasioplay.obj
 0003:00004934       ??_R0?AVasxRecorderASIO@@@8 10097934     asxasiorec.obj
 0003:00004954       ??_R0?AVasxRecorder@@@8    10097954     asxasiorec.obj
 0003:00004970       ??_R0?AVasxSystem@@@8      10097970     asxclass.obj
 0003:00004988       ??_R0?AVasxMixer@@@8       10097988     asxclass.obj
 0003:000049a0       ??_R0?AVasxNode@@@8        100979a0     asxclass.obj
 0003:000049b8       ??_R0?AVasxAbstractAdapter@@@8 100979b8     asxclass.obj
 0003:000049dc       ??_R0?AVasxBlockProperty@@@8 100979dc     asxclass.obj
 0003:000049fc       ??_R0?AVasxSubSystemDSND@@@8 100979fc     asxdsnd.obj
 0003:00004a1c       ??_R0?AVasxAdapterDSND@@@8 10097a1c     asxdsnd.obj
 0003:00004a3c       ??_R0?AVasxMixerScannerDSND@@@8 10097a3c     asxdsnd.obj
 0003:00004a60       ??_R0?AVasxPlayerDSND@@@8  10097a60     asxdsndplay.obj
 0003:00004a7c       ??_R0?AVasxRecorderDSND@@@8 10097a7c     asxdsndrec.obj
 0003:00004a9c       ??_R0?AVasxCobranetContainer@@@8 10097a9c     asxhpi.obj
 0003:00004ac0       ??_R0?AVasxMeter@@@8       10097ac0     asxhpi.obj
 0003:00004ad8       ??_R0?AVasxVolume@@@8      10097ad8     asxhpi.obj
 0003:00004af0       ??_R0?AVasxLevel@@@8       10097af0     asxhpi.obj
 0003:00004b08       ??_R0?AVasxMux@@@8         10097b08     asxhpi.obj
 0003:00004b20       ??_R0?AVasxMode@@@8        10097b20     asxhpi.obj
 0003:00004b38       ??_R0?AVasxTuner@@@8       10097b38     asxhpi.obj
 0003:00004b50       ??_R0?AVasxPad@@@8         10097b50     asxhpi.obj
 0003:00004b68       ??_R0?AVasxSampleClock@@@8 10097b68     asxhpi.obj
 0003:00004b88       ??_R0?AVasxAes3Tx@@@8      10097b88     asxhpi.obj
 0003:00004ba0       ??_R0?AVasxAes3Rx@@@8      10097ba0     asxhpi.obj
 0003:00004bb8       ??_R0?AVasxGpio@@@8        10097bb8     asxhpi.obj
 0003:00004bd0       ??_R0?AVasxVox@@@8         10097bd0     asxhpi.obj
 0003:00004be8       ??_R0?AVasxBitStream@@@8   10097be8     asxhpi.obj
 0003:00004c04       ??_R0?AVasxMic@@@8         10097c04     asxhpi.obj
 0003:00004c1c       ??_R0?AVasxParametricEQ@@@8 10097c1c     asxhpi.obj
 0003:00004c3c       ??_R0?AVasxCompander@@@8   10097c3c     asxhpi.obj
 0003:00004c58       ??_R0?AVasxCobranet@@@8    10097c58     asxhpi.obj
 0003:00004c74       ??_R0?AVasxCobranetRx@@@8  10097c74     asxhpi.obj
 0003:00004c90       ??_R0?AVasxCobranetRxContainer@@@8 10097c90     asxhpi.obj
 0003:00004cb8       ??_R0?AVasxCobranetTx@@@8  10097cb8     asxhpi.obj
 0003:00004cd4       ??_R0?AVasxCobranetTxContainer@@@8 10097cd4     asxhpi.obj
 0003:00004cfc       ??_R0?AVasxToneDetector@@@8 10097cfc     asxhpi.obj
 0003:00004d1c       ??_R0?AVasxSilenceDetector@@@8 10097d1c     asxhpi.obj
 0003:00004d40       ??_R0?AVasxGenericControl@@@8 10097d40     asxhpi.obj
 0003:00004d60       ??_R0?AVasxBlock@@@8       10097d60     asxhpi.obj
 0003:00004d78       ??_R0?AVasxSubSystemHPI@@@8 10097d78     asxhpi.obj
 0003:00004d98       ??_R0?AVasxAdapterHPI@@@8  10097d98     asxhpi.obj
 0003:00004db4       ??_R0?AVasxMixerScannerHPI@@@8 10097db4     asxhpi.obj
 0003:00004dd8       ??_R0?AVasxAdapterHPIDuplicateIndex@@@8 10097dd8     asxhpi.obj
 0003:00004e04       ??_R0?AVasxMixerScannerHPIDuplicateIndex@@@8 10097e04     asxhpi.obj
 0003:00004e34       ??_R0?AVasxControlHPI@@@8  10097e34     asxhpi.obj
 0003:00004e50       ??_R0?AVasxControlBaseHPI@@@8 10097e50     asxhpi.obj
 0003:00004e70       ??_R0?AVasxGenericHPI@@@8  10097e70     asxhpi.obj
 0003:00004e8c       ??_R0?AVasxVolumeHPI@@@8   10097e8c     asxhpi.obj
 0003:00004ea8       ??_R0?AVasxLevelHPI@@@8    10097ea8     asxhpi.obj
 0003:00004ec4       ??_R0?AVasxMeterHPI@@@8    10097ec4     asxhpi.obj
 0003:00004ee0       ??_R0?AVasxMuxHPI@@@8      10097ee0     asxhpi.obj
 0003:00004ef8       ??_R0?AVasxModeHPI@@@8     10097ef8     asxhpi.obj
 0003:00004f14       ??_R0?AVasxSampleClockHPI@@@8 10097f14     asxhpi.obj
 0003:00004f34       ??_R0?AVasxTunerHPI@@@8    10097f34     asxhpi.obj
 0003:00004f50       ??_R0?AVasxAes3TxHPI@@@8   10097f50     asxhpi.obj
 0003:00004f6c       ??_R0?AVasxAesebuReceiverHPI@@@8 10097f6c     asxhpi.obj
 0003:00004f90       ??_R0?AVasxGpioHPI@@@8     10097f90     asxhpi.obj
 0003:00004fac       ??_R0?AVasxVoxHPI@@@8      10097fac     asxhpi.obj
 0003:00004fc4       ??_R0?AVasxMicHPI@@@8      10097fc4     asxhpi.obj
 0003:00004fdc       ??_R0?AVasxParametricEqHPI@@@8 10097fdc     asxhpi.obj
 0003:00005000       ??_R0?AVasxCompanderHPI@@@8 10098000     asxhpi.obj
 0003:00005020       ??_R0?AVasxCompanderHPI_Legacy@@@8 10098020     asxhpi.obj
 0003:00005048       ??_R0?AVasxCobranetHPI@@@8 10098048     asxhpi.obj
 0003:00005068       ??_R0?AVasxCobranetRxHPI@@@8 10098068     asxhpi.obj
 0003:00005088       ??_R0?AVasxCobranetTxHPI@@@8 10098088     asxhpi.obj
 0003:000050a8       ??_R0?AVasxToneDetectorHPI@@@8 100980a8     asxhpi.obj
 0003:000050cc       ??_R0?AVasxSilenceDetectorHPI@@@8 100980cc     asxhpi.obj
 0003:000050f0       ??_R0?AVasxPadHPI@@@8      100980f0     asxhpi.obj
 0003:00005108       ??_R0?AVasxBlockPropertyHPI@@@8 10098108     asxhpi.obj
 0003:0000512c       ??_R0?AVasxBlockHPI@@@8    1009812c     asxhpi.obj
 0003:00005148       ??_R0?AVasxPlayerHPI@@@8   10098148     asxhpiplay.obj
 0003:00005164       ??_R0?AVasxPlayerHPIWithInt@@@8 10098164     asxhpiplayi.obj
 0003:00005188       ??_R0?AVasxRecorderHPI@@@8 10098188     asxhpirec.obj
 0003:000051a8       ??_R0?AVasxRecorderHPIWithInt@@@8 100981a8     asxhpireci.obj
 0003:000051cc       ??_R0?AVasxCallbackObject@@@8 100981cc     asxplay.obj
 0003:000051ec       ??_R0?AVPlayerDoneCallback@@@8 100981ec     asxplay.obj
 0003:00005210       ??_R0?AVasxAdapterSNMP@@@8 10098210     asxsnmp.obj
 0003:00005230       ??_R0?AVasxSubSystemSNMP@@@8 10098230     asxsnmp.obj
 0003:00005250       ??_R0?AVasxMixerScannerSNMP@@@8 10098250     asxsnmp.obj
 0003:00005274       ??_R0?AVasxCobranetSNMP@@@8 10098274     asxsnmp.obj
 0003:00005294       ??_R0?AVasxCobranetTxSNMP@@@8 10098294     asxsnmp.obj
 0003:000052b4       ??_R0?AVasxCobranetRxSNMP@@@8 100982b4     asxsnmp.obj
 0003:000052d4       ??_R0?AVasxMixerScannerUnreachableSNMP@@@8 100982d4     asxsnmp.obj
 0003:00005304       ??_R0?AVasxCobranetUnreachableSNMP@@@8 10098304     asxsnmp.obj
 0003:00005330       ??_R0?AVasxLevelTR800@@@8  10098330     asxtr800.obj
 0003:0000534c       ??_R0?AVasxControlBaseTR800@@@8 1009834c     asxtr800.obj
 0003:00005370       ??_R0?AVasxMeterTR800@@@8  10098370     asxtr800.obj
 0003:0000538c       ??_R0?AVasxGpioTR800@@@8   1009838c     asxtr800.obj
 0003:000053a8       ??_R0?AVasxBlockTR800OptoMode@@@8 100983a8     asxtr800.obj
 0003:000053cc       ??_R0?AVasxBlockTR800Status@@@8 100983cc     asxtr800.obj
 0003:000053f0       ??_R0?AVasxSubSystemWAVE@@@8 100983f0     asxwave.obj
 0003:00005410       ??_R0?AVasxAdapterWAVE@@@8 10098410     asxwave.obj
 0003:00005430       ??_R0?AVasxMixerScannerWAVE@@@8 10098430     asxwave.obj
 0003:00005454       ??_R0?AVasxVolumeWAVE@@@8  10098454     asxwave.obj
 0003:00005470       ??_R0?AVasxMeterWAVE@@@8   10098470     asxwave.obj
 0003:0000548c       ??_R0?AVasxLevelWAVE@@@8   1009848c     asxwave.obj
 0003:000054a8       ??_R0?AVasxMuxWAVE@@@8     100984a8     asxwave.obj
 0003:000054c4       ??_R0?AVasxModeWAVE@@@8    100984c4     asxwave.obj
 0003:000054e0       ??_R0?AVasxTunerWAVE@@@8   100984e0     asxwave.obj
 0003:000054fc       ??_R0?AVasxCobranetWAVE@@@8 100984fc     asxwave.obj
 0003:0000551c       ??_R0?AVasxToneDetectorWAVE@@@8 1009851c     asxwave.obj
 0003:00005540       ??_R0?AVasxSilenceDetectorWAVE@@@8 10098540     asxwave.obj
 0003:00005568       ??_R0?AVasxPlayerWAVE@@@8  10098568     asxwaveplay.obj
 0003:00005584       ??_R0?AVasxRecorderWAVE@@@8 10098584     asxwaverec.obj
 0003:000055a4       ??_R0?AVTWavFileBase@@@8   100985a4     twavfile.obj
 0003:000055c0       ??_R0?AVTWavFmt@@@8        100985c0     twavfile.obj
 0003:000055d8       ??_R0?AVTWavFileTypeWav@@@8 100985d8     twavfile.obj
 0003:000055f8       ??_R0?AVTWavFileTypeMP23@@@8 100985f8     twavfile.obj
 0003:00005618       ??_R0?AVTWavFileTypeDAF@@@8 10098618     twavfile.obj
 0003:00005638       ??_R0?AVTWavFileTypeRaw@@@8 10098638     twavfile.obj
 0003:00005658       ??_R0?AVTWavFileTypeNullRecord@@@8 10098658     twavfile.obj
 0003:00005680       ??_R0?AVTWavFileTypeGenerator@@@8 10098680     twavfile.obj
 0003:000056a4       ??_R0?AVTWavFileWithFifo@@@8 100986a4     twavfilefifo.obj
 0003:000056c4       ??_R0?AVbad_alloc@std@@@8  100986c4     LIBCMT:new.obj
 0003:000056e0       ??_R0?AVexception@std@@@8  100986e0     LIBCMT:new.obj
 0003:000056fc       ??_R0?AVtype_info@@@8      100986fc     LIBCMT:typinfo.obj
 0003:00005714       ??_R0?AV__non_rtti_object@std@@@8 10098714     LIBCMT:rtti.obj
 0003:00005738       ??_R0?AVbad_typeid@std@@@8 10098738     LIBCMT:rtti.obj
 0003:00005758       ??_R0?AVbad_cast@std@@@8   10098758     LIBCMT:rtti.obj
 0003:00005774       ??_R0?AVbad_exception@std@@@8 10098774     LIBCMT:frame.obj
 0003:00005794       ??_R0?AVDNameNode@@@8      10098794     LIBCMT:undname.obj
 0003:000057ac       ??_R0?AVcharNode@@@8       100987ac     LIBCMT:undname.obj
 0003:000057c4       ??_R0?AVpcharNode@@@8      100987c4     LIBCMT:undname.obj
 0003:000057dc       ??_R0?AVpDNameNode@@@8     100987dc     LIBCMT:undname.obj
 0003:000057f8       ??_R0?AVDNameStatusNode@@@8 100987f8     LIBCMT:undname.obj
 0003:00005818       ??_R0?AVpairNode@@@8       10098818     LIBCMT:undname.obj
 0003:00005830       ??_R0?AVinvalid_argument@std@@@8 10098830     libcpmt:xthrow.obj
 0003:00005854       ??_R0?AVlogic_error@std@@@8 10098854     libcpmt:xthrow.obj
 0003:00005874       ??_R0?AVlength_error@std@@@8 10098874     libcpmt:xthrow.obj
 0003:00005894       ??_R0?AVout_of_range@std@@@8 10098894     libcpmt:xthrow.obj
 0003:000058b4       ??_R0?AVoverflow_error@std@@@8 100988b4     libcpmt:xthrow.obj
 0003:000058d8       ??_R0?AVruntime_error@std@@@8 100988d8     libcpmt:xthrow.obj
 0003:000058f8       ??_R0?AVbad_function_call@std@@@8 100988f8     libcpmt:xthrow.obj
 0003:0000591c       ??_R0?AVregex_error@std@@@8 1009891c     libcpmt:xthrow.obj
 0003:0000593c       __imp__create_net_interface@0 1009893c     avdecc-lib_controller32:avdecc-lib_controller32.dll
 0003:00005940       __imp__create_controller@16 10098940     avdecc-lib_controller32:avdecc-lib_controller32.dll
 0003:00005944       __imp__create_system@12    10098944     avdecc-lib_controller32:avdecc-lib_controller32.dll
 0003:00005948       __imp_?aem_cmd_value_to_name@utility@avdecc_lib@@YGPBDG@Z 10098948     avdecc-lib_controller32:avdecc-lib_controller32.dll
 0003:0000594c       __imp_?aem_desc_value_to_name@utility@avdecc_lib@@YGPBDG@Z 1009894c     avdecc-lib_controller32:avdecc-lib_controller32.dll
 0003:00005950       __imp_?aem_cmd_status_value_to_name@utility@avdecc_lib@@YGPBDI@Z 10098950     avdecc-lib_controller32:avdecc-lib_controller32.dll
 0003:00005954       __imp_?acmp_cmd_value_to_name@utility@avdecc_lib@@YGPBDI@Z 10098954     avdecc-lib_controller32:avdecc-lib_controller32.dll
 0003:00005958       __imp_?acmp_cmd_status_value_to_name@utility@avdecc_lib@@YGPBDI@Z 10098958     avdecc-lib_controller32:avdecc-lib_controller32.dll
 0003:0000595c       __imp_?notification_value_to_name@utility@avdecc_lib@@YGPBDG@Z 1009895c     avdecc-lib_controller32:avdecc-lib_controller32.dll
 0003:00005960       \177avdecc-lib_controller32_NULL_THUNK_DATA_DLA 10098960     avdecc-lib_controller32:avdecc-lib_controller32.dll
 0003:00005984       ?pCreatePcapInterface@@3P6A?AW4acndERROR@@VasiIpAddr@@PAPAVPcapInterface@@@ZA 10098984     asicndload.obj
 0003:00005988       ?pDeletePcapInterface@@3P6A?AW4acndERROR@@PAPAVPcapInterface@@@ZA 10098988     asicndload.obj
 0003:0000598c       ?pCreateAsiCobraNetDiscovery@@3P6A?AW4acndERROR@@PAVPcapInterface@@PAPAVAsiCobraNetDiscovery@@@ZA 1009898c     asicndload.obj
 0003:00005990       ?pDeleteAsiCobraNetDiscovery@@3P6A?AW4acndERROR@@PAPAVAsiCobraNetDiscovery@@@ZA 10098990     asicndload.obj
 0003:00005994       ?pCreateAsiAutoAssignIpTracker@@3P6A?AW4acndERROR@@PAPAVAsiAutoassignIpTracker@@@ZA 10098994     asicndload.obj
 0003:00005998       ?pDeleteAsiAutoAssignIpTracker@@3P6A?AW4acndERROR@@PAPAVAsiAutoassignIpTracker@@@ZA 10098998     asicndload.obj
 0003:0000599c       ?pCreateAsiAutoAssign@@3P6A?AW4acndERROR@@PAVPcapInterface@@PAVAsiCobraNetDiscovery@@PAVAsiAutoassignIpTracker@@PAPAVAsiAutoAssign@@@ZA 1009899c     asicndload.obj
 0003:000059a0       ?pDeleteAsiAutoAssign@@3P6A?AW4acndERROR@@PAPAVAsiAutoAssign@@@ZA 100989a0     asicndload.obj
 0003:000059a4       ?pAsiCnDiscoStart@@3P8AsiCobraNetDiscovery@@AEXXZQ1@ 100989a4     asicndload.obj
 0003:000059a8       ?pAsiCnDiscoStop@@3P8AsiCobraNetDiscovery@@AEXXZQ1@ 100989a8     asicndload.obj
 0003:000059ac       ?pAsiCnDiscoCreateNotificationClient@@3P8AsiCobraNetDiscovery@@AEPAVNotificationClient@@XZQ1@ 100989ac     asicndload.obj
 0003:000059b0       ?pAsiCnDiscoFreeNotificationClient@@3P8AsiCobraNetDiscovery@@AEXPAPAVNotificationClient@@@ZQ1@ 100989b0     asicndload.obj
 0003:000059b4       ?pNotificationClientGetEvent@@3P8NotificationClient@@AE_NPAW4EventType@NotificationEvent@@PAVasiMacAddr@@PAVasiIpAddr@@_N@ZQ1@ 100989b4     asicndload.obj
 0003:000059b8       ?pAutoAssignStart@@3P8AsiAutoAssign@@AEXXZQ1@ 100989b8     asicndload.obj
 0003:000059bc       ?pAutoAssignStop@@3P8AsiAutoAssign@@AEXXZQ1@ 100989bc     asicndload.obj
 0003:000059c0       ?pAutoAssignGetStatusForMac@@3P8AsiAutoAssign@@AE?AW4AsiAutoAssignNodeStatus@@PBVasiMacAddr@@@ZQ1@ 100989c0     asicndload.obj
 0003:000059c4       ?pAutoAssignAssignIpToMac@@3P8AsiAutoAssign@@AE?AW4AsiAutoAssignNodeStatus@@PBVasiMacAddr@@PBVasiIpAddr@@@ZQ1@ 100989c4     asicndload.obj
 0003:000059c8       ?targetDll@@3PAUHINSTANCE__@@A 100989c8     asicndload.obj
 0003:000059cc       ?m_pFirst@asiMibGroup@@0PAV1@A 100989cc     asimib.obj
 0003:000059d8       ?avdecc_subsys@@3PAVasxSubSystemAVDECC@@A 100989d8     asxavdecc.obj
 0003:000059e4       ?id@?$num_put@DV?$back_insert_iterator@V?$basic_string@DU?$char_traits@D@std@@V?$allocator@D@2@@std@@@std@@@std@@2V0locale@2@A 100989e4     asxavdecc.obj
 0003:000059e8       ?id@?$num_put@_WV?$back_insert_iterator@V?$basic_string@_WU?$char_traits@_W@std@@V?$allocator@_W@2@@std@@@std@@@std@@2V0locale@2@A 100989e8     asxavdecc.obj
 0003:000059ec       ?id@?$numpunct@D@std@@2V0locale@2@A 100989ec     asxavdecc.obj
 0003:000059f0       ?id@?$numpunct@_W@std@@2V0locale@2@A 100989f0     asxavdecc.obj
 0003:00005c78       ?pCallback@asxBase@@1P6AXPAXPBD00@ZA 10098c78     asxclass.obj
 0003:00005c7c       ?pUser1@asxBase@@1PAXA     10098c7c     asxclass.obj
 0003:00005c80       ?pUser2@asxBase@@1PAXA     10098c80     asxclass.obj
 0003:00005c84       ?pFirst@asxSystem@@0PAV1@A 10098c84     asxclass.obj
 0003:00005c8c       ?asxDebug@@3VasxDebugClass@@A 10098c8c     asxdebug.obj
 0003:00005c9c       ?phSS@@3PAUhpi_hsubsys@@A  10098c9c     asxhpi.obj
 0003:00005cd0       ?firmwareMinorVersionOID@CobraNetNode@@0VasiOID@@A 10098cd0     cobranet.obj
 0003:00005ce4       ?txReceiversOid@CobraNetNode@@0VasiOID@@A 10098ce4     cobranet.obj
 0003:00005cf8       ?modeRateStatusOID@CobraNetNode@@0VasiOID@@A 10098cf8     cobranet.obj
 0003:00005d0c       ?txSubMapOid@CobraNetNode@@0VasiOID@@A 10098d0c     cobranet.obj
 0003:00005d20       ?serialPPeriodOID@CobraNetNode@@0VasiOID@@A 10098d20     cobranet.obj
 0003:00005d34       ?flashPersistEnableOID@CobraNetNode@@0VasiOID@@A 10098d34     cobranet.obj
 0003:00005d48       ?serialTxMacOID@CobraNetNode@@0VasiOID@@A 10098d48     cobranet.obj
 0003:00005d5c       ?serialTxPriorityOID@CobraNetNode@@0VasiOID@@A 10098d5c     cobranet.obj
 0003:00005d70       ?sysDescriptionOID@CobraNetNode@@0VasiOID@@A 10098d70     cobranet.obj
 0003:00005d84       ?rxDropoutsOid@CobraNetNode@@0VasiOID@@A 10098d84     cobranet.obj
 0003:00005d98       ?errorDisplayOID@CobraNetNode@@0VasiOID@@A 10098d98     cobranet.obj
 0003:00005dac       ?stdUserIntegerOid@CobraNetNode@@0VasiOID@@A 10098dac     cobranet.obj
 0003:00005dc0       ?serialFormatOID@CobraNetNode@@0VasiOID@@A 10098dc0     cobranet.obj
 0003:00005dd4       ?errorLastOID@CobraNetNode@@0VasiOID@@A 10098dd4     cobranet.obj
 0003:00005de8       ?rxStatusOid@CobraNetNode@@0VasiOID@@A 10098de8     cobranet.obj
 0003:00005dfc       ?sysContactOID@CobraNetNode@@0VasiOID@@A 10098dfc     cobranet.obj
 0003:00005e10       ?txPositionOid@CobraNetNode@@0VasiOID@@A 10098e10     cobranet.obj
 0003:00005e24       ?serialBaudOID@CobraNetNode@@0VasiOID@@A 10098e24     cobranet.obj
 0003:00005e38       ?txPriorityOid@CobraNetNode@@0VasiOID@@A 10098e38     cobranet.obj
 0003:00005e4c       ?rxBundleOid@CobraNetNode@@0VasiOID@@A 10098e4c     cobranet.obj
 0003:00005e60       ?rxPriorityOid@CobraNetNode@@0VasiOID@@A 10098e60     cobranet.obj
 0003:00005e74       ?txBundleOid@CobraNetNode@@0VasiOID@@A 10098e74     cobranet.obj
 0003:00005e88       ?modeRateControlOID@CobraNetNode@@0VasiOID@@A 10098e88     cobranet.obj
 0003:00005e9c       ?ipmonStaticIpOID@CobraNetNode@@0VasiOID@@A 10098e9c     cobranet.obj
 0003:00005eb0       ?sysNameOID@CobraNetNode@@0VasiOID@@A 10098eb0     cobranet.obj
 0003:00005ec4       ?ipmonCurrentIpOID@CobraNetNode@@0VasiOID@@A 10098ec4     cobranet.obj
 0003:00005ed8       ?rxSourceMACOid@CobraNetNode@@0VasiOID@@A 10098ed8     cobranet.obj
 0003:00005eec       ?firmwareMajorVersionOID@CobraNetNode@@0VasiOID@@A 10098eec     cobranet.obj
 0003:00005f00       ?txSubFormatOid@CobraNetNode@@0VasiOID@@A 10098f00     cobranet.obj
 0003:00005f14       ?conductorPriorityOID@CobraNetNode@@0VasiOID@@A 10098f14     cobranet.obj
 0003:00005f28       ?txSubCountOid@CobraNetNode@@0VasiOID@@A 10098f28     cobranet.obj
 0003:00005f3c       ?rxSubMapOid@CobraNetNode@@0VasiOID@@A 10098f3c     cobranet.obj
 0003:00005f50       ?rxMinDelayOid@CobraNetNode@@0VasiOID@@A 10098f50     cobranet.obj
 0003:00005f64       ?audioMetersOid@CobraNetNode@@0VasiOID@@A 10098f64     cobranet.obj
 0003:00005f78       ?serialRxMacOID@CobraNetNode@@0VasiOID@@A 10098f78     cobranet.obj
 0003:00005f8c       ?errorCountOID@CobraNetNode@@0VasiOID@@A 10098f8c     cobranet.obj
 0003:00005fa0       ?rxDelayOid@CobraNetNode@@0VasiOID@@A 10098fa0     cobranet.obj
 0003:00005fb4       ?txMaxUnicastOid@CobraNetNode@@0VasiOID@@A 10098fb4     cobranet.obj
 0003:00005fc8       ?sysLocationOID@CobraNetNode@@0VasiOID@@A 10098fc8     cobranet.obj
 0003:00005fdc       ?txUnicastModeOid@CobraNetNode@@0VasiOID@@A 10098fdc     cobranet.obj
 0003:00005ff0       ?conductorStatusOID@CobraNetNode@@0VasiOID@@A 10098ff0     cobranet.obj
 0003:00006004       ?rxSubFormatOid@CobraNetNode@@0VasiOID@@A 10099004     cobranet.obj
 0003:00006018       ?txDropoutsOid@CobraNetNode@@0VasiOID@@A 10099018     cobranet.obj
 0003:00006030       ?syncEntryTable@@3PAVasiMibEntry@@A 10099030     mibtbl.obj
 0003:00006110       ?rxGroup@@3VasiMibGroup@@A 10099110     mibtbl.obj
 0003:00006128       ?ipGroup@@3VasiMibGroup@@A 10099128     mibtbl.obj
 0003:00006140       ?rxEntryTable@@3PAVasiMibEntry@@A 10099140     mibtbl.obj
 0003:000062b0       ?snmpEntryTable@@3PAVasiMibEntry@@A 100992b0     mibtbl.obj
 0003:00006618       ?audioEntryTable@@3PAVasiMibEntry@@A 10099618     mibtbl.obj
 0003:00006880       ?errorEntryTable@@3PAVasiMibEntry@@A 10099880     mibtbl.obj
 0003:00006928       ?udpEntryTable@@3PAVasiMibEntry@@A 10099928     mibtbl.obj
 0003:000069b8       ?mimonEntryTable@@3PAVasiMibEntry@@A 100999b8     mibtbl.obj
 0003:00006a44       ?txGroup@@3VasiMibGroup@@A 10099a44     mibtbl.obj
 0003:00006a60       ?ifEntryTable@@3PAVasiMibEntry@@A 10099a60     mibtbl.obj
 0003:00006d00       ?txEntryTable@@3PAVasiMibEntry@@A 10099d00     mibtbl.obj
 0003:00006ea8       ?sysEntryTable@@3PAVasiMibEntry@@A 10099ea8     mibtbl.obj
 0003:00006f88       ?stdGroup@@3VasiMibGroup@@A 10099f88     mibtbl.obj
 0003:00006fa0       ?serialGroup@@3VasiMibGroup@@A 10099fa0     mibtbl.obj
 0003:00006fb8       ?ipmonEntryTable@@3PAVasiMibEntry@@A 10099fb8     mibtbl.obj
 0003:00007044       ?audioGroup@@3VasiMibGroup@@A 1009a044     mibtbl.obj
 0003:0000705c       ?ipmonGroup@@3VasiMibGroup@@A 1009a05c     mibtbl.obj
 0003:00007074       ?mimonGroup@@3VasiMibGroup@@A 1009a074     mibtbl.obj
 0003:00007090       ?ipEntryTable@@3PAVasiMibEntry@@A 1009a090     mibtbl.obj
 0003:00007368       ?ifGroup@@3VasiMibGroup@@A 1009a368     mibtbl.obj
 0003:00007380       ?flashGroup@@3VasiMibGroup@@A 1009a380     mibtbl.obj
 0003:00007398       ?modeEntryTable@@3PAVasiMibEntry@@A 1009a398     mibtbl.obj
 0003:000073ec       ?snmpGroup@@3VasiMibGroup@@A 1009a3ec     mibtbl.obj
 0003:00007408       ?stdEntryTable@@3PAVasiMibEntry@@A 1009a408     mibtbl.obj
 0003:00007498       ?conductorEntryTable@@3PAVasiMibEntry@@A 1009a498     mibtbl.obj
 0003:000075b0       ?syncGroup@@3VasiMibGroup@@A 1009a5b0     mibtbl.obj
 0003:000075c8       ?serialEntryTable@@3PAVasiMibEntry@@A 1009a5c8     mibtbl.obj
 0003:000076a8       ?ifmEntryTable@@3PAVasiMibEntry@@A 1009a6a8     mibtbl.obj
 0003:0000776c       ?modeGroup@@3VasiMibGroup@@A 1009a76c     mibtbl.obj
 0003:00007784       ?conductorGroup@@3VasiMibGroup@@A 1009a784     mibtbl.obj
 0003:0000779c       ?sysGroup@@3VasiMibGroup@@A 1009a79c     mibtbl.obj
 0003:000077b4       ?firmwareGroup@@3VasiMibGroup@@A 1009a7b4     mibtbl.obj
 0003:000077cc       ?errorGroup@@3VasiMibGroup@@A 1009a7cc     mibtbl.obj
 0003:000077e8       ?firmwareEntryTable@@3PAVasiMibEntry@@A 1009a7e8     mibtbl.obj
 0003:00007938       ?flashEntryTable@@3PAVasiMibEntry@@A 1009a938     mibtbl.obj
 0003:00007a34       ?ifmGroup@@3VasiMibGroup@@A 1009aa34     mibtbl.obj
 0003:00007a4c       ?udpGroup@@3VasiMibGroup@@A 1009aa4c     mibtbl.obj
 0003:00007a68       __hmod__avdecc_lib_controller32_dll 1009aa68     avdecc-lib_controller32:avdecc-lib_controller32.dll
 0003:00007a6c       ___pfnDliNotifyHook2       1009aa6c     Delayimp:delayhk2.obj
 0003:00007a70       ___pfnDliFailureHook2      1009aa70     Delayimp:delayhk1.obj
 0003:00007d9c       ___fastflag                1009ad9c     LIBCMT:fpinit.obj
 0003:00007da4       __aenvptr                  1009ada4     LIBCMT:dllcrt0.obj
 0003:00007da8       __wenvptr                  1009ada8     LIBCMT:dllcrt0.obj
 0003:00007dac       ___mbcodepage              1009adac     LIBCMT:mbctype.obj
 0003:00007db0       ___ismbcodepage            1009adb0     LIBCMT:mbctype.obj
 0003:00007db4       ___mbulinfo                1009adb4     LIBCMT:mbctype.obj
 0003:00007dc0       ___mblocalename            1009adc0     LIBCMT:mbctype.obj
 0003:00007dc8       ___locale_changed          1009adc8     LIBCMT:wsetloca.obj
 0003:00007dcc       ___pInvalidArgHandler      1009adcc     LIBCMT:invarg.obj
 0003:00007dd0       ___isa_available           1009add0     LIBCMT:cpu_disp.obj
 0003:00007dd4       ___favor                   1009add4     LIBCMT:cpu_disp.obj
 0003:00007dd8       __crtheap                  1009add8     LIBCMT:heapinit.obj
 0003:00007ddc       ?_pnhHeap@@3P6AHI@ZA       1009addc     LIBCMT:handler.obj
 0003:00007de0       __C_Exit_Done              1009ade0     LIBCMT:crt0dat.obj
 0003:00007de4       ___argc                    1009ade4     LIBCMT:crt0dat.obj
 0003:00007de8       ___argv                    1009ade8     LIBCMT:crt0dat.obj
 0003:00007dec       ___wargv                   1009adec     LIBCMT:crt0dat.obj
 0003:00007df0       __environ                  1009adf0     LIBCMT:crt0dat.obj
 0003:00007df4       __wenviron                 1009adf4     LIBCMT:crt0dat.obj
 0003:00007df8       __pgmptr                   1009adf8     LIBCMT:crt0dat.obj
 0003:00007dfc       __wpgmptr                  1009adfc     LIBCMT:crt0dat.obj
 0003:00007e00       __umaskval                 1009ae00     LIBCMT:crt0dat.obj
 0003:00007e04       __exitflag                 1009ae04     LIBCMT:crt0dat.obj
 0003:00007e08       __C_Termination_Done       1009ae08     LIBCMT:crt0dat.obj
 0003:00007e0c       ___winitenv                1009ae0c     LIBCMT:crt0dat.obj
 0003:00007e10       ___initenv                 1009ae10     LIBCMT:crt0dat.obj
 0003:00007e18       ___app_type                1009ae18     LIBCMT:crt0msg.obj
 0003:00008448       __newmode                  1009b448     LIBCMT:_newmode.obj
 0003:0000844c       __cflush                   1009b44c     LIBCMT:_file.obj
 0003:00008450       __stdbuf                   1009b450     LIBCMT:_sftbuf.obj
 0003:00008460       ___pPurecall               1009b460     LIBCMT:inithelp.obj
 0003:00008464       __maxwait                  1009b464     LIBCMT:crtheap.obj
 0003:00008468       ?__pInconsistency@@3P6AXXZA 1009b468     LIBCMT:hooks.obj
 0003:0000846c       ?g_OutOfMemoryExceptionCallback@@3P6GPAXXZA 1009b46c     LIBCMT:frame.obj
 0003:000085c8       ___pioinfo                 1009b5c8     LIBCMT:ioinit.obj
 0003:000087d0       ___lconv_static_null       1009b7d0     LIBCMT:lconv.obj
 0003:000087d4       ___lconv_static_W_null     1009b7d4     LIBCMT:lconv.obj
 0003:000087f4       ___error_mode              1009b7f4     LIBCMT:errmode.obj
 0003:0000880c       ?pArgList@UnDecorator@@0PAVReplicator@@A 1009b80c     LIBCMT:undname.obj
 0003:00008810       ?pZNameList@UnDecorator@@0PAVReplicator@@A 1009b810     LIBCMT:undname.obj
 0003:00008814       ?pTemplateArgList@UnDecorator@@0PAVReplicator@@A 1009b814     LIBCMT:undname.obj
 0003:00008818       ?gName@UnDecorator@@0PBDB  1009b818     LIBCMT:undname.obj
 0003:0000881c       ?name@UnDecorator@@0PBDB   1009b81c     LIBCMT:undname.obj
 0003:00008820       ?outputString@UnDecorator@@0PADA 1009b820     LIBCMT:undname.obj
 0003:00008824       ?maxStringLength@UnDecorator@@0HA 1009b824     LIBCMT:undname.obj
 0003:00008828       ?disableFlags@UnDecorator@@0KA 1009b828     LIBCMT:undname.obj
 0003:0000882c       ?fExplicitTemplateParams@UnDecorator@@0_NA 1009b82c     LIBCMT:undname.obj
 0003:0000882d       ?fGetTemplateArgumentList@UnDecorator@@0_NA 1009b82d     LIBCMT:undname.obj
 0003:00008830       ?m_pGetParameter@UnDecorator@@0P6APADJ@ZA 1009b830     LIBCMT:undname.obj
 0003:00008848       ?nodes@?1??make@DNameStatusNode@@SAPAV2@W4DNameStatus@@@Z@4PAV2@A 1009b848     LIBCMT:undname.obj
 0003:00008878       ??_B?1??make@DNameStatusNode@@SAPAV1@W4DNameStatus@@@Z@51 1009b878     LIBCMT:undname.obj
 0003:0000887c       __outputformat             1009b87c     LIBCMT:outputformat.obj
 0003:00008880       __commode                  1009b880     LIBCMT:ncommode.obj
 0003:00008884       __fmode                    1009b884     LIBCMT:txtmode.obj
 0003:00008890       ___use_sse2_mathfcns       1009b890     <common>
 0003:00008894       __nhandle                  1009b894     <common>
 0003:00008898       __pmatherr                 1009b898     <common>
 0003:000088a0       __bufin                    1009b8a0     <common>
 0003:000098a0       ___piob                    1009c8a0     <common>
 0003:000098a4       __nstream                  1009c8a4     <common>
 0003:000098a8       ___dyn_tls_init_callback   1009c8a8     <common>
 0003:000098ac       ___onexitend               1009c8ac     <common>
 0003:000098b0       ___onexitbegin             1009c8b0     <common>
 0003:000098b4       ___mbctype_initialized     1009c8b4     <common>
 0003:000098b8       ___env_initialized         1009c8b8     <common>
 0003:000098bc       ___unguarded_readlc_active 1009c8bc     <common>
 0003:000098c0       ___setlc_active            1009c8c0     <common>
 0003:000098e0       _encodedKERNEL32Functions  1009c8e0     <common>
 0003:00009964       __debugger_hook_dummy      1009c964     <common>
 0003:00009968       __acmdln                   1009c968     <common>

 entry point at        0001:0003e19a

 Static symbols

 0002:fff98000       ?_System_object$initializer$@?$_Error_objects@H@std@@2P6AXXZA 10000000     libcpmt:xthrow.obj
 0002:fff98000       ?_Iostream_object$initializer$@?$_Error_objects@H@std@@2P6AXXZA 10000000     libcpmt:xthrow.obj
 0002:fff98000       ?_Generic_object$initializer$@?$_Error_objects@H@std@@2P6AXXZA 10000000     libcpmt:xthrow.obj
 0002:fff98000       __catchsym$?_Copy@?$basic_string@DU?$char_traits@D@std@@V?$allocator@D@2@@std@@QAEXII@Z$5 10000000     libcpmt:xthrow.obj
 0000:fff5a000       .debug$S                   10000000     dsound:DSOUND.dll
 0000:fff5a000       .debug$S                   10000000     wsock32:WSOCK32.dll
 0000:fff5a000       .debug$S                   10000000     wsock32:WSOCK32.dll
 0000:fff5a000       .debug$S                   10000000     dsound:DSOUND.dll
 0000:fff5a000       .debug$S                   10000000     wsnmp32:wsnmp32.dll
 0000:fff5a000       .debug$S                   10000000     wsnmp32:wsnmp32.dll
 0000:fff5a000       .debug$S                   10000000     wsnmp32:wsnmp32.dll
 0001:fffff000       __ehhandler$?_Copy@?$basic_string@DU?$char_traits@D@std@@V?$allocator@D@2@@std@@QAEXII@Z 10000000 f   libcpmt:xthrow.obj
 0000:fff5a000       .debug$S                   10000000     wsnmp32:wsnmp32.dll
 0000:fff5a000       .debug$S                   10000000     wsnmp32:wsnmp32.dll
 0000:fff5a000       .debug$S                   10000000     wsnmp32:wsnmp32.dll
 0000:fff5a000       .debug$S                   10000000     wsnmp32:wsnmp32.dll
 0000:fff5a000       .debug$S                   10000000     wsnmp32:wsnmp32.dll
 0000:fff5a000       .debug$S                   10000000     wsnmp32:wsnmp32.dll
 0002:fff98000       ?_System_object$initializer$@?$_Error_objects@H@std@@2P6AXXZA 10000000     libcpmt:syserror.obj
 0002:fff98000       ?_Iostream_object$initializer$@?$_Error_objects@H@std@@2P6AXXZA 10000000     libcpmt:syserror.obj
 0002:fff98000       ?_Generic_object$initializer$@?$_Error_objects@H@std@@2P6AXXZA 10000000     libcpmt:syserror.obj
 0002:fff98000       __catchsym$?_Copy@?$basic_string@DU?$char_traits@D@std@@V?$allocator@D@2@@std@@QAEXII@Z$5 10000000     libcpmt:syserror.obj
 0000:fff5a000       .debug$S                   10000000     wsnmp32:wsnmp32.dll
 0000:fff5a000       .debug$S                   10000000     wsnmp32:wsnmp32.dll
 0000:fff5a000       .debug$S                   10000000     wsnmp32:wsnmp32.dll
 0000:fff5a000       .debug$S                   10000000     wsnmp32:wsnmp32.dll
 0000:fff5a000       .debug$S                   10000000     wsnmp32:wsnmp32.dll
 0000:fff5a000       .debug$S                   10000000     wsnmp32:wsnmp32.dll
 0001:fffff000       __ehhandler$?_Copy@?$basic_string@DU?$char_traits@D@std@@V?$allocator@D@2@@std@@QAEXII@Z 10000000 f   libcpmt:syserror.obj
 0000:fff5a000       .debug$S                   10000000     wsnmp32:wsnmp32.dll
 0000:fff5a000       .debug$S                   10000000     wsnmp32:wsnmp32.dll
 0000:fff5a000       .debug$S                   10000000     wsnmp32:wsnmp32.dll
 0000:fff5a000       .debug$S                   10000000     wsnmp32:wsnmp32.dll
 0000:fff5a000       .debug$S                   10000000     wsnmp32:wsnmp32.dll
 0000:fff5a000       .debug$S                   10000000     wsnmp32:wsnmp32.dll
 0000:fff5a000       .debug$S                   10000000     wsnmp32:wsnmp32.dll
 0000:fff5a000       .debug$S                   10000000     wsnmp32:wsnmp32.dll
 0000:fff5a000       .debug$S                   10000000     wsnmp32:wsnmp32.dll
 0000:fff5a000       .debug$S                   10000000     wsnmp32:wsnmp32.dll
 0000:fff5a000       .debug$S                   10000000     wsnmp32:wsnmp32.dll
 0000:fff5a000       .debug$S                   10000000     wsnmp32:wsnmp32.dll
 0000:fff5a000       .debug$S                   10000000     dsound:DSOUND.dll
 0000:fff5a000       .debug$S                   10000000     asihpi32:ASIHPI32.dll
 0000:fff5a000       .debug$S                   10000000     asihpi32:ASIHPI32.dll
 0000:fff5a000       .debug$S                   10000000     asihpi32:ASIHPI32.dll
 0000:fff5a000       .debug$S                   10000000     asihpi32:ASIHPI32.dll
 0000:fff5a000       .debug$S                   10000000     asihpi32:ASIHPI32.dll
 0000:fff5a000       .debug$S                   10000000     asihpi32:ASIHPI32.dll
 0000:fff5a000       .debug$S                   10000000     asihpi32:ASIHPI32.dll
 0000:fff5a000       .debug$S                   10000000     asihpi32:ASIHPI32.dll
 0000:fff5a000       .debug$S                   10000000     asihpi32:ASIHPI32.dll
 0000:fff5a000       .debug$S                   10000000     asihpi32:ASIHPI32.dll
 0000:fff5a000       .debug$S                   10000000     asihpi32:ASIHPI32.dll
 0000:fff5a000       .debug$S                   10000000     asihpi32:ASIHPI32.dll
 0000:fff5a000       .debug$S                   10000000     asihpi32:ASIHPI32.dll
 0000:fff5a000       .debug$S                   10000000     asihpi32:ASIHPI32.dll
 0000:fff5a000       .debug$S                   10000000     asihpi32:ASIHPI32.dll
 0000:fff5a000       .debug$S                   10000000     asihpi32:ASIHPI32.dll
 0000:fff5a000       .debug$S                   10000000     asihpi32:ASIHPI32.dll
 0000:fff5a000       .debug$S                   10000000     asihpi32:ASIHPI32.dll
 0000:fff5a000       .debug$S                   10000000     asihpi32:ASIHPI32.dll
 0000:fff5a000       .debug$S                   10000000     asihpi32:ASIHPI32.dll
 0000:fff5a000       .debug$S                   10000000     asihpi32:ASIHPI32.dll
 0000:fff5a000       .debug$S                   10000000     asihpi32:ASIHPI32.dll
 0000:fff5a000       .debug$S                   10000000     asihpi32:ASIHPI32.dll
 0000:fff5a000       .debug$S                   10000000     asihpi32:ASIHPI32.dll
 0000:fff5a000       .debug$S                   10000000     asihpi32:ASIHPI32.dll
 0000:fff5a000       .debug$S                   10000000     asihpi32:ASIHPI32.dll
 0000:fff5a000       .debug$S                   10000000     asihpi32:ASIHPI32.dll
 0000:fff5a000       .debug$S                   10000000     asihpi32:ASIHPI32.dll
 0000:fff5a000       .debug$S                   10000000     asihpi32:ASIHPI32.dll
 0000:fff5a000       .debug$S                   10000000     asihpi32:ASIHPI32.dll
 0000:fff5a000       .debug$S                   10000000     asihpi32:ASIHPI32.dll
 0000:fff5a000       .debug$S                   10000000     asihpi32:ASIHPI32.dll
 0000:fff5a000       .debug$S                   10000000     asihpi32:ASIHPI32.dll
 0000:fff5a000       .debug$S                   10000000     asihpi32:ASIHPI32.dll
 0000:fff5a000       .debug$S                   10000000     asihpi32:ASIHPI32.dll
 0000:fff5a000       .debug$S                   10000000     asihpi32:ASIHPI32.dll
 0000:fff5a000       .debug$S                   10000000     asihpi32:ASIHPI32.dll
 0000:fff5a000       .debug$S                   10000000     asihpi32:ASIHPI32.dll
 0000:fff5a000       .debug$S                   10000000     asihpi32:ASIHPI32.dll
 0000:fff5a000       .debug$S                   10000000     asihpi32:ASIHPI32.dll
 0000:fff5a000       .debug$S                   10000000     asihpi32:ASIHPI32.dll
 0000:fff5a000       .debug$S                   10000000     asihpi32:ASIHPI32.dll
 0000:fff5a000       .debug$S                   10000000     asihpi32:ASIHPI32.dll
 0000:fff5a000       .debug$S                   10000000     asihpi32:ASIHPI32.dll
 0000:fff5a000       .debug$S                   10000000     asihpi32:ASIHPI32.dll
 0000:fff5a000       .debug$S                   10000000     asihpi32:ASIHPI32.dll
 0000:fff5a000       .debug$S                   10000000     asihpi32:ASIHPI32.dll
 0000:fff5a000       .debug$S                   10000000     asihpi32:ASIHPI32.dll
 0000:fff5a000       .debug$S                   10000000     asihpi32:ASIHPI32.dll
 0000:fff5a000       .debug$S                   10000000     asihpi32:ASIHPI32.dll
 0000:fff5a000       .debug$S                   10000000     asihpi32:ASIHPI32.dll
 0000:fff5a000       .debug$S                   10000000     asihpi32:ASIHPI32.dll
 0000:fff5a000       .debug$S                   10000000     asihpi32:ASIHPI32.dll
 0000:fff5a000       .debug$S                   10000000     asihpi32:ASIHPI32.dll
 0000:fff5a000       .debug$S                   10000000     asihpi32:ASIHPI32.dll
 0000:fff5a000       .debug$S                   10000000     asihpi32:ASIHPI32.dll
 0000:fff5a000       .debug$S                   10000000     asihpi32:ASIHPI32.dll
 0000:fff5a000       .debug$S                   10000000     asihpi32:ASIHPI32.dll
 0000:fff5a000       .debug$S                   10000000     asihpi32:ASIHPI32.dll
 0000:fff5a000       .debug$S                   10000000     asihpi32:ASIHPI32.dll
 0000:fff5a000       .debug$S                   10000000     asihpi32:ASIHPI32.dll
 0000:fff5a000       .debug$S                   10000000     asihpi32:ASIHPI32.dll
 0000:fff5a000       .debug$S                   10000000     asihpi32:ASIHPI32.dll
 0000:fff5a000       .debug$S                   10000000     asihpi32:ASIHPI32.dll
 0000:fff5a000       .debug$S                   10000000     asihpi32:ASIHPI32.dll
 0000:fff5a000       .debug$S                   10000000     asihpi32:ASIHPI32.dll
 0000:fff5a000       .debug$S                   10000000     asihpi32:ASIHPI32.dll
 0000:fff5a000       .debug$S                   10000000     asihpi32:ASIHPI32.dll
 0000:fff5a000       .debug$S                   10000000     asihpi32:ASIHPI32.dll
 0000:fff5a000       .debug$S                   10000000     asihpi32:ASIHPI32.dll
 0000:fff5a000       .debug$S                   10000000     asihpi32:ASIHPI32.dll
 0000:fff5a000       .debug$S                   10000000     asihpi32:ASIHPI32.dll
 0000:fff5a000       .debug$S                   10000000     asihpi32:ASIHPI32.dll
 0000:fff5a000       .debug$S                   10000000     asihpi32:ASIHPI32.dll
 0000:fff5a000       .debug$S                   10000000     asihpi32:ASIHPI32.dll
 0000:fff5a000       .debug$S                   10000000     asihpi32:ASIHPI32.dll
 0000:fff5a000       .debug$S                   10000000     asihpi32:ASIHPI32.dll
 0000:fff5a000       .debug$S                   10000000     asihpi32:ASIHPI32.dll
 0000:fff5a000       .debug$S                   10000000     asihpi32:ASIHPI32.dll
 0000:fff5a000       .debug$S                   10000000     asihpi32:ASIHPI32.dll
 0000:fff5a000       .debug$S                   10000000     asihpi32:ASIHPI32.dll
 0000:fff5a000       .debug$S                   10000000     asihpi32:ASIHPI32.dll
 0000:fff5a000       .debug$S                   10000000     asihpi32:ASIHPI32.dll
 0000:fff5a000       .debug$S                   10000000     asihpi32:ASIHPI32.dll
 0000:fff5a000       .debug$S                   10000000     asihpi32:ASIHPI32.dll
 0000:fff5a000       .debug$S                   10000000     asihpi32:ASIHPI32.dll
 0000:fff5a000       .debug$S                   10000000     asihpi32:ASIHPI32.dll
 0000:fff5a000       .debug$S                   10000000     asihpi32:ASIHPI32.dll
 0000:fff5a000       .debug$S                   10000000     asihpi32:ASIHPI32.dll
 0000:fff5a000       .debug$S                   10000000     asihpi32:ASIHPI32.dll
 0000:fff5a000       .debug$S                   10000000     asihpi32:ASIHPI32.dll
 0000:fff5a000       .debug$S                   10000000     asihpi32:ASIHPI32.dll
 0000:fff5a000       .debug$S                   10000000     asihpi32:ASIHPI32.dll
 0000:fff5a000       .debug$S                   10000000     asihpi32:ASIHPI32.dll
 0000:fff5a000       .debug$S                   10000000     asihpi32:ASIHPI32.dll
 0000:fff5a000       .debug$S                   10000000     asihpi32:ASIHPI32.dll
 0000:fff5a000       .debug$S                   10000000     asihpi32:ASIHPI32.dll
 0000:fff5a000       .debug$S                   10000000     asihpi32:ASIHPI32.dll
 0000:fff5a000       .debug$S                   10000000     asihpi32:ASIHPI32.dll
 0000:fff5a000       .debug$S                   10000000     asihpi32:ASIHPI32.dll
 0000:fff5a000       .debug$S                   10000000     asihpi32:ASIHPI32.dll
 0000:fff5a000       .debug$S                   10000000     asihpi32:ASIHPI32.dll
 0000:fff5a000       .debug$S                   10000000     asihpi32:ASIHPI32.dll
 0000:fff5a000       .debug$S                   10000000     asihpi32:ASIHPI32.dll
 0000:fff5a000       .debug$S                   10000000     asihpi32:ASIHPI32.dll
 0000:fff5a000       .debug$S                   10000000     asihpi32:ASIHPI32.dll
 0000:fff5a000       .debug$S                   10000000     asihpi32:ASIHPI32.dll
 0000:fff5a000       .debug$S                   10000000     asihpi32:ASIHPI32.dll
 0000:fff5a000       .debug$S                   10000000     asihpi32:ASIHPI32.dll
 0000:fff5a000       .debug$S                   10000000     asihpi32:ASIHPI32.dll
 0000:fff5a000       .debug$S                   10000000     asihpi32:ASIHPI32.dll
 0000:fff5a000       .debug$S                   10000000     asihpi32:ASIHPI32.dll
 0000:fff5a000       .debug$S                   10000000     asihpi32:ASIHPI32.dll
 0000:fff5a000       .debug$S                   10000000     asihpi32:ASIHPI32.dll
 0000:fff5a000       .debug$S                   10000000     asihpi32:ASIHPI32.dll
 0000:fff5a000       .debug$S                   10000000     asihpi32:ASIHPI32.dll
 0000:fff5a000       .debug$S                   10000000     asihpi32:ASIHPI32.dll
 0000:fff5a000       .debug$S                   10000000     asihpi32:ASIHPI32.dll
 0000:fff5a000       .debug$S                   10000000     asihpi32:ASIHPI32.dll
 0000:fff5a000       .debug$S                   10000000     asihpi32:ASIHPI32.dll
 0000:fff5a000       .debug$S                   10000000     asihpi32:ASIHPI32.dll
 0000:fff5a000       .debug$S                   10000000     asihpi32:ASIHPI32.dll
 0000:fff5a000       .debug$S                   10000000     asihpi32:ASIHPI32.dll
 0000:fff5a000       .debug$S                   10000000     asihpi32:ASIHPI32.dll
 0000:fff5a000       .debug$S                   10000000     asihpi32:ASIHPI32.dll
 0000:fff5a000       .debug$S                   10000000     asihpi32:ASIHPI32.dll
 0000:fff5a000       .debug$S                   10000000     asihpi32:ASIHPI32.dll
 0000:fff5a000       .debug$S                   10000000     asihpi32:ASIHPI32.dll
 0000:fff5a000       .debug$S                   10000000     asihpi32:ASIHPI32.dll
 0000:fff5a000       .debug$S                   10000000     asihpi32:ASIHPI32.dll
 0000:fff5a000       .debug$S                   10000000     asihpi32:ASIHPI32.dll
 0000:fff5a000       .debug$S                   10000000     asihpi32:ASIHPI32.dll
 0000:fff5a000       .debug$S                   10000000     asihpi32:ASIHPI32.dll
 0000:fff5a000       .debug$S                   10000000     asihpi32:ASIHPI32.dll
 0000:fff5a000       .debug$S                   10000000     asihpi32:ASIHPI32.dll
 0000:fff5a000       .debug$S                   10000000     asihpi32:ASIHPI32.dll
 0000:fff5a000       .debug$S                   10000000     asihpi32:ASIHPI32.dll
 0000:fff5a000       .debug$S                   10000000     asihpi32:ASIHPI32.dll
 0000:fff5a000       .debug$S                   10000000     asihpi32:ASIHPI32.dll
 0000:fff5a000       .debug$S                   10000000     asihpi32:ASIHPI32.dll
 0000:fff5a000       .debug$S                   10000000     asihpi32:ASIHPI32.dll
 0000:fff5a000       .debug$S                   10000000     asihpi32:ASIHPI32.dll
 0000:fff5a000       .debug$S                   10000000     asihpi32:ASIHPI32.dll
 0000:fff5a000       .debug$S                   10000000     asihpi32:ASIHPI32.dll
 0000:fff5a000       .debug$S                   10000000     asihpi32:ASIHPI32.dll
 0000:fff5a000       .debug$S                   10000000     asihpi32:ASIHPI32.dll
 0000:fff5a000       .debug$S                   10000000     asihpi32:ASIHPI32.dll
 0000:fff5a000       .debug$S                   10000000     asihpi32:ASIHPI32.dll
 0000:fff5a000       .debug$S                   10000000     asihpi32:ASIHPI32.dll
 0000:fff5a000       .debug$S                   10000000     asihpi32:ASIHPI32.dll
 0000:fff5a000       .debug$S                   10000000     asihpi32:ASIHPI32.dll
 0000:fff5a000       .debug$S                   10000000     asihpi32:ASIHPI32.dll
 0000:fff5a000       .debug$S                   10000000     asihpi32:ASIHPI32.dll
 0000:fff5a000       .debug$S                   10000000     asihpi32:ASIHPI32.dll
 0000:fff5a000       .debug$S                   10000000     asihpi32:ASIHPI32.dll
 0000:fff5a000       .debug$S                   10000000     asihpi32:ASIHPI32.dll
 0000:fff5a000       .debug$S                   10000000     asihpi32:ASIHPI32.dll
 0000:fff5a000       .debug$S                   10000000     asihpi32:ASIHPI32.dll
 0000:fff5a000       .debug$S                   10000000     asihpi32:ASIHPI32.dll
 0000:fff5a000       .debug$S                   10000000     asihpi32:ASIHPI32.dll
 0000:fff5a000       .debug$S                   10000000     asihpi32:ASIHPI32.dll
 0000:fff5a000       .debug$S                   10000000     asihpi32:ASIHPI32.dll
 0000:fff5a000       .debug$S                   10000000     asihpi32:ASIHPI32.dll
 0000:fff5a000       .debug$S                   10000000     asihpi32:ASIHPI32.dll
 0000:fff5a000       .debug$S                   10000000     asihpi32:ASIHPI32.dll
 0000:fff5a000       .debug$S                   10000000     asihpi32:ASIHPI32.dll
 0000:fff5a000       .debug$S                   10000000     asihpi32:ASIHPI32.dll
 0000:fff5a000       .debug$S                   10000000     asihpi32:ASIHPI32.dll
 0000:fff5a000       .debug$S                   10000000     asihpi32:ASIHPI32.dll
 0000:fff5a000       .debug$S                   10000000     asihpi32:ASIHPI32.dll
 0000:fff5a000       .debug$S                   10000000     asihpi32:ASIHPI32.dll
 0000:fff5a000       .debug$S                   10000000     asihpi32:ASIHPI32.dll
 0000:fff5a000       .debug$S                   10000000     asihpi32:ASIHPI32.dll
 0000:fff5a000       .debug$S                   10000000     asihpi32:ASIHPI32.dll
 0000:fff5a000       .debug$S                   10000000     asihpi32:ASIHPI32.dll
 0000:fff5a000       .debug$S                   10000000     asihpi32:ASIHPI32.dll
 0000:fff5a000       .debug$S                   10000000     asihpi32:ASIHPI32.dll
 0000:fff5a000       .debug$S                   10000000     asihpi32:ASIHPI32.dll
 0000:fff5a000       .debug$S                   10000000     asihpi32:ASIHPI32.dll
 0000:fff5a000       .debug$S                   10000000     asihpi32:ASIHPI32.dll
 0000:fff5a000       .debug$S                   10000000     asihpi32:ASIHPI32.dll
 0000:fff5a000       .debug$S                   10000000     asihpi32:ASIHPI32.dll
 0000:fff5a000       .debug$S                   10000000     asihpi32:ASIHPI32.dll
 0000:fff5a000       .debug$S                   10000000     asihpi32:ASIHPI32.dll
 0000:fff5a000       .debug$S                   10000000     asihpi32:ASIHPI32.dll
 0000:fff5a000       .debug$S                   10000000     asihpi32:ASIHPI32.dll
 0000:fff5a000       .debug$S                   10000000     asihpi32:ASIHPI32.dll
 0000:fff5a000       .debug$S                   10000000     asihpi32:ASIHPI32.dll
 0000:fff5a000       .debug$S                   10000000     asihpi32:ASIHPI32.dll
 0000:fff5a000       .debug$S                   10000000     asihpi32:ASIHPI32.dll
 0000:fff5a000       .debug$S                   10000000     asihpi32:ASIHPI32.dll
 0000:fff5a000       .debug$S                   10000000     asihpi32:ASIHPI32.dll
 0000:fff5a000       .debug$S                   10000000     avdecc-lib_controller32:avdecc-lib_controller32.dll
 0000:fff5a000       .debug$S                   10000000     winmm:WINMM.dll
 0000:fff5a000       .debug$S                   10000000     winmm:WINMM.dll
 0000:fff5a000       .debug$S                   10000000     winmm:WINMM.dll
 0000:fff5a000       .debug$S                   10000000     winmm:WINMM.dll
 0000:fff5a000       .debug$S                   10000000     winmm:WINMM.dll
 0000:fff5a000       .debug$S                   10000000     winmm:WINMM.dll
 0000:fff5a000       .debug$S                   10000000     winmm:WINMM.dll
 0000:fff5a000       .debug$S                   10000000     winmm:WINMM.dll
 0000:fff5a000       .debug$S                   10000000     winmm:WINMM.dll
 0000:fff5a000       .debug$S                   10000000     winmm:WINMM.dll
 0000:fff5a000       .debug$S                   10000000     winmm:WINMM.dll
 0000:fff5a000       .debug$S                   10000000     winmm:WINMM.dll
 0000:fff5a000       .debug$S                   10000000     winmm:WINMM.dll
 0000:fff5a000       .debug$S                   10000000     winmm:WINMM.dll
 0000:fff5a000       .debug$S                   10000000     winmm:WINMM.dll
 0000:fff5a000       .debug$S                   10000000     winmm:WINMM.dll
 0000:fff5a000       .debug$S                   10000000     winmm:WINMM.dll
 0000:fff5a000       .debug$S                   10000000     winmm:WINMM.dll
 0000:fff5a000       .debug$S                   10000000     winmm:WINMM.dll
 0000:fff5a000       .debug$S                   10000000     winmm:WINMM.dll
 0000:fff5a000       .debug$S                   10000000     winmm:WINMM.dll
 0000:fff5a000       .debug$S                   10000000     winmm:WINMM.dll
 0000:fff5a000       .debug$S                   10000000     winmm:WINMM.dll
 0000:fff5a000       .debug$S                   10000000     winmm:WINMM.dll
 0000:fff5a000       .debug$S                   10000000     winmm:WINMM.dll
 0000:fff5a000       .debug$S                   10000000     winmm:WINMM.dll
 0000:fff5a000       .debug$S                   10000000     winmm:WINMM.dll
 0000:fff5a000       .debug$S                   10000000     winmm:WINMM.dll
 0000:fff5a000       .debug$S                   10000000     winmm:WINMM.dll
 0000:fff5a000       .debug$S                   10000000     winmm:WINMM.dll
 0000:fff5a000       .debug$S                   10000000     winmm:WINMM.dll
 0000:fff5a000       .debug$S                   10000000     winmm:WINMM.dll
 0000:fff5a000       .debug$S                   10000000     winmm:WINMM.dll
 0000:fff5a000       .debug$S                   10000000     winmm:WINMM.dll
 0000:fff5a000       .debug$S                   10000000     winmm:WINMM.dll
 0000:fff5a000       .debug$S                   10000000     winmm:WINMM.dll
 0000:fff5a000       .debug$S                   10000000     winmm:WINMM.dll
 0000:fff5a000       .debug$S                   10000000     winmm:WINMM.dll
 0000:fff5a000       .debug$S                   10000000     winmm:WINMM.dll
 0000:fff5a000       .debug$S                   10000000     avdecc-lib_controller32:avdecc-lib_controller32.dll
 0000:fff5a000       .debug$S                   10000000     avdecc-lib_controller32:avdecc-lib_controller32.dll
 0000:fff5a000       .debug$S                   10000000     avdecc-lib_controller32:avdecc-lib_controller32.dll
 0000:fff5a000       .debug$S                   10000000     avdecc-lib_controller32:avdecc-lib_controller32.dll
 0000:fff5a000       .debug$S                   10000000     avdecc-lib_controller32:avdecc-lib_controller32.dll
 0000:fff5a000       .debug$S                   10000000     avdecc-lib_controller32:avdecc-lib_controller32.dll
 0000:fff5a000       .debug$S                   10000000     avdecc-lib_controller32:avdecc-lib_controller32.dll
 0000:fff5a000       .debug$S                   10000000     avdecc-lib_controller32:avdecc-lib_controller32.dll
 0000:fff5a000       .debug$S                   10000000     kernel32:KERNEL32.dll
 0000:fff5a000       .debug$S                   10000000     kernel32:KERNEL32.dll
 0000:fff5a000       .debug$S                   10000000     kernel32:KERNEL32.dll
 0000:fff5a000       .debug$S                   10000000     kernel32:KERNEL32.dll
 0000:fff5a000       .debug$S                   10000000     kernel32:KERNEL32.dll
 0000:fff5a000       .debug$S                   10000000     kernel32:KERNEL32.dll
 0000:fff5a000       .debug$S                   10000000     kernel32:KERNEL32.dll
 0000:fff5a000       .debug$S                   10000000     kernel32:KERNEL32.dll
 0000:fff5a000       .debug$S                   10000000     kernel32:KERNEL32.dll
 0000:fff5a000       .debug$S                   10000000     kernel32:KERNEL32.dll
 0000:fff5a000       .debug$S                   10000000     kernel32:KERNEL32.dll
 0000:fff5a000       .debug$S                   10000000     kernel32:KERNEL32.dll
 0000:fff5a000       .debug$S                   10000000     kernel32:KERNEL32.dll
 0000:fff5a000       .debug$S                   10000000     kernel32:KERNEL32.dll
 0000:fff5a000       .debug$S                   10000000     kernel32:KERNEL32.dll
 0000:fff5a000       .debug$S                   10000000     kernel32:KERNEL32.dll
 0000:fff5a000       .debug$S                   10000000     kernel32:KERNEL32.dll
 0000:fff5a000       .debug$S                   10000000     kernel32:KERNEL32.dll
 0000:fff5a000       .debug$S                   10000000     kernel32:KERNEL32.dll
 0000:fff5a000       .debug$S                   10000000     kernel32:KERNEL32.dll
 0000:fff5a000       .debug$S                   10000000     kernel32:KERNEL32.dll
 0000:fff5a000       .debug$S                   10000000     kernel32:KERNEL32.dll
 0000:fff5a000       .debug$S                   10000000     kernel32:KERNEL32.dll
 0000:fff5a000       .debug$S                   10000000     kernel32:KERNEL32.dll
 0000:fff5a000       .debug$S                   10000000     kernel32:KERNEL32.dll
 0000:fff5a000       .debug$S                   10000000     kernel32:KERNEL32.dll
 0000:fff5a000       .debug$S                   10000000     kernel32:KERNEL32.dll
 0000:fff5a000       .debug$S                   10000000     kernel32:KERNEL32.dll
 0000:fff5a000       .debug$S                   10000000     kernel32:KERNEL32.dll
 0000:fff5a000       .debug$S                   10000000     kernel32:KERNEL32.dll
 0000:fff5a000       .debug$S                   10000000     kernel32:KERNEL32.dll
 0000:fff5a000       .debug$S                   10000000     kernel32:KERNEL32.dll
 0000:fff5a000       .debug$S                   10000000     kernel32:KERNEL32.dll
 0000:fff5a000       .debug$S                   10000000     kernel32:KERNEL32.dll
 0000:fff5a000       .debug$S                   10000000     kernel32:KERNEL32.dll
 0000:fff5a000       .debug$S                   10000000     kernel32:KERNEL32.dll
 0000:fff5a000       .debug$S                   10000000     kernel32:KERNEL32.dll
 0000:fff5a000       .debug$S                   10000000     kernel32:KERNEL32.dll
 0000:fff5a000       .debug$S                   10000000     kernel32:KERNEL32.dll
 0000:fff5a000       .debug$S                   10000000     kernel32:KERNEL32.dll
 0000:fff5a000       .debug$S                   10000000     kernel32:KERNEL32.dll
 0000:fff5a000       .debug$S                   10000000     kernel32:KERNEL32.dll
 0000:fff5a000       .debug$S                   10000000     kernel32:KERNEL32.dll
 0000:fff5a000       .debug$S                   10000000     kernel32:KERNEL32.dll
 0000:fff5a000       .debug$S                   10000000     kernel32:KERNEL32.dll
 0000:fff5a000       .debug$S                   10000000     kernel32:KERNEL32.dll
 0000:fff5a000       .debug$S                   10000000     kernel32:KERNEL32.dll
 0000:fff5a000       .debug$S                   10000000     kernel32:KERNEL32.dll
 0000:fff5a000       .debug$S                   10000000     kernel32:KERNEL32.dll
 0000:fff5a000       .debug$S                   10000000     kernel32:KERNEL32.dll
 0000:fff5a000       .debug$S                   10000000     kernel32:KERNEL32.dll
 0000:fff5a000       .debug$S                   10000000     kernel32:KERNEL32.dll
 0000:fff5a000       .debug$S                   10000000     kernel32:KERNEL32.dll
 0000:fff5a000       .debug$S                   10000000     kernel32:KERNEL32.dll
 0000:fff5a000       .debug$S                   10000000     kernel32:KERNEL32.dll
 0000:fff5a000       .debug$S                   10000000     kernel32:KERNEL32.dll
 0000:fff5a000       .debug$S                   10000000     kernel32:KERNEL32.dll
 0000:fff5a000       .debug$S                   10000000     kernel32:KERNEL32.dll
 0000:fff5a000       .debug$S                   10000000     kernel32:KERNEL32.dll
 0000:fff5a000       .debug$S                   10000000     kernel32:KERNEL32.dll
 0000:fff5a000       .debug$S                   10000000     kernel32:KERNEL32.dll
 0000:fff5a000       .debug$S                   10000000     kernel32:KERNEL32.dll
 0000:fff5a000       .debug$S                   10000000     kernel32:KERNEL32.dll
 0000:fff5a000       .debug$S                   10000000     kernel32:KERNEL32.dll
 0000:fff5a000       .debug$S                   10000000     kernel32:KERNEL32.dll
 0000:fff5a000       .debug$S                   10000000     kernel32:KERNEL32.dll
 0000:fff5a000       .debug$S                   10000000     kernel32:KERNEL32.dll
 0000:fff5a000       .debug$S                   10000000     kernel32:KERNEL32.dll
 0000:fff5a000       .debug$S                   10000000     kernel32:KERNEL32.dll
 0000:fff5a000       .debug$S                   10000000     kernel32:KERNEL32.dll
 0000:fff5a000       .debug$S                   10000000     kernel32:KERNEL32.dll
 0000:fff5a000       .debug$S                   10000000     kernel32:KERNEL32.dll
 0000:fff5a000       .debug$S                   10000000     kernel32:KERNEL32.dll
 0000:fff5a000       .debug$S                   10000000     kernel32:KERNEL32.dll
 0000:fff5a000       .debug$S                   10000000     kernel32:KERNEL32.dll
 0000:fff5a000       .debug$S                   10000000     kernel32:KERNEL32.dll
 0000:fff5a000       .debug$S                   10000000     kernel32:KERNEL32.dll
 0000:fff5a000       .debug$S                   10000000     kernel32:KERNEL32.dll
 0000:fff5a000       .debug$S                   10000000     kernel32:KERNEL32.dll
 0000:fff5a000       .debug$S                   10000000     kernel32:KERNEL32.dll
 0000:fff5a000       .debug$S                   10000000     kernel32:KERNEL32.dll
 0000:fff5a000       .debug$S                   10000000     kernel32:KERNEL32.dll
 0000:fff5a000       .debug$S                   10000000     kernel32:KERNEL32.dll
 0000:fff5a000       .debug$S                   10000000     kernel32:KERNEL32.dll
 0000:fff5a000       .debug$S                   10000000     kernel32:KERNEL32.dll
 0000:fff5a000       .debug$S                   10000000     kernel32:KERNEL32.dll
 0000:fff5a000       .debug$S                   10000000     kernel32:KERNEL32.dll
 0000:fff5a000       .debug$S                   10000000     kernel32:KERNEL32.dll
 0000:fff5a000       .debug$S                   10000000     kernel32:KERNEL32.dll
 0000:fff5a000       .debug$S                   10000000     kernel32:KERNEL32.dll
 0000:fff5a000       .debug$S                   10000000     kernel32:KERNEL32.dll
 0000:fff5a000       .debug$S                   10000000     kernel32:KERNEL32.dll
 0000:fff5a000       .debug$S                   10000000     kernel32:KERNEL32.dll
 0000:fff5a000       .debug$S                   10000000     kernel32:KERNEL32.dll
 0000:fff5a000       .debug$S                   10000000     kernel32:KERNEL32.dll
 0000:fff5a000       .debug$S                   10000000     kernel32:KERNEL32.dll
 0000:fff5a000       .debug$S                   10000000     kernel32:KERNEL32.dll
 0000:fff5a000       .debug$S                   10000000     kernel32:KERNEL32.dll
 0000:fff5a000       .debug$S                   10000000     kernel32:KERNEL32.dll
 0000:fff5a000       .debug$S                   10000000     kernel32:KERNEL32.dll
 0000:fff5a000       .debug$S                   10000000     user32:USER32.dll
 0000:fff5a000       .debug$S                   10000000     user32:USER32.dll
 0000:fff5a000       .debug$S                   10000000     user32:USER32.dll
 0000:fff5a000       .debug$S                   10000000     advapi32:ADVAPI32.dll
 0000:fff5a000       .debug$S                   10000000     advapi32:ADVAPI32.dll
 0000:fff5a000       .debug$S                   10000000     advapi32:ADVAPI32.dll
 0000:fff5a000       .debug$S                   10000000     advapi32:ADVAPI32.dll
 0000:fff5a000       .debug$S                   10000000     advapi32:ADVAPI32.dll
 0000:fff5a000       .debug$S                   10000000     advapi32:ADVAPI32.dll
 0000:fff5a000       .debug$S                   10000000     advapi32:ADVAPI32.dll
 0000:fff5a000       .debug$S                   10000000     advapi32:ADVAPI32.dll
 0000:fff5a000       .debug$S                   10000000     ole32:ole32.dll
 0000:fff5a000       .debug$S                   10000000     ole32:ole32.dll
 0000:fff5a000       .debug$S                   10000000     ole32:ole32.dll
 0002:fff98000       __unwindtable$??_GasxCobranetTxContainer@@UAEPAXI@Z 10000000     asxsnmp.obj
 0002:fff98000       __unwindtable$??1asxCobranetTxContainer@@UAE@XZ 10000000     asxsnmp.obj
 0002:fff98000       __unwindtable$??_GasxCobranetRxContainer@@UAEPAXI@Z 10000000     asxsnmp.obj
 0002:fff98000       __unwindtable$??1asxCobranetRxContainer@@UAE@XZ 10000000     asxsnmp.obj
 0002:fff98000       __unwindtable$??_GasxCobranetContainer@@UAEPAXI@Z 10000000     asxsnmp.obj
 0002:fff98000       __unwindtable$??1asxCobranetContainer@@UAE@XZ 10000000     asxsnmp.obj
 0000:fff5a000       .debug$S                   10000000     dsound:DSOUND.dll
 0001:fffff000       __unwindfunclet$??_GasxCobranetTxContainer@@UAEPAXI@Z$0 10000000 f   asxsnmp.obj
 0001:fffff000       __unwindfunclet$??1asxCobranetTxContainer@@UAE@XZ$0 10000000 f   asxsnmp.obj
 0001:fffff000       __unwindfunclet$??_GasxCobranetRxContainer@@UAEPAXI@Z$0 10000000 f   asxsnmp.obj
 0001:fffff000       __unwindfunclet$??1asxCobranetRxContainer@@UAE@XZ$0 10000000 f   asxsnmp.obj
 0001:fffff000       __unwindfunclet$??_GasxCobranetContainer@@UAEPAXI@Z$0 10000000 f   asxsnmp.obj
 0001:fffff000       __unwindfunclet$??1asxCobranetContainer@@UAE@XZ$0 10000000 f   asxsnmp.obj
 0002:fff98000       __unwindtable$??_GasxBlock@@UAEPAXI@Z 10000000     asxtr800.obj
 0002:fff98000       __unwindtable$??1asxBlock@@UAE@XZ 10000000     asxtr800.obj
 0001:fffff000       __unwindfunclet$??_GasxBlock@@UAEPAXI@Z$0 10000000 f   asxtr800.obj
 0001:fffff000       __unwindfunclet$??1asxBlock@@UAE@XZ$0 10000000 f   asxtr800.obj
 0002:fff98000       __unwindtable$??_GasxCobranetContainer@@UAEPAXI@Z 10000000     asxwave.obj
 0002:fff98000       __unwindtable$??1asxCobranetContainer@@UAE@XZ 10000000     asxwave.obj
 0002:fff98000       __unwindtable$??_GasxTuner@@UAEPAXI@Z 10000000     asxwave.obj
 0002:fff98000       __unwindtable$??1asxTuner@@UAE@XZ 10000000     asxwave.obj
 0002:fff98000       __unwindtable$??_GasxMode@@UAEPAXI@Z 10000000     asxwave.obj
 0002:fff98000       __unwindtable$??1asxMode@@UAE@XZ 10000000     asxwave.obj
 0002:fff98000       __unwindtable$??_GasxMux@@UAEPAXI@Z 10000000     asxwave.obj
 0002:fff98000       __unwindtable$??1asxMux@@UAE@XZ 10000000     asxwave.obj
 0001:fffff000       __unwindfunclet$??_GasxCobranetContainer@@UAEPAXI@Z$0 10000000 f   asxwave.obj
 0001:fffff000       __unwindfunclet$??1asxCobranetContainer@@UAE@XZ$0 10000000 f   asxwave.obj
 0001:fffff000       __unwindfunclet$??_GasxTuner@@UAEPAXI@Z$0 10000000 f   asxwave.obj
 0001:fffff000       __unwindfunclet$??1asxTuner@@UAE@XZ$0 10000000 f   asxwave.obj
 0001:fffff000       __unwindfunclet$??_GasxMode@@UAEPAXI@Z$0 10000000 f   asxwave.obj
 0001:fffff000       __unwindfunclet$??1asxMode@@UAE@XZ$0 10000000 f   asxwave.obj
 0001:fffff000       __unwindfunclet$??_GasxMux@@UAEPAXI@Z$0 10000000 f   asxwave.obj
 0001:fffff000       __unwindfunclet$??1asxMux@@UAE@XZ$0 10000000 f   asxwave.obj
 0002:fff98008       __ehfuncinfo$??1asxCobranetRxContainer@@UAE@XZ 10000008     asxsnmp.obj
 0001:fffff008       __ehhandler$??_GasxCobranetRxContainer@@UAEPAXI@Z 10000008 f   asxsnmp.obj
 0001:fffff008       __ehhandler$??_GasxCobranetContainer@@UAEPAXI@Z 10000008 f   asxwave.obj
 0001:fffff008       __ehhandler$??1asxCobranetRxContainer@@UAE@XZ 10000008 f   asxsnmp.obj
 0001:fffff008       __ehhandler$??1asxCobranetContainer@@UAE@XZ 10000008 f   asxwave.obj
 0001:fffff008       __ehhandler$??_GasxCobranetContainer@@UAEPAXI@Z 10000008 f   asxsnmp.obj
 0002:fff98008       __ehfuncinfo$??_GasxCobranetTxContainer@@UAEPAXI@Z 10000008     asxsnmp.obj
 0001:fffff008       __ehhandler$??1asxCobranetContainer@@UAE@XZ 10000008 f   asxsnmp.obj
 0002:fff98008       __ehfuncinfo$??1asxCobranetTxContainer@@UAE@XZ 10000008     asxsnmp.obj
 0001:fffff008       __unwindfunclet$??_GasxTuner@@UAEPAXI@Z$1 10000008 f   asxwave.obj
 0002:fff98008       __ehfuncinfo$??_GasxBlock@@UAEPAXI@Z 10000008     asxtr800.obj
 0002:fff98008       __ehfuncinfo$??1asxBlock@@UAE@XZ 10000008     asxtr800.obj
 0001:fffff008       __unwindfunclet$??1asxTuner@@UAE@XZ$1 10000008 f   asxwave.obj
 0001:fffff008       __ehhandler$??_GasxCobranetTxContainer@@UAEPAXI@Z 10000008 f   asxsnmp.obj
 0001:fffff008       __ehhandler$??_GasxBlock@@UAEPAXI@Z 10000008 f   asxtr800.obj
 0001:fffff008       __ehhandler$??_GasxMode@@UAEPAXI@Z 10000008 f   asxwave.obj
 0001:fffff008       __ehhandler$??1asxMode@@UAE@XZ 10000008 f   asxwave.obj
 0001:fffff008       __unwindfunclet$??_GasxMux@@UAEPAXI@Z$1 10000008 f   asxwave.obj
 0001:fffff008       __ehhandler$??1asxBlock@@UAE@XZ 10000008 f   asxtr800.obj
 0001:fffff008       __unwindfunclet$??1asxMux@@UAE@XZ$1 10000008 f   asxwave.obj
 0002:fff98008       __ehfuncinfo$??_GasxCobranetContainer@@UAEPAXI@Z 10000008     asxwave.obj
 0002:fff98008       __ehfuncinfo$??1asxCobranetContainer@@UAE@XZ 10000008     asxwave.obj
 0002:fff98008       __ehfuncinfo$??_GasxCobranetRxContainer@@UAEPAXI@Z 10000008     asxsnmp.obj
 0002:fff98008       __ehfuncinfo$??_GasxMode@@UAEPAXI@Z 10000008     asxwave.obj
 0002:fff98008       __ehfuncinfo$??_GasxCobranetContainer@@UAEPAXI@Z 10000008     asxsnmp.obj
 0001:fffff008       __ehhandler$??1asxCobranetTxContainer@@UAE@XZ 10000008 f   asxsnmp.obj
 0002:fff98008       __ehfuncinfo$??1asxCobranetContainer@@UAE@XZ 10000008     asxsnmp.obj
 0002:fff98008       __ehfuncinfo$??1asxMode@@UAE@XZ 10000008     asxwave.obj
 0002:fff98010       __ehfuncinfo$??1asxMux@@UAE@XZ 10000010     asxwave.obj
 0002:fff98010       __catchsym$?_Copy@?$basic_string@DU?$char_traits@D@std@@V?$allocator@D@2@@std@@QAEXII@Z$4 10000010     libcpmt:xthrow.obj
 0002:fff98010       __ehfuncinfo$??_GasxMux@@UAEPAXI@Z 10000010     asxwave.obj
 0002:fff98010       __ehfuncinfo$??_GasxTuner@@UAEPAXI@Z 10000010     asxwave.obj
 0002:fff98010       __catchsym$?_Copy@?$basic_string@DU?$char_traits@D@std@@V?$allocator@D@2@@std@@QAEXII@Z$4 10000010     libcpmt:syserror.obj
 0002:fff98010       __ehfuncinfo$??1asxTuner@@UAE@XZ 10000010     asxwave.obj
 0001:fffff013       __ehhandler$??_GasxTuner@@UAEPAXI@Z 10000013 f   asxwave.obj
 0001:fffff013       __ehhandler$??1asxTuner@@UAE@XZ 10000013 f   asxwave.obj
 0001:fffff013       __ehhandler$??_GasxMux@@UAEPAXI@Z 10000013 f   asxwave.obj
 0001:fffff013       __ehhandler$??1asxMux@@UAE@XZ 10000013 f   asxwave.obj
 0002:fff98020       __unwindtable$?_Copy@?$basic_string@DU?$char_traits@D@std@@V?$allocator@D@2@@std@@QAEXII@Z 10000020     libcpmt:xthrow.obj
 0002:fff98020       __unwindtable$?_Copy@?$basic_string@DU?$char_traits@D@std@@V?$allocator@D@2@@std@@QAEXII@Z 10000020     libcpmt:syserror.obj
 0001:fffff03c       $LN11                      1000003c     asxsnmp.obj
 0002:fff98040       __ehfuncinfo$?_Copy@?$basic_string@DU?$char_traits@D@std@@V?$allocator@D@2@@std@@QAEXII@Z 10000040     libcpmt:syserror.obj
 0002:fff98040       __ehfuncinfo$?_Copy@?$basic_string@DU?$char_traits@D@std@@V?$allocator@D@2@@std@@QAEXII@Z 10000040     libcpmt:xthrow.obj
 0001:fffff063       __catch$?_Copy@?$basic_string@DU?$char_traits@D@std@@V?$allocator@D@2@@std@@QAEXII@Z$0 10000063 f   libcpmt:xthrow.obj
 0001:fffff063       __catch$?_Copy@?$basic_string@DU?$char_traits@D@std@@V?$allocator@D@2@@std@@QAEXII@Z$0 10000063 f   libcpmt:syserror.obj
 0002:fff98064       __tryblocktable$?_Copy@?$basic_string@DU?$char_traits@D@std@@V?$allocator@D@2@@std@@QAEXII@Z 10000064     libcpmt:syserror.obj
 0002:fff98064       __tryblocktable$?_Copy@?$basic_string@DU?$char_traits@D@std@@V?$allocator@D@2@@std@@QAEXII@Z 10000064     libcpmt:xthrow.obj
 0001:fffff0a4       $LN23                      100000a4     asxsnmp.obj
 0001:fffff0e2       __catch$?_Copy@?$basic_string@DU?$char_traits@D@std@@V?$allocator@D@2@@std@@QAEXII@Z$1 100000e2 f   libcpmt:xthrow.obj
 0001:fffff0e2       __catch$?_Copy@?$basic_string@DU?$char_traits@D@std@@V?$allocator@D@2@@std@@QAEXII@Z$1 100000e2 f   libcpmt:syserror.obj
 0001:00000000       ??__E?_Generic_object@?$_Error_objects@H@std@@2V_Generic_error_category@2@A@@YAXXZ 10001000 f   asxavdecc.obj
 0001:00000010       ??__E?_Iostream_object@?$_Error_objects@H@std@@2V_Iostream_error_category@2@A@@YAXXZ 10001010 f   asxavdecc.obj
 0001:00000020       ??__E?_System_object@?$_Error_objects@H@std@@2V_System_error_category@2@A@@YAXXZ 10001020 f   asxavdecc.obj
 0001:00000030       ??__EasxDebug@@YAXXZ       10001030 f   asxdebug.obj
 0001:00000040       ??__E?audioMetersOid@CobraNetNode@@0VasiOID@@A@@YAXXZ 10001040 f   cobranet.obj
 0001:00000050       ??__E?conductorPriorityOID@CobraNetNode@@0VasiOID@@A@@YAXXZ 10001050 f   cobranet.obj
 0001:00000060       ??__E?conductorStatusOID@CobraNetNode@@0VasiOID@@A@@YAXXZ 10001060 f   cobranet.obj
 0001:00000070       ??__E?errorCountOID@CobraNetNode@@0VasiOID@@A@@YAXXZ 10001070 f   cobranet.obj
 0001:00000080       ??__E?errorDisplayOID@CobraNetNode@@0VasiOID@@A@@YAXXZ 10001080 f   cobranet.obj
 0001:00000090       ??__E?errorLastOID@CobraNetNode@@0VasiOID@@A@@YAXXZ 10001090 f   cobranet.obj
 0001:000000a0       ??__E?firmwareMajorVersionOID@CobraNetNode@@0VasiOID@@A@@YAXXZ 100010a0 f   cobranet.obj
 0001:000000b0       ??__E?firmwareMinorVersionOID@CobraNetNode@@0VasiOID@@A@@YAXXZ 100010b0 f   cobranet.obj
 0001:000000c0       ??__E?flashPersistEnableOID@CobraNetNode@@0VasiOID@@A@@YAXXZ 100010c0 f   cobranet.obj
 0001:000000d0       ??__E?ipmonCurrentIpOID@CobraNetNode@@0VasiOID@@A@@YAXXZ 100010d0 f   cobranet.obj
 0001:000000e0       ??__E?ipmonStaticIpOID@CobraNetNode@@0VasiOID@@A@@YAXXZ 100010e0 f   cobranet.obj
 0001:000000f0       ??__E?modeRateControlOID@CobraNetNode@@0VasiOID@@A@@YAXXZ 100010f0 f   cobranet.obj
 0001:00000100       ??__E?modeRateStatusOID@CobraNetNode@@0VasiOID@@A@@YAXXZ 10001100 f   cobranet.obj
 0001:00000110       ??__E?rxBundleOid@CobraNetNode@@0VasiOID@@A@@YAXXZ 10001110 f   cobranet.obj
 0001:00000120       ??__E?rxDelayOid@CobraNetNode@@0VasiOID@@A@@YAXXZ 10001120 f   cobranet.obj
 0001:00000130       ??__E?rxDropoutsOid@CobraNetNode@@0VasiOID@@A@@YAXXZ 10001130 f   cobranet.obj
 0001:00000140       ??__E?rxMinDelayOid@CobraNetNode@@0VasiOID@@A@@YAXXZ 10001140 f   cobranet.obj
 0001:00000150       ??__E?rxPriorityOid@CobraNetNode@@0VasiOID@@A@@YAXXZ 10001150 f   cobranet.obj
 0001:00000160       ??__E?rxSourceMACOid@CobraNetNode@@0VasiOID@@A@@YAXXZ 10001160 f   cobranet.obj
 0001:00000170       ??__E?rxStatusOid@CobraNetNode@@0VasiOID@@A@@YAXXZ 10001170 f   cobranet.obj
 0001:00000180       ??__E?rxSubFormatOid@CobraNetNode@@0VasiOID@@A@@YAXXZ 10001180 f   cobranet.obj
 0001:00000190       ??__E?rxSubMapOid@CobraNetNode@@0VasiOID@@A@@YAXXZ 10001190 f   cobranet.obj
 0001:000001a0       ??__E?serialBaudOID@CobraNetNode@@0VasiOID@@A@@YAXXZ 100011a0 f   cobranet.obj
 0001:000001b0       ??__E?serialFormatOID@CobraNetNode@@0VasiOID@@A@@YAXXZ 100011b0 f   cobranet.obj
 0001:000001c0       ??__E?serialPPeriodOID@CobraNetNode@@0VasiOID@@A@@YAXXZ 100011c0 f   cobranet.obj
 0001:000001d0       ??__E?serialRxMacOID@CobraNetNode@@0VasiOID@@A@@YAXXZ 100011d0 f   cobranet.obj
 0001:000001e0       ??__E?serialTxMacOID@CobraNetNode@@0VasiOID@@A@@YAXXZ 100011e0 f   cobranet.obj
 0001:000001f0       ??__E?serialTxPriorityOID@CobraNetNode@@0VasiOID@@A@@YAXXZ 100011f0 f   cobranet.obj
 0001:00000200       ??__E?stdUserIntegerOid@CobraNetNode@@0VasiOID@@A@@YAXXZ 10001200 f   cobranet.obj
 0001:00000210       ??__E?sysContactOID@CobraNetNode@@0VasiOID@@A@@YAXXZ 10001210 f   cobranet.obj
 0001:00000220       ??__E?sysDescriptionOID@CobraNetNode@@0VasiOID@@A@@YAXXZ 10001220 f   cobranet.obj
 0001:00000230       ??__E?sysLocationOID@CobraNetNode@@0VasiOID@@A@@YAXXZ 10001230 f   cobranet.obj
 0001:00000240       ??__E?sysNameOID@CobraNetNode@@0VasiOID@@A@@YAXXZ 10001240 f   cobranet.obj
 0001:00000250       ??__E?txBundleOid@CobraNetNode@@0VasiOID@@A@@YAXXZ 10001250 f   cobranet.obj
 0001:00000260       ??__E?txDropoutsOid@CobraNetNode@@0VasiOID@@A@@YAXXZ 10001260 f   cobranet.obj
 0001:00000270       ??__E?txMaxUnicastOid@CobraNetNode@@0VasiOID@@A@@YAXXZ 10001270 f   cobranet.obj
 0001:00000280       ??__E?txPositionOid@CobraNetNode@@0VasiOID@@A@@YAXXZ 10001280 f   cobranet.obj
 0001:00000290       ??__E?txPriorityOid@CobraNetNode@@0VasiOID@@A@@YAXXZ 10001290 f   cobranet.obj
 0001:000002a0       ??__E?txReceiversOid@CobraNetNode@@0VasiOID@@A@@YAXXZ 100012a0 f   cobranet.obj
 0001:000002b0       ??__E?txSubCountOid@CobraNetNode@@0VasiOID@@A@@YAXXZ 100012b0 f   cobranet.obj
 0001:000002c0       ??__E?txSubFormatOid@CobraNetNode@@0VasiOID@@A@@YAXXZ 100012c0 f   cobranet.obj
 0001:000002d0       ??__E?txSubMapOid@CobraNetNode@@0VasiOID@@A@@YAXXZ 100012d0 f   cobranet.obj
 0001:000002e0       ??__E?txUnicastModeOid@CobraNetNode@@0VasiOID@@A@@YAXXZ 100012e0 f   cobranet.obj
 0001:000002f0       ??__EaudioEntryTable@@YAXXZ 100012f0 f   mibtbl.obj
 0001:000005a0       ??__EaudioGroup@@YAXXZ     100015a0 f   mibtbl.obj
 0001:000005c0       ??__EconductorEntryTable@@YAXXZ 100015c0 f   mibtbl.obj
 0001:00000700       ??__EconductorGroup@@YAXXZ 10001700 f   mibtbl.obj
 0001:00000720       ??__EerrorEntryTable@@YAXXZ 10001720 f   mibtbl.obj
 0001:000007e0       ??__EerrorGroup@@YAXXZ     100017e0 f   mibtbl.obj
 0001:00000800       ??__EfirmwareEntryTable@@YAXXZ 10001800 f   mibtbl.obj
 0001:00000970       ??__EfirmwareGroup@@YAXXZ  10001970 f   mibtbl.obj
 0001:00000990       ??__EflashEntryTable@@YAXXZ 10001990 f   mibtbl.obj
 0001:00000ab0       ??__EflashGroup@@YAXXZ     10001ab0 f   mibtbl.obj
 0001:00000ad0       ??__EifEntryTable@@YAXXZ   10001ad0 f   mibtbl.obj
 0001:00000dc0       ??__EifGroup@@YAXXZ        10001dc0 f   mibtbl.obj
 0001:00000de0       ??__EifmEntryTable@@YAXXZ  10001de0 f   mibtbl.obj
 0001:00000ec0       ??__EifmGroup@@YAXXZ       10001ec0 f   mibtbl.obj
 0001:00000f20       ??__EipEntryTable@@YAXXZ   10001f20 f   mibtbl.obj
 0001:00001250       ??__EipGroup@@YAXXZ        10002250 f   mibtbl.obj
 0001:00001270       ??__EipmonEntryTable@@YAXXZ 10002270 f   mibtbl.obj
 0001:00001310       ??__EipmonGroup@@YAXXZ     10002310 f   mibtbl.obj
 0001:00001330       ??__EmimonEntryTable@@YAXXZ 10002330 f   mibtbl.obj
 0001:000013d0       ??__EmimonGroup@@YAXXZ     100023d0 f   mibtbl.obj
 0001:000013f0       ??__EmodeEntryTable@@YAXXZ 100023f0 f   mibtbl.obj
 0001:00001450       ??__EmodeGroup@@YAXXZ      10002450 f   mibtbl.obj
 0001:00001470       ??__ErxEntryTable@@YAXXZ   10002470 f   mibtbl.obj
 0001:00001600       ??__ErxGroup@@YAXXZ        10002600 f   mibtbl.obj
 0001:00001620       ??__EserialEntryTable@@YAXXZ 10002620 f   mibtbl.obj
 0001:00001720       ??__EserialGroup@@YAXXZ    10002720 f   mibtbl.obj
 0001:00001740       ??__EsnmpEntryTable@@YAXXZ 10002740 f   mibtbl.obj
 0001:00001b00       ??__EsnmpGroup@@YAXXZ      10002b00 f   mibtbl.obj
 0001:00001b20       ??__EstdEntryTable@@YAXXZ  10002b20 f   mibtbl.obj
 0001:00001bc0       ??__EstdGroup@@YAXXZ       10002bc0 f   mibtbl.obj
 0001:00001be0       ??__EsyncEntryTable@@YAXXZ 10002be0 f   mibtbl.obj
 0001:00001ce0       ??__EsyncGroup@@YAXXZ      10002ce0 f   mibtbl.obj
 0001:00001d00       ??__EsysEntryTable@@YAXXZ  10002d00 f   mibtbl.obj
 0001:00001e00       ??__EsysGroup@@YAXXZ       10002e00 f   mibtbl.obj
 0001:00001e20       ??__EtxEntryTable@@YAXXZ   10002e20 f   mibtbl.obj
 0001:00002000       ??__EtxGroup@@YAXXZ        10003000 f   mibtbl.obj
 0001:00002020       ??__EudpEntryTable@@YAXXZ  10003020 f   mibtbl.obj
 0001:000020c0       ??__EudpGroup@@YAXXZ       100030c0 f   mibtbl.obj
 0001:000020de       ??__E?_Generic_object@?$_Error_objects@H@std@@2V_Generic_error_category@2@A@@YAXXZ 100030de f   libcpmt:xthrow.obj
 0001:000020ea       ??__E?_Iostream_object@?$_Error_objects@H@std@@2V_Iostream_error_category@2@A@@YAXXZ 100030ea f   libcpmt:xthrow.obj
 0001:000020f6       ??__E?_System_object@?$_Error_objects@H@std@@2V_System_error_category@2@A@@YAXXZ 100030f6 f   libcpmt:xthrow.obj
 0001:00002102       ??__E?_Generic_object@?$_Error_objects@H@std@@2V_Generic_error_category@2@A@@YAXXZ 10003102 f   libcpmt:syserror.obj
 0001:0000210e       ??__E?_Iostream_object@?$_Error_objects@H@std@@2V_Iostream_error_category@2@A@@YAXXZ 1000310e f   libcpmt:syserror.obj
 0001:0000211a       ??__E?_System_object@?$_Error_objects@H@std@@2V_System_error_category@2@A@@YAXXZ 1000311a f   libcpmt:syserror.obj
 0001:000031ac       $LN14                      100041ac     asios.obj
 0001:00003a80       $LN36                      10004a80     asisnmp.obj
 0001:00003a94       $LN31                      10004a94     asisnmp.obj
 0001:00003fe4       $LN63                      10004fe4     asisnmp.obj
 0001:00004000       $LN54                      10005000     asisnmp.obj
 0001:00004800       ?oidMatches@@YA_NPAVasiOID@@PAKH@Z 10005800 f   asisnmp.obj
 0001:0000e495       __catch$?_Copy@?$basic_string@DU?$char_traits@D@std@@V?$allocator@D@2@@std@@QAEXII@Z$0 1000f495 f i asxavdecc.obj
 0001:0000e4d2       __catch$?_Copy@?$basic_string@DU?$char_traits@D@std@@V?$allocator@D@2@@std@@QAEXII@Z$1 1000f4d2 f i asxavdecc.obj
 0001:0000ecac       $LN11                      1000fcac     asxavdecc.obj
 0001:0000f084       $LN23                      10010084     asxavdecc.obj
 0001:0000f280       ?bufferSwitch@@YAXJJ@Z     10010280 f   asxasio.obj
 0001:0000f2a0       ?sampleRateDidChange@@YAXN@Z 100102a0 f   asxasio.obj
 0001:0000f2b0       ?asioMessage@@YAJJJPAXPAN@Z 100102b0 f   asxasio.obj
 0001:0000f2c0       ?bufferSwitchTimeInfo@@YAPAUASIOTime@@PAU1@JJ@Z 100102c0 f   asxasio.obj
 0001:00010348       $LN25                      10011348     asxasioplay.obj
 0001:000108e8       $LN20                      100118e8     asxasiorec.obj
 0001:00014be4       $LN31                      10015be4     asxclass.obj
 0001:00014c44       $LN9                       10015c44     asxclass.obj
 0001:00014c4c       $LN7                       10015c4c     asxclass.obj
 0001:00017970       $LN62                      10018970     asxhpi.obj
 0001:00017988       $LN63                      10018988     asxhpi.obj
 0001:0001bdf0       $LN15                      1001cdf0     asxhpi.obj
 0001:0001ddd8       $LN37                      1001edd8     asxhpi.obj
 0001:0001ddfc       $LN31                      1001edfc     asxhpi.obj
 0001:0001de0c       $LN38                      1001ee0c     asxhpi.obj
 0001:0001ecd0       ?HpiTranslateNode@@YAHH@Z  1001fcd0 f   asxhpi.obj
 0001:0001f668       $LN19                      10020668     asxhpi.obj
 0001:0001fcb4       $LN74                      10020cb4     asxhpi.obj
 0001:0001fcd4       $LN58                      10020cd4     asxhpi.obj
 0001:00021028       $LN337                     10022028     asxhpi.obj
 0001:00021600       $LN15                      10022600     asxhpi.obj
 0001:00023328       $LN48                      10024328     asxhpi.obj
 0001:0002334c       $LN44                      1002434c     asxhpi.obj
 0001:00023420       $LN49                      10024420     asxhpi.obj
 0001:00023448       $LN45                      10024448     asxhpi.obj
 0001:00023684       $LN11                      10024684     asxhpi.obj
 0001:00024714       $LN25                      10025714     asxhpirec.obj
 0001:00024730       $LN26                      10025730     asxhpirec.obj
 0001:00025ca4       $LN32                      10026ca4     asxplay.obj
 0001:00025dac       $LN29                      10026dac     asxplay.obj
 0001:000260e0       $LN39                      100270e0     asxplay.obj
 0001:00026504       $LN35                      10027504     asxplay.obj
 0001:0002667c       $LN35                      1002767c     asxplay.obj
 0001:00026820       $LN18                      10027820     asxplay.obj
 0001:0002695c       $LN13                      1002795c     asxplay.obj
 0001:00026f28       $LN57                      10027f28     asxrec.obj
 0001:00027310       $LN24                      10028310     asxrec.obj
 0001:000273ac       $LN15                      100283ac     asxrec.obj
 0001:000274d4       $LN26                      100284d4     asxrec.obj
 0001:000274e8       $LN27                      100284e8     asxrec.obj
 0001:0002765c       $LN18                      1002865c     asxrec.obj
 0001:00027708       $LN12                      10028708     asxrec.obj
 0001:000277b4       $LN15                      100287b4     asxrec.obj
 0001:0002824c       $LN11                      1002924c     asxsnmp.obj
 0001:00028a14       $LN31                      10029a14     asxsnmp.obj
 0001:00028db0       $LN13                      10029db0     asxsnmp.obj
 0001:00029be0       $LN99                      1002abe0     asxsnmp.obj
 0001:0002b054       $LN31                      1002c054     asxsnmp.obj
 0001:0002dc20       ?AddCobranet@@YAXPAVasxMixer@@PAVasxSubSystem@@PAVControlTracker@@PAUHMIXEROBJ__@@PAVasxNode@@4PAUtagMIXERCONTROLA@@H@Z 1002ec20 f   asxwave.obj
 0001:0002e6fc       $LN183                     1002f6fc     asxwave.obj
 0001:0002e740       ?AddTuner@@YAXPAVasxMixer@@PAVasxSubSystem@@PAVControlTracker@@PAUHMIXEROBJ__@@PAVasxNode@@4PAUtagMIXERCONTROLA@@H@Z 1002f740 f   asxwave.obj
 0001:00030308       $LN162                     10031308     asxwave.obj
 0001:00030c80       $LN14                      10031c80     asxwave.obj
 0001:00030c98       $LN12                      10031c98     asxwave.obj
 0001:00030cc0       ?extractIndexFromName@@YAHPAD@Z 10031cc0 f   asxwave.obj
 0001:00030d70       ?mapWAVEError@@YA?AW4asxERROR@@H@Z 10031d70 f   asxwave.obj
 0001:00030d80       ?translateLineNameToId@@YAHPADPBUNAMEMAPPING@@@Z 10031d80 f   asxwave.obj
 0001:00030de0       ?waveLinearTodB@@YAMJ@Z    10031de0 f   asxwave.obj
 0001:00030e20       ?wavedBToLinear@@YAJM@Z    10031e20 f   asxwave.obj
 0001:000325cc       $LN29                      100335cc     cobranet.obj
 0001:0003301c       $LN29                      1003401c     cobranet.obj
 0001:000338f8       $LN49                      100348f8     rifffile.obj
 0001:000344dc       $LN21                      100354dc     twavfile.obj
 0001:00034e14       $LN103                     10035e14     twavfile.obj
 0001:00034e34       $LN73                      10035e34     twavfile.obj
 0001:00037014       $LN95                      10038014     twavgen.obj
 0001:00037028       $LN91                      10038028     twavgen.obj
 0001:00037915       ?FLoadedAtPreferredAddress@@YG_NPAU_IMAGE_NT_HEADERS@@PAUHINSTANCE__@@@Z 10038915 f   Delayimp:delayhlp.obj
 0001:0003793e       ?OverlayIAT@@YGXPAU_IMAGE_THUNK_DATA32@@PBU1@@Z 1003893e f   Delayimp:delayhlp.obj
 0001:00037972       ?PiddFromDllName@@YGPBUImgDelayDescr@@PBD@Z 10038972 f   Delayimp:delayhlp.obj
 0001:000379f7       ?PinhFromImageBase@@YGPAU_IMAGE_NT_HEADERS@@PAUHINSTANCE__@@@Z 100389f7 f   Delayimp:delayhlp.obj
 0001:00037a08       ?TimeStampOfImage@@YGKPAU_IMAGE_NT_HEADERS@@@Z 10038a08 f   Delayimp:delayhlp.obj
 0001:00037a17       ?__memcmp@@YGHPBX0I@Z      10038a17 f   Delayimp:delayhlp.obj
 0001:00037a48       ?__memcpy@@YGPAXPAXPBXI@Z  10038a48 f   Delayimp:delayhlp.obj
 0001:00037a6f       ?__strlen@@YGIPBD@Z        10038a6f f   Delayimp:delayhlp.obj
 0001:00038800       $$000000                   10039800     LIBCMT:strncpy.obj
 0001:00038924       ?strtoxl@@YAKPAUlocaleinfo_struct@@PBDPAPBDHH@Z 10039924 f   LIBCMT:strtol.obj
 0001:00038d90       $$000000                   10039d90     LIBCMT:memcpy.obj
 0001:00038fe0       LeadUpVec                  10039fe0     LIBCMT:memcpy.obj
 0001:0003905c       UnwindUpVec                1003a05c     LIBCMT:memcpy.obj
 0001:000390c8       TrailUpVec                 1003a0c8     LIBCMT:memcpy.obj
 0001:0003916c       LeadDownVec                1003a16c     LIBCMT:memcpy.obj
 0001:000391f8       UnwindDownVec              1003a1f8     LIBCMT:memcpy.obj
 0001:00039264       TrailDownVec               1003a264     LIBCMT:memcpy.obj
 0001:00039770       $$000000                   1003a770     LIBCMT:lldiv.obj
 0001:00039820       $$000000                   1003a820     LIBCMT:llmul.obj
 0001:00039920       $$000000                   1003a920     LIBCMT:memmove.obj
 0001:00039b70       LeadUpVec                  1003ab70     LIBCMT:memmove.obj
 0001:00039bec       UnwindUpVec                1003abec     LIBCMT:memmove.obj
 0001:00039c58       TrailUpVec                 1003ac58     LIBCMT:memmove.obj
 0001:00039cfc       LeadDownVec                1003acfc     LIBCMT:memmove.obj
 0001:00039d88       UnwindDownVec              1003ad88     LIBCMT:memmove.obj
 0001:00039df4       TrailDownVec               1003adf4     LIBCMT:memmove.obj
 0001:0003a18d       __onexit_nolock            1003b18d f   LIBCMT:onexit.obj
 0001:0003a260       $$000000                   1003b260     LIBCMT:strstr.obj
 0001:0003a4c3       ?strtoxq@@YA_KPAUlocaleinfo_struct@@PBDPAPBDHH@Z 1003b4c3 f   LIBCMT:strtoq.obj
 0001:0003a894       __hypothlp                 1003b894 f   LIBCMT:hypot.obj
 0001:0003ab43       ?CatchGuardHandler@@YA?AW4_EXCEPTION_DISPOSITION@@PAUEHExceptionRecord@@PAUCatchGuardRN@@PAX2@Z 1003bb43 f   LIBCMT:_trnsctrl_.obj
 0001:0003ab74       ?TranslatorGuardHandler@@YA?AW4_EXCEPTION_DISPOSITION@@PAUEHExceptionRecord@@PAUTranslatorGuardRN@@PAX2@Z 1003bb74 f   LIBCMT:_trnsctrl_.obj
 0001:0003afd0       $$000000                   1003bfd0     LIBCMT:memset.obj
 0001:0003b060       $$000000                   1003c060     LIBCMT:ftol3.obj
 0001:0003b500       $$000000                   1003c500     LIBCMT:strncmp.obj
 0001:0003b578       ?FindCompleteObject@@YAPAXPAPAX@Z 1003c578 f   LIBCMT:rtti.obj
 0001:0003b595       ?FindMITargetTypeInstance@@YAPBU_s_RTTIBaseClassDescriptor@@PAXPBU_s_RTTICompleteObjectLocator@@PAUTypeDescriptor@@H2@Z 1003c595 f   LIBCMT:rtti.obj
 0001:0003b6aa       ?FindSITargetTypeInstance@@YAPBU_s_RTTIBaseClassDescriptor@@PBU_s_RTTICompleteObjectLocator@@PAUTypeDescriptor@@1@Z 1003c6aa f   LIBCMT:rtti.obj
 0001:0003b732       ?FindVITargetTypeInstance@@YAPBU_s_RTTIBaseClassDescriptor@@PAXPBU_s_RTTICompleteObjectLocator@@PAUTypeDescriptor@@H2@Z 1003c732 f   LIBCMT:rtti.obj
 0001:0003b8b1       ?PMDtoOffset@@YAHPAXABUPMD@@@Z 1003c8b1 f   LIBCMT:rtti.obj
 0001:0003bc2d       __dupenv_s_helper          1003cc2d f   LIBCMT:getenv.obj
 0001:0003bd4d       __getenv_s_helper          1003cd4d f   LIBCMT:getenv.obj
 0001:0003bfd0       $$000000                   1003cfd0     LIBCMT:ulldiv.obj
 0001:0003c040       $$000000                   1003d040     LIBCMT:log10_sse2_precise.obj
 0001:0003c2f0       $$000000                   1003d2f0     LIBCMT:pow_sse2_precise.obj
 0001:0003de60       $$000000                   1003ee60     LIBCMT:sin_sse2_precise.obj
 0001:0003e1bd       ___DllMainCRTStartup       1003f1bd f   LIBCMT:dllcrt0.obj
 0001:0003e2f8       ___IsPackagedAppHelper     1003f2f8 f   LIBCMT:winapisupp.obj
 0001:0003ecd0       ?CPtoLocaleName@@YAPB_WH@Z 1003fcd0 f   LIBCMT:mbctype.obj
 0001:0003ed0a       ?getSystemCP@@YAHH@Z       1003fd0a f   LIBCMT:mbctype.obj
 0001:0003ed78       ?setSBCS@@YAXPAUthreadmbcinfostruct@@@Z 1003fd78 f   LIBCMT:mbctype.obj
 0001:0003edd7       ?setSBUpLow@@YAXPAUthreadmbcinfostruct@@@Z 1003fdd7 f   LIBCMT:mbctype.obj
 0001:0003fac9       __copytlocinfo_nolock      10040ac9 f   LIBCMT:wsetloca.obj
 0001:00040247       __wsetlocale_get_all       10041247 f   LIBCMT:wsetloca.obj
 0001:000403b4       __wsetlocale_nolock        100413b4 f   LIBCMT:wsetloca.obj
 0001:0004063d       __wsetlocale_set_cat       1004163d f   LIBCMT:wsetloca.obj
 0001:000409e7       _sync_legacy_variables_lk  100419e7 f   LIBCMT:wsetloca.obj
 0001:00041e41       $LN277                     10042e41     LIBCMT:output.obj
 0001:00041e95       _write_char                10042e95 f   LIBCMT:output.obj
 0001:00041edd       _write_multi_char          10042edd f   LIBCMT:output.obj
 0001:00041f09       _write_string              10042f09 f   LIBCMT:output.obj
 0001:000425cf       __initterm                 100435cf f   LIBCMT:crt0dat.obj
 0001:00042639       _doexit                    10043639 f   LIBCMT:crt0dat.obj
 0001:00042bf0       $$000000                   10043bf0     LIBCMT:sehprolg4.obj
 0001:00042c50       _ValidateLocalCookies      10043c50 f   LIBCMT:chandler4.obj
 0001:000439a0       $LN296                     100449a0     LIBCMT:outputs.obj
 0001:000439c0       _write_char                100449c0 f   LIBCMT:outputs.obj
 0001:00043a08       _write_multi_char          10044a08 f   LIBCMT:outputs.obj
 0001:00043a34       _write_string              10044a34 f   LIBCMT:outputs.obj
 0001:00044dc4       $LN736                     10045dc4     LIBCMT:outputp.obj
 0001:00044f2d       _write_char                10045f2d f   LIBCMT:outputp.obj
 0001:00044f75       _write_multi_char          10045f75 f   LIBCMT:outputp.obj
 0001:00044fa1       _write_string              10045fa1 f   LIBCMT:outputp.obj
 0001:00045290       $$000000                   10046290     LIBCMT:strcmp.obj
 0001:00045ac2       __cftoe2_l                 10046ac2 f   LIBCMT:cvt.obj
 0001:00045cfc       __cftof2_l                 10046cfc f   LIBCMT:cvt.obj
 0001:00046150       __shift                    10047150 f   LIBCMT:cvt.obj
 0001:000465a0       $$000000                   100475a0     LIBCMT:strchr.obj
 0001:000468f0       $$000000                   100478f0     LIBCMT:ulldvrm.obj
 0001:00046990       $$000000                   10047990     LIBCMT:sqrt.obj
 0001:00046ded       __get_fname                10047ded f   LIBCMT:fpexcept.obj
 0001:00047670       $$000000                   10048670     LIBCMT:lowhelpr.obj
 0001:0004783e       ?CallCatchBlock@@YAPAXPAUEHExceptionRecord@@PAUEHRegistrationNode@@PAU_CONTEXT@@PBU_s_FuncInfo@@PAXHK@Z 1004883e f   LIBCMT:frame.obj
 0001:00047a04       ?CallUnexpected@@YAXPBU_s_ESTypeList@@@Z 10048a04 f   LIBCMT:frame.obj
 0001:00047a2c       __catch$?CallUnexpected@@YAXPBU_s_ESTypeList@@@Z$0 10048a2c f   LIBCMT:frame.obj
 0001:00047a44       ?CatchIt@@YAXPAUEHExceptionRecord@@PAUEHRegistrationNode@@PAU_CONTEXT@@PAXPBU_s_FuncInfo@@PBU_s_HandlerType@@PBU_s_CatchableType@@PBU_s_TryBlockMapEntry@@H1E@Z 10048a44 f   LIBCMT:frame.obj
 0001:00047abf       ?ExFilterRethrow@@YAHPAU_EXCEPTION_POINTERS@@@Z 10048abf f   LIBCMT:frame.obj
 0001:00047b0c       ?FindHandler@@YAXPAUEHExceptionRecord@@PAUEHRegistrationNode@@PAU_CONTEXT@@PAXPBU_s_FuncInfo@@EH1@Z 10048b0c f   LIBCMT:frame.obj
 0001:00047ea9       ?FindHandlerForForeignException@@YAXPAUEHExceptionRecord@@PAUEHRegistrationNode@@PAU_CONTEXT@@PAXPBU_s_FuncInfo@@HH1@Z 10048ea9 f   LIBCMT:frame.obj
 0001:00047fc5       ?IsInExceptionSpec@@YAEPAUEHExceptionRecord@@PBU_s_ESTypeList@@@Z 10048fc5 f   LIBCMT:frame.obj
 0001:0004804d       ?Is_bad_exception_allowed@@YAEPBU_s_ESTypeList@@@Z 1004904d f   LIBCMT:frame.obj
 0001:00048b30       $$000000                   10049b30     LIBCMT:strlen.obj
 0001:000491a7       $LN79                      1004a1a7     LIBCMT:libm_error.obj
 0001:00049210       $$000000                   1004a210     LIBCMT:log10.obj
 0001:00049360       $$000000                   1004a360     LIBCMT:pow.obj
 0001:000498bf       _flsall                    1004a8bf f   LIBCMT:fflush.obj
 0001:00049d40       $$000000                   1004ad40     LIBCMT:exsup4.obj
 0001:00049dd0       __unwind_handler4          1004add0 f   LIBCMT:exsup4.obj
 0001:0004abe0       $$000000                   1004bbe0     LIBCMT:chkstk.obj
 0001:0004bc96       ?__crtLCMapStringA_stat@@YAHPAUlocaleinfo_struct@@PB_WKPBDHPADHHH@Z 1004cc96 f   LIBCMT:a_map.obj
 0001:0004be9a       ?strncnt@@YAHPBDH@Z        1004ce9a f   LIBCMT:a_map.obj
 0001:0004bff0       $$000000                   1004cff0     LIBCMT:sin.obj
 0001:0004c292       _xcptlookup                1004d292 f   LIBCMT:winxfltr.obj
 0001:0004c386       _parse_cmdline             1004d386 f   LIBCMT:stdargv.obj
 0001:0004cbe9       _fix_grouping              1004dbe9 f   LIBCMT:initmon.obj
 0001:0004ce8e       _fix_grouping              1004de8e f   LIBCMT:initnum.obj
 0001:0004d2c2       __get_lc_time              1004e2c2 f   LIBCMT:inittime.obj
 0001:0004dadb       ?__crtGetStringTypeA_stat@@YAHPAUlocaleinfo_struct@@KPBDHPAGHH@Z 1004eadb f   LIBCMT:a_str.obj
 0001:0004e08e       _cmpBYTE                   1004f08e f   LIBCMT:memcmp.obj
 0001:0004e0b3       _cmpDWORD                  1004f0b3 f   LIBCMT:memcmp.obj
 0001:0004e13e       _cmpResult                 1004f13e f   LIBCMT:memcmp.obj
 0001:0004e15a       _cmpWORD                   1004f15a f   LIBCMT:memcmp.obj
 0001:0004f8a3       $LN1281                    100508a3     LIBCMT:memcmp.obj
 0001:0004f923       _unaligned_memcmp          10050923 f   LIBCMT:memcmp.obj
 0001:0005103f       $LN1269                    1005203f     LIBCMT:memcmp.obj
 0001:0005137e       _GetLocaleNameFromDefault  1005237e f   LIBCMT:getqloc.obj
 0001:000513f7       _GetLocaleNameFromLangCountry 100523f7 f   LIBCMT:getqloc.obj
 0001:0005146b       _GetLocaleNameFromLanguage 1005246b f   LIBCMT:getqloc.obj
 0001:000514b5       _GetPrimaryLen             100524b5 f   LIBCMT:getqloc.obj
 0001:000514e7       _LangCountryEnumProcEx@12  100524e7 f   LIBCMT:getqloc.obj
 0001:00051707       _LanguageEnumProcEx@12     10052707 f   LIBCMT:getqloc.obj
 0001:000517ba       _ProcessCodePage           100527ba f   LIBCMT:getqloc.obj
 0001:0005184f       _TestDefaultCountry        1005284f f   LIBCMT:getqloc.obj
 0001:0005189b       _TestDefaultLanguage       1005289b f   LIBCMT:getqloc.obj
 0001:000518d6       _TranslateName             100528d6 f   LIBCMT:getqloc.obj
 0001:00051b04       _CountryEnumProc@4         10052b04 f   LIBCMT:getqloc_downlevel.obj
 0001:00051bb4       _GetLcidFromCountry        10052bb4 f   LIBCMT:getqloc_downlevel.obj
 0001:00051bf4       _GetLcidFromDefault        10052bf4 f   LIBCMT:getqloc_downlevel.obj
 0001:00051c10       _GetLcidFromLangCountry    10052c10 f   LIBCMT:getqloc_downlevel.obj
 0001:00051c8d       _GetLcidFromLanguage       10052c8d f   LIBCMT:getqloc_downlevel.obj
 0001:00051ce6       _GetPrimaryLen             10052ce6 f   LIBCMT:getqloc_downlevel.obj
 0001:00051d10       _LangCountryEnumProc@4     10052d10 f   LIBCMT:getqloc_downlevel.obj
 0001:00051f05       _LanguageEnumProc@4        10052f05 f   LIBCMT:getqloc_downlevel.obj
 0001:00051fe0       _LcidFromHexString         10052fe0 f   LIBCMT:getqloc_downlevel.obj
 0001:0005202f       _ProcessCodePage           1005302f f   LIBCMT:getqloc_downlevel.obj
 0001:000520ba       _TestDefaultCountry        100530ba f   LIBCMT:getqloc_downlevel.obj
 0001:000520dc       _TestDefaultLanguage       100530dc f   LIBCMT:getqloc_downlevel.obj
 0001:00052146       _TranslateName             10053146 f   LIBCMT:getqloc_downlevel.obj
 0001:00052541       ___crtEnumLocalesProc@4    10053541 f   LIBCMT:winapinls.obj
 0001:00052b2c       _ctrlevent_capture@4       10053b2c f   LIBCMT:winsig.obj
 0001:00052d8c       _siglookup                 10053d8c f   LIBCMT:winsig.obj
 0001:00055591       $LN113                     10056591     LIBCMT:undname.obj
 0001:000555a9       $LN105                     100565a9     LIBCMT:undname.obj
 0001:00056309       $LN27                      10057309     LIBCMT:undname.obj
 0001:00058986       $LN129                     10059986     LIBCMT:undname.obj
 0001:00058f83       ?und_memcpy@@YAXPADPBDI@Z  10059f83 f   LIBCMT:undname.obj
 0001:00058fa2       ?und_strlen@@YAIPBD@Z      10059fa2 f   LIBCMT:undname.obj
 0001:00058fb7       ?und_strncmp@@YAIPBD0I@Z   10059fb7 f   LIBCMT:undname.obj
 0001:00059130       $$000000                   1005a130     LIBCMT:strrchr.obj
 0001:00059470       $$000000                   1005a470     LIBCMT:lldvrm.obj
 0001:00059550       $$000000                   1005a550     LIBCMT:ullshr.obj
 0001:000596b1       ?__crtGetLocaleInfoA_stat@@YAHPAUlocaleinfo_struct@@PB_WKPADH@Z 1005a6b1 f   LIBCMT:a_loc.obj
 0001:0005bb74       $LN333                     1005cb74     LIBCMT:strgtold.obj
 0001:0005bbb0       $$000000                   1005cbb0     LIBCMT:87disp.obj
 0001:0005bd80       $$000000                   1005cd80     LIBCMT:genexcep.obj
 0001:0005bde0       $$000000                   1005cde0     LIBCMT:common.obj
 0001:0005bf70       $$000000                   1005cf70     LIBCMT:exsup.obj
 0001:0005bf90       __unwind_handler           1005cf90 f   LIBCMT:exsup.obj
 0001:0005c426       _copy_environ              1005d426 f   LIBCMT:setenv.obj
 0001:0005c486       _findenv                   1005d486 f   LIBCMT:setenv.obj
 0001:0005c5cd       ?__crtCompareStringA_stat@@YAHPAUlocaleinfo_struct@@PB_WKPBDH2HH@Z 1005d5cd f   LIBCMT:a_cmp.obj
 0001:0005c851       ?strncnt@@YAHPBDH@Z        1005d851 f   LIBCMT:a_cmp.obj
 0001:0005c8f0       $$000000                   1005d8f0     LIBCMT:log10_pentium4.obj
 0001:0005cb80       $$000000                   1005db80     LIBCMT:87tran.obj
 0001:0005cd80       $$000000                   1005dd80     LIBCMT:pow_pentium4.obj
 0001:0005e770       $$000000                   1005f770     LIBCMT:alloca16.obj
 0001:0005e7a0       $$000000                   1005f7a0     LIBCMT:sin_pentium4.obj
 0001:0005e968       ?x_ismbbtype_l@@YAHPAUlocaleinfo_struct@@IHH@Z 1005f968 f   LIBCMT:ismbbyte.obj
 0001:0005ec3c       @x64tow_s@24               1005fc3c f   LIBCMT:xtows.obj
 0001:0005ee0f       _xtow_s@20                 1005fe0f f   LIBCMT:xtows.obj
 0001:0005fe39       ___abstract_cw_sse2        10060e39 f   LIBCMT:ieee87.obj
 0001:0005fee2       ___abstract_sw_sse2        10060ee2 f   LIBCMT:ieee87.obj
 0001:0005ff23       ___clearfp_sse2            10060f23 f   LIBCMT:ieee87.obj
 0001:0006028d       ___control87_sse2          1006128d f   LIBCMT:ieee87.obj
 0001:00060410       ___fpreset_sse2            10061410 f   LIBCMT:ieee87.obj
 0001:0006041c       ___hw_cw_sse2              1006141c f   LIBCMT:ieee87.obj
 0001:000604c5       ___statusfp_sse2           100614c5 f   LIBCMT:ieee87.obj
 0001:00060506       __abstract_cw              10061506 f   LIBCMT:ieee87.obj
 0001:000605a5       __abstract_sw              100615a5 f   LIBCMT:ieee87.obj
 0001:00060d0a       __hw_cw                    10061d0a f   LIBCMT:ieee87.obj
 0001:000618ea       ___createFile              100628ea f   LIBCMT:wopen.obj
 0001:000622c5       ?wcstoxl@@YAKPB_WPAPB_WHH@Z 100632c5 f   LIBCMT:wcstol.obj
 0001:00062506       ?wcstoxq@@YA_KPAUlocaleinfo_struct@@PB_WPAPB_WHH@Z 10063506 f   LIBCMT:wcstoq.obj
 0001:00062a50       $$000000                   10063a50     LIBCMT:_strnicm.obj
 0001:00063d94       $LN323                     10064d94     LIBCMT:wstrgtold.obj
 0001:00064150       $LN22                      10065150     libcpmt:xthrow.obj
 0001:000644e6       ?_strupr_s_l_stat@@YAHPADIPAUlocaleinfo_struct@@@Z 100654e6 f   LIBCMT:strupr.obj
 0001:00064720       __unwindfunclet$??0asxAdapterAVDECC@@QAE@PAVcontroller@avdecc_lib@@PAVsystem@2@PAVasxSystem@@PADH3@Z$0 10065720 f   asxavdecc.obj
 0001:00064728       __ehhandler$??0asxAdapterAVDECC@@QAE@PAVcontroller@avdecc_lib@@PAVsystem@2@PAVasxSystem@@PADH3@Z 10065728 f   asxavdecc.obj
 0001:00064750       __unwindfunclet$??0asxSubSystemAVDECC@@QAE@PAVasxSystem@@@Z$0 10065750 f   asxavdecc.obj
 0001:00064758       __ehhandler$??0asxSubSystemAVDECC@@QAE@PAVasxSystem@@@Z 10065758 f   asxavdecc.obj
 0001:00064780       __unwindfunclet$??1asxSubSystemAVDECC@@UAE@XZ$0 10065780 f   asxavdecc.obj
 0001:00064788       __ehhandler$??1asxSubSystemAVDECC@@UAE@XZ 10065788 f   asxavdecc.obj
 0001:000647b0       __unwindfunclet$?CheckSubSystems@asxAdapterAVDECC@@UAE?AW4asxERROR@@PAI0@Z$0 100657b0 f   asxavdecc.obj
 0001:000647b8       __ehhandler$?CheckSubSystems@asxAdapterAVDECC@@UAE?AW4asxERROR@@PAI0@Z 100657b8 f   asxavdecc.obj
 0001:000647e0       __unwindfunclet$?ReScan@asxSubSystemAVDECC@@UAEXXZ$0 100657e0 f   asxavdecc.obj
 0001:000647e8       __unwindfunclet$?ReScan@asxSubSystemAVDECC@@UAEXXZ$1 100657e8 f   asxavdecc.obj
 0001:000647f3       __unwindfunclet$?ReScan@asxSubSystemAVDECC@@UAEXXZ$2 100657f3 f   asxavdecc.obj
 0001:000647fb       __unwindfunclet$?ReScan@asxSubSystemAVDECC@@UAEXXZ$3 100657fb f   asxavdecc.obj
 0001:00064806       __ehhandler$?ReScan@asxSubSystemAVDECC@@UAEXXZ 10065806 f   asxavdecc.obj
 0001:00064830       __unwindfunclet$?SetDetails@asxAdapterAVDECC@@QAEXXZ$0 10065830 f   asxavdecc.obj
 0001:00064838       __ehhandler$?SetDetails@asxAdapterAVDECC@@QAEXXZ 10065838 f   asxavdecc.obj
 0001:00064860       __unwindfunclet$?UpdateAdapterProperties@asxAdapterAVDECC@@UAE?AW4asxERROR@@XZ$0 10065860 f   asxavdecc.obj
 0001:00064868       __ehhandler$?UpdateAdapterProperties@asxAdapterAVDECC@@UAE?AW4asxERROR@@XZ 10065868 f   asxavdecc.obj
 0001:00064890       __ehhandler$?_Copy@?$basic_string@DU?$char_traits@D@std@@V?$allocator@D@2@@std@@QAEXII@Z 10065890 f   asxavdecc.obj
 0001:000648b0       __unwindfunclet$??0asxAdapterASIO@@QAE@PAVasxSystem@@PAU_GUID@@PBD@Z$0 100658b0 f   asxasio.obj
 0001:000648b8       __ehhandler$??0asxAdapterASIO@@QAE@PAVasxSystem@@PAU_GUID@@PBD@Z 100658b8 f   asxasio.obj
 0001:000648e0       __unwindfunclet$??1asxAdapterASIO@@UAE@XZ$0 100658e0 f   asxasio.obj
 0001:000648e8       __ehhandler$??1asxAdapterASIO@@UAE@XZ 100658e8 f   asxasio.obj
 0001:00064910       __unwindfunclet$?Scan@asxMixerScannerASIO@@EAEXPAVasxMixer@@@Z$0 10065910 f   asxasio.obj
 0001:0006491b       __unwindfunclet$?Scan@asxMixerScannerASIO@@EAEXPAVasxMixer@@@Z$1 1006591b f   asxasio.obj
 0001:00064926       __unwindfunclet$?Scan@asxMixerScannerASIO@@EAEXPAVasxMixer@@@Z$2 10065926 f   asxasio.obj
 0001:00064931       __unwindfunclet$?Scan@asxMixerScannerASIO@@EAEXPAVasxMixer@@@Z$3 10065931 f   asxasio.obj
 0001:0006493c       __unwindfunclet$?Scan@asxMixerScannerASIO@@EAEXPAVasxMixer@@@Z$4 1006593c f   asxasio.obj
 0001:00064947       __ehhandler$?Scan@asxMixerScannerASIO@@EAEXPAVasxMixer@@@Z 10065947 f   asxasio.obj
 0001:00064970       __unwindfunclet$?Scan@asxSubSystemASIO@@UAEXXZ$0 10065970 f   asxasio.obj
 0001:0006497e       __ehhandler$?Scan@asxSubSystemASIO@@UAEXXZ 1006597e f   asxasio.obj
 0001:000649b0       __unwindfunclet$??1asxPlayerASIO@@UAE@XZ$0 100659b0 f   asxasioplay.obj
 0001:000649b8       __ehhandler$??1asxPlayerASIO@@UAE@XZ 100659b8 f   asxasioplay.obj
 0001:000649e0       __unwindfunclet$??1asxRecorderASIO@@UAE@XZ$0 100659e0 f   asxasiorec.obj
 0001:000649e8       __ehhandler$??1asxRecorderASIO@@UAE@XZ 100659e8 f   asxasiorec.obj
 0001:00064a10       __unwindfunclet$??0asxAbstractAdapter@@QAE@PAVasxAdapter@@@Z$0 10065a10 f   asxclass.obj
 0001:00064a18       __ehhandler$??0asxAbstractAdapter@@QAE@PAVasxAdapter@@@Z 10065a18 f   asxclass.obj
 0001:00064a40       __unwindfunclet$??0asxBlockProperty@@QAE@W4asxUCONTROL_PTYPE@@W4asxUCONTROL_PFLAGS@@IPBDPAUasxParameterRangeInfo@@2@Z$0 10065a40 f   asxclass.obj
 0001:00064a4b       __ehhandler$??0asxBlockProperty@@QAE@W4asxUCONTROL_PTYPE@@W4asxUCONTROL_PFLAGS@@IPBDPAUasxParameterRangeInfo@@2@Z 10065a4b f   asxclass.obj
 0001:00064a70       __unwindfunclet$??1asxAbstractAdapter@@UAE@XZ$0 10065a70 f   asxclass.obj
 0001:00064a78       __ehhandler$??1asxAbstractAdapter@@UAE@XZ 10065a78 f   asxclass.obj
 0001:00064aa0       __unwindfunclet$??1asxAdapter@@UAE@XZ$0 10065aa0 f   asxclass.obj
 0001:00064aa8       __unwindfunclet$??1asxAdapter@@UAE@XZ$1 10065aa8 f   asxclass.obj
 0001:00064ab3       __ehhandler$??1asxAdapter@@UAE@XZ 10065ab3 f   asxclass.obj
 0001:00064ad0       __unwindfunclet$??1asxMixer@@UAE@XZ$0 10065ad0 f   asxclass.obj
 0001:00064ad8       __unwindfunclet$??1asxMixer@@UAE@XZ$1 10065ad8 f   asxclass.obj
 0001:00064ae3       __unwindfunclet$??1asxMixer@@UAE@XZ$2 10065ae3 f   asxclass.obj
 0001:00064aee       __unwindfunclet$??1asxMixer@@UAE@XZ$3 10065aee f   asxclass.obj
 0001:00064af9       __unwindfunclet$??1asxMixer@@UAE@XZ$4 10065af9 f   asxclass.obj
 0001:00064b04       __ehhandler$??1asxMixer@@UAE@XZ 10065b04 f   asxclass.obj
 0001:00064b20       __unwindfunclet$??1asxSystem@@UAE@XZ$0 10065b20 f   asxclass.obj
 0001:00064b28       __unwindfunclet$??1asxSystem@@UAE@XZ$1 10065b28 f   asxclass.obj
 0001:00064b33       __unwindfunclet$??1asxSystem@@UAE@XZ$2 10065b33 f   asxclass.obj
 0001:00064b3e       __unwindfunclet$??1asxSystem@@UAE@XZ$3 10065b3e f   asxclass.obj
 0001:00064b49       __ehhandler$??1asxSystem@@UAE@XZ 10065b49 f   asxclass.obj
 0001:00064b70       __unwindfunclet$?AddAdapter@asxSystem@@QAE?AW4asxERROR@@PAVasxAdapter@@PAVasxMixerScanner@@@Z$0 10065b70 f   asxclass.obj
 0001:00064b7b       __ehhandler$?AddAdapter@asxSystem@@QAE?AW4asxERROR@@PAVasxAdapter@@PAVasxMixerScanner@@@Z 10065b7b f   asxclass.obj
 0001:00064ba0       __unwindfunclet$?asxCreateSubSystem@@YA?AW4asxERROR@@PAVasxSystem@@HPAPAVasxSubSystem@@@Z$0 10065ba0 f   asxclass.obj
 0001:00064bab       __unwindfunclet$?asxCreateSubSystem@@YA?AW4asxERROR@@PAVasxSystem@@HPAPAVasxSubSystem@@@Z$1 10065bab f   asxclass.obj
 0001:00064bb6       __unwindfunclet$?asxCreateSubSystem@@YA?AW4asxERROR@@PAVasxSystem@@HPAPAVasxSubSystem@@@Z$2 10065bb6 f   asxclass.obj
 0001:00064bc1       __unwindfunclet$?asxCreateSubSystem@@YA?AW4asxERROR@@PAVasxSystem@@HPAPAVasxSubSystem@@@Z$3 10065bc1 f   asxclass.obj
 0001:00064bcc       __unwindfunclet$?asxCreateSubSystem@@YA?AW4asxERROR@@PAVasxSystem@@HPAPAVasxSubSystem@@@Z$4 10065bcc f   asxclass.obj
 0001:00064bd7       __unwindfunclet$?asxCreateSubSystem@@YA?AW4asxERROR@@PAVasxSystem@@HPAPAVasxSubSystem@@@Z$5 10065bd7 f   asxclass.obj
 0001:00064be2       __ehhandler$?asxCreateSubSystem@@YA?AW4asxERROR@@PAVasxSystem@@HPAPAVasxSubSystem@@@Z 10065be2 f   asxclass.obj
 0001:00064c00       __unwindfunclet$??1asxMixerScannerDSND@@UAE@XZ$0 10065c00 f   asxdsnd.obj
 0001:00064c08       __ehhandler$??1asxMixerScannerDSND@@UAE@XZ 10065c08 f   asxdsnd.obj
 0001:00064c30       __unwindfunclet$?Scan@asxMixerScannerDSND@@EAEXPAVasxMixer@@@Z$0 10065c30 f   asxdsnd.obj
 0001:00064c3b       __unwindfunclet$?Scan@asxMixerScannerDSND@@EAEXPAVasxMixer@@@Z$1 10065c3b f   asxdsnd.obj
 0001:00064c46       __unwindfunclet$?Scan@asxMixerScannerDSND@@EAEXPAVasxMixer@@@Z$2 10065c46 f   asxdsnd.obj
 0001:00064c51       __unwindfunclet$?Scan@asxMixerScannerDSND@@EAEXPAVasxMixer@@@Z$3 10065c51 f   asxdsnd.obj
 0001:00064c5c       __ehhandler$?Scan@asxMixerScannerDSND@@EAEXPAVasxMixer@@@Z 10065c5c f   asxdsnd.obj
 0001:00064c80       __unwindfunclet$?Scan@asxSubSystemDSND@@UAEXXZ$0 10065c80 f   asxdsnd.obj
 0001:00064c88       __unwindfunclet$?Scan@asxSubSystemDSND@@UAEXXZ$1 10065c88 f   asxdsnd.obj
 0001:00064c93       __ehhandler$?Scan@asxSubSystemDSND@@UAEXXZ 10065c93 f   asxdsnd.obj
 0001:00064cb0       __unwindfunclet$??0asxPlayerDSND@@QAE@PAVasxSubSystem@@PAVasxNode@@1PBU_GUID@@@Z$0 10065cb0 f   asxdsndplay.obj
 0001:00064cb8       __ehhandler$??0asxPlayerDSND@@QAE@PAVasxSubSystem@@PAVasxNode@@1PBU_GUID@@@Z 10065cb8 f   asxdsndplay.obj
 0001:00064ce0       __unwindfunclet$??1asxPlayerDSND@@UAE@XZ$0 10065ce0 f   asxdsndplay.obj
 0001:00064ce8       __ehhandler$??1asxPlayerDSND@@UAE@XZ 10065ce8 f   asxdsndplay.obj
 0001:00064d10       __unwindfunclet$??1asxRecorderDSND@@UAE@XZ$0 10065d10 f   asxdsndrec.obj
 0001:00064d18       __ehhandler$??1asxRecorderDSND@@UAE@XZ 10065d18 f   asxdsndrec.obj
 0001:00064d40       __unwindfunclet$??0asxAdapterHPI@@QAE@PAVasxSystem@@HPBD@Z$0 10065d40 f   asxhpi.obj
 0001:00064d4b       __unwindfunclet$??0asxAdapterHPI@@QAE@PAVasxSystem@@HPBD@Z$1 10065d4b f   asxhpi.obj
 0001:00064d5c       __ehhandler$??0asxAdapterHPI@@QAE@PAVasxSystem@@HPBD@Z 10065d5c f   asxhpi.obj
 0001:00064d90       __unwindfunclet$??0asxAes3TxHPI@@QAE@PAVasxSubSystem@@PAVasxNode@@1I@Z$0 10065d90 f   asxhpi.obj
 0001:00064d98       __ehhandler$??0asxAes3TxHPI@@QAE@PAVasxSubSystem@@PAVasxNode@@1I@Z 10065d98 f   asxhpi.obj
 0001:00064dc0       __unwindfunclet$??0asxAesebuReceiverHPI@@QAE@PAVasxSubSystem@@PAVasxNode@@1I@Z$0 10065dc0 f   asxhpi.obj
 0001:00064dc8       __ehhandler$??0asxAesebuReceiverHPI@@QAE@PAVasxSubSystem@@PAVasxNode@@1I@Z 10065dc8 f   asxhpi.obj
 0001:00064df0       __unwindfunclet$??0asxCobranetHPI@@QAE@PAVasxSubSystem@@PAVasxNode@@1IH@Z$0 10065df0 f   asxhpi.obj
 0001:00064df8       __ehhandler$??0asxCobranetHPI@@QAE@PAVasxSubSystem@@PAVasxNode@@1IH@Z 10065df8 f   asxhpi.obj
 0001:00064e20       __unwindfunclet$??0asxCobranetRxHPI@@QAE@PAVasxSubSystem@@PAVasxNode@@1IH@Z$0 10065e20 f   asxhpi.obj
 0001:00064e28       __ehhandler$??0asxCobranetRxHPI@@QAE@PAVasxSubSystem@@PAVasxNode@@1IH@Z 10065e28 f   asxhpi.obj
 0001:00064e50       __unwindfunclet$??0asxCobranetTxHPI@@QAE@PAVasxSubSystem@@PAVasxNode@@1IH@Z$0 10065e50 f   asxhpi.obj
 0001:00064e58       __ehhandler$??0asxCobranetTxHPI@@QAE@PAVasxSubSystem@@PAVasxNode@@1IH@Z 10065e58 f   asxhpi.obj
 0001:00064e80       __unwindfunclet$??0asxCompanderHPI_Legacy@@QAE@PAVasxSubSystem@@PAVasxNode@@1I@Z$0 10065e80 f   asxhpi.obj
 0001:00064e88       __ehhandler$??0asxCompanderHPI_Legacy@@QAE@PAVasxSubSystem@@PAVasxNode@@1I@Z 10065e88 f   asxhpi.obj
 0001:00064eb0       __unwindfunclet$??0asxGpioHPI@@QAE@PAVasxSubSystem@@PAVasxNode@@1IHH@Z$0 10065eb0 f   asxhpi.obj
 0001:00064eb8       __ehhandler$??0asxGpioHPI@@QAE@PAVasxSubSystem@@PAVasxNode@@1IHH@Z 10065eb8 f   asxhpi.obj
 0001:00064ee0       __unwindfunclet$??0asxModeHPI@@QAE@PAVasxSubSystem@@PAVasxNode@@1I@Z$0 10065ee0 f   asxhpi.obj
 0001:00064ee8       __unwindfunclet$??0asxModeHPI@@QAE@PAVasxSubSystem@@PAVasxNode@@1I@Z$1 10065ee8 f   asxhpi.obj
 0001:00064ef3       __ehhandler$??0asxModeHPI@@QAE@PAVasxSubSystem@@PAVasxNode@@1I@Z 10065ef3 f   asxhpi.obj
 0001:00064f10       __unwindfunclet$??0asxMuxHPI@@QAE@PAVasxSubSystem@@PAVasxNode@@1I@Z$0 10065f10 f   asxhpi.obj
 0001:00064f18       __unwindfunclet$??0asxMuxHPI@@QAE@PAVasxSubSystem@@PAVasxNode@@1I@Z$1 10065f18 f   asxhpi.obj
 0001:00064f23       __unwindfunclet$??0asxMuxHPI@@QAE@PAVasxSubSystem@@PAVasxNode@@1I@Z$2 10065f23 f   asxhpi.obj
 0001:00064f2e       __ehhandler$??0asxMuxHPI@@QAE@PAVasxSubSystem@@PAVasxNode@@1I@Z 10065f2e f   asxhpi.obj
 0001:00064f50       __unwindfunclet$??0asxSampleClockHPI@@QAE@PAVasxSubSystem@@PAVasxNode@@1I@Z$0 10065f50 f   asxhpi.obj
 0001:00064f58       __unwindfunclet$??0asxSampleClockHPI@@QAE@PAVasxSubSystem@@PAVasxNode@@1I@Z$1 10065f58 f   asxhpi.obj
 0001:00064f63       __unwindfunclet$??0asxSampleClockHPI@@QAE@PAVasxSubSystem@@PAVasxNode@@1I@Z$2 10065f63 f   asxhpi.obj
 0001:00064f6e       __ehhandler$??0asxSampleClockHPI@@QAE@PAVasxSubSystem@@PAVasxNode@@1I@Z 10065f6e f   asxhpi.obj
 0001:00064fa0       __unwindfunclet$??0asxSubSystemHPI@@QAE@PAVasxSystem@@H@Z$0 10065fa0 f   asxhpi.obj
 0001:00064fa8       __ehhandler$??0asxSubSystemHPI@@QAE@PAVasxSystem@@H@Z 10065fa8 f   asxhpi.obj
 0001:00064fd0       __unwindfunclet$??0asxTunerHPI@@QAE@PAVasxSubSystem@@PAVasxNode@@1I@Z$0 10065fd0 f   asxhpi.obj
 0001:00064fd8       __ehhandler$??0asxTunerHPI@@QAE@PAVasxSubSystem@@PAVasxNode@@1I@Z 10065fd8 f   asxhpi.obj
 0001:00065000       __unwindfunclet$??1asxAdapterHPI@@UAE@XZ$0 10066000 f   asxhpi.obj
 0001:00065008       __ehhandler$??1asxAdapterHPI@@UAE@XZ 10066008 f   asxhpi.obj
 0001:00065030       __unwindfunclet$??1asxAes3Rx@@UAE@XZ$0 10066030 f   asxhpi.obj
 0001:00065038       __ehhandler$??1asxAes3Rx@@UAE@XZ 10066038 f   asxhpi.obj
 0001:00065060       __unwindfunclet$??1asxAes3Tx@@UAE@XZ$0 10066060 f   asxhpi.obj
 0001:00065068       __ehhandler$??1asxAes3Tx@@UAE@XZ 10066068 f   asxhpi.obj
 0001:00065090       __unwindfunclet$??1asxAes3TxHPI@@UAE@XZ$1 10066090 f   asxhpi.obj
 0001:00065098       __ehhandler$??1asxAes3TxHPI@@UAE@XZ 10066098 f   asxhpi.obj
 0001:000650c0       __unwindfunclet$??1asxAesebuReceiverHPI@@UAE@XZ$1 100660c0 f   asxhpi.obj
 0001:000650c8       __ehhandler$??1asxAesebuReceiverHPI@@UAE@XZ 100660c8 f   asxhpi.obj
 0001:000650f0       __unwindfunclet$??1asxBlock@@UAE@XZ$0 100660f0 f   asxhpi.obj
 0001:000650f8       __ehhandler$??1asxBlock@@UAE@XZ 100660f8 f   asxhpi.obj
 0001:00065120       __unwindfunclet$??1asxBlockHPI@@UAE@XZ$1 10066120 f   asxhpi.obj
 0001:00065128       __ehhandler$??1asxBlockHPI@@UAE@XZ 10066128 f   asxhpi.obj
 0001:00065150       __unwindfunclet$??1asxCobranetContainer@@UAE@XZ$0 10066150 f   asxhpi.obj
 0001:00065158       __ehhandler$??1asxCobranetContainer@@UAE@XZ 10066158 f   asxhpi.obj
 0001:00065180       __unwindfunclet$??1asxCobranetRxContainer@@UAE@XZ$0 10066180 f   asxhpi.obj
 0001:00065188       __ehhandler$??1asxCobranetRxContainer@@UAE@XZ 10066188 f   asxhpi.obj
 0001:000651b0       __unwindfunclet$??1asxCobranetTxContainer@@UAE@XZ$0 100661b0 f   asxhpi.obj
 0001:000651b8       __ehhandler$??1asxCobranetTxContainer@@UAE@XZ 100661b8 f   asxhpi.obj
 0001:000651e0       __unwindfunclet$??1asxGpioHPI@@UAE@XZ$0 100661e0 f   asxhpi.obj
 0001:000651e8       __ehhandler$??1asxGpioHPI@@UAE@XZ 100661e8 f   asxhpi.obj
 0001:00065210       __unwindfunclet$??1asxMode@@UAE@XZ$0 10066210 f   asxhpi.obj
 0001:00065218       __ehhandler$??1asxMode@@UAE@XZ 10066218 f   asxhpi.obj
 0001:00065240       __unwindfunclet$??1asxModeHPI@@UAE@XZ$0 10066240 f   asxhpi.obj
 0001:00065248       __unwindfunclet$??1asxModeHPI@@UAE@XZ$2 10066248 f   asxhpi.obj
 0001:00065250       __ehhandler$??1asxModeHPI@@UAE@XZ 10066250 f   asxhpi.obj
 0001:00065270       __unwindfunclet$??1asxMux@@UAE@XZ$0 10066270 f   asxhpi.obj
 0001:00065278       __unwindfunclet$??1asxMux@@UAE@XZ$1 10066278 f   asxhpi.obj
 0001:00065283       __ehhandler$??1asxMux@@UAE@XZ 10066283 f   asxhpi.obj
 0001:000652a0       __unwindfunclet$??1asxMuxHPI@@UAE@XZ$0 100662a0 f   asxhpi.obj
 0001:000652a8       __unwindfunclet$??1asxMuxHPI@@UAE@XZ$2 100662a8 f   asxhpi.obj
 0001:000652b0       __unwindfunclet$??1asxMuxHPI@@UAE@XZ$3 100662b0 f   asxhpi.obj
 0001:000652bb       __ehhandler$??1asxMuxHPI@@UAE@XZ 100662bb f   asxhpi.obj
 0001:000652e0       __unwindfunclet$??1asxSampleClock@@UAE@XZ$0 100662e0 f   asxhpi.obj
 0001:000652e8       __unwindfunclet$??1asxSampleClock@@UAE@XZ$1 100662e8 f   asxhpi.obj
 0001:000652f3       __ehhandler$??1asxSampleClock@@UAE@XZ 100662f3 f   asxhpi.obj
 0001:00065310       __unwindfunclet$??1asxSampleClockHPI@@UAE@XZ$0 10066310 f   asxhpi.obj
 0001:00065318       __unwindfunclet$??1asxSampleClockHPI@@UAE@XZ$1 10066318 f   asxhpi.obj
 0001:00065323       __unwindfunclet$??1asxSampleClockHPI@@UAE@XZ$3 10066323 f   asxhpi.obj
 0001:0006532b       __unwindfunclet$??1asxSampleClockHPI@@UAE@XZ$4 1006632b f   asxhpi.obj
 0001:00065336       __ehhandler$??1asxSampleClockHPI@@UAE@XZ 10066336 f   asxhpi.obj
 0001:00065360       __unwindfunclet$??1asxTuner@@UAE@XZ$0 10066360 f   asxhpi.obj
 0001:00065368       __unwindfunclet$??1asxTuner@@UAE@XZ$1 10066368 f   asxhpi.obj
 0001:00065373       __ehhandler$??1asxTuner@@UAE@XZ 10066373 f   asxhpi.obj
 0001:00065390       __unwindfunclet$??1asxTunerHPI@@UAE@XZ$1 10066390 f   asxhpi.obj
 0001:00065398       __unwindfunclet$??1asxTunerHPI@@UAE@XZ$2 10066398 f   asxhpi.obj
 0001:000653a3       __ehhandler$??1asxTunerHPI@@UAE@XZ 100663a3 f   asxhpi.obj
 0001:000653c0       __unwindfunclet$??_GasxAes3Rx@@UAEPAXI@Z$0 100663c0 f   asxhpi.obj
 0001:000653c8       __ehhandler$??_GasxAes3Rx@@UAEPAXI@Z 100663c8 f   asxhpi.obj
 0001:000653f0       __unwindfunclet$??_GasxAes3Tx@@UAEPAXI@Z$0 100663f0 f   asxhpi.obj
 0001:000653f8       __ehhandler$??_GasxAes3Tx@@UAEPAXI@Z 100663f8 f   asxhpi.obj
 0001:00065420       __unwindfunclet$??_GasxBlock@@UAEPAXI@Z$0 10066420 f   asxhpi.obj
 0001:00065428       __ehhandler$??_GasxBlock@@UAEPAXI@Z 10066428 f   asxhpi.obj
 0001:00065450       __unwindfunclet$??_GasxCobranetContainer@@UAEPAXI@Z$0 10066450 f   asxhpi.obj
 0001:00065458       __ehhandler$??_GasxCobranetContainer@@UAEPAXI@Z 10066458 f   asxhpi.obj
 0001:00065480       __unwindfunclet$??_GasxCobranetRxContainer@@UAEPAXI@Z$0 10066480 f   asxhpi.obj
 0001:00065488       __ehhandler$??_GasxCobranetRxContainer@@UAEPAXI@Z 10066488 f   asxhpi.obj
 0001:000654b0       __unwindfunclet$??_GasxCobranetTxContainer@@UAEPAXI@Z$0 100664b0 f   asxhpi.obj
 0001:000654b8       __ehhandler$??_GasxCobranetTxContainer@@UAEPAXI@Z 100664b8 f   asxhpi.obj
 0001:000654e0       __unwindfunclet$??_GasxMode@@UAEPAXI@Z$0 100664e0 f   asxhpi.obj
 0001:000654e8       __ehhandler$??_GasxMode@@UAEPAXI@Z 100664e8 f   asxhpi.obj
 0001:00065510       __unwindfunclet$??_GasxMux@@UAEPAXI@Z$0 10066510 f   asxhpi.obj
 0001:00065518       __unwindfunclet$??_GasxMux@@UAEPAXI@Z$1 10066518 f   asxhpi.obj
 0001:00065523       __ehhandler$??_GasxMux@@UAEPAXI@Z 10066523 f   asxhpi.obj
 0001:00065540       __unwindfunclet$??_GasxSampleClock@@UAEPAXI@Z$0 10066540 f   asxhpi.obj
 0001:00065548       __unwindfunclet$??_GasxSampleClock@@UAEPAXI@Z$1 10066548 f   asxhpi.obj
 0001:00065553       __ehhandler$??_GasxSampleClock@@UAEPAXI@Z 10066553 f   asxhpi.obj
 0001:00065570       __unwindfunclet$??_GasxTuner@@UAEPAXI@Z$0 10066570 f   asxhpi.obj
 0001:00065578       __unwindfunclet$??_GasxTuner@@UAEPAXI@Z$1 10066578 f   asxhpi.obj
 0001:00065583       __ehhandler$??_GasxTuner@@UAEPAXI@Z 10066583 f   asxhpi.obj
 0001:000655a0       __unwindfunclet$?AddDuplicateIndexAdapter@asxSubSystemHPI@@AAEXIGG@Z$0 100665a0 f   asxhpi.obj
 0001:000655ae       __ehhandler$?AddDuplicateIndexAdapter@asxSubSystemHPI@@AAEXIGG@Z 100665ae f   asxhpi.obj
 0001:000655e0       __unwindfunclet$?AddProperty@asxBlockHPI@@QAE?AW4asxERROR@@I@Z$20 100665e0 f   asxhpi.obj
 0001:000655ee       __ehhandler$?AddProperty@asxBlockHPI@@QAE?AW4asxERROR@@I@Z 100665ee f   asxhpi.obj
 0001:00065620       __unwindfunclet$?AddSingleAdapter@asxSubSystemHPI@@AAEHIG@Z$0 10066620 f   asxhpi.obj
 0001:0006562e       __unwindfunclet$?AddSingleAdapter@asxSubSystemHPI@@AAEHIG@Z$1 1006662e f   asxhpi.obj
 0001:0006563c       __ehhandler$?AddSingleAdapter@asxSubSystemHPI@@AAEHIG@Z 1006663c f   asxhpi.obj
 0001:00065670       __unwindfunclet$?CreateUniversalControl@asxMixerScannerHPI@@QAEPAVasxControlBase@@PAHPAVasxNode@@1I@Z$0 10066670 f   asxhpi.obj
 0001:0006567b       __ehhandler$?CreateUniversalControl@asxMixerScannerHPI@@QAEPAVasxControlBase@@PAHPAVasxNode@@1I@Z 1006667b f   asxhpi.obj
 0001:000656a0       __unwindfunclet$?Scan@asxMixerScannerHPI@@UAEXPAVasxMixer@@@Z$0 100666a0 f   asxhpi.obj
 0001:000656ae       __unwindfunclet$?Scan@asxMixerScannerHPI@@UAEXPAVasxMixer@@@Z$1 100666ae f   asxhpi.obj
 0001:000656bc       __unwindfunclet$?Scan@asxMixerScannerHPI@@UAEXPAVasxMixer@@@Z$2 100666bc f   asxhpi.obj
 0001:000656ca       __unwindfunclet$?Scan@asxMixerScannerHPI@@UAEXPAVasxMixer@@@Z$3 100666ca f   asxhpi.obj
 0001:000656d8       __unwindfunclet$?Scan@asxMixerScannerHPI@@UAEXPAVasxMixer@@@Z$4 100666d8 f   asxhpi.obj
 0001:000656e6       __unwindfunclet$?Scan@asxMixerScannerHPI@@UAEXPAVasxMixer@@@Z$5 100666e6 f   asxhpi.obj
 0001:000656f4       __unwindfunclet$?Scan@asxMixerScannerHPI@@UAEXPAVasxMixer@@@Z$6 100666f4 f   asxhpi.obj
 0001:00065702       __unwindfunclet$?Scan@asxMixerScannerHPI@@UAEXPAVasxMixer@@@Z$7 10066702 f   asxhpi.obj
 0001:00065710       __unwindfunclet$?Scan@asxMixerScannerHPI@@UAEXPAVasxMixer@@@Z$8 10066710 f   asxhpi.obj
 0001:0006571e       __unwindfunclet$?Scan@asxMixerScannerHPI@@UAEXPAVasxMixer@@@Z$9 1006671e f   asxhpi.obj
 0001:0006572c       __unwindfunclet$?Scan@asxMixerScannerHPI@@UAEXPAVasxMixer@@@Z$10 1006672c f   asxhpi.obj
 0001:0006573a       __unwindfunclet$?Scan@asxMixerScannerHPI@@UAEXPAVasxMixer@@@Z$11 1006673a f   asxhpi.obj
 0001:00065748       __unwindfunclet$?Scan@asxMixerScannerHPI@@UAEXPAVasxMixer@@@Z$12 10066748 f   asxhpi.obj
 0001:00065756       __unwindfunclet$?Scan@asxMixerScannerHPI@@UAEXPAVasxMixer@@@Z$13 10066756 f   asxhpi.obj
 0001:00065764       __unwindfunclet$?Scan@asxMixerScannerHPI@@UAEXPAVasxMixer@@@Z$14 10066764 f   asxhpi.obj
 0001:00065772       __unwindfunclet$?Scan@asxMixerScannerHPI@@UAEXPAVasxMixer@@@Z$15 10066772 f   asxhpi.obj
 0001:00065780       __unwindfunclet$?Scan@asxMixerScannerHPI@@UAEXPAVasxMixer@@@Z$16 10066780 f   asxhpi.obj
 0001:0006578e       __unwindfunclet$?Scan@asxMixerScannerHPI@@UAEXPAVasxMixer@@@Z$17 1006678e f   asxhpi.obj
 0001:0006579c       __unwindfunclet$?Scan@asxMixerScannerHPI@@UAEXPAVasxMixer@@@Z$18 1006679c f   asxhpi.obj
 0001:000657aa       __unwindfunclet$?Scan@asxMixerScannerHPI@@UAEXPAVasxMixer@@@Z$19 100667aa f   asxhpi.obj
 0001:000657b8       __unwindfunclet$?Scan@asxMixerScannerHPI@@UAEXPAVasxMixer@@@Z$20 100667b8 f   asxhpi.obj
 0001:000657c6       __unwindfunclet$?Scan@asxMixerScannerHPI@@UAEXPAVasxMixer@@@Z$21 100667c6 f   asxhpi.obj
 0001:000657d4       __unwindfunclet$?Scan@asxMixerScannerHPI@@UAEXPAVasxMixer@@@Z$22 100667d4 f   asxhpi.obj
 0001:000657e2       __unwindfunclet$?Scan@asxMixerScannerHPI@@UAEXPAVasxMixer@@@Z$23 100667e2 f   asxhpi.obj
 0001:000657f0       __unwindfunclet$?Scan@asxMixerScannerHPI@@UAEXPAVasxMixer@@@Z$24 100667f0 f   asxhpi.obj
 0001:000657fe       __unwindfunclet$?Scan@asxMixerScannerHPI@@UAEXPAVasxMixer@@@Z$25 100667fe f   asxhpi.obj
 0001:0006580c       __unwindfunclet$?Scan@asxMixerScannerHPI@@UAEXPAVasxMixer@@@Z$26 1006680c f   asxhpi.obj
 0001:0006581a       __unwindfunclet$?Scan@asxMixerScannerHPI@@UAEXPAVasxMixer@@@Z$27 1006681a f   asxhpi.obj
 0001:00065828       __unwindfunclet$?Scan@asxMixerScannerHPI@@UAEXPAVasxMixer@@@Z$28 10066828 f   asxhpi.obj
 0001:00065836       __unwindfunclet$?Scan@asxMixerScannerHPI@@UAEXPAVasxMixer@@@Z$29 10066836 f   asxhpi.obj
 0001:00065844       __unwindfunclet$?Scan@asxMixerScannerHPI@@UAEXPAVasxMixer@@@Z$30 10066844 f   asxhpi.obj
 0001:00065852       __unwindfunclet$?Scan@asxMixerScannerHPI@@UAEXPAVasxMixer@@@Z$31 10066852 f   asxhpi.obj
 0001:00065860       __unwindfunclet$?Scan@asxMixerScannerHPI@@UAEXPAVasxMixer@@@Z$32 10066860 f   asxhpi.obj
 0001:0006586e       __unwindfunclet$?Scan@asxMixerScannerHPI@@UAEXPAVasxMixer@@@Z$33 1006686e f   asxhpi.obj
 0001:0006587c       __unwindfunclet$?Scan@asxMixerScannerHPI@@UAEXPAVasxMixer@@@Z$34 1006687c f   asxhpi.obj
 0001:0006588a       __unwindfunclet$?Scan@asxMixerScannerHPI@@UAEXPAVasxMixer@@@Z$35 1006688a f   asxhpi.obj
 0001:00065898       __unwindfunclet$?Scan@asxMixerScannerHPI@@UAEXPAVasxMixer@@@Z$36 10066898 f   asxhpi.obj
 0001:000658a6       __ehhandler$?Scan@asxMixerScannerHPI@@UAEXPAVasxMixer@@@Z 100668a6 f   asxhpi.obj
 0001:000658d0       __unwindfunclet$??1asxPlayerHPI@@UAE@XZ$0 100668d0 f   asxhpiplay.obj
 0001:000658d8       __ehhandler$??1asxPlayerHPI@@UAE@XZ 100668d8 f   asxhpiplay.obj
 0001:00065900       __unwindfunclet$??1asxRecorderHPI@@UAE@XZ$0 10066900 f   asxhpirec.obj
 0001:00065908       __ehhandler$??1asxRecorderHPI@@UAE@XZ 10066908 f   asxhpirec.obj
 0001:00065930       __unwindfunclet$??1asxPlayer@@UAE@XZ$0 10066930 f   asxplay.obj
 0001:00065938       __unwindfunclet$??1asxPlayer@@UAE@XZ$1 10066938 f   asxplay.obj
 0001:00065943       __ehhandler$??1asxPlayer@@UAE@XZ 10066943 f   asxplay.obj
 0001:00065960       __unwindfunclet$?AddFile@asxPlayerFileList@@QAEXPBD@Z$0 10066960 f   asxplay.obj
 0001:0006596b       __ehhandler$?AddFile@asxPlayerFileList@@QAEXPBD@Z 1006696b f   asxplay.obj
 0001:00065990       __unwindfunclet$?Close@asxPlayer@@UAE?AW4asxERROR@@XZ$0 10066990 f   asxplay.obj
 0001:00065998       __ehhandler$?Close@asxPlayer@@UAE?AW4asxERROR@@XZ 10066998 f   asxplay.obj
 0001:000659c0       __unwindfunclet$?Open@asxPlayerFile@@QAE?AW4asxERROR@@XZ$0 100669c0 f   asxplay.obj
 0001:000659cb       __ehhandler$?Open@asxPlayerFile@@QAE?AW4asxERROR@@XZ 100669cb f   asxplay.obj
 0001:000659f0       __unwindfunclet$?OpenPlaylist@asxPlayer@@UAE?AW4asxERROR@@PAPBDI@Z$0 100669f0 f   asxplay.obj
 0001:000659f8       __ehhandler$?OpenPlaylist@asxPlayer@@UAE?AW4asxERROR@@PAPBDI@Z 100669f8 f   asxplay.obj
 0001:00065a20       __unwindfunclet$?Pause@asxPlayer@@UAE?AW4asxERROR@@XZ$0 10066a20 f   asxplay.obj
 0001:00065a28       __ehhandler$?Pause@asxPlayer@@UAE?AW4asxERROR@@XZ 10066a28 f   asxplay.obj
 0001:00065a50       __unwindfunclet$?PreLoad@asxPlayer@@UAE?AW4asxERROR@@W4asxTIMESCALE@@K@Z$0 10066a50 f   asxplay.obj
 0001:00065a58       __ehhandler$?PreLoad@asxPlayer@@UAE?AW4asxERROR@@W4asxTIMESCALE@@K@Z 10066a58 f   asxplay.obj
 0001:00065a80       __unwindfunclet$?Start@asxPlayer@@UAE?AW4asxERROR@@XZ$0 10066a80 f   asxplay.obj
 0001:00065a88       __ehhandler$?Start@asxPlayer@@UAE?AW4asxERROR@@XZ 10066a88 f   asxplay.obj
 0001:00065ab0       __unwindfunclet$?Stop@asxPlayer@@UAE?AW4asxERROR@@XZ$0 10066ab0 f   asxplay.obj
 0001:00065ab8       __ehhandler$?Stop@asxPlayer@@UAE?AW4asxERROR@@XZ 10066ab8 f   asxplay.obj
 0001:00065ae0       __unwindfunclet$??1asxRecorder@@UAE@XZ$0 10066ae0 f   asxrec.obj
 0001:00065ae8       __ehhandler$??1asxRecorder@@UAE@XZ 10066ae8 f   asxrec.obj
 0001:00065b10       __unwindfunclet$?CreateFileA@asxRecorder@@MAE?AW4asxERROR@@XZ$0 10066b10 f   asxrec.obj
 0001:00065b1b       __ehhandler$?CreateFileA@asxRecorder@@MAE?AW4asxERROR@@XZ 10066b1b f   asxrec.obj
 0001:00065b40       __unwindfunclet$??0asxAdapterSNMP@@QAE@PAVasxSystem@@PADPBD2PAVSnmpSession@@@Z$0 10066b40 f   asxsnmp.obj
 0001:00065b48       __unwindfunclet$??0asxAdapterSNMP@@QAE@PAVasxSystem@@PADPBD2PAVSnmpSession@@@Z$1 10066b48 f   asxsnmp.obj
 0001:00065b53       __ehhandler$??0asxAdapterSNMP@@QAE@PAVasxSystem@@PADPBD2PAVSnmpSession@@@Z 10066b53 f   asxsnmp.obj
 0001:00065b80       __unwindfunclet$??0asxCobranetSNMP@@QAE@PAVasxSubSystem@@PAVasxNode@@1PAVCobraNetNode@@PBD@Z$0 10066b80 f   asxsnmp.obj
 0001:00065b8b       __ehhandler$??0asxCobranetSNMP@@QAE@PAVasxSubSystem@@PAVasxNode@@1PAVCobraNetNode@@PBD@Z 10066b8b f   asxsnmp.obj
 0001:00065bc0       __unwindfunclet$??0asxSubSystemSNMP@@QAE@PAVasxSystem@@@Z$0 10066bc0 f   asxsnmp.obj
 0001:00065bc8       __unwindfunclet$??0asxSubSystemSNMP@@QAE@PAVasxSystem@@@Z$1 10066bc8 f   asxsnmp.obj
 0001:00065bd3       __ehhandler$??0asxSubSystemSNMP@@QAE@PAVasxSystem@@@Z 10066bd3 f   asxsnmp.obj
 0001:00065c00       __unwindfunclet$??1asxAdapterSNMP@@UAE@XZ$0 10066c00 f   asxsnmp.obj
 0001:00065c08       __ehhandler$??1asxAdapterSNMP@@UAE@XZ 10066c08 f   asxsnmp.obj
 0001:00065c30       __unwindfunclet$??1asxSubSystemSNMP@@UAE@XZ$0 10066c30 f   asxsnmp.obj
 0001:00065c38       __unwindfunclet$??1asxSubSystemSNMP@@UAE@XZ$1 10066c38 f   asxsnmp.obj
 0001:00065c43       __ehhandler$??1asxSubSystemSNMP@@UAE@XZ 10066c43 f   asxsnmp.obj
 0001:00065c60       __unwindfunclet$?NewIpAddress@asxAdapterSNMP@@QAEXPBD@Z$0 10066c60 f   asxsnmp.obj
 0001:00065c6b       __ehhandler$?NewIpAddress@asxAdapterSNMP@@QAEXPBD@Z 10066c6b f   asxsnmp.obj
 0001:00065c90       __unwindfunclet$?ReScan@asxSubSystemSNMP@@UAEXXZ$0 10066c90 f   asxsnmp.obj
 0001:00065c9e       __unwindfunclet$?ReScan@asxSubSystemSNMP@@UAEXXZ$1 10066c9e f   asxsnmp.obj
 0001:00065cac       __unwindfunclet$?ReScan@asxSubSystemSNMP@@UAEXXZ$4 10066cac f   asxsnmp.obj
 0001:00065cb7       __ehhandler$?ReScan@asxSubSystemSNMP@@UAEXXZ 10066cb7 f   asxsnmp.obj
 0001:00065ce0       __unwindfunclet$?Scan@asxMixerScannerSNMP@@UAEXPAVasxMixer@@@Z$0 10066ce0 f   asxsnmp.obj
 0001:00065cee       __unwindfunclet$?Scan@asxMixerScannerSNMP@@UAEXPAVasxMixer@@@Z$1 10066cee f   asxsnmp.obj
 0001:00065cfc       __unwindfunclet$?Scan@asxMixerScannerSNMP@@UAEXPAVasxMixer@@@Z$2 10066cfc f   asxsnmp.obj
 0001:00065d0a       __unwindfunclet$?Scan@asxMixerScannerSNMP@@UAEXPAVasxMixer@@@Z$3 10066d0a f   asxsnmp.obj
 0001:00065d18       __unwindfunclet$?Scan@asxMixerScannerSNMP@@UAEXPAVasxMixer@@@Z$7 10066d18 f   asxsnmp.obj
 0001:00065d26       __unwindfunclet$?Scan@asxMixerScannerSNMP@@UAEXPAVasxMixer@@@Z$4 10066d26 f   asxsnmp.obj
 0001:00065d34       __unwindfunclet$?Scan@asxMixerScannerSNMP@@UAEXPAVasxMixer@@@Z$5 10066d34 f   asxsnmp.obj
 0001:00065d42       __unwindfunclet$?Scan@asxMixerScannerSNMP@@UAEXPAVasxMixer@@@Z$6 10066d42 f   asxsnmp.obj
 0001:00065d50       __unwindfunclet$?Scan@asxMixerScannerSNMP@@UAEXPAVasxMixer@@@Z$8 10066d50 f   asxsnmp.obj
 0001:00065d5e       __unwindfunclet$?Scan@asxMixerScannerSNMP@@UAEXPAVasxMixer@@@Z$9 10066d5e f   asxsnmp.obj
 0001:00065d6c       __unwindfunclet$?Scan@asxMixerScannerSNMP@@UAEXPAVasxMixer@@@Z$10 10066d6c f   asxsnmp.obj
 0001:00065d7a       __ehhandler$?Scan@asxMixerScannerSNMP@@UAEXPAVasxMixer@@@Z 10066d7a f   asxsnmp.obj
 0001:00065db0       __unwindfunclet$?Scan@asxMixerScannerUnreachableSNMP@@UAEXPAVasxMixer@@@Z$0 10066db0 f   asxsnmp.obj
 0001:00065dbb       __unwindfunclet$?Scan@asxMixerScannerUnreachableSNMP@@UAEXPAVasxMixer@@@Z$1 10066dbb f   asxsnmp.obj
 0001:00065dc6       __unwindfunclet$?Scan@asxMixerScannerUnreachableSNMP@@UAEXPAVasxMixer@@@Z$2 10066dc6 f   asxsnmp.obj
 0001:00065dd1       __ehhandler$?Scan@asxMixerScannerUnreachableSNMP@@UAEXPAVasxMixer@@@Z 10066dd1 f   asxsnmp.obj
 0001:00065df0       __unwindfunclet$??0asxBlockTR800OptoMode@@QAE@PAVasxSubSystem@@PAVasxTR800helperthread@@PAVasxNode@@2@Z$0 10066df0 f   asxtr800.obj
 0001:00065df8       __unwindfunclet$??0asxBlockTR800OptoMode@@QAE@PAVasxSubSystem@@PAVasxTR800helperthread@@PAVasxNode@@2@Z$1 10066df8 f   asxtr800.obj
 0001:00065e03       __ehhandler$??0asxBlockTR800OptoMode@@QAE@PAVasxSubSystem@@PAVasxTR800helperthread@@PAVasxNode@@2@Z 10066e03 f   asxtr800.obj
 0001:00065e30       __unwindfunclet$??0asxBlockTR800Status@@QAE@PAVasxSubSystem@@PAVasxNode@@1_N@Z$0 10066e30 f   asxtr800.obj
 0001:00065e38       __unwindfunclet$??0asxBlockTR800Status@@QAE@PAVasxSubSystem@@PAVasxNode@@1_N@Z$1 10066e38 f   asxtr800.obj
 0001:00065e43       __ehhandler$??0asxBlockTR800Status@@QAE@PAVasxSubSystem@@PAVasxNode@@1_N@Z 10066e43 f   asxtr800.obj
 0001:00065e70       __unwindfunclet$??0asxLevelTR800@@QAE@PAVasxSubSystem@@PAVasxTR800helperthread@@PAVasxNode@@2@Z$0 10066e70 f   asxtr800.obj
 0001:00065e78       __ehhandler$??0asxLevelTR800@@QAE@PAVasxSubSystem@@PAVasxTR800helperthread@@PAVasxNode@@2@Z 10066e78 f   asxtr800.obj
 0001:00065ea0       __unwindfunclet$??1asxBlockTR800OptoMode@@UAE@XZ$1 10066ea0 f   asxtr800.obj
 0001:00065ea8       __ehhandler$??1asxBlockTR800OptoMode@@UAE@XZ 10066ea8 f   asxtr800.obj
 0001:00065ed0       __unwindfunclet$??1asxBlockTR800Status@@UAE@XZ$1 10066ed0 f   asxtr800.obj
 0001:00065ed8       __ehhandler$??1asxBlockTR800Status@@UAE@XZ 10066ed8 f   asxtr800.obj
 0001:00065f00       __unwindfunclet$??_GasxBlockTR800OptoMode@@UAEPAXI@Z$1 10066f00 f   asxtr800.obj
 0001:00065f08       __ehhandler$??_GasxBlockTR800OptoMode@@UAEPAXI@Z 10066f08 f   asxtr800.obj
 0001:00065f30       __unwindfunclet$??_GasxBlockTR800Status@@UAEPAXI@Z$1 10066f30 f   asxtr800.obj
 0001:00065f38       __ehhandler$??_GasxBlockTR800Status@@UAEPAXI@Z 10066f38 f   asxtr800.obj
 0001:00065f60       __unwindfunclet$?asxTR800_Create@@YAXPAVasxSubSystem@@PAVCobraNetNode@@PAVasxMixer@@@Z$0 10066f60 f   asxtr800.obj
 0001:00065f6b       __unwindfunclet$?asxTR800_Create@@YAXPAVasxSubSystem@@PAVCobraNetNode@@PAVasxMixer@@@Z$1 10066f6b f   asxtr800.obj
 0001:00065f76       __unwindfunclet$?asxTR800_Create@@YAXPAVasxSubSystem@@PAVCobraNetNode@@PAVasxMixer@@@Z$2 10066f76 f   asxtr800.obj
 0001:00065f81       __unwindfunclet$?asxTR800_Create@@YAXPAVasxSubSystem@@PAVCobraNetNode@@PAVasxMixer@@@Z$3 10066f81 f   asxtr800.obj
 0001:00065f8c       __unwindfunclet$?asxTR800_Create@@YAXPAVasxSubSystem@@PAVCobraNetNode@@PAVasxMixer@@@Z$4 10066f8c f   asxtr800.obj
 0001:00065f97       __unwindfunclet$?asxTR800_Create@@YAXPAVasxSubSystem@@PAVCobraNetNode@@PAVasxMixer@@@Z$5 10066f97 f   asxtr800.obj
 0001:00065fa2       __unwindfunclet$?asxTR800_Create@@YAXPAVasxSubSystem@@PAVCobraNetNode@@PAVasxMixer@@@Z$6 10066fa2 f   asxtr800.obj
 0001:00065fad       __unwindfunclet$?asxTR800_Create@@YAXPAVasxSubSystem@@PAVCobraNetNode@@PAVasxMixer@@@Z$7 10066fad f   asxtr800.obj
 0001:00065fb8       __unwindfunclet$?asxTR800_Create@@YAXPAVasxSubSystem@@PAVCobraNetNode@@PAVasxMixer@@@Z$8 10066fb8 f   asxtr800.obj
 0001:00065fc3       __unwindfunclet$?asxTR800_Create@@YAXPAVasxSubSystem@@PAVCobraNetNode@@PAVasxMixer@@@Z$9 10066fc3 f   asxtr800.obj
 0001:00065fce       __unwindfunclet$?asxTR800_Create@@YAXPAVasxSubSystem@@PAVCobraNetNode@@PAVasxMixer@@@Z$10 10066fce f   asxtr800.obj
 0001:00065fd9       __ehhandler$?asxTR800_Create@@YAXPAVasxSubSystem@@PAVCobraNetNode@@PAVasxMixer@@@Z 10066fd9 f   asxtr800.obj
 0001:00066000       __unwindfunclet$??0asxCobranetWAVE@@QAE@PAVasxSubSystem@@PAUHMIXEROBJ__@@PAVasxNode@@2HPAUtagMIXERCONTROLA@@3@Z$0 10067000 f   asxwave.obj
 0001:00066008       __ehhandler$??0asxCobranetWAVE@@QAE@PAVasxSubSystem@@PAUHMIXEROBJ__@@PAVasxNode@@2HPAUtagMIXERCONTROLA@@3@Z 10067008 f   asxwave.obj
 0001:00066030       __unwindfunclet$??0asxLevelWAVE@@QAE@PAVasxSubSystem@@PAUHMIXEROBJ__@@PAVasxNode@@2PAUtagMIXERCONTROLA@@H@Z$0 10067030 f   asxwave.obj
 0001:00066038       __ehhandler$??0asxLevelWAVE@@QAE@PAVasxSubSystem@@PAUHMIXEROBJ__@@PAVasxNode@@2PAUtagMIXERCONTROLA@@H@Z 10067038 f   asxwave.obj
 0001:00066060       __unwindfunclet$??0asxMeterWAVE@@QAE@PAVasxSubSystem@@PAUHMIXEROBJ__@@PAVasxNode@@2PAUtagMIXERCONTROLA@@H@Z$0 10067060 f   asxwave.obj
 0001:00066068       __ehhandler$??0asxMeterWAVE@@QAE@PAVasxSubSystem@@PAUHMIXEROBJ__@@PAVasxNode@@2PAUtagMIXERCONTROLA@@H@Z 10067068 f   asxwave.obj
 0001:00066090       __unwindfunclet$??0asxModeWAVE@@QAE@PAVasxSubSystem@@PAUHMIXEROBJ__@@PAVasxNode@@2PAUtagMIXERCONTROLA@@H@Z$0 10067090 f   asxwave.obj
 0001:00066098       __ehhandler$??0asxModeWAVE@@QAE@PAVasxSubSystem@@PAUHMIXEROBJ__@@PAVasxNode@@2PAUtagMIXERCONTROLA@@H@Z 10067098 f   asxwave.obj
 0001:000660c0       __unwindfunclet$??0asxMuxWAVE@@QAE@PAVasxSubSystem@@PAUHMIXEROBJ__@@PAVasxNode@@2PAUtagMIXERCONTROLA@@H@Z$0 100670c0 f   asxwave.obj
 0001:000660c8       __ehhandler$??0asxMuxWAVE@@QAE@PAVasxSubSystem@@PAUHMIXEROBJ__@@PAVasxNode@@2PAUtagMIXERCONTROLA@@H@Z 100670c8 f   asxwave.obj
 0001:000660f0       __unwindfunclet$??0asxSilenceDetectorWAVE@@QAE@PAVasxSubSystem@@PAUHMIXEROBJ__@@PAVasxNode@@2PAUtagMIXERCONTROLA@@H@Z$0 100670f0 f   asxwave.obj
 0001:000660f8       __ehhandler$??0asxSilenceDetectorWAVE@@QAE@PAVasxSubSystem@@PAUHMIXEROBJ__@@PAVasxNode@@2PAUtagMIXERCONTROLA@@H@Z 100670f8 f   asxwave.obj
 0001:00066120       __unwindfunclet$??0asxToneDetectorWAVE@@QAE@PAVasxSubSystem@@PAUHMIXEROBJ__@@PAVasxNode@@2PAUtagMIXERCONTROLA@@H@Z$0 10067120 f   asxwave.obj
 0001:00066128       __ehhandler$??0asxToneDetectorWAVE@@QAE@PAVasxSubSystem@@PAUHMIXEROBJ__@@PAVasxNode@@2PAUtagMIXERCONTROLA@@H@Z 10067128 f   asxwave.obj
 0001:00066150       __unwindfunclet$??0asxTunerWAVE@@QAE@PAVasxSubSystem@@PAUHMIXEROBJ__@@PAVasxNode@@2HPAUtagMIXERCONTROLA@@3333@Z$0 10067150 f   asxwave.obj
 0001:00066158       __unwindfunclet$??0asxTunerWAVE@@QAE@PAVasxSubSystem@@PAUHMIXEROBJ__@@PAVasxNode@@2HPAUtagMIXERCONTROLA@@3333@Z$1 10067158 f   asxwave.obj
 0001:00066163       __ehhandler$??0asxTunerWAVE@@QAE@PAVasxSubSystem@@PAUHMIXEROBJ__@@PAVasxNode@@2HPAUtagMIXERCONTROLA@@3333@Z 10067163 f   asxwave.obj
 0001:00066180       __unwindfunclet$??0asxVolumeWAVE@@QAE@PAVasxSubSystem@@PAUHMIXEROBJ__@@PAVasxNode@@2PAUtagMIXERCONTROLA@@H3@Z$0 10067180 f   asxwave.obj
 0001:00066188       __ehhandler$??0asxVolumeWAVE@@QAE@PAVasxSubSystem@@PAUHMIXEROBJ__@@PAVasxNode@@2PAUtagMIXERCONTROLA@@H3@Z 10067188 f   asxwave.obj
 0001:000661b0       __unwindfunclet$??0waveControlMuxHelper@@QAE@PAUHMIXEROBJ__@@PAVwaveControlInfo@@PAV?$TASIArray@VTASICString@@@@@Z$0 100671b0 f   asxwave.obj
 0001:000661bb       __ehhandler$??0waveControlMuxHelper@@QAE@PAUHMIXEROBJ__@@PAVwaveControlInfo@@PAV?$TASIArray@VTASICString@@@@@Z 100671bb f   asxwave.obj
 0001:000661e0       __unwindfunclet$??1asxAdapterWAVE@@UAE@XZ$0 100671e0 f   asxwave.obj
 0001:000661e8       __ehhandler$??1asxAdapterWAVE@@UAE@XZ 100671e8 f   asxwave.obj
 0001:00066210       __unwindfunclet$??1asxMixerScannerWAVE@@UAE@XZ$0 10067210 f   asxwave.obj
 0001:00066218       __unwindfunclet$??1asxMixerScannerWAVE@@UAE@XZ$1 10067218 f   asxwave.obj
 0001:00066223       __ehhandler$??1asxMixerScannerWAVE@@UAE@XZ 10067223 f   asxwave.obj
 0001:00066240       __unwindfunclet$??1asxModeWAVE@@UAE@XZ$1 10067240 f   asxwave.obj
 0001:00066248       __ehhandler$??1asxModeWAVE@@UAE@XZ 10067248 f   asxwave.obj
 0001:00066270       __unwindfunclet$??1asxMuxWAVE@@UAE@XZ$1 10067270 f   asxwave.obj
 0001:00066278       __unwindfunclet$??1asxMuxWAVE@@UAE@XZ$2 10067278 f   asxwave.obj
 0001:00066283       __ehhandler$??1asxMuxWAVE@@UAE@XZ 10067283 f   asxwave.obj
 0001:000662a0       __unwindfunclet$??1asxTunerWAVE@@UAE@XZ$0 100672a0 f   asxwave.obj
 0001:000662a8       __unwindfunclet$??1asxTunerWAVE@@UAE@XZ$2 100672a8 f   asxwave.obj
 0001:000662b0       __unwindfunclet$??1asxTunerWAVE@@UAE@XZ$3 100672b0 f   asxwave.obj
 0001:000662bb       __ehhandler$??1asxTunerWAVE@@UAE@XZ 100672bb f   asxwave.obj
 0001:000662e0       __unwindfunclet$?AddCobranet@@YAXPAVasxMixer@@PAVasxSubSystem@@PAVControlTracker@@PAUHMIXEROBJ__@@PAVasxNode@@4PAUtagMIXERCONTROLA@@H@Z$0 100672e0 f   asxwave.obj
 0001:000662ee       __unwindfunclet$?AddCobranet@@YAXPAVasxMixer@@PAVasxSubSystem@@PAVControlTracker@@PAUHMIXEROBJ__@@PAVasxNode@@4PAUtagMIXERCONTROLA@@H@Z$1 100672ee f   asxwave.obj
 0001:000662fc       __ehhandler$?AddCobranet@@YAXPAVasxMixer@@PAVasxSubSystem@@PAVControlTracker@@PAUHMIXEROBJ__@@PAVasxNode@@4PAUtagMIXERCONTROLA@@H@Z 100672fc f   asxwave.obj
 0001:00066330       __unwindfunclet$?AddControl@asxMixerScannerWAVE@@AAEXPAVasxMixer@@PAVControlTracker@@PAUHMIXEROBJ__@@PAVasxNode@@3PAUtagMIXERCONTROLA@@H@Z$2 10067330 f   asxwave.obj
 0001:0006633b       __unwindfunclet$?AddControl@asxMixerScannerWAVE@@AAEXPAVasxMixer@@PAVControlTracker@@PAUHMIXEROBJ__@@PAVasxNode@@3PAUtagMIXERCONTROLA@@H@Z$5 1006733b f   asxwave.obj
 0001:00066346       __unwindfunclet$?AddControl@asxMixerScannerWAVE@@AAEXPAVasxMixer@@PAVControlTracker@@PAUHMIXEROBJ__@@PAVasxNode@@3PAUtagMIXERCONTROLA@@H@Z$6 10067346 f   asxwave.obj
 0001:00066351       __unwindfunclet$?AddControl@asxMixerScannerWAVE@@AAEXPAVasxMixer@@PAVControlTracker@@PAUHMIXEROBJ__@@PAVasxNode@@3PAUtagMIXERCONTROLA@@H@Z$19 10067351 f   asxwave.obj
 0001:0006635c       __unwindfunclet$?AddControl@asxMixerScannerWAVE@@AAEXPAVasxMixer@@PAVControlTracker@@PAUHMIXEROBJ__@@PAVasxNode@@3PAUtagMIXERCONTROLA@@H@Z$20 1006735c f   asxwave.obj
 0001:00066367       __unwindfunclet$?AddControl@asxMixerScannerWAVE@@AAEXPAVasxMixer@@PAVControlTracker@@PAUHMIXEROBJ__@@PAVasxNode@@3PAUtagMIXERCONTROLA@@H@Z$21 10067367 f   asxwave.obj
 0001:00066372       __unwindfunclet$?AddControl@asxMixerScannerWAVE@@AAEXPAVasxMixer@@PAVControlTracker@@PAUHMIXEROBJ__@@PAVasxNode@@3PAUtagMIXERCONTROLA@@H@Z$22 10067372 f   asxwave.obj
 0001:0006637d       __unwindfunclet$?AddControl@asxMixerScannerWAVE@@AAEXPAVasxMixer@@PAVControlTracker@@PAUHMIXEROBJ__@@PAVasxNode@@3PAUtagMIXERCONTROLA@@H@Z$23 1006737d f   asxwave.obj
 0001:00066388       __unwindfunclet$?AddControl@asxMixerScannerWAVE@@AAEXPAVasxMixer@@PAVControlTracker@@PAUHMIXEROBJ__@@PAVasxNode@@3PAUtagMIXERCONTROLA@@H@Z$24 10067388 f   asxwave.obj
 0001:00066393       __unwindfunclet$?AddControl@asxMixerScannerWAVE@@AAEXPAVasxMixer@@PAVControlTracker@@PAUHMIXEROBJ__@@PAVasxNode@@3PAUtagMIXERCONTROLA@@H@Z$25 10067393 f   asxwave.obj
 0001:0006639e       __unwindfunclet$?AddControl@asxMixerScannerWAVE@@AAEXPAVasxMixer@@PAVControlTracker@@PAUHMIXEROBJ__@@PAVasxNode@@3PAUtagMIXERCONTROLA@@H@Z$26 1006739e f   asxwave.obj
 0001:000663a9       __unwindfunclet$?AddControl@asxMixerScannerWAVE@@AAEXPAVasxMixer@@PAVControlTracker@@PAUHMIXEROBJ__@@PAVasxNode@@3PAUtagMIXERCONTROLA@@H@Z$27 100673a9 f   asxwave.obj
 0001:000663b4       __unwindfunclet$?AddControl@asxMixerScannerWAVE@@AAEXPAVasxMixer@@PAVControlTracker@@PAUHMIXEROBJ__@@PAVasxNode@@3PAUtagMIXERCONTROLA@@H@Z$28 100673b4 f   asxwave.obj
 0001:000663bf       __unwindfunclet$?AddControl@asxMixerScannerWAVE@@AAEXPAVasxMixer@@PAVControlTracker@@PAUHMIXEROBJ__@@PAVasxNode@@3PAUtagMIXERCONTROLA@@H@Z$3 100673bf f   asxwave.obj
 0001:000663ca       __unwindfunclet$?AddControl@asxMixerScannerWAVE@@AAEXPAVasxMixer@@PAVControlTracker@@PAUHMIXEROBJ__@@PAVasxNode@@3PAUtagMIXERCONTROLA@@H@Z$16 100673ca f   asxwave.obj
 0001:000663d5       __unwindfunclet$?AddControl@asxMixerScannerWAVE@@AAEXPAVasxMixer@@PAVControlTracker@@PAUHMIXEROBJ__@@PAVasxNode@@3PAUtagMIXERCONTROLA@@H@Z$9 100673d5 f   asxwave.obj
 0001:000663e0       __unwindfunclet$?AddControl@asxMixerScannerWAVE@@AAEXPAVasxMixer@@PAVControlTracker@@PAUHMIXEROBJ__@@PAVasxNode@@3PAUtagMIXERCONTROLA@@H@Z$11 100673e0 f   asxwave.obj
 0001:000663eb       __unwindfunclet$?AddControl@asxMixerScannerWAVE@@AAEXPAVasxMixer@@PAVControlTracker@@PAUHMIXEROBJ__@@PAVasxNode@@3PAUtagMIXERCONTROLA@@H@Z$17 100673eb f   asxwave.obj
 0001:000663f6       __unwindfunclet$?AddControl@asxMixerScannerWAVE@@AAEXPAVasxMixer@@PAVControlTracker@@PAUHMIXEROBJ__@@PAVasxNode@@3PAUtagMIXERCONTROLA@@H@Z$15 100673f6 f   asxwave.obj
 0001:00066401       __unwindfunclet$?AddControl@asxMixerScannerWAVE@@AAEXPAVasxMixer@@PAVControlTracker@@PAUHMIXEROBJ__@@PAVasxNode@@3PAUtagMIXERCONTROLA@@H@Z$10 10067401 f   asxwave.obj
 0001:0006640c       __unwindfunclet$?AddControl@asxMixerScannerWAVE@@AAEXPAVasxMixer@@PAVControlTracker@@PAUHMIXEROBJ__@@PAVasxNode@@3PAUtagMIXERCONTROLA@@H@Z$4 1006740c f   asxwave.obj
 0001:00066417       __unwindfunclet$?AddControl@asxMixerScannerWAVE@@AAEXPAVasxMixer@@PAVControlTracker@@PAUHMIXEROBJ__@@PAVasxNode@@3PAUtagMIXERCONTROLA@@H@Z$0 10067417 f   asxwave.obj
 0001:00066422       __unwindfunclet$?AddControl@asxMixerScannerWAVE@@AAEXPAVasxMixer@@PAVControlTracker@@PAUHMIXEROBJ__@@PAVasxNode@@3PAUtagMIXERCONTROLA@@H@Z$1 10067422 f   asxwave.obj
 0001:0006642d       __unwindfunclet$?AddControl@asxMixerScannerWAVE@@AAEXPAVasxMixer@@PAVControlTracker@@PAUHMIXEROBJ__@@PAVasxNode@@3PAUtagMIXERCONTROLA@@H@Z$8 1006742d f   asxwave.obj
 0001:00066438       __unwindfunclet$?AddControl@asxMixerScannerWAVE@@AAEXPAVasxMixer@@PAVControlTracker@@PAUHMIXEROBJ__@@PAVasxNode@@3PAUtagMIXERCONTROLA@@H@Z$12 10067438 f   asxwave.obj
 0001:00066443       __unwindfunclet$?AddControl@asxMixerScannerWAVE@@AAEXPAVasxMixer@@PAVControlTracker@@PAUHMIXEROBJ__@@PAVasxNode@@3PAUtagMIXERCONTROLA@@H@Z$13 10067443 f   asxwave.obj
 0001:0006644e       __unwindfunclet$?AddControl@asxMixerScannerWAVE@@AAEXPAVasxMixer@@PAVControlTracker@@PAUHMIXEROBJ__@@PAVasxNode@@3PAUtagMIXERCONTROLA@@H@Z$14 1006744e f   asxwave.obj
 0001:00066459       __unwindfunclet$?AddControl@asxMixerScannerWAVE@@AAEXPAVasxMixer@@PAVControlTracker@@PAUHMIXEROBJ__@@PAVasxNode@@3PAUtagMIXERCONTROLA@@H@Z$18 10067459 f   asxwave.obj
 0001:00066464       __unwindfunclet$?AddControl@asxMixerScannerWAVE@@AAEXPAVasxMixer@@PAVControlTracker@@PAUHMIXEROBJ__@@PAVasxNode@@3PAUtagMIXERCONTROLA@@H@Z$7 10067464 f   asxwave.obj
 0001:0006646f       __ehhandler$?AddControl@asxMixerScannerWAVE@@AAEXPAVasxMixer@@PAVControlTracker@@PAUHMIXEROBJ__@@PAVasxNode@@3PAUtagMIXERCONTROLA@@H@Z 1006746f f   asxwave.obj
 0001:00066490       __unwindfunclet$?AddTuner@@YAXPAVasxMixer@@PAVasxSubSystem@@PAVControlTracker@@PAUHMIXEROBJ__@@PAVasxNode@@4PAUtagMIXERCONTROLA@@H@Z$0 10067490 f   asxwave.obj
 0001:0006649e       __ehhandler$?AddTuner@@YAXPAVasxMixer@@PAVasxSubSystem@@PAVControlTracker@@PAUHMIXEROBJ__@@PAVasxNode@@4PAUtagMIXERCONTROLA@@H@Z 1006749e f   asxwave.obj
 0001:000664d0       __unwindfunclet$?Scan@asxMixerScannerWAVE@@UAEXPAVasxMixer@@@Z$0 100674d0 f   asxwave.obj
 0001:000664db       __unwindfunclet$?Scan@asxMixerScannerWAVE@@UAEXPAVasxMixer@@@Z$1 100674db f   asxwave.obj
 0001:000664e9       __unwindfunclet$?Scan@asxMixerScannerWAVE@@UAEXPAVasxMixer@@@Z$2 100674e9 f   asxwave.obj
 0001:000664f7       __unwindfunclet$?Scan@asxMixerScannerWAVE@@UAEXPAVasxMixer@@@Z$3 100674f7 f   asxwave.obj
 0001:00066505       __unwindfunclet$?Scan@asxMixerScannerWAVE@@UAEXPAVasxMixer@@@Z$4 10067505 f   asxwave.obj
 0001:00066513       __unwindfunclet$?Scan@asxMixerScannerWAVE@@UAEXPAVasxMixer@@@Z$5 10067513 f   asxwave.obj
 0001:0006651e       __unwindfunclet$?Scan@asxMixerScannerWAVE@@UAEXPAVasxMixer@@@Z$6 1006751e f   asxwave.obj
 0001:00066529       __unwindfunclet$?Scan@asxMixerScannerWAVE@@UAEXPAVasxMixer@@@Z$7 10067529 f   asxwave.obj
 0001:00066537       __unwindfunclet$?Scan@asxMixerScannerWAVE@@UAEXPAVasxMixer@@@Z$8 10067537 f   asxwave.obj
 0001:00066545       __ehhandler$?Scan@asxMixerScannerWAVE@@UAEXPAVasxMixer@@@Z 10067545 f   asxwave.obj
 0001:00066570       __unwindfunclet$?Scan@asxSubSystemWAVE@@UAEXXZ$0 10067570 f   asxwave.obj
 0001:0006657b       __ehhandler$?Scan@asxSubSystemWAVE@@UAEXXZ 1006757b f   asxwave.obj
 0001:000665a0       __unwindfunclet$??1asxPlayerWAVE@@UAE@XZ$0 100675a0 f   asxwaveplay.obj
 0001:000665a8       __ehhandler$??1asxPlayerWAVE@@UAE@XZ 100675a8 f   asxwaveplay.obj
 0001:000665d0       __unwindfunclet$??1asxRecorderWAVE@@UAE@XZ$0 100675d0 f   asxwaverec.obj
 0001:000665d8       __ehhandler$??1asxRecorderWAVE@@UAE@XZ 100675d8 f   asxwaverec.obj
 0001:00066600       __unwindfunclet$??0TWavFileTypeGenerator@@QAE@PBD0PAJ@Z$0 10067600 f   twavfile.obj
 0001:00066608       __ehhandler$??0TWavFileTypeGenerator@@QAE@PBD0PAJ@Z 10067608 f   twavfile.obj
 0001:00066630       __unwindfunclet$??1TWavFileTypeWav@@UAE@XZ$0 10067630 f   twavfile.obj
 0001:00066638       __ehhandler$??1TWavFileTypeWav@@UAE@XZ 10067638 f   twavfile.obj
 0001:00066660       __unwindfunclet$??_GTWavFileTypeWav@@UAEPAXI@Z$0 10067660 f   twavfile.obj
 0001:00066668       __ehhandler$??_GTWavFileTypeWav@@UAEPAXI@Z 10067668 f   twavfile.obj
 0001:00066690       __unwindfunclet$?OpenWavFile@@YAPAVTWavFileBase@@PBD0PAJ@Z$0 10067690 f   twavfile.obj
 0001:0006669b       __unwindfunclet$?OpenWavFile@@YAPAVTWavFileBase@@PBD0PAJ@Z$1 1006769b f   twavfile.obj
 0001:000666a6       __unwindfunclet$?OpenWavFile@@YAPAVTWavFileBase@@PBD0PAJ@Z$2 100676a6 f   twavfile.obj
 0001:000666b1       __unwindfunclet$?OpenWavFile@@YAPAVTWavFileBase@@PBD0PAJ@Z$3 100676b1 f   twavfile.obj
 0001:000666bc       __unwindfunclet$?OpenWavFile@@YAPAVTWavFileBase@@PBD0PAJ@Z$4 100676bc f   twavfile.obj
 0001:000666c7       __ehhandler$?OpenWavFile@@YAPAVTWavFileBase@@PBD0PAJ@Z 100676c7 f   twavfile.obj
 0001:000666f0       __unwindfunclet$??0TWavFileWithFifo@@QAE@PAVTWavFileBase@@JW4FifoDirection@0@@Z$0 100676f0 f   twavfilefifo.obj
 0001:000666f8       __unwindfunclet$??0TWavFileWithFifo@@QAE@PAVTWavFileBase@@JW4FifoDirection@0@@Z$1 100676f8 f   twavfilefifo.obj
 0001:00066706       __ehhandler$??0TWavFileWithFifo@@QAE@PAVTWavFileBase@@JW4FifoDirection@0@@Z 10067706 f   twavfilefifo.obj
 0001:00066730       __unwindfunclet$??1TWavFileWithFifo@@UAE@XZ$0 10067730 f   twavfilefifo.obj
 0001:00066738       __unwindfunclet$??1TWavFileWithFifo@@UAE@XZ$1 10067738 f   twavfilefifo.obj
 0001:00066746       __ehhandler$??1TWavFileWithFifo@@UAE@XZ 10067746 f   twavfilefifo.obj
 0001:00066761       __ehhandler$?CallUnexpected@@YAXPBU_s_ESTypeList@@@Z 10067761 f   LIBCMT:frame.obj
 0001:00066780       ??__F?_Generic_object@?$_Error_objects@H@std@@2V_Generic_error_category@2@A@@YAXXZ 10067780 f   asxavdecc.obj
 0001:00066790       ??__F?_Iostream_object@?$_Error_objects@H@std@@2V_Iostream_error_category@2@A@@YAXXZ 10067790 f   asxavdecc.obj
 0001:000667a0       ??__F?_System_object@?$_Error_objects@H@std@@2V_System_error_category@2@A@@YAXXZ 100677a0 f   asxavdecc.obj
 0001:000667b0       ??__F?audioMetersOid@CobraNetNode@@0VasiOID@@A@@YAXXZ 100677b0 f   cobranet.obj
 0001:000667d0       ??__F?conductorPriorityOID@CobraNetNode@@0VasiOID@@A@@YAXXZ 100677d0 f   cobranet.obj
 0001:000667f0       ??__F?conductorStatusOID@CobraNetNode@@0VasiOID@@A@@YAXXZ 100677f0 f   cobranet.obj
 0001:00066810       ??__F?errorCountOID@CobraNetNode@@0VasiOID@@A@@YAXXZ 10067810 f   cobranet.obj
 0001:00066830       ??__F?errorDisplayOID@CobraNetNode@@0VasiOID@@A@@YAXXZ 10067830 f   cobranet.obj
 0001:00066850       ??__F?errorLastOID@CobraNetNode@@0VasiOID@@A@@YAXXZ 10067850 f   cobranet.obj
 0001:00066870       ??__F?firmwareMajorVersionOID@CobraNetNode@@0VasiOID@@A@@YAXXZ 10067870 f   cobranet.obj
 0001:00066890       ??__F?firmwareMinorVersionOID@CobraNetNode@@0VasiOID@@A@@YAXXZ 10067890 f   cobranet.obj
 0001:000668b0       ??__F?flashPersistEnableOID@CobraNetNode@@0VasiOID@@A@@YAXXZ 100678b0 f   cobranet.obj
 0001:000668d0       ??__F?ipmonCurrentIpOID@CobraNetNode@@0VasiOID@@A@@YAXXZ 100678d0 f   cobranet.obj
 0001:000668f0       ??__F?ipmonStaticIpOID@CobraNetNode@@0VasiOID@@A@@YAXXZ 100678f0 f   cobranet.obj
 0001:00066910       ??__F?modeRateControlOID@CobraNetNode@@0VasiOID@@A@@YAXXZ 10067910 f   cobranet.obj
 0001:00066930       ??__F?modeRateStatusOID@CobraNetNode@@0VasiOID@@A@@YAXXZ 10067930 f   cobranet.obj
 0001:00066950       ??__F?rxBundleOid@CobraNetNode@@0VasiOID@@A@@YAXXZ 10067950 f   cobranet.obj
 0001:00066970       ??__F?rxDelayOid@CobraNetNode@@0VasiOID@@A@@YAXXZ 10067970 f   cobranet.obj
 0001:00066990       ??__F?rxDropoutsOid@CobraNetNode@@0VasiOID@@A@@YAXXZ 10067990 f   cobranet.obj
 0001:000669b0       ??__F?rxMinDelayOid@CobraNetNode@@0VasiOID@@A@@YAXXZ 100679b0 f   cobranet.obj
 0001:000669d0       ??__F?rxPriorityOid@CobraNetNode@@0VasiOID@@A@@YAXXZ 100679d0 f   cobranet.obj
 0001:000669f0       ??__F?rxSourceMACOid@CobraNetNode@@0VasiOID@@A@@YAXXZ 100679f0 f   cobranet.obj
 0001:00066a10       ??__F?rxStatusOid@CobraNetNode@@0VasiOID@@A@@YAXXZ 10067a10 f   cobranet.obj
 0001:00066a30       ??__F?rxSubFormatOid@CobraNetNode@@0VasiOID@@A@@YAXXZ 10067a30 f   cobranet.obj
 0001:00066a50       ??__F?rxSubMapOid@CobraNetNode@@0VasiOID@@A@@YAXXZ 10067a50 f   cobranet.obj
 0001:00066a70       ??__F?serialBaudOID@CobraNetNode@@0VasiOID@@A@@YAXXZ 10067a70 f   cobranet.obj
 0001:00066a90       ??__F?serialFormatOID@CobraNetNode@@0VasiOID@@A@@YAXXZ 10067a90 f   cobranet.obj
 0001:00066ab0       ??__F?serialPPeriodOID@CobraNetNode@@0VasiOID@@A@@YAXXZ 10067ab0 f   cobranet.obj
 0001:00066ad0       ??__F?serialRxMacOID@CobraNetNode@@0VasiOID@@A@@YAXXZ 10067ad0 f   cobranet.obj
 0001:00066af0       ??__F?serialTxMacOID@CobraNetNode@@0VasiOID@@A@@YAXXZ 10067af0 f   cobranet.obj
 0001:00066b10       ??__F?serialTxPriorityOID@CobraNetNode@@0VasiOID@@A@@YAXXZ 10067b10 f   cobranet.obj
 0001:00066b30       ??__F?stdUserIntegerOid@CobraNetNode@@0VasiOID@@A@@YAXXZ 10067b30 f   cobranet.obj
 0001:00066b50       ??__F?sysContactOID@CobraNetNode@@0VasiOID@@A@@YAXXZ 10067b50 f   cobranet.obj
 0001:00066b70       ??__F?sysDescriptionOID@CobraNetNode@@0VasiOID@@A@@YAXXZ 10067b70 f   cobranet.obj
 0001:00066b90       ??__F?sysLocationOID@CobraNetNode@@0VasiOID@@A@@YAXXZ 10067b90 f   cobranet.obj
 0001:00066bb0       ??__F?sysNameOID@CobraNetNode@@0VasiOID@@A@@YAXXZ 10067bb0 f   cobranet.obj
 0001:00066bd0       ??__F?txBundleOid@CobraNetNode@@0VasiOID@@A@@YAXXZ 10067bd0 f   cobranet.obj
 0001:00066bf0       ??__F?txDropoutsOid@CobraNetNode@@0VasiOID@@A@@YAXXZ 10067bf0 f   cobranet.obj
 0001:00066c10       ??__F?txMaxUnicastOid@CobraNetNode@@0VasiOID@@A@@YAXXZ 10067c10 f   cobranet.obj
 0001:00066c30       ??__F?txPositionOid@CobraNetNode@@0VasiOID@@A@@YAXXZ 10067c30 f   cobranet.obj
 0001:00066c50       ??__F?txPriorityOid@CobraNetNode@@0VasiOID@@A@@YAXXZ 10067c50 f   cobranet.obj
 0001:00066c70       ??__F?txReceiversOid@CobraNetNode@@0VasiOID@@A@@YAXXZ 10067c70 f   cobranet.obj
 0001:00066c90       ??__F?txSubCountOid@CobraNetNode@@0VasiOID@@A@@YAXXZ 10067c90 f   cobranet.obj
 0001:00066cb0       ??__F?txSubFormatOid@CobraNetNode@@0VasiOID@@A@@YAXXZ 10067cb0 f   cobranet.obj
 0001:00066cd0       ??__F?txSubMapOid@CobraNetNode@@0VasiOID@@A@@YAXXZ 10067cd0 f   cobranet.obj
 0001:00066cf0       ??__F?txUnicastModeOid@CobraNetNode@@0VasiOID@@A@@YAXXZ 10067cf0 f   cobranet.obj
 0001:00066d0e       ??__F?_Generic_object@?$_Error_objects@H@std@@2V_Generic_error_category@2@A@@YAXXZ 10067d0e f   libcpmt:xthrow.obj
 0001:00066d19       ??__F?_Iostream_object@?$_Error_objects@H@std@@2V_Iostream_error_category@2@A@@YAXXZ 10067d19 f   libcpmt:xthrow.obj
 0001:00066d24       ??__F?_System_object@?$_Error_objects@H@std@@2V_System_error_category@2@A@@YAXXZ 10067d24 f   libcpmt:xthrow.obj
 0001:00066d2f       ??__F?_Generic_object@?$_Error_objects@H@std@@2V_Generic_error_category@2@A@@YAXXZ 10067d2f f   libcpmt:syserror.obj
 0001:00066d3a       ??__F?_Iostream_object@?$_Error_objects@H@std@@2V_Iostream_error_category@2@A@@YAXXZ 10067d3a f   libcpmt:syserror.obj
 0001:00066d45       ??__F?_System_object@?$_Error_objects@H@std@@2V_System_error_category@2@A@@YAXXZ 10067d45 f   libcpmt:syserror.obj
 0002:00000610       ?_Generic_object$initializer$@?$_Error_objects@H@std@@2P6AXXZA 10068610     asxavdecc.obj
 0002:00000614       ?_Iostream_object$initializer$@?$_Error_objects@H@std@@2P6AXXZA 10068614     asxavdecc.obj
 0002:00000618       ?_System_object$initializer$@?$_Error_objects@H@std@@2P6AXXZA 10068618     asxavdecc.obj
 0002:0000061c       _asxDebug$initializer$     1006861c     asxdebug.obj
 0002:00000620       ?sysDescriptionOID$initializer$@CobraNetNode@@0P6AXXZA 10068620     cobranet.obj
 0002:00000624       ?sysNameOID$initializer$@CobraNetNode@@0P6AXXZA 10068624     cobranet.obj
 0002:00000628       ?sysLocationOID$initializer$@CobraNetNode@@0P6AXXZA 10068628     cobranet.obj
 0002:0000062c       ?sysContactOID$initializer$@CobraNetNode@@0P6AXXZA 1006862c     cobranet.obj
 0002:00000630       ?firmwareMajorVersionOID$initializer$@CobraNetNode@@0P6AXXZA 10068630     cobranet.obj
 0002:00000634       ?firmwareMinorVersionOID$initializer$@CobraNetNode@@0P6AXXZA 10068634     cobranet.obj
 0002:00000638       ?flashPersistEnableOID$initializer$@CobraNetNode@@0P6AXXZA 10068638     cobranet.obj
 0002:0000063c       ?modeRateControlOID$initializer$@CobraNetNode@@0P6AXXZA 1006863c     cobranet.obj
 0002:00000640       ?errorDisplayOID$initializer$@CobraNetNode@@0P6AXXZA 10068640     cobranet.obj
 0002:00000644       ?errorCountOID$initializer$@CobraNetNode@@0P6AXXZA 10068644     cobranet.obj
 0002:00000648       ?errorLastOID$initializer$@CobraNetNode@@0P6AXXZA 10068648     cobranet.obj
 0002:0000064c       ?modeRateStatusOID$initializer$@CobraNetNode@@0P6AXXZA 1006864c     cobranet.obj
 0002:00000650       ?conductorStatusOID$initializer$@CobraNetNode@@0P6AXXZA 10068650     cobranet.obj
 0002:00000654       ?conductorPriorityOID$initializer$@CobraNetNode@@0P6AXXZA 10068654     cobranet.obj
 0002:00000658       ?ipmonCurrentIpOID$initializer$@CobraNetNode@@0P6AXXZA 10068658     cobranet.obj
 0002:0000065c       ?ipmonStaticIpOID$initializer$@CobraNetNode@@0P6AXXZA 1006865c     cobranet.obj
 0002:00000660       ?serialFormatOID$initializer$@CobraNetNode@@0P6AXXZA 10068660     cobranet.obj
 0002:00000664       ?serialBaudOID$initializer$@CobraNetNode@@0P6AXXZA 10068664     cobranet.obj
 0002:00000668       ?serialPPeriodOID$initializer$@CobraNetNode@@0P6AXXZA 10068668     cobranet.obj
 0002:0000066c       ?serialRxMacOID$initializer$@CobraNetNode@@0P6AXXZA 1006866c     cobranet.obj
 0002:00000670       ?serialTxMacOID$initializer$@CobraNetNode@@0P6AXXZA 10068670     cobranet.obj
 0002:00000674       ?serialTxPriorityOID$initializer$@CobraNetNode@@0P6AXXZA 10068674     cobranet.obj
 0002:00000678       ?txBundleOid$initializer$@CobraNetNode@@0P6AXXZA 10068678     cobranet.obj
 0002:0000067c       ?txPriorityOid$initializer$@CobraNetNode@@0P6AXXZA 1006867c     cobranet.obj
 0002:00000680       ?txSubCountOid$initializer$@CobraNetNode@@0P6AXXZA 10068680     cobranet.obj
 0002:00000684       ?txMaxUnicastOid$initializer$@CobraNetNode@@0P6AXXZA 10068684     cobranet.obj
 0002:00000688       ?txUnicastModeOid$initializer$@CobraNetNode@@0P6AXXZA 10068688     cobranet.obj
 0002:0000068c       ?txSubMapOid$initializer$@CobraNetNode@@0P6AXXZA 1006868c     cobranet.obj
 0002:00000690       ?txSubFormatOid$initializer$@CobraNetNode@@0P6AXXZA 10068690     cobranet.obj
 0002:00000694       ?txPositionOid$initializer$@CobraNetNode@@0P6AXXZA 10068694     cobranet.obj
 0002:00000698       ?txDropoutsOid$initializer$@CobraNetNode@@0P6AXXZA 10068698     cobranet.obj
 0002:0000069c       ?txReceiversOid$initializer$@CobraNetNode@@0P6AXXZA 1006869c     cobranet.obj
 0002:000006a0       ?rxBundleOid$initializer$@CobraNetNode@@0P6AXXZA 100686a0     cobranet.obj
 0002:000006a4       ?rxSourceMACOid$initializer$@CobraNetNode@@0P6AXXZA 100686a4     cobranet.obj
 0002:000006a8       ?rxPriorityOid$initializer$@CobraNetNode@@0P6AXXZA 100686a8     cobranet.obj
 0002:000006ac       ?rxStatusOid$initializer$@CobraNetNode@@0P6AXXZA 100686ac     cobranet.obj
 0002:000006b0       ?rxDropoutsOid$initializer$@CobraNetNode@@0P6AXXZA 100686b0     cobranet.obj
 0002:000006b4       ?rxDelayOid$initializer$@CobraNetNode@@0P6AXXZA 100686b4     cobranet.obj
 0002:000006b8       ?rxMinDelayOid$initializer$@CobraNetNode@@0P6AXXZA 100686b8     cobranet.obj
 0002:000006bc       ?rxSubMapOid$initializer$@CobraNetNode@@0P6AXXZA 100686bc     cobranet.obj
 0002:000006c0       ?rxSubFormatOid$initializer$@CobraNetNode@@0P6AXXZA 100686c0     cobranet.obj
 0002:000006c4       ?audioMetersOid$initializer$@CobraNetNode@@0P6AXXZA 100686c4     cobranet.obj
 0002:000006c8       ?stdUserIntegerOid$initializer$@CobraNetNode@@0P6AXXZA 100686c8     cobranet.obj
 0002:000006cc       _sysEntryTable$initializer$ 100686cc     mibtbl.obj
 0002:000006d0       _sysGroup$initializer$     100686d0     mibtbl.obj
 0002:000006d4       _ifEntryTable$initializer$ 100686d4     mibtbl.obj
 0002:000006d8       _ifGroup$initializer$      100686d8     mibtbl.obj
 0002:000006dc       _ipEntryTable$initializer$ 100686dc     mibtbl.obj
 0002:000006e0       _ipGroup$initializer$      100686e0     mibtbl.obj
 0002:000006e4       _udpEntryTable$initializer$ 100686e4     mibtbl.obj
 0002:000006e8       _udpGroup$initializer$     100686e8     mibtbl.obj
 0002:000006ec       _snmpEntryTable$initializer$ 100686ec     mibtbl.obj
 0002:000006f0       _snmpGroup$initializer$    100686f0     mibtbl.obj
 0002:000006f4       _firmwareEntryTable$initializer$ 100686f4     mibtbl.obj
 0002:000006f8       _firmwareGroup$initializer$ 100686f8     mibtbl.obj
 0002:000006fc       _flashEntryTable$initializer$ 100686fc     mibtbl.obj
 0002:00000700       _flashGroup$initializer$   10068700     mibtbl.obj
 0002:00000704       _errorEntryTable$initializer$ 10068704     mibtbl.obj
 0002:00000708       _errorGroup$initializer$   10068708     mibtbl.obj
 0002:0000070c       _modeEntryTable$initializer$ 1006870c     mibtbl.obj
 0002:00000710       _modeGroup$initializer$    10068710     mibtbl.obj
 0002:00000714       _conductorEntryTable$initializer$ 10068714     mibtbl.obj
 0002:00000718       _conductorGroup$initializer$ 10068718     mibtbl.obj
 0002:0000071c       _audioEntryTable$initializer$ 1006871c     mibtbl.obj
 0002:00000720       _audioGroup$initializer$   10068720     mibtbl.obj
 0002:00000724       _rxEntryTable$initializer$ 10068724     mibtbl.obj
 0002:00000728       _rxGroup$initializer$      10068728     mibtbl.obj
 0002:0000072c       _txEntryTable$initializer$ 1006872c     mibtbl.obj
 0002:00000730       _txGroup$initializer$      10068730     mibtbl.obj
 0002:00000734       _syncEntryTable$initializer$ 10068734     mibtbl.obj
 0002:00000738       _syncGroup$initializer$    10068738     mibtbl.obj
 0002:0000073c       _mimonEntryTable$initializer$ 1006873c     mibtbl.obj
 0002:00000740       _mimonGroup$initializer$   10068740     mibtbl.obj
 0002:00000744       _ipmonEntryTable$initializer$ 10068744     mibtbl.obj
 0002:00000748       _ipmonGroup$initializer$   10068748     mibtbl.obj
 0002:0000074c       _ifmEntryTable$initializer$ 1006874c     mibtbl.obj
 0002:00000750       _ifmGroup$initializer$     10068750     mibtbl.obj
 0002:00000754       _serialEntryTable$initializer$ 10068754     mibtbl.obj
 0002:00000758       _serialGroup$initializer$  10068758     mibtbl.obj
 0002:0000075c       _stdEntryTable$initializer$ 1006875c     mibtbl.obj
 0002:00000760       _stdGroup$initializer$     10068760     mibtbl.obj
 0002:0000076c       _pinit                     1006876c     LIBCMT:onexit.obj
 0002:00000770       _pinit                     10068770     LIBCMT:mbctype.obj
 0002:00000774       _pinit                     10068774     LIBCMT:cpu_disp.obj
 0002:00000778       _pinit                     10068778     LIBCMT:_file.obj
 0002:0000077c       _pinit                     1006877c     LIBCMT:mathfcns.obj
 0002:00000788       _pterm                     10068788     LIBCMT:wsetloca.obj
 0002:0000078c       _pterm                     1006878c     LIBCMT:initcon.obj
 0002:00000790       _pterm                     10068790     LIBCMT:_file.obj
 0002:00009138       _aErrorList                10071138     asxclass.obj
 0002:0000af14       _aFormatTranslate          10072f14     asxhpi.obj
 0002:0000d2a8       _channelModeNameMapping    100752a8     asxwave.obj
 0002:0000d338       _tunerBandNameMapping      10075338     asxwave.obj
 0002:0000d3b0       _tunerStatusNameMapping    100753b0     asxwave.obj
 0002:0000d440       _waveLineNameMapping       10075440     asxwave.obj
 0002:0000ecbc       _GS_ExceptionPointers      10076cbc     LIBCMT:gs_report.obj
 0002:0000ed00       ?ExceptionTemplate@?1??_CxxThrowException@@9@8@4UEHExceptionRecord@@B 10076d00     LIBCMT:throw.obj
 0002:0000ed20       _Int32ToUInt32             10076d20     LIBCMT:ftol3.obj
 0002:0000ed30       _MantissaMask              10076d30     LIBCMT:ftol3.obj
 0002:0000ed38       _IntegerBit                10076d38     LIBCMT:ftol3.obj
 0002:0000ed40       _SignBit64                 10076d40     LIBCMT:ftol3.obj
 0002:0000ed48       _MinFP64                   10076d48     LIBCMT:ftol3.obj
 0002:0000ed50       _MinInt64                  10076d50     LIBCMT:ftol3.obj
 0002:0000ed58       _MaxInt64                  10076d58     LIBCMT:ftol3.obj
 0002:0000ed60       _MaxUInt64                 10076d60     LIBCMT:ftol3.obj
 0002:0000ed68       _MaxFP32                   10076d68     LIBCMT:ftol3.obj
 0002:0000ed70       _MinFP32                   10076d70     LIBCMT:ftol3.obj
 0002:0000ed78       _MinSubInexact             10076d78     LIBCMT:ftol3.obj
 0002:0000ed80       _FpExcptTable              10076d80     LIBCMT:ftol3.obj
 0002:0000ed90       _i1075                     10076d90     LIBCMT:ftol3.obj
 0002:0000ed94       _i1087                     10076d94     LIBCMT:ftol3.obj
 0002:0000ed98       _x0800                     10076d98     LIBCMT:ftol3.obj
 0002:0000ed9c       _x17FF                     10076d9c     LIBCMT:ftol3.obj
 0002:0000eda0       _CWMask                    10076da0     LIBCMT:ftol3.obj
 0002:0000ee30       emask                      10076e30     LIBCMT:log10_sse2_precise.obj
 0002:0000ee40       CC                         10076e40     LIBCMT:log10_sse2_precise.obj
 0002:0000ee50       Magic                      10076e50     LIBCMT:log10_sse2_precise.obj
 0002:0000ee60       hi_mask                    10076e60     LIBCMT:log10_sse2_precise.obj
 0002:0000ee70       LOG10_2                    10076e70     LIBCMT:log10_sse2_precise.obj
 0002:0000ee80       place_L                    10076e80     LIBCMT:log10_sse2_precise.obj
 0002:0000eea0       One                        10076ea0     LIBCMT:log10_sse2_precise.obj
 0002:0000eeb0       Zero                       10076eb0     LIBCMT:log10_sse2_precise.obj
 0002:0000eec0       Two52                      10076ec0     LIBCMT:log10_sse2_precise.obj
 0002:0000eed0       Infs                       10076ed0     LIBCMT:log10_sse2_precise.obj
 0002:0000eee0       NaN                        10076ee0     LIBCMT:log10_sse2_precise.obj
 0002:0000eef0       coeff                      10076ef0     LIBCMT:log10_sse2_precise.obj
 0002:0000ef30       T_Tbl                      10076f30     LIBCMT:log10_sse2_precise.obj
 0002:0000f340       CB_Tbl                     10077340     LIBCMT:log10_sse2_precise.obj
 0002:0000f750       rcp_t1                     10077750     LIBCMT:pow_sse2_precise.obj
 0002:0000fb60       log2_t1                    10077b60     LIBCMT:pow_sse2_precise.obj
 0002:00010370       rcp_t2                     10078370     LIBCMT:pow_sse2_precise.obj
 0002:00010780       log2_t2                    10078780     LIBCMT:pow_sse2_precise.obj
 0002:00010f90       rcp_t3                     10078f90     LIBCMT:pow_sse2_precise.obj
 0002:000117a0       log2_t3                    100797a0     LIBCMT:pow_sse2_precise.obj
 0002:000127b0       clv                        1007a7b0     LIBCMT:pow_sse2_precise.obj
 0002:000127d0       exp2_tbl                   1007a7d0     LIBCMT:pow_sse2_precise.obj
 0002:00012fd0       Shifter                    1007afd0     LIBCMT:pow_sse2_precise.obj
 0002:00012fe0       SIGMASK                    1007afe0     LIBCMT:pow_sse2_precise.obj
 0002:00012ff0       ONEMASK                    1007aff0     LIBCMT:pow_sse2_precise.obj
 0002:00013000       ABSVALMASK                 1007b000     LIBCMT:pow_sse2_precise.obj
 0002:00013010       cev                        1007b010     LIBCMT:pow_sse2_precise.obj
 0002:00013038       HALFSIG                    1007b038     LIBCMT:pow_sse2_precise.obj
 0002:00013040       LHN                        1007b040     LIBCMT:pow_sse2_precise.obj
 0002:00013048       sNaN                       1007b048     LIBCMT:pow_sse2_precise.obj
 0002:00013050       INF                        1007b050     LIBCMT:pow_sse2_precise.obj
 0002:00013058       NEG_INF                    1007b058     LIBCMT:pow_sse2_precise.obj
 0002:00013060       NEG_ZERO                   1007b060     LIBCMT:pow_sse2_precise.obj
 0002:00013068       NEG_BIG                    1007b068     LIBCMT:pow_sse2_precise.obj
 0002:00013070       POS_BIG                    1007b070     LIBCMT:pow_sse2_precise.obj
 0002:00013078       EMIN                       1007b078     LIBCMT:pow_sse2_precise.obj
 0002:00013080       QIND                       1007b080     LIBCMT:pow_sse2_precise.obj
 0002:00013090       Ctable                     1007b090     LIBCMT:sin_sse2_precise.obj
 0002:00013890       SC_1                       1007b890     LIBCMT:sin_sse2_precise.obj
 0002:000138a0       SC_2                       1007b8a0     LIBCMT:sin_sse2_precise.obj
 0002:000138b0       SC_3                       1007b8b0     LIBCMT:sin_sse2_precise.obj
 0002:000138c0       SC_4                       1007b8c0     LIBCMT:sin_sse2_precise.obj
 0002:000138d0       PI32INV                    1007b8d0     LIBCMT:sin_sse2_precise.obj
 0002:000138d8       SHIFTER                    1007b8d8     LIBCMT:sin_sse2_precise.obj
 0002:000138e0       P_2                        1007b8e0     LIBCMT:sin_sse2_precise.obj
 0002:000138f0       P_1                        1007b8f0     LIBCMT:sin_sse2_precise.obj
 0002:000138f8       P_3                        1007b8f8     LIBCMT:sin_sse2_precise.obj
 0002:00013900       TWO_POW_55                 1007b900     LIBCMT:sin_sse2_precise.obj
 0002:00013908       TWO_POW_M55                1007b908     LIBCMT:sin_sse2_precise.obj
 0002:00013910       ALL_ONES                   1007b910     LIBCMT:sin_sse2_precise.obj
 0002:00013918       NEG_ZERO                   1007b918     LIBCMT:sin_sse2_precise.obj
 0002:00013920       ONE                        1007b920     LIBCMT:sin_sse2_precise.obj
 0002:00013c14       __mb_locale_names          1007bc14     LIBCMT:mbctype.obj
 0002:00014078       __first_127char            1007c078     LIBCMT:wsetloca.obj
 0002:000141c0       _rterrs                    1007c1c0     LIBCMT:crt0msg.obj
 0002:00014db8       _INF                       1007cdb8     LIBCMT:libm_error.obj
 0002:00014dc8       _BIG                       1007cdc8     LIBCMT:libm_error.obj
 0002:00014dd8       _ZERO                      1007cdd8     LIBCMT:libm_error.obj
 0002:00014de8       _INF_32                    1007cde8     LIBCMT:libm_error.obj
 0002:00014df0       _NAN_32                    1007cdf0     LIBCMT:libm_error.obj
 0002:00014df8       _ZERO_32                   1007cdf8     LIBCMT:libm_error.obj
 0002:00014e00       _libm_largef               1007ce00     LIBCMT:libm_error.obj
 0002:00014e08       _libm_smallf               1007ce08     LIBCMT:libm_error.obj
 0002:00014e10       _libm_small                1007ce10     LIBCMT:libm_error.obj
 0002:00014e30       ?ccsField@?P@??_openfile@@9@9 1007ce30     LIBCMT:_open.obj
 0002:00014e34       ?utf8encoding@?P@??_openfile@@9@9 1007ce34     LIBCMT:_open.obj
 0002:00014e3c       ?utf16encoding@?P@??_openfile@@9@9 1007ce3c     LIBCMT:_open.obj
 0002:00014e48       ?unicodeencoding@?P@??_openfile@@9@9 1007ce48     LIBCMT:_open.obj
 0002:000185d0       _tokenTable                100805d0     LIBCMT:undname.obj
 0002:00018608       _nameTable                 10080608     LIBCMT:undname.obj
 0002:00018748       _rttiTable                 10080748     LIBCMT:undname.obj
 0002:000190f4       One                        100810f4     LIBCMT:87disp.obj
 0002:000190fc       XAMtoTagTab                100810fc     LIBCMT:87disp.obj
 0002:00019110       One                        10081110     LIBCMT:common.obj
 0002:00019124       DblMax                     10081124     LIBCMT:common.obj
 0002:0001912c       DblMin                     1008112c     LIBCMT:common.obj
 0002:00019134       IeeeAdjO                   10081134     LIBCMT:common.obj
 0002:0001913c       IeeeAdjU                   1008113c     LIBCMT:common.obj
 0002:00019144       _infinity                  10081144     LIBCMT:common.obj
 0002:0001914c       _zero                      1008114c     LIBCMT:common.obj
 0002:00019160       emask                      10081160     LIBCMT:log10_pentium4.obj
 0002:00019170       CC                         10081170     LIBCMT:log10_pentium4.obj
 0002:00019180       Magic                      10081180     LIBCMT:log10_pentium4.obj
 0002:00019190       hi_mask                    10081190     LIBCMT:log10_pentium4.obj
 0002:000191a0       LOG10_2                    100811a0     LIBCMT:log10_pentium4.obj
 0002:000191b0       place_L                    100811b0     LIBCMT:log10_pentium4.obj
 0002:000191d0       One                        100811d0     LIBCMT:log10_pentium4.obj
 0002:000191e0       Zero                       100811e0     LIBCMT:log10_pentium4.obj
 0002:000191f0       Two52                      100811f0     LIBCMT:log10_pentium4.obj
 0002:00019200       Infs                       10081200     LIBCMT:log10_pentium4.obj
 0002:00019210       NaN                        10081210     LIBCMT:log10_pentium4.obj
 0002:00019220       coeff                      10081220     LIBCMT:log10_pentium4.obj
 0002:00019260       T_Tbl                      10081260     LIBCMT:log10_pentium4.obj
 0002:00019670       CB_Tbl                     10081670     LIBCMT:log10_pentium4.obj
 0002:00019a9e       _log2max                   10081a9e     LIBCMT:87tran.obj
 0002:00019aa8       _smallarg                  10081aa8     LIBCMT:87tran.obj
 0002:00019ab2       _half                      10081ab2     LIBCMT:87tran.obj
 0002:00019ae0       rcp_t1                     10081ae0     LIBCMT:pow_pentium4.obj
 0002:00019ef0       log2_t1                    10081ef0     LIBCMT:pow_pentium4.obj
 0002:0001a700       rcp_t2                     10082700     LIBCMT:pow_pentium4.obj
 0002:0001ab10       log2_t2                    10082b10     LIBCMT:pow_pentium4.obj
 0002:0001b320       rcp_t3                     10083320     LIBCMT:pow_pentium4.obj
 0002:0001bb30       log2_t3                    10083b30     LIBCMT:pow_pentium4.obj
 0002:0001cb40       clv                        10084b40     LIBCMT:pow_pentium4.obj
 0002:0001cb60       exp2_tbl                   10084b60     LIBCMT:pow_pentium4.obj
 0002:0001d360       Shifter                    10085360     LIBCMT:pow_pentium4.obj
 0002:0001d370       SIGMASK                    10085370     LIBCMT:pow_pentium4.obj
 0002:0001d380       ONEMASK                    10085380     LIBCMT:pow_pentium4.obj
 0002:0001d390       ABSVALMASK                 10085390     LIBCMT:pow_pentium4.obj
 0002:0001d3a0       cev                        100853a0     LIBCMT:pow_pentium4.obj
 0002:0001d3c8       HALFSIG                    100853c8     LIBCMT:pow_pentium4.obj
 0002:0001d3d0       LHN                        100853d0     LIBCMT:pow_pentium4.obj
 0002:0001d3d8       sNaN                       100853d8     LIBCMT:pow_pentium4.obj
 0002:0001d3e0       INF                        100853e0     LIBCMT:pow_pentium4.obj
 0002:0001d3e8       NEG_INF                    100853e8     LIBCMT:pow_pentium4.obj
 0002:0001d3f0       NEG_ZERO                   100853f0     LIBCMT:pow_pentium4.obj
 0002:0001d3f8       NEG_BIG                    100853f8     LIBCMT:pow_pentium4.obj
 0002:0001d400       POS_BIG                    10085400     LIBCMT:pow_pentium4.obj
 0002:0001d408       EMIN                       10085408     LIBCMT:pow_pentium4.obj
 0002:0001d410       QIND                       10085410     LIBCMT:pow_pentium4.obj
 0002:0001d430       Ctable                     10085430     LIBCMT:sin_pentium4.obj
 0002:0001dc30       SC_1                       10085c30     LIBCMT:sin_pentium4.obj
 0002:0001dc40       SC_2                       10085c40     LIBCMT:sin_pentium4.obj
 0002:0001dc50       SC_3                       10085c50     LIBCMT:sin_pentium4.obj
 0002:0001dc60       SC_4                       10085c60     LIBCMT:sin_pentium4.obj
 0002:0001dc70       PI32INV                    10085c70     LIBCMT:sin_pentium4.obj
 0002:0001dc78       SHIFTER                    10085c78     LIBCMT:sin_pentium4.obj
 0002:0001dc80       P_2                        10085c80     LIBCMT:sin_pentium4.obj
 0002:0001dc90       P_1                        10085c90     LIBCMT:sin_pentium4.obj
 0002:0001dc98       P_3                        10085c98     LIBCMT:sin_pentium4.obj
 0002:0001dca0       TWO_POW_55                 10085ca0     LIBCMT:sin_pentium4.obj
 0002:0001dca8       TWO_POW_M55                10085ca8     LIBCMT:sin_pentium4.obj
 0002:0001dcb0       ALL_ONES                   10085cb0     LIBCMT:sin_pentium4.obj
 0002:0001dcb8       NEG_ZERO                   10085cb8     LIBCMT:sin_pentium4.obj
 0002:0001dcc0       ONE                        10085cc0     LIBCMT:sin_pentium4.obj
 0002:0001e9e0       __Win_errtab               100869e0     libcpmt:syserror.obj
 0002:0001ec38       __Sys_errtab               10086c38     libcpmt:syserror.obj
 0002:00022680       __catchsym$?_Copy@?$basic_string@DU?$char_traits@D@std@@V?$allocator@D@2@@std@@QAEXII@Z$5 1008a680     asxavdecc.obj
 0002:00022690       __catchsym$?_Copy@?$basic_string@DU?$char_traits@D@std@@V?$allocator@D@2@@std@@QAEXII@Z$4 1008a690     asxavdecc.obj
 0002:000226a0       __unwindtable$?_Copy@?$basic_string@DU?$char_traits@D@std@@V?$allocator@D@2@@std@@QAEXII@Z 1008a6a0     asxavdecc.obj
 0002:000226c0       __ehfuncinfo$?_Copy@?$basic_string@DU?$char_traits@D@std@@V?$allocator@D@2@@std@@QAEXII@Z 1008a6c0     asxavdecc.obj
 0002:000226e4       __tryblocktable$?_Copy@?$basic_string@DU?$char_traits@D@std@@V?$allocator@D@2@@std@@QAEXII@Z 1008a6e4     asxavdecc.obj
 0002:0002270c       __unwindtable$??0asxSubSystemAVDECC@@QAE@PAVasxSystem@@@Z 1008a70c     asxavdecc.obj
 0002:00022714       __ehfuncinfo$??0asxSubSystemAVDECC@@QAE@PAVasxSystem@@@Z 1008a714     asxavdecc.obj
 0002:00022738       __unwindtable$??1asxSubSystemAVDECC@@UAE@XZ 1008a738     asxavdecc.obj
 0002:00022740       __ehfuncinfo$??1asxSubSystemAVDECC@@UAE@XZ 1008a740     asxavdecc.obj
 0002:00022764       __unwindtable$?ReScan@asxSubSystemAVDECC@@UAEXXZ 1008a764     asxavdecc.obj
 0002:00022784       __ehfuncinfo$?ReScan@asxSubSystemAVDECC@@UAEXXZ 1008a784     asxavdecc.obj
 0002:000227a8       __unwindtable$??0asxAdapterAVDECC@@QAE@PAVcontroller@avdecc_lib@@PAVsystem@2@PAVasxSystem@@PADH3@Z 1008a7a8     asxavdecc.obj
 0002:000227b0       __ehfuncinfo$??0asxAdapterAVDECC@@QAE@PAVcontroller@avdecc_lib@@PAVsystem@2@PAVasxSystem@@PADH3@Z 1008a7b0     asxavdecc.obj
 0002:000227d4       __unwindtable$?SetDetails@asxAdapterAVDECC@@QAEXXZ 1008a7d4     asxavdecc.obj
 0002:000227dc       __ehfuncinfo$?SetDetails@asxAdapterAVDECC@@QAEXXZ 1008a7dc     asxavdecc.obj
 0002:00022800       __unwindtable$?CheckSubSystems@asxAdapterAVDECC@@UAE?AW4asxERROR@@PAI0@Z 1008a800     asxavdecc.obj
 0002:00022808       __ehfuncinfo$?CheckSubSystems@asxAdapterAVDECC@@UAE?AW4asxERROR@@PAI0@Z 1008a808     asxavdecc.obj
 0002:0002282c       __unwindtable$?UpdateAdapterProperties@asxAdapterAVDECC@@UAE?AW4asxERROR@@XZ 1008a82c     asxavdecc.obj
 0002:00022834       __ehfuncinfo$?UpdateAdapterProperties@asxAdapterAVDECC@@UAE?AW4asxERROR@@XZ 1008a834     asxavdecc.obj
 0002:00022858       __unwindtable$?Scan@asxSubSystemASIO@@UAEXXZ 1008a858     asxasio.obj
 0002:00022860       __ehfuncinfo$?Scan@asxSubSystemASIO@@UAEXXZ 1008a860     asxasio.obj
 0002:00022884       __unwindtable$??0asxAdapterASIO@@QAE@PAVasxSystem@@PAU_GUID@@PBD@Z 1008a884     asxasio.obj
 0002:0002288c       __ehfuncinfo$??0asxAdapterASIO@@QAE@PAVasxSystem@@PAU_GUID@@PBD@Z 1008a88c     asxasio.obj
 0002:000228b0       __unwindtable$??1asxAdapterASIO@@UAE@XZ 1008a8b0     asxasio.obj
 0002:000228b8       __ehfuncinfo$??1asxAdapterASIO@@UAE@XZ 1008a8b8     asxasio.obj
 0002:000228dc       __ehfuncinfo$?Scan@asxMixerScannerASIO@@EAEXPAVasxMixer@@@Z 1008a8dc     asxasio.obj
 0002:00022900       __unwindtable$?Scan@asxMixerScannerASIO@@EAEXPAVasxMixer@@@Z 1008a900     asxasio.obj
 0002:00022928       __unwindtable$??1asxPlayerASIO@@UAE@XZ 1008a928     asxasioplay.obj
 0002:00022930       __ehfuncinfo$??1asxPlayerASIO@@UAE@XZ 1008a930     asxasioplay.obj
 0002:00022954       __unwindtable$??1asxRecorderASIO@@UAE@XZ 1008a954     asxasiorec.obj
 0002:0002295c       __ehfuncinfo$??1asxRecorderASIO@@UAE@XZ 1008a95c     asxasiorec.obj
 0002:00022980       __ehfuncinfo$?asxCreateSubSystem@@YA?AW4asxERROR@@PAVasxSystem@@HPAPAVasxSubSystem@@@Z 1008a980     asxclass.obj
 0002:000229a4       __unwindtable$?asxCreateSubSystem@@YA?AW4asxERROR@@PAVasxSystem@@HPAPAVasxSubSystem@@@Z 1008a9a4     asxclass.obj
 0002:000229d4       __unwindtable$??1asxAdapter@@UAE@XZ 1008a9d4     asxclass.obj
 0002:000229e4       __ehfuncinfo$??1asxAdapter@@UAE@XZ 1008a9e4     asxclass.obj
 0002:00022a08       __unwindtable$??0asxAbstractAdapter@@QAE@PAVasxAdapter@@@Z 1008aa08     asxclass.obj
 0002:00022a10       __ehfuncinfo$??0asxAbstractAdapter@@QAE@PAVasxAdapter@@@Z 1008aa10     asxclass.obj
 0002:00022a34       __unwindtable$??1asxAbstractAdapter@@UAE@XZ 1008aa34     asxclass.obj
 0002:00022a3c       __ehfuncinfo$??1asxAbstractAdapter@@UAE@XZ 1008aa3c     asxclass.obj
 0002:00022a60       __unwindtable$??1asxSystem@@UAE@XZ 1008aa60     asxclass.obj
 0002:00022a80       __ehfuncinfo$??1asxSystem@@UAE@XZ 1008aa80     asxclass.obj
 0002:00022aa4       __unwindtable$?AddAdapter@asxSystem@@QAE?AW4asxERROR@@PAVasxAdapter@@PAVasxMixerScanner@@@Z 1008aaa4     asxclass.obj
 0002:00022aac       __ehfuncinfo$?AddAdapter@asxSystem@@QAE?AW4asxERROR@@PAVasxAdapter@@PAVasxMixerScanner@@@Z 1008aaac     asxclass.obj
 0002:00022ad0       __ehfuncinfo$??1asxMixer@@UAE@XZ 1008aad0     asxclass.obj
 0002:00022af4       __unwindtable$??1asxMixer@@UAE@XZ 1008aaf4     asxclass.obj
 0002:00022b1c       __unwindtable$??0asxBlockProperty@@QAE@W4asxUCONTROL_PTYPE@@W4asxUCONTROL_PFLAGS@@IPBDPAUasxParameterRangeInfo@@2@Z 1008ab1c     asxclass.obj
 0002:00022b24       __ehfuncinfo$??0asxBlockProperty@@QAE@W4asxUCONTROL_PTYPE@@W4asxUCONTROL_PFLAGS@@IPBDPAUasxParameterRangeInfo@@2@Z 1008ab24     asxclass.obj
 0002:00022b48       __unwindtable$?Scan@asxSubSystemDSND@@UAEXXZ 1008ab48     asxdsnd.obj
 0002:00022b58       __ehfuncinfo$?Scan@asxSubSystemDSND@@UAEXXZ 1008ab58     asxdsnd.obj
 0002:00022b7c       __unwindtable$??1asxMixerScannerDSND@@UAE@XZ 1008ab7c     asxdsnd.obj
 0002:00022b84       __ehfuncinfo$??1asxMixerScannerDSND@@UAE@XZ 1008ab84     asxdsnd.obj
 0002:00022ba8       __unwindtable$?Scan@asxMixerScannerDSND@@EAEXPAVasxMixer@@@Z 1008aba8     asxdsnd.obj
 0002:00022bc8       __ehfuncinfo$?Scan@asxMixerScannerDSND@@EAEXPAVasxMixer@@@Z 1008abc8     asxdsnd.obj
 0002:00022bec       __unwindtable$??0asxPlayerDSND@@QAE@PAVasxSubSystem@@PAVasxNode@@1PBU_GUID@@@Z 1008abec     asxdsndplay.obj
 0002:00022bf4       __ehfuncinfo$??0asxPlayerDSND@@QAE@PAVasxSubSystem@@PAVasxNode@@1PBU_GUID@@@Z 1008abf4     asxdsndplay.obj
 0002:00022c18       __unwindtable$??1asxPlayerDSND@@UAE@XZ 1008ac18     asxdsndplay.obj
 0002:00022c20       __ehfuncinfo$??1asxPlayerDSND@@UAE@XZ 1008ac20     asxdsndplay.obj
 0002:00022c44       __unwindtable$??1asxRecorderDSND@@UAE@XZ 1008ac44     asxdsndrec.obj
 0002:00022c4c       __ehfuncinfo$??1asxRecorderDSND@@UAE@XZ 1008ac4c     asxdsndrec.obj
 0002:00022c70       __unwindtable$??1asxMux@@UAE@XZ 1008ac70     asxhpi.obj
 0002:00022c80       __ehfuncinfo$??1asxMux@@UAE@XZ 1008ac80     asxhpi.obj
 0002:00022ca4       __unwindtable$??_GasxMux@@UAEPAXI@Z 1008aca4     asxhpi.obj
 0002:00022cb4       __ehfuncinfo$??_GasxMux@@UAEPAXI@Z 1008acb4     asxhpi.obj
 0002:00022cd8       __unwindtable$??1asxMode@@UAE@XZ 1008acd8     asxhpi.obj
 0002:00022ce0       __ehfuncinfo$??1asxMode@@UAE@XZ 1008ace0     asxhpi.obj
 0002:00022d04       __unwindtable$??_GasxMode@@UAEPAXI@Z 1008ad04     asxhpi.obj
 0002:00022d0c       __ehfuncinfo$??_GasxMode@@UAEPAXI@Z 1008ad0c     asxhpi.obj
 0002:00022d30       __unwindtable$??1asxTuner@@UAE@XZ 1008ad30     asxhpi.obj
 0002:00022d40       __ehfuncinfo$??1asxTuner@@UAE@XZ 1008ad40     asxhpi.obj
 0002:00022d64       __unwindtable$??_GasxTuner@@UAEPAXI@Z 1008ad64     asxhpi.obj
 0002:00022d74       __ehfuncinfo$??_GasxTuner@@UAEPAXI@Z 1008ad74     asxhpi.obj
 0002:00022d98       __unwindtable$??1asxSampleClock@@UAE@XZ 1008ad98     asxhpi.obj
 0002:00022da8       __ehfuncinfo$??1asxSampleClock@@UAE@XZ 1008ada8     asxhpi.obj
 0002:00022dcc       __unwindtable$??_GasxSampleClock@@UAEPAXI@Z 1008adcc     asxhpi.obj
 0002:00022ddc       __ehfuncinfo$??_GasxSampleClock@@UAEPAXI@Z 1008addc     asxhpi.obj
 0002:00022e00       __unwindtable$??1asxAes3Tx@@UAE@XZ 1008ae00     asxhpi.obj
 0002:00022e08       __ehfuncinfo$??1asxAes3Tx@@UAE@XZ 1008ae08     asxhpi.obj
 0002:00022e2c       __unwindtable$??_GasxAes3Tx@@UAEPAXI@Z 1008ae2c     asxhpi.obj
 0002:00022e34       __ehfuncinfo$??_GasxAes3Tx@@UAEPAXI@Z 1008ae34     asxhpi.obj
 0002:00022e58       __unwindtable$??1asxAes3Rx@@UAE@XZ 1008ae58     asxhpi.obj
 0002:00022e60       __ehfuncinfo$??1asxAes3Rx@@UAE@XZ 1008ae60     asxhpi.obj
 0002:00022e84       __unwindtable$??_GasxAes3Rx@@UAEPAXI@Z 1008ae84     asxhpi.obj
 0002:00022e8c       __ehfuncinfo$??_GasxAes3Rx@@UAEPAXI@Z 1008ae8c     asxhpi.obj
 0002:00022eb0       __unwindtable$??1asxCobranetContainer@@UAE@XZ 1008aeb0     asxhpi.obj
 0002:00022eb8       __ehfuncinfo$??1asxCobranetContainer@@UAE@XZ 1008aeb8     asxhpi.obj
 0002:00022edc       __unwindtable$??_GasxCobranetContainer@@UAEPAXI@Z 1008aedc     asxhpi.obj
 0002:00022ee4       __ehfuncinfo$??_GasxCobranetContainer@@UAEPAXI@Z 1008aee4     asxhpi.obj
 0002:00022f08       __unwindtable$??1asxCobranetRxContainer@@UAE@XZ 1008af08     asxhpi.obj
 0002:00022f10       __ehfuncinfo$??1asxCobranetRxContainer@@UAE@XZ 1008af10     asxhpi.obj
 0002:00022f34       __unwindtable$??_GasxCobranetRxContainer@@UAEPAXI@Z 1008af34     asxhpi.obj
 0002:00022f3c       __ehfuncinfo$??_GasxCobranetRxContainer@@UAEPAXI@Z 1008af3c     asxhpi.obj
 0002:00022f60       __unwindtable$??1asxCobranetTxContainer@@UAE@XZ 1008af60     asxhpi.obj
 0002:00022f68       __ehfuncinfo$??1asxCobranetTxContainer@@UAE@XZ 1008af68     asxhpi.obj
 0002:00022f8c       __unwindtable$??_GasxCobranetTxContainer@@UAEPAXI@Z 1008af8c     asxhpi.obj
 0002:00022f94       __ehfuncinfo$??_GasxCobranetTxContainer@@UAEPAXI@Z 1008af94     asxhpi.obj
 0002:00022fb8       __unwindtable$??1asxBlock@@UAE@XZ 1008afb8     asxhpi.obj
 0002:00022fc0       __ehfuncinfo$??1asxBlock@@UAE@XZ 1008afc0     asxhpi.obj
 0002:00022fe4       __unwindtable$??_GasxBlock@@UAEPAXI@Z 1008afe4     asxhpi.obj
 0002:00022fec       __ehfuncinfo$??_GasxBlock@@UAEPAXI@Z 1008afec     asxhpi.obj
 0002:00023010       __unwindtable$??0asxSubSystemHPI@@QAE@PAVasxSystem@@H@Z 1008b010     asxhpi.obj
 0002:00023018       __ehfuncinfo$??0asxSubSystemHPI@@QAE@PAVasxSystem@@H@Z 1008b018     asxhpi.obj
 0002:0002303c       __unwindtable$?AddSingleAdapter@asxSubSystemHPI@@AAEHIG@Z 1008b03c     asxhpi.obj
 0002:0002304c       __ehfuncinfo$?AddSingleAdapter@asxSubSystemHPI@@AAEHIG@Z 1008b04c     asxhpi.obj
 0002:00023070       __unwindtable$?AddDuplicateIndexAdapter@asxSubSystemHPI@@AAEXIGG@Z 1008b070     asxhpi.obj
 0002:00023078       __ehfuncinfo$?AddDuplicateIndexAdapter@asxSubSystemHPI@@AAEXIGG@Z 1008b078     asxhpi.obj
 0002:0002309c       __unwindtable$??0asxAdapterHPI@@QAE@PAVasxSystem@@HPBD@Z 1008b09c     asxhpi.obj
 0002:000230ac       __ehfuncinfo$??0asxAdapterHPI@@QAE@PAVasxSystem@@HPBD@Z 1008b0ac     asxhpi.obj
 0002:000230d0       __unwindtable$??1asxAdapterHPI@@UAE@XZ 1008b0d0     asxhpi.obj
 0002:000230d8       __ehfuncinfo$??1asxAdapterHPI@@UAE@XZ 1008b0d8     asxhpi.obj
 0002:000230fc       __ehfuncinfo$?Scan@asxMixerScannerHPI@@UAEXPAVasxMixer@@@Z 1008b0fc     asxhpi.obj
 0002:00023120       __unwindtable$?Scan@asxMixerScannerHPI@@UAEXPAVasxMixer@@@Z 1008b120     asxhpi.obj
 0002:00023248       __unwindtable$?CreateUniversalControl@asxMixerScannerHPI@@QAEPAVasxControlBase@@PAHPAVasxNode@@1I@Z 1008b248     asxhpi.obj
 0002:00023250       __ehfuncinfo$?CreateUniversalControl@asxMixerScannerHPI@@QAEPAVasxControlBase@@PAHPAVasxNode@@1I@Z 1008b250     asxhpi.obj
 0002:00023274       __unwindtable$??0asxMuxHPI@@QAE@PAVasxSubSystem@@PAVasxNode@@1I@Z 1008b274     asxhpi.obj
 0002:0002328c       __ehfuncinfo$??0asxMuxHPI@@QAE@PAVasxSubSystem@@PAVasxNode@@1I@Z 1008b28c     asxhpi.obj
 0002:000232b0       __unwindtable$??1asxMuxHPI@@UAE@XZ 1008b2b0     asxhpi.obj
 0002:000232c8       __ehfuncinfo$??1asxMuxHPI@@UAE@XZ 1008b2c8     asxhpi.obj
 0002:000232ec       __unwindtable$??0asxModeHPI@@QAE@PAVasxSubSystem@@PAVasxNode@@1I@Z 1008b2ec     asxhpi.obj
 0002:000232fc       __ehfuncinfo$??0asxModeHPI@@QAE@PAVasxSubSystem@@PAVasxNode@@1I@Z 1008b2fc     asxhpi.obj
 0002:00023320       __unwindtable$??1asxModeHPI@@UAE@XZ 1008b320     asxhpi.obj
 0002:00023330       __ehfuncinfo$??1asxModeHPI@@UAE@XZ 1008b330     asxhpi.obj
 0002:00023354       __unwindtable$??0asxSampleClockHPI@@QAE@PAVasxSubSystem@@PAVasxNode@@1I@Z 1008b354     asxhpi.obj
 0002:0002336c       __ehfuncinfo$??0asxSampleClockHPI@@QAE@PAVasxSubSystem@@PAVasxNode@@1I@Z 1008b36c     asxhpi.obj
 0002:00023390       __unwindtable$??1asxSampleClockHPI@@UAE@XZ 1008b390     asxhpi.obj
 0002:000233b0       __ehfuncinfo$??1asxSampleClockHPI@@UAE@XZ 1008b3b0     asxhpi.obj
 0002:000233d4       __unwindtable$??0asxTunerHPI@@QAE@PAVasxSubSystem@@PAVasxNode@@1I@Z 1008b3d4     asxhpi.obj
 0002:000233dc       __ehfuncinfo$??0asxTunerHPI@@QAE@PAVasxSubSystem@@PAVasxNode@@1I@Z 1008b3dc     asxhpi.obj
 0002:00023400       __unwindtable$??1asxTunerHPI@@UAE@XZ 1008b400     asxhpi.obj
 0002:00023410       __ehfuncinfo$??1asxTunerHPI@@UAE@XZ 1008b410     asxhpi.obj
 0002:00023434       __unwindtable$??0asxAes3TxHPI@@QAE@PAVasxSubSystem@@PAVasxNode@@1I@Z 1008b434     asxhpi.obj
 0002:0002343c       __ehfuncinfo$??0asxAes3TxHPI@@QAE@PAVasxSubSystem@@PAVasxNode@@1I@Z 1008b43c     asxhpi.obj
 0002:00023460       __unwindtable$??1asxAes3TxHPI@@UAE@XZ 1008b460     asxhpi.obj
 0002:00023468       __ehfuncinfo$??1asxAes3TxHPI@@UAE@XZ 1008b468     asxhpi.obj
 0002:0002348c       __unwindtable$??0asxAesebuReceiverHPI@@QAE@PAVasxSubSystem@@PAVasxNode@@1I@Z 1008b48c     asxhpi.obj
 0002:00023494       __ehfuncinfo$??0asxAesebuReceiverHPI@@QAE@PAVasxSubSystem@@PAVasxNode@@1I@Z 1008b494     asxhpi.obj
 0002:000234b8       __unwindtable$??1asxAesebuReceiverHPI@@UAE@XZ 1008b4b8     asxhpi.obj
 0002:000234c0       __ehfuncinfo$??1asxAesebuReceiverHPI@@UAE@XZ 1008b4c0     asxhpi.obj
 0002:000234e4       __unwindtable$??0asxGpioHPI@@QAE@PAVasxSubSystem@@PAVasxNode@@1IHH@Z 1008b4e4     asxhpi.obj
 0002:000234ec       __ehfuncinfo$??0asxGpioHPI@@QAE@PAVasxSubSystem@@PAVasxNode@@1IHH@Z 1008b4ec     asxhpi.obj
 0002:00023510       __unwindtable$??1asxGpioHPI@@UAE@XZ 1008b510     asxhpi.obj
 0002:00023518       __ehfuncinfo$??1asxGpioHPI@@UAE@XZ 1008b518     asxhpi.obj
 0002:0002353c       __unwindtable$??0asxCompanderHPI_Legacy@@QAE@PAVasxSubSystem@@PAVasxNode@@1I@Z 1008b53c     asxhpi.obj
 0002:00023544       __ehfuncinfo$??0asxCompanderHPI_Legacy@@QAE@PAVasxSubSystem@@PAVasxNode@@1I@Z 1008b544     asxhpi.obj
 0002:00023568       __unwindtable$??0asxCobranetHPI@@QAE@PAVasxSubSystem@@PAVasxNode@@1IH@Z 1008b568     asxhpi.obj
 0002:00023570       __ehfuncinfo$??0asxCobranetHPI@@QAE@PAVasxSubSystem@@PAVasxNode@@1IH@Z 1008b570     asxhpi.obj
 0002:00023594       __unwindtable$??0asxCobranetRxHPI@@QAE@PAVasxSubSystem@@PAVasxNode@@1IH@Z 1008b594     asxhpi.obj
 0002:0002359c       __ehfuncinfo$??0asxCobranetRxHPI@@QAE@PAVasxSubSystem@@PAVasxNode@@1IH@Z 1008b59c     asxhpi.obj
 0002:000235c0       __unwindtable$??0asxCobranetTxHPI@@QAE@PAVasxSubSystem@@PAVasxNode@@1IH@Z 1008b5c0     asxhpi.obj
 0002:000235c8       __ehfuncinfo$??0asxCobranetTxHPI@@QAE@PAVasxSubSystem@@PAVasxNode@@1IH@Z 1008b5c8     asxhpi.obj
 0002:000235ec       __unwindtable$??1asxBlockHPI@@UAE@XZ 1008b5ec     asxhpi.obj
 0002:000235f4       __ehfuncinfo$??1asxBlockHPI@@UAE@XZ 1008b5f4     asxhpi.obj
 0002:00023618       __unwindtable$?AddProperty@asxBlockHPI@@QAE?AW4asxERROR@@I@Z 1008b618     asxhpi.obj
 0002:00023620       __ehfuncinfo$?AddProperty@asxBlockHPI@@QAE?AW4asxERROR@@I@Z 1008b620     asxhpi.obj
 0002:00023644       __unwindtable$??1asxPlayerHPI@@UAE@XZ 1008b644     asxhpiplay.obj
 0002:0002364c       __ehfuncinfo$??1asxPlayerHPI@@UAE@XZ 1008b64c     asxhpiplay.obj
 0002:00023670       __unwindtable$??1asxRecorderHPI@@UAE@XZ 1008b670     asxhpirec.obj
 0002:00023678       __ehfuncinfo$??1asxRecorderHPI@@UAE@XZ 1008b678     asxhpirec.obj
 0002:0002369c       __unwindtable$?Open@asxPlayerFile@@QAE?AW4asxERROR@@XZ 1008b69c     asxplay.obj
 0002:000236a4       __ehfuncinfo$?Open@asxPlayerFile@@QAE?AW4asxERROR@@XZ 1008b6a4     asxplay.obj
 0002:000236c8       __unwindtable$?AddFile@asxPlayerFileList@@QAEXPBD@Z 1008b6c8     asxplay.obj
 0002:000236d0       __ehfuncinfo$?AddFile@asxPlayerFileList@@QAEXPBD@Z 1008b6d0     asxplay.obj
 0002:000236f4       __unwindtable$??1asxPlayer@@UAE@XZ 1008b6f4     asxplay.obj
 0002:00023704       __ehfuncinfo$??1asxPlayer@@UAE@XZ 1008b704     asxplay.obj
 0002:00023728       __unwindtable$?PreLoad@asxPlayer@@UAE?AW4asxERROR@@W4asxTIMESCALE@@K@Z 1008b728     asxplay.obj
 0002:00023730       __ehfuncinfo$?PreLoad@asxPlayer@@UAE?AW4asxERROR@@W4asxTIMESCALE@@K@Z 1008b730     asxplay.obj
 0002:00023754       __unwindtable$?Start@asxPlayer@@UAE?AW4asxERROR@@XZ 1008b754     asxplay.obj
 0002:0002375c       __ehfuncinfo$?Start@asxPlayer@@UAE?AW4asxERROR@@XZ 1008b75c     asxplay.obj
 0002:00023780       __unwindtable$?OpenPlaylist@asxPlayer@@UAE?AW4asxERROR@@PAPBDI@Z 1008b780     asxplay.obj
 0002:00023788       __ehfuncinfo$?OpenPlaylist@asxPlayer@@UAE?AW4asxERROR@@PAPBDI@Z 1008b788     asxplay.obj
 0002:000237ac       __unwindtable$?Pause@asxPlayer@@UAE?AW4asxERROR@@XZ 1008b7ac     asxplay.obj
 0002:000237b4       __ehfuncinfo$?Pause@asxPlayer@@UAE?AW4asxERROR@@XZ 1008b7b4     asxplay.obj
 0002:000237d8       __unwindtable$?Stop@asxPlayer@@UAE?AW4asxERROR@@XZ 1008b7d8     asxplay.obj
 0002:000237e0       __ehfuncinfo$?Stop@asxPlayer@@UAE?AW4asxERROR@@XZ 1008b7e0     asxplay.obj
 0002:00023804       __unwindtable$?Close@asxPlayer@@UAE?AW4asxERROR@@XZ 1008b804     asxplay.obj
 0002:0002380c       __ehfuncinfo$?Close@asxPlayer@@UAE?AW4asxERROR@@XZ 1008b80c     asxplay.obj
 0002:00023830       __unwindtable$?CreateFileA@asxRecorder@@MAE?AW4asxERROR@@XZ 1008b830     asxrec.obj
 0002:00023838       __ehfuncinfo$?CreateFileA@asxRecorder@@MAE?AW4asxERROR@@XZ 1008b838     asxrec.obj
 0002:0002385c       __unwindtable$??1asxRecorder@@UAE@XZ 1008b85c     asxrec.obj
 0002:00023864       __ehfuncinfo$??1asxRecorder@@UAE@XZ 1008b864     asxrec.obj
 0002:00023888       __unwindtable$??0asxSubSystemSNMP@@QAE@PAVasxSystem@@@Z 1008b888     asxsnmp.obj
 0002:00023898       __ehfuncinfo$??0asxSubSystemSNMP@@QAE@PAVasxSystem@@@Z 1008b898     asxsnmp.obj
 0002:000238bc       __unwindtable$??1asxSubSystemSNMP@@UAE@XZ 1008b8bc     asxsnmp.obj
 0002:000238cc       __ehfuncinfo$??1asxSubSystemSNMP@@UAE@XZ 1008b8cc     asxsnmp.obj
 0002:000238f0       __unwindtable$?ReScan@asxSubSystemSNMP@@UAEXXZ 1008b8f0     asxsnmp.obj
 0002:00023908       __ehfuncinfo$?ReScan@asxSubSystemSNMP@@UAEXXZ 1008b908     asxsnmp.obj
 0002:0002392c       __unwindtable$??0asxAdapterSNMP@@QAE@PAVasxSystem@@PADPBD2PAVSnmpSession@@@Z 1008b92c     asxsnmp.obj
 0002:0002393c       __ehfuncinfo$??0asxAdapterSNMP@@QAE@PAVasxSystem@@PADPBD2PAVSnmpSession@@@Z 1008b93c     asxsnmp.obj
 0002:00023960       __unwindtable$??1asxAdapterSNMP@@UAE@XZ 1008b960     asxsnmp.obj
 0002:00023968       __ehfuncinfo$??1asxAdapterSNMP@@UAE@XZ 1008b968     asxsnmp.obj
 0002:0002398c       __unwindtable$?NewIpAddress@asxAdapterSNMP@@QAEXPBD@Z 1008b98c     asxsnmp.obj
 0002:00023994       __ehfuncinfo$?NewIpAddress@asxAdapterSNMP@@QAEXPBD@Z 1008b994     asxsnmp.obj
 0002:000239b8       __ehfuncinfo$?Scan@asxMixerScannerSNMP@@UAEXPAVasxMixer@@@Z 1008b9b8     asxsnmp.obj
 0002:000239dc       __unwindtable$?Scan@asxMixerScannerSNMP@@UAEXPAVasxMixer@@@Z 1008b9dc     asxsnmp.obj
 0002:00023a34       __unwindtable$??0asxCobranetSNMP@@QAE@PAVasxSubSystem@@PAVasxNode@@1PAVCobraNetNode@@PBD@Z 1008ba34     asxsnmp.obj
 0002:00023a3c       __ehfuncinfo$??0asxCobranetSNMP@@QAE@PAVasxSubSystem@@PAVasxNode@@1PAVCobraNetNode@@PBD@Z 1008ba3c     asxsnmp.obj
 0002:00023a60       __unwindtable$?Scan@asxMixerScannerUnreachableSNMP@@UAEXPAVasxMixer@@@Z 1008ba60     asxsnmp.obj
 0002:00023a78       __ehfuncinfo$?Scan@asxMixerScannerUnreachableSNMP@@UAEXPAVasxMixer@@@Z 1008ba78     asxsnmp.obj
 0002:00023a9c       __ehfuncinfo$?asxTR800_Create@@YAXPAVasxSubSystem@@PAVCobraNetNode@@PAVasxMixer@@@Z 1008ba9c     asxtr800.obj
 0002:00023ac0       __unwindtable$?asxTR800_Create@@YAXPAVasxSubSystem@@PAVCobraNetNode@@PAVasxMixer@@@Z 1008bac0     asxtr800.obj
 0002:00023b18       __unwindtable$??0asxLevelTR800@@QAE@PAVasxSubSystem@@PAVasxTR800helperthread@@PAVasxNode@@2@Z 1008bb18     asxtr800.obj
 0002:00023b20       __ehfuncinfo$??0asxLevelTR800@@QAE@PAVasxSubSystem@@PAVasxTR800helperthread@@PAVasxNode@@2@Z 1008bb20     asxtr800.obj
 0002:00023b44       __unwindtable$??0asxBlockTR800OptoMode@@QAE@PAVasxSubSystem@@PAVasxTR800helperthread@@PAVasxNode@@2@Z 1008bb44     asxtr800.obj
 0002:00023b54       __ehfuncinfo$??0asxBlockTR800OptoMode@@QAE@PAVasxSubSystem@@PAVasxTR800helperthread@@PAVasxNode@@2@Z 1008bb54     asxtr800.obj
 0002:00023b78       __unwindtable$??1asxBlockTR800OptoMode@@UAE@XZ 1008bb78     asxtr800.obj
 0002:00023b80       __ehfuncinfo$??1asxBlockTR800OptoMode@@UAE@XZ 1008bb80     asxtr800.obj
 0002:00023ba4       __unwindtable$??_GasxBlockTR800OptoMode@@UAEPAXI@Z 1008bba4     asxtr800.obj
 0002:00023bac       __ehfuncinfo$??_GasxBlockTR800OptoMode@@UAEPAXI@Z 1008bbac     asxtr800.obj
 0002:00023bd0       __unwindtable$??0asxBlockTR800Status@@QAE@PAVasxSubSystem@@PAVasxNode@@1_N@Z 1008bbd0     asxtr800.obj
 0002:00023be0       __ehfuncinfo$??0asxBlockTR800Status@@QAE@PAVasxSubSystem@@PAVasxNode@@1_N@Z 1008bbe0     asxtr800.obj
 0002:00023c04       __unwindtable$??1asxBlockTR800Status@@UAE@XZ 1008bc04     asxtr800.obj
 0002:00023c0c       __ehfuncinfo$??1asxBlockTR800Status@@UAE@XZ 1008bc0c     asxtr800.obj
 0002:00023c30       __unwindtable$??_GasxBlockTR800Status@@UAEPAXI@Z 1008bc30     asxtr800.obj
 0002:00023c38       __ehfuncinfo$??_GasxBlockTR800Status@@UAEPAXI@Z 1008bc38     asxtr800.obj
 0002:00023c5c       __unwindtable$?Scan@asxSubSystemWAVE@@UAEXXZ 1008bc5c     asxwave.obj
 0002:00023c64       __ehfuncinfo$?Scan@asxSubSystemWAVE@@UAEXXZ 1008bc64     asxwave.obj
 0002:00023c88       __unwindtable$??1asxAdapterWAVE@@UAE@XZ 1008bc88     asxwave.obj
 0002:00023c90       __ehfuncinfo$??1asxAdapterWAVE@@UAE@XZ 1008bc90     asxwave.obj
 0002:00023cb4       __ehfuncinfo$?AddControl@asxMixerScannerWAVE@@AAEXPAVasxMixer@@PAVControlTracker@@PAUHMIXEROBJ__@@PAVasxNode@@3PAUtagMIXERCONTROLA@@H@Z 1008bcb4     asxwave.obj
 0002:00023cd8       __unwindtable$?AddControl@asxMixerScannerWAVE@@AAEXPAVasxMixer@@PAVControlTracker@@PAUHMIXEROBJ__@@PAVasxNode@@3PAUtagMIXERCONTROLA@@H@Z 1008bcd8     asxwave.obj
 0002:00023dc0       __unwindtable$??1asxMixerScannerWAVE@@UAE@XZ 1008bdc0     asxwave.obj
 0002:00023dd0       __ehfuncinfo$??1asxMixerScannerWAVE@@UAE@XZ 1008bdd0     asxwave.obj
 0002:00023df4       __ehfuncinfo$?Scan@asxMixerScannerWAVE@@UAEXPAVasxMixer@@@Z 1008bdf4     asxwave.obj
 0002:00023e18       __unwindtable$?Scan@asxMixerScannerWAVE@@UAEXPAVasxMixer@@@Z 1008be18     asxwave.obj
 0002:00023e60       __unwindtable$??0waveControlMuxHelper@@QAE@PAUHMIXEROBJ__@@PAVwaveControlInfo@@PAV?$TASIArray@VTASICString@@@@@Z 1008be60     asxwave.obj
 0002:00023e68       __ehfuncinfo$??0waveControlMuxHelper@@QAE@PAUHMIXEROBJ__@@PAVwaveControlInfo@@PAV?$TASIArray@VTASICString@@@@@Z 1008be68     asxwave.obj
 0002:00023e8c       __unwindtable$??0asxVolumeWAVE@@QAE@PAVasxSubSystem@@PAUHMIXEROBJ__@@PAVasxNode@@2PAUtagMIXERCONTROLA@@H3@Z 1008be8c     asxwave.obj
 0002:00023e94       __ehfuncinfo$??0asxVolumeWAVE@@QAE@PAVasxSubSystem@@PAUHMIXEROBJ__@@PAVasxNode@@2PAUtagMIXERCONTROLA@@H3@Z 1008be94     asxwave.obj
 0002:00023eb8       __unwindtable$??0asxMeterWAVE@@QAE@PAVasxSubSystem@@PAUHMIXEROBJ__@@PAVasxNode@@2PAUtagMIXERCONTROLA@@H@Z 1008beb8     asxwave.obj
 0002:00023ec0       __ehfuncinfo$??0asxMeterWAVE@@QAE@PAVasxSubSystem@@PAUHMIXEROBJ__@@PAVasxNode@@2PAUtagMIXERCONTROLA@@H@Z 1008bec0     asxwave.obj
 0002:00023ee4       __unwindtable$??0asxLevelWAVE@@QAE@PAVasxSubSystem@@PAUHMIXEROBJ__@@PAVasxNode@@2PAUtagMIXERCONTROLA@@H@Z 1008bee4     asxwave.obj
 0002:00023eec       __ehfuncinfo$??0asxLevelWAVE@@QAE@PAVasxSubSystem@@PAUHMIXEROBJ__@@PAVasxNode@@2PAUtagMIXERCONTROLA@@H@Z 1008beec     asxwave.obj
 0002:00023f10       __unwindtable$??0asxMuxWAVE@@QAE@PAVasxSubSystem@@PAUHMIXEROBJ__@@PAVasxNode@@2PAUtagMIXERCONTROLA@@H@Z 1008bf10     asxwave.obj
 0002:00023f18       __ehfuncinfo$??0asxMuxWAVE@@QAE@PAVasxSubSystem@@PAUHMIXEROBJ__@@PAVasxNode@@2PAUtagMIXERCONTROLA@@H@Z 1008bf18     asxwave.obj
 0002:00023f3c       __unwindtable$??1asxMuxWAVE@@UAE@XZ 1008bf3c     asxwave.obj
 0002:00023f4c       __ehfuncinfo$??1asxMuxWAVE@@UAE@XZ 1008bf4c     asxwave.obj
 0002:00023f70       __unwindtable$??0asxModeWAVE@@QAE@PAVasxSubSystem@@PAUHMIXEROBJ__@@PAVasxNode@@2PAUtagMIXERCONTROLA@@H@Z 1008bf70     asxwave.obj
 0002:00023f78       __ehfuncinfo$??0asxModeWAVE@@QAE@PAVasxSubSystem@@PAUHMIXEROBJ__@@PAVasxNode@@2PAUtagMIXERCONTROLA@@H@Z 1008bf78     asxwave.obj
 0002:00023f9c       __unwindtable$??1asxModeWAVE@@UAE@XZ 1008bf9c     asxwave.obj
 0002:00023fa4       __ehfuncinfo$??1asxModeWAVE@@UAE@XZ 1008bfa4     asxwave.obj
 0002:00023fc8       __unwindtable$??0asxTunerWAVE@@QAE@PAVasxSubSystem@@PAUHMIXEROBJ__@@PAVasxNode@@2HPAUtagMIXERCONTROLA@@3333@Z 1008bfc8     asxwave.obj
 0002:00023fd8       __ehfuncinfo$??0asxTunerWAVE@@QAE@PAVasxSubSystem@@PAUHMIXEROBJ__@@PAVasxNode@@2HPAUtagMIXERCONTROLA@@3333@Z 1008bfd8     asxwave.obj
 0002:00023ffc       __unwindtable$??1asxTunerWAVE@@UAE@XZ 1008bffc     asxwave.obj
 0002:00024014       __ehfuncinfo$??1asxTunerWAVE@@UAE@XZ 1008c014     asxwave.obj
 0002:00024038       __unwindtable$??0asxCobranetWAVE@@QAE@PAVasxSubSystem@@PAUHMIXEROBJ__@@PAVasxNode@@2HPAUtagMIXERCONTROLA@@3@Z 1008c038     asxwave.obj
 0002:00024040       __ehfuncinfo$??0asxCobranetWAVE@@QAE@PAVasxSubSystem@@PAUHMIXEROBJ__@@PAVasxNode@@2HPAUtagMIXERCONTROLA@@3@Z 1008c040     asxwave.obj
 0002:00024064       __unwindtable$??0asxToneDetectorWAVE@@QAE@PAVasxSubSystem@@PAUHMIXEROBJ__@@PAVasxNode@@2PAUtagMIXERCONTROLA@@H@Z 1008c064     asxwave.obj
 0002:0002406c       __ehfuncinfo$??0asxToneDetectorWAVE@@QAE@PAVasxSubSystem@@PAUHMIXEROBJ__@@PAVasxNode@@2PAUtagMIXERCONTROLA@@H@Z 1008c06c     asxwave.obj
 0002:00024090       __unwindtable$??0asxSilenceDetectorWAVE@@QAE@PAVasxSubSystem@@PAUHMIXEROBJ__@@PAVasxNode@@2PAUtagMIXERCONTROLA@@H@Z 1008c090     asxwave.obj
 0002:00024098       __ehfuncinfo$??0asxSilenceDetectorWAVE@@QAE@PAVasxSubSystem@@PAUHMIXEROBJ__@@PAVasxNode@@2PAUtagMIXERCONTROLA@@H@Z 1008c098     asxwave.obj
 0002:000240bc       __unwindtable$?AddCobranet@@YAXPAVasxMixer@@PAVasxSubSystem@@PAVControlTracker@@PAUHMIXEROBJ__@@PAVasxNode@@4PAUtagMIXERCONTROLA@@H@Z 1008c0bc     asxwave.obj
 0002:000240cc       __ehfuncinfo$?AddCobranet@@YAXPAVasxMixer@@PAVasxSubSystem@@PAVControlTracker@@PAUHMIXEROBJ__@@PAVasxNode@@4PAUtagMIXERCONTROLA@@H@Z 1008c0cc     asxwave.obj
 0002:000240f0       __unwindtable$?AddTuner@@YAXPAVasxMixer@@PAVasxSubSystem@@PAVControlTracker@@PAUHMIXEROBJ__@@PAVasxNode@@4PAUtagMIXERCONTROLA@@H@Z 1008c0f0     asxwave.obj
 0002:000240f8       __ehfuncinfo$?AddTuner@@YAXPAVasxMixer@@PAVasxSubSystem@@PAVControlTracker@@PAUHMIXEROBJ__@@PAVasxNode@@4PAUtagMIXERCONTROLA@@H@Z 1008c0f8     asxwave.obj
 0002:0002411c       __unwindtable$??1asxPlayerWAVE@@UAE@XZ 1008c11c     asxwaveplay.obj
 0002:00024124       __ehfuncinfo$??1asxPlayerWAVE@@UAE@XZ 1008c124     asxwaveplay.obj
 0002:00024148       __unwindtable$??1asxRecorderWAVE@@UAE@XZ 1008c148     asxwaverec.obj
 0002:00024150       __ehfuncinfo$??1asxRecorderWAVE@@UAE@XZ 1008c150     asxwaverec.obj
 0002:00024174       __unwindtable$??1TWavFileTypeWav@@UAE@XZ 1008c174     twavfile.obj
 0002:0002417c       __ehfuncinfo$??1TWavFileTypeWav@@UAE@XZ 1008c17c     twavfile.obj
 0002:000241a0       __unwindtable$??_GTWavFileTypeWav@@UAEPAXI@Z 1008c1a0     twavfile.obj
 0002:000241a8       __ehfuncinfo$??_GTWavFileTypeWav@@UAEPAXI@Z 1008c1a8     twavfile.obj
 0002:000241cc       __unwindtable$??0TWavFileTypeGenerator@@QAE@PBD0PAJ@Z 1008c1cc     twavfile.obj
 0002:000241d4       __ehfuncinfo$??0TWavFileTypeGenerator@@QAE@PBD0PAJ@Z 1008c1d4     twavfile.obj
 0002:000241f8       __ehfuncinfo$?OpenWavFile@@YAPAVTWavFileBase@@PBD0PAJ@Z 1008c1f8     twavfile.obj
 0002:0002421c       __unwindtable$?OpenWavFile@@YAPAVTWavFileBase@@PBD0PAJ@Z 1008c21c     twavfile.obj
 0002:00024244       __unwindtable$??0TWavFileWithFifo@@QAE@PAVTWavFileBase@@JW4FifoDirection@0@@Z 1008c244     twavfilefifo.obj
 0002:00024254       __ehfuncinfo$??0TWavFileWithFifo@@QAE@PAVTWavFileBase@@JW4FifoDirection@0@@Z 1008c254     twavfilefifo.obj
 0002:00024278       __unwindtable$??1TWavFileWithFifo@@UAE@XZ 1008c278     twavfilefifo.obj
 0002:00024288       __ehfuncinfo$??1TWavFileWithFifo@@UAE@XZ 1008c288     twavfilefifo.obj
 0002:000242b0       __sehtable$_printf         1008c2b0     LIBCMT:printf.obj
 0002:000242d0       __sehtable$_vprintf_helper 1008c2d0     LIBCMT:vprintf.obj
 0002:00024340       __sehtable$__onexit        1008c340     LIBCMT:onexit.obj
 0002:00024360       __sehtable$___RTDynamicCast 1008c360     LIBCMT:rtti.obj
 0002:00024380       __sehtable$___RTtypeid     1008c380     LIBCMT:rtti.obj
 0002:000243a0       __sehtable$___RTCastToVoid 1008c3a0     LIBCMT:rtti.obj
 0002:00024468       __sehtable$_getenv         1008c468     LIBCMT:getenv.obj
 0002:00024488       __sehtable$_getenv_s       1008c488     LIBCMT:getenv.obj
 0002:000244a8       __sehtable$__dupenv_s      1008c4a8     LIBCMT:getenv.obj
 0002:000244c8       __sehtable$_fclose         1008c4c8     LIBCMT:fclose.obj
 0002:000244e8       __sehtable$__fsopen        1008c4e8     LIBCMT:fopen.obj
 0002:00024508       __sehtable$_fread_s        1008c508     LIBCMT:fread.obj
 0002:00024528       __sehtable$_fseek          1008c528     LIBCMT:fseek.obj
 0002:00024548       __sehtable$_ftell          1008c548     LIBCMT:ftell.obj
 0002:00024568       __sehtable$_fwrite         1008c568     LIBCMT:fwrite.obj
 0002:00024588       __sehtable$__CRT_INIT@12   1008c588     LIBCMT:dllcrt0.obj
 0002:000245a8       __sehtable$___DllMainCRTStartup 1008c5a8     LIBCMT:dllcrt0.obj
 0002:000245c8       __sehtable$___updatetlocinfo 1008c5c8     LIBCMT:localref.obj
 0002:000245e8       __sehtable$___updatetmbcinfo 1008c5e8     LIBCMT:mbctype.obj
 0002:00024608       __sehtable$__setmbcp       1008c608     LIBCMT:mbctype.obj
 0002:00024628       __sehtable$__freefls@4     1008c628     LIBCMT:tidtable.obj
 0002:00024650       __sehtable$__initptd       1008c650     LIBCMT:tidtable.obj
 0002:00024678       __sehtable$__get_current_locale 1008c678     LIBCMT:wsetloca.obj
 0002:000246a0       __sehtable$__free_locale   1008c6a0     LIBCMT:wsetloca.obj
 0002:000246c8       __sehtable$__wsetlocale    1008c6c8     LIBCMT:wsetloca.obj
 0002:00024700       __sehtable$__locterm       1008c700     LIBCMT:wsetloca.obj
 0002:00024720       __sehtable$_doexit         1008c720     LIBCMT:crt0dat.obj
 0002:00024740       __sehtable$?_Name_base@type_info@@CAPBDPBV1@PAU__type_info_node@@@Z 1008c740     LIBCMT:typname.obj
 0002:00024760       __sehtable$?_Type_info_dtor@type_info@@CAXPAV1@@Z 1008c760     LIBCMT:typname.obj
 0002:00024780       __sehtable$?_Name_base_internal@type_info@@CAPBDPBV1@PAU__type_info_node@@@Z 1008c780     LIBCMT:typname.obj
 0002:000247a0       __sehtable$?_Type_info_dtor_internal@type_info@@CAXPAV1@@Z 1008c7a0     LIBCMT:typname.obj
 0002:000247c0       __sehtable$___clean_type_info_names_internal 1008c7c0     LIBCMT:typname.obj
 0002:000247e0       __sehtable$___set_fpsr_sse2 1008c7e0     LIBCMT:fpctrl.obj
 0002:00024800       __sehtable$?terminate@@YAXXZ 1008c800     LIBCMT:hooks.obj
 0002:00024820       __sehtable$?_inconsistency@@YAXXZ 1008c820     LIBCMT:hooks.obj
 0002:00024840       __sehtable$___FrameUnwindToState 1008c840     LIBCMT:frame.obj
 0002:00024868       __sehtable$?CallCatchBlock@@YAPAXPAUEHExceptionRecord@@PAUEHRegistrationNode@@PAU_CONTEXT@@PBU_s_FuncInfo@@PAXHK@Z 1008c868     LIBCMT:frame.obj
 0002:00024890       __sehtable$___BuildCatchObject 1008c890     LIBCMT:frame.obj
 0002:000248b0       __sehtable$___DestructExceptionObject 1008c8b0     LIBCMT:frame.obj
 0002:000248cc       __catchsym$?CallUnexpected@@YAXPBU_s_ESTypeList@@@Z$2 1008c8cc     LIBCMT:frame.obj
 0002:000248dc       __unwindtable$?CallUnexpected@@YAXPBU_s_ESTypeList@@@Z 1008c8dc     LIBCMT:frame.obj
 0002:000248ec       __tryblocktable$?CallUnexpected@@YAXPBU_s_ESTypeList@@@Z 1008c8ec     LIBCMT:frame.obj
 0002:00024900       __ehfuncinfo$?CallUnexpected@@YAXPBU_s_ESTypeList@@@Z 1008c900     LIBCMT:frame.obj
 0002:00024928       __sehtable$___BuildCatchObjectHelper 1008c928     LIBCMT:frame.obj
 0002:00024980       __sehtable$__mtinitlocknum 1008c980     LIBCMT:mlock.obj
 0002:000249a0       __sehtable$__close         1008c9a0     LIBCMT:close.obj
 0002:000249c0       __sehtable$_fflush         1008c9c0     LIBCMT:fflush.obj
 0002:000249e0       __sehtable$_flsall         1008c9e0     LIBCMT:fflush.obj
 0002:00024a08       __sehtable$__getstream     1008ca08     LIBCMT:stream.obj
 0002:00024a28       __sehtable$__read          1008ca28     LIBCMT:read.obj
 0002:00024a48       __sehtable$__lseek         1008ca48     LIBCMT:lseek.obj
 0002:00024a68       __sehtable$__lseeki64      1008ca68     LIBCMT:lseeki64.obj
 0002:00024a88       __sehtable$__ioinit        1008ca88     LIBCMT:ioinit.obj
 0002:00024aa8       __sehtable$__write         1008caa8     LIBCMT:write.obj
 0002:00024ac8       __sehtable$__IsNonwritableInCurrentImage 1008cac8     LIBCMT:pesect.obj
 0002:00024ae8       __sehtable$_signal         1008cae8     LIBCMT:winsig.obj
 0002:00024b08       __sehtable$_raise          1008cb08     LIBCMT:winsig.obj
 0002:00024b28       __sehtable$_ctrlevent_capture@4 1008cb28     LIBCMT:winsig.obj
 0002:00024b48       __sehtable$__fcloseall     1008cb48     LIBCMT:closeall.obj
 0002:00024b68       __sehtable$___unDName      1008cb68     LIBCMT:undname.obj
 0002:00024b88       __sehtable$___unDNameEx    1008cb88     LIBCMT:undname.obj
 0002:00024ba8       __sehtable$__alloc_osfhnd  1008cba8     LIBCMT:osfinfo.obj
 0002:00024bd0       __sehtable$___lock_fhandle 1008cbd0     LIBCMT:osfinfo.obj
 0002:00024bf0       __sehtable$__open_osfhandle 1008cbf0     LIBCMT:osfinfo.obj
 0002:00024c10       __sehtable$__commit        1008cc10     LIBCMT:commit.obj
 0002:00024c30       __sehtable$__sopen_helper  1008cc30     LIBCMT:open.obj
 0002:00024c50       __sehtable$__open          1008cc50     LIBCMT:open.obj
 0002:00024c70       __sehtable$__putwch        1008cc70     LIBCMT:putwch.obj
 0002:00024c90       __sehtable$__wsopen_helper 1008cc90     LIBCMT:wopen.obj
 0002:00024cb0       __sehtable$__wopen         1008ccb0     LIBCMT:wopen.obj
 0002:00024cd0       __sehtable$__chsize_s      1008ccd0     LIBCMT:chsize.obj
 0002:00024cf0       __sehtable$__setmode       1008ccf0     LIBCMT:setmode.obj
 0002:00025100       .edata                     1008d100     asx32.exp
 0002:00025128       rgpv                       1008d128     asx32.exp
 0002:00025590       rgszName                   1008d590     asx32.exp
 0002:000259f8       rgwOrd                     1008d9f8     asx32.exp
 0002:00025c2c       szName                     1008dc2c     asx32.exp
 0002:00025c36       $N00001                    1008dc36     asx32.exp
 0002:00025c4d       $N00002                    1008dc4d     asx32.exp
 0002:00025c64       $N00003                    1008dc64     asx32.exp
 0002:00025c87       $N00004                    1008dc87     asx32.exp
 0002:00025ca9       $N00005                    1008dca9     asx32.exp
 0002:00025cc6       $N00006                    1008dcc6     asx32.exp
 0002:00025ce7       $N00007                    1008dce7     asx32.exp
 0002:00025d04       $N00008                    1008dd04     asx32.exp
 0002:00025d2a       $N00009                    1008dd2a     asx32.exp
 0002:00025d4a       $N00010                    1008dd4a     asx32.exp
 0002:00025d6a       $N00011                    1008dd6a     asx32.exp
 0002:00025d86       $N00012                    1008dd86     asx32.exp
 0002:00025da0       $N00013                    1008dda0     asx32.exp
 0002:00025dbe       $N00014                    1008ddbe     asx32.exp
 0002:00025dde       $N00015                    1008ddde     asx32.exp
 0002:00025dfa       $N00016                    1008ddfa     asx32.exp
 0002:00025e18       $N00017                    1008de18     asx32.exp
 0002:00025e38       $N00018                    1008de38     asx32.exp
 0002:00025e58       $N00019                    1008de58     asx32.exp
 0002:00025e6d       $N00020                    1008de6d     asx32.exp
 0002:00025e86       $N00021                    1008de86     asx32.exp
 0002:00025ea0       $N00022                    1008dea0     asx32.exp
 0002:00025eb5       $N00023                    1008deb5     asx32.exp
 0002:00025ec9       $N00024                    1008dec9     asx32.exp
 0002:00025edd       $N00025                    1008dedd     asx32.exp
 0002:00025efd       $N00026                    1008defd     asx32.exp
 0002:00025f19       $N00027                    1008df19     asx32.exp
 0002:00025f2f       $N00028                    1008df2f     asx32.exp
 0002:00025f48       $N00029                    1008df48     asx32.exp
 0002:00025f5c       $N00030                    1008df5c     asx32.exp
 0002:00025f73       $N00031                    1008df73     asx32.exp
 0002:00025f8d       $N00032                    1008df8d     asx32.exp
 0002:00025f9f       $N00033                    1008df9f     asx32.exp
 0002:00025fb7       $N00034                    1008dfb7     asx32.exp
 0002:00025fdb       $N00035                    1008dfdb     asx32.exp
 0002:00025ffb       $N00036                    1008dffb     asx32.exp
 0002:00026018       $N00037                    1008e018     asx32.exp
 0002:00026034       $N00038                    1008e034     asx32.exp
 0002:00026051       $N00039                    1008e051     asx32.exp
 0002:0002606d       $N00040                    1008e06d     asx32.exp
 0002:0002608a       $N00041                    1008e08a     asx32.exp
 0002:000260a2       $N00042                    1008e0a2     asx32.exp
 0002:000260bc       $N00043                    1008e0bc     asx32.exp
 0002:000260d0       $N00044                    1008e0d0     asx32.exp
 0002:000260e4       $N00045                    1008e0e4     asx32.exp
 0002:000260fd       $N00046                    1008e0fd     asx32.exp
 0002:0002611a       $N00047                    1008e11a     asx32.exp
 0002:00026139       $N00048                    1008e139     asx32.exp
 0002:00026155       $N00049                    1008e155     asx32.exp
 0002:0002616e       $N00050                    1008e16e     asx32.exp
 0002:00026187       $N00051                    1008e187     asx32.exp
 0002:000261a4       $N00052                    1008e1a4     asx32.exp
 0002:000261c3       $N00053                    1008e1c3     asx32.exp
 0002:000261df       $N00054                    1008e1df     asx32.exp
 0002:000261f8       $N00055                    1008e1f8     asx32.exp
 0002:00026217       $N00056                    1008e217     asx32.exp
 0002:00026234       $N00057                    1008e234     asx32.exp
 0002:0002624d       $N00058                    1008e24d     asx32.exp
 0002:00026266       $N00059                    1008e266     asx32.exp
 0002:00026284       $N00060                    1008e284     asx32.exp
 0002:0002629d       $N00061                    1008e29d     asx32.exp
 0002:000262bc       $N00062                    1008e2bc     asx32.exp
 0002:000262d9       $N00063                    1008e2d9     asx32.exp
 0002:000262f2       $N00064                    1008e2f2     asx32.exp
 0002:00026310       $N00065                    1008e310     asx32.exp
 0002:0002632c       $N00066                    1008e32c     asx32.exp
 0002:0002634e       $N00067                    1008e34e     asx32.exp
 0002:0002636e       $N00068                    1008e36e     asx32.exp
 0002:0002638a       $N00069                    1008e38a     asx32.exp
 0002:000263a4       $N00070                    1008e3a4     asx32.exp
 0002:000263c5       $N00071                    1008e3c5     asx32.exp
 0002:000263df       $N00072                    1008e3df     asx32.exp
 0002:000263f8       $N00073                    1008e3f8     asx32.exp
 0002:0002641d       $N00074                    1008e41d     asx32.exp
 0002:00026436       $N00075                    1008e436     asx32.exp
 0002:00026451       $N00076                    1008e451     asx32.exp
 0002:00026466       $N00077                    1008e466     asx32.exp
 0002:0002647b       $N00078                    1008e47b     asx32.exp
 0002:00026497       $N00079                    1008e497     asx32.exp
 0002:000264b4       $N00080                    1008e4b4     asx32.exp
 0002:000264d1       $N00081                    1008e4d1     asx32.exp
 0002:000264f1       $N00082                    1008e4f1     asx32.exp
 0002:00026513       $N00083                    1008e513     asx32.exp
 0002:0002652d       $N00084                    1008e52d     asx32.exp
 0002:00026552       $N00085                    1008e552     asx32.exp
 0002:0002656b       $N00086                    1008e56b     asx32.exp
 0002:00026580       $N00087                    1008e580     asx32.exp
 0002:00026595       $N00088                    1008e595     asx32.exp
 0002:000265b1       $N00089                    1008e5b1     asx32.exp
 0002:000265ce       $N00090                    1008e5ce     asx32.exp
 0002:000265eb       $N00091                    1008e5eb     asx32.exp
 0002:0002660b       $N00092                    1008e60b     asx32.exp
 0002:0002661d       $N00093                    1008e61d     asx32.exp
 0002:00026641       $N00094                    1008e641     asx32.exp
 0002:00026664       $N00095                    1008e664     asx32.exp
 0002:0002667c       $N00096                    1008e67c     asx32.exp
 0002:00026698       $N00097                    1008e698     asx32.exp
 0002:000266af       $N00098                    1008e6af     asx32.exp
 0002:000266ca       $N00099                    1008e6ca     asx32.exp
 0002:000266dc       $N00100                    1008e6dc     asx32.exp
 0002:00026700       $N00101                    1008e700     asx32.exp
 0002:00026723       $N00102                    1008e723     asx32.exp
 0002:0002673b       $N00103                    1008e73b     asx32.exp
 0002:00026757       $N00104                    1008e757     asx32.exp
 0002:0002676e       $N00105                    1008e76e     asx32.exp
 0002:00026789       $N00106                    1008e789     asx32.exp
 0002:000267a8       $N00107                    1008e7a8     asx32.exp
 0002:000267c2       $N00108                    1008e7c2     asx32.exp
 0002:000267dc       $N00109                    1008e7dc     asx32.exp
 0002:000267f5       $N00110                    1008e7f5     asx32.exp
 0002:00026809       $N00111                    1008e809     asx32.exp
 0002:00026818       $N00112                    1008e818     asx32.exp
 0002:00026827       $N00113                    1008e827     asx32.exp
 0002:00026836       $N00114                    1008e836     asx32.exp
 0002:00026846       $N00115                    1008e846     asx32.exp
 0002:00026856       $N00116                    1008e856     asx32.exp
 0002:00026868       $N00117                    1008e868     asx32.exp
 0002:00026880       $N00118                    1008e880     asx32.exp
 0002:00026897       $N00119                    1008e897     asx32.exp
 0002:000268a9       $N00120                    1008e8a9     asx32.exp
 0002:000268bc       $N00121                    1008e8bc     asx32.exp
 0002:000268cf       $N00122                    1008e8cf     asx32.exp
 0002:000268e9       $N00123                    1008e8e9     asx32.exp
 0002:000268fc       $N00124                    1008e8fc     asx32.exp
 0002:0002690a       $N00125                    1008e90a     asx32.exp
 0002:0002691d       $N00126                    1008e91d     asx32.exp
 0002:0002692b       $N00127                    1008e92b     asx32.exp
 0002:00026943       $N00128                    1008e943     asx32.exp
 0002:00026959       $N00129                    1008e959     asx32.exp
 0002:0002696b       $N00130                    1008e96b     asx32.exp
 0002:0002697c       $N00131                    1008e97c     asx32.exp
 0002:00026994       $N00132                    1008e994     asx32.exp
 0002:000269ac       $N00133                    1008e9ac     asx32.exp
 0002:000269c4       $N00134                    1008e9c4     asx32.exp
 0002:000269f0       $N00135                    1008e9f0     asx32.exp
 0002:00026a05       $N00136                    1008ea05     asx32.exp
 0002:00026a20       $N00137                    1008ea20     asx32.exp
 0002:00026a47       $N00138                    1008ea47     asx32.exp
 0002:00026a61       $N00139                    1008ea61     asx32.exp
 0002:00026a7e       $N00140                    1008ea7e     asx32.exp
 0002:00026aa0       $N00141                    1008eaa0     asx32.exp
 0002:00026ab8       $N00142                    1008eab8     asx32.exp
 0002:00026acf       $N00143                    1008eacf     asx32.exp
 0002:00026ae5       $N00144                    1008eae5     asx32.exp
 0002:00026b00       $N00145                    1008eb00     asx32.exp
 0002:00026b18       $N00146                    1008eb18     asx32.exp
 0002:00026b35       $N00147                    1008eb35     asx32.exp
 0002:00026b4d       $N00148                    1008eb4d     asx32.exp
 0002:00026b67       $N00149                    1008eb67     asx32.exp
 0002:00026b7b       $N00150                    1008eb7b     asx32.exp
 0002:00026b8f       $N00151                    1008eb8f     asx32.exp
 0002:00026ba1       $N00152                    1008eba1     asx32.exp
 0002:00026bb6       $N00153                    1008ebb6     asx32.exp
 0002:00026bc7       $N00154                    1008ebc7     asx32.exp
 0002:00026bdd       $N00155                    1008ebdd     asx32.exp
 0002:00026bee       $N00156                    1008ebee     asx32.exp
 0002:00026c00       $N00157                    1008ec00     asx32.exp
 0002:00026c17       $N00158                    1008ec17     asx32.exp
 0002:00026c2a       $N00159                    1008ec2a     asx32.exp
 0002:00026c41       $N00160                    1008ec41     asx32.exp
 0002:00026c5e       $N00161                    1008ec5e     asx32.exp
 0002:00026c6f       $N00162                    1008ec6f     asx32.exp
 0002:00026c80       $N00163                    1008ec80     asx32.exp
 0002:00026c91       $N00164                    1008ec91     asx32.exp
 0002:00026cae       $N00165                    1008ecae     asx32.exp
 0002:00026cca       $N00166                    1008ecca     asx32.exp
 0002:00026ce1       $N00167                    1008ece1     asx32.exp
 0002:00026cf8       $N00168                    1008ecf8     asx32.exp
 0002:00026d0f       $N00169                    1008ed0f     asx32.exp
 0002:00026d23       $N00170                    1008ed23     asx32.exp
 0002:00026d3b       $N00171                    1008ed3b     asx32.exp
 0002:00026d4b       $N00172                    1008ed4b     asx32.exp
 0002:00026d63       $N00173                    1008ed63     asx32.exp
 0002:00026d74       $N00174                    1008ed74     asx32.exp
 0002:00026d8e       $N00175                    1008ed8e     asx32.exp
 0002:00026da6       $N00176                    1008eda6     asx32.exp
 0002:00026db9       $N00177                    1008edb9     asx32.exp
 0002:00026dd5       $N00178                    1008edd5     asx32.exp
 0002:00026dec       $N00179                    1008edec     asx32.exp
 0002:00026e03       $N00180                    1008ee03     asx32.exp
 0002:00026e1b       $N00181                    1008ee1b     asx32.exp
 0002:00026e2c       $N00182                    1008ee2c     asx32.exp
 0002:00026e3c       $N00183                    1008ee3c     asx32.exp
 0002:00026e4c       $N00184                    1008ee4c     asx32.exp
 0002:00026e5f       $N00185                    1008ee5f     asx32.exp
 0002:00026e7c       $N00186                    1008ee7c     asx32.exp
 0002:00026e95       $N00187                    1008ee95     asx32.exp
 0002:00026eae       $N00188                    1008eeae     asx32.exp
 0002:00026ec4       $N00189                    1008eec4     asx32.exp
 0002:00026ed6       $N00190                    1008eed6     asx32.exp
 0002:00026ee9       $N00191                    1008eee9     asx32.exp
 0002:00026efc       $N00192                    1008eefc     asx32.exp
 0002:00026f0e       $N00193                    1008ef0e     asx32.exp
 0002:00026f33       $N00194                    1008ef33     asx32.exp
 0002:00026f56       $N00195                    1008ef56     asx32.exp
 0002:00026f7a       $N00196                    1008ef7a     asx32.exp
 0002:00026f98       $N00197                    1008ef98     asx32.exp
 0002:00026fb7       $N00198                    1008efb7     asx32.exp
 0002:00026fd4       $N00199                    1008efd4     asx32.exp
 0002:00026ff5       $N00200                    1008eff5     asx32.exp
 0002:00027013       $N00201                    1008f013     asx32.exp
 0002:00027031       $N00202                    1008f031     asx32.exp
 0002:00027050       $N00203                    1008f050     asx32.exp
 0002:0002706d       $N00204                    1008f06d     asx32.exp
 0002:0002708e       $N00205                    1008f08e     asx32.exp
 0002:000270ac       $N00206                    1008f0ac     asx32.exp
 0002:000270c9       $N00207                    1008f0c9     asx32.exp
 0002:000270e7       $N00208                    1008f0e7     asx32.exp
 0002:0002710a       $N00209                    1008f10a     asx32.exp
 0002:00027127       $N00210                    1008f127     asx32.exp
 0002:00027148       $N00211                    1008f148     asx32.exp
 0002:00027165       $N00212                    1008f165     asx32.exp
 0002:00027183       $N00213                    1008f183     asx32.exp
 0002:000271a6       $N00214                    1008f1a6     asx32.exp
 0002:000271c7       $N00215                    1008f1c7     asx32.exp
 0002:000271d9       $N00216                    1008f1d9     asx32.exp
 0002:000271f4       $N00217                    1008f1f4     asx32.exp
 0002:00027206       $N00218                    1008f206     asx32.exp
 0002:0002721c       $N00219                    1008f21c     asx32.exp
 0002:00027237       $N00220                    1008f237     asx32.exp
 0002:0002725d       $N00221                    1008f25d     asx32.exp
 0002:0002727a       $N00222                    1008f27a     asx32.exp
 0002:0002728d       $N00223                    1008f28d     asx32.exp
 0002:000272a3       $N00224                    1008f2a3     asx32.exp
 0002:000272c4       $N00225                    1008f2c4     asx32.exp
 0002:000272e2       $N00226                    1008f2e2     asx32.exp
 0002:00027308       $N00227                    1008f308     asx32.exp
 0002:0002732b       $N00228                    1008f32b     asx32.exp
 0002:00027348       $N00229                    1008f348     asx32.exp
 0002:00027365       $N00230                    1008f365     asx32.exp
 0002:00027380       $N00231                    1008f380     asx32.exp
 0002:000273a0       $N00232                    1008f3a0     asx32.exp
 0002:000273be       $N00233                    1008f3be     asx32.exp
 0002:000273d8       $N00234                    1008f3d8     asx32.exp
 0002:000273f6       $N00235                    1008f3f6     asx32.exp
 0002:00027411       $N00236                    1008f411     asx32.exp
 0002:00027431       $N00237                    1008f431     asx32.exp
 0002:0002744f       $N00238                    1008f44f     asx32.exp
 0002:00027467       $N00239                    1008f467     asx32.exp
 0002:00027485       $N00240                    1008f485     asx32.exp
 0002:000274a0       $N00241                    1008f4a0     asx32.exp
 0002:000274bb       $N00242                    1008f4bb     asx32.exp
 0002:000274cd       $N00243                    1008f4cd     asx32.exp
 0002:000274e7       $N00244                    1008f4e7     asx32.exp
 0002:00027509       $N00245                    1008f509     asx32.exp
 0002:0002752a       $N00246                    1008f52a     asx32.exp
 0002:00027546       $N00247                    1008f546     asx32.exp
 0002:00027564       $N00248                    1008f564     asx32.exp
 0002:0002757e       $N00249                    1008f57e     asx32.exp
 0002:00027596       $N00250                    1008f596     asx32.exp
 0002:000275b8       $N00251                    1008f5b8     asx32.exp
 0002:000275d5       $N00252                    1008f5d5     asx32.exp
 0002:000275ec       $N00253                    1008f5ec     asx32.exp
 0002:00027608       $N00254                    1008f608     asx32.exp
 0002:0002761a       $N00255                    1008f61a     asx32.exp
 0002:00027631       $N00256                    1008f631     asx32.exp
 0002:00027646       $N00257                    1008f646     asx32.exp
 0002:00027665       $N00258                    1008f665     asx32.exp
 0002:00027684       $N00259                    1008f684     asx32.exp
 0002:000276a6       $N00260                    1008f6a6     asx32.exp
 0002:000276b8       $N00261                    1008f6b8     asx32.exp
 0002:000276cd       $N00262                    1008f6cd     asx32.exp
 0002:000276e2       $N00263                    1008f6e2     asx32.exp
 0002:000276fa       $N00264                    1008f6fa     asx32.exp
 0002:0002770e       $N00265                    1008f70e     asx32.exp
 0002:00027720       $N00266                    1008f720     asx32.exp
 0002:0002773d       $N00267                    1008f73d     asx32.exp
 0002:00027755       $N00268                    1008f755     asx32.exp
 0002:0002776c       $N00269                    1008f76c     asx32.exp
 0002:0002777e       $N00270                    1008f77e     asx32.exp
 0002:00027793       $N00271                    1008f793     asx32.exp
 0002:000277a5       $N00272                    1008f7a5     asx32.exp
 0002:000277ba       $N00273                    1008f7ba     asx32.exp
 0002:000277d1       $N00274                    1008f7d1     asx32.exp
 0002:000277e4       $N00275                    1008f7e4     asx32.exp
 0002:000277f7       $N00276                    1008f7f7     asx32.exp
 0002:0002780b       $N00277                    1008f80b     asx32.exp
 0002:00027822       $N00278                    1008f822     asx32.exp
 0002:00027835       $N00279                    1008f835     asx32.exp
 0002:00027848       $N00280                    1008f848     asx32.exp
 0002:00027859       $N00281                    1008f859     asx32.exp
 0002:0002786a       $N00282                    1008f86a     asx32.exp
 0002:000281f4       .idata$6                   100901f4     winmm:WINMM.dll
 0002:000298f2       .idata$6                   100918f2     asihpi32:ASIHPI32.dll
 0002:00029900       .idata$6                   10091900     wsnmp32:wsnmp32.dll
 0002:0002990c       .idata$6                   1009190c     wsock32:WSOCK32.dll
 0002:00029918       .idata$6                   10091918     dsound:DSOUND.dll
 0002:00029b36       .idata$6                   10091b36     kernel32:KERNEL32.dll
 0002:00029b88       .idata$6                   10091b88     user32:USER32.dll
 0002:00029c1e       .idata$6                   10091c1e     advapi32:ADVAPI32.dll
 0002:00029c62       .idata$6                   10091c62     ole32:ole32.dll
 0003:000000a8       _PcmSubformatGUID          100930a8     asxasioplay.obj
 0003:000000b8       _IeeeFloatSubformatGUID    100930b8     asxasioplay.obj
 0003:000000c8       _PcmSubformatGUID          100930c8     asxasiorec.obj
 0003:000000d8       _IeeeFloatSubformatGUID    100930d8     asxasiorec.obj
 0003:000000e8       _hpi_asx_node_map          100930e8     asxhpi.obj
 0003:000001e0       _FormatTable               100931e0     asxplay.obj
 0003:00002214       _szNoFound                 10095214     asxstring.obj
 0003:00002220       _mode_rate_table           10095220     cobranet.obj
 0003:00002238       _subformat_table           10095238     cobranet.obj
 0003:00002280       _maxchans_table            10095280     cobranet.obj
 0003:000031e0       _adwMpegBr                 100961e0     twavfile.obj
 0003:00003220       _adwMp3Br                  10096220     twavfile.obj
 0003:00003320       _adwMpegRate               10096320     twavfile.obj
 0003:00003360       _awMpegChannels            10096360     twavfile.obj
 0003:00003368       _PcmSubformatGUID          10096368     twavfmt.obj
 0003:00003378       _FloatSubformatGUID        10096378     twavfmt.obj
 0003:000033b0       ?isPackaged@?1??__crtIsPackagedApp@@9@9 100963b0     LIBCMT:winapisupp.obj
 0003:000037e0       ___rgctypeflag             100967e0     LIBCMT:mbctype.obj
 0003:000037e8       ___rgcode_page_info        100967e8     LIBCMT:mbctype.obj
 0003:00003b14       __ctype_loc_style          10096b14     LIBCMT:wsetloca.obj
 0003:00003b18       _errtable                  10096b18     LIBCMT:dosmap.obj
 0003:00003c80       _ErrnoNoMem                10096c80     LIBCMT:dosmap.obj
 0003:00003c84       _DoserrorNoMem             10096c84     LIBCMT:dosmap.obj
 0003:00003f50       _NAME_                     10096f50     LIBCMT:sqrt.obj
 0003:00003f80       ?_names@?1??_get_fname@@9@9 10096f80     LIBCMT:fpexcept.obj
 0003:00004068       _over                      10097068     LIBCMT:fpctrl.obj
 0003:00004074       _under                     10097074     LIBCMT:fpctrl.obj
 0003:00004080       ?__DAZ_ENABLED@?1??__set_fpsr_sse2@@9@9 10097080     LIBCMT:fpctrl.obj
 0003:00004090       __locktable                10097090     LIBCMT:mlock.obj
 0003:000041b0       LOG_name                   100971b0     LIBCMT:log10.obj
 0003:000041c8       POW_name                   100971c8     LIBCMT:pow.obj
 0003:00004320       _NAME_                     10097320     LIBCMT:sin.obj
 0003:00004390       _DoubleFormat              10097390     LIBCMT:intrncvt.obj
 0003:000043a8       _FloatFormat               100973a8     LIBCMT:intrncvt.obj
 0003:00005980       _asios_module_log_state    10098980     asicndload.obj
 0003:000059d0       _asios_module_log_state    100989d0     asios.obj
 0003:000059d4       _asios_module_log_state    100989d4     asx.obj
 0003:000059dc       _asios_module_log_state    100989dc     asxavdecc.obj
 0003:000059e0       _allocator_arg             100989e0     asxavdecc.obj
 0003:000059e1       _piecewise_construct       100989e1     asxavdecc.obj
 0003:000059f4       _asios_module_log_state    100989f4     asx32.obj
 0003:000059f8       _asios_module_log_state    100989f8     asxasio.obj
 0003:000059fc       _gpAdapter                 100989fc     asxasio.obj
 0003:00005a00       _asios_module_log_state    10098a00     asxasioplay.obj
 0003:00005a04       _asios_module_log_state    10098a04     asxasiorec.obj
 0003:00005a08       _gszNetworkInterface       10098a08     asxclass.obj
 0003:00005a48       _gszAvdeccInterface        10098a48     asxclass.obj
 0003:00005c48       _gCAP                      10098c48     asxclass.obj
 0003:00005c74       _asios_module_log_state    10098c74     asxclass.obj
 0003:00005c88       _allocator_arg             10098c88     asxclass.obj
 0003:00005c89       _piecewise_construct       10098c89     asxclass.obj
 0003:00005c90       _asios_module_log_state    10098c90     asxdsnd.obj
 0003:00005c94       _asios_module_log_state    10098c94     asxdsndplay.obj
 0003:00005c98       _asios_module_log_state    10098c98     asxdsndrec.obj
 0003:00005ca0       _asios_module_log_state    10098ca0     asxhpi.obj
 0003:00005ca4       _asios_module_log_state    10098ca4     asxhpiplay.obj
 0003:00005ca8       _asios_module_log_state    10098ca8     asxhpiplayi.obj
 0003:00005cac       _asios_module_log_state    10098cac     asxhpirec.obj
 0003:00005cb0       _asios_module_log_state    10098cb0     asxhpireci.obj
 0003:00005cb4       _asios_module_log_state    10098cb4     asxplay.obj
 0003:00005cb8       _asios_module_log_state    10098cb8     asxrec.obj
 0003:00005cbc       _asios_module_log_state    10098cbc     asxsnmp.obj
 0003:00005cc0       _asios_module_log_state    10098cc0     asxtr800.obj
 0003:00005cc4       _asios_module_log_state    10098cc4     asxwave.obj
 0003:00005cc8       _asios_module_log_state    10098cc8     asxwaveplay.obj
 0003:00005ccc       _asios_module_log_state    10098ccc     asxwaverec.obj
 0003:00007a64       _asios_module_log_state    1009aa64     twavfilefifo.obj
 0003:00007a78       _GS_ExceptionRecord        1009aa78     LIBCMT:gs_report.obj
 0003:00007ac8       _GS_ContextRecord          1009aac8     LIBCMT:gs_report.obj
 0003:00007d94       _DebuggerWasPresent        1009ad94     LIBCMT:gs_report.obj
 0003:00007d98       ___enable_percent_n        1009ad98     LIBCMT:printf.obj
 0003:00007da0       ___proc_attached           1009ada0     LIBCMT:dllcrt0.obj
 0003:00007dc4       _fSystemSet                1009adc4     LIBCMT:mbctype.obj
 0003:00007e20       ?outmsg@?8??_NMSG_WRITE@@9@9 1009ae20     LIBCMT:crt0msg.obj
 0003:00008458       ___type_info_root_node     1009b458     LIBCMT:typname.obj
 0003:00008470       _lclcritsects              1009b470     LIBCMT:mlock.obj
 0003:000085c0       __pmatherr_set             1009b5c0     LIBCMT:libm_error.obj
 0003:000086c8       ?_pgmname@?1??_setargv@@9@9 1009b6c8     LIBCMT:stdargv.obj
 0003:000087d8       ___crtCallProc             1009b7d8     LIBCMT:winapinls.obj
 0003:000087dc       _ctrlc_action              1009b7dc     LIBCMT:winsig.obj
 0003:000087e0       _ctrlbreak_action          1009b7e0     LIBCMT:winsig.obj
 0003:000087e4       _abort_action              1009b7e4     LIBCMT:winsig.obj
 0003:000087e8       _term_action               1009b7e8     LIBCMT:winsig.obj
 0003:000087ec       _ConsoleCtrlHandler_Installed 1009b7ec     LIBCMT:winsig.obj
 0003:000087f0       _g_pfnRtlGenRandom         1009b7f0     LIBCMT:rand_s.obj
 0003:000087f8       ?pfnMessageBox@?1??__crtMessageBoxW@@9@9 1009b7f8     LIBCMT:crtmboxw.obj
 0003:000087fc       ?pfnGetActiveWindow@?1??__crtMessageBoxW@@9@9 1009b7fc     LIBCMT:crtmboxw.obj
 0003:00008800       ?pfnGetLastActivePopup@?1??__crtMessageBoxW@@9@9 1009b800     LIBCMT:crtmboxw.obj
 0003:00008804       ?pfnGetProcessWindowStation@?1??__crtMessageBoxW@@9@9 1009b804     LIBCMT:crtmboxw.obj
 0003:00008808       ?pfnGetUserObjectInformation@?1??__crtMessageBoxW@@9@9 1009b808     LIBCMT:crtmboxw.obj
 0003:00008834       _heap                      1009b834     LIBCMT:undname.obj
 0003:00008888       __Tuple_alloc              1009b888     libcpmt:xthrow.obj
 0003:00008889       _ignore                    1009b889     libcpmt:xthrow.obj
 0003:0000888a       _allocator_arg             1009b88a     libcpmt:xthrow.obj
 0003:0000888b       _piecewise_construct       1009b88b     libcpmt:xthrow.obj
 0003:0000888c       _allocator_arg             1009b88c     libcpmt:syserror.obj
 0003:0000888d       _piecewise_construct       1009b88d     libcpmt:syserror.obj
 0004:000000a0       $R000000                   1009d0a0     asx32.res
 0004:00000400       $R000360                   1009d400     asx32.res
